 fontmanager

 Timestamp is a670f7cb (reproducible build file hash)

 Preferred load address is 0000000180000000

 Start         Length     Name                   Class
 0001:00000000 000a9270H .text$mn                CODE
 0001:000a9270 00000036H .text$mn$00             CODE
 0001:000a92a6 00000092H .text$x                 CODE
 0002:00000000 000004c0H .idata$5                DATA
 0002:000004c0 00000038H .00cfg                  DATA
 0002:000004f8 00000008H .CRT$XCA                DATA
 0002:00000500 00000008H .CRT$XCZ                DATA
 0002:00000508 00000008H .CRT$XIA                DATA
 0002:00000510 00000008H .CRT$XIZ                DATA
 0002:00000518 00000008H .CRT$XPA                DATA
 0002:00000520 00000008H .CRT$XPZ                DATA
 0002:00000528 00000008H .CRT$XTA                DATA
 0002:00000530 00000010H .CRT$XTZ                DATA
 0002:00000538 00000000H .gehcont$y              DATA
 0002:00000538 00000000H .gfids$y                DATA
 0002:00000540 00028ec0H .rdata                  DATA
 0002:00029400 00000000H .rdata$CastGuardVftablesA DATA
 0002:00029400 00000000H .rdata$CastGuardVftablesC DATA
 0002:00029400 00000d24H .rdata$voltmd           DATA
 0002:0002a124 000002ccH .rdata$zzzdbg           DATA
 0002:0002a3f0 00000008H .rtc$IAA                DATA
 0002:0002a3f8 00000008H .rtc$IZZ                DATA
 0002:0002a400 00000008H .rtc$TAA                DATA
 0002:0002a408 00000008H .rtc$TZZ                DATA
 0002:0002a410 00009f00H .xdata                  DATA
 0002:00034310 000008c0H .edata                  DATA
 0002:00034bd0 0000012cH .idata$2                DATA
 0002:00034cfc 00000014H .idata$3                DATA
 0002:00034d10 000004c0H .idata$4                DATA
 0002:000351d0 00000af4H .idata$6                DATA
 0003:00000000 00000b00H .data                   DATA
 0003:00000b00 00001800H .bss                    DATA
 0004:00000000 00007b3cH .pdata                  DATA
 0005:00000000 00000030H _RDATA                  DATA
 0006:00000000 00000060H .rsrc$01                DATA
 0006:00000060 00000340H .rsrc$02                DATA

  Address         Publics by Value              Rva+Base               Lib:Object

 0000:00000000       __guard_iat_count          0000000000000000     <absolute>
 0000:00000000       __dynamic_value_reloc_table 0000000000000000     <absolute>
 0000:00000000       __guard_iat_table          0000000000000000     <absolute>
 0000:00000000       __arm64x_redirection_metadata 0000000000000000     <absolute>
 0000:00000000       __hybrid_auxiliary_iat     0000000000000000     <absolute>
 0000:00000000       __hybrid_auxiliary_iat_copy 0000000000000000     <absolute>
 0000:00000000       __x64_code_ranges_to_entry_points_count 0000000000000000     <absolute>
 0000:00000000       ___safe_se_handler_table   0000000000000000     <absolute>
 0000:00000000       __AbsoluteZero             0000000000000000     <absolute>
 0000:00000000       __guard_longjmp_count      0000000000000000     <absolute>
 0000:00000000       __guard_check_icall_a64n_fptr 0000000000000000     <absolute>
 0000:00000000       __guard_fids_table         0000000000000000     <absolute>
 0000:00000000       __guard_longjmp_table      0000000000000000     <absolute>
 0000:00000000       __x64_code_ranges_to_entry_points 0000000000000000     <absolute>
 0000:00000000       __guard_eh_cont_count      0000000000000000     <absolute>
 0000:00000000       __guard_fids_count         0000000000000000     <absolute>
 0000:00000000       __arm64x_redirection_metadata_count 0000000000000000     <absolute>
 0000:00000000       __enclave_config           0000000000000000     <absolute>
 0000:00000000       __arm64x_extra_rfe_table   0000000000000000     <absolute>
 0000:00000000       __guard_eh_cont_table      0000000000000000     <absolute>
 0000:00000000       __arm64x_native_entrypoint 0000000000000000     <absolute>
 0000:00000000       __hybrid_code_map          0000000000000000     <absolute>
 0000:00000000       __arm64x_extra_rfe_table_size 0000000000000000     <absolute>
 0000:00000000       __hybrid_code_map_count    0000000000000000     <absolute>
 0000:00000000       ___safe_se_handler_count   0000000000000000     <absolute>
 0000:00000100       __guard_flags              0000000000000100     <absolute>
 0000:00000000       __ImageBase                0000000180000000     <linker-defined>
 0001:000000b0       Java_sun_font_ColorGlyphSurfaceData_initOps 00000001800010b0 f   ColorGlyphSurfaceData.obj
 0001:00000100       Java_sun_font_ColorGlyphSurfaceData_setCurrentGlyph 0000000180001100 f   ColorGlyphSurfaceData.obj
 0001:00000120       Java_sun_java2d_loops_DrawGlyphListAA_DrawGlyphListAA 0000000180001120 f   DrawGlyphList.obj
 0001:00000120       Java_sun_java2d_loops_DrawGlyphList_DrawGlyphList 0000000180001120 f   DrawGlyphList.obj
 0001:00000200       Java_sun_java2d_loops_DrawGlyphListLCD_DrawGlyphListLCD 0000000180001200 f   DrawGlyphList.obj
 0001:00000320       RefineBounds               0000000180001320 f   DrawGlyphList.obj
 0001:000008c0       initLCDGammaTables         00000001800018c0 f   DrawGlyphList.obj
 0001:00000910       initLUT                    0000000180001910 f   DrawGlyphList.obj
 0001:00000ab0       setupBlitVector            0000000180001ab0 f   DrawGlyphList.obj
 0001:00000ee0       setupLCDBlitVector         0000000180001ee0 f   DrawGlyphList.obj
 0001:00001520       Java_sun_font_SunLayoutEngine_shape 0000000180002520 f   HBShaper.obj
 0001:00001990       storeGVData                0000000180002990 f   HBShaper.obj
 0001:00002200       jdk_hb_shape               0000000180003200 f   HBShaper_Panama.obj
 0001:00002b00       Java_sun_awt_Win32FontManager_getFontPath 0000000180003b00 f   fontpath.obj
 0001:00002e30       Java_sun_awt_Win32FontManager_populateFontFileNameMap0 0000000180003e30 f   fontpath.obj
 0001:00003ac0       Java_sun_font_FreetypeFontScaler_createScalerContextNative 0000000180004ac0 f   freetypeScaler.obj
 0001:00003d60       Java_sun_font_FreetypeFontScaler_disposeNativeScaler 0000000180004d60 f   freetypeScaler.obj
 0001:00003dd0       Java_sun_font_FreetypeFontScaler_getFontMetricsNative 0000000180004dd0 f   freetypeScaler.obj
 0001:000041c0       Java_sun_font_FreetypeFontScaler_getGlyphAdvanceNative 00000001800051c0 f   freetypeScaler.obj
 0001:00004220       Java_sun_font_FreetypeFontScaler_getGlyphCodeNative 0000000180005220 f   freetypeScaler.obj
 0001:000042d0       Java_sun_font_FreetypeFontScaler_getGlyphImageNative 00000001800052d0 f   freetypeScaler.obj
 0001:00004300       Java_sun_font_FreetypeFontScaler_getGlyphMetricsNative 0000000180005300 f   freetypeScaler.obj
 0001:000043c0       Java_sun_font_FreetypeFontScaler_getGlyphOutlineBoundsNative 00000001800053c0 f   freetypeScaler.obj
 0001:00004520       Java_sun_font_FreetypeFontScaler_getGlyphOutlineNative 0000000180005520 f   freetypeScaler.obj
 0001:00004590       Java_sun_font_FreetypeFontScaler_getGlyphPointNative 0000000180005590 f   freetypeScaler.obj
 0001:00004660       Java_sun_font_FreetypeFontScaler_getGlyphVectorOutlineNative 0000000180005660 f   freetypeScaler.obj
 0001:00004960       ??$cache_func_to@U?$SingleSubstFormat2_4@USmallTypes@Layout@OT@@@GSUB_impl@Layout@OT@@@hb_accelerate_subtables_context_t@OT@@SAPEAXPEAXW4hb_ot_lookup_cache_op_t@1@@Z 0000000180005960 f   hb-ot-layout.obj
 0001:00004960       ??$cache_func_to@UContextFormat3@OT@@@hb_accelerate_subtables_context_t@OT@@SAPEAXPEAXW4hb_ot_lookup_cache_op_t@1@@Z 0000000180005960 f   hb-ot-layout.obj
 0001:00004960       ??$cache_func_to@U?$MarkLigPosFormat1_2@USmallTypes@Layout@OT@@@GPOS_impl@Layout@OT@@@hb_accelerate_subtables_context_t@OT@@SAPEAXPEAXW4hb_ot_lookup_cache_op_t@1@@Z 0000000180005960 f   hb-ot-layout.obj
 0001:00004960       ??$cache_func_to@U?$MarkMarkPosFormat1_2@USmallTypes@Layout@OT@@@GPOS_impl@Layout@OT@@@hb_accelerate_subtables_context_t@OT@@SAPEAXPEAXW4hb_ot_lookup_cache_op_t@1@@Z 0000000180005960 f   hb-ot-layout.obj
 0001:00004960       ??$cache_func_to@UReverseChainSingleSubstFormat1@GSUB_impl@Layout@OT@@@hb_accelerate_subtables_context_t@OT@@SAPEAXPEAXW4hb_ot_lookup_cache_op_t@1@@Z 0000000180005960 f   hb-ot-layout.obj
 0001:00004960       ??$cache_func_to@USinglePosFormat2@GPOS_impl@Layout@OT@@@hb_accelerate_subtables_context_t@OT@@SAPEAXPEAXW4hb_ot_lookup_cache_op_t@1@@Z 0000000180005960 f   hb-ot-layout.obj
 0001:00004960       ??$cache_func_to@USinglePosFormat1@GPOS_impl@Layout@OT@@@hb_accelerate_subtables_context_t@OT@@SAPEAXPEAXW4hb_ot_lookup_cache_op_t@1@@Z 0000000180005960 f   hb-ot-layout.obj
 0001:00004960       Java_sun_font_FreetypeFontScaler_getMissingGlyphCodeNative 0000000180005960 f   freetypeScaler.obj
 0001:00004960       ??$cache_func_to@UChainContextFormat3@OT@@@hb_accelerate_subtables_context_t@OT@@SAPEAXPEAXW4hb_ot_lookup_cache_op_t@1@@Z 0000000180005960 f   hb-ot-layout.obj
 0001:00004960       __scrt_stub_for_is_c_termination_complete 0000000180005960 f   MSVCRT:ucrt_stubs.obj
 0001:00004960       ??$cache_func_to@UCursivePosFormat1@GPOS_impl@Layout@OT@@@hb_accelerate_subtables_context_t@OT@@SAPEAXPEAXW4hb_ot_lookup_cache_op_t@1@@Z 0000000180005960 f   hb-ot-layout.obj
 0001:00004960       ??$cache_func_to@U?$MultipleSubstFormat1_2@USmallTypes@Layout@OT@@@GSUB_impl@Layout@OT@@@hb_accelerate_subtables_context_t@OT@@SAPEAXPEAXW4hb_ot_lookup_cache_op_t@1@@Z 0000000180005960 f   hb-ot-layout.obj
 0001:00004960       ??$cache_func_to@U?$AlternateSubstFormat1_2@USmallTypes@Layout@OT@@@GSUB_impl@Layout@OT@@@hb_accelerate_subtables_context_t@OT@@SAPEAXPEAXW4hb_ot_lookup_cache_op_t@1@@Z 0000000180005960 f   hb-ot-layout.obj
 0001:00004960       ??$cache_func_to@U?$ChainContextFormat1_4@USmallTypes@Layout@OT@@@OT@@@hb_accelerate_subtables_context_t@OT@@SAPEAXPEAXW4hb_ot_lookup_cache_op_t@1@@Z 0000000180005960 f   hb-ot-layout.obj
 0001:00004960       ??$cache_func_to@U?$ContextFormat1_4@USmallTypes@Layout@OT@@@OT@@@hb_accelerate_subtables_context_t@OT@@SAPEAXPEAXW4hb_ot_lookup_cache_op_t@1@@Z 0000000180005960 f   hb-ot-layout.obj
 0001:00004960       _is_c_termination_complete 0000000180005960 f   MSVCRT:ucrt_stubs.obj
 0001:00004960       ??$cache_func_to@U?$MarkBasePosFormat1_2@USmallTypes@Layout@OT@@@GPOS_impl@Layout@OT@@@hb_accelerate_subtables_context_t@OT@@SAPEAXPEAXW4hb_ot_lookup_cache_op_t@1@@Z 0000000180005960 f   hb-ot-layout.obj
 0001:00004960       ??$cache_func_to@U?$SingleSubstFormat1_3@USmallTypes@Layout@OT@@@GSUB_impl@Layout@OT@@@hb_accelerate_subtables_context_t@OT@@SAPEAXPEAXW4hb_ot_lookup_cache_op_t@1@@Z 0000000180005960 f   hb-ot-layout.obj
 0001:00004970       Java_sun_font_FreetypeFontScaler_getNumGlyphsNative 0000000180005970 f   freetypeScaler.obj
 0001:00004a20       Java_sun_font_FreetypeFontScaler_getUnitsPerEMNative 0000000180005a20 f   freetypeScaler.obj
 0001:00004a40       Java_sun_font_FreetypeFontScaler_initIDs 0000000180005a40 f   freetypeScaler.obj
 0001:00004aa0       Java_sun_font_FreetypeFontScaler_initNativeScaler 0000000180005aa0 f   freetypeScaler.obj
 0001:00005950       _hb_fallback_shaper_font_data_destroy 0000000180006950 f   hb-fallback-shape.obj
 0001:00005950       ?hb_ot_layout_position_finish_advances@@YAXPEAUhb_font_t@@PEAUhb_buffer_t@@@Z 0000000180006950 f   hb-ot-layout.obj
 0001:00005950       _hb_ot_shaper_face_data_destroy 0000000180006950 f   hb-ot-shape.obj
 0001:00005950       _guard_check_icall_nop     0000000180006950 f   MSVCRT:guard_support.obj
 0001:00005950       _hb_fallback_shaper_face_data_destroy 0000000180006950 f   hb-fallback-shape.obj
 0001:00005960       ??$add_array@I@hb_bit_set_t@@QEAAXPEBIII@Z 0000000180006960 f i hb-aat-layout.obj
 0001:00005b60       ??$add_array@UHBGlyphID16@OT@@@hb_bit_set_t@@QEAAXPEBUHBGlyphID16@OT@@II@Z 0000000180006b60 f i hb-aat-layout.obj
 0001:00005d70       ??$check_array@U?$Entry@X@AAT@@@hb_sanitize_context_t@@QEBA_NPEBU?$Entry@X@AAT@@I@Z 0000000180006d70 f i hb-aat-layout.obj
 0001:00005d70       ??$check_array@U?$IntType@I$03@OT@@@hb_sanitize_context_t@@QEBA_NPEBU?$IntType@I$03@OT@@I@Z 0000000180006d70 f i hb-common.obj
 0001:00005e60       ??$check_array@UFeature@AAT@@@hb_sanitize_context_t@@QEBA_NPEBUFeature@AAT@@I@Z 0000000180006e60 f i hb-aat-layout.obj
 0001:00005f50       ??$check_array@UHBGlyphID16@OT@@@hb_sanitize_context_t@@QEBA_NPEBUHBGlyphID16@OT@@I@Z 0000000180006f50 f i hb-aat-layout.obj
 0001:00005f50       ??$check_array@U?$IntType@G$01@OT@@@hb_sanitize_context_t@@QEBA_NPEBU?$IntType@G$01@OT@@I@Z 0000000180006f50 f i hb-common.obj
 0001:00006040       ??$check_range@U?$IntType@E$00@OT@@@hb_sanitize_context_t@@QEBA_NPEBU?$IntType@E$00@OT@@II@Z 0000000180007040 f i hb-aat-layout.obj
 0001:00006040       ??$check_range@U?$IntType@G$01@OT@@@hb_sanitize_context_t@@QEBA_NPEBU?$IntType@G$01@OT@@II@Z 0000000180007040 f i hb-aat-layout.obj
 0001:00006040       ??$check_range@U?$IntType@F$01@OT@@@hb_sanitize_context_t@@QEBA_NPEBU?$IntType@F$01@OT@@II@Z 0000000180007040 f i hb-aat-layout.obj
 0001:00006140       ??$collect_coverage@Uhb_set_digest_t@@@?$CoverageFormat2_4@USmallTypes@Layout@OT@@@Common@Layout@OT@@AEBA_NPEAUhb_set_digest_t@@@Z 0000000180007140 f i hb-aat-layout.obj
 0001:00006310       ??$collect_coverage@Uhb_set_digest_t@@@MarkGlyphSetsFormat1@OT@@QEBAXAEAU?$hb_vector_t@Uhb_set_digest_t@@$0A@@@@Z 0000000180007310 f i hb-aat-layout.obj
 0001:00006540       ??$collect_glyphs@Uhb_bit_set_t@@@?$ClassTable@U?$IntType@E$00@OT@@@AAT@@QEBAXAEAUhb_bit_set_t@@I@Z 0000000180007540 f i hb-aat-layout.obj
 0001:00006600       ??$collect_glyphs@Uhb_bit_set_t@@@?$Lookup@UHBGlyphID16@OT@@@AAT@@QEBAXAEAUhb_bit_set_t@@I@Z 0000000180007600 f i hb-aat-layout.obj
 0001:00006600       ??$collect_glyphs@Uhb_bit_set_t@@@?$Lookup@U?$IntType@I$03@OT@@@AAT@@QEBAXAEAUhb_bit_set_t@@I@Z 0000000180007600 f i hb-aat-layout.obj
 0001:00006600       ??$collect_glyphs@Uhb_bit_set_t@@@?$Lookup@U?$IntType@G$01@OT@@@AAT@@QEBAXAEAUhb_bit_set_t@@I@Z 0000000180007600 f i hb-aat-layout.obj
 0001:00006940       ??$collect_glyphs@Uhb_bit_set_t@@@KerxSubTable@AAT@@QEBAXAEAUhb_bit_set_t@@0I@Z 0000000180007940 f i hb-aat-layout.obj
 0001:00006bd0       ??$collect_glyphs_filtered@Uhb_bit_set_t@@Uhb_bit_page_t@@@?$ClassTable@U?$IntType@E$00@OT@@@AAT@@QEBAXAEAUhb_bit_set_t@@IAEBUhb_bit_page_t@@@Z 0000000180007bd0 f i hb-aat-layout.obj
 0001:00006cc0       ??$collect_glyphs_filtered@Uhb_bit_set_t@@Uhb_bit_page_t@@@?$Lookup@U?$IntType@G$01@OT@@@AAT@@QEBAXAEAUhb_bit_set_t@@IAEBUhb_bit_page_t@@@Z 0000000180007cc0 f i hb-aat-layout.obj
 0001:00007090       ??$collect_glyphs_filtered@Uhb_bit_set_t@@Uhb_bit_page_t@@@?$LookupFormat4@U?$IntType@G$01@OT@@@AAT@@AEBAXAEAUhb_bit_set_t@@AEBUhb_bit_page_t@@@Z 0000000180008090 f i hb-aat-layout.obj
 0001:00007220       ??$collect_initial_glyphs@Uhb_bit_set_t@@U?$ContextualSubtable@UExtendedTypes@AAT@@@AAT@@@?$StateTable@UExtendedTypes@AAT@@UEntryData@?$ContextualSubtable@UExtendedTypes@AAT@@@2@@AAT@@QEBAXAEAUhb_bit_set_t@@IAEBU?$ContextualSubtable@UExtendedTypes@AAT@@@1@@Z 0000000180008220 f i hb-aat-layout.obj
 0001:00007500       ??$collect_initial_glyphs@Uhb_bit_set_t@@U?$ContextualSubtable@UObsoleteTypes@AAT@@@AAT@@@?$StateTable@UObsoleteTypes@AAT@@UEntryData@?$ContextualSubtable@UObsoleteTypes@AAT@@@2@@AAT@@QEBAXAEAUhb_bit_set_t@@IAEBU?$ContextualSubtable@UObsoleteTypes@AAT@@@1@@Z 0000000180008500 f i hb-aat-layout.obj
 0001:00007740       ??$collect_initial_glyphs@Uhb_bit_set_t@@U?$InsertionSubtable@UExtendedTypes@AAT@@@AAT@@@?$StateTable@UExtendedTypes@AAT@@UEntryData@?$InsertionSubtable@UExtendedTypes@AAT@@@2@@AAT@@QEBAXAEAUhb_bit_set_t@@IAEBU?$InsertionSubtable@UExtendedTypes@AAT@@@1@@Z 0000000180008740 f i hb-aat-layout.obj
 0001:00007a40       ??$collect_initial_glyphs@Uhb_bit_set_t@@U?$InsertionSubtable@UObsoleteTypes@AAT@@@AAT@@@?$StateTable@UObsoleteTypes@AAT@@UEntryData@?$InsertionSubtable@UObsoleteTypes@AAT@@@2@@AAT@@QEBAXAEAUhb_bit_set_t@@IAEBU?$InsertionSubtable@UObsoleteTypes@AAT@@@1@@Z 0000000180008a40 f i hb-aat-layout.obj
 0001:00007cb0       ??$collect_initial_glyphs@Uhb_bit_set_t@@U?$KerxSubTableFormat4@UKerxSubTableHeader@AAT@@@AAT@@@?$StateTable@UExtendedTypes@AAT@@UEntryData@?$KerxSubTableFormat4@UKerxSubTableHeader@AAT@@@2@@AAT@@QEBAXAEAUhb_bit_set_t@@IAEBU?$KerxSubTableFormat4@UKerxSubTableHeader@AAT@@@1@@Z 0000000180008cb0 f i hb-aat-layout.obj
 0001:00007cb0       ??$collect_initial_glyphs@Uhb_bit_set_t@@U?$KerxSubTableFormat1@UKerxSubTableHeader@AAT@@@AAT@@@?$StateTable@UExtendedTypes@AAT@@UEntryData@?$Format1Entry@$00@2@@AAT@@QEBAXAEAUhb_bit_set_t@@IAEBU?$KerxSubTableFormat1@UKerxSubTableHeader@AAT@@@1@@Z 0000000180008cb0 f i hb-aat-layout.obj
 0001:00007f80       ??$collect_initial_glyphs@Uhb_bit_set_t@@U?$LigatureSubtable@UExtendedTypes@AAT@@@AAT@@@?$StateTable@UExtendedTypes@AAT@@UEntryData@?$LigatureEntry@$00@2@@AAT@@QEBAXAEAUhb_bit_set_t@@IAEBU?$LigatureSubtable@UExtendedTypes@AAT@@@1@@Z 0000000180008f80 f i hb-aat-layout.obj
 0001:00008220       ??$collect_initial_glyphs@Uhb_bit_set_t@@U?$KerxSubTableFormat1@UKernAATSubTableHeader@OT@@@AAT@@@?$StateTable@UObsoleteTypes@AAT@@X@AAT@@QEBAXAEAUhb_bit_set_t@@IAEBU?$KerxSubTableFormat1@UKernAATSubTableHeader@OT@@@1@@Z 0000000180009220 f i hb-ot-layout.obj
 0001:00008220       ??$collect_initial_glyphs@Uhb_bit_set_t@@U?$LigatureSubtable@UObsoleteTypes@AAT@@@AAT@@@?$StateTable@UObsoleteTypes@AAT@@X@AAT@@QEBAXAEAUhb_bit_set_t@@IAEBU?$LigatureSubtable@UObsoleteTypes@AAT@@@1@@Z 0000000180009220 f i hb-aat-layout.obj
 0001:00008220       ??$collect_initial_glyphs@Uhb_bit_set_t@@U?$KerxSubTableFormat1@UKernOTSubTableHeader@OT@@@AAT@@@?$StateTable@UObsoleteTypes@AAT@@X@AAT@@QEBAXAEAUhb_bit_set_t@@IAEBU?$KerxSubTableFormat1@UKernOTSubTableHeader@OT@@@1@@Z 0000000180009220 f i hb-ot-layout.obj
 0001:00008430       ??$collect_initial_glyphs@Uhb_bit_set_t@@U?$RearrangementSubtable@UExtendedTypes@AAT@@@AAT@@@?$StateTable@UExtendedTypes@AAT@@X@AAT@@QEBAXAEAUhb_bit_set_t@@IAEBU?$RearrangementSubtable@UExtendedTypes@AAT@@@1@@Z 0000000180009430 f i hb-aat-layout.obj
 0001:000086d0       ??$collect_initial_glyphs@Uhb_bit_set_t@@U?$RearrangementSubtable@UObsoleteTypes@AAT@@@AAT@@@?$StateTable@UObsoleteTypes@AAT@@X@AAT@@QEBAXAEAUhb_bit_set_t@@IAEBU?$RearrangementSubtable@UObsoleteTypes@AAT@@@1@@Z 00000001800096d0 f i hb-aat-layout.obj
 0001:000088d0       ??$dispatch@U?$ChainRuleSet@USmallTypes@Layout@OT@@@OT@@$$V@hb_sanitize_context_t@@QEAA_NAEBU?$ChainRuleSet@USmallTypes@Layout@OT@@@OT@@@Z 00000001800098d0 f i hb-aat-layout.obj
 0001:000089b0       ??$dispatch@U?$ClassTable@U?$IntType@E$00@OT@@@AAT@@$$V@hb_sanitize_context_t@@QEAA_NAEBU?$ClassTable@U?$IntType@E$00@OT@@@AAT@@@Z 00000001800099b0 f i hb-aat-layout.obj
 0001:00008a70       ??$dispatch@U?$Ligature@USmallTypes@Layout@OT@@@GSUB_impl@Layout@OT@@$$V@hb_sanitize_context_t@@QEAA_NAEBU?$Ligature@USmallTypes@Layout@OT@@@GSUB_impl@Layout@OT@@@Z 0000000180009a70 f i hb-aat-layout.obj
 0001:00008b20       ??$dispatch@U?$LigatureSet@USmallTypes@Layout@OT@@@GSUB_impl@Layout@OT@@$$V@hb_sanitize_context_t@@QEAA_NAEBU?$LigatureSet@USmallTypes@Layout@OT@@@GSUB_impl@Layout@OT@@@Z 0000000180009b20 f i hb-aat-layout.obj
 0001:00008c00       ??$dispatch@U?$List16OfOffsetTo@USubstLookup@GSUB_impl@Layout@OT@@U?$IntType@G$01@4@@OT@@$$V@hb_sanitize_context_t@@QEAA_NAEBU?$List16OfOffsetTo@USubstLookup@GSUB_impl@Layout@OT@@U?$IntType@G$01@4@@OT@@@Z 0000000180009c00 f i hb-aat-layout.obj
 0001:00008ce0       ??$dispatch@U?$RecordListOf@UFeature@OT@@@OT@@$$V@hb_sanitize_context_t@@QEAA_NAEBU?$RecordListOf@UFeature@OT@@@OT@@@Z 0000000180009ce0 f i hb-aat-layout.obj
 0001:00008ea0       ??$dispatch@U?$Rule@USmallTypes@Layout@OT@@@OT@@$$V@hb_sanitize_context_t@@QEAA_NAEBU?$Rule@USmallTypes@Layout@OT@@@OT@@@Z 0000000180009ea0 f i hb-aat-layout.obj
 0001:00009030       ??$dispatch@U?$RuleSet@USmallTypes@Layout@OT@@@OT@@$$V@hb_sanitize_context_t@@QEAA_NAEBU?$RuleSet@USmallTypes@Layout@OT@@@OT@@@Z 000000018000a030 f i hb-aat-layout.obj
 0001:00009110       ??$dispatch@U?$UnsizedArrayOf@U?$OffsetTo@U?$ArrayOf@UAnchor@AAT@@U?$IntType@I$03@OT@@@OT@@U?$IntType@G$01@2@X$0A@@OT@@@OT@@IAEAPEBX@hb_sanitize_context_t@@QEAA_NAEBU?$UnsizedArrayOf@U?$OffsetTo@U?$ArrayOf@UAnchor@AAT@@U?$IntType@I$03@OT@@@OT@@U?$IntType@G$01@2@X$0A@@OT@@@OT@@$$QEAIAEAPEBX@Z 000000018000a110 f i hb-aat-layout.obj
 0001:000091c0       ??$dispatch@UAttachList@OT@@$$V@hb_sanitize_context_t@@QEAA_NAEBUAttachList@OT@@@Z 000000018000a1c0 f i hb-aat-layout.obj
 0001:000092f0       ??$dispatch@UClassDef@OT@@$$V@hb_sanitize_context_t@@QEAA_NAEBUClassDef@OT@@@Z 000000018000a2f0 f i hb-aat-layout.obj
 0001:00009450       ??$dispatch@UConditionSet@OT@@$$V@hb_sanitize_context_t@@QEAA_NAEBUConditionSet@OT@@@Z 000000018000a450 f i hb-aat-layout.obj
 0001:00009530       ??$dispatch@UCoverage@Common@Layout@OT@@$$V@hb_sanitize_context_t@@QEAA_NAEBUCoverage@Common@Layout@OT@@@Z 000000018000a530 f i hb-aat-layout.obj
 0001:00009630       ??$dispatch@ULigCaretList@OT@@$$V@hb_sanitize_context_t@@QEAA_NAEBULigCaretList@OT@@@Z 000000018000a630 f i hb-aat-layout.obj
 0001:00009760       ??$dispatch@ULigGlyph@OT@@$$V@hb_sanitize_context_t@@QEAA_NAEBULigGlyph@OT@@@Z 000000018000a760 f i hb-aat-layout.obj
 0001:00009840       ??$dispatch@UMarkGlyphSets@OT@@$$V@hb_sanitize_context_t@@QEAA_NAEBUMarkGlyphSets@OT@@@Z 000000018000a840 f i hb-aat-layout.obj
 0001:000099a0       ??$dispatch@URecordListOfScript@OT@@$$V@hb_sanitize_context_t@@QEAA_NAEBURecordListOfScript@OT@@@Z 000000018000a9a0 f i hb-aat-layout.obj
 0001:00009b40       ??$dispatch@UVarData@OT@@$$V@hb_sanitize_context_t@@QEAA_NAEBUVarData@OT@@@Z 000000018000ab40 f i hb-aat-layout.obj
 0001:00009c90       ??$dispatch@UVarRegionList@OT@@$$V@hb_sanitize_context_t@@QEAA_NAEBUVarRegionList@OT@@@Z 000000018000ac90 f i hb-aat-layout.obj
 0001:00009d80       ??$dispatch@Uhb_aat_apply_context_t@AAT@@$$V@?$ChainSubtable@UExtendedTypes@AAT@@@AAT@@QEBA_NPEAUhb_aat_apply_context_t@1@@Z 000000018000ad80 f i hb-aat-layout.obj
 0001:0000a030       ??$dispatch@Uhb_aat_apply_context_t@AAT@@$$V@?$ChainSubtable@UObsoleteTypes@AAT@@@AAT@@QEBA_NPEAUhb_aat_apply_context_t@1@@Z 000000018000b030 f i hb-aat-layout.obj
 0001:0000a260       ??$dispatch@Uhb_aat_apply_context_t@AAT@@$$V@KerxSubTable@AAT@@QEBA_NPEAUhb_aat_apply_context_t@1@@Z 000000018000b260 f i hb-aat-layout.obj
 0001:0000a510       ??$dispatch@Uhb_accelerate_subtables_context_t@AAT@@$$V@?$ChainSubtable@UExtendedTypes@AAT@@@AAT@@QEBA?AUhb_empty_t@@PEAUhb_accelerate_subtables_context_t@1@@Z 000000018000b510 f i hb-aat-layout.obj
 0001:0000a7b0       ??$dispatch@Uhb_accelerate_subtables_context_t@AAT@@$$V@?$ChainSubtable@UObsoleteTypes@AAT@@@AAT@@QEBA?AUhb_empty_t@@PEAUhb_accelerate_subtables_context_t@1@@Z 000000018000b7b0 f i hb-aat-layout.obj
 0001:0000aa50       ??$dispatch@Uhb_sanitize_context_t@@$$V@?$ChainSubtable@UExtendedTypes@AAT@@@AAT@@QEBA_NPEAUhb_sanitize_context_t@@@Z 000000018000ba50 f i hb-aat-layout.obj
 0001:0000add0       ??$dispatch@Uhb_sanitize_context_t@@$$V@?$ChainSubtable@UObsoleteTypes@AAT@@@AAT@@QEBA_NPEAUhb_sanitize_context_t@@@Z 000000018000bdd0 f i hb-aat-layout.obj
 0001:0000b050       ??$dispatch@Uhb_sanitize_context_t@@$$V@?$Extension@UExtensionSubst@GSUB_impl@Layout@OT@@@OT@@QEBA_NPEAUhb_sanitize_context_t@@@Z 000000018000c050 f i hb-aat-layout.obj
 0001:0000b200       ??$dispatch@Uhb_sanitize_context_t@@$$V@MultipleSubst@GSUB_impl@Layout@OT@@QEBA_NPEAUhb_sanitize_context_t@@@Z 000000018000c200 f i hb-aat-layout.obj
 0001:0000b200       ??$dispatch@Uhb_sanitize_context_t@@$$V@AlternateSubst@GSUB_impl@Layout@OT@@QEBA_NPEAUhb_sanitize_context_t@@@Z 000000018000c200 f i hb-aat-layout.obj
 0001:0000b3f0       ??$dispatch@Uhb_sanitize_context_t@@$$V@ChainContext@OT@@QEBA_NPEAUhb_sanitize_context_t@@@Z 000000018000c3f0 f i hb-aat-layout.obj
 0001:0000b620       ??$dispatch@Uhb_sanitize_context_t@@$$V@Context@OT@@QEBA_NPEAUhb_sanitize_context_t@@@Z 000000018000c620 f i hb-aat-layout.obj
 0001:0000b850       ??$dispatch@Uhb_sanitize_context_t@@$$V@LigatureSubst@GSUB_impl@Layout@OT@@QEBA_NPEAUhb_sanitize_context_t@@@Z 000000018000c850 f i hb-aat-layout.obj
 0001:0000ba40       ??$dispatch@Uhb_sanitize_context_t@@$$V@SingleSubst@GSUB_impl@Layout@OT@@QEBA_NPEAUhb_sanitize_context_t@@@Z 000000018000ca40 f i hb-aat-layout.obj
 0001:0000bc90       ??$dispatch@Uhb_sanitize_context_t@@$$V@SubstLookupSubTable@GSUB_impl@Layout@OT@@QEBA_NPEAUhb_sanitize_context_t@@I@Z 000000018000cc90 f i hb-aat-layout.obj
 0001:0000be30       ??$drive@Udriver_context_t@?$ContextualSubtable@UExtendedTypes@AAT@@@AAT@@@?$StateTableDriver@UExtendedTypes@AAT@@UEntryData@?$ContextualSubtable@UExtendedTypes@AAT@@@2@W4Flags@42@@AAT@@QEAAXPEAUdriver_context_t@?$ContextualSubtable@UExtendedTypes@AAT@@@1@PEAUhb_aat_apply_context_t@1@@Z 000000018000ce30 f i hb-aat-layout.obj
 0001:0000c4a0       ??$drive@Udriver_context_t@?$ContextualSubtable@UObsoleteTypes@AAT@@@AAT@@@?$StateTableDriver@UObsoleteTypes@AAT@@UEntryData@?$ContextualSubtable@UObsoleteTypes@AAT@@@2@W4Flags@42@@AAT@@QEAAXPEAUdriver_context_t@?$ContextualSubtable@UObsoleteTypes@AAT@@@1@PEAUhb_aat_apply_context_t@1@@Z 000000018000d4a0 f i hb-aat-layout.obj
 0001:0000c960       ??$drive@Udriver_context_t@?$InsertionSubtable@UExtendedTypes@AAT@@@AAT@@@?$StateTableDriver@UExtendedTypes@AAT@@UEntryData@?$InsertionSubtable@UExtendedTypes@AAT@@@2@W4Flags@42@@AAT@@QEAAXPEAUdriver_context_t@?$InsertionSubtable@UExtendedTypes@AAT@@@1@PEAUhb_aat_apply_context_t@1@@Z 000000018000d960 f i hb-aat-layout.obj
 0001:0000ce80       ??$drive@Udriver_context_t@?$InsertionSubtable@UObsoleteTypes@AAT@@@AAT@@@?$StateTableDriver@UObsoleteTypes@AAT@@UEntryData@?$InsertionSubtable@UObsoleteTypes@AAT@@@2@W4Flags@42@@AAT@@QEAAXPEAUdriver_context_t@?$InsertionSubtable@UObsoleteTypes@AAT@@@1@PEAUhb_aat_apply_context_t@1@@Z 000000018000de80 f i hb-aat-layout.obj
 0001:0000d380       ??$drive@Udriver_context_t@?$KerxSubTableFormat1@UKerxSubTableHeader@AAT@@@AAT@@@?$StateTableDriver@UExtendedTypes@AAT@@UEntryData@?$Format1Entry@$00@2@W4Flags@?$KerxSubTableFormat1@UKerxSubTableHeader@AAT@@@2@@AAT@@QEAAXPEAUdriver_context_t@?$KerxSubTableFormat1@UKerxSubTableHeader@AAT@@@1@PEAUhb_aat_apply_context_t@1@@Z 000000018000e380 f i hb-aat-layout.obj
 0001:0000d7e0       ??$drive@Udriver_context_t@?$KerxSubTableFormat4@UKerxSubTableHeader@AAT@@@AAT@@@?$StateTableDriver@UExtendedTypes@AAT@@UEntryData@?$KerxSubTableFormat4@UKerxSubTableHeader@AAT@@@2@W4Flags@42@@AAT@@QEAAXPEAUdriver_context_t@?$KerxSubTableFormat4@UKerxSubTableHeader@AAT@@@1@PEAUhb_aat_apply_context_t@1@@Z 000000018000e7e0 f i hb-aat-layout.obj
 0001:0000dc30       ??$drive@Udriver_context_t@?$LigatureSubtable@UExtendedTypes@AAT@@@AAT@@@?$StateTableDriver@UExtendedTypes@AAT@@UEntryData@?$LigatureEntry@$00@2@W4Flags@?$LigatureSubtable@UExtendedTypes@AAT@@@2@@AAT@@QEAAXPEAUdriver_context_t@?$LigatureSubtable@UExtendedTypes@AAT@@@1@PEAUhb_aat_apply_context_t@1@@Z 000000018000ec30 f i hb-aat-layout.obj
 0001:0000e080       ??$drive@Udriver_context_t@?$LigatureSubtable@UObsoleteTypes@AAT@@@AAT@@@?$StateTableDriver@UObsoleteTypes@AAT@@XW4Flags@?$LigatureSubtable@UObsoleteTypes@AAT@@@2@@AAT@@QEAAXPEAUdriver_context_t@?$LigatureSubtable@UObsoleteTypes@AAT@@@1@PEAUhb_aat_apply_context_t@1@@Z 000000018000f080 f i hb-aat-layout.obj
 0001:0000e480       ??$drive@Udriver_context_t@?$RearrangementSubtable@UExtendedTypes@AAT@@@AAT@@@?$StateTableDriver@UExtendedTypes@AAT@@XW4Flags@?$RearrangementSubtable@UExtendedTypes@AAT@@@2@@AAT@@QEAAXPEAUdriver_context_t@?$RearrangementSubtable@UExtendedTypes@AAT@@@1@PEAUhb_aat_apply_context_t@1@@Z 000000018000f480 f i hb-aat-layout.obj
 0001:0000e870       ??$drive@Udriver_context_t@?$RearrangementSubtable@UObsoleteTypes@AAT@@@AAT@@@?$StateTableDriver@UObsoleteTypes@AAT@@XW4Flags@?$RearrangementSubtable@UObsoleteTypes@AAT@@@2@@AAT@@QEAAXPEAUdriver_context_t@?$RearrangementSubtable@UObsoleteTypes@AAT@@@1@PEAUhb_aat_apply_context_t@1@@Z 000000018000f870 f i hb-aat-layout.obj
 0001:0000ec10       ??$get_subtable@UPosLookupSubTable@GPOS_impl@Layout@OT@@@Lookup@OT@@QEBAAEBUPosLookupSubTable@GPOS_impl@Layout@1@I@Z 000000018000fc10 f i hb-ot-layout.obj
 0001:0000ec10       ??$get_subtable@USubstLookupSubTable@GSUB_impl@Layout@OT@@@Lookup@OT@@QEBAAEBUSubstLookupSubTable@GSUB_impl@Layout@1@I@Z 000000018000fc10 f i hb-aat-layout.obj
 0001:0000ec80       ??$output_glyphs@UHBGlyphID16@OT@@@hb_aat_apply_context_t@AAT@@QEAA_NIPEBUHBGlyphID16@OT@@@Z 000000018000fc80 f i hb-aat-layout.obj
 0001:0000eee0       ??$realloc_vector@Ukern_subtable_accelerator_data_t@AAT@@$0A@@?$hb_vector_t@Ukern_subtable_accelerator_data_t@AAT@@$0A@@@QEAAPEAUkern_subtable_accelerator_data_t@AAT@@IU?$hb_priority@$0A@@@@Z 000000018000fee0 f i hb-aat-layout.obj
 0001:0000f0f0       ??$sanitize@$$V@?$UnsizedListOfOffset16To@U?$Lookup@UHBGlyphID16@OT@@@AAT@@U?$IntType@G$01@OT@@X$0A@@OT@@QEBA_NPEAUhb_sanitize_context_t@@I@Z 00000001800100f0 f i hb-aat-layout.obj
 0001:0000f1a0       ??$sanitize@$$V@?$UnsizedListOfOffset16To@U?$Lookup@UHBGlyphID16@OT@@@AAT@@U?$IntType@I$03@OT@@X$0A@@OT@@QEBA_NPEAUhb_sanitize_context_t@@I@Z 00000001800101a0 f i hb-aat-layout.obj
 0001:0000f250       ??$sanitize@USubstLookup@GSUB_impl@Layout@OT@@@?$GSUBGPOSVersion1_2@USmallTypes@Layout@OT@@@OT@@QEBA_NPEAUhb_sanitize_context_t@@@Z 0000000180010250 f i hb-aat-layout.obj
 0001:0000f400       ??$sanitize@USubstLookupSubTable@GSUB_impl@Layout@OT@@@Lookup@OT@@QEBA_NPEAUhb_sanitize_context_t@@@Z 0000000180010400 f i hb-aat-layout.obj
 0001:0000f660       ??$sanitize_blob@UGDEF@OT@@@hb_sanitize_context_t@@QEAAPEAUhb_blob_t@@PEAU1@@Z 0000000180010660 f i hb-aat-layout.obj
 0001:0000f880       ??$sanitize_blob@UGSUB@Layout@OT@@@hb_sanitize_context_t@@QEAAPEAUhb_blob_t@@PEAU1@@Z 0000000180010880 f i hb-aat-layout.obj
 0001:0000faa0       ??$sanitize_blob@Uankr@AAT@@@hb_sanitize_context_t@@QEAAPEAUhb_blob_t@@PEAU1@@Z 0000000180010aa0 f i hb-aat-layout.obj
 0001:0000fe00       ??$sanitize_blob@Ufeat@AAT@@@hb_sanitize_context_t@@QEAAPEAUhb_blob_t@@PEAU1@@Z 0000000180010e00 f i hb-aat-layout.obj
 0001:00010120       ??$sanitize_blob@Ukerx@AAT@@@hb_sanitize_context_t@@QEAAPEAUhb_blob_t@@PEAU1@@Z 0000000180011120 f i hb-aat-layout.obj
 0001:000102b0       ??$sanitize_blob@Ultag@AAT@@@hb_sanitize_context_t@@QEAAPEAUhb_blob_t@@PEAU1@@Z 00000001800112b0 f i hb-aat-layout.obj
 0001:000105d0       ??$sanitize_blob@Umort@AAT@@@hb_sanitize_context_t@@QEAAPEAUhb_blob_t@@PEAU1@@Z 00000001800115d0 f i hb-aat-layout.obj
 0001:00010ae0       ??$sanitize_blob@Umorx@AAT@@@hb_sanitize_context_t@@QEAAPEAUhb_blob_t@@PEAU1@@Z 0000000180011ae0 f i hb-aat-layout.obj
 0001:00010de0       ??$sanitize_blob@Utrak@AAT@@@hb_sanitize_context_t@@QEAAPEAUhb_blob_t@@PEAU1@@Z 0000000180011de0 f i hb-aat-layout.obj
 0001:000110a0       ??0?$accelerator_t@UGSUB@Layout@OT@@@GSUBGPOS@OT@@QEAA@PEAUhb_face_t@@@Z 00000001800120a0 f i hb-aat-layout.obj
 0001:00011260       ??0?$hb_cache_t@$0P@$07$06$00@@QEAA@XZ 0000000180012260 f i hb-aat-layout.obj
 0001:00011350       ??0accelerator_t@?$KerxTable@Ukerx@AAT@@@AAT@@QEAA@PEAUhb_face_t@@@Z 0000000180012350 f i hb-aat-layout.obj
 0001:000114f0       ??0accelerator_t@?$mortmorx@Umorx@AAT@@UExtendedTypes@2@$0GNGPHCHI@@AAT@@QEAA@PEAUhb_face_t@@@Z 00000001800124f0 f i hb-aat-layout.obj
 0001:00011750       ??0accelerator_t@GDEF@OT@@QEAA@PEAUhb_face_t@@@Z 0000000180012750 f i hb-aat-layout.obj
 0001:00011960       ??0hb_aat_apply_context_t@AAT@@QEAA@PEBUhb_ot_shape_plan_t@@PEAUhb_font_t@@PEAUhb_buffer_t@@PEAUhb_blob_t@@@Z 0000000180012960 f   hb-aat-layout.obj
 0001:00011ab0       ??0hb_ot_apply_context_t@OT@@QEAA@IPEAUhb_font_t@@PEAUhb_buffer_t@@PEAUhb_blob_t@@PEAU?$hb_atomic_t@H@@@Z 0000000180012ab0 f i hb-aat-layout.obj
 0001:00011d70       ??1?$accelerator_t@UGPOS@Layout@OT@@@GSUBGPOS@OT@@QEAA@XZ 0000000180012d70 f i hb-ot-layout.obj
 0001:00011d70       ??1?$accelerator_t@UGSUB@Layout@OT@@@GSUBGPOS@OT@@QEAA@XZ 0000000180012d70 f i hb-aat-layout.obj
 0001:00011df0       ??1accelerator_t@?$KerxTable@Ukerx@AAT@@@AAT@@QEAA@XZ 0000000180012df0 f i hb-aat-layout.obj
 0001:00011df0       ??1accelerator_t@kern@OT@@QEAA@XZ 0000000180012df0 f i hb-ot-layout.obj
 0001:00011e60       ??1accelerator_t@?$mortmorx@Umort@AAT@@UObsoleteTypes@2@$0GNGPHCHE@@AAT@@QEAA@XZ 0000000180012e60 f i hb-aat-layout.obj
 0001:00011e60       ??1accelerator_t@?$mortmorx@Umorx@AAT@@UExtendedTypes@2@$0GNGPHCHI@@AAT@@QEAA@XZ 0000000180012e60 f i hb-aat-layout.obj
 0001:00011fa0       ??1hb_aat_apply_context_t@AAT@@QEAA@XZ 0000000180012fa0 f   hb-aat-layout.obj
 0001:00011fd0       ??1hb_aat_scratch_t@AAT@@QEAA@XZ 0000000180012fd0 f i hb-aat-layout.obj
 0001:00012040       ??4hb_bit_set_t@@QEAAAEAU0@$$QEAU0@@Z 0000000180013040 f i hb-aat-layout.obj
 0001:000120d0       ??C?$hb_lazy_loader_t@Ufeat@AAT@@U?$hb_table_lazy_loader_t@Ufeat@AAT@@$0CC@$0A@@@Uhb_face_t@@$0CC@Uhb_blob_t@@@@QEBAPEBUfeat@AAT@@XZ 00000001800130d0 f i hb-aat-layout.obj
 0001:00012240       ??C?$hb_lazy_loader_t@Ultag@AAT@@U?$hb_table_lazy_loader_t@Ultag@AAT@@$0CB@$0A@@@Uhb_face_t@@$0CB@Uhb_blob_t@@@@QEBAPEBUltag@AAT@@XZ 0000000180013240 f i hb-aat-layout.obj
 0001:000123b0       ?_infos_find_min_cluster@hb_buffer_t@@QEAAIPEBUhb_glyph_info_t@@III@Z 00000001800133b0 f i hb-aat-layout.obj
 0001:00012440       ?_infos_set_glyph_flags@hb_buffer_t@@QEAAXPEAUhb_glyph_info_t@@IIII@Z 0000000180013440 f i hb-aat-layout.obj
 0001:00012530       ?add_range@hb_bit_page_t@@QEAAXII@Z 0000000180013530 f i hb-aat-layout.obj
 0001:000125f0       ?add_range@hb_bit_set_t@@QEAA_NII@Z 00000001800135f0 f i hb-aat-layout.obj
 0001:00012730       ?alloc@?$hb_vector_t@Uhb_bit_page_t@@$0A@@@QEAA_NI_N@Z 0000000180013730 f i hb-aat-layout.obj
 0001:000127f0       ?alloc@?$hb_vector_t@Upage_map_t@hb_bit_set_t@@$00@@QEAA_NI_N@Z 00000001800137f0 f i hb-aat-layout.obj
 0001:000128b0       ?apply@?$Chain@UExtendedTypes@AAT@@@AAT@@QEBAXPEAUhb_aat_apply_context_t@2@PEBUhb_aat_layout_chain_accelerator_t@2@@Z 00000001800138b0 f i hb-aat-layout.obj
 0001:00012cf0       ?apply@?$Chain@UObsoleteTypes@AAT@@@AAT@@QEBAXPEAUhb_aat_apply_context_t@2@PEBUhb_aat_layout_chain_accelerator_t@2@@Z 0000000180013cf0 f i hb-aat-layout.obj
 0001:000130f0       ?apply@?$KerxTable@Ukerx@AAT@@@AAT@@QEBA_NPEAUhb_aat_apply_context_t@2@AEBUkern_accelerator_data_t@2@@Z 00000001800140f0 f i hb-aat-layout.obj
 0001:00013520       ?apply@?$NoncontextualSubtable@UExtendedTypes@AAT@@@AAT@@QEBA_NPEAUhb_aat_apply_context_t@2@@Z 0000000180014520 f i hb-aat-layout.obj
 0001:00013520       ?apply@?$NoncontextualSubtable@UObsoleteTypes@AAT@@@AAT@@QEBA_NPEAUhb_aat_apply_context_t@2@@Z 0000000180014520 f i hb-aat-layout.obj
 0001:00013730       ?apply@?$mortmorx@Umort@AAT@@UObsoleteTypes@2@$0GNGPHCHE@@AAT@@QEBAXPEAUhb_aat_apply_context_t@2@AEBUhb_aat_map_t@@AEBUaccelerator_t@12@@Z 0000000180014730 f i hb-aat-layout.obj
 0001:000139d0       ?apply@?$mortmorx@Umorx@AAT@@UExtendedTypes@2@$0GNGPHCHI@@AAT@@QEBAXPEAUhb_aat_apply_context_t@2@AEBUhb_aat_map_t@@AEBUaccelerator_t@12@@Z 00000001800149d0 f i hb-aat-layout.obj
 0001:00013cd0       ?apply@trak@AAT@@QEBA_NPEAUhb_aat_apply_context_t@2@M@Z 0000000180014cd0 f i hb-aat-layout.obj
 0001:00013ee0       ?backtrack_len@hb_buffer_t@@QEBAIXZ 0000000180014ee0 f i hb-aat-layout.obj
 0001:00013ef0       ?clear@hb_bit_set_t@@QEAAXXZ 0000000180014ef0 f i hb-aat-layout.obj
 0001:00013fd0       ?compile_flags@?$Chain@UExtendedTypes@AAT@@@AAT@@QEBAIPEBUhb_aat_map_builder_t@@@Z 0000000180014fd0 f i hb-aat-layout.obj
 0001:00014200       ?compile_flags@?$Chain@UObsoleteTypes@AAT@@@AAT@@QEBAIPEBUhb_aat_map_builder_t@@@Z 0000000180015200 f i hb-aat-layout.obj
 0001:00014420       ?compile_flags@?$mortmorx@Umort@AAT@@UObsoleteTypes@2@$0GNGPHCHE@@AAT@@QEBAXPEBUhb_aat_map_builder_t@@PEAUhb_aat_map_t@@@Z 0000000180015420 f i hb-aat-layout.obj
 0001:000146b0       ?compile_flags@?$mortmorx@Umorx@AAT@@UExtendedTypes@2@$0GNGPHCHI@@AAT@@QEBAXPEBUhb_aat_map_builder_t@@PEAUhb_aat_map_t@@@Z 00000001800156b0 f i hb-aat-layout.obj
 0001:00014940       ?copy_glyph@hb_buffer_t@@QEAA_NXZ 0000000180015940 f i hb-aat-layout.obj
 0001:000149b0       ?create_accelerator_data@?$KerxTable@Ukerx@AAT@@@AAT@@QEBA?AUkern_accelerator_data_t@2@I@Z 00000001800159b0 f i hb-aat-layout.obj
 0001:00014da0       ?create_buffer_glyph_set@hb_aat_scratch_t@AAT@@QEBAPEAUhb_bit_set_t@@XZ 0000000180015da0 f i hb-aat-layout.obj
 0001:00014e00       ?end_processing@hb_sanitize_context_t@@QEAAXXZ 0000000180015e00 f i hb-aat-layout.obj
 0001:00014e80       ?fini@object_t@hb_serialize_context_t@@QEAAXXZ 0000000180015e80 f i hb-face-builder.obj
 0001:00014e80       ?fini@hb_bit_set_t@@QEAAXXZ 0000000180015e80 f i hb-aat-layout.obj
 0001:00014ee0       ?get@?$hb_lazy_loader_t@UGDEF_accelerator_t@OT@@U?$hb_face_lazy_loader_t@UGDEF_accelerator_t@OT@@$0BI@@@Uhb_face_t@@$0BI@U12@@@QEBAPEBUGDEF_accelerator_t@OT@@XZ 0000000180015ee0 f i hb-aat-layout.obj
 0001:00014fb0       ?get@?$hb_lazy_loader_t@Ukerx_accelerator_t@AAT@@U?$hb_face_lazy_loader_t@Ukerx_accelerator_t@AAT@@$0BO@@@Uhb_face_t@@$0BO@U12@@@QEBAPEBUkerx_accelerator_t@AAT@@XZ 0000000180015fb0 f i hb-aat-layout.obj
 0001:00015060       ?get@?$hb_lazy_loader_t@Umorx_accelerator_t@AAT@@U?$hb_face_lazy_loader_t@Umorx_accelerator_t@AAT@@$0BM@@@Uhb_face_t@@$0BM@U12@@@QEBAPEBUmorx_accelerator_t@AAT@@XZ 0000000180016060 f i hb-aat-layout.obj
 0001:00015110       ?get@?$hb_lazy_loader_t@Utrak@AAT@@U?$hb_table_lazy_loader_t@Utrak@AAT@@$0CA@$0A@@@Uhb_face_t@@$0CA@Uhb_blob_t@@@@QEBAPEBUtrak@AAT@@XZ 0000000180016110 f i hb-aat-layout.obj
 0001:00015280       ?get@hb_bit_set_t@@QEBA_NI@Z 0000000180016280 f i hb-aat-layout.obj
 0001:00015370       ?get_anchor@ankr@AAT@@QEBAAEBUAnchor@2@III@Z 0000000180016370 f i hb-aat-layout.obj
 0001:000154e0       ?get_class@ClassDef@OT@@QEBAII@Z 00000001800164e0 f i hb-aat-layout.obj
 0001:000155f0       ?get_coverage@?$CoverageFormat1_3@USmallTypes@Layout@OT@@@Common@Layout@OT@@AEBAII@Z 00000001800165f0 f i hb-aat-layout.obj
 0001:00015670       ?get_coverage@?$CoverageFormat2_4@USmallTypes@Layout@OT@@@Common@Layout@OT@@AEBAII@Z 0000000180016670 f i hb-aat-layout.obj
 0001:00015760       ?get_feature@feat@AAT@@QEBAAEBUFeatureName@2@W4hb_aat_layout_feature_type_t@@@Z 0000000180016760 f i hb-aat-layout.obj
 0001:000157e0       ?get_glyph_contour_point_for_origin@hb_font_t@@QEAAHIIW4hb_direction_t@@PEAH1@Z 00000001800167e0 f i hb-aat-layout.obj
 0001:00015a40       ?get_glyph_props@GDEF@OT@@QEBAII@Z 0000000180016a40 f i hb-aat-layout.obj
 0001:00015b30       ?get_kerning@?$KerxSubTableFormat0@UKerxSubTableHeader@AAT@@@AAT@@QEBAHIIPEAUhb_aat_apply_context_t@2@@Z 0000000180016b30 f i hb-aat-layout.obj
 0001:00015c80       ?get_kerning@?$KerxSubTableFormat2@UKerxSubTableHeader@AAT@@@AAT@@QEBAHIIPEAUhb_aat_apply_context_t@2@@Z 0000000180016c80 f i hb-aat-layout.obj
 0001:00015e80       ?get_kerning@?$KerxSubTableFormat6@UKerxSubTableHeader@AAT@@@AAT@@QEBAHIIPEAUhb_aat_apply_context_t@2@@Z 0000000180016e80 f i hb-aat-layout.obj
 0001:00016230       ?get_length@?$VarSizedBinSearchArrayOf@U?$LookupSegmentSingle@U?$IntType@G$01@OT@@@AAT@@@OT@@QEBAIXZ 0000000180017230 f i hb-aat-layout.obj
 0001:00016230       ?get_length@?$VarSizedBinSearchArrayOf@U?$LookupSegmentArray@U?$IntType@I$03@OT@@@AAT@@@OT@@QEBAIXZ 0000000180017230 f i hb-aat-layout.obj
 0001:00016230       ?get_length@?$VarSizedBinSearchArrayOf@U?$LookupSegmentArray@U?$IntType@G$01@OT@@@AAT@@@OT@@QEBAIXZ 0000000180017230 f i hb-aat-layout.obj
 0001:00016230       ?get_length@?$VarSizedBinSearchArrayOf@U?$LookupSegmentSingle@U?$OffsetTo@U?$ArrayOf@UAnchor@AAT@@U?$IntType@I$03@OT@@@OT@@U?$IntType@G$01@2@X$0A@@OT@@@AAT@@@OT@@QEBAIXZ 0000000180017230 f i hb-aat-layout.obj
 0001:00016230       ?get_length@?$VarSizedBinSearchArrayOf@U?$LookupSegmentArray@U?$OffsetTo@U?$ArrayOf@UAnchor@AAT@@U?$IntType@I$03@OT@@@OT@@U?$IntType@G$01@2@X$0A@@OT@@@AAT@@@OT@@QEBAIXZ 0000000180017230 f i hb-aat-layout.obj
 0001:00016230       ?get_length@?$VarSizedBinSearchArrayOf@U?$LookupSegmentArray@UHBGlyphID16@OT@@@AAT@@@OT@@QEBAIXZ 0000000180017230 f i hb-aat-layout.obj
 0001:00016230       ?get_length@?$VarSizedBinSearchArrayOf@U?$LookupSegmentSingle@UHBGlyphID16@OT@@@AAT@@@OT@@QEBAIXZ 0000000180017230 f i hb-aat-layout.obj
 0001:00016230       ?get_length@?$VarSizedBinSearchArrayOf@U?$LookupSegmentSingle@U?$IntType@I$03@OT@@@AAT@@@OT@@QEBAIXZ 0000000180017230 f i hb-aat-layout.obj
 0001:000162d0       ?get_length@?$VarSizedBinSearchArrayOf@U?$LookupSingle@U?$IntType@I$03@OT@@@AAT@@@OT@@QEBAIXZ 00000001800172d0 f i hb-aat-layout.obj
 0001:000162d0       ?get_length@?$VarSizedBinSearchArrayOf@U?$LookupSingle@UHBGlyphID16@OT@@@AAT@@@OT@@QEBAIXZ 00000001800172d0 f i hb-aat-layout.obj
 0001:000162d0       ?get_length@?$VarSizedBinSearchArrayOf@U?$LookupSingle@U?$OffsetTo@U?$ArrayOf@UAnchor@AAT@@U?$IntType@I$03@OT@@@OT@@U?$IntType@G$01@2@X$0A@@OT@@@AAT@@@OT@@QEBAIXZ 00000001800172d0 f i hb-aat-layout.obj
 0001:000162d0       ?get_length@?$VarSizedBinSearchArrayOf@U?$LookupSingle@U?$IntType@G$01@OT@@@AAT@@@OT@@QEBAIXZ 00000001800172d0 f i hb-aat-layout.obj
 0001:00016370       ?get_population@Coverage@Common@Layout@OT@@QEBAIXZ 0000000180017370 f i hb-aat-layout.obj
 0001:00016440       ?get_size@HintingDevice@OT@@QEBAIXZ 0000000180017440 f i hb-aat-layout.obj
 0001:000164b0       ?get_stored@?$hb_lazy_loader_t@Umort_accelerator_t@AAT@@U?$hb_face_lazy_loader_t@Umort_accelerator_t@AAT@@$0BN@@@Uhb_face_t@@$0BN@U12@@@QEBAPEAUmort_accelerator_t@AAT@@XZ 00000001800174b0 f i hb-aat-layout.obj
 0001:000166a0       ?get_tracking@TrackData@AAT@@QEBAMPEBXMM@Z 00000001800176a0 f i hb-aat-layout.obj
 0001:00016b00       ?get_value@?$Lookup@UHBGlyphID16@OT@@@AAT@@QEBAPEBUHBGlyphID16@OT@@II@Z 0000000180017b00 f i hb-aat-layout.obj
 0001:00016b00       ?get_value@?$Lookup@U?$IntType@G$01@OT@@@AAT@@QEBAPEBU?$IntType@G$01@OT@@II@Z 0000000180017b00 f i hb-aat-layout.obj
 0001:00016b90       ?get_value@?$LookupFormat2@UHBGlyphID16@OT@@@AAT@@AEBAPEBUHBGlyphID16@OT@@I@Z 0000000180017b90 f i hb-aat-layout.obj
 0001:00016b90       ?get_value@?$LookupFormat2@U?$IntType@G$01@OT@@@AAT@@AEBAPEBU?$IntType@G$01@OT@@I@Z 0000000180017b90 f i hb-aat-layout.obj
 0001:00016b90       ?get_value@?$LookupFormat2@U?$IntType@I$03@OT@@@AAT@@AEBAPEBU?$IntType@I$03@OT@@I@Z 0000000180017b90 f i hb-aat-layout.obj
 0001:00016b90       ?get_value@?$LookupFormat2@U?$OffsetTo@U?$ArrayOf@UAnchor@AAT@@U?$IntType@I$03@OT@@@OT@@U?$IntType@G$01@2@X$0A@@OT@@@AAT@@AEBAPEBU?$OffsetTo@U?$ArrayOf@UAnchor@AAT@@U?$IntType@I$03@OT@@@OT@@U?$IntType@G$01@2@X$0A@@OT@@I@Z 0000000180017b90 f i hb-aat-layout.obj
 0001:00016cd0       ?get_value@?$LookupFormat4@U?$IntType@G$01@OT@@@AAT@@AEBAPEBU?$IntType@G$01@OT@@I@Z 0000000180017cd0 f i hb-aat-layout.obj
 0001:00016cd0       ?get_value@?$LookupFormat4@U?$OffsetTo@U?$ArrayOf@UAnchor@AAT@@U?$IntType@I$03@OT@@@OT@@U?$IntType@G$01@2@X$0A@@OT@@@AAT@@AEBAPEBU?$OffsetTo@U?$ArrayOf@UAnchor@AAT@@U?$IntType@I$03@OT@@@OT@@U?$IntType@G$01@2@X$0A@@OT@@I@Z 0000000180017cd0 f i hb-aat-layout.obj
 0001:00016cd0       ?get_value@?$LookupFormat4@UHBGlyphID16@OT@@@AAT@@AEBAPEBUHBGlyphID16@OT@@I@Z 0000000180017cd0 f i hb-aat-layout.obj
 0001:00016e50       ?get_value@?$LookupFormat4@U?$IntType@I$03@OT@@@AAT@@AEBAPEBU?$IntType@I$03@OT@@I@Z 0000000180017e50 f i hb-aat-layout.obj
 0001:00016fd0       ?get_value@?$LookupFormat6@UHBGlyphID16@OT@@@AAT@@AEBAPEBUHBGlyphID16@OT@@I@Z 0000000180017fd0 f i hb-aat-layout.obj
 0001:00016fd0       ?get_value@?$LookupFormat6@U?$OffsetTo@U?$ArrayOf@UAnchor@AAT@@U?$IntType@I$03@OT@@@OT@@U?$IntType@G$01@2@X$0A@@OT@@@AAT@@AEBAPEBU?$OffsetTo@U?$ArrayOf@UAnchor@AAT@@U?$IntType@I$03@OT@@@OT@@U?$IntType@G$01@2@X$0A@@OT@@I@Z 0000000180017fd0 f i hb-aat-layout.obj
 0001:00016fd0       ?get_value@?$LookupFormat6@U?$IntType@G$01@OT@@@AAT@@AEBAPEBU?$IntType@G$01@OT@@I@Z 0000000180017fd0 f i hb-aat-layout.obj
 0001:00016fd0       ?get_value@?$LookupFormat6@U?$IntType@I$03@OT@@@AAT@@AEBAPEBU?$IntType@I$03@OT@@I@Z 0000000180017fd0 f i hb-aat-layout.obj
 0001:00017100       ?get_value@TrackTableEntry@AAT@@QEBAMMPEBXU?$hb_array_t@$$CBU?$HBFixed@U?$IntType@H$03@OT@@$0BA@@OT@@@@@Z 0000000180018100 f i hb-aat-layout.obj
 0001:000172a0       ?get_value_or_null@?$Lookup@U?$IntType@G$01@OT@@@AAT@@QEBA?BGII@Z 00000001800182a0 f i hb-aat-layout.obj
 0001:00017380       ?get_value_or_null@?$Lookup@U?$IntType@I$03@OT@@@AAT@@QEBA?BIII@Z 0000000180018380 f i hb-aat-layout.obj
 0001:00017500       ?guess_v_origin_minus_h_origin@hb_font_t@@QEAAXIPEAH0@Z 0000000180018500 f i hb-aat-layout.obj
 0001:00017600       ?hb_aat_layout_compile_map@@YAXPEBUhb_aat_map_builder_t@@PEAUhb_aat_map_t@@@Z 0000000180018600 f   hb-aat-layout.obj
 0001:000176d0       ?hb_aat_layout_find_feature_mapping@@YAPEBUhb_aat_feature_mapping_t@@I@Z 00000001800186d0 f   hb-aat-layout.obj
 0001:00017730       ?hb_aat_layout_position@@YAXPEBUhb_ot_shape_plan_t@@PEAUhb_font_t@@PEAUhb_buffer_t@@@Z 0000000180018730 f   hb-aat-layout.obj
 0001:000179c0       ?hb_aat_layout_remove_deleted_glyphs@@YAXPEAUhb_buffer_t@@@Z 00000001800189c0 f   hb-aat-layout.obj
 0001:000179e0       ?hb_aat_layout_substitute@@YAXPEBUhb_ot_shape_plan_t@@PEAUhb_font_t@@PEAUhb_buffer_t@@PEBUhb_feature_t@@I@Z 00000001800189e0 f   hb-aat-layout.obj
 0001:00017d40       ?hb_aat_layout_track@@YAXPEBUhb_ot_shape_plan_t@@PEAUhb_font_t@@PEAUhb_buffer_t@@@Z 0000000180018d40 f   hb-aat-layout.obj
 0001:00017de0       ?init_iters@hb_ot_apply_context_t@OT@@QEAAXXZ 0000000180018de0 f i hb-aat-layout.obj
 0001:00017ef0       ?interpolate_at@TrackTableEntry@AAT@@QEBAMIMPEBXU?$hb_array_t@$$CBU?$HBFixed@U?$IntType@H$03@OT@@$0BA@@OT@@@@@Z 0000000180018ef0 f i hb-aat-layout.obj
 0001:000180b0       ?kern@?$hb_kern_machine_t@Uaccelerator_t@?$KerxSubTableFormat0@UKerxSubTableHeader@AAT@@@AAT@@@OT@@QEBAXPEAUhb_font_t@@PEAUhb_buffer_t@@I_N@Z 00000001800190b0 f i hb-aat-layout.obj
 0001:00018590       ?kern@?$hb_kern_machine_t@Uaccelerator_t@?$KerxSubTableFormat2@UKerxSubTableHeader@AAT@@@AAT@@@OT@@QEBAXPEAUhb_font_t@@PEAUhb_buffer_t@@I_N@Z 0000000180019590 f i hb-aat-layout.obj
 0001:00018a70       ?kern@?$hb_kern_machine_t@Uaccelerator_t@?$KerxSubTableFormat6@UKerxSubTableHeader@AAT@@@AAT@@@OT@@QEBAXPEAUhb_font_t@@PEAUhb_buffer_t@@I_N@Z 0000000180019a70 f i hb-aat-layout.obj
 0001:00018f50       ?mark_set_covers@GDEF@OT@@QEBA_NII@Z 0000000180019f50 f i hb-aat-layout.obj
 0001:000190c0       ?match_properties_mark@hb_ot_apply_context_t@OT@@QEBA_NIII@Z 000000018001a0c0 f i hb-aat-layout.obj
 0001:000191b0       ?may_edit@hb_sanitize_context_t@@QEAA_NPEBXI@Z 000000018001a1b0 f i hb-aat-layout.obj
 0001:00019260       ?message@hb_buffer_t@@QEAA_NPEAUhb_font_t@@PEBDZZ 000000018001a260 f i hb-aat-layout.obj
 0001:00019290       ?neuter@?$OffsetTo@UScript@OT@@U?$IntType@G$01@2@X$00@OT@@QEBA_NPEAUhb_sanitize_context_t@@@Z 000000018001a290 f i hb-aat-layout.obj
 0001:00019290       ?neuter@?$OffsetTo@UFeatureParams@OT@@U?$IntType@G$01@2@X$00@OT@@QEBA_NPEAUhb_sanitize_context_t@@@Z 000000018001a290 f i hb-aat-layout.obj
 0001:00019290       ?neuter@?$OffsetTo@UCoverage@Common@Layout@OT@@U?$IntType@G$01@4@X$00@OT@@QEBA_NPEAUhb_sanitize_context_t@@@Z 000000018001a290 f i hb-aat-layout.obj
 0001:00019290       ?neuter@?$OffsetTo@UAxisValue@OT@@U?$IntType@G$01@2@X$00@OT@@QEBA_NPEAUhb_sanitize_context_t@@@Z 000000018001a290 f i hb-ot-shape.obj
 0001:00019290       ?neuter@?$OffsetTo@UPosLookupSubTable@GPOS_impl@Layout@OT@@U?$IntType@G$01@4@X$00@OT@@QEBA_NPEAUhb_sanitize_context_t@@@Z 000000018001a290 f i hb-ot-layout.obj
 0001:00019290       ?neuter@?$OffsetTo@UCaretValue@OT@@U?$IntType@G$01@2@X$00@OT@@QEBA_NPEAUhb_sanitize_context_t@@@Z 000000018001a290 f i hb-aat-layout.obj
 0001:00019290       ?neuter@?$OffsetTo@UAttachList@OT@@U?$IntType@G$01@2@X$00@OT@@QEBA_NPEAUhb_sanitize_context_t@@@Z 000000018001a290 f i hb-aat-layout.obj
 0001:00019290       ?neuter@?$OffsetTo@UItemVariationStore@OT@@U?$IntType@G$01@2@X$00@OT@@QEBA_NPEAUhb_sanitize_context_t@@@Z 000000018001a290 f i hb-ot-metrics.obj
 0001:00019290       ?neuter@?$OffsetTo@U?$Rule@USmallTypes@Layout@OT@@@OT@@U?$IntType@G$01@2@X$00@OT@@QEBA_NPEAUhb_sanitize_context_t@@@Z 000000018001a290 f i hb-aat-layout.obj
 0001:00019290       ?neuter@?$OffsetTo@UClassDef@OT@@U?$IntType@G$01@2@X$00@OT@@QEBA_NPEAUhb_sanitize_context_t@@@Z 000000018001a290 f i hb-aat-layout.obj
 0001:00019290       ?neuter@?$OffsetTo@U?$LigatureSet@USmallTypes@Layout@OT@@@GSUB_impl@Layout@OT@@U?$IntType@G$01@4@X$00@OT@@QEBA_NPEAUhb_sanitize_context_t@@@Z 000000018001a290 f i hb-aat-layout.obj
 0001:00019290       ?neuter@?$OffsetTo@UDevice@OT@@U?$IntType@G$01@2@X$00@OT@@QEBA_NPEAUhb_sanitize_context_t@@@Z 000000018001a290 f i hb-aat-layout.obj
 0001:00019290       ?neuter@?$OffsetTo@ULigGlyph@OT@@U?$IntType@G$01@2@X$00@OT@@QEBA_NPEAUhb_sanitize_context_t@@@Z 000000018001a290 f i hb-aat-layout.obj
 0001:00019290       ?neuter@?$OffsetTo@UTrackData@AAT@@U?$IntType@G$01@OT@@X$00@OT@@QEBA_NPEAUhb_sanitize_context_t@@@Z 000000018001a290 f i hb-aat-layout.obj
 0001:00019290       ?neuter@?$OffsetTo@ULigatureArray@GPOS_impl@Layout@OT@@U?$IntType@G$01@4@X$00@OT@@QEBA_NPEAUhb_sanitize_context_t@@@Z 000000018001a290 f i hb-ot-layout.obj
 0001:00019290       ?neuter@?$OffsetTo@UMarkArray@GPOS_impl@Layout@OT@@U?$IntType@G$01@4@X$00@OT@@QEBA_NPEAUhb_sanitize_context_t@@@Z 000000018001a290 f i hb-ot-layout.obj
 0001:00019290       ?neuter@?$OffsetTo@U?$List16OfOffsetTo@UPosLookup@GPOS_impl@Layout@OT@@U?$IntType@G$01@4@@OT@@U?$IntType@G$01@2@X$00@OT@@QEBA_NPEAUhb_sanitize_context_t@@@Z 000000018001a290 f i hb-ot-layout.obj
 0001:00019290       ?neuter@?$OffsetTo@U?$Ligature@USmallTypes@Layout@OT@@@GSUB_impl@Layout@OT@@U?$IntType@G$01@4@X$00@OT@@QEBA_NPEAUhb_sanitize_context_t@@@Z 000000018001a290 f i hb-aat-layout.obj
 0001:00019290       ?neuter@?$OffsetTo@UAnchor@GPOS_impl@Layout@OT@@U?$IntType@G$01@4@UAnchorMatrix@234@$00@OT@@QEBA_NPEAUhb_sanitize_context_t@@@Z 000000018001a290 f i hb-ot-layout.obj
 0001:00019290       ?neuter@?$OffsetTo@U?$List16OfOffsetTo@USubstLookup@GSUB_impl@Layout@OT@@U?$IntType@G$01@4@@OT@@U?$IntType@G$01@2@X$00@OT@@QEBA_NPEAUhb_sanitize_context_t@@@Z 000000018001a290 f i hb-aat-layout.obj
 0001:00019290       ?neuter@?$OffsetTo@USubstLookup@GSUB_impl@Layout@OT@@U?$IntType@G$01@4@X$00@OT@@QEBA_NPEAUhb_sanitize_context_t@@@Z 000000018001a290 f i hb-aat-layout.obj
 0001:00019290       ?neuter@?$OffsetTo@UFeature@OT@@U?$IntType@G$01@2@X$00@OT@@QEBA_NPEAUhb_sanitize_context_t@@@Z 000000018001a290 f i hb-aat-layout.obj
 0001:00019290       ?neuter@?$OffsetTo@U?$PairSet@USmallTypes@Layout@OT@@@GPOS_impl@Layout@OT@@U?$IntType@G$01@4@X$00@OT@@QEBA_NPEAUhb_sanitize_context_t@@@Z 000000018001a290 f i hb-ot-layout.obj
 0001:00019290       ?neuter@?$OffsetTo@ULangSys@OT@@U?$IntType@G$01@2@X$00@OT@@QEBA_NPEAUhb_sanitize_context_t@@@Z 000000018001a290 f i hb-aat-layout.obj
 0001:00019290       ?neuter@?$OffsetTo@URecordListOfScript@OT@@U?$IntType@G$01@2@X$00@OT@@QEBA_NPEAUhb_sanitize_context_t@@@Z 000000018001a290 f i hb-aat-layout.obj
 0001:00019290       ?neuter@?$OffsetTo@U?$RecordListOf@UFeature@OT@@@OT@@U?$IntType@G$01@2@X$00@OT@@QEBA_NPEAUhb_sanitize_context_t@@@Z 000000018001a290 f i hb-aat-layout.obj
 0001:00019290       ?neuter@?$OffsetTo@U?$Sequence@USmallTypes@Layout@OT@@@GSUB_impl@Layout@OT@@U?$IntType@G$01@4@X$00@OT@@QEBA_NPEAUhb_sanitize_context_t@@@Z 000000018001a290 f i hb-aat-layout.obj
 0001:00019290       ?neuter@?$OffsetTo@USubstLookupSubTable@GSUB_impl@Layout@OT@@U?$IntType@G$01@4@X$00@OT@@QEBA_NPEAUhb_sanitize_context_t@@@Z 000000018001a290 f i hb-aat-layout.obj
 0001:00019290       ?neuter@?$OffsetTo@UAnchor@GPOS_impl@Layout@OT@@U?$IntType@G$01@4@X$00@OT@@QEBA_NPEAUhb_sanitize_context_t@@@Z 000000018001a290 f i hb-ot-layout.obj
 0001:00019290       ?neuter@?$OffsetTo@UMarkGlyphSets@OT@@U?$IntType@G$01@2@X$00@OT@@QEBA_NPEAUhb_sanitize_context_t@@@Z 000000018001a290 f i hb-aat-layout.obj
 0001:00019290       ?neuter@?$OffsetTo@U?$RuleSet@USmallTypes@Layout@OT@@@OT@@U?$IntType@G$01@2@X$00@OT@@QEBA_NPEAUhb_sanitize_context_t@@@Z 000000018001a290 f i hb-aat-layout.obj
 0001:00019290       ?neuter@?$OffsetTo@UDevice@OT@@U?$IntType@G$01@2@UValueBase@GPOS_impl@Layout@2@$00@OT@@QEBA_NPEAUhb_sanitize_context_t@@@Z 000000018001a290 f i hb-ot-layout.obj
 0001:00019290       ?neuter@?$OffsetTo@ULigCaretList@OT@@U?$IntType@G$01@2@X$00@OT@@QEBA_NPEAUhb_sanitize_context_t@@@Z 000000018001a290 f i hb-aat-layout.obj
 0001:00019290       ?neuter@?$OffsetTo@UAnchorMatrix@GPOS_impl@Layout@OT@@U?$IntType@G$01@4@X$00@OT@@QEBA_NPEAUhb_sanitize_context_t@@@Z 000000018001a290 f i hb-ot-layout.obj
 0001:00019290       ?neuter@?$OffsetTo@U?$AlternateSet@USmallTypes@Layout@OT@@@GSUB_impl@Layout@OT@@U?$IntType@G$01@4@X$00@OT@@QEBA_NPEAUhb_sanitize_context_t@@@Z 000000018001a290 f i hb-aat-layout.obj
 0001:00019290       ?neuter@?$OffsetTo@UPosLookup@GPOS_impl@Layout@OT@@U?$IntType@G$01@4@X$00@OT@@QEBA_NPEAUhb_sanitize_context_t@@@Z 000000018001a290 f i hb-ot-layout.obj
 0001:00019290       ?neuter@?$OffsetTo@U?$ChainRule@USmallTypes@Layout@OT@@@OT@@U?$IntType@G$01@2@X$00@OT@@QEBA_NPEAUhb_sanitize_context_t@@@Z 000000018001a290 f i hb-aat-layout.obj
 0001:00019290       ?neuter@?$OffsetTo@U?$ChainRuleSet@USmallTypes@Layout@OT@@@OT@@U?$IntType@G$01@2@X$00@OT@@QEBA_NPEAUhb_sanitize_context_t@@@Z 000000018001a290 f i hb-aat-layout.obj
 0001:00019290       ?neuter@?$OffsetTo@UAnchor@GPOS_impl@Layout@OT@@U?$IntType@G$01@4@UCursivePosFormat1@234@$00@OT@@QEBA_NPEAUhb_sanitize_context_t@@@Z 000000018001a290 f i hb-ot-layout.obj
 0001:00019290       ?neuter@?$OffsetTo@UAttachPoint@OT@@U?$IntType@G$01@2@X$00@OT@@QEBA_NPEAUhb_sanitize_context_t@@@Z 000000018001a290 f i hb-aat-layout.obj
 0001:000192d0       ?neuter@?$OffsetTo@UCmapSubtable@OT@@U?$IntType@I$03@2@X$00@OT@@QEBA_NPEAUhb_sanitize_context_t@@@Z 000000018001a2d0 f i hb-face.obj
 0001:000192d0       ?neuter@?$OffsetTo@UDeltaSetIndexMap@OT@@U?$IntType@I$03@2@X$00@OT@@QEBA_NPEAUhb_sanitize_context_t@@@Z 000000018001a2d0 f i hb-common.obj
 0001:000192d0       ?neuter@?$OffsetTo@UClipList@OT@@U?$IntType@I$03@2@X$00@OT@@QEBA_NPEAUhb_sanitize_context_t@@@Z 000000018001a2d0 f i hb-ot-color.obj
 0001:000192d0       ?neuter@?$OffsetTo@UBaseGlyphList@OT@@U?$IntType@I$03@2@X$00@OT@@QEBA_NPEAUhb_sanitize_context_t@@@Z 000000018001a2d0 f i hb-ot-color.obj
 0001:000192d0       ?neuter@?$OffsetTo@UFeatureTableSubstitution@OT@@U?$IntType@I$03@2@X$00@OT@@QEBA_NPEAUhb_sanitize_context_t@@@Z 000000018001a2d0 f i hb-aat-layout.obj
 0001:000192d0       ?neuter@?$OffsetTo@UNonDefaultUVS@OT@@U?$IntType@I$03@2@X$00@OT@@QEBA_NPEAUhb_sanitize_context_t@@@Z 000000018001a2d0 f i hb-face.obj
 0001:000192d0       ?neuter@?$OffsetTo@UDefaultUVS@OT@@U?$IntType@I$03@2@X$00@OT@@QEBA_NPEAUhb_sanitize_context_t@@@Z 000000018001a2d0 f i hb-face.obj
 0001:000192d0       ?neuter@?$OffsetTo@USBIXStrike@OT@@U?$IntType@I$03@2@X$00@OT@@QEBA_NPEAUhb_sanitize_context_t@@@Z 000000018001a2d0 f i hb-ot-color.obj
 0001:000192d0       ?neuter@?$OffsetTo@UItemVariationStore@OT@@U?$IntType@I$03@2@X$00@OT@@QEBA_NPEAUhb_sanitize_context_t@@@Z 000000018001a2d0 f i hb-aat-layout.obj
 0001:000192d0       ?neuter@?$OffsetTo@UConditionSet@OT@@U?$IntType@I$03@2@X$00@OT@@QEBA_NPEAUhb_sanitize_context_t@@@Z 000000018001a2d0 f i hb-aat-layout.obj
 0001:000192d0       ?neuter@?$OffsetTo@UOpenTypeOffsetTable@OT@@U?$IntType@I$03@2@X$00@OT@@QEBA_NPEAUhb_sanitize_context_t@@@Z 000000018001a2d0 f i hb-face.obj
 0001:000192d0       ?neuter@?$OffsetTo@U?$Lookup@U?$OffsetTo@U?$ArrayOf@UAnchor@AAT@@U?$IntType@I$03@OT@@@OT@@U?$IntType@G$01@2@X$0A@@OT@@@AAT@@U?$IntType@I$03@OT@@X$00@OT@@QEBA_NPEAUhb_sanitize_context_t@@@Z 000000018001a2d0 f i hb-aat-layout.obj
 0001:000192d0       ?neuter@?$OffsetTo@UPaint@OT@@U?$IntType@I$03@2@X$00@OT@@QEBA_NPEAUhb_sanitize_context_t@@@Z 000000018001a2d0 f i hb-ot-color.obj
 0001:000192d0       ?neuter@?$OffsetTo@UVarRegionList@OT@@U?$IntType@I$03@2@X$00@OT@@QEBA_NPEAUhb_sanitize_context_t@@@Z 000000018001a2d0 f i hb-aat-layout.obj
 0001:000192d0       ?neuter@?$OffsetTo@UVarData@OT@@U?$IntType@I$03@2@X$00@OT@@QEBA_NPEAUhb_sanitize_context_t@@@Z 000000018001a2d0 f i hb-aat-layout.obj
 0001:000192d0       ?neuter@?$OffsetTo@UCondition@OT@@U?$IntType@I$03@2@X$00@OT@@QEBA_NPEAUhb_sanitize_context_t@@@Z 000000018001a2d0 f i hb-aat-layout.obj
 0001:000192d0       ?neuter@?$OffsetTo@UFeatureVariations@OT@@U?$IntType@I$03@2@X$00@OT@@QEBA_NPEAUhb_sanitize_context_t@@@Z 000000018001a2d0 f i hb-aat-layout.obj
 0001:000192d0       ?neuter@?$OffsetTo@UCoverage@Common@Layout@OT@@U?$IntType@I$03@4@X$00@OT@@QEBA_NPEAUhb_sanitize_context_t@@@Z 000000018001a2d0 f i hb-aat-layout.obj
 0001:000192d0       ?neuter@?$OffsetTo@ULayerList@OT@@U?$IntType@I$03@2@X$00@OT@@QEBA_NPEAUhb_sanitize_context_t@@@Z 000000018001a2d0 f i hb-ot-color.obj
 0001:000192d0       ?neuter@?$OffsetTo@UFeature@OT@@U?$IntType@I$03@2@X$00@OT@@QEBA_NPEAUhb_sanitize_context_t@@@Z 000000018001a2d0 f i hb-aat-layout.obj
 0001:000192d0       ?neuter@?$OffsetTo@UIndexSubtable@OT@@U?$IntType@I$03@2@X$00@OT@@QEBA_NPEAUhb_sanitize_context_t@@@Z 000000018001a2d0 f i hb-ot-color.obj
 0001:00019310       ?neuter@?$OffsetTo@UPaint@OT@@U?$IntType@I$02@2@X$00@OT@@QEBA_NPEAUhb_sanitize_context_t@@@Z 000000018001a310 f i hb-ot-color.obj
 0001:00019310       ?neuter@?$OffsetTo@UCondition@OT@@U?$IntType@I$02@2@X$00@OT@@QEBA_NPEAUhb_sanitize_context_t@@@Z 000000018001a310 f i hb-aat-layout.obj
 0001:00019310       ?neuter@?$OffsetTo@U?$NoVariable@UAffine2x3@OT@@@OT@@U?$IntType@I$02@2@X$00@OT@@QEBA_NPEAUhb_sanitize_context_t@@@Z 000000018001a310 f i hb-ot-color.obj
 0001:00019310       ?neuter@?$OffsetTo@U?$Variable@UAffine2x3@OT@@@OT@@U?$IntType@I$02@2@X$00@OT@@QEBA_NPEAUhb_sanitize_context_t@@@Z 000000018001a310 f i hb-ot-color.obj
 0001:00019310       ?neuter@?$OffsetTo@UClipBox@OT@@U?$IntType@I$02@2@X$00@OT@@QEBA_NPEAUhb_sanitize_context_t@@@Z 000000018001a310 f i hb-ot-color.obj
 0001:00019310       ?neuter@?$OffsetTo@U?$ColorLine@UNoVariable@OT@@@OT@@U?$IntType@I$02@2@X$00@OT@@QEBA_NPEAUhb_sanitize_context_t@@@Z 000000018001a310 f i hb-ot-color.obj
 0001:00019310       ?neuter@?$OffsetTo@U?$ColorLine@UVariable@OT@@@OT@@U?$IntType@I$02@2@X$00@OT@@QEBA_NPEAUhb_sanitize_context_t@@@Z 000000018001a310 f i hb-ot-color.obj
 0001:00019350       ?next_glyph@hb_buffer_t@@QEAA_NXZ 000000018001a350 f i hb-aat-layout.obj
 0001:000193f0       ?page_for@hb_bit_set_t@@IEAAPEAUhb_bit_page_t@@I_N@Z 000000018001a3f0 f i hb-aat-layout.obj
 0001:00019570       ?replace_glyph@hb_aat_apply_context_t@AAT@@QEAA_NI@Z 000000018001a570 f i hb-aat-layout.obj
 0001:00019670       ?replace_glyph@hb_buffer_t@@QEAA_NI@Z 000000018001a670 f i hb-aat-layout.obj
 0001:00019700       ?replace_glyph_inplace@hb_aat_apply_context_t@AAT@@QEAAXII@Z 000000018001a700 f i hb-aat-layout.obj
 0001:000197c0       ?resize@?$hb_vector_t@Uhb_bit_page_t@@$0A@@@QEAA_NH_N0@Z 000000018001a7c0 f i hb-aat-layout.obj
 0001:00019860       ?resize@?$hb_vector_t@Upage_map_t@hb_bit_set_t@@$00@@QEAA_NH_N0@Z 000000018001a860 f i hb-aat-layout.obj
 0001:000198e0       ?resize@hb_bit_set_t@@QEAA_NI_N0@Z 000000018001a8e0 f i hb-aat-layout.obj
 0001:00019990       ?reverse_range@hb_buffer_t@@QEAAXII@Z 000000018001a990 f i hb-aat-layout.obj
 0001:00019ac0       ?sanitize@?$Chain@UExtendedTypes@AAT@@@AAT@@QEBA_NPEAUhb_sanitize_context_t@@I@Z 000000018001aac0 f i hb-aat-layout.obj
 0001:00019e70       ?sanitize@?$Chain@UObsoleteTypes@AAT@@@AAT@@QEBA_NPEAUhb_sanitize_context_t@@I@Z 000000018001ae70 f i hb-aat-layout.obj
 0001:0001a0a0       ?sanitize@?$ChainContextFormat2_5@USmallTypes@Layout@OT@@@OT@@QEBA_NPEAUhb_sanitize_context_t@@@Z 000000018001b0a0 f i hb-aat-layout.obj
 0001:0001a2c0       ?sanitize@?$ChainRule@USmallTypes@Layout@OT@@@OT@@QEBA_NPEAUhb_sanitize_context_t@@@Z 000000018001b2c0 f i hb-aat-layout.obj
 0001:0001a4a0       ?sanitize@?$ChainSubtable@UObsoleteTypes@AAT@@@AAT@@QEBA_NPEAUhb_sanitize_context_t@@@Z 000000018001b4a0 f i hb-aat-layout.obj
 0001:0001a620       ?sanitize@?$ContextFormat2_5@USmallTypes@Layout@OT@@@OT@@QEBA_NPEAUhb_sanitize_context_t@@@Z 000000018001b620 f i hb-aat-layout.obj
 0001:0001a7a0       ?sanitize@?$GDEFVersion1_2@USmallTypes@Layout@OT@@@OT@@QEBA_NPEAUhb_sanitize_context_t@@@Z 000000018001b7a0 f i hb-aat-layout.obj
 0001:0001aa90       ?sanitize@?$IntType@G$01@OT@@QEBA_NPEAUhb_sanitize_context_t@@@Z 000000018001ba90 f i hb-aat-layout.obj
 0001:0001ab20       ?sanitize@?$IntType@H$03@OT@@QEBA_NPEAUhb_sanitize_context_t@@@Z 000000018001bb20 f i hb-aat-layout.obj
 0001:0001ab20       ?sanitize@?$IntType@I$03@OT@@QEBA_NPEAUhb_sanitize_context_t@@@Z 000000018001bb20 f i hb-aat-layout.obj
 0001:0001abb0       ?sanitize@?$KerxSubTableFormat2@UKerxSubTableHeader@AAT@@@AAT@@QEBA_NPEAUhb_sanitize_context_t@@@Z 000000018001bbb0 f i hb-aat-layout.obj
 0001:0001add0       ?sanitize@?$KerxSubTableFormat6@UKerxSubTableHeader@AAT@@@AAT@@QEBA_NPEAUhb_sanitize_context_t@@@Z 000000018001bdd0 f i hb-aat-layout.obj
 0001:0001b230       ?sanitize@?$KerxTable@Ukerx@AAT@@@AAT@@QEBA_NPEAUhb_sanitize_context_t@@@Z 000000018001c230 f i hb-aat-layout.obj
 0001:0001b4f0       ?sanitize@?$Lookup@U?$IntType@G$01@OT@@@AAT@@QEBA_NPEAUhb_sanitize_context_t@@@Z 000000018001c4f0 f i hb-aat-layout.obj
 0001:0001b7b0       ?sanitize@?$Lookup@U?$IntType@I$03@OT@@@AAT@@QEBA_NPEAUhb_sanitize_context_t@@@Z 000000018001c7b0 f i hb-aat-layout.obj
 0001:0001ba70       ?sanitize@?$Lookup@U?$OffsetTo@U?$ArrayOf@UAnchor@AAT@@U?$IntType@I$03@OT@@@OT@@U?$IntType@G$01@2@X$0A@@OT@@@AAT@@QEBA_NPEAUhb_sanitize_context_t@@PEBX@Z 000000018001ca70 f i hb-aat-layout.obj
 0001:0001bf10       ?sanitize@?$Lookup@UHBGlyphID16@OT@@@AAT@@QEBA_NPEAUhb_sanitize_context_t@@@Z 000000018001cf10 f i hb-aat-layout.obj
 0001:0001c1c0       ?sanitize@?$LookupFormat4@U?$IntType@G$01@OT@@@AAT@@AEBA_NPEAUhb_sanitize_context_t@@@Z 000000018001d1c0 f i hb-aat-layout.obj
 0001:0001c390       ?sanitize@?$LookupFormat4@U?$IntType@I$03@OT@@@AAT@@AEBA_NPEAUhb_sanitize_context_t@@@Z 000000018001d390 f i hb-aat-layout.obj
 0001:0001c550       ?sanitize@?$LookupFormat4@U?$OffsetTo@U?$ArrayOf@UAnchor@AAT@@U?$IntType@I$03@OT@@@OT@@U?$IntType@G$01@2@X$0A@@OT@@@AAT@@AEBA_NPEAUhb_sanitize_context_t@@PEBX@Z 000000018001d550 f i hb-aat-layout.obj
 0001:0001c730       ?sanitize@?$LookupFormat4@UHBGlyphID16@OT@@@AAT@@AEBA_NPEAUhb_sanitize_context_t@@@Z 000000018001d730 f i hb-aat-layout.obj
 0001:0001c8f0       ?sanitize@?$StateTable@UExtendedTypes@AAT@@UEntryData@?$ContextualSubtable@UExtendedTypes@AAT@@@2@@AAT@@QEBA_NPEAUhb_sanitize_context_t@@PEAI@Z 000000018001d8f0 f i hb-aat-layout.obj
 0001:0001c8f0       ?sanitize@?$StateTable@UExtendedTypes@AAT@@UEntryData@?$InsertionSubtable@UExtendedTypes@AAT@@@2@@AAT@@QEBA_NPEAUhb_sanitize_context_t@@PEAI@Z 000000018001d8f0 f i hb-aat-layout.obj
 0001:0001cd70       ?sanitize@?$StateTable@UExtendedTypes@AAT@@UEntryData@?$Format1Entry@$00@2@@AAT@@QEBA_NPEAUhb_sanitize_context_t@@PEAI@Z 000000018001dd70 f i hb-aat-layout.obj
 0001:0001cd70       ?sanitize@?$StateTable@UExtendedTypes@AAT@@UEntryData@?$KerxSubTableFormat4@UKerxSubTableHeader@AAT@@@2@@AAT@@QEBA_NPEAUhb_sanitize_context_t@@PEAI@Z 000000018001dd70 f i hb-aat-layout.obj
 0001:0001cd70       ?sanitize@?$StateTable@UExtendedTypes@AAT@@UEntryData@?$LigatureEntry@$00@2@@AAT@@QEBA_NPEAUhb_sanitize_context_t@@PEAI@Z 000000018001dd70 f i hb-aat-layout.obj
 0001:0001d200       ?sanitize@?$StateTable@UExtendedTypes@AAT@@X@AAT@@QEBA_NPEAUhb_sanitize_context_t@@PEAI@Z 000000018001e200 f i hb-aat-layout.obj
 0001:0001d5d0       ?sanitize@?$StateTable@UObsoleteTypes@AAT@@UEntryData@?$InsertionSubtable@UObsoleteTypes@AAT@@@2@@AAT@@QEBA_NPEAUhb_sanitize_context_t@@PEAI@Z 000000018001e5d0 f i hb-aat-layout.obj
 0001:0001d5d0       ?sanitize@?$StateTable@UObsoleteTypes@AAT@@UEntryData@?$ContextualSubtable@UObsoleteTypes@AAT@@@2@@AAT@@QEBA_NPEAUhb_sanitize_context_t@@PEAI@Z 000000018001e5d0 f i hb-aat-layout.obj
 0001:0001d9f0       ?sanitize@?$StateTable@UObsoleteTypes@AAT@@X@AAT@@QEBA_NPEAUhb_sanitize_context_t@@PEAI@Z 000000018001e9f0 f i hb-aat-layout.obj
 0001:0001dd70       ?sanitize@?$mortmorx@Umort@AAT@@UObsoleteTypes@2@$0GNGPHCHE@@AAT@@QEBA_NPEAUhb_sanitize_context_t@@@Z 000000018001ed70 f i hb-aat-layout.obj
 0001:0001ded0       ?sanitize@?$mortmorx@Umorx@AAT@@UExtendedTypes@2@$0GNGPHCHI@@AAT@@QEBA_NPEAUhb_sanitize_context_t@@@Z 000000018001eed0 f i hb-aat-layout.obj
 0001:0001e030       ?sanitize@CaretValue@OT@@QEBA_NPEAUhb_sanitize_context_t@@@Z 000000018001f030 f i hb-aat-layout.obj
 0001:0001e240       ?sanitize@ChainContextFormat3@OT@@QEBA_NPEAUhb_sanitize_context_t@@@Z 000000018001f240 f i hb-aat-layout.obj
 0001:0001e4b0       ?sanitize@Condition@OT@@QEBA_NPEAUhb_sanitize_context_t@@@Z 000000018001f4b0 f i hb-aat-layout.obj
 0001:0001e7d0       ?sanitize@ContextFormat3@OT@@QEBA_NPEAUhb_sanitize_context_t@@@Z 000000018001f7d0 f i hb-aat-layout.obj
 0001:0001ea70       ?sanitize@Device@OT@@QEBA_NPEAUhb_sanitize_context_t@@@Z 000000018001fa70 f i hb-aat-layout.obj
 0001:0001ecc0       ?sanitize@Feature@OT@@QEBA_NPEAUhb_sanitize_context_t@@PEBURecord_sanitize_closure_t@2@@Z 000000018001fcc0 f i hb-aat-layout.obj
 0001:0001ef10       ?sanitize@FeatureParams@OT@@QEBA_NPEAUhb_sanitize_context_t@@I@Z 000000018001ff10 f i hb-aat-layout.obj
 0001:0001f1b0       ?sanitize@FeatureTableSubstitution@OT@@QEBA_NPEAUhb_sanitize_context_t@@@Z 00000001800201b0 f i hb-aat-layout.obj
 0001:0001f3a0       ?sanitize@FeatureVariations@OT@@QEBA_NPEAUhb_sanitize_context_t@@@Z 00000001800203a0 f i hb-aat-layout.obj
 0001:0001f580       ?sanitize@GDEF@OT@@QEBA_NPEAUhb_sanitize_context_t@@@Z 0000000180020580 f i hb-aat-layout.obj
 0001:0001f650       ?sanitize@GSUB@Layout@OT@@QEBA_NPEAUhb_sanitize_context_t@@@Z 0000000180020650 f i hb-aat-layout.obj
 0001:0001f720       ?sanitize@ItemVariationStore@OT@@QEBA_NPEAUhb_sanitize_context_t@@@Z 0000000180020720 f i hb-aat-layout.obj
 0001:0001f8e0       ?sanitize@KerxSubTable@AAT@@QEBA_NPEAUhb_sanitize_context_t@@@Z 00000001800208e0 f i hb-aat-layout.obj
 0001:0001fbb0       ?sanitize@LangSys@OT@@QEBA_NPEAUhb_sanitize_context_t@@PEBURecord_sanitize_closure_t@2@@Z 0000000180020bb0 f i hb-aat-layout.obj
 0001:0001fc70       ?sanitize@ReverseChainSingleSubstFormat1@GSUB_impl@Layout@OT@@QEBA_NPEAUhb_sanitize_context_t@@@Z 0000000180020c70 f i hb-aat-layout.obj
 0001:0001fe70       ?sanitize@Script@OT@@QEBA_NPEAUhb_sanitize_context_t@@PEBURecord_sanitize_closure_t@2@@Z 0000000180020e70 f i hb-aat-layout.obj
 0001:00020030       ?sanitize@SubtableGlyphCoverage@AAT@@QEBA_NPEAUhb_sanitize_context_t@@I@Z 0000000180021030 f i hb-aat-layout.obj
 0001:000201e0       ?sanitize@TrackData@AAT@@QEBA_NPEAUhb_sanitize_context_t@@PEBX@Z 00000001800211e0 f i hb-aat-layout.obj
 0001:00020420       ?sanitize@ankr@AAT@@QEBA_NPEAUhb_sanitize_context_t@@@Z 0000000180021420 f i hb-aat-layout.obj
 0001:00020630       ?sanitize@feat@AAT@@QEBA_NPEAUhb_sanitize_context_t@@@Z 0000000180021630 f i hb-aat-layout.obj
 0001:00020800       ?sanitize@ltag@AAT@@QEBA_NPEAUhb_sanitize_context_t@@@Z 0000000180021800 f i hb-aat-layout.obj
 0001:000209e0       ?sanitize@trak@AAT@@QEBA_NPEAUhb_sanitize_context_t@@@Z 00000001800219e0 f i hb-aat-layout.obj
 0001:00020b60       ?sanitize_shallow@?$ArrayOf@U?$IntType@E$00@OT@@U?$IntType@G$01@2@@OT@@QEBA_NPEAUhb_sanitize_context_t@@@Z 0000000180021b60 f i hb-aat-layout.obj
 0001:00020cd0       ?sanitize_shallow@?$ArrayOf@U?$Offset@U?$IntType@G$01@OT@@$00@OT@@U?$IntType@G$01@2@@OT@@QEBA_NPEAUhb_sanitize_context_t@@@Z 0000000180021cd0 f i hb-aat-layout.obj
 0001:00020cd0       ?sanitize_shallow@?$ArrayOf@U?$OffsetTo@UAnchorMatrix@GPOS_impl@Layout@OT@@U?$IntType@G$01@4@X$00@OT@@U?$IntType@G$01@2@@OT@@QEBA_NPEAUhb_sanitize_context_t@@@Z 0000000180021cd0 f i hb-ot-layout.obj
 0001:00020cd0       ?sanitize_shallow@?$ArrayOf@U?$OffsetTo@U?$Ligature@USmallTypes@Layout@OT@@@GSUB_impl@Layout@OT@@U?$IntType@G$01@4@X$00@OT@@U?$IntType@G$01@2@@OT@@QEBA_NPEAUhb_sanitize_context_t@@@Z 0000000180021cd0 f i hb-aat-layout.obj
 0001:00020cd0       ?sanitize_shallow@?$ArrayOf@U?$OffsetTo@U?$PairSet@USmallTypes@Layout@OT@@@GPOS_impl@Layout@OT@@U?$IntType@G$01@4@X$00@OT@@U?$IntType@G$01@2@@OT@@QEBA_NPEAUhb_sanitize_context_t@@@Z 0000000180021cd0 f i hb-ot-layout.obj
 0001:00020cd0       ?sanitize_shallow@?$ArrayOf@U?$OffsetTo@U?$LigatureSet@USmallTypes@Layout@OT@@@GSUB_impl@Layout@OT@@U?$IntType@G$01@4@X$00@OT@@U?$IntType@G$01@2@@OT@@QEBA_NPEAUhb_sanitize_context_t@@@Z 0000000180021cd0 f i hb-aat-layout.obj
 0001:00020cd0       ?sanitize_shallow@?$ArrayOf@UHBGlyphID16@OT@@U?$IntType@G$01@2@@OT@@QEBA_NPEAUhb_sanitize_context_t@@@Z 0000000180021cd0 f i hb-aat-layout.obj
 0001:00020cd0       ?sanitize_shallow@?$ArrayOf@U?$IntType@G$01@OT@@U12@@OT@@QEBA_NPEAUhb_sanitize_context_t@@@Z 0000000180021cd0 f i hb-aat-layout.obj
 0001:00020cd0       ?sanitize_shallow@?$ArrayOf@U?$OffsetTo@UPosLookup@GPOS_impl@Layout@OT@@U?$IntType@G$01@4@X$00@OT@@U?$IntType@G$01@2@@OT@@QEBA_NPEAUhb_sanitize_context_t@@@Z 0000000180021cd0 f i hb-ot-layout.obj
 0001:00020cd0       ?sanitize_shallow@?$ArrayOf@U?$OffsetTo@U?$ChainRule@USmallTypes@Layout@OT@@@OT@@U?$IntType@G$01@2@X$00@OT@@U?$IntType@G$01@2@@OT@@QEBA_NPEAUhb_sanitize_context_t@@@Z 0000000180021cd0 f i hb-aat-layout.obj
 0001:00020cd0       ?sanitize_shallow@?$ArrayOf@U?$OffsetTo@USubstLookupSubTable@GSUB_impl@Layout@OT@@U?$IntType@G$01@4@X$00@OT@@U?$IntType@G$01@2@@OT@@QEBA_NPEAUhb_sanitize_context_t@@@Z 0000000180021cd0 f i hb-aat-layout.obj
 0001:00020cd0       ?sanitize_shallow@?$ArrayOf@U?$OffsetTo@U?$AlternateSet@USmallTypes@Layout@OT@@@GSUB_impl@Layout@OT@@U?$IntType@G$01@4@X$00@OT@@U?$IntType@G$01@2@@OT@@QEBA_NPEAUhb_sanitize_context_t@@@Z 0000000180021cd0 f i hb-aat-layout.obj
 0001:00020cd0       ?sanitize_shallow@?$ArrayOf@UIndex@OT@@U?$IntType@G$01@2@@OT@@QEBA_NPEAUhb_sanitize_context_t@@@Z 0000000180021cd0 f i hb-aat-layout.obj
 0001:00020cd0       ?sanitize_shallow@?$ArrayOf@U?$OffsetTo@U?$RuleSet@USmallTypes@Layout@OT@@@OT@@U?$IntType@G$01@2@X$00@OT@@U?$IntType@G$01@2@@OT@@QEBA_NPEAUhb_sanitize_context_t@@@Z 0000000180021cd0 f i hb-aat-layout.obj
 0001:00020cd0       ?sanitize_shallow@?$ArrayOf@U?$OffsetTo@UAttachPoint@OT@@U?$IntType@G$01@2@X$00@OT@@U?$IntType@G$01@2@@OT@@QEBA_NPEAUhb_sanitize_context_t@@@Z 0000000180021cd0 f i hb-aat-layout.obj
 0001:00020cd0       ?sanitize_shallow@?$ArrayOf@U?$OffsetTo@UCoverage@Common@Layout@OT@@U?$IntType@G$01@4@X$00@OT@@U?$IntType@G$01@2@@OT@@QEBA_NPEAUhb_sanitize_context_t@@@Z 0000000180021cd0 f i hb-aat-layout.obj
 0001:00020cd0       ?sanitize_shallow@?$ArrayOf@U?$OffsetTo@ULigGlyph@OT@@U?$IntType@G$01@2@X$00@OT@@U?$IntType@G$01@2@@OT@@QEBA_NPEAUhb_sanitize_context_t@@@Z 0000000180021cd0 f i hb-aat-layout.obj
 0001:00020cd0       ?sanitize_shallow@?$ArrayOf@U?$OffsetTo@U?$Rule@USmallTypes@Layout@OT@@@OT@@U?$IntType@G$01@2@X$00@OT@@U?$IntType@G$01@2@@OT@@QEBA_NPEAUhb_sanitize_context_t@@@Z 0000000180021cd0 f i hb-aat-layout.obj
 0001:00020cd0       ?sanitize_shallow@?$ArrayOf@U?$OffsetTo@UPosLookupSubTable@GPOS_impl@Layout@OT@@U?$IntType@G$01@4@X$00@OT@@U?$IntType@G$01@2@@OT@@QEBA_NPEAUhb_sanitize_context_t@@@Z 0000000180021cd0 f i hb-ot-layout.obj
 0001:00020cd0       ?sanitize_shallow@?$ArrayOf@U?$OffsetTo@UCaretValue@OT@@U?$IntType@G$01@2@X$00@OT@@U?$IntType@G$01@2@@OT@@QEBA_NPEAUhb_sanitize_context_t@@@Z 0000000180021cd0 f i hb-aat-layout.obj
 0001:00020cd0       ?sanitize_shallow@?$ArrayOf@U?$OffsetTo@USubstLookup@GSUB_impl@Layout@OT@@U?$IntType@G$01@4@X$00@OT@@U?$IntType@G$01@2@@OT@@QEBA_NPEAUhb_sanitize_context_t@@@Z 0000000180021cd0 f i hb-aat-layout.obj
 0001:00020cd0       ?sanitize_shallow@?$ArrayOf@U?$OffsetTo@U?$ChainRuleSet@USmallTypes@Layout@OT@@@OT@@U?$IntType@G$01@2@X$00@OT@@U?$IntType@G$01@2@@OT@@QEBA_NPEAUhb_sanitize_context_t@@@Z 0000000180021cd0 f i hb-aat-layout.obj
 0001:00020cd0       ?sanitize_shallow@?$ArrayOf@U?$OffsetTo@U?$Sequence@USmallTypes@Layout@OT@@@GSUB_impl@Layout@OT@@U?$IntType@G$01@4@X$00@OT@@U?$IntType@G$01@2@@OT@@QEBA_NPEAUhb_sanitize_context_t@@@Z 0000000180021cd0 f i hb-aat-layout.obj
 0001:00020e30       ?sanitize_shallow@?$ArrayOf@U?$FDSelect3_4_Range@U?$IntType@G$01@OT@@U?$IntType@E$00@2@@CFF@@U?$IntType@G$01@OT@@@OT@@QEBA_NPEAUhb_sanitize_context_t@@@Z 0000000180021e30 f i hb-ot-font.obj
 0001:00020e30       ?sanitize_shallow@?$ArrayOf@U?$IntType@I$02@OT@@U?$IntType@G$01@2@@OT@@QEBA_NPEAUhb_sanitize_context_t@@@Z 0000000180021e30 f i hb-aat-layout.obj
 0001:00020f90       ?sanitize_shallow@?$ArrayOf@U?$OffsetTo@UCondition@OT@@U?$IntType@I$02@2@X$00@OT@@U?$IntType@E$00@2@@OT@@QEBA_NPEAUhb_sanitize_context_t@@@Z 0000000180021f90 f i hb-aat-layout.obj
 0001:00020f90       ?sanitize_shallow@?$ArrayOf@USuppEncoding@CFF@@U?$IntType@E$00@OT@@@OT@@QEBA_NPEAUhb_sanitize_context_t@@@Z 0000000180021f90 f i hb-ot-font.obj
 0001:000210f0       ?sanitize_shallow@?$ArrayOf@U?$OffsetTo@UCoverage@Common@Layout@OT@@U?$IntType@I$03@4@X$00@OT@@U?$IntType@G$01@2@@OT@@QEBA_NPEAUhb_sanitize_context_t@@@Z 00000001800220f0 f i hb-aat-layout.obj
 0001:000210f0       ?sanitize_shallow@?$ArrayOf@U?$OffsetTo@UCondition@OT@@U?$IntType@I$03@2@X$00@OT@@U?$IntType@G$01@2@@OT@@QEBA_NPEAUhb_sanitize_context_t@@@Z 00000001800220f0 f i hb-aat-layout.obj
 0001:000210f0       ?sanitize_shallow@?$ArrayOf@ULookupRecord@OT@@U?$IntType@G$01@2@@OT@@QEBA_NPEAUhb_sanitize_context_t@@@Z 00000001800220f0 f i hb-aat-layout.obj
 0001:000210f0       ?sanitize_shallow@?$ArrayOf@UAxisValueMap@OT@@U?$IntType@G$01@2@@OT@@QEBA_NPEAUhb_sanitize_context_t@@@Z 00000001800220f0 f i hb-font.obj
 0001:000210f0       ?sanitize_shallow@?$ArrayOf@UVertOriginMetric@OT@@U?$IntType@G$01@2@@OT@@QEBA_NPEAUhb_sanitize_context_t@@@Z 00000001800220f0 f i hb-ot-font.obj
 0001:000210f0       ?sanitize_shallow@?$ArrayOf@UEntryExitRecord@GPOS_impl@Layout@OT@@U?$IntType@G$01@4@@OT@@QEBA_NPEAUhb_sanitize_context_t@@@Z 00000001800220f0 f i hb-ot-layout.obj
 0001:000210f0       ?sanitize_shallow@?$ArrayOf@U?$OffsetTo@UVarData@OT@@U?$IntType@I$03@2@X$00@OT@@U?$IntType@G$01@2@@OT@@QEBA_NPEAUhb_sanitize_context_t@@@Z 00000001800220f0 f i hb-aat-layout.obj
 0001:000210f0       ?sanitize_shallow@?$ArrayOf@UMarkRecord@GPOS_impl@Layout@OT@@U?$IntType@G$01@4@@OT@@QEBA_NPEAUhb_sanitize_context_t@@@Z 00000001800220f0 f i hb-ot-layout.obj
 0001:00021260       ?sanitize_shallow@?$ArrayOf@U?$NoVariable@UColorStop@OT@@@OT@@U?$IntType@G$01@2@@OT@@QEBA_NPEAUhb_sanitize_context_t@@@Z 0000000180022260 f i hb-ot-color.obj
 0001:00021260       ?sanitize_shallow@?$ArrayOf@U?$Record@ULangSys@OT@@@OT@@U?$IntType@G$01@2@@OT@@QEBA_NPEAUhb_sanitize_context_t@@@Z 0000000180022260 f i hb-aat-layout.obj
 0001:00021260       ?sanitize_shallow@?$ArrayOf@U?$Record@UFeature@OT@@@OT@@U?$IntType@G$01@2@@OT@@QEBA_NPEAUhb_sanitize_context_t@@@Z 0000000180022260 f i hb-aat-layout.obj
 0001:00021260       ?sanitize_shallow@?$ArrayOf@U?$Record@UScript@OT@@@OT@@U?$IntType@G$01@2@@OT@@QEBA_NPEAUhb_sanitize_context_t@@@Z 0000000180022260 f i hb-aat-layout.obj
 0001:00021260       ?sanitize_shallow@?$ArrayOf@U?$RangeRecord@USmallTypes@Layout@OT@@@Common@Layout@OT@@U?$IntType@G$01@4@@OT@@QEBA_NPEAUhb_sanitize_context_t@@@Z 0000000180022260 f i hb-aat-layout.obj
 0001:00021260       ?sanitize_shallow@?$ArrayOf@UFeatureTableSubstitutionRecord@OT@@U?$IntType@G$01@2@@OT@@QEBA_NPEAUhb_sanitize_context_t@@@Z 0000000180022260 f i hb-aat-layout.obj
 0001:000213d0       ?sanitize_shallow@?$ArrayOf@UFTStringRange@AAT@@U?$IntType@I$03@OT@@@OT@@QEBA_NPEAUhb_sanitize_context_t@@@Z 00000001800223d0 f i hb-aat-layout.obj
 0001:000213d0       ?sanitize_shallow@?$ArrayOf@U?$OffsetTo@UOpenTypeOffsetTable@OT@@U?$IntType@I$03@2@X$00@OT@@U?$IntType@I$03@2@@OT@@QEBA_NPEAUhb_sanitize_context_t@@@Z 00000001800223d0 f i hb-face.obj
 0001:000213d0       ?sanitize_shallow@?$ArrayOf@U?$OffsetTo@UPaint@OT@@U?$IntType@I$03@2@X$00@OT@@U?$IntType@I$03@2@@OT@@QEBA_NPEAUhb_sanitize_context_t@@@Z 00000001800223d0 f i hb-ot-color.obj
 0001:000213d0       ?sanitize_shallow@?$ArrayOf@UAnchor@AAT@@U?$IntType@I$03@OT@@@OT@@QEBA_NPEAUhb_sanitize_context_t@@@Z 00000001800223d0 f i hb-aat-layout.obj
 0001:000213d0       ?sanitize_shallow@?$ArrayOf@UUnicodeValueRange@OT@@U?$IntType@I$03@2@@OT@@QEBA_NPEAUhb_sanitize_context_t@@@Z 00000001800223d0 f i hb-face.obj
 0001:000213d0       ?sanitize_shallow@?$ArrayOf@U?$OffsetTo@USBIXStrike@OT@@U?$IntType@I$03@2@X$00@OT@@U?$IntType@I$03@2@@OT@@QEBA_NPEAUhb_sanitize_context_t@@@Z 00000001800223d0 f i hb-ot-color.obj
 0001:00021550       ?sanitize_shallow@?$ArrayOf@UFeatureVariationRecord@OT@@U?$IntType@I$03@2@@OT@@QEBA_NPEAUhb_sanitize_context_t@@@Z 0000000180022550 f i hb-aat-layout.obj
 0001:000216d0       ?sanitize_shallow@?$ArrayOf@UKernPair@AAT@@U?$BinSearchHeader@U?$IntType@I$03@OT@@@OT@@@OT@@QEBA_NPEAUhb_sanitize_context_t@@@Z 00000001800226d0 f i hb-aat-layout.obj
 0001:00021860       ?sanitize_shallow@?$HeadlessArrayOf@UHBGlyphID16@OT@@U?$IntType@G$01@2@@OT@@AEBA_NPEAUhb_sanitize_context_t@@@Z 0000000180022860 f i hb-aat-layout.obj
 0001:000219e0       ?sanitize_shallow@?$OffsetTo@ULigCaretList@OT@@U?$IntType@G$01@2@X$00@OT@@QEBA_NPEAUhb_sanitize_context_t@@PEBX@Z 00000001800229e0 f i hb-aat-layout.obj
 0001:000219e0       ?sanitize_shallow@?$OffsetTo@UPosLookupSubTable@GPOS_impl@Layout@OT@@U?$IntType@G$01@4@X$00@OT@@QEBA_NPEAUhb_sanitize_context_t@@PEBX@Z 00000001800229e0 f i hb-ot-layout.obj
 0001:000219e0       ?sanitize_shallow@?$OffsetTo@UCoverage@Common@Layout@OT@@U?$IntType@G$01@4@X$00@OT@@QEBA_NPEAUhb_sanitize_context_t@@PEBX@Z 00000001800229e0 f i hb-aat-layout.obj
 0001:000219e0       ?sanitize_shallow@?$OffsetTo@U?$RuleSet@USmallTypes@Layout@OT@@@OT@@U?$IntType@G$01@2@X$00@OT@@QEBA_NPEAUhb_sanitize_context_t@@PEBX@Z 00000001800229e0 f i hb-aat-layout.obj
 0001:000219e0       ?sanitize_shallow@?$OffsetTo@UMarkGlyphSets@OT@@U?$IntType@G$01@2@X$00@OT@@QEBA_NPEAUhb_sanitize_context_t@@PEBX@Z 00000001800229e0 f i hb-aat-layout.obj
 0001:000219e0       ?sanitize_shallow@?$OffsetTo@U?$RecordListOf@UFeature@OT@@@OT@@U?$IntType@G$01@2@X$00@OT@@QEBA_NPEAUhb_sanitize_context_t@@PEBX@Z 00000001800229e0 f i hb-aat-layout.obj
 0001:000219e0       ?sanitize_shallow@?$OffsetTo@U?$ArrayOfM1@UResourceTypeRecord@OT@@U?$IntType@G$01@2@@OT@@U?$IntType@G$01@2@X$0A@@OT@@QEBA_NPEAUhb_sanitize_context_t@@PEBX@Z 00000001800229e0 f i hb-face.obj
 0001:000219e0       ?sanitize_shallow@?$OffsetTo@U?$ClassTable@U?$IntType@E$00@OT@@@AAT@@U?$IntType@G$01@OT@@X$0A@@OT@@QEBA_NPEAUhb_sanitize_context_t@@PEBX@Z 00000001800229e0 f i hb-aat-layout.obj
 0001:000219e0       ?sanitize_shallow@?$OffsetTo@U?$List16OfOffsetTo@USubstLookup@GSUB_impl@Layout@OT@@U?$IntType@G$01@4@@OT@@U?$IntType@G$01@2@X$00@OT@@QEBA_NPEAUhb_sanitize_context_t@@PEBX@Z 00000001800229e0 f i hb-aat-layout.obj
 0001:000219e0       ?sanitize_shallow@?$OffsetTo@URecordListOfScript@OT@@U?$IntType@G$01@2@X$00@OT@@QEBA_NPEAUhb_sanitize_context_t@@PEBX@Z 00000001800229e0 f i hb-aat-layout.obj
 0001:000219e0       ?sanitize_shallow@?$OffsetTo@UDevice@OT@@U?$IntType@G$01@2@UValueBase@GPOS_impl@Layout@2@$00@OT@@QEBA_NPEAUhb_sanitize_context_t@@PEBUValueBase@GPOS_impl@Layout@2@@Z 00000001800229e0 f i hb-ot-layout.obj
 0001:000219e0       ?sanitize_shallow@?$OffsetTo@UAxisValue@OT@@U?$IntType@G$01@2@X$00@OT@@QEBA_NPEAUhb_sanitize_context_t@@PEBX@Z 00000001800229e0 f i hb-ot-shape.obj
 0001:000219e0       ?sanitize_shallow@?$OffsetTo@UCaretValue@OT@@U?$IntType@G$01@2@X$00@OT@@QEBA_NPEAUhb_sanitize_context_t@@PEBX@Z 00000001800229e0 f i hb-aat-layout.obj
 0001:000219e0       ?sanitize_shallow@?$OffsetTo@UFeature@OT@@U?$IntType@G$01@2@X$00@OT@@QEBA_NPEAUhb_sanitize_context_t@@PEBX@Z 00000001800229e0 f i hb-aat-layout.obj
 0001:000219e0       ?sanitize_shallow@?$OffsetTo@U?$LigatureSet@USmallTypes@Layout@OT@@@GSUB_impl@Layout@OT@@U?$IntType@G$01@4@X$00@OT@@QEBA_NPEAUhb_sanitize_context_t@@PEBX@Z 00000001800229e0 f i hb-aat-layout.obj
 0001:000219e0       ?sanitize_shallow@?$OffsetTo@UTrackData@AAT@@U?$IntType@G$01@OT@@X$00@OT@@QEBA_NPEAUhb_sanitize_context_t@@PEBX@Z 00000001800229e0 f i hb-aat-layout.obj
 0001:000219e0       ?sanitize_shallow@?$OffsetTo@ULigGlyph@OT@@U?$IntType@G$01@2@X$00@OT@@QEBA_NPEAUhb_sanitize_context_t@@PEBX@Z 00000001800229e0 f i hb-aat-layout.obj
 0001:000219e0       ?sanitize_shallow@?$OffsetTo@U?$ClassTable@U?$IntType@G$01@OT@@@AAT@@U?$IntType@G$01@OT@@X$0A@@OT@@QEBA_NPEAUhb_sanitize_context_t@@PEBX@Z 00000001800229e0 f i hb-ot-layout.obj
 0001:000219e0       ?sanitize_shallow@?$OffsetTo@U?$Sequence@USmallTypes@Layout@OT@@@GSUB_impl@Layout@OT@@U?$IntType@G$01@4@X$00@OT@@QEBA_NPEAUhb_sanitize_context_t@@PEBX@Z 00000001800229e0 f i hb-aat-layout.obj
 0001:000219e0       ?sanitize_shallow@?$OffsetTo@U?$UnsizedArrayOf@U?$IntType@F$01@OT@@@OT@@U?$IntType@G$01@2@X$0A@@OT@@QEBA_NPEAUhb_sanitize_context_t@@PEBX@Z 00000001800229e0 f i hb-aat-layout.obj
 0001:000219e0       ?sanitize_shallow@?$OffsetTo@U?$AlternateSet@USmallTypes@Layout@OT@@@GSUB_impl@Layout@OT@@U?$IntType@G$01@4@X$00@OT@@QEBA_NPEAUhb_sanitize_context_t@@PEBX@Z 00000001800229e0 f i hb-aat-layout.obj
 0001:000219e0       ?sanitize_shallow@?$OffsetTo@U?$ArrayOf@UAnchor@AAT@@U?$IntType@I$03@OT@@@OT@@U?$IntType@G$01@2@X$0A@@OT@@QEBA_NPEAUhb_sanitize_context_t@@PEBX@Z 00000001800229e0 f i hb-aat-layout.obj
 0001:000219e0       ?sanitize_shallow@?$OffsetTo@U?$ChainRuleSet@USmallTypes@Layout@OT@@@OT@@U?$IntType@G$01@2@X$00@OT@@QEBA_NPEAUhb_sanitize_context_t@@PEBX@Z 00000001800229e0 f i hb-aat-layout.obj
 0001:000219e0       ?sanitize_shallow@?$OffsetTo@UFeatureParams@OT@@U?$IntType@G$01@2@X$00@OT@@QEBA_NPEAUhb_sanitize_context_t@@PEBX@Z 00000001800229e0 f i hb-aat-layout.obj
 0001:000219e0       ?sanitize_shallow@?$OffsetTo@U?$UnsizedArrayOf@U?$IntType@G$01@OT@@@OT@@U?$IntType@G$01@2@X$0A@@OT@@QEBA_NPEAUhb_sanitize_context_t@@PEBX@Z 00000001800229e0 f i hb-aat-layout.obj
 0001:000219e0       ?sanitize_shallow@?$OffsetTo@USubstLookupSubTable@GSUB_impl@Layout@OT@@U?$IntType@G$01@4@X$00@OT@@QEBA_NPEAUhb_sanitize_context_t@@PEBX@Z 00000001800229e0 f i hb-aat-layout.obj
 0001:000219e0       ?sanitize_shallow@?$OffsetTo@UAttachList@OT@@U?$IntType@G$01@2@X$00@OT@@QEBA_NPEAUhb_sanitize_context_t@@PEBX@Z 00000001800229e0 f i hb-aat-layout.obj
 0001:000219e0       ?sanitize_shallow@?$OffsetTo@ULigatureArray@GPOS_impl@Layout@OT@@U?$IntType@G$01@4@X$00@OT@@QEBA_NPEAUhb_sanitize_context_t@@PEBX@Z 00000001800229e0 f i hb-ot-layout.obj
 0001:000219e0       ?sanitize_shallow@?$OffsetTo@U?$Rule@USmallTypes@Layout@OT@@@OT@@U?$IntType@G$01@2@X$00@OT@@QEBA_NPEAUhb_sanitize_context_t@@PEBX@Z 00000001800229e0 f i hb-aat-layout.obj
 0001:000219e0       ?sanitize_shallow@?$OffsetTo@UPosLookup@GPOS_impl@Layout@OT@@U?$IntType@G$01@4@X$00@OT@@QEBA_NPEAUhb_sanitize_context_t@@PEBX@Z 00000001800229e0 f i hb-ot-layout.obj
 0001:000219e0       ?sanitize_shallow@?$OffsetTo@UMarkArray@GPOS_impl@Layout@OT@@U?$IntType@G$01@4@X$00@OT@@QEBA_NPEAUhb_sanitize_context_t@@PEBX@Z 00000001800229e0 f i hb-ot-layout.obj
 0001:000219e0       ?sanitize_shallow@?$OffsetTo@ULangSys@OT@@U?$IntType@G$01@2@X$00@OT@@QEBA_NPEAUhb_sanitize_context_t@@PEBX@Z 00000001800229e0 f i hb-aat-layout.obj
 0001:000219e0       ?sanitize_shallow@?$OffsetTo@U?$UnsizedListOfOffset16To@U?$Lookup@UHBGlyphID16@OT@@@AAT@@U?$IntType@G$01@OT@@X$0A@@OT@@U?$IntType@G$01@2@X$0A@@OT@@QEBA_NPEAUhb_sanitize_context_t@@PEBX@Z 00000001800229e0 f i hb-aat-layout.obj
 0001:000219e0       ?sanitize_shallow@?$OffsetTo@UItemVariationStore@OT@@U?$IntType@G$01@2@X$00@OT@@QEBA_NPEAUhb_sanitize_context_t@@PEBX@Z 00000001800229e0 f i hb-ot-metrics.obj
 0001:000219e0       ?sanitize_shallow@?$OffsetTo@UAnchor@GPOS_impl@Layout@OT@@U?$IntType@G$01@4@X$00@OT@@QEBA_NPEAUhb_sanitize_context_t@@PEBX@Z 00000001800229e0 f i hb-ot-layout.obj
 0001:000219e0       ?sanitize_shallow@?$OffsetTo@UDevice@OT@@U?$IntType@G$01@2@X$00@OT@@QEBA_NPEAUhb_sanitize_context_t@@PEBX@Z 00000001800229e0 f i hb-aat-layout.obj
 0001:000219e0       ?sanitize_shallow@?$OffsetTo@UAnchor@GPOS_impl@Layout@OT@@U?$IntType@G$01@4@UAnchorMatrix@234@$00@OT@@QEBA_NPEAUhb_sanitize_context_t@@PEBUAnchorMatrix@GPOS_impl@Layout@2@@Z 00000001800229e0 f i hb-ot-layout.obj
 0001:000219e0       ?sanitize_shallow@?$OffsetTo@U?$PairSet@USmallTypes@Layout@OT@@@GPOS_impl@Layout@OT@@U?$IntType@G$01@4@X$00@OT@@QEBA_NPEAUhb_sanitize_context_t@@PEBX@Z 00000001800229e0 f i hb-ot-layout.obj
 0001:000219e0       ?sanitize_shallow@?$OffsetTo@UAttachPoint@OT@@U?$IntType@G$01@2@X$00@OT@@QEBA_NPEAUhb_sanitize_context_t@@PEBX@Z 00000001800229e0 f i hb-aat-layout.obj
 0001:000219e0       ?sanitize_shallow@?$OffsetTo@U?$List16OfOffsetTo@UPosLookup@GPOS_impl@Layout@OT@@U?$IntType@G$01@4@@OT@@U?$IntType@G$01@2@X$00@OT@@QEBA_NPEAUhb_sanitize_context_t@@PEBX@Z 00000001800229e0 f i hb-ot-layout.obj
 0001:000219e0       ?sanitize_shallow@?$OffsetTo@U?$UnsizedArrayOf@UResourceRecord@OT@@@OT@@U?$IntType@G$01@2@X$0A@@OT@@QEBA_NPEAUhb_sanitize_context_t@@PEBX@Z 00000001800229e0 f i hb-face.obj
 0001:000219e0       ?sanitize_shallow@?$OffsetTo@UScript@OT@@U?$IntType@G$01@2@X$00@OT@@QEBA_NPEAUhb_sanitize_context_t@@PEBX@Z 00000001800229e0 f i hb-aat-layout.obj
 0001:000219e0       ?sanitize_shallow@?$OffsetTo@UAnchorMatrix@GPOS_impl@Layout@OT@@U?$IntType@G$01@4@X$00@OT@@QEBA_NPEAUhb_sanitize_context_t@@PEBX@Z 00000001800229e0 f i hb-ot-layout.obj
 0001:000219e0       ?sanitize_shallow@?$OffsetTo@U?$Ligature@USmallTypes@Layout@OT@@@GSUB_impl@Layout@OT@@U?$IntType@G$01@4@X$00@OT@@QEBA_NPEAUhb_sanitize_context_t@@PEBX@Z 00000001800229e0 f i hb-aat-layout.obj
 0001:000219e0       ?sanitize_shallow@?$OffsetTo@U?$ChainRule@USmallTypes@Layout@OT@@@OT@@U?$IntType@G$01@2@X$00@OT@@QEBA_NPEAUhb_sanitize_context_t@@PEBX@Z 00000001800229e0 f i hb-aat-layout.obj
 0001:000219e0       ?sanitize_shallow@?$OffsetTo@UAnchor@GPOS_impl@Layout@OT@@U?$IntType@G$01@4@UCursivePosFormat1@234@$00@OT@@QEBA_NPEAUhb_sanitize_context_t@@PEBUCursivePosFormat1@GPOS_impl@Layout@2@@Z 00000001800229e0 f i hb-ot-layout.obj
 0001:000219e0       ?sanitize_shallow@?$OffsetTo@U?$UnsizedArrayOf@U?$IntType@I$03@OT@@@OT@@U?$IntType@G$01@2@X$0A@@OT@@QEBA_NPEAUhb_sanitize_context_t@@PEBX@Z 00000001800229e0 f i hb-aat-layout.obj
 0001:000219e0       ?sanitize_shallow@?$OffsetTo@U?$Lookup@UHBGlyphID16@OT@@@AAT@@U?$IntType@G$01@OT@@X$0A@@OT@@QEBA_NPEAUhb_sanitize_context_t@@PEBX@Z 00000001800229e0 f i hb-aat-layout.obj
 0001:000219e0       ?sanitize_shallow@?$OffsetTo@U?$UnsizedArrayOf@UHBGlyphID16@OT@@@OT@@U?$IntType@G$01@2@X$0A@@OT@@QEBA_NPEAUhb_sanitize_context_t@@PEBX@Z 00000001800229e0 f i hb-aat-layout.obj
 0001:000219e0       ?sanitize_shallow@?$OffsetTo@UClassDef@OT@@U?$IntType@G$01@2@X$00@OT@@QEBA_NPEAUhb_sanitize_context_t@@PEBX@Z 00000001800229e0 f i hb-aat-layout.obj
 0001:000219e0       ?sanitize_shallow@?$OffsetTo@USubstLookup@GSUB_impl@Layout@OT@@U?$IntType@G$01@4@X$00@OT@@QEBA_NPEAUhb_sanitize_context_t@@PEBX@Z 00000001800229e0 f i hb-aat-layout.obj
 0001:000219e0       ?sanitize_shallow@?$OffsetTo@U?$UnsizedArrayOf@U?$OffsetTo@U?$ArrayOf@UAnchor@AAT@@U?$IntType@I$03@OT@@@OT@@U?$IntType@G$01@2@X$0A@@OT@@@OT@@U?$IntType@G$01@2@X$0A@@OT@@QEBA_NPEAUhb_sanitize_context_t@@PEBX@Z 00000001800229e0 f i hb-aat-layout.obj
 0001:00021ab0       ?sanitize_shallow@?$OffsetTo@U?$UnsizedArrayOf@U?$HBFixed@U?$IntType@H$03@OT@@$0BA@@OT@@@OT@@U?$IntType@I$03@2@X$0A@@OT@@QEBA_NPEAUhb_sanitize_context_t@@PEBX@Z 0000000180022ab0 f i hb-aat-layout.obj
 0001:00021ab0       ?sanitize_shallow@?$OffsetTo@UCoverage@Common@Layout@OT@@U?$IntType@I$03@4@X$00@OT@@QEBA_NPEAUhb_sanitize_context_t@@PEBX@Z 0000000180022ab0 f i hb-aat-layout.obj
 0001:00021ab0       ?sanitize_shallow@?$OffsetTo@UDefaultUVS@OT@@U?$IntType@I$03@2@X$00@OT@@QEBA_NPEAUhb_sanitize_context_t@@PEBX@Z 0000000180022ab0 f i hb-face.obj
 0001:00021ab0       ?sanitize_shallow@?$OffsetTo@UNonDefaultUVS@OT@@U?$IntType@I$03@2@X$00@OT@@QEBA_NPEAUhb_sanitize_context_t@@PEBX@Z 0000000180022ab0 f i hb-face.obj
 0001:00021ab0       ?sanitize_shallow@?$OffsetTo@U?$UnsizedArrayOf@UStatAxisRecord@OT@@@OT@@U?$IntType@I$03@2@X$0A@@OT@@QEBA_NPEAUhb_sanitize_context_t@@PEBX@Z 0000000180022ab0 f i hb-ot-shape.obj
 0001:00021ab0       ?sanitize_shallow@?$OffsetTo@UItemVariationStore@OT@@U?$IntType@I$03@2@X$00@OT@@QEBA_NPEAUhb_sanitize_context_t@@PEBX@Z 0000000180022ab0 f i hb-aat-layout.obj
 0001:00021ab0       ?sanitize_shallow@?$OffsetTo@UConditionSet@OT@@U?$IntType@I$03@2@X$00@OT@@QEBA_NPEAUhb_sanitize_context_t@@PEBX@Z 0000000180022ab0 f i hb-aat-layout.obj
 0001:00021ab0       ?sanitize_shallow@?$OffsetTo@UFeatureTableSubstitution@OT@@U?$IntType@I$03@2@X$00@OT@@QEBA_NPEAUhb_sanitize_context_t@@PEBX@Z 0000000180022ab0 f i hb-aat-layout.obj
 0001:00021ab0       ?sanitize_shallow@?$OffsetTo@UAxisValueOffsetArray@OT@@U?$IntType@I$03@2@X$0A@@OT@@QEBA_NPEAUhb_sanitize_context_t@@PEBX@Z 0000000180022ab0 f i hb-ot-shape.obj
 0001:00021ab0       ?sanitize_shallow@?$OffsetTo@UFeatureVariations@OT@@U?$IntType@I$03@2@X$00@OT@@QEBA_NPEAUhb_sanitize_context_t@@PEBX@Z 0000000180022ab0 f i hb-aat-layout.obj
 0001:00021ab0       ?sanitize_shallow@?$OffsetTo@UCondition@OT@@U?$IntType@I$03@2@X$00@OT@@QEBA_NPEAUhb_sanitize_context_t@@PEBX@Z 0000000180022ab0 f i hb-aat-layout.obj
 0001:00021ab0       ?sanitize_shallow@?$OffsetTo@U?$Lookup@U?$OffsetTo@U?$ArrayOf@UAnchor@AAT@@U?$IntType@I$03@OT@@@OT@@U?$IntType@G$01@2@X$0A@@OT@@@AAT@@U?$IntType@I$03@OT@@X$00@OT@@QEBA_NPEAUhb_sanitize_context_t@@PEBX@Z 0000000180022ab0 f i hb-aat-layout.obj
 0001:00021ab0       ?sanitize_shallow@?$OffsetTo@U?$UnsizedArrayOf@U?$IntType@E$00@OT@@@OT@@U?$IntType@I$03@2@X$0A@@OT@@QEBA_NPEAUhb_sanitize_context_t@@PEBX@Z 0000000180022ab0 f i hb-aat-layout.obj
 0001:00021ab0       ?sanitize_shallow@?$OffsetTo@UCmapSubtable@OT@@U?$IntType@I$03@2@X$00@OT@@QEBA_NPEAUhb_sanitize_context_t@@PEBX@Z 0000000180022ab0 f i hb-face.obj
 0001:00021ab0       ?sanitize_shallow@?$OffsetTo@UResourceMap@OT@@U?$IntType@I$03@2@X$0A@@OT@@QEBA_NPEAUhb_sanitize_context_t@@PEBX@Z 0000000180022ab0 f i hb-face.obj
 0001:00021ab0       ?sanitize_shallow@?$OffsetTo@UIndexSubtableArray@OT@@U?$IntType@I$03@2@X$0A@@OT@@QEBA_NPEAUhb_sanitize_context_t@@PEBX@Z 0000000180022ab0 f i hb-ot-color.obj
 0001:00021ab0       ?sanitize_shallow@?$OffsetTo@UFeature@OT@@U?$IntType@I$03@2@X$00@OT@@QEBA_NPEAUhb_sanitize_context_t@@PEBX@Z 0000000180022ab0 f i hb-aat-layout.obj
 0001:00021ab0       ?sanitize_shallow@?$OffsetTo@U?$Lookup@U?$IntType@I$03@OT@@@AAT@@U?$IntType@I$03@OT@@X$0A@@OT@@QEBA_NPEAUhb_sanitize_context_t@@PEBX@Z 0000000180022ab0 f i hb-aat-layout.obj
 0001:00021ab0       ?sanitize_shallow@?$OffsetTo@U?$Lookup@UHBGlyphID16@OT@@@AAT@@U?$IntType@I$03@OT@@X$0A@@OT@@QEBA_NPEAUhb_sanitize_context_t@@PEBX@Z 0000000180022ab0 f i hb-aat-layout.obj
 0001:00021ab0       ?sanitize_shallow@?$OffsetTo@UVarRegionList@OT@@U?$IntType@I$03@2@X$00@OT@@QEBA_NPEAUhb_sanitize_context_t@@PEBX@Z 0000000180022ab0 f i hb-aat-layout.obj
 0001:00021ab0       ?sanitize_shallow@?$OffsetTo@UIndexSubtable@OT@@U?$IntType@I$03@2@X$00@OT@@QEBA_NPEAUhb_sanitize_context_t@@PEBX@Z 0000000180022ab0 f i hb-ot-color.obj
 0001:00021ab0       ?sanitize_shallow@?$OffsetTo@UBaseGlyphList@OT@@U?$IntType@I$03@2@X$00@OT@@QEBA_NPEAUhb_sanitize_context_t@@PEBX@Z 0000000180022ab0 f i hb-ot-color.obj
 0001:00021ab0       ?sanitize_shallow@?$OffsetTo@U?$UnsizedArrayOf@U?$HBFixed@U?$IntType@F$01@OT@@$0O@@OT@@@OT@@U?$IntType@I$03@2@X$0A@@OT@@QEBA_NPEAUhb_sanitize_context_t@@PEBX@Z 0000000180022ab0 f i hb-common.obj
 0001:00021ab0       ?sanitize_shallow@?$OffsetTo@ULayerList@OT@@U?$IntType@I$03@2@X$00@OT@@QEBA_NPEAUhb_sanitize_context_t@@PEBX@Z 0000000180022ab0 f i hb-ot-color.obj
 0001:00021ab0       ?sanitize_shallow@?$OffsetTo@U?$Lookup@U?$IntType@G$01@OT@@@AAT@@U?$IntType@I$03@OT@@X$0A@@OT@@QEBA_NPEAUhb_sanitize_context_t@@PEBX@Z 0000000180022ab0 f i hb-aat-layout.obj
 0001:00021ab0       ?sanitize_shallow@?$OffsetTo@UClipList@OT@@U?$IntType@I$03@2@X$00@OT@@QEBA_NPEAUhb_sanitize_context_t@@PEBX@Z 0000000180022ab0 f i hb-ot-color.obj
 0001:00021ab0       ?sanitize_shallow@?$OffsetTo@UOpenTypeOffsetTable@OT@@U?$IntType@I$03@2@X$00@OT@@QEBA_NPEAUhb_sanitize_context_t@@PEBX@Z 0000000180022ab0 f i hb-face.obj
 0001:00021ab0       ?sanitize_shallow@?$OffsetTo@UVarData@OT@@U?$IntType@I$03@2@X$00@OT@@QEBA_NPEAUhb_sanitize_context_t@@PEBX@Z 0000000180022ab0 f i hb-aat-layout.obj
 0001:00021ab0       ?sanitize_shallow@?$OffsetTo@USBIXStrike@OT@@U?$IntType@I$03@2@X$00@OT@@QEBA_NPEAUhb_sanitize_context_t@@PEBX@Z 0000000180022ab0 f i hb-ot-color.obj
 0001:00021ab0       ?sanitize_shallow@?$OffsetTo@U?$UnsizedListOfOffset16To@U?$Lookup@UHBGlyphID16@OT@@@AAT@@U?$IntType@I$03@OT@@X$0A@@OT@@U?$IntType@I$03@2@X$0A@@OT@@QEBA_NPEAUhb_sanitize_context_t@@PEBX@Z 0000000180022ab0 f i hb-aat-layout.obj
 0001:00021ab0       ?sanitize_shallow@?$OffsetTo@UPaint@OT@@U?$IntType@I$03@2@X$00@OT@@QEBA_NPEAUhb_sanitize_context_t@@PEBX@Z 0000000180022ab0 f i hb-ot-color.obj
 0001:00021ab0       ?sanitize_shallow@?$OffsetTo@UDeltaSetIndexMap@OT@@U?$IntType@I$03@2@X$00@OT@@QEBA_NPEAUhb_sanitize_context_t@@PEBX@Z 0000000180022ab0 f i hb-common.obj
 0001:00021b90       ?sanitize_shallow@?$OffsetTo@UCondition@OT@@U?$IntType@I$02@2@X$00@OT@@QEBA_NPEAUhb_sanitize_context_t@@PEBX@Z 0000000180022b90 f i hb-aat-layout.obj
 0001:00021b90       ?sanitize_shallow@?$OffsetTo@UClipBox@OT@@U?$IntType@I$02@2@X$00@OT@@QEBA_NPEAUhb_sanitize_context_t@@PEBX@Z 0000000180022b90 f i hb-ot-color.obj
 0001:00021b90       ?sanitize_shallow@?$OffsetTo@U?$Variable@UAffine2x3@OT@@@OT@@U?$IntType@I$02@2@X$00@OT@@QEBA_NPEAUhb_sanitize_context_t@@PEBX@Z 0000000180022b90 f i hb-ot-color.obj
 0001:00021b90       ?sanitize_shallow@?$OffsetTo@UPaint@OT@@U?$IntType@I$02@2@X$00@OT@@QEBA_NPEAUhb_sanitize_context_t@@PEBX@Z 0000000180022b90 f i hb-ot-color.obj
 0001:00021b90       ?sanitize_shallow@?$OffsetTo@U?$ColorLine@UVariable@OT@@@OT@@U?$IntType@I$02@2@X$00@OT@@QEBA_NPEAUhb_sanitize_context_t@@PEBX@Z 0000000180022b90 f i hb-ot-color.obj
 0001:00021b90       ?sanitize_shallow@?$OffsetTo@U?$NoVariable@UAffine2x3@OT@@@OT@@U?$IntType@I$02@2@X$00@OT@@QEBA_NPEAUhb_sanitize_context_t@@PEBX@Z 0000000180022b90 f i hb-ot-color.obj
 0001:00021b90       ?sanitize_shallow@?$OffsetTo@U?$ArrayOf@U?$IntType@E$00@OT@@U?$IntType@I$03@2@@OT@@U?$IntType@I$02@2@X$0A@@OT@@QEBA_NPEAUhb_sanitize_context_t@@PEBX@Z 0000000180022b90 f i hb-face.obj
 0001:00021b90       ?sanitize_shallow@?$OffsetTo@U?$ColorLine@UNoVariable@OT@@@OT@@U?$IntType@I$02@2@X$00@OT@@QEBA_NPEAUhb_sanitize_context_t@@PEBX@Z 0000000180022b90 f i hb-ot-color.obj
 0001:00021c70       ?sanitize_shallow@?$UnsizedArrayOf@ULayerRecord@OT@@@OT@@QEBA_NPEAUhb_sanitize_context_t@@I@Z 0000000180022c70 f i hb-ot-color.obj
 0001:00021c70       ?sanitize_shallow@?$UnsizedArrayOf@U?$HBFixed@U?$IntType@H$03@OT@@$0BA@@OT@@@OT@@QEBA_NPEAUhb_sanitize_context_t@@I@Z 0000000180022c70 f i hb-aat-layout.obj
 0001:00021c70       ?sanitize_shallow@?$UnsizedArrayOf@USettingName@AAT@@@OT@@QEBA_NPEAUhb_sanitize_context_t@@I@Z 0000000180022c70 f i hb-aat-layout.obj
 0001:00021c70       ?sanitize_shallow@?$UnsizedArrayOf@U?$OffsetTo@U?$Lookup@UHBGlyphID16@OT@@@AAT@@U?$IntType@I$03@OT@@X$0A@@OT@@@OT@@QEBA_NPEAUhb_sanitize_context_t@@I@Z 0000000180022c70 f i hb-aat-layout.obj
 0001:00021c70       ?sanitize_shallow@?$UnsizedArrayOf@U?$Offset@U?$IntType@I$03@OT@@$00@OT@@@OT@@QEBA_NPEAUhb_sanitize_context_t@@I@Z 0000000180022c70 f i hb-ot-color.obj
 0001:00021c70       ?sanitize_shallow@?$UnsizedArrayOf@U?$IntType@I$03@OT@@@OT@@QEBA_NPEAUhb_sanitize_context_t@@I@Z 0000000180022c70 f i hb-aat-layout.obj
 0001:00021d60       ?sanitize_shallow@?$UnsizedArrayOf@U?$OffsetTo@U?$Lookup@UHBGlyphID16@OT@@@AAT@@U?$IntType@G$01@OT@@X$0A@@OT@@@OT@@QEBA_NPEAUhb_sanitize_context_t@@I@Z 0000000180022d60 f i hb-aat-layout.obj
 0001:00021d60       ?sanitize_shallow@?$UnsizedArrayOf@U?$Offset@U?$IntType@G$01@OT@@$00@OT@@@OT@@QEBA_NPEAUhb_sanitize_context_t@@I@Z 0000000180022d60 f i hb-ot-color.obj
 0001:00021d60       ?sanitize_shallow@?$UnsizedArrayOf@UIndex@OT@@@OT@@QEBA_NPEAUhb_sanitize_context_t@@I@Z 0000000180022d60 f i hb-ot-color.obj
 0001:00021d60       ?sanitize_shallow@?$UnsizedArrayOf@U?$OffsetTo@UAxisValue@OT@@U?$IntType@G$01@2@X$00@OT@@@OT@@QEBA_NPEAUhb_sanitize_context_t@@I@Z 0000000180022d60 f i hb-ot-shape.obj
 0001:00021d60       ?sanitize_shallow@?$UnsizedArrayOf@U?$HBFixed@U?$IntType@F$01@OT@@$0O@@OT@@@OT@@QEBA_NPEAUhb_sanitize_context_t@@I@Z 0000000180022d60 f i hb-common.obj
 0001:00021d60       ?sanitize_shallow@?$UnsizedArrayOf@U?$OffsetTo@U?$ArrayOf@UAnchor@AAT@@U?$IntType@I$03@OT@@@OT@@U?$IntType@G$01@2@X$0A@@OT@@@OT@@QEBA_NPEAUhb_sanitize_context_t@@I@Z 0000000180022d60 f i hb-aat-layout.obj
 0001:00021d60       ?sanitize_shallow@?$UnsizedArrayOf@U?$IntType@G$01@OT@@@OT@@QEBA_NPEAUhb_sanitize_context_t@@I@Z 0000000180022d60 f i hb-ot-color.obj
 0001:00021e50       ?sanitize_shallow@?$UnsizedArrayOf@UResourceRecord@OT@@@OT@@QEBA_NPEAUhb_sanitize_context_t@@I@Z 0000000180022e50 f i hb-face.obj
 0001:00021e50       ?sanitize_shallow@?$UnsizedArrayOf@UFeatureName@AAT@@@OT@@QEBA_NPEAUhb_sanitize_context_t@@I@Z 0000000180022e50 f i hb-aat-layout.obj
 0001:00021f40       ?sanitize_shallow@?$UnsizedArrayOf@UStatAxisRecord@OT@@@OT@@QEBA_NPEAUhb_sanitize_context_t@@I@Z 0000000180022f40 f i hb-ot-shape.obj
 0001:00021f40       ?sanitize_shallow@?$UnsizedArrayOf@UTrackTableEntry@AAT@@@OT@@QEBA_NPEAUhb_sanitize_context_t@@I@Z 0000000180022f40 f i hb-aat-layout.obj
 0001:00021f40       ?sanitize_shallow@?$UnsizedArrayOf@UIndexSubtableRecord@OT@@@OT@@QEBA_NPEAUhb_sanitize_context_t@@I@Z 0000000180022f40 f i hb-ot-color.obj
 0001:00022030       ?sanitize_shallow@?$UnsizedArrayOf@UBaseGlyphRecord@OT@@@OT@@QEBA_NPEAUhb_sanitize_context_t@@I@Z 0000000180023030 f i hb-ot-color.obj
 0001:00022030       ?sanitize_shallow@?$UnsizedArrayOf@UAxisValueRecord@OT@@@OT@@QEBA_NPEAUhb_sanitize_context_t@@I@Z 0000000180023030 f i hb-ot-shape.obj
 0001:00022030       ?sanitize_shallow@?$UnsizedArrayOf@UVarRegionAxis@OT@@@OT@@QEBA_NPEAUhb_sanitize_context_t@@I@Z 0000000180023030 f i hb-aat-layout.obj
 0001:00022120       ?sanitize_shallow@?$VarSizedBinSearchArrayOf@U?$LookupSegmentArray@U?$IntType@G$01@OT@@@AAT@@@OT@@AEBA_NPEAUhb_sanitize_context_t@@@Z 0000000180023120 f i hb-aat-layout.obj
 0001:00022120       ?sanitize_shallow@?$VarSizedBinSearchArrayOf@U?$LookupSegmentArray@U?$OffsetTo@U?$ArrayOf@UAnchor@AAT@@U?$IntType@I$03@OT@@@OT@@U?$IntType@G$01@2@X$0A@@OT@@@AAT@@@OT@@AEBA_NPEAUhb_sanitize_context_t@@@Z 0000000180023120 f i hb-aat-layout.obj
 0001:00022120       ?sanitize_shallow@?$VarSizedBinSearchArrayOf@U?$LookupSingle@U?$IntType@I$03@OT@@@AAT@@@OT@@AEBA_NPEAUhb_sanitize_context_t@@@Z 0000000180023120 f i hb-aat-layout.obj
 0001:00022120       ?sanitize_shallow@?$VarSizedBinSearchArrayOf@U?$LookupSegmentArray@UHBGlyphID16@OT@@@AAT@@@OT@@AEBA_NPEAUhb_sanitize_context_t@@@Z 0000000180023120 f i hb-aat-layout.obj
 0001:00022120       ?sanitize_shallow@?$VarSizedBinSearchArrayOf@U?$LookupSegmentSingle@UHBGlyphID16@OT@@@AAT@@@OT@@AEBA_NPEAUhb_sanitize_context_t@@@Z 0000000180023120 f i hb-aat-layout.obj
 0001:00022120       ?sanitize_shallow@?$VarSizedBinSearchArrayOf@U?$LookupSegmentSingle@U?$OffsetTo@U?$ArrayOf@UAnchor@AAT@@U?$IntType@I$03@OT@@@OT@@U?$IntType@G$01@2@X$0A@@OT@@@AAT@@@OT@@AEBA_NPEAUhb_sanitize_context_t@@@Z 0000000180023120 f i hb-aat-layout.obj
 0001:00022120       ?sanitize_shallow@?$VarSizedBinSearchArrayOf@U?$LookupSegmentArray@U?$IntType@I$03@OT@@@AAT@@@OT@@AEBA_NPEAUhb_sanitize_context_t@@@Z 0000000180023120 f i hb-aat-layout.obj
 0001:00022120       ?sanitize_shallow@?$VarSizedBinSearchArrayOf@U?$LookupSegmentSingle@U?$IntType@G$01@OT@@@AAT@@@OT@@AEBA_NPEAUhb_sanitize_context_t@@@Z 0000000180023120 f i hb-aat-layout.obj
 0001:00022220       ?sanitize_shallow@?$VarSizedBinSearchArrayOf@U?$LookupSegmentSingle@U?$IntType@I$03@OT@@@AAT@@@OT@@AEBA_NPEAUhb_sanitize_context_t@@@Z 0000000180023220 f i hb-aat-layout.obj
 0001:00022320       ?sanitize_shallow@?$VarSizedBinSearchArrayOf@U?$LookupSingle@UHBGlyphID16@OT@@@AAT@@@OT@@AEBA_NPEAUhb_sanitize_context_t@@@Z 0000000180023320 f i hb-aat-layout.obj
 0001:00022320       ?sanitize_shallow@?$VarSizedBinSearchArrayOf@U?$LookupSingle@U?$OffsetTo@U?$ArrayOf@UAnchor@AAT@@U?$IntType@I$03@OT@@@OT@@U?$IntType@G$01@2@X$0A@@OT@@@AAT@@@OT@@AEBA_NPEAUhb_sanitize_context_t@@@Z 0000000180023320 f i hb-aat-layout.obj
 0001:00022320       ?sanitize_shallow@?$VarSizedBinSearchArrayOf@U?$LookupSingle@U?$IntType@G$01@OT@@@AAT@@@OT@@AEBA_NPEAUhb_sanitize_context_t@@@Z 0000000180023320 f i hb-aat-layout.obj
 0001:00022420       ?setup_buffer_glyph_set@hb_aat_apply_context_t@AAT@@QEAAXXZ 0000000180023420 f i hb-aat-layout.obj
 0001:00022490       ?shrink_vector@?$hb_vector_t@U?$hb_vector_t@Urange_flags_t@hb_aat_map_t@@$00@@$0A@@@QEAAXI@Z 0000000180023490 f i hb-aat-layout.obj
 0001:00022530       ?shrink_vector@?$hb_vector_t@Ukern_subtable_accelerator_data_t@AAT@@$0A@@@QEAAXI@Z 0000000180023530 f i hb-aat-layout.obj
 0001:00022640       ?start_processing@hb_sanitize_context_t@@QEAAXXZ 0000000180023640 f i hb-aat-layout.obj
 0001:00022710       ?transition@driver_context_t@?$ContextualSubtable@UObsoleteTypes@AAT@@@AAT@@QEAAXPEAUhb_buffer_t@@PEAU?$StateTableDriver@UObsoleteTypes@AAT@@UEntryData@?$ContextualSubtable@UObsoleteTypes@AAT@@@2@W4Flags@42@@3@AEBU?$Entry@UEntryData@?$ContextualSubtable@UObsoleteTypes@AAT@@@AAT@@@3@@Z 0000000180023710 f i hb-aat-layout.obj
 0001:000229b0       ?transition@driver_context_t@?$InsertionSubtable@UObsoleteTypes@AAT@@@AAT@@QEAAXPEAUhb_buffer_t@@PEAU?$StateTableDriver@UObsoleteTypes@AAT@@UEntryData@?$InsertionSubtable@UObsoleteTypes@AAT@@@2@W4Flags@42@@3@AEBU?$Entry@UEntryData@?$InsertionSubtable@UObsoleteTypes@AAT@@@AAT@@@3@@Z 00000001800239b0 f i hb-aat-layout.obj
 0001:000229b0       ?transition@driver_context_t@?$InsertionSubtable@UExtendedTypes@AAT@@@AAT@@QEAAXPEAUhb_buffer_t@@PEAU?$StateTableDriver@UExtendedTypes@AAT@@UEntryData@?$InsertionSubtable@UExtendedTypes@AAT@@@2@W4Flags@42@@3@AEBU?$Entry@UEntryData@?$InsertionSubtable@UExtendedTypes@AAT@@@AAT@@@3@@Z 00000001800239b0 f i hb-aat-layout.obj
 0001:00022c00       ?transition@driver_context_t@?$KerxSubTableFormat1@UKerxSubTableHeader@AAT@@@AAT@@QEAAXPEAUhb_buffer_t@@PEAU?$StateTableDriver@UExtendedTypes@AAT@@UEntryData@?$Format1Entry@$00@2@W4Flags@?$KerxSubTableFormat1@UKerxSubTableHeader@AAT@@@2@@3@AEBU?$Entry@UEntryData@?$Format1Entry@$00@AAT@@@3@@Z 0000000180023c00 f i hb-aat-layout.obj
 0001:00022ee0       ?transition@driver_context_t@?$KerxSubTableFormat4@UKerxSubTableHeader@AAT@@@AAT@@QEAAXPEAUhb_buffer_t@@PEAU?$StateTableDriver@UExtendedTypes@AAT@@UEntryData@?$KerxSubTableFormat4@UKerxSubTableHeader@AAT@@@2@W4Flags@42@@3@AEBU?$Entry@UEntryData@?$KerxSubTableFormat4@UKerxSubTableHeader@AAT@@@AAT@@@3@@Z 0000000180023ee0 f i hb-aat-layout.obj
 0001:00023350       ?transition@driver_context_t@?$LigatureSubtable@UExtendedTypes@AAT@@@AAT@@QEAAXPEAUhb_buffer_t@@PEAU?$StateTableDriver@UExtendedTypes@AAT@@UEntryData@?$LigatureEntry@$00@2@W4Flags@?$LigatureSubtable@UExtendedTypes@AAT@@@2@@3@AEBU?$Entry@UEntryData@?$LigatureEntry@$00@AAT@@@3@@Z 0000000180024350 f i hb-aat-layout.obj
 0001:00023790       ?transition@driver_context_t@?$LigatureSubtable@UObsoleteTypes@AAT@@@AAT@@QEAAXPEAUhb_buffer_t@@PEAU?$StateTableDriver@UObsoleteTypes@AAT@@XW4Flags@?$LigatureSubtable@UObsoleteTypes@AAT@@@2@@3@AEBU?$Entry@X@3@@Z 0000000180024790 f i hb-aat-layout.obj
 0001:00023c20       ?transition@driver_context_t@?$RearrangementSubtable@UExtendedTypes@AAT@@@AAT@@QEAAXPEAUhb_buffer_t@@PEAU?$StateTableDriver@UExtendedTypes@AAT@@XW4Flags@?$RearrangementSubtable@UExtendedTypes@AAT@@@2@@3@AEBU?$Entry@X@3@@Z 0000000180024c20 f i hb-aat-layout.obj
 0001:00023c20       ?transition@driver_context_t@?$RearrangementSubtable@UObsoleteTypes@AAT@@@AAT@@QEAAXPEAUhb_buffer_t@@PEAU?$StateTableDriver@UObsoleteTypes@AAT@@XW4Flags@?$RearrangementSubtable@UObsoleteTypes@AAT@@@2@@3@AEBU?$Entry@X@3@@Z 0000000180024c20 f i hb-aat-layout.obj
 0001:00023f40       ?unsafe_to_break@hb_buffer_t@@QEAAXII@Z 0000000180024f40 f i hb-aat-layout.obj
 0001:00023fc0       ?unsafe_to_break_from_outbuffer@hb_buffer_t@@QEAAXII@Z 0000000180024fc0 f i hb-aat-layout.obj
 0001:000240b0       hb_aat_layout_has_positioning 00000001800250b0 f   hb-aat-layout.obj
 0001:00024100       hb_aat_layout_has_substitution 0000000180025100 f   hb-aat-layout.obj
 0001:000241b0       hb_aat_layout_has_tracking 00000001800251b0 f   hb-aat-layout.obj
 0001:00024560       ?add_feature@hb_aat_map_builder_t@@QEAAXAEBUhb_feature_t@@@Z 0000000180025560 f   hb-aat-map.obj
 0001:00024720       ?alloc@?$hb_vector_t@Ufeature_info_t@hb_aat_map_builder_t@@$00@@QEAA_NI_N@Z 0000000180025720 f i hb-aat-map.obj
 0001:000247e0       ?cmp@feature_event_t@hb_aat_map_builder_t@@SAHPEBX0@Z 00000001800257e0 f i hb-aat-map.obj
 0001:00024810       ?cmp@feature_info_t@hb_aat_map_builder_t@@SAHPEBX0@Z 0000000180025810 f i hb-aat-map.obj
 0001:00024870       ?compile@hb_aat_map_builder_t@@QEAAXAEAUhb_aat_map_t@@@Z 0000000180025870 f   hb-aat-map.obj
 0001:000253f0       ?push@?$hb_vector_t@Ufeature_event_t@hb_aat_map_builder_t@@$0A@@@QEAAPEAUfeature_event_t@hb_aat_map_builder_t@@XZ 00000001800263f0 f i hb-aat-map.obj
 0001:000253f0       ?push@?$hb_vector_t@Ufeature_range_t@hb_aat_map_builder_t@@$00@@QEAAPEAUfeature_range_t@hb_aat_map_builder_t@@XZ 00000001800263f0 f i hb-aat-map.obj
 0001:000255d0       ?fini@hb_user_data_array_t@@QEAAXXZ 00000001800265d0 f i hb-blob.obj
 0001:00025710       ?try_make_writable@hb_blob_t@@QEAA_NXZ 0000000180026710 f   hb-blob.obj
 0001:00025840       hb_blob_create             0000000180026840 f   hb-blob.obj
 0001:00025890       hb_blob_create_from_file_or_fail 0000000180026890 f   hb-blob.obj
 0001:00025b00       hb_blob_create_or_fail     0000000180026b00 f   hb-blob.obj
 0001:00025bf0       hb_blob_create_sub_blob    0000000180026bf0 f   hb-blob.obj
 0001:00025d80       hb_blob_destroy            0000000180026d80 f   hb-blob.obj
 0001:00025e10       hb_blob_get_data           0000000180026e10 f   hb-blob.obj
 0001:00025e20       hb_blob_get_data_writable  0000000180026e20 f   hb-blob.obj
 0001:00025e80       hb_blob_get_empty          0000000180026e80 f   hb-blob.obj
 0001:00025e90       hb_blob_is_immutable       0000000180026e90 f   hb-blob.obj
 0001:00025ea0       hb_draw_funcs_make_immutable 0000000180026ea0 f   hb-draw.obj
 0001:00025ea0       hb_paint_funcs_make_immutable 0000000180026ea0 f   hb-paint.obj
 0001:00025ea0       hb_blob_make_immutable     0000000180026ea0 f   hb-blob.obj
 0001:00025ea0       hb_unicode_funcs_make_immutable 0000000180026ea0 f   hb-unicode.obj
 0001:00025ea0       hb_font_funcs_make_immutable 0000000180026ea0 f   hb-font.obj
 0001:00025ea0       hb_face_make_immutable     0000000180026ea0 f   hb-face.obj
 0001:00025eb0       hb_unicode_funcs_reference 0000000180026eb0 f   hb-unicode.obj
 0001:00025eb0       hb_font_reference          0000000180026eb0 f   hb-font.obj
 0001:00025eb0       hb_face_reference          0000000180026eb0 f   hb-face.obj
 0001:00025eb0       hb_blob_reference          0000000180026eb0 f   hb-blob.obj
 0001:00025ed0       __local_stdio_printf_options 0000000180026ed0 f i hb-buffer-serialize.obj
 0001:00025ee0       hb_buffer_serialize_unicode 0000000180026ee0 f   hb-buffer-serialize.obj
 0001:00026210       snprintf                   0000000180027210 f i hb-buffer-serialize.obj
 0001:00026a20       ?verify@hb_buffer_t@@QEAA_NPEAU1@PEAUhb_font_t@@PEBUhb_feature_t@@IPEBQEBD@Z 0000000180027a20 f   hb-buffer-verify.obj
 0001:00026c40       fprintf                    0000000180027c40 f i hb-buffer-verify.obj
 0001:00026f30       ??$reverse_groups@$$A6A_NAEBUhb_glyph_info_t@@0@Z@hb_buffer_t@@QEAAXA6A_NAEBUhb_glyph_info_t@@0@Z_N@Z 0000000180027f30 f i hb-buffer.obj
 0001:00027110       ?clear_output@hb_buffer_t@@QEAAXXZ 0000000180028110 f   hb-buffer.obj
 0001:00027130       ?clear_positions@hb_buffer_t@@QEAAXXZ 0000000180028130 f   hb-buffer.obj
 0001:00027170       ?delete_glyph@hb_buffer_t@@QEAAXXZ 0000000180028170 f   hb-buffer.obj
 0001:00027240       ?delete_glyphs_inplace@hb_buffer_t@@QEAAXP6A_NPEBUhb_glyph_info_t@@@Z@Z 0000000180028240 f   hb-buffer.obj
 0001:000273a0       ?enlarge@hb_buffer_t@@QEAA_NI@Z 00000001800283a0 f   hb-buffer.obj
 0001:000274c0       ?ensure@hb_buffer_t@@QEAA_NI@Z 00000001800284c0 f i hb-buffer.obj
 0001:000275e0       ?enter@hb_buffer_t@@QEAAXXZ 00000001800285e0 f   hb-buffer.obj
 0001:00027640       ?leave@hb_buffer_t@@QEAAXXZ 0000000180028640 f   hb-buffer.obj
 0001:00027660       ?make_room_for@hb_buffer_t@@QEAA_NII@Z 0000000180028660 f   hb-buffer.obj
 0001:000276e0       ?merge_clusters_impl@hb_buffer_t@@QEAAXII@Z 00000001800286e0 f   hb-buffer.obj
 0001:000278f0       ?merge_out_clusters@hb_buffer_t@@QEAAXII@Z 00000001800288f0 f   hb-buffer.obj
 0001:00027a70       ?message_impl@hb_buffer_t@@QEAA_NPEAUhb_font_t@@PEBDPEAD@Z 0000000180028a70 f   hb-buffer.obj
 0001:00027b10       ?move_to@hb_buffer_t@@QEAA_NI@Z 0000000180028b10 f   hb-buffer.obj
 0001:00027c90       ?reset@hb_buffer_t@@QEAAXXZ 0000000180028c90 f   hb-buffer.obj
 0001:00027d30       ?set_masks@hb_buffer_t@@QEAAXIIII@Z 0000000180028d30 f   hb-buffer.obj
 0001:00027da0       ?sort@hb_buffer_t@@QEAAXIIP6AHPEBUhb_glyph_info_t@@0@Z@Z 0000000180028da0 f   hb-buffer.obj
 0001:00027f00       ?sync@hb_buffer_t@@QEAA_NXZ 0000000180028f00 f   hb-buffer.obj
 0001:00027fd0       ?sync_so_far@hb_buffer_t@@QEAAHXZ 0000000180028fd0 f   hb-buffer.obj
 0001:000280e0       hb_buffer_add_utf16        00000001800290e0 f   hb-buffer.obj
 0001:000280f0       hb_buffer_append           00000001800290f0 f   hb-buffer.obj
 0001:00028550       hb_buffer_clear_contents   0000000180029550 f   hb-buffer.obj
 0001:000285b0       hb_buffer_create           00000001800295b0 f   hb-buffer.obj
 0001:00028630       hb_buffer_create_similar   0000000180029630 f   hb-buffer.obj
 0001:000286f0       hb_buffer_destroy          00000001800296f0 f   hb-buffer.obj
 0001:00028790       hb_buffer_diff             0000000180029790 f   hb-buffer.obj
 0001:00028940       hb_buffer_get_direction    0000000180029940 f   hb-buffer.obj
 0001:00028950       hb_buffer_get_flags        0000000180029950 f   hb-buffer.obj
 0001:00028960       hb_buffer_get_glyph_infos  0000000180029960 f   hb-buffer.obj
 0001:00028970       hb_buffer_get_glyph_positions 0000000180029970 f   hb-buffer.obj
 0001:000289e0       hb_buffer_get_length       00000001800299e0 f   hb-buffer.obj
 0001:000289f0       hb_buffer_get_segment_properties 00000001800299f0 f   hb-buffer.obj
 0001:00028a00       hb_buffer_reverse          0000000180029a00 f   hb-buffer.obj
 0001:00028a10       hb_buffer_set_cluster_level 0000000180029a10 f   hb-buffer.obj
 0001:00028a20       hb_buffer_set_direction    0000000180029a20 f   hb-buffer.obj
 0001:00028a30       hb_buffer_set_flags        0000000180029a30 f   hb-buffer.obj
 0001:00028a40       hb_buffer_set_invisible_glyph 0000000180029a40 f   hb-buffer.obj
 0001:00028a50       hb_buffer_set_language     0000000180029a50 f   hb-buffer.obj
 0001:00028a60       hb_buffer_set_length       0000000180029a60 f   hb-buffer.obj
 0001:00028b30       hb_buffer_set_script       0000000180029b30 f   hb-buffer.obj
 0001:00028b40       hb_buffer_set_segment_properties 0000000180029b40 f   hb-buffer.obj
 0001:00028b60       hb_segment_properties_equal 0000000180029b60 f   hb-buffer.obj
 0001:00028ba0       ??$decompile@H@TupleValues@OT@@SA_NAEAPEBU?$IntType@E$00@1@AEAU?$hb_vector_t@H$0A@@@PEBU21@_N@Z 0000000180029ba0 f i hb-common.obj
 0001:000290d0       ??$get_points@Uglyf_accelerator_t@OT@@@Glyph@glyf_impl@OT@@QEBA_NPEAUhb_font_t@@AEBUglyf_accelerator_t@2@AEAUcontour_point_vector_t@@AEAUhb_glyf_scratch_t@@PEAU5@PEAUhead_maxp_info_t@@PEAI_N77U?$hb_array_t@$$CBH@@I6@Z 000000018002a0d0 f i hb-common.obj
 0001:0002a790       ??$get_points@Upoints_aggregator_t@glyf_accelerator_t@OT@@@glyf_accelerator_t@OT@@IEBA_NPEAUhb_font_t@@IUpoints_aggregator_t@01@U?$hb_array_t@$$CBH@@AEAUhb_glyf_scratch_t@@@Z 000000018002b790 f i hb-common.obj
 0001:0002af80       ??$sanitize_blob@U?$gvar_GVAR@U?$IntType@G$01@OT@@$0GHHGGBHC@@OT@@@hb_sanitize_context_t@@QEAAPEAUhb_blob_t@@PEAU1@@Z 000000018002bf80 f i hb-common.obj
 0001:0002b110       ??$sanitize_blob@UHVAR@OT@@@hb_sanitize_context_t@@QEAAPEAUhb_blob_t@@PEAU1@@Z 000000018002c110 f i hb-common.obj
 0001:0002b2a0       ??$sanitize_blob@UVVAR@OT@@@hb_sanitize_context_t@@QEAAPEAUhb_blob_t@@PEAU1@@Z 000000018002c2a0 f i hb-common.obj
 0001:0002b540       ??$sanitize_blob@Uhead@OT@@@hb_sanitize_context_t@@QEAAPEAUhb_blob_t@@PEAU1@@Z 000000018002c540 f i hb-common.obj
 0001:0002b780       ??$sanitize_blob@Uhhea@OT@@@hb_sanitize_context_t@@QEAAPEAUhb_blob_t@@PEAU1@@Z 000000018002c780 f i hb-common.obj
 0001:0002b780       ??$sanitize_blob@Uvhea@OT@@@hb_sanitize_context_t@@QEAAPEAUhb_blob_t@@PEAU1@@Z 000000018002c780 f i hb-common.obj
 0001:0002b9a0       ??$sanitize_blob@Umaxp@OT@@@hb_sanitize_context_t@@QEAAPEAUhb_blob_t@@PEAU1@@Z 000000018002c9a0 f i hb-common.obj
 0001:0002bc50       ??0accelerator_t@?$gvar_GVAR@U?$IntType@G$01@OT@@$0GHHGGBHC@@OT@@QEAA@PEAUhb_face_t@@@Z 000000018002cc50 f i hb-common.obj
 0001:0002bfc0       ??0accelerator_t@?$hmtxvmtx@Uhmtx@OT@@Uhhea@2@UHVAR@2@@OT@@QEAA@PEAUhb_face_t@@@Z 000000018002cfc0 f i hb-common.obj
 0001:0002c2a0       ??0accelerator_t@?$hmtxvmtx@Uvmtx@OT@@Uvhea@2@UVVAR@2@@OT@@QEAA@PEAUhb_face_t@@@Z 000000018002d2a0 f i hb-common.obj
 0001:0002c580       ??0glyf_accelerator_t@OT@@QEAA@PEAUhb_face_t@@@Z 000000018002d580 f i hb-common.obj
 0001:0002c9a0       ??1hb_glyf_scratch_t@@QEAA@XZ 000000018002d9a0 f i hb-common.obj
 0001:0002cab0       ??C?$hb_lazy_loader_t@Uglyf_accelerator_t@OT@@U?$hb_face_lazy_loader_t@Uglyf_accelerator_t@OT@@$0P@@@Uhb_face_t@@$0P@U12@@@QEBAPEBUglyf_accelerator_t@OT@@XZ 000000018002dab0 f i hb-common.obj
 0001:0002cb80       ??C?$hb_lazy_loader_t@Uhhea@OT@@U?$hb_table_lazy_loader_t@Uhhea@OT@@$03$00@@Uhb_face_t@@$03Uhb_blob_t@@@@QEBAPEBUhhea@OT@@XZ 000000018002db80 f i hb-common.obj
 0001:0002cce0       ??C?$hb_lazy_loader_t@Umaxp@OT@@U?$hb_table_lazy_loader_t@Umaxp@OT@@$01$00@@Uhb_face_t@@$01Uhb_blob_t@@@@QEBAPEBUmaxp@OT@@XZ 000000018002dce0 f i hb-common.obj
 0001:0002ce40       ??C?$hb_lazy_loader_t@Uvhea@OT@@U?$hb_table_lazy_loader_t@Uvhea@OT@@$0L@$00@@Uhb_face_t@@$0L@Uhb_blob_t@@@@QEBAPEBUvhea@OT@@XZ 000000018002de40 f i hb-common.obj
 0001:0002cfa0       ?_glyf_get_advance_with_var_unscaled@@YAIPEAUhb_font_t@@I_N@Z 000000018002dfa0 f   hb-common.obj
 0001:0002cff0       ?_glyf_get_leading_bearing_with_var_unscaled@@YA_NPEAUhb_font_t@@I_NPEAH@Z 000000018002dff0 f   hb-common.obj
 0001:0002d050       ?_hb_options_init@@YAXXZ   000000018002e050 f   hb-common.obj
 0001:0002d140       ?alloc@?$hb_vector_t@Ucontour_point_t@@$0A@@@QEAA_NI_N@Z 000000018002e140 f i hb-common.obj
 0001:0002d200       ?apply_deltas_to_points@accelerator_t@?$gvar_GVAR@U?$IntType@G$01@OT@@$0GHHGGBHC@@OT@@QEBA_NIU?$hb_array_t@$$CBH@@U?$hb_array_t@Ucontour_point_t@@@@AEAUhb_glyf_scratch_t@@_N@Z 000000018002e200 f i hb-common.obj
 0001:0002e8c0       ?calculate_scalar@TupleVariationHeader@OT@@QEBANU?$hb_array_t@$$CBH@@IU?$hb_array_t@$$CBU?$HBFixed@U?$IntType@F$01@OT@@$0O@@OT@@@@PEBU?$hb_vector_t@U?$hb_pair_t@HH@@$0A@@@@Z 000000018002f8c0 f i hb-common.obj
 0001:0002eb40       ?decompile_points@?$TupleVariationData@U?$IntType@G$01@OT@@@OT@@SA_NAEAPEBU?$IntType@E$00@2@AEAU?$hb_vector_t@I$0A@@@PEBU32@@Z 000000018002fb40 f i hb-common.obj
 0001:0002ed30       ?extend@?$hb_vector_t@Ucontour_point_t@@$0A@@@QEAAXU?$hb_array_t@Ucontour_point_t@@@@@Z 000000018002fd30 f i hb-common.obj
 0001:0002ee20       ?get@?$hb_lazy_loader_t@Uhead@OT@@U?$hb_table_lazy_loader_t@Uhead@OT@@$00$00@@Uhb_face_t@@$00Uhb_blob_t@@@@QEBAPEBUhead@OT@@XZ 000000018002fe20 f i hb-common.obj
 0001:0002ef80       ?get@?$hb_lazy_loader_t@Uhmtx_accelerator_t@OT@@U?$hb_face_lazy_loader_t@Uhmtx_accelerator_t@OT@@$04@@Uhb_face_t@@$04U12@@@QEBAPEBUhmtx_accelerator_t@OT@@XZ 000000018002ff80 f i hb-common.obj
 0001:0002f040       ?get@?$hb_lazy_loader_t@Uvmtx_accelerator_t@OT@@U?$hb_face_lazy_loader_t@Uvmtx_accelerator_t@OT@@$0M@@@Uhb_face_t@@$0M@U12@@@QEBAPEBUvmtx_accelerator_t@OT@@XZ 0000000180030040 f i hb-common.obj
 0001:0002f100       ?get_advance_with_var_unscaled@glyf_accelerator_t@OT@@QEBAIPEAUhb_font_t@@I_N@Z 0000000180030100 f i hb-common.obj
 0001:0002f3f0       ?get_advance_without_var_unscaled@accelerator_t@?$hmtxvmtx@Uhmtx@OT@@Uhhea@2@UHVAR@2@@OT@@QEBAII@Z 00000001800303f0 f i hb-common.obj
 0001:0002f3f0       ?get_advance_without_var_unscaled@accelerator_t@?$hmtxvmtx@Uvmtx@OT@@Uvhea@2@UVVAR@2@@OT@@QEBAII@Z 00000001800303f0 f i hb-common.obj
 0001:0002f450       ?get_contour_points@SimpleGlyph@glyf_impl@OT@@QEBA_NAEAUcontour_point_vector_t@@_N@Z 0000000180030450 f i hb-common.obj
 0001:0002f7f0       ?get_glyph_var_data_bytes@?$gvar_GVAR@U?$IntType@G$01@OT@@$0GHHGGBHC@@OT@@IEBA?BU?$hb_array_t@$$CBD@@PEAUhb_blob_t@@II@Z 00000001800307f0 f i hb-common.obj
 0001:0002f980       ?get_leading_bearing_with_var_unscaled@glyf_accelerator_t@OT@@QEBA_NPEAUhb_font_t@@I_NPEAH@Z 0000000180030980 f i hb-common.obj
 0001:0002fbf0       ?get_transformation@CompositeGlyphRecord@glyf_impl@OT@@QEBA_NAEAY03MAEAUcontour_point_t@@@Z 0000000180030bf0 f i hb-common.obj
 0001:0002fe30       ?glyph_for_gid@glyf_accelerator_t@OT@@QEBA?BUGlyph@glyf_impl@2@I_N@Z 0000000180030e30 f i hb-common.obj
 0001:000300f0       ?is_valid@tuple_iterator_t@?$TupleVariationData@U?$IntType@G$01@OT@@@OT@@QEBA_NXZ 00000001800310f0 f i hb-common.obj
 0001:00030300       ?load_num_glyphs@hb_face_t@@AEBAIXZ 0000000180031300 f   hb-common.obj
 0001:00030330       ?load_upem@hb_face_t@@AEBAIXZ 0000000180031330 f   hb-common.obj
 0001:000308d0       ?read_points@SimpleGlyph@glyf_impl@OT@@SA_NAEAPEBU?$IntType@E$00@3@U?$hb_array_t@Ucontour_point_t@@@@PEBU43@PEQcontour_point_t@@MW4simple_glyph_flag_t@123@4@Z 00000001800318d0 f i hb-common.obj
 0001:000309b0       ?resize@?$hb_vector_t@Ucontour_point_t@@$0A@@@QEAA_NH_N0@Z 00000001800319b0 f i hb-common.obj
 0001:00030a40       ?sanitize@?$_hea@Uvhea@OT@@@OT@@QEBA_NPEAUhb_sanitize_context_t@@@Z 0000000180031a40 f i hb-common.obj
 0001:00030a40       ?sanitize@?$_hea@Uhhea@OT@@@OT@@QEBA_NPEAUhb_sanitize_context_t@@@Z 0000000180031a40 f i hb-common.obj
 0001:00030b00       ?sanitize@DeltaSetIndexMap@OT@@QEBA_NPEAUhb_sanitize_context_t@@@Z 0000000180031b00 f i hb-common.obj
 0001:00030d00       ?sanitize@HVARVVAR@OT@@QEBA_NPEAUhb_sanitize_context_t@@@Z 0000000180031d00 f i hb-common.obj
 0001:00030f30       ?sanitize@VVAR@OT@@QEBA_NPEAUhb_sanitize_context_t@@@Z 0000000180031f30 f i hb-common.obj
 0001:00030fd0       ?sanitize@head@OT@@QEBA_NPEAUhb_sanitize_context_t@@@Z 0000000180031fd0 f i hb-common.obj
 0001:000310c0       ?sanitize@maxp@OT@@QEBA_NPEAUhb_sanitize_context_t@@@Z 00000001800320c0 f i hb-common.obj
 0001:00031220       ?sanitize_shallow@?$gvar_GVAR@U?$IntType@G$01@OT@@$0GHHGGBHC@@OT@@QEBA_NPEAUhb_sanitize_context_t@@@Z 0000000180032220 f i hb-common.obj
 0001:000313a0       ?scale_glyph_extents@hb_font_t@@QEAAXPEAUhb_glyph_extents_t@@@Z 00000001800323a0 f i hb-common.obj
 0001:000314d0       ?translate@CompositeGlyphRecord@glyf_impl@OT@@SAXAEBUcontour_point_t@@U?$hb_array_t@Ucontour_point_t@@@@@Z 00000001800324d0 f i hb-common.obj
 0001:000315b0       ?trim_padding@SimpleGlyph@glyf_impl@OT@@QEBA?BU?$hb_array_t@$$CBD@@XZ 00000001800325b0 f i hb-common.obj
 0001:00031710       hb_calloc                  0000000180032710 f   hb-common.obj
 0001:00031720       hb_feature_from_string     0000000180032720 f   hb-common.obj
 0001:00031790       hb_free                    0000000180032790 f   hb-common.obj
 0001:000317a0       hb_language_from_string    00000001800327a0 f   hb-common.obj
 0001:00031840       hb_language_matches        0000000180032840 f   hb-common.obj
 0001:000318e0       hb_language_to_string      00000001800328e0 f   hb-common.obj
 0001:000318f0       hb_malloc                  00000001800328f0 f   hb-common.obj
 0001:00031900       hb_realloc                 0000000180032900 f   hb-common.obj
 0001:00031910       hb_script_get_horizontal_direction 0000000180032910 f   hb-common.obj
 0001:00031ad0       hb_tag_from_string         0000000180032ad0 f   hb-common.obj
 0001:00031b80       hb_tag_to_string           0000000180032b80 f   hb-common.obj
 0001:00031c40       ?add_point@hb_extents_t@@QEAAXMM@Z 0000000180032c40 f i hb-draw.obj
 0001:00031cc0       ?create@hb_draw_extents_funcs_lazy_loader_t@@SAPEAUhb_draw_funcs_t@@XZ 0000000180032cc0 f i hb-draw.obj
 0001:00031f00       ?hb_draw_extents_get_funcs@@YAPEAUhb_draw_funcs_t@@XZ 0000000180032f00 f   hb-draw.obj
 0001:00031fd0       hb_draw_funcs_create       0000000180032fd0 f   hb-draw.obj
 0001:00032050       hb_draw_funcs_destroy      0000000180033050 f   hb-draw.obj
 0001:00032180       hb_draw_funcs_get_empty    0000000180033180 f   hb-draw.obj
 0001:00032190       hb_draw_funcs_set_close_path_func 0000000180033190 f   hb-draw.obj
 0001:000322b0       hb_draw_funcs_set_cubic_to_func 00000001800332b0 f   hb-draw.obj
 0001:000323d0       hb_draw_funcs_set_line_to_func 00000001800333d0 f   hb-draw.obj
 0001:000324f0       hb_draw_funcs_set_move_to_func 00000001800334f0 f   hb-draw.obj
 0001:00032600       hb_draw_funcs_set_quadratic_to_func 0000000180033600 f   hb-draw.obj
 0001:00032720       ??$set_with_hash@AEAPEAUobject_t@hb_serialize_context_t@@AEAI@?$hb_hashmap_t@PEBUobject_t@hb_serialize_context_t@@I$0A@@@QEAA_NAEAPEAUobject_t@hb_serialize_context_t@@IAEAI_N@Z 0000000180033720 f i hb-face-builder.obj
 0001:00032960       ??0hb_serialize_context_t@@QEAA@PEAXI@Z 0000000180033960 f i hb-face-builder.obj
 0001:00032bf0       ??1?$hb_pool_t@Uobject_t@hb_serialize_context_t@@$0CA@@@QEAA@XZ 0000000180033bf0 f i hb-face-builder.obj
 0001:00032c80       ?alloc@?$hb_hashmap_t@PEBUobject_t@hb_serialize_context_t@@I$0A@@@QEAA_NI@Z 0000000180033c80 f i hb-face-builder.obj
 0001:00033120       ?alloc@?$hb_pool_t@Uobject_t@hb_serialize_context_t@@$0CA@@@QEAAPEAUobject_t@hb_serialize_context_t@@XZ 0000000180034120 f i hb-face-builder.obj
 0001:00033580       ?fetch_item@?$hb_hashmap_t@PEBUobject_t@hb_serialize_context_t@@I$0A@@@QEBAPEAUitem_t@1@AEBQEBUobject_t@hb_serialize_context_t@@I@Z 0000000180034580 f i hb-face-builder.obj
 0001:000336d0       ?fini@hb_serialize_context_t@@QEAAXXZ 00000001800346d0 f i hb-face-builder.obj
 0001:00033820       ?pop_pack@hb_serialize_context_t@@QEAAI_N@Z 0000000180034820 f i hb-face-builder.obj
 0001:00033bb0       ?resolve_links@hb_serialize_context_t@@QEAAXXZ 0000000180034bb0 f i hb-face-builder.obj
 0001:00033e80       hb_face_create_or_fail     0000000180034e80 f   hb-face.obj
 0001:00034010       hb_face_create_from_file_or_fail 0000000180035010 f   hb-face.obj
 0001:000341e0       ??$bsearch@I@?$SortedArrayOf@UCmapSubtableLongGroup@OT@@U?$IntType@I$03@2@@OT@@QEBAAEBUCmapSubtableLongGroup@1@AEBIAEBU21@@Z 00000001800351e0 f i hb-face.obj
 0001:000342a0       ??$dispatch@U?$ArrayOfM1@UResourceTypeRecord@OT@@U?$IntType@G$01@2@@OT@@PEBU12@AEAPEBX@hb_sanitize_context_t@@QEAA_NAEBU?$ArrayOfM1@UResourceTypeRecord@OT@@U?$IntType@G$01@2@@OT@@$$QEAPEBU12@AEAPEBX@Z 00000001800352a0 f i hb-face.obj
 0001:00034470       ??$dispatch@U?$UnsizedArrayOf@UResourceRecord@OT@@@OT@@IAEAPEBX@hb_sanitize_context_t@@QEAA_NAEBU?$UnsizedArrayOf@UResourceRecord@OT@@@OT@@$$QEAIAEAPEBX@Z 0000000180035470 f i hb-face.obj
 0001:00034600       ??$dispatch@UResourceMap@OT@@PEBU?$UnsizedArrayOf@U?$IntType@E$00@OT@@@2@@hb_sanitize_context_t@@QEAA_NAEBUResourceMap@OT@@$$QEAPEBU?$UnsizedArrayOf@U?$IntType@E$00@OT@@@2@@Z 0000000180035600 f i hb-face.obj
 0001:00034710       ??$get_glyph_from@UCmapSubtable@OT@@@accelerator_t@cmap@OT@@KA_NPEBXIPEAI@Z 0000000180035710 f i hb-face.obj
 0001:00034720       ??$get_glyph_from@UCmapSubtableFormat12@OT@@@accelerator_t@cmap@OT@@KA_NPEBXIPEAI@Z 0000000180035720 f i hb-face.obj
 0001:00034770       ??$get_glyph_from_ascii@UCmapSubtable@OT@@@accelerator_t@cmap@OT@@KA_NPEBXIPEAI@Z 0000000180035770 f i hb-face.obj
 0001:000347a0       ??$get_glyph_from_macroman@UCmapSubtable@OT@@@accelerator_t@cmap@OT@@KA_NPEBXIPEAI@Z 00000001800357a0 f i hb-face.obj
 0001:00034b10       ??$sanitize_blob@UOS2@OT@@@hb_sanitize_context_t@@QEAAPEAUhb_blob_t@@PEAU1@@Z 0000000180035b10 f i hb-face.obj
 0001:00034ca0       ??$sanitize_blob@UOpenTypeFontFile@OT@@@hb_sanitize_context_t@@QEAAPEAUhb_blob_t@@PEAU1@@Z 0000000180035ca0 f i hb-face.obj
 0001:00034e30       ??$sanitize_blob@Ucmap@OT@@@hb_sanitize_context_t@@QEAAPEAUhb_blob_t@@PEAU1@@Z 0000000180035e30 f i hb-face.obj
 0001:00034fc0       ??$set_with_hash@AEBIAEAI@?$hb_hashmap_t@II$00@@QEAA_NAEBIIAEAI_N@Z 0000000180035fc0 f i hb-face.obj
 0001:00035120       ??0accelerator_t@cmap@OT@@QEAA@PEAUhb_face_t@@@Z 0000000180036120 f i hb-face.obj
 0001:000356e0       ??C?$hb_lazy_loader_t@Ucmap_accelerator_t@OT@@U?$hb_face_lazy_loader_t@Ucmap_accelerator_t@OT@@$02@@Uhb_face_t@@$02U12@@@QEBAPEBUcmap_accelerator_t@OT@@XZ 00000001800366e0 f i hb-face.obj
 0001:00035b80       ?alloc@?$hb_hashmap_t@II$00@@QEAA_NI@Z 0000000180036b80 f i hb-face.obj
 0001:00035f10       ?compact@hb_bit_set_t@@AEAAXAEAU?$hb_vector_t@I$0A@@@I@Z 0000000180036f10 f i hb-face.obj
 0001:00036110       ?find_subtable@cmap@OT@@IEBAPEBUCmapSubtable@2@II@Z 0000000180037110 f i hb-face.obj
 0001:000362c0       ?find_table_index@OpenTypeOffsetTable@OT@@QEBA_NIPEAI@Z 00000001800372c0 f i hb-face.obj
 0001:00036490       ?get_face@OpenTypeFontFile@OT@@QEBAAEBUOpenTypeOffsetTable@2@IPEAI@Z 0000000180037490 f i hb-face.obj
 0001:000365e0       ?get_face@ResourceForkHeader@OT@@QEBAAEBUOpenTypeOffsetTable@2@IPEAI@Z 00000001800375e0 f i hb-face.obj
 0001:00036770       ?get_face_count@OpenTypeFontFile@OT@@QEBAIXZ 0000000180037770 f i hb-face.obj
 0001:00036950       ?get_glyph@?$CmapSubtableLongSegmented@UCmapSubtableFormat12@OT@@@OT@@QEBA_NIPEAI@Z 0000000180037950 f i hb-face.obj
 0001:000369a0       ?get_glyph@CmapSubtable@OT@@QEBA_NIPEAI@Z 00000001800379a0 f i hb-face.obj
 0001:00036bf0       ?get_glyph@accelerator_t@CmapSubtableFormat4@OT@@QEBA_NIPEAI@Z 0000000180037bf0 f i hb-face.obj
 0001:00036d40       ?get_glyph_func@accelerator_t@CmapSubtableFormat4@OT@@SA_NPEBXIPEAI@Z 0000000180037d40 f i hb-face.obj
 0001:00036d50       ?group_get_glyph@CmapSubtableFormat12@OT@@SAIAEBUCmapSubtableLongGroup@2@I@Z 0000000180037d50 f i hb-face.obj
 0001:00036e00       ?sanitize@CmapSubtable@OT@@QEBA_NPEAUhb_sanitize_context_t@@@Z 0000000180037e00 f i hb-face.obj
 0001:00037100       ?sanitize@CmapSubtableFormat14@OT@@QEBA_NPEAUhb_sanitize_context_t@@@Z 0000000180038100 f i hb-face.obj
 0001:00037330       ?sanitize@CmapSubtableFormat4@OT@@QEBA_NPEAUhb_sanitize_context_t@@@Z 0000000180038330 f i hb-face.obj
 0001:00037500       ?sanitize@OS2@OT@@QEBA_NPEAUhb_sanitize_context_t@@@Z 0000000180038500 f i hb-face.obj
 0001:00037730       ?sanitize@OpenTypeFontFile@OT@@QEBA_NPEAUhb_sanitize_context_t@@@Z 0000000180038730 f i hb-face.obj
 0001:000379a0       ?sanitize@OpenTypeOffsetTable@OT@@QEBA_NPEAUhb_sanitize_context_t@@@Z 00000001800389a0 f i hb-face.obj
 0001:00037a60       ?sanitize@ResourceForkHeader@OT@@QEBA_NPEAUhb_sanitize_context_t@@@Z 0000000180038a60 f i hb-face.obj
 0001:00037c10       ?sanitize@cmap@OT@@QEBA_NPEAUhb_sanitize_context_t@@@Z 0000000180038c10 f i hb-face.obj
 0001:00037df0       ?sanitize_shallow@?$ArrayOf@U?$IntType@E$00@OT@@U?$IntType@I$03@2@@OT@@QEBA_NPEAUhb_sanitize_context_t@@@Z 0000000180038df0 f i hb-face.obj
 0001:00037f80       ?sanitize_shallow@?$ArrayOf@UCmapSubtableLongGroup@OT@@U?$IntType@I$03@2@@OT@@QEBA_NPEAUhb_sanitize_context_t@@@Z 0000000180038f80 f i hb-face.obj
 0001:00038110       ?sanitize_shallow@?$ArrayOf@UEncodingRecord@OT@@U?$IntType@G$01@2@@OT@@QEBA_NPEAUhb_sanitize_context_t@@@Z 0000000180039110 f i hb-face.obj
 0001:00038280       ?sanitize_shallow@?$ArrayOf@UHBGlyphID16@OT@@U?$IntType@I$03@2@@OT@@QEBA_NPEAUhb_sanitize_context_t@@@Z 0000000180039280 f i hb-face.obj
 0001:00038400       ?sanitize_shallow@?$ArrayOf@UTableRecord@OT@@U?$BinSearchHeader@U?$IntType@G$01@OT@@@2@@OT@@QEBA_NPEAUhb_sanitize_context_t@@@Z 0000000180039400 f i hb-face.obj
 0001:00038570       ?sanitize_shallow@?$ArrayOf@UUVSMapping@OT@@U?$IntType@I$03@2@@OT@@QEBA_NPEAUhb_sanitize_context_t@@@Z 0000000180039570 f i hb-face.obj
 0001:000386f0       ?sanitize_shallow@?$ArrayOf@UVariationSelectorRecord@OT@@U?$IntType@I$03@2@@OT@@QEBA_NPEAUhb_sanitize_context_t@@@Z 00000001800396f0 f i hb-face.obj
 0001:00038870       ?sanitize_shallow@?$ArrayOfM1@UResourceTypeRecord@OT@@U?$IntType@G$01@2@@OT@@AEBA_NPEAUhb_sanitize_context_t@@@Z 0000000180039870 f i hb-face.obj
 0001:000389e0       hb_face_create             00000001800399e0 f   hb-face.obj
 0001:00038bc0       hb_face_create_for_tables  0000000180039bc0 f   hb-face.obj
 0001:00038c40       hb_face_destroy            0000000180039c40 f   hb-face.obj
 0001:00038d40       hb_face_get_empty          0000000180039d40 f   hb-face.obj
 0001:00038d50       hb_face_get_glyph_count    0000000180039d50 f   hb-face.obj
 0001:00038d60       hb_face_get_upem           0000000180039d60 f   hb-face.obj
 0001:00038d70       hb_face_reference_table    0000000180039d70 f   hb-face.obj
 0001:00038da0       _hb_fallback_shape         0000000180039da0 f   hb-fallback-shape.obj
 0001:00039240       _get_startup_argv_mode     000000018003a240 f   MSVCRT:argv_mode.obj
 0001:00039240       _hb_fallback_shaper_face_data_create 000000018003a240 f   hb-fallback-shape.obj
 0001:00039240       _hb_fallback_shaper_font_data_create 000000018003a240 f   hb-fallback-shape.obj
 0001:00039240       _hb_ot_shaper_face_data_create 000000018003a240 f   hb-ot-shape.obj
 0001:0003a440       ??$sanitize_blob@Uavar@OT@@@hb_sanitize_context_t@@QEAAPEAUhb_blob_t@@PEAU1@@Z 000000018003b440 f i hb-font.obj
 0001:0003a5d0       ??$sanitize_blob@Ufvar@OT@@@hb_sanitize_context_t@@QEAAPEAUhb_blob_t@@PEAU1@@Z 000000018003b5d0 f i hb-font.obj
 0001:0003a900       ?alloc@?$hb_vector_t@Uhb_bounds_t@@$0A@@@QEAA_NI_N@Z 000000018003b900 f i hb-font.obj
 0001:0003a9c0       ?alloc@?$hb_vector_t@Uhb_transform_t@@$0A@@@QEAA_NI_N@Z 000000018003b9c0 f i hb-font.obj
 0001:0003aa80       ?changed@hb_font_t@@QEAAXXZ 000000018003ba80 f i hb-font.obj
 0001:0003ac00       ?clear@hb_paint_extents_context_t@@QEAAXXZ 000000018003bc00 f i hb-font.obj
 0001:0003ad90       ?draw_glyph_or_fail@hb_font_t@@QEAA_NIPEAUhb_draw_funcs_t@@PEAX_N@Z 000000018003bd90 f i hb-font.obj
 0001:0003afb0       ?get@?$hb_lazy_loader_t@Ufvar@OT@@U?$hb_table_lazy_loader_t@Ufvar@OT@@$0BC@$00@@Uhb_face_t@@$0BC@Uhb_blob_t@@@@QEBAPEBUfvar@OT@@XZ 000000018003bfb0 f i hb-font.obj
 0001:0003b120       ?get_glyph_extents@hb_font_t@@QEAAHIPEAUhb_glyph_extents_t@@_N@Z 000000018003c120 f i hb-font.obj
 0001:0003b590       ?get_h_extents_with_fallback@hb_font_t@@QEAAXPEAUhb_font_extents_t@@@Z 000000018003c590 f i hb-font.obj
 0001:0003b630       ?has_func@hb_font_t@@QEAA_NI@Z 000000018003c630 f   hb-font.obj
 0001:0003b680       ?map@SegmentMaps@OT@@QEBAHHII@Z 000000018003c680 f i hb-font.obj
 0001:0003b8c0       ?paint_glyph_or_fail@hb_font_t@@QEAA_NIPEAUhb_paint_funcs_t@@PEAXII_N@Z 000000018003c8c0 f i hb-font.obj
 0001:0003b9c0       ?sanitize@avar@OT@@QEBA_NPEAUhb_sanitize_context_t@@@Z 000000018003c9c0 f i hb-font.obj
 0001:0003bc20       ?sanitize@fvar@OT@@QEBA_NPEAUhb_sanitize_context_t@@@Z 000000018003cc20 f i hb-font.obj
 0001:0003bf80       hb_font_create             000000018003cf80 f   hb-font.obj
 0001:0003c0e0       hb_font_create_sub_font    000000018003d0e0 f   hb-font.obj
 0001:0003c230       hb_font_destroy            000000018003d230 f   hb-font.obj
 0001:0003c330       hb_font_draw_glyph         000000018003d330 f   hb-font.obj
 0001:0003c350       hb_font_funcs_create       000000018003d350 f   hb-font.obj
 0001:0003c430       hb_font_funcs_destroy      000000018003d430 f   hb-font.obj
 0001:0003c720       hb_font_funcs_get_empty    000000018003d720 f   hb-font.obj
 0001:0003c730       hb_font_funcs_set_draw_glyph_or_fail_func 000000018003d730 f   hb-font.obj
 0001:0003c860       hb_font_funcs_set_font_h_extents_func 000000018003d860 f   hb-font.obj
 0001:0003c980       hb_font_funcs_set_font_v_extents_func 000000018003d980 f   hb-font.obj
 0001:0003caa0       hb_font_funcs_set_glyph_contour_point_func 000000018003daa0 f   hb-font.obj
 0001:0003cbc0       hb_font_funcs_set_glyph_extents_func 000000018003dbc0 f   hb-font.obj
 0001:0003cce0       hb_font_funcs_set_glyph_from_name_func 000000018003dce0 f   hb-font.obj
 0001:0003ce10       hb_font_funcs_set_glyph_h_advance_func 000000018003de10 f   hb-font.obj
 0001:0003cf30       hb_font_funcs_set_glyph_h_advances_func 000000018003df30 f   hb-font.obj
 0001:0003d050       hb_font_funcs_set_glyph_h_kerning_func 000000018003e050 f   hb-font.obj
 0001:0003d170       hb_font_funcs_set_glyph_h_origin_func 000000018003e170 f   hb-font.obj
 0001:0003d290       hb_font_funcs_set_glyph_name_func 000000018003e290 f   hb-font.obj
 0001:0003d3b0       hb_font_funcs_set_glyph_v_advance_func 000000018003e3b0 f   hb-font.obj
 0001:0003d4d0       hb_font_funcs_set_glyph_v_advances_func 000000018003e4d0 f   hb-font.obj
 0001:0003d5f0       hb_font_funcs_set_glyph_v_kerning_func 000000018003e5f0 f   hb-font.obj
 0001:0003d710       hb_font_funcs_set_glyph_v_origin_func 000000018003e710 f   hb-font.obj
 0001:0003d830       hb_font_funcs_set_nominal_glyph_func 000000018003e830 f   hb-font.obj
 0001:0003d950       hb_font_funcs_set_nominal_glyphs_func 000000018003e950 f   hb-font.obj
 0001:0003da70       hb_font_funcs_set_paint_glyph_or_fail_func 000000018003ea70 f   hb-font.obj
 0001:0003dba0       hb_font_funcs_set_variation_glyph_func 000000018003eba0 f   hb-font.obj
 0001:0003dcc0       hb_font_get_glyph          000000018003ecc0 f   hb-font.obj
 0001:0003dd40       hb_font_get_glyph_extents  000000018003ed40 f   hb-font.obj
 0001:0003dd50       hb_font_get_glyph_h_advance 000000018003ed50 f   hb-font.obj
 0001:0003ddb0       hb_font_get_nominal_glyph  000000018003edb0 f   hb-font.obj
 0001:0003ddf0       hb_font_set_funcs          000000018003edf0 f   hb-font.obj
 0001:0003dec0       hb_font_set_scale          000000018003eec0 f   hb-font.obj
 0001:0003dee0       hb_font_set_synthetic_bold 000000018003eee0 f   hb-font.obj
 0001:0003df30       hb_font_set_synthetic_slant 000000018003ef30 f   hb-font.obj
 0001:0003df50       hb_font_set_var_coords_normalized 000000018003ef50 f   hb-font.obj
 0001:0003e420       hb_font_set_variations     000000018003f420 f   hb-font.obj
 0001:0003e880       HBCreateFace               000000018003f880 f   hb-jdk-font-p.obj
 0001:0003e8a0       HBCreateFontFuncs          000000018003f8a0 f   hb-jdk-font-p.obj
 0001:0003e9e0       HBDisposeFace              000000018003f9e0 f   hb-jdk-font-p.obj
 0001:0003e9f0       jdk_font_create_hbp        000000018003f9f0 f   hb-jdk-font-p.obj
 0001:0003ea60       ?CallIntMethod@JNIEnv_@@QEAAHPEAV_jobject@@PEAU_jmethodID@@ZZ 000000018003fa60 f i hb-jdk-font.obj
 0001:0003ea90       ?CallObjectMethod@JNIEnv_@@QEAAPEAV_jobject@@PEAV2@PEAU_jmethodID@@ZZ 000000018003fa90 f i hb-jdk-font.obj
 0001:0003eef0       Java_sun_font_SunLayoutEngine_createFace 000000018003fef0 f   hb-jdk-font.obj
 0001:0003ef90       Java_sun_font_SunLayoutEngine_disposeFace 000000018003ff90 f   hb-jdk-font.obj
 0001:0003efa0       hb_jdk_font_create         000000018003ffa0 f   hb-jdk-font.obj
 0001:0003f130       ?fetch_item@?$hb_hashmap_t@II$00@@QEBAPEAUitem_t@1@AEBII@Z 0000000180040130 f i hb-map.obj
 0001:0003f1c0       ?hb_parse_double@@YA_NPEAPEBDPEBDPEAN_N@Z 00000001800401c0 f   hb-number.obj
 0001:0003f230       ?hb_parse_int@@YA_NPEAPEBDPEBDPEAH_N@Z 0000000180040230 f   hb-number.obj
 0001:0003f600       ??0?$cff_stack_t@Ucall_context_t@CFF@@$09@CFF@@QEAA@XZ 0000000180040600 f i hb-ot-cff1-table.obj
 0001:0003f6c0       ??0?$cs_interp_env_t@Unumber_t@CFF@@U?$Subrs@U?$IntType@G$01@OT@@@2@@CFF@@QEAA@AEBU?$hb_array_t@$$CBE@@PEBU?$Subrs@U?$IntType@G$01@OT@@@1@1@Z 00000001800406c0 f i hb-ot-cff1-table.obj
 0001:0003f880       ??A?$CFFIndex@U?$IntType@G$01@OT@@@OT@@QEBA?AU?$hb_array_t@$$CBE@@I@Z 0000000180040880 f i hb-ot-cff1-table.obj
 0001:0003fcb0       ?call_subr@?$cs_interp_env_t@Unumber_t@CFF@@U?$Subrs@U?$IntType@G$01@OT@@@2@@CFF@@QEAAXAEBU?$biased_subrs_t@U?$Subrs@U?$IntType@G$01@OT@@@CFF@@@2@W4cs_type_t@2@@Z 0000000180040cb0 f i hb-ot-cff1-table.obj
 0001:0003fe40       ?check_width@?$cff1_cs_opset_t@Ucff1_cs_opset_path_t@@Ucff1_path_param_t@@Ucff1_path_procs_path_t@@@CFF@@SAXIAEAUcff1_cs_interp_env_t@2@AEAUcff1_path_param_t@@@Z 0000000180040e40 f i hb-ot-cff1-table.obj
 0001:0003fe40       ?check_width@?$cff1_cs_opset_t@Ucff1_cs_opset_extents_t@@Ucff1_extents_param_t@@Ucff1_path_procs_extents_t@@@CFF@@SAXIAEAUcff1_cs_interp_env_t@2@AEAUcff1_extents_param_t@@@Z 0000000180040e40 f i hb-ot-cff1-table.obj
 0001:0003ff10       ?curve@cff1_path_procs_extents_t@@SAXAEAUcff1_cs_interp_env_t@CFF@@AEAUcff1_extents_param_t@@AEBUpoint_t@3@22@Z 0000000180040f10 f i hb-ot-cff1-table.obj
 0001:000400d0       ?curve@cff1_path_procs_path_t@@SAXAEAUcff1_cs_interp_env_t@CFF@@AEAUcff1_path_param_t@@AEBUpoint_t@3@22@Z 00000001800410d0 f i hb-ot-cff1-table.obj
 0001:000402b0       ?end_path@cff1_path_param_t@@QEAAXXZ 00000001800412b0 f i hb-ot-cff1-table.obj
 0001:00040380       ?flex1@?$path_procs_t@Ucff1_path_procs_extents_t@@Ucff1_cs_interp_env_t@CFF@@Ucff1_extents_param_t@@@CFF@@SAXAEAUcff1_cs_interp_env_t@2@AEAUcff1_extents_param_t@@@Z 0000000180041380 f i hb-ot-cff1-table.obj
 0001:000406d0       ?flex1@?$path_procs_t@Ucff1_path_procs_path_t@@Ucff1_cs_interp_env_t@CFF@@Ucff1_path_param_t@@@CFF@@SAXAEAUcff1_cs_interp_env_t@2@AEAUcff1_path_param_t@@@Z 00000001800416d0 f i hb-ot-cff1-table.obj
 0001:00040a20       ?flex@?$path_procs_t@Ucff1_path_procs_extents_t@@Ucff1_cs_interp_env_t@CFF@@Ucff1_extents_param_t@@@CFF@@SAXAEAUcff1_cs_interp_env_t@2@AEAUcff1_extents_param_t@@@Z 0000000180041a20 f i hb-ot-cff1-table.obj
 0001:00040cd0       ?flex@?$path_procs_t@Ucff1_path_procs_path_t@@Ucff1_cs_interp_env_t@CFF@@Ucff1_path_param_t@@@CFF@@SAXAEAUcff1_cs_interp_env_t@2@AEAUcff1_path_param_t@@@Z 0000000180041cd0 f i hb-ot-cff1-table.obj
 0001:00040f80       ?get_extents@accelerator_t@cff1@OT@@QEBA_NPEAUhb_font_t@@IPEAUhb_glyph_extents_t@@@Z 0000000180041f80 f   hb-ot-cff1-table.obj
 0001:000411c0       ?get_fd@FDSelect@CFF@@QEBAII@Z 00000001800421c0 f i hb-ot-cff1-table.obj
 0001:000412b0       ?get_glyph@Charset@CFF@@QEBAIII@Z 00000001800422b0 f i hb-ot-cff1-table.obj
 0001:00041450       ?get_path@accelerator_t@cff1@OT@@QEBA_NPEAUhb_font_t@@IAEAUhb_draw_session_t@@@Z 0000000180042450 f   hb-ot-cff1-table.obj
 0001:00041470       ?hflex1@?$path_procs_t@Ucff1_path_procs_extents_t@@Ucff1_cs_interp_env_t@CFF@@Ucff1_extents_param_t@@@CFF@@SAXAEAUcff1_cs_interp_env_t@2@AEAUcff1_extents_param_t@@@Z 0000000180042470 f i hb-ot-cff1-table.obj
 0001:000416c0       ?hflex1@?$path_procs_t@Ucff1_path_procs_path_t@@Ucff1_cs_interp_env_t@CFF@@Ucff1_path_param_t@@@CFF@@SAXAEAUcff1_cs_interp_env_t@2@AEAUcff1_path_param_t@@@Z 00000001800426c0 f i hb-ot-cff1-table.obj
 0001:00041910       ?hflex@?$path_procs_t@Ucff1_path_procs_extents_t@@Ucff1_cs_interp_env_t@CFF@@Ucff1_extents_param_t@@@CFF@@SAXAEAUcff1_cs_interp_env_t@2@AEAUcff1_extents_param_t@@@Z 0000000180042910 f i hb-ot-cff1-table.obj
 0001:00041b20       ?hflex@?$path_procs_t@Ucff1_path_procs_path_t@@Ucff1_cs_interp_env_t@CFF@@Ucff1_path_param_t@@@CFF@@SAXAEAUcff1_cs_interp_env_t@2@AEAUcff1_path_param_t@@@Z 0000000180042b20 f i hb-ot-cff1-table.obj
 0001:00041d30       ?hhcurveto@?$path_procs_t@Ucff1_path_procs_extents_t@@Ucff1_cs_interp_env_t@CFF@@Ucff1_extents_param_t@@@CFF@@SAXAEAUcff1_cs_interp_env_t@2@AEAUcff1_extents_param_t@@@Z 0000000180042d30 f i hb-ot-cff1-table.obj
 0001:00042040       ?hhcurveto@?$path_procs_t@Ucff1_path_procs_path_t@@Ucff1_cs_interp_env_t@CFF@@Ucff1_path_param_t@@@CFF@@SAXAEAUcff1_cs_interp_env_t@2@AEAUcff1_path_param_t@@@Z 0000000180043040 f i hb-ot-cff1-table.obj
 0001:00042370       ?hlineto@?$path_procs_t@Ucff1_path_procs_extents_t@@Ucff1_cs_interp_env_t@CFF@@Ucff1_extents_param_t@@@CFF@@SAXAEAUcff1_cs_interp_env_t@2@AEAUcff1_extents_param_t@@@Z 0000000180043370 f i hb-ot-cff1-table.obj
 0001:000426f0       ?hlineto@?$path_procs_t@Ucff1_path_procs_path_t@@Ucff1_cs_interp_env_t@CFF@@Ucff1_path_param_t@@@CFF@@SAXAEAUcff1_cs_interp_env_t@2@AEAUcff1_path_param_t@@@Z 00000001800436f0 f i hb-ot-cff1-table.obj
 0001:00042a30       ?hvcurveto@?$path_procs_t@Ucff1_path_procs_extents_t@@Ucff1_cs_interp_env_t@CFF@@Ucff1_extents_param_t@@@CFF@@SAXAEAUcff1_cs_interp_env_t@2@AEAUcff1_extents_param_t@@@Z 0000000180043a30 f i hb-ot-cff1-table.obj
 0001:00043790       ?hvcurveto@?$path_procs_t@Ucff1_path_procs_path_t@@Ucff1_cs_interp_env_t@CFF@@Ucff1_path_param_t@@@CFF@@SAXAEAUcff1_cs_interp_env_t@2@AEAUcff1_path_param_t@@@Z 0000000180044790 f i hb-ot-cff1-table.obj
 0001:00044230       ?interpret@?$cs_interpreter_t@Ucff1_cs_interp_env_t@CFF@@Ucff1_cs_opset_extents_t@@Ucff1_extents_param_t@@@CFF@@QEAA_NAEAUcff1_extents_param_t@@@Z 0000000180045230 f i hb-ot-cff1-table.obj
 0001:000443a0       ?interpret@?$cs_interpreter_t@Ucff1_cs_interp_env_t@CFF@@Ucff1_cs_opset_path_t@@Ucff1_path_param_t@@@CFF@@QEAA_NAEAUcff1_path_param_t@@@Z 00000001800453a0 f i hb-ot-cff1-table.obj
 0001:00044510       ?line@cff1_path_procs_path_t@@SAXAEAUcff1_cs_interp_env_t@CFF@@AEAUcff1_path_param_t@@AEBUpoint_t@3@@Z 0000000180045510 f i hb-ot-cff1-table.obj
 0001:00044630       ?lookup_expert_charset_for_glyph@cff1@OT@@KAII@Z 0000000180045630 f   hb-ot-cff1-table.obj
 0001:00044670       ?lookup_expert_charset_for_sid@cff1@OT@@KAII@Z 0000000180045670 f   hb-ot-cff1-table.obj
 0001:00044690       ?lookup_expert_subset_charset_for_glyph@cff1@OT@@KAII@Z 0000000180045690 f   hb-ot-cff1-table.obj
 0001:000446d0       ?lookup_expert_subset_charset_for_sid@cff1@OT@@KAII@Z 00000001800456d0 f   hb-ot-cff1-table.obj
 0001:000446f0       ?merge@bounds_t@@QEAAXAEBU1@@Z 00000001800456f0 f i hb-ot-cff1-table.obj
 0001:00044790       ?moveto@cff1_path_procs_path_t@@SAXAEAUcff1_cs_interp_env_t@CFF@@AEAUcff1_path_param_t@@AEBUpoint_t@3@@Z 0000000180045790 f i hb-ot-cff1-table.obj
 0001:000448e0       ?offset_at@?$CFFIndex@U?$IntType@G$01@OT@@@OT@@AEBAII@Z 00000001800458e0 f i hb-ot-cff1-table.obj
 0001:00044970       ?process_op@?$cs_opset_t@Unumber_t@CFF@@Ucff1_cs_opset_extents_t@@Ucff1_cs_interp_env_t@2@Ucff1_extents_param_t@@Ucff1_path_procs_extents_t@@@CFF@@SAXIAEAUcff1_cs_interp_env_t@2@AEAUcff1_extents_param_t@@@Z 0000000180045970 f i hb-ot-cff1-table.obj
 0001:00044f40       ?process_op@?$cs_opset_t@Unumber_t@CFF@@Ucff1_cs_opset_path_t@@Ucff1_cs_interp_env_t@2@Ucff1_path_param_t@@Ucff1_path_procs_path_t@@@CFF@@SAXIAEAUcff1_cs_interp_env_t@2@AEAUcff1_path_param_t@@@Z 0000000180045f40 f i hb-ot-cff1-table.obj
 0001:00045520       ?process_op@?$opset_t@Unumber_t@CFF@@@CFF@@SAXIAEAU?$interp_env_t@Unumber_t@CFF@@@2@@Z 0000000180046520 f i hb-ot-cff1-table.obj
 0001:00045810       ?process_post_move@?$cs_opset_t@Unumber_t@CFF@@Ucff1_cs_opset_path_t@@Ucff1_cs_interp_env_t@2@Ucff1_path_param_t@@Ucff1_path_procs_path_t@@@CFF@@SAXIAEAUcff1_cs_interp_env_t@2@AEAUcff1_path_param_t@@@Z 0000000180046810 f i hb-ot-cff1-table.obj
 0001:00045810       ?process_post_move@?$cs_opset_t@Unumber_t@CFF@@Ucff1_cs_opset_extents_t@@Ucff1_cs_interp_env_t@2@Ucff1_extents_param_t@@Ucff1_path_procs_extents_t@@@CFF@@SAXIAEAUcff1_cs_interp_env_t@2@AEAUcff1_extents_param_t@@@Z 0000000180046810 f i hb-ot-cff1-table.obj
 0001:000458a0       ?process_seac@cff1_cs_opset_extents_t@@SAXAEAUcff1_cs_interp_env_t@CFF@@AEAUcff1_extents_param_t@@@Z 00000001800468a0 f i hb-ot-cff1-table.obj
 0001:00045b40       ?process_seac@cff1_cs_opset_path_t@@SAXAEAUcff1_cs_interp_env_t@CFF@@AEAUcff1_path_param_t@@@Z 0000000180046b40 f i hb-ot-cff1-table.obj
 0001:00045d60       ?push_fixed_from_substr@?$arg_stack_t@Unumber_t@CFF@@@CFF@@QEAA_NAEAUbyte_str_ref_t@2@@Z 0000000180046d60 f i hb-ot-cff1-table.obj
 0001:00045e00       ?push_int@?$arg_stack_t@Unumber_t@CFF@@@CFF@@QEAAXH@Z 0000000180046e00 f i hb-ot-cff1-table.obj
 0001:00045e30       ?rcurveline@?$path_procs_t@Ucff1_path_procs_extents_t@@Ucff1_cs_interp_env_t@CFF@@Ucff1_extents_param_t@@@CFF@@SAXAEAUcff1_cs_interp_env_t@2@AEAUcff1_extents_param_t@@@Z 0000000180046e30 f i hb-ot-cff1-table.obj
 0001:000462d0       ?rcurveline@?$path_procs_t@Ucff1_path_procs_path_t@@Ucff1_cs_interp_env_t@CFF@@Ucff1_path_param_t@@@CFF@@SAXAEAUcff1_cs_interp_env_t@2@AEAUcff1_path_param_t@@@Z 00000001800472d0 f i hb-ot-cff1-table.obj
 0001:000466e0       ?return_from_subr@?$cs_interp_env_t@Unumber_t@CFF@@U?$Subrs@U?$IntType@I$03@OT@@@2@@CFF@@QEAAXXZ 00000001800476e0 f i hb-ot-cff2-table.obj
 0001:000466e0       ?return_from_subr@?$cs_interp_env_t@Unumber_t@CFF@@U?$Subrs@U?$IntType@G$01@OT@@@2@@CFF@@QEAAXXZ 00000001800476e0 f i hb-ot-cff1-table.obj
 0001:00046770       ?rlinecurve@?$path_procs_t@Ucff1_path_procs_extents_t@@Ucff1_cs_interp_env_t@CFF@@Ucff1_extents_param_t@@@CFF@@SAXAEAUcff1_cs_interp_env_t@2@AEAUcff1_extents_param_t@@@Z 0000000180047770 f i hb-ot-cff1-table.obj
 0001:00046c20       ?rlinecurve@?$path_procs_t@Ucff1_path_procs_path_t@@Ucff1_cs_interp_env_t@CFF@@Ucff1_path_param_t@@@CFF@@SAXAEAUcff1_cs_interp_env_t@2@AEAUcff1_path_param_t@@@Z 0000000180047c20 f i hb-ot-cff1-table.obj
 0001:00046fa0       ?rlineto@?$path_procs_t@Ucff1_path_procs_extents_t@@Ucff1_cs_interp_env_t@CFF@@Ucff1_extents_param_t@@@CFF@@SAXAEAUcff1_cs_interp_env_t@2@AEAUcff1_extents_param_t@@@Z 0000000180047fa0 f i hb-ot-cff1-table.obj
 0001:00047130       ?rlineto@?$path_procs_t@Ucff1_path_procs_path_t@@Ucff1_cs_interp_env_t@CFF@@Ucff1_path_param_t@@@CFF@@SAXAEAUcff1_cs_interp_env_t@2@AEAUcff1_path_param_t@@@Z 0000000180048130 f i hb-ot-cff1-table.obj
 0001:00047310       ?rrcurveto@?$path_procs_t@Ucff1_path_procs_extents_t@@Ucff1_cs_interp_env_t@CFF@@Ucff1_extents_param_t@@@CFF@@SAXAEAUcff1_cs_interp_env_t@2@AEAUcff1_extents_param_t@@@Z 0000000180048310 f i hb-ot-cff1-table.obj
 0001:00047640       ?rrcurveto@?$path_procs_t@Ucff1_path_procs_path_t@@Ucff1_cs_interp_env_t@CFF@@Ucff1_path_param_t@@@CFF@@SAXAEAUcff1_cs_interp_env_t@2@AEAUcff1_path_param_t@@@Z 0000000180048640 f i hb-ot-cff1-table.obj
 0001:00047980       ?vhcurveto@?$path_procs_t@Ucff1_path_procs_extents_t@@Ucff1_cs_interp_env_t@CFF@@Ucff1_extents_param_t@@@CFF@@SAXAEAUcff1_cs_interp_env_t@2@AEAUcff1_extents_param_t@@@Z 0000000180048980 f i hb-ot-cff1-table.obj
 0001:000486d0       ?vhcurveto@?$path_procs_t@Ucff1_path_procs_path_t@@Ucff1_cs_interp_env_t@CFF@@Ucff1_path_param_t@@@CFF@@SAXAEAUcff1_cs_interp_env_t@2@AEAUcff1_path_param_t@@@Z 00000001800496d0 f i hb-ot-cff1-table.obj
 0001:00049160       ?vlineto@?$path_procs_t@Ucff1_path_procs_extents_t@@Ucff1_cs_interp_env_t@CFF@@Ucff1_extents_param_t@@@CFF@@SAXAEAUcff1_cs_interp_env_t@2@AEAUcff1_extents_param_t@@@Z 000000018004a160 f i hb-ot-cff1-table.obj
 0001:000494e0       ?vlineto@?$path_procs_t@Ucff1_path_procs_path_t@@Ucff1_cs_interp_env_t@CFF@@Ucff1_path_param_t@@@CFF@@SAXAEAUcff1_cs_interp_env_t@2@AEAUcff1_path_param_t@@@Z 000000018004a4e0 f i hb-ot-cff1-table.obj
 0001:00049820       ?vvcurveto@?$path_procs_t@Ucff1_path_procs_extents_t@@Ucff1_cs_interp_env_t@CFF@@Ucff1_extents_param_t@@@CFF@@SAXAEAUcff1_cs_interp_env_t@2@AEAUcff1_extents_param_t@@@Z 000000018004a820 f i hb-ot-cff1-table.obj
 0001:00049b30       ?vvcurveto@?$path_procs_t@Ucff1_path_procs_path_t@@Ucff1_cs_interp_env_t@CFF@@Ucff1_path_param_t@@@CFF@@SAXAEAUcff1_cs_interp_env_t@2@AEAUcff1_path_param_t@@@Z 000000018004ab30 f i hb-ot-cff1-table.obj
 0001:00049e60       ??$?0$$CBUaccelerator_t@cff2@OT@@@?$cff2_cs_interp_env_t@Unumber_t@CFF@@@CFF@@QEAA@AEBU?$hb_array_t@$$CBE@@AEBUaccelerator_t@cff2@OT@@IPEBHI@Z 000000018004ae60 f i hb-ot-cff2-table.obj
 0001:0004a110       ??A?$CFFIndex@U?$IntType@I$03@OT@@@OT@@QEBA?AU?$hb_array_t@$$CBE@@I@Z 000000018004b110 f i hb-ot-cff2-table.obj
 0001:0004a260       ?blend_deltas@?$cff2_cs_interp_env_t@Unumber_t@CFF@@@CFF@@QEBANU?$hb_array_t@$$CBUnumber_t@CFF@@@@@Z 000000018004b260 f i hb-ot-cff2-table.obj
 0001:0004a3b0       ?call_subr@?$cs_interp_env_t@Unumber_t@CFF@@U?$Subrs@U?$IntType@I$03@OT@@@2@@CFF@@QEAAXAEBU?$biased_subrs_t@U?$Subrs@U?$IntType@I$03@OT@@@CFF@@@2@W4cs_type_t@2@@Z 000000018004b3b0 f i hb-ot-cff2-table.obj
 0001:0004a560       ?curve@cff2_path_procs_extents_t@@SAXAEAU?$cff2_cs_interp_env_t@Unumber_t@CFF@@@CFF@@AEAUcff2_extents_param_t@@AEBUpoint_t@3@22@Z 000000018004b560 f i hb-ot-cff2-table.obj
 0001:0004a710       ?curve@cff2_path_procs_path_t@@SAXAEAU?$cff2_cs_interp_env_t@Unumber_t@CFF@@@CFF@@AEAUcff2_path_param_t@@AEBUpoint_t@3@22@Z 000000018004b710 f i hb-ot-cff2-table.obj
 0001:0004a8b0       ?flex1@?$path_procs_t@Ucff2_path_procs_extents_t@@U?$cff2_cs_interp_env_t@Unumber_t@CFF@@@CFF@@Ucff2_extents_param_t@@@CFF@@SAXAEAU?$cff2_cs_interp_env_t@Unumber_t@CFF@@@2@AEAUcff2_extents_param_t@@@Z 000000018004b8b0 f i hb-ot-cff2-table.obj
 0001:0004ac10       ?flex1@?$path_procs_t@Ucff2_path_procs_path_t@@U?$cff2_cs_interp_env_t@Unumber_t@CFF@@@CFF@@Ucff2_path_param_t@@@CFF@@SAXAEAU?$cff2_cs_interp_env_t@Unumber_t@CFF@@@2@AEAUcff2_path_param_t@@@Z 000000018004bc10 f i hb-ot-cff2-table.obj
 0001:0004af70       ?flex@?$path_procs_t@Ucff2_path_procs_extents_t@@U?$cff2_cs_interp_env_t@Unumber_t@CFF@@@CFF@@Ucff2_extents_param_t@@@CFF@@SAXAEAU?$cff2_cs_interp_env_t@Unumber_t@CFF@@@2@AEAUcff2_extents_param_t@@@Z 000000018004bf70 f i hb-ot-cff2-table.obj
 0001:0004b220       ?flex@?$path_procs_t@Ucff2_path_procs_path_t@@U?$cff2_cs_interp_env_t@Unumber_t@CFF@@@CFF@@Ucff2_path_param_t@@@CFF@@SAXAEAU?$cff2_cs_interp_env_t@Unumber_t@CFF@@@2@AEAUcff2_path_param_t@@@Z 000000018004c220 f i hb-ot-cff2-table.obj
 0001:0004b4d0       ?get_extents@accelerator_t@cff2@OT@@QEBA_NPEAUhb_font_t@@IPEAUhb_glyph_extents_t@@@Z 000000018004c4d0 f   hb-ot-cff2-table.obj
 0001:0004b520       ?get_extents_at@accelerator_t@cff2@OT@@QEBA_NPEAUhb_font_t@@IPEAUhb_glyph_extents_t@@U?$hb_array_t@$$CBH@@@Z 000000018004c520 f   hb-ot-cff2-table.obj
 0001:0004bab0       ?get_fd@CFF2FDSelect@CFF@@QEBAII@Z 000000018004cab0 f i hb-ot-cff2-table.obj
 0001:0004bd00       ?get_path@accelerator_t@cff2@OT@@QEBA_NPEAUhb_font_t@@IAEAUhb_draw_session_t@@@Z 000000018004cd00 f   hb-ot-cff2-table.obj
 0001:0004bd50       ?get_path_at@accelerator_t@cff2@OT@@QEBA_NPEAUhb_font_t@@IAEAUhb_draw_session_t@@U?$hb_array_t@$$CBH@@@Z 000000018004cd50 f   hb-ot-cff2-table.obj
 0001:0004c0d0       ?get_region_scalars@VarData@OT@@QEBAXPEBHIAEBUVarRegionList@2@PEAMI@Z 000000018004d0d0 f i hb-ot-cff2-table.obj
 0001:0004c350       ?hflex1@?$path_procs_t@Ucff2_path_procs_extents_t@@U?$cff2_cs_interp_env_t@Unumber_t@CFF@@@CFF@@Ucff2_extents_param_t@@@CFF@@SAXAEAU?$cff2_cs_interp_env_t@Unumber_t@CFF@@@2@AEAUcff2_extents_param_t@@@Z 000000018004d350 f i hb-ot-cff2-table.obj
 0001:0004c5a0       ?hflex1@?$path_procs_t@Ucff2_path_procs_path_t@@U?$cff2_cs_interp_env_t@Unumber_t@CFF@@@CFF@@Ucff2_path_param_t@@@CFF@@SAXAEAU?$cff2_cs_interp_env_t@Unumber_t@CFF@@@2@AEAUcff2_path_param_t@@@Z 000000018004d5a0 f i hb-ot-cff2-table.obj
 0001:0004c7f0       ?hflex@?$path_procs_t@Ucff2_path_procs_extents_t@@U?$cff2_cs_interp_env_t@Unumber_t@CFF@@@CFF@@Ucff2_extents_param_t@@@CFF@@SAXAEAU?$cff2_cs_interp_env_t@Unumber_t@CFF@@@2@AEAUcff2_extents_param_t@@@Z 000000018004d7f0 f i hb-ot-cff2-table.obj
 0001:0004ca00       ?hflex@?$path_procs_t@Ucff2_path_procs_path_t@@U?$cff2_cs_interp_env_t@Unumber_t@CFF@@@CFF@@Ucff2_path_param_t@@@CFF@@SAXAEAU?$cff2_cs_interp_env_t@Unumber_t@CFF@@@2@AEAUcff2_path_param_t@@@Z 000000018004da00 f i hb-ot-cff2-table.obj
 0001:0004cc10       ?hhcurveto@?$path_procs_t@Ucff2_path_procs_extents_t@@U?$cff2_cs_interp_env_t@Unumber_t@CFF@@@CFF@@Ucff2_extents_param_t@@@CFF@@SAXAEAU?$cff2_cs_interp_env_t@Unumber_t@CFF@@@2@AEAUcff2_extents_param_t@@@Z 000000018004dc10 f i hb-ot-cff2-table.obj
 0001:0004cf30       ?hhcurveto@?$path_procs_t@Ucff2_path_procs_path_t@@U?$cff2_cs_interp_env_t@Unumber_t@CFF@@@CFF@@Ucff2_path_param_t@@@CFF@@SAXAEAU?$cff2_cs_interp_env_t@Unumber_t@CFF@@@2@AEAUcff2_path_param_t@@@Z 000000018004df30 f i hb-ot-cff2-table.obj
 0001:0004d230       ?hlineto@?$path_procs_t@Ucff2_path_procs_extents_t@@U?$cff2_cs_interp_env_t@Unumber_t@CFF@@@CFF@@Ucff2_extents_param_t@@@CFF@@SAXAEAU?$cff2_cs_interp_env_t@Unumber_t@CFF@@@2@AEAUcff2_extents_param_t@@@Z 000000018004e230 f i hb-ot-cff2-table.obj
 0001:0004d5b0       ?hlineto@?$path_procs_t@Ucff2_path_procs_path_t@@U?$cff2_cs_interp_env_t@Unumber_t@CFF@@@CFF@@Ucff2_path_param_t@@@CFF@@SAXAEAU?$cff2_cs_interp_env_t@Unumber_t@CFF@@@2@AEAUcff2_path_param_t@@@Z 000000018004e5b0 f i hb-ot-cff2-table.obj
 0001:0004d8d0       ?hvcurveto@?$path_procs_t@Ucff2_path_procs_extents_t@@U?$cff2_cs_interp_env_t@Unumber_t@CFF@@@CFF@@Ucff2_extents_param_t@@@CFF@@SAXAEAU?$cff2_cs_interp_env_t@Unumber_t@CFF@@@2@AEAUcff2_extents_param_t@@@Z 000000018004e8d0 f i hb-ot-cff2-table.obj
 0001:0004e620       ?hvcurveto@?$path_procs_t@Ucff2_path_procs_path_t@@U?$cff2_cs_interp_env_t@Unumber_t@CFF@@@CFF@@Ucff2_path_param_t@@@CFF@@SAXAEAU?$cff2_cs_interp_env_t@Unumber_t@CFF@@@2@AEAUcff2_path_param_t@@@Z 000000018004f620 f i hb-ot-cff2-table.obj
 0001:0004f010       ?in_error@?$cs_interp_env_t@Unumber_t@CFF@@U?$Subrs@U?$IntType@I$03@OT@@@2@@CFF@@QEBA_NXZ 0000000180050010 f i hb-ot-cff2-table.obj
 0001:0004f030       ?line@cff2_path_procs_path_t@@SAXAEAU?$cff2_cs_interp_env_t@Unumber_t@CFF@@@CFF@@AEAUcff2_path_param_t@@AEBUpoint_t@3@@Z 0000000180050030 f i hb-ot-cff2-table.obj
 0001:0004f140       ?moveto@cff2_path_procs_path_t@@SAXAEAU?$cff2_cs_interp_env_t@Unumber_t@CFF@@@CFF@@AEAUcff2_path_param_t@@AEBUpoint_t@3@@Z 0000000180050140 f i hb-ot-cff2-table.obj
 0001:0004f260       ?offset_at@?$CFFIndex@U?$IntType@I$03@OT@@@OT@@AEBAII@Z 0000000180050260 f i hb-ot-cff2-table.obj
 0001:0004f2f0       ?process_blend@?$cff2_cs_interp_env_t@Unumber_t@CFF@@@CFF@@QEAAXXZ 00000001800502f0 f i hb-ot-cff2-table.obj
 0001:0004f630       ?process_op@?$cs_opset_t@Unumber_t@CFF@@Ucff2_cs_opset_extents_t@@U?$cff2_cs_interp_env_t@Unumber_t@CFF@@@2@Ucff2_extents_param_t@@Ucff2_path_procs_extents_t@@@CFF@@SAXIAEAU?$cff2_cs_interp_env_t@Unumber_t@CFF@@@2@AEAUcff2_extents_param_t@@@Z 0000000180050630 f i hb-ot-cff2-table.obj
 0001:0004fda0       ?process_op@?$cs_opset_t@Unumber_t@CFF@@Ucff2_cs_opset_path_t@@U?$cff2_cs_interp_env_t@Unumber_t@CFF@@@2@Ucff2_path_param_t@@Ucff2_path_procs_path_t@@@CFF@@SAXIAEAU?$cff2_cs_interp_env_t@Unumber_t@CFF@@@2@AEAUcff2_path_param_t@@@Z 0000000180050da0 f i hb-ot-cff2-table.obj
 0001:000502d0       ?process_vsindex@?$cff2_cs_interp_env_t@Unumber_t@CFF@@@CFF@@QEAAXXZ 00000001800512d0 f i hb-ot-cff2-table.obj
 0001:00050340       ?rcurveline@?$path_procs_t@Ucff2_path_procs_extents_t@@U?$cff2_cs_interp_env_t@Unumber_t@CFF@@@CFF@@Ucff2_extents_param_t@@@CFF@@SAXAEAU?$cff2_cs_interp_env_t@Unumber_t@CFF@@@2@AEAUcff2_extents_param_t@@@Z 0000000180051340 f i hb-ot-cff2-table.obj
 0001:00050800       ?rcurveline@?$path_procs_t@Ucff2_path_procs_path_t@@U?$cff2_cs_interp_env_t@Unumber_t@CFF@@@CFF@@Ucff2_path_param_t@@@CFF@@SAXAEAU?$cff2_cs_interp_env_t@Unumber_t@CFF@@@2@AEAUcff2_path_param_t@@@Z 0000000180051800 f i hb-ot-cff2-table.obj
 0001:00050bd0       ?rlinecurve@?$path_procs_t@Ucff2_path_procs_extents_t@@U?$cff2_cs_interp_env_t@Unumber_t@CFF@@@CFF@@Ucff2_extents_param_t@@@CFF@@SAXAEAU?$cff2_cs_interp_env_t@Unumber_t@CFF@@@2@AEAUcff2_extents_param_t@@@Z 0000000180051bd0 f i hb-ot-cff2-table.obj
 0001:00051090       ?rlinecurve@?$path_procs_t@Ucff2_path_procs_path_t@@U?$cff2_cs_interp_env_t@Unumber_t@CFF@@@CFF@@Ucff2_path_param_t@@@CFF@@SAXAEAU?$cff2_cs_interp_env_t@Unumber_t@CFF@@@2@AEAUcff2_path_param_t@@@Z 0000000180052090 f i hb-ot-cff2-table.obj
 0001:00051400       ?rlineto@?$path_procs_t@Ucff2_path_procs_path_t@@U?$cff2_cs_interp_env_t@Unumber_t@CFF@@@CFF@@Ucff2_path_param_t@@@CFF@@SAXAEAU?$cff2_cs_interp_env_t@Unumber_t@CFF@@@2@AEAUcff2_path_param_t@@@Z 0000000180052400 f i hb-ot-cff2-table.obj
 0001:000515c0       ?rrcurveto@?$path_procs_t@Ucff2_path_procs_extents_t@@U?$cff2_cs_interp_env_t@Unumber_t@CFF@@@CFF@@Ucff2_extents_param_t@@@CFF@@SAXAEAU?$cff2_cs_interp_env_t@Unumber_t@CFF@@@2@AEAUcff2_extents_param_t@@@Z 00000001800525c0 f i hb-ot-cff2-table.obj
 0001:00051900       ?rrcurveto@?$path_procs_t@Ucff2_path_procs_path_t@@U?$cff2_cs_interp_env_t@Unumber_t@CFF@@@CFF@@Ucff2_path_param_t@@@CFF@@SAXAEAU?$cff2_cs_interp_env_t@Unumber_t@CFF@@@2@AEAUcff2_path_param_t@@@Z 0000000180052900 f i hb-ot-cff2-table.obj
 0001:00051c10       ?vhcurveto@?$path_procs_t@Ucff2_path_procs_extents_t@@U?$cff2_cs_interp_env_t@Unumber_t@CFF@@@CFF@@Ucff2_extents_param_t@@@CFF@@SAXAEAU?$cff2_cs_interp_env_t@Unumber_t@CFF@@@2@AEAUcff2_extents_param_t@@@Z 0000000180052c10 f i hb-ot-cff2-table.obj
 0001:00052950       ?vhcurveto@?$path_procs_t@Ucff2_path_procs_path_t@@U?$cff2_cs_interp_env_t@Unumber_t@CFF@@@CFF@@Ucff2_path_param_t@@@CFF@@SAXAEAU?$cff2_cs_interp_env_t@Unumber_t@CFF@@@2@AEAUcff2_path_param_t@@@Z 0000000180053950 f i hb-ot-cff2-table.obj
 0001:00053340       ?vlineto@?$path_procs_t@Ucff2_path_procs_extents_t@@U?$cff2_cs_interp_env_t@Unumber_t@CFF@@@CFF@@Ucff2_extents_param_t@@@CFF@@SAXAEAU?$cff2_cs_interp_env_t@Unumber_t@CFF@@@2@AEAUcff2_extents_param_t@@@Z 0000000180054340 f i hb-ot-cff2-table.obj
 0001:000536c0       ?vlineto@?$path_procs_t@Ucff2_path_procs_path_t@@U?$cff2_cs_interp_env_t@Unumber_t@CFF@@@CFF@@Ucff2_path_param_t@@@CFF@@SAXAEAU?$cff2_cs_interp_env_t@Unumber_t@CFF@@@2@AEAUcff2_path_param_t@@@Z 00000001800546c0 f i hb-ot-cff2-table.obj
 0001:000539e0       ?vvcurveto@?$path_procs_t@Ucff2_path_procs_extents_t@@U?$cff2_cs_interp_env_t@Unumber_t@CFF@@@CFF@@Ucff2_extents_param_t@@@CFF@@SAXAEAU?$cff2_cs_interp_env_t@Unumber_t@CFF@@@2@AEAUcff2_extents_param_t@@@Z 00000001800549e0 f i hb-ot-cff2-table.obj
 0001:00053d00       ?vvcurveto@?$path_procs_t@Ucff2_path_procs_path_t@@U?$cff2_cs_interp_env_t@Unumber_t@CFF@@@CFF@@Ucff2_path_param_t@@@CFF@@SAXAEAU?$cff2_cs_interp_env_t@Unumber_t@CFF@@@2@AEAUcff2_path_param_t@@@Z 0000000180054d00 f i hb-ot-cff2-table.obj
 0001:00054000       ??$_dispatch@UIndexSubtableArray@OT@@AEBU?$IntType@I$03@2@@hb_sanitize_context_t@@AEAA_NAEBUIndexSubtableArray@OT@@U?$hb_priority@$00@@AEBU?$IntType@I$03@2@@Z 0000000180055000 f i hb-ot-color.obj
 0001:000541e0       ??$dispatch@U?$ColorLine@UNoVariable@OT@@@OT@@$$V@hb_sanitize_context_t@@QEAA_NAEBU?$ColorLine@UNoVariable@OT@@@OT@@@Z 00000001800551e0 f i hb-ot-color.obj
 0001:000542a0       ??$dispatch@U?$ColorLine@UVariable@OT@@@OT@@$$V@hb_sanitize_context_t@@QEAA_NAEBU?$ColorLine@UVariable@OT@@@OT@@@Z 00000001800552a0 f i hb-ot-color.obj
 0001:00054360       ??$dispatch@U?$NoVariable@UAffine2x3@OT@@@OT@@$$V@hb_sanitize_context_t@@QEAA_NAEBU?$NoVariable@UAffine2x3@OT@@@OT@@@Z 0000000180055360 f i hb-ot-color.obj
 0001:00054480       ??$dispatch@U?$Variable@UAffine2x3@OT@@@OT@@$$V@hb_sanitize_context_t@@QEAA_NAEBU?$Variable@UAffine2x3@OT@@@OT@@@Z 0000000180055480 f i hb-ot-color.obj
 0001:000545a0       ??$dispatch@ULayerList@OT@@$$V@hb_sanitize_context_t@@QEAA_NAEBULayerList@OT@@@Z 00000001800555a0 f i hb-ot-color.obj
 0001:000546a0       ??$dispatch@USBIXStrike@OT@@$$V@hb_sanitize_context_t@@QEAA_NAEBUSBIXStrike@OT@@@Z 00000001800556a0 f i hb-ot-color.obj
 0001:00054810       ??$dispatch@Uhb_sanitize_context_t@@$$V@ClipBox@OT@@QEBA_NPEAUhb_sanitize_context_t@@@Z 0000000180055810 f i hb-ot-color.obj
 0001:000549f0       ??$dispatch@Uhb_sanitize_context_t@@$$V@Paint@OT@@QEBA_NPEAUhb_sanitize_context_t@@@Z 00000001800559f0 f i hb-ot-color.obj
 0001:000558e0       ??$sanitize@$$V@Paint@OT@@QEBA_NPEAUhb_sanitize_context_t@@@Z 00000001800568e0 f i hb-ot-color.obj
 0001:00055910       ??$sanitize_blob@UCBDT@OT@@@hb_sanitize_context_t@@QEAAPEAUhb_blob_t@@PEAU1@@Z 0000000180056910 f i hb-ot-color.obj
 0001:00055b30       ??$sanitize_blob@UCBLC@OT@@@hb_sanitize_context_t@@QEAAPEAUhb_blob_t@@PEAU1@@Z 0000000180056b30 f i hb-ot-color.obj
 0001:00055db0       ??$sanitize_blob@UCOLR@OT@@@hb_sanitize_context_t@@QEAAPEAUhb_blob_t@@PEAU1@@Z 0000000180056db0 f i hb-ot-color.obj
 0001:00055f40       ??$sanitize_blob@UCPAL@OT@@@hb_sanitize_context_t@@QEAAPEAUhb_blob_t@@PEAU1@@Z 0000000180056f40 f i hb-ot-color.obj
 0001:000560d0       ??$sanitize_blob@USVG@OT@@@hb_sanitize_context_t@@QEAAPEAUhb_blob_t@@PEAU1@@Z 00000001800570d0 f i hb-ot-color.obj
 0001:00056420       ??$sanitize_blob@Usbix@OT@@@hb_sanitize_context_t@@QEAAPEAUhb_blob_t@@PEAU1@@Z 0000000180057420 f i hb-ot-color.obj
 0001:000566d0       ??1accelerator_t@COLR@OT@@QEAA@XZ 00000001800576d0 f i hb-ot-color.obj
 0001:00056740       ??1hb_paint_extents_context_t@@QEAA@XZ 0000000180057740 f i hb-ot-color.obj
 0001:000567b0       ??C?$hb_lazy_loader_t@UCOLR_accelerator_t@OT@@U?$hb_face_lazy_loader_t@UCOLR_accelerator_t@OT@@$0CD@@@Uhb_face_t@@$0CD@U12@@@QEBAPEBUCOLR_accelerator_t@OT@@XZ 00000001800577b0 f i hb-ot-color.obj
 0001:00056960       ??C?$hb_lazy_loader_t@UCPAL@OT@@U?$hb_table_lazy_loader_t@UCPAL@OT@@$0CE@$00@@Uhb_face_t@@$0CE@Uhb_blob_t@@@@QEBAPEBUCPAL@OT@@XZ 0000000180057960 f i hb-ot-color.obj
 0001:00056ad0       ??C?$hb_lazy_loader_t@Usbix_accelerator_t@OT@@U?$hb_face_lazy_loader_t@Usbix_accelerator_t@OT@@$0CG@@@Uhb_face_t@@$0CG@U12@@@QEBAPEBUsbix_accelerator_t@OT@@XZ 0000000180057ad0 f i hb-ot-color.obj
 0001:00056c70       ?choose_strike@CBLC@OT@@IEBAAEBUBitmapSizeTable@2@PEAUhb_font_t@@@Z 0000000180057c70 f i hb-ot-color.obj
 0001:00056d70       ?choose_strike@accelerator_t@sbix@OT@@AEBAAEBUSBIXStrike@3@PEAUhb_font_t@@@Z 0000000180057d70 f i hb-ot-color.obj
 0001:00056f50       ?find_table@IndexSubtableArray@OT@@QEBAPEBUIndexSubtableRecord@2@II@Z 0000000180057f50 f i hb-ot-color.obj
 0001:00056fc0       ?get_base_glyph_paint@COLR@OT@@QEBAPEBUPaint@2@I@Z 0000000180057fc0 f i hb-ot-color.obj
 0001:000570f0       ?get_glyph_blob@SBIXStrike@OT@@QEBAPEAUhb_blob_t@@IPEAU3@IPEAH1IPEAI@Z 00000001800580f0 f i hb-ot-color.obj
 0001:00057320       ?get_image_data@IndexSubtable@OT@@QEBA_NIPEAI00@Z 0000000180058320 f i hb-ot-color.obj
 0001:00057500       ?get_stored@?$hb_lazy_loader_t@UCBDT_accelerator_t@OT@@U?$hb_face_lazy_loader_t@UCBDT_accelerator_t@OT@@$0CF@@@Uhb_face_t@@$0CF@U12@@@QEBAPEAUCBDT_accelerator_t@OT@@XZ 0000000180058500 f i hb-ot-color.obj
 0001:00057730       ?get_strike@sbix@OT@@QEBAAEBUSBIXStrike@2@I@Z 0000000180058730 f i hb-ot-color.obj
 0001:000577e0       ?reference_blob_for_glyph@accelerator_t@SVG@OT@@QEBAPEAUhb_blob_t@@I@Z 00000001800587e0 f i hb-ot-color.obj
 0001:00057940       ?reference_png@accelerator_t@CBDT@OT@@QEBAPEAUhb_blob_t@@PEAUhb_font_t@@I@Z 0000000180058940 f i hb-ot-color.obj
 0001:00057bf0       ?sanitize@BaseGlyphList@OT@@QEBA_NPEAUhb_sanitize_context_t@@@Z 0000000180058bf0 f i hb-ot-color.obj
 0001:00057d90       ?sanitize@BitmapSizeTable@OT@@QEBA_NPEAUhb_sanitize_context_t@@PEBX@Z 0000000180058d90 f i hb-ot-color.obj
 0001:00057f70       ?sanitize@CBDT@OT@@QEBA_NPEAUhb_sanitize_context_t@@@Z 0000000180058f70 f i hb-ot-color.obj
 0001:00058040       ?sanitize@CBLC@OT@@QEBA_NPEAUhb_sanitize_context_t@@@Z 0000000180059040 f i hb-ot-color.obj
 0001:00058180       ?sanitize@COLR@OT@@QEBA_NPEAUhb_sanitize_context_t@@@Z 0000000180059180 f i hb-ot-color.obj
 0001:000584a0       ?sanitize@CPAL@OT@@QEBA_NPEAUhb_sanitize_context_t@@@Z 00000001800594a0 f i hb-ot-color.obj
 0001:00058730       ?sanitize@ClipList@OT@@QEBA_NPEAUhb_sanitize_context_t@@@Z 0000000180059730 f i hb-ot-color.obj
 0001:00058910       ?sanitize@IndexSubtable@OT@@QEBA_NPEAUhb_sanitize_context_t@@I@Z 0000000180059910 f i hb-ot-color.obj
 0001:00058ad0       ?sanitize@PaintScaleUniform@OT@@QEBA_NPEAUhb_sanitize_context_t@@@Z 0000000180059ad0 f i hb-ot-color.obj
 0001:00058ad0       ?sanitize@PaintRotate@OT@@QEBA_NPEAUhb_sanitize_context_t@@@Z 0000000180059ad0 f i hb-ot-color.obj
 0001:00058bd0       ?sanitize@PaintRotateAroundCenter@OT@@QEBA_NPEAUhb_sanitize_context_t@@@Z 0000000180059bd0 f i hb-ot-color.obj
 0001:00058bd0       ?sanitize@PaintScaleUniformAroundCenter@OT@@QEBA_NPEAUhb_sanitize_context_t@@@Z 0000000180059bd0 f i hb-ot-color.obj
 0001:00058cd0       ?sanitize@PaintScale@OT@@QEBA_NPEAUhb_sanitize_context_t@@@Z 0000000180059cd0 f i hb-ot-color.obj
 0001:00058cd0       ?sanitize@PaintTranslate@OT@@QEBA_NPEAUhb_sanitize_context_t@@@Z 0000000180059cd0 f i hb-ot-color.obj
 0001:00058cd0       ?sanitize@PaintSkew@OT@@QEBA_NPEAUhb_sanitize_context_t@@@Z 0000000180059cd0 f i hb-ot-color.obj
 0001:00058dd0       ?sanitize@PaintSkewAroundCenter@OT@@QEBA_NPEAUhb_sanitize_context_t@@@Z 0000000180059dd0 f i hb-ot-color.obj
 0001:00058dd0       ?sanitize@PaintScaleAroundCenter@OT@@QEBA_NPEAUhb_sanitize_context_t@@@Z 0000000180059dd0 f i hb-ot-color.obj
 0001:00058ed0       ?sanitize@SVG@OT@@QEBA_NPEAUhb_sanitize_context_t@@@Z 0000000180059ed0 f i hb-ot-color.obj
 0001:000590d0       ?sanitize@sbix@OT@@QEBA_NPEAUhb_sanitize_context_t@@@Z 000000018005a0d0 f i hb-ot-color.obj
 0001:00059240       ?sanitize_shallow@?$ArrayOf@U?$Variable@UColorStop@OT@@@OT@@U?$IntType@G$01@2@@OT@@QEBA_NPEAUhb_sanitize_context_t@@@Z 000000018005a240 f i hb-ot-color.obj
 0001:000593b0       ?sanitize_shallow@?$ArrayOf@U?$FDSelect3_4_Range@U?$IntType@I$03@OT@@U?$IntType@G$01@2@@CFF@@U?$IntType@I$03@OT@@@OT@@QEBA_NPEAUhb_sanitize_context_t@@@Z 000000018005a3b0 f i hb-ot-font.obj
 0001:000593b0       ?sanitize_shallow@?$ArrayOf@UBaseGlyphPaintRecord@OT@@U?$IntType@I$03@2@@OT@@QEBA_NPEAUhb_sanitize_context_t@@@Z 000000018005a3b0 f i hb-ot-color.obj
 0001:00059540       ?sanitize_shallow@?$ArrayOf@UBitmapSizeTable@OT@@U?$IntType@I$03@2@@OT@@QEBA_NPEAUhb_sanitize_context_t@@@Z 000000018005a540 f i hb-ot-color.obj
 0001:000596d0       ?sanitize_shallow@?$ArrayOf@UClipRecord@OT@@U?$IntType@I$03@2@@OT@@QEBA_NPEAUhb_sanitize_context_t@@@Z 000000018005a6d0 f i hb-ot-color.obj
 0001:00059850       ??1?$accelerator_templ_t@Ucff1_private_dict_opset_t@CFF@@U?$cff1_private_dict_values_base_t@Udict_val_t@CFF@@@2@@cff1@OT@@QEAA@XZ 000000018005a850 f i hb-ot-face.obj
 0001:00059920       ??1?$accelerator_templ_t@Ucff2_private_dict_opset_t@CFF@@U?$cff2_private_dict_values_base_t@Udict_val_t@CFF@@@2@@cff2@OT@@QEAA@XZ 000000018005a920 f i hb-ot-face.obj
 0001:000599e0       ??1kern_accelerator_data_t@AAT@@QEAA@XZ 000000018005a9e0 f i hb-ot-face.obj
 0001:00059a30       ??_Ghb_colr_scratch_t@@QEAAPEAXI@Z 000000018005aa30 f i hb-ot-face.obj
 0001:00059aa0       ?_fini@?$accelerator_templ_t@Ucff1_private_dict_opset_t@CFF@@U?$cff1_private_dict_values_base_t@Udict_val_t@CFF@@@2@@cff1@OT@@QEAAXXZ 000000018005aaa0 f i hb-ot-face.obj
 0001:00059b70       ?_fini@?$accelerator_templ_t@Ucff2_private_dict_opset_t@CFF@@U?$cff2_private_dict_values_base_t@Udict_val_t@CFF@@@2@@cff2@OT@@QEAAXXZ 000000018005ab70 f i hb-ot-face.obj
 0001:00059c70       ?fini@hb_ot_face_t@@QEAAXXZ 000000018005ac70 f   hb-ot-face.obj
 0001:0005a630       ?init0@hb_ot_face_t@@QEAAXPEAUhb_face_t@@@Z 000000018005b630 f   hb-ot-face.obj
 0001:0005a640       ?shrink_vector@?$hb_vector_t@U?$cff1_private_dict_values_base_t@Udict_val_t@CFF@@@CFF@@$0A@@@QEAAXI@Z 000000018005b640 f i hb-ot-face.obj
 0001:0005a640       ?shrink_vector@?$hb_vector_t@Ucff1_font_dict_values_t@CFF@@$0A@@@QEAAXI@Z 000000018005b640 f i hb-ot-face.obj
 0001:0005a640       ?shrink_vector@?$hb_vector_t@Ucff2_font_dict_values_t@CFF@@$0A@@@QEAAXI@Z 000000018005b640 f i hb-ot-face.obj
 0001:0005a6e0       ?shrink_vector@?$hb_vector_t@U?$cff2_private_dict_values_base_t@Udict_val_t@CFF@@@CFF@@$0A@@@QEAAXI@Z 000000018005b6e0 f i hb-ot-face.obj
 0001:0005a920       ??$dispatch@Uhb_paint_context_t@OT@@$$V@Paint@OT@@QEBA?AUhb_empty_t@@PEAUhb_paint_context_t@1@@Z 000000018005b920 f i hb-ot-font.obj
 0001:0005b0c0       ??$get_extents_without_var_scaled@Uglyf_accelerator_t@OT@@@GlyphHeader@glyf_impl@OT@@QEBA_NPEAUhb_font_t@@AEBUglyf_accelerator_t@2@IPEAUhb_glyph_extents_t@@@Z 000000018005c0c0 f i hb-ot-font.obj
 0001:0005b320       ??$get_points@Upath_builder_t@glyf_impl@OT@@@glyf_accelerator_t@OT@@IEBA_NPEAUhb_font_t@@IUpath_builder_t@glyf_impl@1@U?$hb_array_t@$$CBH@@AEAUhb_glyf_scratch_t@@@Z 000000018005c320 f i hb-ot-font.obj
 0001:0005c320       ??$sanitize@Uhb_sanitize_context_t@@@?$hb_array_t@$$CBE@@QEBA_NPEAUhb_sanitize_context_t@@@Z 000000018005d320 f i hb-ot-font.obj
 0001:0005c400       ??$sanitize_blob@UVORG@OT@@@hb_sanitize_context_t@@QEAAPEAUhb_blob_t@@PEAU1@@Z 000000018005d400 f i hb-ot-font.obj
 0001:0005c630       ??$sanitize_blob@Ucff1@OT@@@hb_sanitize_context_t@@QEAAPEAUhb_blob_t@@PEAU1@@Z 000000018005d630 f i hb-ot-font.obj
 0001:0005c830       ??$sanitize_blob@Ucff2@OT@@@hb_sanitize_context_t@@QEAAPEAUhb_blob_t@@PEAU1@@Z 000000018005d830 f i hb-ot-font.obj
 0001:0005ca30       ??$sanitize_blob@Upost@OT@@@hb_sanitize_context_t@@QEAAPEAUhb_blob_t@@PEAU1@@Z 000000018005da30 f i hb-ot-font.obj
 0001:0005d040       ??0?$accelerator_templ_t@Ucff1_private_dict_opset_t@CFF@@U?$cff1_private_dict_values_base_t@Udict_val_t@CFF@@@2@@cff1@OT@@QEAA@PEAUhb_face_t@@@Z 000000018005e040 f i hb-ot-font.obj
 0001:0005e200       ??0?$accelerator_templ_t@Ucff2_private_dict_opset_t@CFF@@U?$cff2_private_dict_values_base_t@Udict_val_t@CFF@@@2@@cff2@OT@@QEAA@PEAUhb_face_t@@@Z 000000018005f200 f i hb-ot-font.obj
 0001:0005efe0       ??0accelerator_t@post@OT@@QEAA@PEAUhb_face_t@@@Z 000000018005ffe0 f i hb-ot-font.obj
 0001:0005f320       ??0hb_paint_context_t@OT@@QEAA@PEBXPEAUhb_paint_funcs_t@@PEAXPEAUhb_font_t@@IIAEAUItemVarStoreInstancer@1@@Z 0000000180060320 f i hb-ot-font.obj
 0001:0005f4f0       ??1accelerator_t@cff1@OT@@QEAA@XZ 00000001800604f0 f i hb-ot-font.obj
 0001:0005f550       ??C?$hb_lazy_loader_t@Ucff1_accelerator_t@OT@@U?$hb_face_lazy_loader_t@Ucff1_accelerator_t@OT@@$0BA@@@Uhb_face_t@@$0BA@U12@@@QEBAPEBUcff1_accelerator_t@OT@@XZ 0000000180060550 f i hb-ot-font.obj
 0001:0005f610       ??C?$hb_lazy_loader_t@Ucff2_accelerator_t@OT@@U?$hb_face_lazy_loader_t@Ucff2_accelerator_t@OT@@$0BB@@@Uhb_face_t@@$0BB@U12@@@QEBAPEBUcff2_accelerator_t@OT@@XZ 0000000180060610 f i hb-ot-font.obj
 0001:0005f6c0       ??C?$hb_lazy_loader_t@Upost_accelerator_t@OT@@U?$hb_face_lazy_loader_t@Upost_accelerator_t@OT@@$06@@Uhb_face_t@@$06U12@@@QEBAPEBUpost_accelerator_t@OT@@XZ 00000001800606c0 f i hb-ot-font.obj
 0001:0005f7a0       ??RItemVarStoreInstancer@OT@@QEBAMIG@Z 00000001800607a0 f i hb-ot-font.obj
 0001:0005f820       ?_cached_get@accelerator_t@cmap@OT@@QEBA_NIPEAI@Z 0000000180060820 f i hb-ot-font.obj
 0001:0005f8f0       ?acquire_varStore_cache@advance_cache_t@hb_ot_font_t@@QEBAPEAU?$hb_atomic_t@H@@AEBUItemVariationStore@OT@@@Z 00000001800608f0 f i hb-ot-font.obj
 0001:0005f9c0       ?add_op@?$parsed_values_t@Udict_val_t@CFF@@@CFF@@QEAAXIAEBUbyte_str_ref_t@2@AEBUdict_val_t@2@@Z 00000001800609c0 f i hb-ot-font.obj
 0001:0005f9c0       ?add_op@?$parsed_values_t@Uop_str_t@CFF@@@CFF@@QEAAXIAEBUbyte_str_ref_t@2@AEBUop_str_t@2@@Z 00000001800609c0 f i hb-ot-font.obj
 0001:0005fae0       ?alloc@?$hb_vector_t@U?$cff1_private_dict_values_base_t@Udict_val_t@CFF@@@CFF@@$0A@@@QEAA_NI_N@Z 0000000180060ae0 f i hb-ot-font.obj
 0001:0005fcb0       ?alloc@?$hb_vector_t@U?$cff2_private_dict_values_base_t@Udict_val_t@CFF@@@CFF@@$0A@@@QEAA_NI_N@Z 0000000180060cb0 f i hb-ot-font.obj
 0001:0005fe80       ?alloc@?$hb_vector_t@Ucff1_font_dict_values_t@CFF@@$0A@@@QEAA_NI_N@Z 0000000180060e80 f i hb-ot-font.obj
 0001:00060050       ?alloc@?$hb_vector_t@Ucff2_font_dict_values_t@CFF@@$0A@@@QEAA_NI_N@Z 0000000180061050 f i hb-ot-font.obj
 0001:00060220       ?clear@advance_cache_t@hb_ot_font_t@@QEBAXXZ 0000000180061220 f i hb-ot-font.obj
 0001:000602a0       ?cmp@gname_t@accelerator_t@cff1@OT@@SAHPEBX0@Z 00000001800612a0 f i hb-ot-font.obj
 0001:000602e0       ?cmp_gids@accelerator_t@post@OT@@KAHPEBX0PEAX@Z 00000001800612e0 f i hb-ot-font.obj
 0001:00060370       ?contour_end@path_builder_t@glyf_impl@OT@@QEAAXXZ 0000000180061370 f i hb-ot-font.obj
 0001:00060b90       ?find_glyph_name@accelerator_t@post@OT@@IEBA?AU?$hb_array_t@$$CBD@@I@Z 0000000180061b90 f i hb-ot-font.obj
 0001:00060ca0       ?get_advance_delta_unscaled@HVARVVAR@OT@@QEBAMIPEBHIPEAU?$hb_atomic_t@H@@@Z 0000000180061ca0 f i hb-ot-font.obj
 0001:00060d50       ?get_base_glyph_record@COLR@OT@@QEBAPEBUBaseGlyphRecord@2@I@Z 0000000180061d50 f i hb-ot-font.obj
 0001:00060e00       ?get_clip_box@ClipBoxFormat2@OT@@QEBAXAEAUClipBoxData@2@AEBUItemVarStoreInstancer@2@@Z 0000000180061e00 f i hb-ot-font.obj
 0001:00060fe0       ?get_color@hb_paint_context_t@OT@@QEAAIIMPEAH@Z 0000000180061fe0 f i hb-ot-font.obj
 0001:000610c0       ?get_color_stop@ColorStop@OT@@QEBAXPEAUhb_paint_context_t@2@PEAUhb_color_stop_t@@IAEBUItemVarStoreInstancer@2@@Z 00000001800620c0 f i hb-ot-font.obj
 0001:000611a0       ?get_delta@ItemVariationStore@OT@@QEBAMIPEBHIPEAU?$hb_atomic_t@H@@@Z 00000001800621a0 f i hb-ot-font.obj
 0001:00061270       ?get_delta@VarData@OT@@QEBAMIPEBHIAEBUVarRegionList@2@PEAU?$hb_atomic_t@H@@@Z 0000000180062270 f i hb-ot-font.obj
 0001:00061a50       ?get_delta_set_index_map_ptr@COLR@OT@@QEBAPEBUDeltaSetIndexMap@2@XZ 0000000180062a50 f i hb-ot-font.obj
 0001:00061ac0       ?get_extents@COLR@OT@@QEBA_NPEAUhb_font_t@@IPEAUhb_glyph_extents_t@@AEAUhb_colr_scratch_t@@@Z 0000000180062ac0 f i hb-ot-font.obj
 0001:00061d00       ?get_extents@ClipList@OT@@QEBA_NIPEAUhb_glyph_extents_t@@AEBUItemVarStoreInstancer@2@@Z 0000000180062d00 f i hb-ot-font.obj
 0001:00061e90       ?get_extents@accelerator_t@CBDT@OT@@QEBA_NPEAUhb_font_t@@IPEAUhb_glyph_extents_t@@_N@Z 0000000180062e90 f i hb-ot-font.obj
 0001:00062190       ?get_extents_at@glyf_accelerator_t@OT@@QEBA_NPEAUhb_font_t@@IPEAUhb_glyph_extents_t@@U?$hb_array_t@$$CBH@@@Z 0000000180063190 f i hb-ot-font.obj
 0001:00062400       ?get_glyph@VariationSelectorRecord@OT@@QEBA?AW4glyph_variant_t@2@IPEAIPEBX@Z 0000000180063400 f i hb-ot-font.obj
 0001:000625d0       ?get_glyph_from_name@accelerator_t@cff1@OT@@QEBA_NPEBDHPEAI@Z 00000001800635d0 f i hb-ot-font.obj
 0001:00062a10       ?get_glyph_from_name@accelerator_t@post@OT@@QEBA_NPEBDHPEAI@Z 0000000180063a10 f i hb-ot-font.obj
 0001:00062b90       ?get_png_extents@accelerator_t@sbix@OT@@AEBA_NPEAUhb_font_t@@IPEAUhb_glyph_extents_t@@_N@Z 0000000180063b90 f i hb-ot-font.obj
 0001:00062dc0       ?get_sid@Charset@CFF@@QEBAIIIPEAUcode_pair_t@2@@Z 0000000180063dc0 f i hb-ot-font.obj
 0001:00062f40       ?get_size@?$CFFIndex@U?$IntType@G$01@OT@@@OT@@QEBAIXZ 0000000180063f40 f i hb-ot-font.obj
 0001:00063040       ?get_var_store_ptr@COLR@OT@@QEBAPEBUItemVariationStore@2@XZ 0000000180064040 f i hb-ot-font.obj
 0001:000630b0       ?glyph_to_sid@?$accelerator_templ_t@Ucff1_private_dict_opset_t@CFF@@U?$cff1_private_dict_values_base_t@Udict_val_t@CFF@@@2@@cff1@OT@@QEBAIIPEAUcode_pair_t@CFF@@@Z 00000001800640b0 f i hb-ot-font.obj
 0001:00064ef0       ?interpret@?$dict_interpreter_t@Ucff1_font_dict_opset_t@CFF@@Ucff1_font_dict_values_t@2@U?$interp_env_t@Unumber_t@CFF@@@2@@CFF@@QEAA_NAEAUcff1_font_dict_values_t@2@@Z 0000000180065ef0 f i hb-ot-font.obj
 0001:00065100       ?interpret@?$dict_interpreter_t@Ucff1_private_dict_opset_t@CFF@@U?$cff1_private_dict_values_base_t@Udict_val_t@CFF@@@2@U?$interp_env_t@Unumber_t@CFF@@@2@@CFF@@QEAA_NAEAU?$cff1_private_dict_values_base_t@Udict_val_t@CFF@@@2@@Z 0000000180066100 f i hb-ot-font.obj
 0001:00065340       ?interpret@?$dict_interpreter_t@Ucff1_top_dict_opset_t@CFF@@Ucff1_top_dict_values_t@2@Ucff1_top_dict_interp_env_t@2@@CFF@@QEAA_NAEAUcff1_top_dict_values_t@2@@Z 0000000180066340 f i hb-ot-font.obj
 0001:00065450       ?interpret@?$dict_interpreter_t@Ucff2_font_dict_opset_t@CFF@@Ucff2_font_dict_values_t@2@U?$interp_env_t@Unumber_t@CFF@@@2@@CFF@@QEAA_NAEAUcff2_font_dict_values_t@2@@Z 0000000180066450 f i hb-ot-font.obj
 0001:00065610       ?interpret@?$dict_interpreter_t@Ucff2_private_dict_opset_t@CFF@@U?$cff2_private_dict_values_base_t@Udict_val_t@CFF@@@2@Ucff2_priv_dict_interp_env_t@2@@CFF@@QEAA_NAEAU?$cff2_private_dict_values_base_t@Udict_val_t@CFF@@@2@@Z 0000000180066610 f i hb-ot-font.obj
 0001:000658e0       ?interpret@?$dict_interpreter_t@Ucff2_top_dict_opset_t@CFF@@Ucff2_top_dict_values_t@2@U?$interp_env_t@Unumber_t@CFF@@@2@@CFF@@QEAA_NAEAUcff2_top_dict_values_t@2@@Z 00000001800668e0 f i hb-ot-font.obj
 0001:000659b0       ?map@DeltaSetIndexMap@OT@@QEBAII@Z 00000001800669b0 f i hb-ot-font.obj
 0001:00065ac0       ?paint_glyph@?$PaintLinearGradient@UNoVariable@OT@@@OT@@QEBAXPEAUhb_paint_context_t@2@I@Z 0000000180066ac0 f i hb-ot-font.obj
 0001:00065d50       ?paint_glyph@?$PaintLinearGradient@UVariable@OT@@@OT@@QEBAXPEAUhb_paint_context_t@2@I@Z 0000000180066d50 f i hb-ot-font.obj
 0001:00065fe0       ?paint_glyph@?$PaintRadialGradient@UNoVariable@OT@@@OT@@QEBAXPEAUhb_paint_context_t@2@I@Z 0000000180066fe0 f i hb-ot-font.obj
 0001:00066270       ?paint_glyph@?$PaintRadialGradient@UVariable@OT@@@OT@@QEBAXPEAUhb_paint_context_t@2@I@Z 0000000180067270 f i hb-ot-font.obj
 0001:00066500       ?paint_glyph@?$PaintSweepGradient@UNoVariable@OT@@@OT@@QEBAXPEAUhb_paint_context_t@2@I@Z 0000000180067500 f i hb-ot-font.obj
 0001:00066710       ?paint_glyph@?$PaintSweepGradient@UVariable@OT@@@OT@@QEBAXPEAUhb_paint_context_t@2@I@Z 0000000180067710 f i hb-ot-font.obj
 0001:00066920       ?paint_glyph@Affine2x3@OT@@QEBAXPEAUhb_paint_context_t@2@I@Z 0000000180067920 f i hb-ot-font.obj
 0001:00066b70       ?paint_glyph@COLR@OT@@QEBA_NPEAUhb_font_t@@IPEAUhb_paint_funcs_t@@PEAXII_NAEAUhb_colr_scratch_t@@@Z 0000000180067b70 f i hb-ot-font.obj
 0001:00067150       ?paint_glyph@PaintColrGlyph@OT@@QEBAXPEAUhb_paint_context_t@2@@Z 0000000180068150 f i hb-ot-font.obj
 0001:00067470       ?paint_glyph@PaintColrLayers@OT@@QEBAXPEAUhb_paint_context_t@2@@Z 0000000180068470 f i hb-ot-font.obj
 0001:000676c0       ?paint_glyph@PaintRotate@OT@@QEBAXPEAUhb_paint_context_t@2@I@Z 00000001800686c0 f i hb-ot-font.obj
 0001:00067790       ?paint_glyph@PaintRotateAroundCenter@OT@@QEBAXPEAUhb_paint_context_t@2@I@Z 0000000180068790 f i hb-ot-font.obj
 0001:00067a40       ?paint_glyph@PaintScale@OT@@QEBAXPEAUhb_paint_context_t@2@I@Z 0000000180068a40 f i hb-ot-font.obj
 0001:00067bb0       ?paint_glyph@PaintScaleAroundCenter@OT@@QEBAXPEAUhb_paint_context_t@2@I@Z 0000000180068bb0 f i hb-ot-font.obj
 0001:00067ef0       ?paint_glyph@PaintScaleUniform@OT@@QEBAXPEAUhb_paint_context_t@2@I@Z 0000000180068ef0 f i hb-ot-font.obj
 0001:00068010       ?paint_glyph@PaintScaleUniformAroundCenter@OT@@QEBAXPEAUhb_paint_context_t@2@I@Z 0000000180069010 f i hb-ot-font.obj
 0001:00068300       ?paint_glyph@PaintSkew@OT@@QEBAXPEAUhb_paint_context_t@2@I@Z 0000000180069300 f i hb-ot-font.obj
 0001:00068420       ?paint_glyph@PaintSkewAroundCenter@OT@@QEBAXPEAUhb_paint_context_t@2@I@Z 0000000180069420 f i hb-ot-font.obj
 0001:00068720       ?paint_glyph@PaintSolid@OT@@QEBAXPEAUhb_paint_context_t@2@I@Z 0000000180069720 f i hb-ot-font.obj
 0001:000687c0       ?paint_glyph@PaintTranslate@OT@@QEBAXPEAUhb_paint_context_t@2@I@Z 00000001800697c0 f i hb-ot-font.obj
 0001:00068930       ?parse_bcd@dict_opset_t@CFF@@SANAEAUbyte_str_ref_t@2@@Z 0000000180069930 f i hb-ot-font.obj
 0001:00068a60       ?pop_int@?$arg_stack_t@Unumber_t@CFF@@@CFF@@QEAAHXZ 0000000180069a60 f i hb-ot-font.obj
 0001:00068a90       ?pop_uint@?$arg_stack_t@Unumber_t@CFF@@@CFF@@QEAAIXZ 0000000180069a90 f i hb-ot-font.obj
 0001:00068ad0       ?process_op@cff1_top_dict_opset_t@CFF@@SAXIAEAUcff1_top_dict_interp_env_t@2@AEAUcff1_top_dict_values_t@2@@Z 0000000180069ad0 f i hb-ot-font.obj
 0001:00068ff0       ?process_op@cff2_top_dict_opset_t@CFF@@SAXIAEAU?$interp_env_t@Unumber_t@CFF@@@2@AEAUcff2_top_dict_values_t@2@@Z 0000000180069ff0 f i hb-ot-font.obj
 0001:00069200       ?process_op@dict_opset_t@CFF@@SAXIAEAU?$interp_env_t@Unumber_t@CFF@@@2@@Z 000000018006a200 f i hb-ot-font.obj
 0001:00069330       ?push@?$hb_vector_t@Ucff1_font_dict_values_t@CFF@@$0A@@@QEAAPEAUcff1_font_dict_values_t@CFF@@XZ 000000018006a330 f i hb-ot-font.obj
 0001:00069420       ?push@?$hb_vector_t@Ucff2_font_dict_values_t@CFF@@$0A@@@QEAAPEAUcff2_font_dict_values_t@CFF@@XZ 000000018006a420 f i hb-ot-font.obj
 0001:00069510       ?push_font_transform@hb_paint_funcs_t@@QEAAXPEAXPEBUhb_font_t@@@Z 000000018006a510 f i hb-ot-font.obj
 0001:000695b0       ?push_inverse_font_transform@hb_paint_funcs_t@@QEAAXPEAXPEBUhb_font_t@@@Z 000000018006a5b0 f i hb-ot-font.obj
 0001:00069680       ?push_rotate@hb_paint_funcs_t@@QEAA_NPEAXM@Z 000000018006a680 f i hb-ot-font.obj
 0001:00069740       ?push_skew@hb_paint_funcs_t@@QEAA_NPEAXMM@Z 000000018006a740 f i hb-ot-font.obj
 0001:00069810       ?recurse@hb_paint_context_t@OT@@QEAAXAEBUPaint@2@@Z 000000018006a810 f i hb-ot-font.obj
 0001:00069860       ?release_scratch@accelerator_t@COLR@OT@@AEBAXPEAUhb_colr_scratch_t@@@Z 000000018006a860 f i hb-ot-font.obj
 0001:000698c0       ?sanitize@?$CFFIndex@U?$IntType@G$01@OT@@@OT@@QEBA_NPEAUhb_sanitize_context_t@@@Z 000000018006a8c0 f i hb-ot-font.obj
 0001:00069b30       ?sanitize@?$CFFIndex@U?$IntType@I$03@OT@@@OT@@QEBA_NPEAUhb_sanitize_context_t@@@Z 000000018006ab30 f i hb-ot-font.obj
 0001:00069dc0       ?sanitize@?$FDSelect3_4@U?$IntType@G$01@OT@@U?$IntType@E$00@2@@CFF@@QEBA_NPEAUhb_sanitize_context_t@@I@Z 000000018006adc0 f i hb-ot-font.obj
 0001:0006a0e0       ?sanitize@?$FDSelect3_4@U?$IntType@I$03@OT@@U?$IntType@G$01@2@@CFF@@QEBA_NPEAUhb_sanitize_context_t@@I@Z 000000018006b0e0 f i hb-ot-font.obj
 0001:0006a480       ?sanitize@Charset@CFF@@QEBA_NPEAUhb_sanitize_context_t@@PEAI@Z 000000018006b480 f i hb-ot-font.obj
 0001:0006a710       ?sanitize@FDSelect0@CFF@@QEBA_NPEAUhb_sanitize_context_t@@I@Z 000000018006b710 f i hb-ot-font.obj
 0001:0006a7b0       ?sanitize@VORG@OT@@QEBA_NPEAUhb_sanitize_context_t@@@Z 000000018006b7b0 f i hb-ot-font.obj
 0001:0006a880       ?sanitize@cff1@OT@@QEBA_NPEAUhb_sanitize_context_t@@@Z 000000018006b880 f i hb-ot-font.obj
 0001:0006a930       ?sanitize@cff2@OT@@QEBA_NPEAUhb_sanitize_context_t@@@Z 000000018006b930 f i hb-ot-font.obj
 0001:0006a9e0       ?sanitize@post@OT@@QEBA_NPEAUhb_sanitize_context_t@@@Z 000000018006b9e0 f i hb-ot-font.obj
 0001:0006ab00       ?sanitize_shallow@?$ArrayOf@U?$IntType@E$00@OT@@U12@@OT@@QEBA_NPEAUhb_sanitize_context_t@@@Z 000000018006bb00 f i hb-ot-font.obj
 0001:0006ac50       ?sanitize_shallow@?$ArrayOf@UEncoding1_Range@CFF@@U?$IntType@E$00@OT@@@OT@@QEBA_NPEAUhb_sanitize_context_t@@@Z 000000018006bc50 f i hb-ot-font.obj
 0001:0006adb0       ?sentinel@?$FDSelect3_4@U?$IntType@G$01@OT@@U?$IntType@E$00@2@@CFF@@QEBAAEBU?$IntType@G$01@OT@@XZ 000000018006bdb0 f i hb-ot-font.obj
 0001:0006adf0       ?sentinel@?$FDSelect3_4@U?$IntType@I$03@OT@@U?$IntType@G$01@2@@CFF@@QEBAAEBU?$IntType@I$03@OT@@XZ 000000018006bdf0 f i hb-ot-font.obj
 0001:0006ae50       ?static_get_color_stops@?$ColorLine@UNoVariable@OT@@@OT@@SAIPEAUhb_color_line_t@@PEAXIPEAIPEAUhb_color_stop_t@@1@Z 000000018006be50 f i hb-ot-font.obj
 0001:0006af50       ?static_get_color_stops@?$ColorLine@UVariable@OT@@@OT@@SAIPEAUhb_color_line_t@@PEAXIPEAIPEAUhb_color_stop_t@@1@Z 000000018006bf50 f i hb-ot-font.obj
 0001:0006b060       ?static_get_extend@?$ColorLine@UNoVariable@OT@@@OT@@SA?AW4hb_paint_extend_t@@PEAUhb_color_line_t@@PEAX1@Z 000000018006c060 f i hb-ot-font.obj
 0001:0006b060       ?static_get_extend@?$ColorLine@UVariable@OT@@@OT@@SA?AW4hb_paint_extend_t@@PEAUhb_color_line_t@@PEAX1@Z 000000018006c060 f i hb-ot-font.obj
 0001:0006b070       hb_ot_font_set_funcs       000000018006c070 f   hb-ot-font.obj
 0001:0006b240       ??$apply@UGPOSProxy@@@hb_ot_map_t@@QEBAXAEBUGPOSProxy@@PEBUhb_ot_shape_plan_t@@PEAUhb_font_t@@PEAUhb_buffer_t@@@Z 000000018006c240 f i hb-ot-layout.obj
 0001:0006b780       ??$apply@UGSUBProxy@@@hb_ot_map_t@@QEBAXAEBUGSUBProxy@@PEBUhb_ot_shape_plan_t@@PEAUhb_font_t@@PEAUhb_buffer_t@@@Z 000000018006c780 f i hb-ot-layout.obj
 0001:0006bd90       ??$apply_cached_to@U?$AlternateSubstFormat1_2@USmallTypes@Layout@OT@@@GSUB_impl@Layout@OT@@@hb_accelerate_subtables_context_t@OT@@SA_NPEBXPEAUhb_ot_apply_context_t@1@@Z 000000018006cd90 f i hb-ot-layout.obj
 0001:0006bd90       ??$apply_to@U?$AlternateSubstFormat1_2@USmallTypes@Layout@OT@@@GSUB_impl@Layout@OT@@@hb_accelerate_subtables_context_t@OT@@SA_NPEBXPEAUhb_ot_apply_context_t@1@@Z 000000018006cd90 f i hb-ot-layout.obj
 0001:0006bda0       ??$apply_to@U?$ChainContextFormat1_4@USmallTypes@Layout@OT@@@OT@@@hb_accelerate_subtables_context_t@OT@@SA_NPEBXPEAUhb_ot_apply_context_t@1@@Z 000000018006cda0 f i hb-ot-layout.obj
 0001:0006bda0       ??$apply_cached_to@U?$ChainContextFormat1_4@USmallTypes@Layout@OT@@@OT@@@hb_accelerate_subtables_context_t@OT@@SA_NPEBXPEAUhb_ot_apply_context_t@1@@Z 000000018006cda0 f i hb-ot-layout.obj
 0001:0006bdb0       ??$apply_cached_to@U?$ChainContextFormat2_5@USmallTypes@Layout@OT@@@OT@@@hb_accelerate_subtables_context_t@OT@@SA_NPEBXPEAUhb_ot_apply_context_t@1@@Z 000000018006cdb0 f i hb-ot-layout.obj
 0001:0006bdc0       ??$apply_cached_to@U?$ContextFormat1_4@USmallTypes@Layout@OT@@@OT@@@hb_accelerate_subtables_context_t@OT@@SA_NPEBXPEAUhb_ot_apply_context_t@1@@Z 000000018006cdc0 f i hb-ot-layout.obj
 0001:0006bdc0       ??$apply_to@U?$ContextFormat1_4@USmallTypes@Layout@OT@@@OT@@@hb_accelerate_subtables_context_t@OT@@SA_NPEBXPEAUhb_ot_apply_context_t@1@@Z 000000018006cdc0 f i hb-ot-layout.obj
 0001:0006bdd0       ??$apply_cached_to@U?$ContextFormat2_5@USmallTypes@Layout@OT@@@OT@@@hb_accelerate_subtables_context_t@OT@@SA_NPEBXPEAUhb_ot_apply_context_t@1@@Z 000000018006cdd0 f i hb-ot-layout.obj
 0001:0006bde0       ??$apply_cached_to@U?$LigatureSubstFormat1_2@USmallTypes@Layout@OT@@@GSUB_impl@Layout@OT@@@hb_accelerate_subtables_context_t@OT@@SA_NPEBXPEAUhb_ot_apply_context_t@1@@Z 000000018006cde0 f i hb-ot-layout.obj
 0001:0006bdf0       ??$apply_to@U?$MarkBasePosFormat1_2@USmallTypes@Layout@OT@@@GPOS_impl@Layout@OT@@@hb_accelerate_subtables_context_t@OT@@SA_NPEBXPEAUhb_ot_apply_context_t@1@@Z 000000018006cdf0 f i hb-ot-layout.obj
 0001:0006bdf0       ??$apply_cached_to@U?$MarkBasePosFormat1_2@USmallTypes@Layout@OT@@@GPOS_impl@Layout@OT@@@hb_accelerate_subtables_context_t@OT@@SA_NPEBXPEAUhb_ot_apply_context_t@1@@Z 000000018006cdf0 f i hb-ot-layout.obj
 0001:0006be00       ??$apply_to@U?$MarkLigPosFormat1_2@USmallTypes@Layout@OT@@@GPOS_impl@Layout@OT@@@hb_accelerate_subtables_context_t@OT@@SA_NPEBXPEAUhb_ot_apply_context_t@1@@Z 000000018006ce00 f i hb-ot-layout.obj
 0001:0006be00       ??$apply_cached_to@U?$MarkLigPosFormat1_2@USmallTypes@Layout@OT@@@GPOS_impl@Layout@OT@@@hb_accelerate_subtables_context_t@OT@@SA_NPEBXPEAUhb_ot_apply_context_t@1@@Z 000000018006ce00 f i hb-ot-layout.obj
 0001:0006be10       ??$apply_cached_to@U?$MarkMarkPosFormat1_2@USmallTypes@Layout@OT@@@GPOS_impl@Layout@OT@@@hb_accelerate_subtables_context_t@OT@@SA_NPEBXPEAUhb_ot_apply_context_t@1@@Z 000000018006ce10 f i hb-ot-layout.obj
 0001:0006be10       ??$apply_to@U?$MarkMarkPosFormat1_2@USmallTypes@Layout@OT@@@GPOS_impl@Layout@OT@@@hb_accelerate_subtables_context_t@OT@@SA_NPEBXPEAUhb_ot_apply_context_t@1@@Z 000000018006ce10 f i hb-ot-layout.obj
 0001:0006be20       ??$apply_to@U?$MultipleSubstFormat1_2@USmallTypes@Layout@OT@@@GSUB_impl@Layout@OT@@@hb_accelerate_subtables_context_t@OT@@SA_NPEBXPEAUhb_ot_apply_context_t@1@@Z 000000018006ce20 f i hb-ot-layout.obj
 0001:0006be20       ??$apply_cached_to@U?$MultipleSubstFormat1_2@USmallTypes@Layout@OT@@@GSUB_impl@Layout@OT@@@hb_accelerate_subtables_context_t@OT@@SA_NPEBXPEAUhb_ot_apply_context_t@1@@Z 000000018006ce20 f i hb-ot-layout.obj
 0001:0006be30       ??$apply_cached_to@U?$PairPosFormat1_3@USmallTypes@Layout@OT@@@GPOS_impl@Layout@OT@@@hb_accelerate_subtables_context_t@OT@@SA_NPEBXPEAUhb_ot_apply_context_t@1@@Z 000000018006ce30 f i hb-ot-layout.obj
 0001:0006be40       ??$apply_cached_to@U?$PairPosFormat2_4@USmallTypes@Layout@OT@@@GPOS_impl@Layout@OT@@@hb_accelerate_subtables_context_t@OT@@SA_NPEBXPEAUhb_ot_apply_context_t@1@@Z 000000018006ce40 f i hb-ot-layout.obj
 0001:0006be50       ??$apply_to@U?$SingleSubstFormat1_3@USmallTypes@Layout@OT@@@GSUB_impl@Layout@OT@@@hb_accelerate_subtables_context_t@OT@@SA_NPEBXPEAUhb_ot_apply_context_t@1@@Z 000000018006ce50 f i hb-ot-layout.obj
 0001:0006be50       ??$apply_cached_to@U?$SingleSubstFormat1_3@USmallTypes@Layout@OT@@@GSUB_impl@Layout@OT@@@hb_accelerate_subtables_context_t@OT@@SA_NPEBXPEAUhb_ot_apply_context_t@1@@Z 000000018006ce50 f i hb-ot-layout.obj
 0001:0006be60       ??$apply_to@U?$SingleSubstFormat2_4@USmallTypes@Layout@OT@@@GSUB_impl@Layout@OT@@@hb_accelerate_subtables_context_t@OT@@SA_NPEBXPEAUhb_ot_apply_context_t@1@@Z 000000018006ce60 f i hb-ot-layout.obj
 0001:0006be60       ??$apply_cached_to@U?$SingleSubstFormat2_4@USmallTypes@Layout@OT@@@GSUB_impl@Layout@OT@@@hb_accelerate_subtables_context_t@OT@@SA_NPEBXPEAUhb_ot_apply_context_t@1@@Z 000000018006ce60 f i hb-ot-layout.obj
 0001:0006be70       ??$apply_cached_to@UChainContextFormat3@OT@@@hb_accelerate_subtables_context_t@OT@@SA_NPEBXPEAUhb_ot_apply_context_t@1@@Z 000000018006ce70 f i hb-ot-layout.obj
 0001:0006be70       ??$apply_to@UChainContextFormat3@OT@@@hb_accelerate_subtables_context_t@OT@@SA_NPEBXPEAUhb_ot_apply_context_t@1@@Z 000000018006ce70 f i hb-ot-layout.obj
 0001:0006be80       ??$apply_cached_to@UContextFormat3@OT@@@hb_accelerate_subtables_context_t@OT@@SA_NPEBXPEAUhb_ot_apply_context_t@1@@Z 000000018006ce80 f i hb-ot-layout.obj
 0001:0006be80       ??$apply_to@UContextFormat3@OT@@@hb_accelerate_subtables_context_t@OT@@SA_NPEBXPEAUhb_ot_apply_context_t@1@@Z 000000018006ce80 f i hb-ot-layout.obj
 0001:0006be90       ??$apply_to@UCursivePosFormat1@GPOS_impl@Layout@OT@@@hb_accelerate_subtables_context_t@OT@@SA_NPEBXPEAUhb_ot_apply_context_t@1@@Z 000000018006ce90 f i hb-ot-layout.obj
 0001:0006be90       ??$apply_cached_to@UCursivePosFormat1@GPOS_impl@Layout@OT@@@hb_accelerate_subtables_context_t@OT@@SA_NPEBXPEAUhb_ot_apply_context_t@1@@Z 000000018006ce90 f i hb-ot-layout.obj
 0001:0006bea0       ??$apply_cached_to@UReverseChainSingleSubstFormat1@GSUB_impl@Layout@OT@@@hb_accelerate_subtables_context_t@OT@@SA_NPEBXPEAUhb_ot_apply_context_t@1@@Z 000000018006cea0 f i hb-ot-layout.obj
 0001:0006bea0       ??$apply_to@UReverseChainSingleSubstFormat1@GSUB_impl@Layout@OT@@@hb_accelerate_subtables_context_t@OT@@SA_NPEBXPEAUhb_ot_apply_context_t@1@@Z 000000018006cea0 f i hb-ot-layout.obj
 0001:0006beb0       ??$apply_to@USinglePosFormat1@GPOS_impl@Layout@OT@@@hb_accelerate_subtables_context_t@OT@@SA_NPEBXPEAUhb_ot_apply_context_t@1@@Z 000000018006ceb0 f i hb-ot-layout.obj
 0001:0006beb0       ??$apply_cached_to@USinglePosFormat1@GPOS_impl@Layout@OT@@@hb_accelerate_subtables_context_t@OT@@SA_NPEBXPEAUhb_ot_apply_context_t@1@@Z 000000018006ceb0 f i hb-ot-layout.obj
 0001:0006bec0       ??$apply_cached_to@USinglePosFormat2@GPOS_impl@Layout@OT@@@hb_accelerate_subtables_context_t@OT@@SA_NPEBXPEAUhb_ot_apply_context_t@1@@Z 000000018006cec0 f i hb-ot-layout.obj
 0001:0006bec0       ??$apply_to@USinglePosFormat2@GPOS_impl@Layout@OT@@@hb_accelerate_subtables_context_t@OT@@SA_NPEBXPEAUhb_ot_apply_context_t@1@@Z 000000018006cec0 f i hb-ot-layout.obj
 0001:0006c050       ??$apply_to@U?$ChainContextFormat2_5@USmallTypes@Layout@OT@@@OT@@@hb_accelerate_subtables_context_t@OT@@SA_NPEBXPEAUhb_ot_apply_context_t@1@@Z 000000018006d050 f i hb-ot-layout.obj
 0001:0006c060       ??$apply_to@U?$ContextFormat2_5@USmallTypes@Layout@OT@@@OT@@@hb_accelerate_subtables_context_t@OT@@SA_NPEBXPEAUhb_ot_apply_context_t@1@@Z 000000018006d060 f i hb-ot-layout.obj
 0001:0006c070       ??$apply_to@U?$LigatureSubstFormat1_2@USmallTypes@Layout@OT@@@GSUB_impl@Layout@OT@@@hb_accelerate_subtables_context_t@OT@@SA_NPEBXPEAUhb_ot_apply_context_t@1@@Z 000000018006d070 f i hb-ot-layout.obj
 0001:0006c080       ??$apply_to@U?$PairPosFormat1_3@USmallTypes@Layout@OT@@@GPOS_impl@Layout@OT@@@hb_accelerate_subtables_context_t@OT@@SA_NPEBXPEAUhb_ot_apply_context_t@1@@Z 000000018006d080 f i hb-ot-layout.obj
 0001:0006c090       ??$apply_to@U?$PairPosFormat2_4@USmallTypes@Layout@OT@@@GPOS_impl@Layout@OT@@@hb_accelerate_subtables_context_t@OT@@SA_NPEBXPEAUhb_ot_apply_context_t@1@@Z 000000018006d090 f i hb-ot-layout.obj
 0001:0006c0a0       ??$cache_func_to@U?$ContextFormat2_5@USmallTypes@Layout@OT@@@OT@@@hb_accelerate_subtables_context_t@OT@@SAPEAXPEAXW4hb_ot_lookup_cache_op_t@1@@Z 000000018006d0a0 f i hb-ot-layout.obj
 0001:0006c0a0       ??$cache_func_to@U?$ChainContextFormat2_5@USmallTypes@Layout@OT@@@OT@@@hb_accelerate_subtables_context_t@OT@@SAPEAXPEAXW4hb_ot_lookup_cache_op_t@1@@Z 000000018006d0a0 f i hb-ot-layout.obj
 0001:0006c130       ??$cache_func_to@U?$LigatureSubstFormat1_2@USmallTypes@Layout@OT@@@GSUB_impl@Layout@OT@@@hb_accelerate_subtables_context_t@OT@@SAPEAXPEAXW4hb_ot_lookup_cache_op_t@1@@Z 000000018006d130 f i hb-ot-layout.obj
 0001:0006c130       ??$cache_func_to@U?$PairPosFormat1_3@USmallTypes@Layout@OT@@@GPOS_impl@Layout@OT@@@hb_accelerate_subtables_context_t@OT@@SAPEAXPEAXW4hb_ot_lookup_cache_op_t@1@@Z 000000018006d130 f i hb-ot-layout.obj
 0001:0006c1a0       ??$cache_func_to@U?$PairPosFormat2_4@USmallTypes@Layout@OT@@@GPOS_impl@Layout@OT@@@hb_accelerate_subtables_context_t@OT@@SAPEAXPEAXW4hb_ot_lookup_cache_op_t@1@@Z 000000018006d1a0 f i hb-ot-layout.obj
 0001:0006c250       ??$collect_coverage@Uhb_set_digest_t@@@Coverage@Common@Layout@OT@@QEBA_NPEAUhb_set_digest_t@@@Z 000000018006d250 f i hb-ot-layout.obj
 0001:0006c310       ??$collect_glyphs@Uhb_bit_set_t@@@?$ClassTable@U?$IntType@G$01@OT@@@AAT@@QEBAXAEAUhb_bit_set_t@@I@Z 000000018006d310 f i hb-ot-layout.obj
 0001:0006c400       ??$collect_glyphs@Uhb_bit_set_t@@@?$KernSubTable@UKernAATSubTableHeader@OT@@@OT@@QEBAXAEAUhb_bit_set_t@@0I@Z 000000018006d400 f i hb-ot-layout.obj
 0001:0006c650       ??$collect_glyphs@Uhb_bit_set_t@@@?$KernSubTable@UKernOTSubTableHeader@OT@@@OT@@QEBAXAEAUhb_bit_set_t@@0I@Z 000000018006d650 f i hb-ot-layout.obj
 0001:0006c8b0       ??$create@UPosLookup@GPOS_impl@Layout@OT@@@hb_ot_layout_lookup_accelerator_t@OT@@SAPEAU01@AEBUPosLookup@GPOS_impl@Layout@1@@Z 000000018006d8b0 f i hb-ot-layout.obj
 0001:0006cad0       ??$create@USubstLookup@GSUB_impl@Layout@OT@@@hb_ot_layout_lookup_accelerator_t@OT@@SAPEAU01@AEBUSubstLookup@GSUB_impl@Layout@1@@Z 000000018006dad0 f i hb-ot-layout.obj
 0001:0006ccf0       ??$dispatch@U?$ClassTable@U?$IntType@G$01@OT@@@AAT@@$$V@hb_sanitize_context_t@@QEAA_NAEBU?$ClassTable@U?$IntType@G$01@OT@@@AAT@@@Z 000000018006dcf0 f i hb-ot-layout.obj
 0001:0006cdb0       ??$dispatch@U?$ContextFormat2_5@USmallTypes@Layout@OT@@@OT@@@hb_accelerate_subtables_context_t@OT@@QEAA?AUhb_empty_t@@AEBU?$ContextFormat2_5@USmallTypes@Layout@OT@@@1@@Z 000000018006ddb0 f i hb-ot-layout.obj
 0001:0006cef0       ??$dispatch@U?$LigatureSubstFormat1_2@USmallTypes@Layout@OT@@@GSUB_impl@Layout@OT@@@hb_accelerate_subtables_context_t@OT@@QEAA?AUhb_empty_t@@AEBU?$LigatureSubstFormat1_2@USmallTypes@Layout@OT@@@GSUB_impl@Layout@1@@Z 000000018006def0 f i hb-ot-layout.obj
 0001:0006d020       ??$dispatch@U?$List16OfOffsetTo@UPosLookup@GPOS_impl@Layout@OT@@U?$IntType@G$01@4@@OT@@$$V@hb_sanitize_context_t@@QEAA_NAEBU?$List16OfOffsetTo@UPosLookup@GPOS_impl@Layout@OT@@U?$IntType@G$01@4@@OT@@@Z 000000018006e020 f i hb-ot-layout.obj
 0001:0006d100       ??$dispatch@U?$PairPosFormat1_3@USmallTypes@Layout@OT@@@GPOS_impl@Layout@OT@@@hb_accelerate_subtables_context_t@OT@@QEAA?AUhb_empty_t@@AEBU?$PairPosFormat1_3@USmallTypes@Layout@OT@@@GPOS_impl@Layout@1@@Z 000000018006e100 f i hb-ot-layout.obj
 0001:0006d230       ??$dispatch@ULigatureArray@GPOS_impl@Layout@OT@@I@hb_sanitize_context_t@@QEAA_NAEBULigatureArray@GPOS_impl@Layout@OT@@$$QEAI@Z 000000018006e230 f i hb-ot-layout.obj
 0001:0006d320       ??$dispatch@UMarkArray@GPOS_impl@Layout@OT@@$$V@hb_sanitize_context_t@@QEAA_NAEBUMarkArray@GPOS_impl@Layout@OT@@@Z 000000018006e320 f i hb-ot-layout.obj
 0001:0006d4a0       ??$dispatch@Uhb_aat_apply_context_t@AAT@@$$V@?$KernSubTable@UKernAATSubTableHeader@OT@@@OT@@QEBA_NPEAUhb_aat_apply_context_t@AAT@@@Z 000000018006e4a0 f i hb-ot-layout.obj
 0001:0006d660       ??$dispatch@Uhb_aat_apply_context_t@AAT@@$$V@?$KernSubTable@UKernOTSubTableHeader@OT@@@OT@@QEBA_NPEAUhb_aat_apply_context_t@AAT@@@Z 000000018006e660 f i hb-ot-layout.obj
 0001:0006d820       ??$dispatch@Uhb_accelerate_subtables_context_t@OT@@$$V@ChainContext@OT@@QEBA?AUhb_empty_t@@PEAUhb_accelerate_subtables_context_t@1@@Z 000000018006e820 f i hb-ot-layout.obj
 0001:0006da40       ??$dispatch@Uhb_accelerate_subtables_context_t@OT@@$$V@Context@OT@@QEBA?AUhb_empty_t@@PEAUhb_accelerate_subtables_context_t@1@@Z 000000018006ea40 f i hb-ot-layout.obj
 0001:0006dbb0       ??$dispatch@Uhb_accelerate_subtables_context_t@OT@@$$V@PosLookupSubTable@GPOS_impl@Layout@OT@@QEBA?AUhb_empty_t@@PEAUhb_accelerate_subtables_context_t@3@I@Z 000000018006ebb0 f i hb-ot-layout.obj
 0001:0006dff0       ??$dispatch@Uhb_accelerate_subtables_context_t@OT@@$$V@SubstLookupSubTable@GSUB_impl@Layout@OT@@QEBA?AUhb_empty_t@@PEAUhb_accelerate_subtables_context_t@3@I@Z 000000018006eff0 f i hb-ot-layout.obj
 0001:0006e310       ??$dispatch@Uhb_sanitize_context_t@@$$V@?$Extension@UExtensionPos@GPOS_impl@Layout@OT@@@OT@@QEBA_NPEAUhb_sanitize_context_t@@@Z 000000018006f310 f i hb-ot-layout.obj
 0001:0006e4c0       ??$dispatch@Uhb_sanitize_context_t@@$$V@?$KernSubTable@UKernAATSubTableHeader@OT@@@OT@@QEBA_NPEAUhb_sanitize_context_t@@@Z 000000018006f4c0 f i hb-ot-layout.obj
 0001:0006e740       ??$dispatch@Uhb_sanitize_context_t@@$$V@?$KernSubTable@UKernOTSubTableHeader@OT@@@OT@@QEBA_NPEAUhb_sanitize_context_t@@@Z 000000018006f740 f i hb-ot-layout.obj
 0001:0006e9c0       ??$dispatch@Uhb_sanitize_context_t@@$$V@PosLookupSubTable@GPOS_impl@Layout@OT@@QEBA_NPEAUhb_sanitize_context_t@@I@Z 000000018006f9c0 f i hb-ot-layout.obj
 0001:0006ee80       ??$dispatch@Uhb_would_apply_context_t@OT@@$$V@ChainContext@OT@@QEBA_NPEAUhb_would_apply_context_t@1@@Z 000000018006fe80 f i hb-ot-layout.obj
 0001:0006f180       ??$dispatch@Uhb_would_apply_context_t@OT@@$$V@Context@OT@@QEBA_NPEAUhb_would_apply_context_t@1@@Z 0000000180070180 f i hb-ot-layout.obj
 0001:0006f390       ??$dispatch@Uhb_would_apply_context_t@OT@@$$V@SubstLookupSubTable@GSUB_impl@Layout@OT@@QEBA_NPEAUhb_would_apply_context_t@3@I@Z 0000000180070390 f i hb-ot-layout.obj
 0001:0006f5c0       ??$dispatch_recurse_func@Uhb_ot_apply_context_t@OT@@@PosLookup@GPOS_impl@Layout@OT@@SA_NPEAUhb_ot_apply_context_t@3@I@Z 00000001800705c0 f i hb-ot-layout.obj
 0001:0006f7a0       ??$dispatch_recurse_func@Uhb_ot_apply_context_t@OT@@@SubstLookup@GSUB_impl@Layout@OT@@SA_NPEAUhb_ot_apply_context_t@3@I@Z 00000001800707a0 f i hb-ot-layout.obj
 0001:0006f980       ??$drive@Udriver_context_t@?$KerxSubTableFormat1@UKernAATSubTableHeader@OT@@@AAT@@@?$StateTableDriver@UObsoleteTypes@AAT@@XW4Flags@?$KerxSubTableFormat1@UKernAATSubTableHeader@OT@@@2@@AAT@@QEAAXPEAUdriver_context_t@?$KerxSubTableFormat1@UKernAATSubTableHeader@OT@@@1@PEAUhb_aat_apply_context_t@1@@Z 0000000180070980 f i hb-ot-layout.obj
 0001:0006fd70       ??$drive@Udriver_context_t@?$KerxSubTableFormat1@UKernOTSubTableHeader@OT@@@AAT@@@?$StateTableDriver@UObsoleteTypes@AAT@@XW4Flags@?$KerxSubTableFormat1@UKernOTSubTableHeader@OT@@@2@@AAT@@QEAAXPEAUdriver_context_t@?$KerxSubTableFormat1@UKernOTSubTableHeader@OT@@@1@PEAUhb_aat_apply_context_t@1@@Z 0000000180070d70 f i hb-ot-layout.obj
 0001:00070160       ??$evaluate@UItemVarStoreInstancer@OT@@@Condition@OT@@QEBA_NPEBHIPEAUItemVarStoreInstancer@1@@Z 0000000180071160 f i hb-ot-layout.obj
 0001:00070480       ??$sanitize@UPosLookup@GPOS_impl@Layout@OT@@@?$GSUBGPOSVersion1_2@USmallTypes@Layout@OT@@@OT@@QEBA_NPEAUhb_sanitize_context_t@@@Z 0000000180071480 f i hb-ot-layout.obj
 0001:00070630       ??$sanitize@UPosLookupSubTable@GPOS_impl@Layout@OT@@@Lookup@OT@@QEBA_NPEAUhb_sanitize_context_t@@@Z 0000000180071630 f i hb-ot-layout.obj
 0001:00070890       ??$sanitize_blob@UGPOS@Layout@OT@@@hb_sanitize_context_t@@QEAAPEAUhb_blob_t@@PEAU1@@Z 0000000180071890 f i hb-ot-layout.obj
 0001:00070ab0       ??$sanitize_blob@Ukern@OT@@@hb_sanitize_context_t@@QEAAPEAUhb_blob_t@@PEAU1@@Z 0000000180071ab0 f i hb-ot-layout.obj
 0001:00070d90       ??0accelerator_t@kern@OT@@QEAA@PEAUhb_face_t@@@Z 0000000180071d90 f i hb-ot-layout.obj
 0001:00070fb0       ?_apply@?$ChainContextFormat2_5@USmallTypes@Layout@OT@@@OT@@QEBA_NPEAUhb_ot_apply_context_t@2@_N@Z 0000000180071fb0 f i hb-ot-layout.obj
 0001:000711c0       ?_apply@?$ContextFormat2_5@USmallTypes@Layout@OT@@@OT@@QEBA_NPEAUhb_ot_apply_context_t@2@_N@Z 00000001800721c0 f i hb-ot-layout.obj
 0001:00071350       ?_apply@?$LigatureSubstFormat1_2@USmallTypes@Layout@OT@@@GSUB_impl@Layout@OT@@QEBA_NPEAUhb_ot_apply_context_t@4@_N@Z 0000000180072350 f i hb-ot-layout.obj
 0001:000714e0       ?_apply@?$PairPosFormat1_3@USmallTypes@Layout@OT@@@GPOS_impl@Layout@OT@@QEBA_NPEAUhb_ot_apply_context_t@4@_N@Z 00000001800724e0 f i hb-ot-layout.obj
 0001:00071820       ?_apply@?$PairPosFormat2_4@USmallTypes@Layout@OT@@@GPOS_impl@Layout@OT@@QEBA_NPEAUhb_ot_apply_context_t@4@_N@Z 0000000180072820 f i hb-ot-layout.obj
 0001:00072060       ?_set_glyph_class@hb_ot_apply_context_t@OT@@QEAAXII_N0@Z 0000000180073060 f i hb-ot-layout.obj
 0001:00072180       ?_set_glyph_flags@hb_buffer_t@@QEAAXIII_N0@Z 0000000180073180 f i hb-ot-layout.obj
 0001:00072330       ?apply@?$AlternateSet@USmallTypes@Layout@OT@@@GSUB_impl@Layout@OT@@QEBA_NPEAUhb_ot_apply_context_t@4@@Z 0000000180073330 f i hb-ot-layout.obj
 0001:000724c0       ?apply@?$AlternateSubstFormat1_2@USmallTypes@Layout@OT@@@GSUB_impl@Layout@OT@@QEBA_NPEAUhb_ot_apply_context_t@4@@Z 00000001800734c0 f i hb-ot-layout.obj
 0001:000725d0       ?apply@?$ChainContextFormat1_4@USmallTypes@Layout@OT@@@OT@@QEBA_NPEAUhb_ot_apply_context_t@2@@Z 00000001800735d0 f i hb-ot-layout.obj
 0001:00072710       ?apply@?$ChainRule@USmallTypes@Layout@OT@@@OT@@QEBA_NPEAUhb_ot_apply_context_t@2@AEBUChainContextApplyLookupContext@2@@Z 0000000180073710 f i hb-ot-layout.obj
 0001:000730d0       ?apply@?$ChainRuleSet@USmallTypes@Layout@OT@@@OT@@QEBA_NPEAUhb_ot_apply_context_t@2@AEBUChainContextApplyLookupContext@2@@Z 00000001800740d0 f i hb-ot-layout.obj
 0001:00073b80       ?apply@?$ContextFormat1_4@USmallTypes@Layout@OT@@@OT@@QEBA_NPEAUhb_ot_apply_context_t@2@@Z 0000000180074b80 f i hb-ot-layout.obj
 0001:00073ca0       ?apply@?$KerxTable@UKernAAT@OT@@@AAT@@QEBA_NPEAUhb_aat_apply_context_t@2@AEBUkern_accelerator_data_t@2@@Z 0000000180074ca0 f i hb-ot-layout.obj
 0001:000740e0       ?apply@?$KerxTable@UKernOT@OT@@@AAT@@QEBA_NPEAUhb_aat_apply_context_t@2@AEBUkern_accelerator_data_t@2@@Z 00000001800750e0 f i hb-ot-layout.obj
 0001:000744c0       ?apply@?$Ligature@USmallTypes@Layout@OT@@@GSUB_impl@Layout@OT@@QEBA_NPEAUhb_ot_apply_context_t@4@@Z 00000001800754c0 f i hb-ot-layout.obj
 0001:00074b90       ?apply@?$LigatureSet@USmallTypes@Layout@OT@@@GSUB_impl@Layout@OT@@QEBA_NPEAUhb_ot_apply_context_t@4@@Z 0000000180075b90 f i hb-ot-layout.obj
 0001:00075020       ?apply@?$MarkBasePosFormat1_2@USmallTypes@Layout@OT@@@GPOS_impl@Layout@OT@@QEBA_NPEAUhb_ot_apply_context_t@4@@Z 0000000180076020 f i hb-ot-layout.obj
 0001:000755a0       ?apply@?$MarkLigPosFormat1_2@USmallTypes@Layout@OT@@@GPOS_impl@Layout@OT@@QEBA_NPEAUhb_ot_apply_context_t@4@@Z 00000001800765a0 f i hb-ot-layout.obj
 0001:00075b70       ?apply@?$MarkMarkPosFormat1_2@USmallTypes@Layout@OT@@@GPOS_impl@Layout@OT@@QEBA_NPEAUhb_ot_apply_context_t@4@@Z 0000000180076b70 f i hb-ot-layout.obj
 0001:000761e0       ?apply@?$MultipleSubstFormat1_2@USmallTypes@Layout@OT@@@GSUB_impl@Layout@OT@@QEBA_NPEAUhb_ot_apply_context_t@4@@Z 00000001800771e0 f i hb-ot-layout.obj
 0001:000762f0       ?apply@?$PairSet@USmallTypes@Layout@OT@@@GPOS_impl@Layout@OT@@QEBA_NPEAUhb_ot_apply_context_t@4@PEBUValueFormat@234@I@Z 00000001800772f0 f i hb-ot-layout.obj
 0001:00076620       ?apply@?$Rule@USmallTypes@Layout@OT@@@OT@@QEBA_NPEAUhb_ot_apply_context_t@2@AEBUContextApplyLookupContext@2@@Z 0000000180077620 f i hb-ot-layout.obj
 0001:00076af0       ?apply@?$RuleSet@USmallTypes@Layout@OT@@@OT@@QEBA_NPEAUhb_ot_apply_context_t@2@AEBUContextApplyLookupContext@2@@Z 0000000180077af0 f i hb-ot-layout.obj
 0001:00077440       ?apply@?$Sequence@USmallTypes@Layout@OT@@@GSUB_impl@Layout@OT@@QEBA_NPEAUhb_ot_apply_context_t@4@@Z 0000000180078440 f i hb-ot-layout.obj
 0001:000777d0       ?apply@?$SingleSubstFormat1_3@USmallTypes@Layout@OT@@@GSUB_impl@Layout@OT@@QEBA_NPEAUhb_ot_apply_context_t@4@@Z 00000001800787d0 f i hb-ot-layout.obj
 0001:00077910       ?apply@?$SingleSubstFormat2_4@USmallTypes@Layout@OT@@@GSUB_impl@Layout@OT@@QEBA_NPEAUhb_ot_apply_context_t@4@@Z 0000000180078910 f i hb-ot-layout.obj
 0001:00077a80       ?apply@ChainContextFormat3@OT@@QEBA_NPEAUhb_ot_apply_context_t@2@@Z 0000000180078a80 f i hb-ot-layout.obj
 0001:00078520       ?apply@ContextFormat3@OT@@QEBA_NPEAUhb_ot_apply_context_t@2@@Z 0000000180079520 f i hb-ot-layout.obj
 0001:00078aa0       ?apply@CursivePosFormat1@GPOS_impl@Layout@OT@@QEBA_NPEAUhb_ot_apply_context_t@4@@Z 0000000180079aa0 f i hb-ot-layout.obj
 0001:00079530       ?apply@MarkArray@GPOS_impl@Layout@OT@@QEBA_NPEAUhb_ot_apply_context_t@4@IIAEBUAnchorMatrix@234@II@Z 000000018007a530 f i hb-ot-layout.obj
 0001:000799d0       ?apply@ReverseChainSingleSubstFormat1@GSUB_impl@Layout@OT@@QEBA_NPEAUhb_ot_apply_context_t@4@@Z 000000018007a9d0 f i hb-ot-layout.obj
 0001:0007a070       ?apply@SinglePosFormat1@GPOS_impl@Layout@OT@@QEBA_NPEAUhb_ot_apply_context_t@4@@Z 000000018007b070 f i hb-ot-layout.obj
 0001:0007a1a0       ?apply@SinglePosFormat2@GPOS_impl@Layout@OT@@QEBA_NPEAUhb_ot_apply_context_t@4@@Z 000000018007b1a0 f i hb-ot-layout.obj
 0001:0007ad80       ?apply_value@ValueFormat@GPOS_impl@Layout@OT@@QEBA_NPEAUhb_ot_apply_context_t@4@PEBUValueBase@234@PEBU?$IntType@G$01@4@AEAUhb_glyph_position_t@@@Z 000000018007bd80 f i hb-ot-layout.obj
 0001:0007b260       ?cache_cost@?$PairPosFormat2_4@USmallTypes@Layout@OT@@@GPOS_impl@Layout@OT@@QEBAIXZ 000000018007c260 f i hb-ot-layout.obj
 0001:0007b3a0       ?create_accelerator_data@?$KerxTable@UKernAAT@OT@@@AAT@@QEBA?AUkern_accelerator_data_t@2@I@Z 000000018007c3a0 f i hb-ot-layout.obj
 0001:0007b790       ?create_accelerator_data@?$KerxTable@UKernOT@OT@@@AAT@@QEBA?AUkern_accelerator_data_t@2@I@Z 000000018007c790 f i hb-ot-layout.obj
 0001:0007bb40       ?find_lang_sys_index@Script@OT@@QEBA_NIPEAI@Z 000000018007cb40 f i hb-ot-layout.obj
 0001:0007bc10       ?find_script_index@GSUBGPOS@OT@@QEBA_NIPEAI@Z 000000018007cc10 f i hb-ot-layout.obj
 0001:0007bd20       ?find_variations_index@GSUBGPOS@OT@@QEBA_NPEBHIPEAIPEAUItemVarStoreInstancer@2@@Z 000000018007cd20 f i hb-ot-layout.obj
 0001:0007bf10       ?get@?$hb_lazy_loader_t@Ukern_accelerator_t@OT@@U?$hb_face_lazy_loader_t@Ukern_accelerator_t@OT@@$0BH@@@Uhb_face_t@@$0BH@U12@@@QEBAPEBUkern_accelerator_t@OT@@XZ 000000018007cf10 f i hb-ot-layout.obj
 0001:0007bfc0       ?get_accel@?$accelerator_t@UGPOS@Layout@OT@@@GSUBGPOS@OT@@QEBAPEAUhb_ot_layout_lookup_accelerator_t@3@I@Z 000000018007cfc0 f i hb-ot-layout.obj
 0001:0007c090       ?get_accel@?$accelerator_t@UGSUB@Layout@OT@@@GSUBGPOS@OT@@QEBAPEAUhb_ot_layout_lookup_accelerator_t@3@I@Z 000000018007d090 f i hb-ot-layout.obj
 0001:0007c160       ?get_anchor@AnchorFormat2@GPOS_impl@Layout@OT@@QEBAXPEAUhb_ot_apply_context_t@4@IPEAM1@Z 000000018007d160 f i hb-ot-layout.obj
 0001:0007c3d0       ?get_anchor@AnchorFormat3@GPOS_impl@Layout@OT@@QEBAXPEAUhb_ot_apply_context_t@4@IPEAM1@Z 000000018007d3d0 f i hb-ot-layout.obj
 0001:0007c600       ?get_class@ClassDef@OT@@QEBAIIPEAU?$hb_cache_t@$0P@$07$06$00@@@Z 000000018007d600 f i hb-ot-layout.obj
 0001:0007c6a0       ?get_coverage@ChainContextFormat3@OT@@QEBAAEBUCoverage@Common@Layout@2@XZ 000000018007d6a0 f i hb-ot-layout.obj
 0001:0007c710       ?get_delta@HintingDevice@OT@@AEBAHIH@Z 000000018007d710 f i hb-ot-layout.obj
 0001:0007c830       ?get_feature@GSUBGPOS@OT@@QEBAAEBUFeature@2@I@Z 000000018007d830 f i hb-ot-layout.obj
 0001:0007c8f0       ?get_feature_tag@GSUBGPOS@OT@@QEBAII@Z 000000018007d8f0 f i hb-ot-layout.obj
 0001:0007c990       ?get_feature_variation@GSUBGPOS@OT@@QEBAAEBUFeature@2@II@Z 000000018007d990 f i hb-ot-layout.obj
 0001:0007cb10       ?get_glyph_props@accelerator_t@GDEF@OT@@QEBAII@Z 000000018007db10 f i hb-ot-layout.obj
 0001:0007cd00       ?get_indexes@IndexArray@OT@@QEBAIIPEAI0@Z 000000018007dd00 f i hb-ot-layout.obj
 0001:0007ce20       ?get_kerning@?$KerxSubTableFormat0@UKernAATSubTableHeader@OT@@@AAT@@QEBAHIIPEAUhb_aat_apply_context_t@2@@Z 000000018007de20 f i hb-ot-layout.obj
 0001:0007cef0       ?get_kerning@?$KerxSubTableFormat0@UKernOTSubTableHeader@OT@@@AAT@@QEBAHIIPEAUhb_aat_apply_context_t@2@@Z 000000018007def0 f i hb-ot-layout.obj
 0001:0007cfc0       ?get_kerning@?$KerxSubTableFormat2@UKernAATSubTableHeader@OT@@@AAT@@QEBAHIIPEAUhb_aat_apply_context_t@2@@Z 000000018007dfc0 f i hb-ot-layout.obj
 0001:0007d150       ?get_kerning@?$KerxSubTableFormat2@UKernOTSubTableHeader@OT@@@AAT@@QEBAHIIPEAUhb_aat_apply_context_t@2@@Z 000000018007e150 f i hb-ot-layout.obj
 0001:0007d2e0       ?get_lang_sys@Script@OT@@QEBAAEBULangSys@2@I@Z 000000018007e2e0 f i hb-ot-layout.obj
 0001:0007d370       ?get_lookup@GSUBGPOS@OT@@QEBAAEBULookup@2@I@Z 000000018007e370 f i hb-ot-layout.obj
 0001:0007d420       ?get_script@GSUBGPOS@OT@@QEBAAEBUScript@2@I@Z 000000018007e420 f i hb-ot-layout.obj
 0001:0007d4d0       ?get_stored@?$hb_lazy_loader_t@UGPOS_accelerator_t@OT@@U?$hb_face_lazy_loader_t@UGPOS_accelerator_t@OT@@$0BK@@@Uhb_face_t@@$0BK@U12@@@QEBAPEAUGPOS_accelerator_t@OT@@XZ 000000018007e4d0 f i hb-ot-layout.obj
 0001:0007d6f0       ?get_stored@?$hb_lazy_loader_t@UGSUB_accelerator_t@OT@@U?$hb_face_lazy_loader_t@UGSUB_accelerator_t@OT@@$0BJ@@@Uhb_face_t@@$0BJ@U12@@@QEBAPEAUGSUB_accelerator_t@OT@@XZ 000000018007e6f0 f i hb-ot-layout.obj
 0001:0007d910       ?get_x_delta@Device@OT@@QEBAHPEAUhb_font_t@@AEBUItemVariationStore@2@PEAU?$hb_atomic_t@H@@@Z 000000018007e910 f i hb-ot-layout.obj
 0001:0007d9d0       ?get_y_delta@Device@OT@@QEBAHPEAUhb_font_t@@AEBUItemVariationStore@2@PEAU?$hb_atomic_t@H@@@Z 000000018007e9d0 f i hb-ot-layout.obj
 0001:0007da90       ?hb_ot_layout_has_cross_kerning@@YA_NPEAUhb_face_t@@@Z 000000018007ea90 f   hb-ot-layout.obj
 0001:0007db90       ?hb_ot_layout_has_kerning@@YA_NPEAUhb_face_t@@@Z 000000018007eb90 f   hb-ot-layout.obj
 0001:0007dbf0       ?hb_ot_layout_has_machine_kerning@@YA_NPEAUhb_face_t@@@Z 000000018007ebf0 f   hb-ot-layout.obj
 0001:0007dcf0       ?hb_ot_layout_kern@@YAXPEBUhb_ot_shape_plan_t@@PEAUhb_font_t@@PEAUhb_buffer_t@@@Z 000000018007ecf0 f   hb-ot-layout.obj
 0001:0007de60       ?hb_ot_layout_position_finish_offsets@@YAXPEAUhb_font_t@@PEAUhb_buffer_t@@@Z 000000018007ee60 f   hb-ot-layout.obj
 0001:0007de70       ?hb_ot_layout_position_start@@YAXPEAUhb_font_t@@PEAUhb_buffer_t@@@Z 000000018007ee70 f   hb-ot-layout.obj
 0001:0007deb0       ?hb_ot_layout_substitute_lookup@@YAXPEAUhb_ot_apply_context_t@OT@@AEBUSubstLookup@GSUB_impl@Layout@2@AEBUhb_ot_layout_lookup_accelerator_t@2@@Z 000000018007eeb0 f   hb-ot-layout.obj
 0001:0007dec0       ?hb_ot_layout_substitute_start@@YAXPEAUhb_font_t@@PEAUhb_buffer_t@@@Z 000000018007eec0 f   hb-ot-layout.obj
 0001:0007ded0       ?hb_ot_layout_table_find_feature@@YA_NPEAUhb_face_t@@IIPEAI@Z 000000018007eed0 f   hb-ot-layout.obj
 0001:0007e020       ?is_blocklisted@GDEF@OT@@QEBA_NPEAUhb_blob_t@@PEAUhb_face_t@@@Z 000000018007f020 f   hb-ot-layout.obj
 0001:0007e380       ?is_blocklisted@GSUB@Layout@OT@@QEBA_NPEAUhb_blob_t@@PEAUhb_face_t@@@Z 000000018007f380 f   hb-ot-layout.obj
 0001:0007e390       ?kern@?$hb_kern_machine_t@U?$KernSubTableFormat3@UKernAATSubTableHeader@OT@@@OT@@@OT@@QEBAXPEAUhb_font_t@@PEAUhb_buffer_t@@I_N@Z 000000018007f390 f i hb-ot-layout.obj
 0001:0007e910       ?kern@?$hb_kern_machine_t@U?$KernSubTableFormat3@UKernOTSubTableHeader@OT@@@OT@@@OT@@QEBAXPEAUhb_font_t@@PEAUhb_buffer_t@@I_N@Z 000000018007f910 f i hb-ot-layout.obj
 0001:0007ee90       ?kern@?$hb_kern_machine_t@Uaccelerator_t@?$KerxSubTableFormat0@UKernAATSubTableHeader@OT@@@AAT@@@OT@@QEBAXPEAUhb_font_t@@PEAUhb_buffer_t@@I_N@Z 000000018007fe90 f i hb-ot-layout.obj
 0001:0007f370       ?kern@?$hb_kern_machine_t@Uaccelerator_t@?$KerxSubTableFormat0@UKernOTSubTableHeader@OT@@@AAT@@@OT@@QEBAXPEAUhb_font_t@@PEAUhb_buffer_t@@I_N@Z 0000000180080370 f i hb-ot-layout.obj
 0001:0007f850       ?kern@?$hb_kern_machine_t@Uaccelerator_t@?$KerxSubTableFormat2@UKernAATSubTableHeader@OT@@@AAT@@@OT@@QEBAXPEAUhb_font_t@@PEAUhb_buffer_t@@I_N@Z 0000000180080850 f i hb-ot-layout.obj
 0001:0007fd30       ?kern@?$hb_kern_machine_t@Uaccelerator_t@?$KerxSubTableFormat2@UKernOTSubTableHeader@OT@@@AAT@@@OT@@QEBAXPEAUhb_font_t@@PEAUhb_buffer_t@@I_N@Z 0000000180080d30 f i hb-ot-layout.obj
 0001:000805c0       __vcrt_initialize          00000001800815c0 f   MSVCRT:ucrt_stubs.obj
 0001:000805c0       __scrt_stub_for_acrt_thread_detach 00000001800815c0 f   MSVCRT:ucrt_stubs.obj
 0001:000805c0       __acrt_uninitialize_critical 00000001800815c0 f   MSVCRT:ucrt_stubs.obj
 0001:000805c0       __acrt_thread_attach       00000001800815c0 f   MSVCRT:ucrt_stubs.obj
 0001:000805c0       __scrt_stub_for_acrt_uninitialize_critical 00000001800815c0 f   MSVCRT:ucrt_stubs.obj
 0001:000805c0       __acrt_initialize          00000001800815c0 f   MSVCRT:ucrt_stubs.obj
 0001:000805c0       __vcrt_thread_detach       00000001800815c0 f   MSVCRT:ucrt_stubs.obj
 0001:000805c0       __vcrt_uninitialize_critical 00000001800815c0 f   MSVCRT:ucrt_stubs.obj
 0001:000805c0       __scrt_stub_for_acrt_uninitialize 00000001800815c0 f   MSVCRT:ucrt_stubs.obj
 0001:000805c0       __vcrt_thread_attach       00000001800815c0 f   MSVCRT:ucrt_stubs.obj
 0001:000805c0       __scrt_stub_for_acrt_thread_attach 00000001800815c0 f   MSVCRT:ucrt_stubs.obj
 0001:000805c0       __vcrt_uninitialize        00000001800815c0 f   MSVCRT:ucrt_stubs.obj
 0001:000805c0       __acrt_uninitialize        00000001800815c0 f   MSVCRT:ucrt_stubs.obj
 0001:000805c0       __acrt_thread_detach       00000001800815c0 f   MSVCRT:ucrt_stubs.obj
 0001:000805c0       __scrt_stub_for_acrt_initialize 00000001800815c0 f   MSVCRT:ucrt_stubs.obj
 0001:00080780       ?position@hb_ot_map_t@@QEBAXPEBUhb_ot_shape_plan_t@@PEAUhb_font_t@@PEAUhb_buffer_t@@@Z 0000000180081780 f   hb-ot-layout.obj
 0001:00080860       ?position_finish_offsets@GPOS@Layout@OT@@SAXPEAUhb_font_t@@PEAUhb_buffer_t@@@Z 0000000180081860 f i hb-ot-layout.obj
 0001:00080a80       ?process_@hb_bit_set_t@@QEAAXP6A?AU?$hb_vector_size_t@_K$0EA@@@AEBU2@0@Z_N2AEBU1@@Z 0000000180081a80 f i hb-ot-layout.obj
 0001:000814a0       ?sanitize@?$KerxSubTableFormat2@UKernAATSubTableHeader@OT@@@AAT@@QEBA_NPEAUhb_sanitize_context_t@@@Z 00000001800824a0 f i hb-ot-layout.obj
 0001:00081680       ?sanitize@?$KerxSubTableFormat2@UKernOTSubTableHeader@OT@@@AAT@@QEBA_NPEAUhb_sanitize_context_t@@@Z 0000000180082680 f i hb-ot-layout.obj
 0001:00081860       ?sanitize@?$KerxTable@UKernAAT@OT@@@AAT@@QEBA_NPEAUhb_sanitize_context_t@@@Z 0000000180082860 f i hb-ot-layout.obj
 0001:00081c80       ?sanitize@?$KerxTable@UKernOT@OT@@@AAT@@QEBA_NPEAUhb_sanitize_context_t@@@Z 0000000180082c80 f i hb-ot-layout.obj
 0001:00082020       ?sanitize@?$MarkMarkPosFormat1_2@USmallTypes@Layout@OT@@@GPOS_impl@Layout@OT@@QEBA_NPEAUhb_sanitize_context_t@@@Z 0000000180083020 f i hb-ot-layout.obj
 0001:00082020       ?sanitize@?$MarkBasePosFormat1_2@USmallTypes@Layout@OT@@@GPOS_impl@Layout@OT@@QEBA_NPEAUhb_sanitize_context_t@@@Z 0000000180083020 f i hb-ot-layout.obj
 0001:00082240       ?sanitize@?$MarkLigPosFormat1_2@USmallTypes@Layout@OT@@@GPOS_impl@Layout@OT@@QEBA_NPEAUhb_sanitize_context_t@@@Z 0000000180083240 f i hb-ot-layout.obj
 0001:00082450       ?sanitize@?$PairPosFormat1_3@USmallTypes@Layout@OT@@@GPOS_impl@Layout@OT@@QEBA_NPEAUhb_sanitize_context_t@@@Z 0000000180083450 f i hb-ot-layout.obj
 0001:000826d0       ?sanitize@?$PairPosFormat2_4@USmallTypes@Layout@OT@@@GPOS_impl@Layout@OT@@QEBA_NPEAUhb_sanitize_context_t@@@Z 00000001800836d0 f i hb-ot-layout.obj
 0001:00082a70       ?sanitize@?$PairSet@USmallTypes@Layout@OT@@@GPOS_impl@Layout@OT@@QEBA_NPEAUhb_sanitize_context_t@@PEBUsanitize_closure_t@1234@@Z 0000000180083a70 f i hb-ot-layout.obj
 0001:00082c60       ?sanitize@Anchor@GPOS_impl@Layout@OT@@QEBA_NPEAUhb_sanitize_context_t@@@Z 0000000180083c60 f i hb-ot-layout.obj
 0001:00082ec0       ?sanitize@AnchorMatrix@GPOS_impl@Layout@OT@@QEBA_NPEAUhb_sanitize_context_t@@I@Z 0000000180083ec0 f i hb-ot-layout.obj
 0001:000830e0       ?sanitize@CursivePosFormat1@GPOS_impl@Layout@OT@@QEBA_NPEAUhb_sanitize_context_t@@@Z 00000001800840e0 f i hb-ot-layout.obj
 0001:00083290       ?sanitize@GPOS@Layout@OT@@QEBA_NPEAUhb_sanitize_context_t@@@Z 0000000180084290 f i hb-ot-layout.obj
 0001:00083360       ?sanitize@SinglePosFormat1@GPOS_impl@Layout@OT@@QEBA_NPEAUhb_sanitize_context_t@@@Z 0000000180084360 f i hb-ot-layout.obj
 0001:000835e0       ?sanitize@SinglePosFormat2@GPOS_impl@Layout@OT@@QEBA_NPEAUhb_sanitize_context_t@@@Z 00000001800845e0 f i hb-ot-layout.obj
 0001:00083790       ?sanitize@kern@OT@@QEBA_NPEAUhb_sanitize_context_t@@@Z 0000000180084790 f i hb-ot-layout.obj
 0001:00083880       ?sanitize_shallow@?$ArrayOf@UKernPair@AAT@@U?$BinSearchHeader@U?$IntType@G$01@OT@@@OT@@@OT@@QEBA_NPEAUhb_sanitize_context_t@@@Z 0000000180084880 f i hb-ot-layout.obj
 0001:000839f0       ?sanitize_value_devices@ValueFormat@GPOS_impl@Layout@OT@@AEBA_NPEAUhb_sanitize_context_t@@PEBUValueBase@234@PEBU?$IntType@G$01@4@@Z 00000001800849f0 f i hb-ot-layout.obj
 0001:00083bd0       ?sanitize_values_stride_unsafe@ValueFormat@GPOS_impl@Layout@OT@@QEBA_NPEAUhb_sanitize_context_t@@PEBUValueBase@234@PEBU?$IntType@G$01@4@II@Z 0000000180084bd0 f i hb-ot-layout.obj
 0001:00083e10       ?substitute@hb_ot_map_t@@QEBAXPEBUhb_ot_shape_plan_t@@PEAUhb_font_t@@PEAUhb_buffer_t@@@Z 0000000180084e10 f   hb-ot-layout.obj
 0001:00083ef0       ?transition@driver_context_t@?$KerxSubTableFormat1@UKernAATSubTableHeader@OT@@@AAT@@QEAAXPEAUhb_buffer_t@@PEAU?$StateTableDriver@UObsoleteTypes@AAT@@XW4Flags@?$KerxSubTableFormat1@UKernAATSubTableHeader@OT@@@2@@3@AEBU?$Entry@X@3@@Z 0000000180084ef0 f i hb-ot-layout.obj
 0001:000841a0       ?transition@driver_context_t@?$KerxSubTableFormat1@UKernOTSubTableHeader@OT@@@AAT@@QEAAXPEAUhb_buffer_t@@PEAU?$StateTableDriver@UObsoleteTypes@AAT@@XW4Flags@?$KerxSubTableFormat1@UKernOTSubTableHeader@OT@@@2@@3@AEBU?$Entry@X@3@@Z 00000001800851a0 f i hb-ot-layout.obj
 0001:00084450       ?would_apply@?$ChainRuleSet@USmallTypes@Layout@OT@@@OT@@QEBA_NPEAUhb_would_apply_context_t@2@AEBUChainContextApplyLookupContext@2@@Z 0000000180085450 f i hb-ot-layout.obj
 0001:00084600       ?would_apply@?$LigatureSubstFormat1_2@USmallTypes@Layout@OT@@@GSUB_impl@Layout@OT@@QEBA_NPEAUhb_would_apply_context_t@4@@Z 0000000180085600 f i hb-ot-layout.obj
 0001:00084840       ?would_apply@?$RuleSet@USmallTypes@Layout@OT@@@OT@@QEBA_NPEAUhb_would_apply_context_t@2@AEBUContextApplyLookupContext@2@@Z 0000000180085840 f i hb-ot-layout.obj
 0001:00084990       hb_ot_layout_collect_features_map 0000000180085990 f   hb-ot-layout.obj
 0001:00084b10       hb_ot_layout_feature_with_variations_get_lookups 0000000180085b10 f   hb-ot-layout.obj
 0001:00084b60       hb_ot_layout_has_glyph_classes 0000000180085b60 f   hb-ot-layout.obj
 0001:00084bd0       hb_ot_layout_has_positioning 0000000180085bd0 f   hb-ot-layout.obj
 0001:00084c30       hb_ot_layout_has_substitution 0000000180085c30 f   hb-ot-layout.obj
 0001:00084c90       hb_ot_layout_language_find_feature 0000000180085c90 f   hb-ot-layout.obj
 0001:00084e20       hb_ot_layout_language_get_required_feature 0000000180085e20 f   hb-ot-layout.obj
 0001:00084ee0       hb_ot_layout_lookup_would_substitute 0000000180085ee0 f   hb-ot-layout.obj
 0001:000850b0       hb_ot_layout_script_select_language 00000001800860b0 f   hb-ot-layout.obj
 0001:000851e0       hb_ot_layout_table_find_feature_variations 00000001800861e0 f   hb-ot-layout.obj
 0001:00085310       hb_ot_layout_table_get_lookup_count 0000000180086310 f   hb-ot-layout.obj
 0001:00085380       hb_ot_layout_table_select_script 0000000180086380 f   hb-ot-layout.obj
 0001:00085570       ??0hb_ot_map_builder_t@@QEAA@PEAUhb_face_t@@AEBUhb_segment_properties_t@@@Z 0000000180086570 f   hb-ot-map.obj
 0001:000856e0       ??1hb_ot_map_builder_t@@QEAA@XZ 00000001800866e0 f   hb-ot-map.obj
 0001:000857c0       ?add_feature@hb_ot_map_builder_t@@QEAAXIW4hb_ot_map_feature_flags_t@@I@Z 00000001800867c0 f   hb-ot-map.obj
 0001:00085930       ?add_lookups@hb_ot_map_builder_t@@AEAAXAEAUhb_ot_map_t@@IIII_N111I@Z 0000000180086930 f   hb-ot-map.obj
 0001:00085bd0       ?add_pause@hb_ot_map_builder_t@@AEAAXIP6A_NPEBUhb_ot_shape_plan_t@@PEAUhb_font_t@@PEAUhb_buffer_t@@@Z@Z 0000000180086bd0 f   hb-ot-map.obj
 0001:00085cf0       ?alloc@?$hb_vector_t@Ufeature_info_t@hb_ot_map_builder_t@@$0A@@@QEAA_NI_N@Z 0000000180086cf0 f i hb-ot-map.obj
 0001:00085db0       ?alloc@?$hb_vector_t@Ulookup_map_t@hb_ot_map_t@@$0A@@@QEAA_NI_N@Z 0000000180086db0 f i hb-ot-map.obj
 0001:00085db0       ?alloc@?$hb_vector_t@Uhb_outline_point_t@@$0A@@@QEAA_NI_N@Z 0000000180086db0 f i hb-outline.obj
 0001:00085e70       ?cmp@feature_info_t@hb_ot_map_builder_t@@SAHPEBX0@Z 0000000180086e70 f i hb-ot-map.obj
 0001:00085ea0       ?cmp@feature_map_t@hb_ot_map_t@@SAHPEBX0@Z 0000000180086ea0 f i hb-ot-map.obj
 0001:00085ec0       ?cmp@lookup_map_t@hb_ot_map_t@@SAHPEBX0@Z 0000000180086ec0 f i hb-ot-map.obj
 0001:00085ee0       ?compile@hb_ot_map_builder_t@@QEAAXAEAUhb_ot_map_t@@AEBUhb_ot_shape_plan_key_t@@@Z 0000000180086ee0 f   hb-ot-map.obj
 0001:00086a70       ?has_feature@hb_ot_map_builder_t@@QEAA_NI@Z 0000000180087a70 f   hb-ot-map.obj
 0001:00086af0       ??$sanitize_blob@UMVAR@OT@@@hb_sanitize_context_t@@QEAAPEAUhb_blob_t@@PEAU1@@Z 0000000180087af0 f i hb-ot-metrics.obj
 0001:00086e10       ??C?$hb_lazy_loader_t@UOS2@OT@@U?$hb_table_lazy_loader_t@UOS2@OT@@$05$00@@Uhb_face_t@@$05Uhb_blob_t@@@@QEBAPEBUOS2@OT@@XZ 0000000180087e10 f i hb-ot-metrics.obj
 0001:00086fb0       ?_hb_ot_metrics_get_position_common@@YA_NPEAUhb_font_t@@W4hb_ot_metrics_tag_t@@PEAH@Z 0000000180087fb0 f   hb-ot-metrics.obj
 0001:00087460       ?get@?$hb_lazy_loader_t@UMVAR@OT@@U?$hb_table_lazy_loader_t@UMVAR@OT@@$0BG@$00@@Uhb_face_t@@$0BG@Uhb_blob_t@@@@QEBAPEBUMVAR@OT@@XZ 0000000180088460 f i hb-ot-metrics.obj
 0001:000875d0       ?get_var@MVAR@OT@@QEBAMIPEBHI@Z 00000001800885d0 f i hb-ot-metrics.obj
 0001:00087700       ?sanitize@MVAR@OT@@QEBA_NPEAUhb_sanitize_context_t@@@Z 0000000180088700 f i hb-ot-metrics.obj
 0001:000878d0       ?_hb_ot_shape_fallback_kern@@YAXPEBUhb_ot_shape_plan_t@@PEAUhb_font_t@@PEAUhb_buffer_t@@@Z 00000001800888d0 f   hb-ot-shape-fallback.obj
 0001:000879c0       ?_hb_ot_shape_fallback_mark_position@@YAXPEBUhb_ot_shape_plan_t@@PEAUhb_font_t@@PEAUhb_buffer_t@@_N@Z 00000001800889c0 f   hb-ot-shape-fallback.obj
 0001:00087ac0       ?_hb_ot_shape_fallback_mark_position_recategorize_marks@@YAXPEBUhb_ot_shape_plan_t@@PEAUhb_font_t@@PEAUhb_buffer_t@@@Z 0000000180088ac0 f   hb-ot-shape-fallback.obj
 0001:00087d50       ?_hb_ot_shape_fallback_spaces@@YAXPEBUhb_ot_shape_plan_t@@PEAUhb_font_t@@PEAUhb_buffer_t@@@Z 0000000180088d50 f   hb-ot-shape-fallback.obj
 0001:000880f0       ?kern@?$hb_kern_machine_t@Uhb_ot_shape_fallback_kern_driver_t@@@OT@@QEBAXPEAUhb_font_t@@PEAUhb_buffer_t@@I_N@Z 00000001800890f0 f i hb-ot-shape-fallback.obj
 0001:00088fd0       ?_hb_ot_shape_normalize@@YAXPEBUhb_ot_shape_plan_t@@PEAUhb_buffer_t@@PEAUhb_font_t@@@Z 0000000180089fd0 f   hb-ot-shape-normalize.obj
 0001:00089ac0       ?compose_unicode@hb_ot_shape_normalize_context_t@@SA_NPEBU1@IIPEAI@Z 000000018008aac0 f i hb-ot-shape-normalize.obj
 0001:0008a010       ?decompose_unicode@hb_ot_shape_normalize_context_t@@SA_NPEBU1@IPEAI1@Z 000000018008b010 f i hb-ot-shape-normalize.obj
 0001:0008a550       ??$dispatch@UAxisValueOffsetArray@OT@@AEBU?$IntType@G$01@2@PEBU12@@hb_sanitize_context_t@@QEAA_NAEBUAxisValueOffsetArray@OT@@AEBU?$IntType@G$01@2@$$QEAPEBU12@@Z 000000018008b550 f i hb-ot-shape.obj
 0001:0008a640       ??$sanitize_blob@USTAT@OT@@@hb_sanitize_context_t@@QEAAPEAUhb_blob_t@@PEAU1@@Z 000000018008b640 f i hb-ot-shape.obj
 0001:0008a990       ?compile@hb_ot_shape_planner_t@@QEAAXAEAUhb_ot_shape_plan_t@@AEBUhb_ot_shape_plan_key_t@@@Z 000000018008b990 f   hb-ot-shape.obj
 0001:0008b020       ?fini@hb_ot_map_t@@QEAAXXZ 000000018008c020 f i hb-ot-shape.obj
 0001:0008b0b0       ?fini@hb_ot_shape_plan_t@@QEAAXXZ 000000018008c0b0 f   hb-ot-shape.obj
 0001:0008b0e0       ?has_glyph@hb_font_t@@QEAA_NI@Z 000000018008c0e0 f i hb-ot-shape.obj
 0001:0008d490       ?init0@hb_ot_shape_plan_t@@QEAA_NPEAUhb_face_t@@PEBUhb_shape_plan_key_t@@@Z 000000018008e490 f   hb-ot-shape.obj
 0001:0008d680       ?sanitize@AxisValue@OT@@QEBA_NPEAUhb_sanitize_context_t@@@Z 000000018008e680 f i hb-ot-shape.obj
 0001:0008d860       ?sanitize@STAT@OT@@QEBA_NPEAUhb_sanitize_context_t@@@Z 000000018008e860 f i hb-ot-shape.obj
 0001:0008dac0       _hb_ot_shape               000000018008eac0 f   hb-ot-shape.obj
 0001:0008db10       _hb_ot_shaper_font_data_create 000000018008eb10 f   hb-ot-shape.obj
 0001:0008dd00       _hb_ot_shaper_font_data_destroy 000000018008ed00 f   hb-ot-shape.obj
 0001:0008e040       ?data_create_arabic@@YAPEAXPEBUhb_ot_shape_plan_t@@@Z 000000018008f040 f   hb-ot-shaper-arabic.obj
 0001:0008e210       ?data_destroy_arabic@@YAXPEAX@Z 000000018008f210 f   hb-ot-shaper-arabic.obj
 0001:0008e3e0       ??$add_link@U?$OffsetTo@U?$Ligature@USmallTypes@Layout@OT@@@GSUB_impl@Layout@OT@@U?$IntType@G$01@4@X$00@OT@@@hb_serialize_context_t@@QEAAXAEAU?$OffsetTo@U?$Ligature@USmallTypes@Layout@OT@@@GSUB_impl@Layout@OT@@U?$IntType@G$01@4@X$00@OT@@IW4whence_t@0@I@Z 000000018008f3e0 f i hb-ot-shaper-arabic.obj
 0001:0008e3e0       ??$add_link@U?$OffsetTo@U?$LigatureSet@USmallTypes@Layout@OT@@@GSUB_impl@Layout@OT@@U?$IntType@G$01@4@X$00@OT@@@hb_serialize_context_t@@QEAAXAEAU?$OffsetTo@U?$LigatureSet@USmallTypes@Layout@OT@@@GSUB_impl@Layout@OT@@U?$IntType@G$01@4@X$00@OT@@IW4whence_t@0@I@Z 000000018008f3e0 f i hb-ot-shaper-arabic.obj
 0001:0008e3e0       ??$add_link@U?$OffsetTo@UCoverage@Common@Layout@OT@@U?$IntType@G$01@4@X$00@OT@@@hb_serialize_context_t@@QEAAXAEAU?$OffsetTo@UCoverage@Common@Layout@OT@@U?$IntType@G$01@4@X$00@OT@@IW4whence_t@0@I@Z 000000018008f3e0 f i hb-ot-shaper-arabic.obj
 0001:0008f780       ??$extend@ULookup@OT@@$$V@hb_serialize_context_t@@QEAAPEAULookup@OT@@PEAU12@@Z 0000000180090780 f i hb-ot-shaper-arabic.obj
 0001:0008f840       ??$extend_min@U?$Ligature@USmallTypes@Layout@OT@@@GSUB_impl@Layout@OT@@@hb_serialize_context_t@@QEAAPEAU?$Ligature@USmallTypes@Layout@OT@@@GSUB_impl@Layout@OT@@PEAU1234@@Z 0000000180090840 f i hb-ot-shaper-arabic.obj
 0001:0008f840       ??$extend_min@U?$CoverageFormat2_4@USmallTypes@Layout@OT@@@Common@Layout@OT@@@hb_serialize_context_t@@QEAAPEAU?$CoverageFormat2_4@USmallTypes@Layout@OT@@@Common@Layout@OT@@PEAU1234@@Z 0000000180090840 f i hb-ot-shaper-arabic.obj
 0001:0008f8f0       ??$extend_min@U?$IntType@G$01@OT@@@hb_serialize_context_t@@QEAAPEAU?$IntType@G$01@OT@@AEAU12@@Z 00000001800908f0 f i hb-ot-shaper-arabic.obj
 0001:0008f8f0       ??$extend_min@U?$LigatureSet@USmallTypes@Layout@OT@@@GSUB_impl@Layout@OT@@@hb_serialize_context_t@@QEAAPEAU?$LigatureSet@USmallTypes@Layout@OT@@@GSUB_impl@Layout@OT@@PEAU1234@@Z 00000001800908f0 f i hb-ot-shaper-arabic.obj
 0001:0008f8f0       ??$extend_min@UCoverage@Common@Layout@OT@@@hb_serialize_context_t@@QEAAPEAUCoverage@Common@Layout@OT@@PEAU1234@@Z 00000001800908f0 f i hb-ot-shaper-arabic.obj
 0001:0008f9a0       ??$extend_min@U?$SingleSubstFormat1_3@USmallTypes@Layout@OT@@@GSUB_impl@Layout@OT@@@hb_serialize_context_t@@QEAAPEAU?$SingleSubstFormat1_3@USmallTypes@Layout@OT@@@GSUB_impl@Layout@OT@@PEAU1234@@Z 00000001800909a0 f i hb-ot-shaper-arabic.obj
 0001:0008f9a0       ??$extend_min@U?$LigatureSubstFormat1_2@USmallTypes@Layout@OT@@@GSUB_impl@Layout@OT@@@hb_serialize_context_t@@QEAAPEAU?$LigatureSubstFormat1_2@USmallTypes@Layout@OT@@@GSUB_impl@Layout@OT@@PEAU1234@@Z 00000001800909a0 f i hb-ot-shaper-arabic.obj
 0001:0008f9a0       ??$extend_min@U?$SingleSubstFormat2_4@USmallTypes@Layout@OT@@@GSUB_impl@Layout@OT@@@hb_serialize_context_t@@QEAAPEAU?$SingleSubstFormat2_4@USmallTypes@Layout@OT@@@GSUB_impl@Layout@OT@@PEAU1234@@Z 00000001800909a0 f i hb-ot-shaper-arabic.obj
 0001:0008f9a0       ??$extend_min@ULookup@OT@@@hb_serialize_context_t@@QEAAPEAULookup@OT@@PEAU12@@Z 00000001800909a0 f i hb-ot-shaper-arabic.obj
 0001:0008fa50       ??$extend_size@U?$ArrayOf@UHBGlyphID16@OT@@U?$IntType@G$01@2@@OT@@@hb_serialize_context_t@@QEAAPEAU?$ArrayOf@UHBGlyphID16@OT@@U?$IntType@G$01@2@@OT@@PEAU12@_K_N@Z 0000000180090a50 f i hb-ot-shaper-arabic.obj
 0001:0008fa50       ??$extend_size@U?$HeadlessArrayOf@UHBGlyphID16@OT@@U?$IntType@G$01@2@@OT@@@hb_serialize_context_t@@QEAAPEAU?$HeadlessArrayOf@UHBGlyphID16@OT@@U?$IntType@G$01@2@@OT@@PEAU12@_K_N@Z 0000000180090a50 f i hb-ot-shaper-arabic.obj
 0001:0008fc20       ??$push@UCoverage@Common@Layout@OT@@@hb_serialize_context_t@@QEAAPEAUCoverage@Common@Layout@OT@@XZ 0000000180090c20 f i hb-ot-shaper-arabic.obj
 0001:000902e0       ??$serialize@U?$hb_sorted_array_t@$$CBUHBGlyphID16@OT@@@@$0A@@?$CoverageFormat2_4@USmallTypes@Layout@OT@@@Common@Layout@OT@@AEAA_NPEAUhb_serialize_context_t@@U?$hb_sorted_array_t@$$CBUHBGlyphID16@OT@@@@@Z 00000001800912e0 f i hb-ot-shaper-arabic.obj
 0001:00090480       ??$serialize@U?$hb_sorted_array_t@$$CBUHBGlyphID16@OT@@@@$0A@@Coverage@Common@Layout@OT@@QEAA_NPEAUhb_serialize_context_t@@U?$hb_sorted_array_t@$$CBUHBGlyphID16@OT@@@@@Z 0000000180091480 f i hb-ot-shaper-arabic.obj
 0001:000906a0       ??$serialize@U?$hb_zip_iter_t@U?$hb_sorted_array_t@UHBGlyphID16@OT@@@@U?$hb_array_t@UHBGlyphID16@OT@@@@@@$0A@@SingleSubst@GSUB_impl@Layout@OT@@QEAA_NPEAUhb_serialize_context_t@@U?$hb_zip_iter_t@U?$hb_sorted_array_t@UHBGlyphID16@OT@@@@U?$hb_array_t@UHBGlyphID16@OT@@@@@@@Z 00000001800916a0 f i hb-ot-shaper-arabic.obj
 0001:00090b80       ??$serialize_serialize@AEAU?$hb_sorted_array_t@$$CBUHBGlyphID16@OT@@@@@?$OffsetTo@UCoverage@Common@Layout@OT@@U?$IntType@G$01@4@X$00@OT@@QEAA_NPEAUhb_serialize_context_t@@AEAU?$hb_sorted_array_t@$$CBUHBGlyphID16@OT@@@@@Z 0000000180091b80 f i hb-ot-shaper-arabic.obj
 0001:00090c30       ??$start_serialize@USubstLookup@GSUB_impl@Layout@OT@@@hb_serialize_context_t@@QEAAPEAUSubstLookup@GSUB_impl@Layout@OT@@XZ 0000000180091c30 f i hb-ot-shaper-arabic.obj
 0001:000922a0       ?cmp@?$IntType@G$01@OT@@SAHPEBU12@0@Z 00000001800932a0 f i hb-ot-shaper-arabic.obj
 0001:000922e0       ?cmp_range@?$RangeRecord@USmallTypes@Layout@OT@@@Common@Layout@OT@@SAHPEBX0@Z 00000001800932e0 f i hb-ot-shaper-arabic.obj
 0001:000923a0       ?discard_stale_objects@hb_serialize_context_t@@QEAAXXZ 00000001800933a0 f i hb-ot-shaper-arabic.obj
 0001:00092610       ?end_serialize@hb_serialize_context_t@@QEAAXXZ 0000000180093610 f i hb-ot-shaper-arabic.obj
 0001:00092880       ?pop_discard@hb_serialize_context_t@@QEAAXXZ 0000000180093880 f i hb-ot-shaper-arabic.obj
 0001:00092900       ?push@?$hb_vector_t@Ulink_t@object_t@hb_serialize_context_t@@$0A@@@QEAAPEAUlink_t@object_t@hb_serialize_context_t@@XZ 0000000180093900 f i hb-ot-shaper-arabic.obj
 0001:00092a80       ?safe_to_insert_tatweel@hb_buffer_t@@QEAAXII@Z 0000000180093a80 f i hb-ot-shaper-arabic.obj
 0001:00092b10       ?serialize@?$ArrayOf@UHBGlyphID16@OT@@U?$IntType@G$01@2@@OT@@QEAA_NPEAUhb_serialize_context_t@@I_N@Z 0000000180093b10 f i hb-ot-shaper-arabic.obj
 0001:00092c20       ?serialize@?$HeadlessArrayOf@UHBGlyphID16@OT@@U?$IntType@G$01@2@@OT@@QEAA_NPEAUhb_serialize_context_t@@I_N@Z 0000000180093c20 f i hb-ot-shaper-arabic.obj
 0001:00092d40       ?serialize@?$LigatureSet@USmallTypes@Layout@OT@@@GSUB_impl@Layout@OT@@QEAA_NPEAUhb_serialize_context_t@@U?$hb_array_t@$$CBUHBGlyphID16@OT@@@@U?$hb_array_t@$$CBI@@AEAU6@@Z 0000000180093d40 f i hb-ot-shaper-arabic.obj
 0001:00093120       ?serialize@?$LigatureSubstFormat1_2@USmallTypes@Layout@OT@@@GSUB_impl@Layout@OT@@QEAA_NPEAUhb_serialize_context_t@@U?$hb_sorted_array_t@$$CBUHBGlyphID16@OT@@@@U?$hb_array_t@$$CBI@@U?$hb_array_t@$$CBUHBGlyphID16@OT@@@@23@Z 0000000180094120 f i hb-ot-shaper-arabic.obj
 0001:000934b0       ?serialize@?$SortedArrayOf@U?$RangeRecord@USmallTypes@Layout@OT@@@Common@Layout@OT@@U?$IntType@G$01@4@@OT@@QEAA_NPEAUhb_serialize_context_t@@I@Z 00000001800944b0 f i hb-ot-shaper-arabic.obj
 0001:00093600       ?serialize@Lookup@OT@@QEAA_NPEAUhb_serialize_context_t@@III@Z 0000000180094600 f i hb-ot-shaper-arabic.obj
 0001:00093800       ?setup_masks_arabic_plan@@YAXPEBUarabic_shape_plan_t@@PEAUhb_buffer_t@@W4hb_script_t@@@Z 0000000180094800 f   hb-ot-shaper-arabic.obj
 0001:000949d0       ?hb_indic_get_categories@@YAGI@Z 00000001800959d0 f   hb-ot-shaper-indic-table.obj
 0001:00095f40       ?find_syllables_indic@@YAXPEAUhb_buffer_t@@@Z 0000000180096f40 f i hb-ot-shaper-indic.obj
 0001:00096640       ?init@hb_indic_would_substitute_feature_t@@QEAAXPEBUhb_ot_map_t@@I_N@Z 0000000180097640 f i hb-ot-shaper-indic.obj
 0001:000978b0       ?would_substitute@hb_indic_would_substitute_feature_t@@QEBA_NPEBIIPEAUhb_face_t@@@Z 00000001800988b0 f i hb-ot-shaper-indic.obj
 0001:00097db0       ?find_syllables_khmer@@YAXPEAUhb_buffer_t@@@Z 0000000180098db0 f i hb-ot-shaper-khmer.obj
 0001:00098850       ?find_syllables_myanmar@@YAXPEAUhb_buffer_t@@@Z 0000000180099850 f i hb-ot-shaper-myanmar.obj
 0001:00099270       ?hb_syllabic_clear_var@@YA_NPEBUhb_ot_shape_plan_t@@PEAUhb_font_t@@PEAUhb_buffer_t@@@Z 000000018009a270 f   hb-ot-shaper-syllabic.obj
 0001:00099280       ?hb_syllabic_insert_dotted_circles@@YA_NPEAUhb_font_t@@PEAUhb_buffer_t@@IIHH@Z 000000018009a280 f   hb-ot-shaper-syllabic.obj
 0001:0009c960       ?_hb_preprocess_text_vowel_constraints@@YAXPEBUhb_ot_shape_plan_t@@PEAUhb_buffer_t@@PEAUhb_font_t@@@Z 000000018009d960 f   hb-ot-shaper-vowel-constraints.obj
 0001:000a0710       hb_ot_tag_to_language      00000001800a1710 f   hb-ot-tag.obj
 0001:000a0890       hb_ot_tags_from_script_and_language 00000001800a1890 f   hb-ot-tag.obj
 0001:000a0ec0       ??C?$hb_lazy_loader_t@Uavar@OT@@U?$hb_table_lazy_loader_t@Uavar@OT@@$0BD@$00@@Uhb_face_t@@$0BD@Uhb_blob_t@@@@QEBAPEBUavar@OT@@XZ 00000001800a1ec0 f i hb-ot-var.obj
 0001:000a1030       ?get_instance@fvar@OT@@QEBAPEBUInstanceRecord@2@I@Z 00000001800a2030 f i hb-ot-var.obj
 0001:000a10b0       ?map_coords@avar@OT@@QEBAXPEAHI@Z 00000001800a20b0 f i hb-ot-var.obj
 0001:000a1620       hb_ot_var_named_instance_get_design_coords 00000001800a2620 f   hb-ot-var.obj
 0001:000a1720       hb_ot_var_normalize_coords 00000001800a2720 f   hb-ot-var.obj
 0001:000a1970       ?control_area@hb_outline_t@@QEBAMXZ 00000001800a2970 f   hb-outline.obj
 0001:000a1bf0       ?embolden@hb_outline_t@@QEAAXMMMM@Z 00000001800a2bf0 f   hb-outline.obj
 0001:000a2330       ?hb_outline_recording_pen_get_funcs@@YAPEAUhb_draw_funcs_t@@XZ 00000001800a3330 f   hb-outline.obj
 0001:000a2640       ?replay@hb_outline_t@@QEBAXPEAUhb_draw_funcs_t@@PEAX@Z 00000001800a3640 f   hb-outline.obj
 0001:000a2bb0       ?slant@hb_outline_t@@QEAAXM@Z 00000001800a3bb0 f   hb-outline.obj
 0001:000a2bf0       ?hb_paint_bounded_get_funcs@@YAPEAUhb_paint_funcs_t@@XZ 00000001800a3bf0 f   hb-paint-bounded.obj
 0001:000a2ef0       ?hb_paint_extents_get_funcs@@YAPEAUhb_paint_funcs_t@@XZ 00000001800a3ef0 f   hb-paint-extents.obj
 0001:000a3480       ?intersect@hb_bounds_t@@QEAAXAEBU1@@Z 00000001800a4480 f i hb-paint-extents.obj
 0001:000a35a0       ?paint@hb_paint_extents_context_t@@QEAAXXZ 00000001800a45a0 f i hb-paint-extents.obj
 0001:000a3620       ?pop_group@hb_paint_extents_context_t@@QEAAXW4hb_paint_composite_mode_t@@@Z 00000001800a4620 f i hb-paint-extents.obj
 0001:000a3800       ?push_clip@hb_paint_extents_context_t@@QEAAXUhb_extents_t@@@Z 00000001800a4800 f i hb-paint-extents.obj
 0001:000a3940       ?transform_extents@hb_transform_t@@QEBAXAEAUhb_extents_t@@@Z 00000001800a4940 f i hb-paint-extents.obj
 0001:000a3b80       ?union_@hb_bounds_t@@QEAAXAEBU1@@Z 00000001800a4b80 f i hb-paint-extents.obj
 0001:000a3c50       hb_paint_funcs_create      00000001800a4c50 f   hb-paint.obj
 0001:000a3d10       hb_paint_funcs_destroy     00000001800a4d10 f   hb-paint.obj
 0001:000a3fb0       hb_paint_funcs_get_empty   00000001800a4fb0 f   hb-paint.obj
 0001:000a3fc0       hb_paint_funcs_set_color_func 00000001800a4fc0 f   hb-paint.obj
 0001:000a40f0       hb_paint_funcs_set_image_func 00000001800a50f0 f   hb-paint.obj
 0001:000a4220       hb_paint_funcs_set_linear_gradient_func 00000001800a5220 f   hb-paint.obj
 0001:000a4350       hb_paint_funcs_set_pop_clip_func 00000001800a5350 f   hb-paint.obj
 0001:000a4480       hb_paint_funcs_set_pop_group_func 00000001800a5480 f   hb-paint.obj
 0001:000a45b0       hb_paint_funcs_set_pop_transform_func 00000001800a55b0 f   hb-paint.obj
 0001:000a46e0       hb_paint_funcs_set_push_clip_glyph_func 00000001800a56e0 f   hb-paint.obj
 0001:000a4810       hb_paint_funcs_set_push_clip_rectangle_func 00000001800a5810 f   hb-paint.obj
 0001:000a4940       hb_paint_funcs_set_push_group_func 00000001800a5940 f   hb-paint.obj
 0001:000a4a70       hb_paint_funcs_set_push_transform_func 00000001800a5a70 f   hb-paint.obj
 0001:000a4ba0       hb_paint_funcs_set_radial_gradient_func 00000001800a5ba0 f   hb-paint.obj
 0001:000a4cd0       hb_paint_funcs_set_sweep_gradient_func 00000001800a5cd0 f   hb-paint.obj
 0001:000a4e00       hb_paint_pop_transform     00000001800a5e00 f   hb-paint.obj
 0001:000a4e20       hb_paint_push_transform    00000001800a5e20 f   hb-paint.obj
 0001:000a4e80       ??1?$hb_vector_t@U?$hb_vector_t@Urange_flags_t@hb_aat_map_t@@$00@@$0A@@@QEAA@XZ 00000001800a5e80 f i hb-shape-plan.obj
 0001:000a4f30       ??1hb_ot_map_t@@QEAA@XZ    00000001800a5f30 f i hb-shape-plan.obj
 0001:000a5190       ?init@hb_shape_plan_key_t@@QEAA_N_NPEAUhb_face_t@@PEBUhb_segment_properties_t@@PEBUhb_feature_t@@IPEBHIPEBQEBD@Z 00000001800a6190 f   hb-shape-plan.obj
 0001:000a54e0       hb_shape_plan_create2      00000001800a64e0 f   hb-shape-plan.obj
 0001:000a56b0       hb_shape_plan_create_cached2 00000001800a66b0 f   hb-shape-plan.obj
 0001:000a5c30       hb_shape_plan_destroy      00000001800a6c30 f   hb-shape-plan.obj
 0001:000a5cd0       hb_shape_plan_execute      00000001800a6cd0 f   hb-shape-plan.obj
 0001:000a5d00       hb_shape_full              00000001800a6d00 f   hb-shape.obj
 0001:000a5e50       ?_hb_shapers_get@@YAPEBUhb_shaper_entry_t@@XZ 00000001800a6e50 f   hb-shaper.obj
 0001:000a5e60       ?get_stored@?$hb_lazy_loader_t@Uhb_shaper_entry_t@@Uhb_shapers_lazy_loader_t@@X$0A@U1@@@QEBAPEAUhb_shaper_entry_t@@XZ 00000001800a6e60 f i hb-shaper.obj
 0001:000a6640       hb_ucd_get_unicode_funcs   00000001800a7640 f   hb-ucd.obj
 0001:000a6780       ?_hb_unicode_is_emoji_Extended_Pictographic@@YA_NI@Z 00000001800a7780 f   hb-unicode.obj
 0001:000a6810       hb_unicode_funcs_create    00000001800a7810 f   hb-unicode.obj
 0001:000a6900       hb_unicode_funcs_destroy   00000001800a7900 f   hb-unicode.obj
 0001:000a6a20       hb_unicode_funcs_get_default 00000001800a7a20 f   hb-unicode.obj
 0001:000a6a30       hb_unicode_funcs_get_empty 00000001800a7a30 f   hb-unicode.obj
 0001:000a6a40       hb_unicode_funcs_set_combining_class_func 00000001800a7a40 f   hb-unicode.obj
 0001:000a6ad0       hb_unicode_funcs_set_compose_func 00000001800a7ad0 f   hb-unicode.obj
 0001:000a6b70       hb_unicode_funcs_set_decompose_func 00000001800a7b70 f   hb-unicode.obj
 0001:000a6c10       hb_unicode_funcs_set_general_category_func 00000001800a7c10 f   hb-unicode.obj
 0001:000a6ca0       hb_unicode_funcs_set_mirroring_func 00000001800a7ca0 f   hb-unicode.obj
 0001:000a6d30       hb_unicode_funcs_set_script_func 00000001800a7d30 f   hb-unicode.obj
 0001:000a6dc0       Java_sun_font_FileFontStrike__1getGlyphImageFromWindows 00000001800a7dc0 f   lcdglyph.obj
 0001:000a7760       getHBScriptCode            00000001800a8760 f   scriptMapping.obj
 0001:000a7780       Java_sun_font_StrikeCache_getInvisibleGlyphPtr 00000001800a8780 f   sunFont.obj
 0001:000a7780       Java_sun_font_NullFontScaler_getGlyphImage 00000001800a8780 f   sunFont.obj
 0001:000a7790       Java_sun_font_NullFontScaler_getNullScalerContext 00000001800a8790 f   sunFont.obj
 0001:000a77c0       Java_sun_font_StrikeCache_freeIntMemory 00000001800a87c0 f   sunFont.obj
 0001:000a78b0       Java_sun_font_StrikeCache_freeIntPointer 00000001800a88b0 f   sunFont.obj
 0001:000a78c0       Java_sun_font_StrikeCache_freeLongMemory 00000001800a88c0 f   sunFont.obj
 0001:000a79b0       Java_sun_font_StrikeCache_freeLongPointer 00000001800a89b0 f   sunFont.obj
 0001:000a79c0       Java_sun_font_SunFontManager_initIDs 00000001800a89c0 f   sunFont.obj
 0001:000a8160       isNullScalerContext        00000001800a9160 f   sunFont.obj
 0001:000a816d       SurfaceData_GetOps         00000001800a916d f   awt:awt.dll
 0001:000a8173       SurfaceData_IntersectBounds 00000001800a9173 f   awt:awt.dll
 0001:000a8179       SurfaceData_InitOps        00000001800a9179 f   awt:awt.dll
 0001:000a817f       GetNativePrim              00000001800a917f f   awt:awt.dll
 0001:000a8185       GrPrim_Sg2dGetCompInfo     00000001800a9185 f   awt:awt.dll
 0001:000a818b       GrPrim_Sg2dGetClip         00000001800a918b f   awt:awt.dll
 0001:000a8191       GrPrim_Sg2dGetPixel        00000001800a9191 f   awt:awt.dll
 0001:000a8197       GrPrim_Sg2dGetEaRGB        00000001800a9197 f   awt:awt.dll
 0001:000a819d       GrPrim_Sg2dGetLCDTextContrast 00000001800a919d f   awt:awt.dll
 0001:000a81a3       AccelGlyphCache_RemoveAllCellInfos 00000001800a91a3 f   awt:awt.dll
 0001:000a81a9       JNU_ThrowOutOfMemoryError  00000001800a91a9 f   java:java.dll
 0001:000a81af       JNU_ThrowInternalError     00000001800a91af f   java:java.dll
 0001:000a81b5       JNU_ThrowArrayIndexOutOfBoundsException 00000001800a91b5 f   java:java.dll
 0001:000a81bb       JNU_NewStringPlatform      00000001800a91bb f   java:java.dll
 0001:000a81c1       JNU_CallStaticMethodByName 00000001800a91c1 f   java:java.dll
 0001:000a81c7       FT_Init_FreeType           00000001800a91c7 f   freetype:freetype.dll
 0001:000a81cd       FT_Done_FreeType           00000001800a91cd f   freetype:freetype.dll
 0001:000a81d3       FT_New_Memory_Face         00000001800a91d3 f   freetype:freetype.dll
 0001:000a81d9       FT_Open_Face               00000001800a91d9 f   freetype:freetype.dll
 0001:000a81df       FT_Done_Face               00000001800a91df f   freetype:freetype.dll
 0001:000a81e5       FT_Set_Char_Size           00000001800a91e5 f   freetype:freetype.dll
 0001:000a81eb       FT_Load_Glyph              00000001800a91eb f   freetype:freetype.dll
 0001:000a81f1       FT_Set_Transform           00000001800a91f1 f   freetype:freetype.dll
 0001:000a81f7       FT_Render_Glyph            00000001800a91f7 f   freetype:freetype.dll
 0001:000a81fd       FT_Get_Char_Index          00000001800a91fd f   freetype:freetype.dll
 0001:000a8203       FT_MulFix                  00000001800a9203 f   freetype:freetype.dll
 0001:000a8209       FT_Matrix_Multiply         00000001800a9209 f   freetype:freetype.dll
 0001:000a820f       FT_Outline_Get_BBox        00000001800a920f f   freetype:freetype.dll
 0001:000a8215       FT_Activate_Size           00000001800a9215 f   freetype:freetype.dll
 0001:000a821b       FT_Outline_Decompose       00000001800a921b f   freetype:freetype.dll
 0001:000a8221       FT_Outline_Get_CBox        00000001800a9221 f   freetype:freetype.dll
 0001:000a8227       FT_Outline_Translate       00000001800a9227 f   freetype:freetype.dll
 0001:000a822d       FT_Outline_Embolden        00000001800a922d f   freetype:freetype.dll
 0001:000a8233       FT_Library_SetLcdFilter    00000001800a9233 f   freetype:freetype.dll
 0001:000a8239       FT_Property_Set            00000001800a9239 f   freetype:freetype.dll
 0001:000a8240       __GSHandlerCheck           00000001800a9240 f   MSVCRT:gshandler.obj
 0001:000a8260       __GSHandlerCheckCommon     00000001800a9260 f   MSVCRT:gshandler.obj
 0001:000a82d0       __security_check_cookie    00000001800a92d0 f   MSVCRT:amdsecgs.obj
 0001:000a82f0       ??3@YAXPEAX_K@Z            00000001800a92f0 f   MSVCRT:delete_scalar_size.obj
 0001:000a82f8       __raise_securityfailure    00000001800a92f8 f   MSVCRT:gs_report.obj
 0001:000a832c       __report_gsfailure         00000001800a932c f   MSVCRT:gs_report.obj
 0001:000a8400       __report_rangecheckfailure 00000001800a9400 f   MSVCRT:gs_report.obj
 0001:000a8414       __report_securityfailure   00000001800a9414 f   MSVCRT:gs_report.obj
 0001:000a85b0       _alloca_probe              00000001800a95b0 f   MSVCRT:chkstk.obj
 0001:000a85b0       __chkstk                   00000001800a95b0 f   MSVCRT:chkstk.obj
 0001:000a8600       __vdecl_floorf4            00000001800a9600 f   MSVCRT:svml_sfloorf4_dispatch.obj
 0001:000a8934       _DllMainCRTStartup         00000001800a9934 f   MSVCRT:dll_dllmain.obj
 0001:000a8974       ??3@YAXPEAX@Z              00000001800a9974 f   MSVCRT:delete_scalar.obj
 0001:000a897c       __isa_available_init       00000001800a997c f   MSVCRT:cpu_disp.obj
 0001:000a8b30       __sse2_floorf4@@16         00000001800a9b30 f   MSVCRT:svml_sfloorf4_sse2.obj
 0001:000a8b80       __sse4_floorf4@@16         00000001800a9b80 f   MSVCRT:svml_sfloorf4_sse4.obj
 0001:000a8b88       __security_init_cookie     00000001800a9b88 f   MSVCRT:gs_support.obj
 0001:000a8c34       DllMain                    00000001800a9c34 f   MSVCRT:dll_dllmain_stub.obj
 0001:000a8c58       ?__scrt_initialize_type_info@@YAXXZ 00000001800a9c58 f   MSVCRT:tncleanup.obj
 0001:000a8c68       ?__scrt_uninitialize_type_info@@YAXXZ 00000001800a9c68 f   MSVCRT:tncleanup.obj
 0001:000a8c74       __local_stdio_scanf_options 00000001800a9c74 f i MSVCRT:default_local_stdio_options.obj
 0001:000a8c7c       __scrt_initialize_default_local_stdio_options 00000001800a9c7c f   MSVCRT:default_local_stdio_options.obj
 0001:000a8c98       __scrt_acquire_startup_lock 00000001800a9c98 f   MSVCRT:utility.obj
 0001:000a8cd4       __scrt_dllmain_after_initialize_c 00000001800a9cd4 f   MSVCRT:utility.obj
 0001:000a8d08       __scrt_dllmain_before_initialize_c 00000001800a9d08 f   MSVCRT:utility.obj
 0001:000a8d20       __scrt_dllmain_crt_thread_attach 00000001800a9d20 f   MSVCRT:utility.obj
 0001:000a8d48       __scrt_dllmain_crt_thread_detach 00000001800a9d48 f   MSVCRT:utility.obj
 0001:000a8d60       __scrt_dllmain_exception_filter 00000001800a9d60 f   MSVCRT:utility.obj
 0001:000a8dc0       __scrt_dllmain_uninitialize_c 00000001800a9dc0 f   MSVCRT:utility.obj
 0001:000a8df0       __scrt_dllmain_uninitialize_critical 00000001800a9df0 f   MSVCRT:utility.obj
 0001:000a8e04       __scrt_initialize_crt      00000001800a9e04 f   MSVCRT:utility.obj
 0001:000a8e50       __scrt_initialize_onexit_tables 00000001800a9e50 f   MSVCRT:utility.obj
 0001:000a8edc       __scrt_is_nonwritable_in_current_image 00000001800a9edc f   MSVCRT:utility.obj
 0001:000a8f74       __scrt_release_startup_lock 00000001800a9f74 f   MSVCRT:utility.obj
 0001:000a8f98       __scrt_uninitialize_crt    00000001800a9f98 f   MSVCRT:utility.obj
 0001:000a8fc4       __scrt_get_dyn_tls_init_callback 00000001800a9fc4 f   MSVCRT:dyn_tls_init.obj
 0001:000a8fcc       __crt_debugger_hook        00000001800a9fcc f   MSVCRT:utility_desktop.obj
 0001:000a8fd4       __scrt_fastfail            00000001800a9fd4 f   MSVCRT:utility_desktop.obj
 0001:000a9120       _RTC_Initialize            00000001800aa120 f   MSVCRT:initsect.obj
 0001:000a915c       _RTC_Terminate             00000001800aa15c f   MSVCRT:initsect.obj
 0001:000a9198       __scrt_is_ucrt_dll_in_use  00000001800aa198 f   MSVCRT:ucrt_detection.obj
 0001:000a91b0       memset                     00000001800aa1b0 f   vcruntime:VCRUNTIME140.dll
 0001:000a91b6       strrchr                    00000001800aa1b6 f   vcruntime:VCRUNTIME140.dll
 0001:000a91bc       wcsrchr                    00000001800aa1bc f   vcruntime:VCRUNTIME140.dll
 0001:000a91c2       wcsstr                     00000001800aa1c2 f   vcruntime:VCRUNTIME140.dll
 0001:000a91c8       strstr                     00000001800aa1c8 f   vcruntime:VCRUNTIME140.dll
 0001:000a91ce       memcpy                     00000001800aa1ce f   vcruntime:VCRUNTIME140.dll
 0001:000a91d4       memmove                    00000001800aa1d4 f   vcruntime:VCRUNTIME140.dll
 0001:000a91da       strchr                     00000001800aa1da f   vcruntime:VCRUNTIME140.dll
 0001:000a91e0       memcmp                     00000001800aa1e0 f   vcruntime:VCRUNTIME140.dll
 0001:000a91e6       __C_specific_handler       00000001800aa1e6 f   vcruntime:VCRUNTIME140.dll
 0001:000a91ec       __std_type_info_destroy_list 00000001800aa1ec f   vcruntime:VCRUNTIME140.dll
 0001:000a91f2       free                       00000001800aa1f2 f   ucrt:api-ms-win-crt-heap-l1-1-0.dll
 0001:000a91f8       floor                      00000001800aa1f8 f   ucrt:api-ms-win-crt-math-l1-1-0.dll
 0001:000a91fe       pow                        00000001800aa1fe f   ucrt:api-ms-win-crt-math-l1-1-0.dll
 0001:000a9204       sqrt                       00000001800aa204 f   ucrt:api-ms-win-crt-math-l1-1-0.dll
 0001:000a920a       floorf                     00000001800aa20a f   ucrt:api-ms-win-crt-math-l1-1-0.dll
 0001:000a9210       ceilf                      00000001800aa210 f   ucrt:api-ms-win-crt-math-l1-1-0.dll
 0001:000a9216       cosf                       00000001800aa216 f   ucrt:api-ms-win-crt-math-l1-1-0.dll
 0001:000a921c       sinf                       00000001800aa21c f   ucrt:api-ms-win-crt-math-l1-1-0.dll
 0001:000a9222       tanf                       00000001800aa222 f   ucrt:api-ms-win-crt-math-l1-1-0.dll
 0001:000a9228       strcmp                     00000001800aa228 f   ucrt:api-ms-win-crt-string-l1-1-0.dll
 0001:000a922e       _hypotf                    00000001800aa22e f   ucrt:api-ms-win-crt-math-l1-1-0.dll
 0001:000a9234       _initterm                  00000001800aa234 f   ucrt:api-ms-win-crt-runtime-l1-1-0.dll
 0001:000a923a       _initterm_e                00000001800aa23a f   ucrt:api-ms-win-crt-runtime-l1-1-0.dll
 0001:000a9240       _seh_filter_dll            00000001800aa240 f   ucrt:api-ms-win-crt-runtime-l1-1-0.dll
 0001:000a9246       _configure_narrow_argv     00000001800aa246 f   ucrt:api-ms-win-crt-runtime-l1-1-0.dll
 0001:000a924c       _initialize_narrow_environment 00000001800aa24c f   ucrt:api-ms-win-crt-runtime-l1-1-0.dll
 0001:000a9252       _initialize_onexit_table   00000001800aa252 f   ucrt:api-ms-win-crt-runtime-l1-1-0.dll
 0001:000a9258       _execute_onexit_table      00000001800aa258 f   ucrt:api-ms-win-crt-runtime-l1-1-0.dll
 0001:000a925e       _cexit                     00000001800aa25e f   ucrt:api-ms-win-crt-runtime-l1-1-0.dll
 0001:000a9280       _guard_dispatch_icall_nop  00000001800aa280 f   MSVCRT:guard_dispatch.obj
 0001:000a92a0       _guard_xfg_dispatch_icall_nop 00000001800aa2a0 f   MSVCRT:guard_xfg_dispatch.obj
 0002:00000000       __imp_RegCloseKey          00000001800ab000     advapi32:ADVAPI32.dll
 0002:00000008       __imp_RegOpenKeyExA        00000001800ab008     advapi32:ADVAPI32.dll
 0002:00000010       __imp_RegQueryInfoKeyW     00000001800ab010     advapi32:ADVAPI32.dll
 0002:00000018       __imp_RegEnumValueW        00000001800ab018     advapi32:ADVAPI32.dll
 0002:00000020       \177ADVAPI32_NULL_THUNK_DATA 00000001800ab020     advapi32:ADVAPI32.dll
 0002:00000028       __imp_GetDeviceCaps        00000001800ab028     gdi32:GDI32.dll
 0002:00000030       __imp_CreateCompatibleBitmap 00000001800ab030     gdi32:GDI32.dll
 0002:00000038       __imp_EnumFontFamiliesExW  00000001800ab038     gdi32:GDI32.dll
 0002:00000040       __imp_CreateFontIndirectW  00000001800ab040     gdi32:GDI32.dll
 0002:00000048       __imp_DeleteObject         00000001800ab048     gdi32:GDI32.dll
 0002:00000050       __imp_GetDIBits            00000001800ab050     gdi32:GDI32.dll
 0002:00000058       __imp_GetFontData          00000001800ab058     gdi32:GDI32.dll
 0002:00000060       __imp_CreateCompatibleDC   00000001800ab060     gdi32:GDI32.dll
 0002:00000068       __imp_SetBkColor           00000001800ab068     gdi32:GDI32.dll
 0002:00000070       __imp_GetStockObject       00000001800ab070     gdi32:GDI32.dll
 0002:00000078       __imp_SelectObject         00000001800ab078     gdi32:GDI32.dll
 0002:00000080       __imp_SetMapMode           00000001800ab080     gdi32:GDI32.dll
 0002:00000088       __imp_SetTextColor         00000001800ab088     gdi32:GDI32.dll
 0002:00000090       __imp_GetTextMetricsA      00000001800ab090     gdi32:GDI32.dll
 0002:00000098       __imp_ExtTextOutW          00000001800ab098     gdi32:GDI32.dll
 0002:000000a0       __imp_GetGlyphOutlineA     00000001800ab0a0     gdi32:GDI32.dll
 0002:000000a8       \177GDI32_NULL_THUNK_DATA  00000001800ab0a8     gdi32:GDI32.dll
 0002:000000b0       __imp_LeaveCriticalSection 00000001800ab0b0     kernel32:KERNEL32.dll
 0002:000000b8       __imp_EnterCriticalSection 00000001800ab0b8     kernel32:KERNEL32.dll
 0002:000000c0       __imp_CloseHandle          00000001800ab0c0     kernel32:KERNEL32.dll
 0002:000000c8       __imp_MapViewOfFile        00000001800ab0c8     kernel32:KERNEL32.dll
 0002:000000d0       __imp_CreateFileW          00000001800ab0d0     kernel32:KERNEL32.dll
 0002:000000d8       __imp_GetWindowsDirectoryA 00000001800ab0d8     kernel32:KERNEL32.dll
 0002:000000e0       __imp_GetSystemDirectoryA  00000001800ab0e0     kernel32:KERNEL32.dll
 0002:000000e8       __imp_DeleteCriticalSection 00000001800ab0e8     kernel32:KERNEL32.dll
 0002:000000f0       __imp_UnmapViewOfFile      00000001800ab0f0     kernel32:KERNEL32.dll
 0002:000000f8       __imp_CreateFileMappingA   00000001800ab0f8     kernel32:KERNEL32.dll
 0002:00000100       __imp_MultiByteToWideChar  00000001800ab100     kernel32:KERNEL32.dll
 0002:00000108       __imp_RtlCaptureContext    00000001800ab108     kernel32:KERNEL32.dll
 0002:00000110       __imp_RtlLookupFunctionEntry 00000001800ab110     kernel32:KERNEL32.dll
 0002:00000118       __imp_RtlVirtualUnwind     00000001800ab118     kernel32:KERNEL32.dll
 0002:00000120       __imp_UnhandledExceptionFilter 00000001800ab120     kernel32:KERNEL32.dll
 0002:00000128       __imp_SetUnhandledExceptionFilter 00000001800ab128     kernel32:KERNEL32.dll
 0002:00000130       __imp_GetCurrentProcess    00000001800ab130     kernel32:KERNEL32.dll
 0002:00000138       __imp_TerminateProcess     00000001800ab138     kernel32:KERNEL32.dll
 0002:00000140       __imp_IsProcessorFeaturePresent 00000001800ab140     kernel32:KERNEL32.dll
 0002:00000148       __imp_QueryPerformanceCounter 00000001800ab148     kernel32:KERNEL32.dll
 0002:00000150       __imp_GetCurrentProcessId  00000001800ab150     kernel32:KERNEL32.dll
 0002:00000158       __imp_GetCurrentThreadId   00000001800ab158     kernel32:KERNEL32.dll
 0002:00000160       __imp_GetSystemTimeAsFileTime 00000001800ab160     kernel32:KERNEL32.dll
 0002:00000168       __imp_DisableThreadLibraryCalls 00000001800ab168     kernel32:KERNEL32.dll
 0002:00000170       __imp_InitializeSListHead  00000001800ab170     kernel32:KERNEL32.dll
 0002:00000178       __imp_IsDebuggerPresent    00000001800ab178     kernel32:KERNEL32.dll
 0002:00000180       __imp_GetFileSize          00000001800ab180     kernel32:KERNEL32.dll
 0002:00000188       \177KERNEL32_NULL_THUNK_DATA 00000001800ab188     kernel32:KERNEL32.dll
 0002:00000190       __imp_SystemParametersInfoA 00000001800ab190     user32:USER32.dll
 0002:00000198       __imp_GetDesktopWindow     00000001800ab198     user32:USER32.dll
 0002:000001a0       __imp_FillRect             00000001800ab1a0     user32:USER32.dll
 0002:000001a8       __imp_GetWindowDC          00000001800ab1a8     user32:USER32.dll
 0002:000001b0       __imp_ReleaseDC            00000001800ab1b0     user32:USER32.dll
 0002:000001b8       __imp_GetDC                00000001800ab1b8     user32:USER32.dll
 0002:000001c0       \177USER32_NULL_THUNK_DATA 00000001800ab1c0     user32:USER32.dll
 0002:000001c8       __imp_memmove              00000001800ab1c8     vcruntime:VCRUNTIME140.dll
 0002:000001d0       __imp_strchr               00000001800ab1d0     vcruntime:VCRUNTIME140.dll
 0002:000001d8       __imp_memcmp               00000001800ab1d8     vcruntime:VCRUNTIME140.dll
 0002:000001e0       __imp___C_specific_handler 00000001800ab1e0     vcruntime:VCRUNTIME140.dll
 0002:000001e8       __imp_memcpy               00000001800ab1e8     vcruntime:VCRUNTIME140.dll
 0002:000001f0       __imp_strstr               00000001800ab1f0     vcruntime:VCRUNTIME140.dll
 0002:000001f8       __imp_wcsstr               00000001800ab1f8     vcruntime:VCRUNTIME140.dll
 0002:00000200       __imp_wcsrchr              00000001800ab200     vcruntime:VCRUNTIME140.dll
 0002:00000208       __imp_strrchr              00000001800ab208     vcruntime:VCRUNTIME140.dll
 0002:00000210       __imp_memset               00000001800ab210     vcruntime:VCRUNTIME140.dll
 0002:00000218       __imp___std_type_info_destroy_list 00000001800ab218     vcruntime:VCRUNTIME140.dll
 0002:00000220       \177VCRUNTIME140_NULL_THUNK_DATA 00000001800ab220     vcruntime:VCRUNTIME140.dll
 0002:00000228       __imp_mbstowcs             00000001800ab228     ucrt:api-ms-win-crt-convert-l1-1-0.dll
 0002:00000230       __imp_strtol               00000001800ab230     ucrt:api-ms-win-crt-convert-l1-1-0.dll
 0002:00000238       \177api-ms-win-crt-convert-l1-1-0_NULL_THUNK_DATA 00000001800ab238     ucrt:api-ms-win-crt-convert-l1-1-0.dll
 0002:00000240       __imp_getenv               00000001800ab240     ucrt:api-ms-win-crt-environment-l1-1-0.dll
 0002:00000248       \177api-ms-win-crt-environment-l1-1-0_NULL_THUNK_DATA 00000001800ab248     ucrt:api-ms-win-crt-environment-l1-1-0.dll
 0002:00000250       __imp_calloc               00000001800ab250     ucrt:api-ms-win-crt-heap-l1-1-0.dll
 0002:00000258       __imp_realloc              00000001800ab258     ucrt:api-ms-win-crt-heap-l1-1-0.dll
 0002:00000260       __imp_free                 00000001800ab260     ucrt:api-ms-win-crt-heap-l1-1-0.dll
 0002:00000268       __imp_malloc               00000001800ab268     ucrt:api-ms-win-crt-heap-l1-1-0.dll
 0002:00000270       \177api-ms-win-crt-heap-l1-1-0_NULL_THUNK_DATA 00000001800ab270     ucrt:api-ms-win-crt-heap-l1-1-0.dll
 0002:00000278       __imp_pow                  00000001800ab278     ucrt:api-ms-win-crt-math-l1-1-0.dll
 0002:00000280       __imp_cosf                 00000001800ab280     ucrt:api-ms-win-crt-math-l1-1-0.dll
 0002:00000288       __imp_sinf                 00000001800ab288     ucrt:api-ms-win-crt-math-l1-1-0.dll
 0002:00000290       __imp_tanf                 00000001800ab290     ucrt:api-ms-win-crt-math-l1-1-0.dll
 0002:00000298       __imp_sqrt                 00000001800ab298     ucrt:api-ms-win-crt-math-l1-1-0.dll
 0002:000002a0       __imp_floorf               00000001800ab2a0     ucrt:api-ms-win-crt-math-l1-1-0.dll
 0002:000002a8       __imp__hypotf              00000001800ab2a8     ucrt:api-ms-win-crt-math-l1-1-0.dll
 0002:000002b0       __imp_ceilf                00000001800ab2b0     ucrt:api-ms-win-crt-math-l1-1-0.dll
 0002:000002b8       __imp_floor                00000001800ab2b8     ucrt:api-ms-win-crt-math-l1-1-0.dll
 0002:000002c0       \177api-ms-win-crt-math-l1-1-0_NULL_THUNK_DATA 00000001800ab2c0     ucrt:api-ms-win-crt-math-l1-1-0.dll
 0002:000002c8       __imp__initterm_e          00000001800ab2c8     ucrt:api-ms-win-crt-runtime-l1-1-0.dll
 0002:000002d0       __imp__cexit               00000001800ab2d0     ucrt:api-ms-win-crt-runtime-l1-1-0.dll
 0002:000002d8       __imp__seh_filter_dll      00000001800ab2d8     ucrt:api-ms-win-crt-runtime-l1-1-0.dll
 0002:000002e0       __imp__execute_onexit_table 00000001800ab2e0     ucrt:api-ms-win-crt-runtime-l1-1-0.dll
 0002:000002e8       __imp__initialize_onexit_table 00000001800ab2e8     ucrt:api-ms-win-crt-runtime-l1-1-0.dll
 0002:000002f0       __imp__initialize_narrow_environment 00000001800ab2f0     ucrt:api-ms-win-crt-runtime-l1-1-0.dll
 0002:000002f8       __imp__configure_narrow_argv 00000001800ab2f8     ucrt:api-ms-win-crt-runtime-l1-1-0.dll
 0002:00000300       __imp__errno               00000001800ab300     ucrt:api-ms-win-crt-runtime-l1-1-0.dll
 0002:00000308       __imp__initterm            00000001800ab308     ucrt:api-ms-win-crt-runtime-l1-1-0.dll
 0002:00000310       \177api-ms-win-crt-runtime-l1-1-0_NULL_THUNK_DATA 00000001800ab310     ucrt:api-ms-win-crt-runtime-l1-1-0.dll
 0002:00000318       __imp_fclose               00000001800ab318     ucrt:api-ms-win-crt-stdio-l1-1-0.dll
 0002:00000320       __imp_ferror               00000001800ab320     ucrt:api-ms-win-crt-stdio-l1-1-0.dll
 0002:00000328       __imp_fopen                00000001800ab328     ucrt:api-ms-win-crt-stdio-l1-1-0.dll
 0002:00000330       __imp___stdio_common_vfprintf 00000001800ab330     ucrt:api-ms-win-crt-stdio-l1-1-0.dll
 0002:00000338       __imp___acrt_iob_func      00000001800ab338     ucrt:api-ms-win-crt-stdio-l1-1-0.dll
 0002:00000340       __imp___stdio_common_vsprintf 00000001800ab340     ucrt:api-ms-win-crt-stdio-l1-1-0.dll
 0002:00000348       __imp_fread                00000001800ab348     ucrt:api-ms-win-crt-stdio-l1-1-0.dll
 0002:00000350       __imp_feof                 00000001800ab350     ucrt:api-ms-win-crt-stdio-l1-1-0.dll
 0002:00000358       \177api-ms-win-crt-stdio-l1-1-0_NULL_THUNK_DATA 00000001800ab358     ucrt:api-ms-win-crt-stdio-l1-1-0.dll
 0002:00000360       __imp_strncmp              00000001800ab360     ucrt:api-ms-win-crt-string-l1-1-0.dll
 0002:00000368       __imp_wcsicmp              00000001800ab368     ucrt:api-ms-win-crt-string-l1-1-0.dll
 0002:00000368       __imp__wcsicmp             00000001800ab368     ucrt:api-ms-win-crt-string-l1-1-0.dll
 0002:00000370       __imp__stricmp             00000001800ab370     ucrt:api-ms-win-crt-string-l1-1-0.dll
 0002:00000370       __imp_stricmp              00000001800ab370     ucrt:api-ms-win-crt-string-l1-1-0.dll
 0002:00000378       __imp_strcmp               00000001800ab378     ucrt:api-ms-win-crt-string-l1-1-0.dll
 0002:00000380       __imp_strncpy              00000001800ab380     ucrt:api-ms-win-crt-string-l1-1-0.dll
 0002:00000388       \177api-ms-win-crt-string-l1-1-0_NULL_THUNK_DATA 00000001800ab388     ucrt:api-ms-win-crt-string-l1-1-0.dll
 0002:00000390       __imp_GrPrim_Sg2dGetClip   00000001800ab390     awt:awt.dll
 0002:00000398       __imp_GrPrim_Sg2dGetCompInfo 00000001800ab398     awt:awt.dll
 0002:000003a0       __imp_GetNativePrim        00000001800ab3a0     awt:awt.dll
 0002:000003a8       __imp_SurfaceData_InitOps  00000001800ab3a8     awt:awt.dll
 0002:000003b0       __imp_SurfaceData_IntersectBounds 00000001800ab3b0     awt:awt.dll
 0002:000003b8       __imp_GrPrim_Sg2dGetPixel  00000001800ab3b8     awt:awt.dll
 0002:000003c0       __imp_GrPrim_Sg2dGetEaRGB  00000001800ab3c0     awt:awt.dll
 0002:000003c8       __imp_AccelGlyphCache_RemoveAllCellInfos 00000001800ab3c8     awt:awt.dll
 0002:000003d0       __imp_GrPrim_Sg2dGetLCDTextContrast 00000001800ab3d0     awt:awt.dll
 0002:000003d8       __imp_SurfaceData_GetOps   00000001800ab3d8     awt:awt.dll
 0002:000003e0       \177awt_NULL_THUNK_DATA    00000001800ab3e0     awt:awt.dll
 0002:000003e8       __imp_FT_Set_Char_Size     00000001800ab3e8     freetype:freetype.dll
 0002:000003f0       __imp_FT_Open_Face         00000001800ab3f0     freetype:freetype.dll
 0002:000003f8       __imp_FT_New_Memory_Face   00000001800ab3f8     freetype:freetype.dll
 0002:00000400       __imp_FT_Done_FreeType     00000001800ab400     freetype:freetype.dll
 0002:00000408       __imp_FT_Load_Glyph        00000001800ab408     freetype:freetype.dll
 0002:00000410       __imp_FT_Init_FreeType     00000001800ab410     freetype:freetype.dll
 0002:00000418       __imp_FT_Property_Set      00000001800ab418     freetype:freetype.dll
 0002:00000420       __imp_FT_Library_SetLcdFilter 00000001800ab420     freetype:freetype.dll
 0002:00000428       __imp_FT_Outline_Embolden  00000001800ab428     freetype:freetype.dll
 0002:00000430       __imp_FT_Outline_Translate 00000001800ab430     freetype:freetype.dll
 0002:00000438       __imp_FT_Outline_Get_CBox  00000001800ab438     freetype:freetype.dll
 0002:00000440       __imp_FT_Outline_Decompose 00000001800ab440     freetype:freetype.dll
 0002:00000448       __imp_FT_Done_Face         00000001800ab448     freetype:freetype.dll
 0002:00000450       __imp_FT_Set_Transform     00000001800ab450     freetype:freetype.dll
 0002:00000458       __imp_FT_Render_Glyph      00000001800ab458     freetype:freetype.dll
 0002:00000460       __imp_FT_Get_Char_Index    00000001800ab460     freetype:freetype.dll
 0002:00000468       __imp_FT_MulFix            00000001800ab468     freetype:freetype.dll
 0002:00000470       __imp_FT_Matrix_Multiply   00000001800ab470     freetype:freetype.dll
 0002:00000478       __imp_FT_Outline_Get_BBox  00000001800ab478     freetype:freetype.dll
 0002:00000480       __imp_FT_Activate_Size     00000001800ab480     freetype:freetype.dll
 0002:00000488       \177freetype_NULL_THUNK_DATA 00000001800ab488     freetype:freetype.dll
 0002:00000490       __imp_JNU_ThrowArrayIndexOutOfBoundsException 00000001800ab490     java:java.dll
 0002:00000498       __imp_JNU_NewStringPlatform 00000001800ab498     java:java.dll
 0002:000004a0       __imp_JNU_CallStaticMethodByName 00000001800ab4a0     java:java.dll
 0002:000004a8       __imp_JNU_ThrowInternalError 00000001800ab4a8     java:java.dll
 0002:000004b0       __imp_JNU_ThrowOutOfMemoryError 00000001800ab4b0     java:java.dll
 0002:000004b8       \177java_NULL_THUNK_DATA   00000001800ab4b8     java:java.dll
 0002:000004c0       __guard_check_icall_fptr   00000001800ab4c0     MSVCRT:guard_support.obj
 0002:000004c8       __guard_xfg_check_icall_fptr 00000001800ab4c8     MSVCRT:guard_support.obj
 0002:000004d0       __guard_dispatch_icall_fptr 00000001800ab4d0     MSVCRT:guard_support.obj
 0002:000004d8       __guard_xfg_dispatch_icall_fptr 00000001800ab4d8     MSVCRT:guard_support.obj
 0002:000004e0       __guard_xfg_table_dispatch_icall_fptr 00000001800ab4e0     MSVCRT:guard_support.obj
 0002:000004e8       __castguard_check_failure_os_handled_fptr 00000001800ab4e8     MSVCRT:guard_support.obj
 0002:000004f0       __guard_memcpy_fptr        00000001800ab4f0     vcruntime:softmemtag.obj
 0002:000004f8       __xc_a                     00000001800ab4f8     MSVCRT:initializers.obj
 0002:00000500       __xc_z                     00000001800ab500     MSVCRT:initializers.obj
 0002:00000508       __xi_a                     00000001800ab508     MSVCRT:initializers.obj
 0002:00000510       __xi_z                     00000001800ab510     MSVCRT:initializers.obj
 0002:00000518       __xp_a                     00000001800ab518     MSVCRT:initializers.obj
 0002:00000520       __xp_z                     00000001800ab520     MSVCRT:initializers.obj
 0002:00000528       __xt_a                     00000001800ab528     MSVCRT:initializers.obj
 0002:00000530       __xt_z                     00000001800ab530     MSVCRT:initializers.obj
 0002:00000540       ??_C@_0CJ@PGKOGMIO@Unsupported?5mode?5for?5glyph?5imag@ 00000001800ab540     ColorGlyphSurfaceData.obj
 0002:00000570       ??_C@_0CP@FKLHLEEM@Initialization?5of?5ColorGlyphSur@ 00000001800ab570     ColorGlyphSurfaceData.obj
 0002:000005a0       __real@3eaaaaaa            00000001800ab5a0     DrawGlyphList.obj
 0002:000005a8       __real@3ff0000000000000    00000001800ab5a8     DrawGlyphList.obj
 0002:000005b0       __real@40400000            00000001800ab5b0     DrawGlyphList.obj
 0002:000005b8       __real@4059000000000000    00000001800ab5b8     DrawGlyphList.obj
 0002:000005c0       __real@406fe00000000000    00000001800ab5c0     DrawGlyphList.obj
 0002:000005c8       __real@beaaaaaa            00000001800ab5c8     DrawGlyphList.obj
 0002:000005d0       ??_C@_0BM@DODCGPJL@sun?1font?1GlyphLayout$GVData@ 00000001800ab5d0     HBShaper.obj
 0002:000005ec       ??_C@_01JPJNBJEM@I@        00000001800ab5ec     HBShaper.obj
 0002:000005f0       ??_C@_06HHPHCOMB@_count@   00000001800ab5f0     HBShaper.obj
 0002:000005f8       ??_C@_06PPHBKICC@_flags@   00000001800ab5f8     HBShaper.obj
 0002:00000600       ??_C@_02EBOMBDPA@?$FLI@    00000001800ab600     HBShaper.obj
 0002:00000608       ??_C@_07PKNHOODJ@_glyphs@  00000001800ab608     HBShaper.obj
 0002:00000610       ??_C@_02MGHEAPDP@?$FLF@    00000001800ab610     HBShaper.obj
 0002:00000618       ??_C@_0L@BHNDECPI@_positions@ 00000001800ab618     HBShaper.obj
 0002:00000628       ??_C@_08MEOKMKLN@_indices@ 00000001800ab628     HBShaper.obj
 0002:00000634       ??_C@_03GAEACAIP@?$CI?$CJV@ 00000001800ab634     HBShaper.obj
 0002:00000638       ??_C@_04PAAMKIIE@grow@     00000001800ab638     HBShaper.obj
 0002:0000063d       ??_C@_00CNPNBAHC@@         00000001800ab63d     HBShaper.obj
 0002:00000640       ??_C@_0L@LCGIKEMB@HB_NODEVTX@ 00000001800ab640     HBShaper.obj
 0002:0000064c       ??_C@_04HHMMLDJI@kern@     00000001800ab64c     HBShaper.obj
 0002:00000654       ??_C@_05LLBOPDMO@?9kern@   00000001800ab654     HBShaper.obj
 0002:0000065c       ??_C@_04BCEPKNGE@liga@     00000001800ab65c     HBShaper.obj
 0002:00000664       ??_C@_05NOJNONDC@?9liga@   00000001800ab664     HBShaper.obj
 0002:0000066c       __real@37800000            00000001800ab66c     HBShaper.obj
 0002:00000670       __real@3f000000            00000001800ab670     HBShaper.obj
 0002:00000674       __real@3f800000            00000001800ab674     HBShaper.obj
 0002:00000680       __xmm@80000000800000008000000080000000 00000001800ab680     HBShaper.obj
 0002:000006f8       ??_C@_11LOCGONAA@@         00000001800ab6f8     fontpath.obj
 0002:00000700       ??_C@_07GCCENIMJ@?2System@ 00000001800ab700     fontpath.obj
 0002:00000708       ??_C@_09FJGNFLHN@?2System32@ 00000001800ab708     fontpath.obj
 0002:00000714       ??_C@_06MIJGMACG@?2Fonts@  00000001800ab714     fontpath.obj
 0002:0000071c       ??_C@_01ICJEACDI@?$DL@     00000001800ab71c     fontpath.obj
 0002:00000720       ??_C@_17BCGMALNF@?$AA?5?$AA?$CG?$AA?5@ 00000001800ab720     fontpath.obj
 0002:00000728       ??_C@_19OLAFNMII@?$AA?4?$AAt?$AAt?$AAf@ 00000001800ab728     fontpath.obj
 0002:00000738       ??_C@_19MKNEPBPF@?$AA?4?$AAo?$AAt?$AAf@ 00000001800ab738     fontpath.obj
 0002:00000748       ??_C@_0BC@LEKPNIDO@java?1util?1HashMap@ 00000001800ab748     fontpath.obj
 0002:00000760       ??_C@_0DJ@FLFJBGBN@?$CILjava?1lang?1Object?$DLLjava?1lang?1O@ 00000001800ab760     fontpath.obj
 0002:0000079c       ??_C@_03KMONJGDG@put@      00000001800ab79c     fontpath.obj
 0002:000007a0       ??_C@_0BG@DHOOFEJE@?$CILjava?1lang?1Object?$DL?$CJZ@ 00000001800ab7a0     fontpath.obj
 0002:000007b8       ??_C@_0M@ILMAKOC@containsKey@ 00000001800ab7b8     fontpath.obj
 0002:000007c8       ??_C@_0BE@GPOIDJOH@java?1util?1ArrayList@ 00000001800ab7c8     fontpath.obj
 0002:000007dc       ??_C@_04PFANPMCN@?$CII?$CJV@ 00000001800ab7dc     fontpath.obj
 0002:000007e4       ??_C@_06FALKBLGB@?$DMinit?$DO@ 00000001800ab7e4     fontpath.obj
 0002:000007ec       ??_C@_03BDGOHNNK@add@      00000001800ab7ec     fontpath.obj
 0002:000007f0       ??_C@_0BB@FLFAIHG@java?1lang?1String@ 00000001800ab7f0     fontpath.obj
 0002:00000808       ??_C@_0CH@BHMNPKMP@?$CILjava?1util?1Locale?$DL?$CJLjava?1lang?1@ 00000001800ab808     fontpath.obj
 0002:00000830       ??_C@_0M@IMBDOEKL@toLowerCase@ 00000001800ab830     fontpath.obj
 0002:00000868       ??_C@_0BB@NIMAMPFF@invalidateScaler@ 00000001800ab868     freetypeScaler.obj
 0002:0000087c       ??_C@_03MMPFGPID@?$CI?$CJZ@ 00000001800ab87c     freetypeScaler.obj
 0002:00000880       ??_C@_0L@NFPPEDEE@debugFonts@ 00000001800ab880     freetypeScaler.obj
 0002:00000890       ??_C@_0BH@MINLIFDD@sun?1font?1FontUtilities@ 00000001800ab890     freetypeScaler.obj
 0002:000008a8       ??_C@_0BE@LLDKDDBI@FREETYPE_PROPERTIES@ 00000001800ab8a8     freetypeScaler.obj
 0002:000008c0       ??_C@_08OKLLNAKL@truetype@ 00000001800ab8c0     freetypeScaler.obj
 0002:000008d0       ??_C@_0BE@OJJAFABD@interpreter?9version@ 00000001800ab8d0     freetypeScaler.obj
 0002:000008e4       __real@3c800000            00000001800ab8e4     freetypeScaler.obj
 0002:000008e8       __real@3ef0000000000000    00000001800ab8e8     freetypeScaler.obj
 0002:000008f0       __real@3f90000000000000    00000001800ab8f0     freetypeScaler.obj
 0002:000008f8       __real@4050000000000000    00000001800ab8f8     freetypeScaler.obj
 0002:00000900       __real@40d0000000000000    00000001800ab900     freetypeScaler.obj
 0002:00000908       __real@42800000            00000001800ab908     freetypeScaler.obj
 0002:0000090c       __real@47800000            00000001800ab90c     freetypeScaler.obj
 0002:00000910       __real@c7800000            00000001800ab910     freetypeScaler.obj
 0002:00000920       __xmm@00010000000000000000366a00010000 00000001800ab920     freetypeScaler.obj
 0002:00000930       __xmm@80000000000000008000000000000000 00000001800ab930     freetypeScaler.obj
 0002:00000e30       ??_C@_08EMNHGPIL@SANITIZE@ 00000001800abe30     hb-aat-layout.obj
 0002:00000e40       ??_C@_0BL@LJCAAAA@start?5?$FL?$CFp?4?4?$CFp?$FN?5?$CI?$CFlu?5bytes?$CJ@ 00000001800abe40     hb-aat-layout.obj
 0002:00000e60       ??_C@_0BO@NFKLCDNJ@end?5?$FL?$CFp?4?4?$CFp?$FN?5?$CFu?5edit?5requests@ 00000001800abe60     hb-aat-layout.obj
 0002:00000e80       ??_C@_02GIPFHKNO@OK@       00000001800abe80     hb-aat-layout.obj
 0002:00000e88       ??_C@_0N@FLBMHONH@OUT?9OF?9RANGE@ 00000001800abe88     hb-aat-layout.obj
 0002:00000e98       ??_C@_0DC@DHOCDOGD@check_range?5?$FL?$CFp?4?4?$CFp?$FN?5?$CI?$CFu?5bytes?$CJ@ 00000001800abe98     hb-aat-layout.obj
 0002:00000ed0       ??_C@_0CD@MJOKIODN@check_point?5?$FL?$CFp?$FN?5in?5?$FL?$CFp?4?4?$CFp?$FN?5?9?$DO@ 00000001800abed0     hb-aat-layout.obj
 0002:00000ef8       ??_C@_07IICDHBMC@GRANTED@  00000001800abef8     hb-aat-layout.obj
 0002:00000f00       ??_C@_06GONJNOIB@DENIED@   00000001800abf00     hb-aat-layout.obj
 0002:00000f08       ??_C@_0DD@ENACFAKI@may_edit?$CI?$CFu?$CJ?5?$FL?$CFp?4?4?$CFp?$FN?5?$CI?$CFu?5bytes@ 00000001800abf08     hb-aat-layout.obj
 0002:00000f40       ??_C@_0BB@HBIIGPNG@start?5table?5morx@ 00000001800abf40     hb-aat-layout.obj
 0002:00000f58       ??_C@_0P@CBPBJJBN@end?5table?5morx@ 00000001800abf58     hb-aat-layout.obj
 0002:00000f68       ??_C@_0BB@NNDNCANK@start?5table?5mort@ 00000001800abf68     hb-aat-layout.obj
 0002:00000f80       ??_C@_0P@INEENGBB@end?5table?5mort@ 00000001800abf80     hb-aat-layout.obj
 0002:00000f90       ??_C@_0BB@JBHFHKBC@start?5table?5kerx@ 00000001800abf90     hb-aat-layout.obj
 0002:00000fa8       ??_C@_0P@MBAMIMNJ@end?5table?5kerx@ 00000001800abfa8     hb-aat-layout.obj
 0002:00000fb8       ??_C@_0CN@KECOGPDB@skipped?5subtable?5?$CFu?5because?5no?5@ 00000001800abfb8     hb-aat-layout.obj
 0002:00000fe8       ??_C@_0BC@JDHEBHPG@start?5subtable?5?$CFu@ 00000001800abfe8     hb-aat-layout.obj
 0002:00001000       ??_C@_0BA@JPJCHFDI@end?5subtable?5?$CFu@ 00000001800ac000     hb-aat-layout.obj
 0002:00001010       ??_C@_0DC@JFNOIBKH@skipped?5chainsubtable?5?$CFu?5becaus@ 00000001800ac010     hb-aat-layout.obj
 0002:00001048       ??_C@_0BH@HOIFGKFM@start?5chainsubtable?5?$CFu@ 00000001800ac048     hb-aat-layout.obj
 0002:00001060       ??_C@_0BF@LIFFOAHA@end?5chainsubtable?5?$CFu@ 00000001800ac060     hb-aat-layout.obj
 0002:00001078       ??_C@_0L@PIONBGHN@start?5kern@ 00000001800ac078     hb-aat-layout.obj
 0002:00001088       ??_C@_08PMCHELIJ@end?5kern@ 00000001800ac088     hb-aat-layout.obj
 0002:00001098       __real@3fe999999999999a    00000001800ac098     hb-aat-layout.obj
 0002:000010a0       __real@41400000            00000001800ac0a0     hb-aat-layout.obj
 0002:000010a4       ??_C@_04HDKFADDE@BLOB@     00000001800ac0a4     hb-blob.obj
 0002:000010b0       ??_C@_0BH@NNGJHJOL@current?5data?5is?5?9?$DO?5?$CFp?6@ 00000001800ac0b0     hb-blob.obj
 0002:000010c8       ??_C@_0DA@EJAJOMDI@bool?5__cdecl?5hb_blob_t?3?3try_mak@ 00000001800ac0c8     hb-blob.obj
 0002:000010f8       ??_C@_0BL@NAAIMIGO@dupped?5successfully?5?9?$DO?5?$CFp?6@ 00000001800ac0f8     hb-blob.obj
 0002:00001114       ??_C@_02JDPG@rb@           00000001800ac114     hb-blob.obj
 0002:00001118       ??_C@_04CIMGMMMG@text@     00000001800ac118     hb-buffer-serialize.obj
 0002:00001120       ??_C@_04CLCAKCEI@json@     00000001800ac120     hb-buffer-serialize.obj
 0002:00002e5c       ??_C@_02GMHACPFF@?$CFu@    00000001800ade5c     hb-buffer-serialize.obj
 0002:00002e60       ??_C@_08ELFBALIN@?0?$CCcl?$CC?3?$CFu@ 00000001800ade60     hb-buffer-serialize.obj
 0002:00002e6c       ??_C@_04MAFNGINP@?$CCu?$CC?3@ 00000001800ade6c     hb-buffer-serialize.obj
 0002:00002e74       ??_C@_03LADEAJCH@?$DN?$CFu@ 00000001800ade74     hb-buffer-serialize.obj
 0002:00002e78       ??_C@_06NGBPNBKB@U?$CL?$CF04X@ 00000001800ade78     hb-buffer-serialize.obj
 0002:00002e80       ??_C@_09CPCAOBOK@harfbuzz?5@ 00000001800ade80     hb-buffer-verify.obj
 0002:00002e8c       ??_C@_01EEMJAFIK@?6@       00000001800ade8c     hb-buffer-verify.obj
 0002:00002e90       ??_C@_0DA@OHKIDNHD@buffer?5verify?5error?3?5clusters?5a@ 00000001800ade90     hb-buffer-verify.obj
 0002:00002ec0       ??_C@_0DC@KJMJOHEC@buffer?5verify?5error?3?5unsafe?9to?9@ 00000001800adec0     hb-buffer-verify.obj
 0002:00002ef8       ??_C@_0DD@CKNGEJOG@buffer?5verify?5error?3?5unsafe?9to?9@ 00000001800adef8     hb-buffer-verify.obj
 0002:00002f30       ??_C@_0CD@DIKIFAKO@buffer?5verify?5error?3?5text?5was?3?5@ 00000001800adf30     hb-buffer-verify.obj
 0002:0000374c       ?_hb_Null_OT_ClipRecord@@3QBEB 00000001800ae74c     hb-common.obj
 0002:00003754       ?_hb_Null_OT_Index@@3QBEB  00000001800ae754     hb-common.obj
 0002:00003760       ?_hb_NullPool@@3QB_KB      00000001800ae760     hb-common.obj
 0002:00003bb0       ?_hb_Null_OT_CmapSubtableLongGroup@@3QBEB 00000001800aebb0     hb-common.obj
 0002:00003bbc       ?_hb_Null_OT_VarIdx@@3QBEB 00000001800aebbc     hb-common.obj
 0002:00003bc0       ?_hb_Null_AAT_Lookup@@3QBEB 00000001800aebc0     hb-common.obj
 0002:00003bc4       ?_hb_Null_AAT_SettingName@@3QBEB 00000001800aebc4     hb-common.obj
 0002:00003bc8       ?minus_1@@3IB              00000001800aebc8     hb-common.obj
 0002:000046f8       ?_hb_Null_OT_LangSys@@3QBEB 00000001800af6f8     hb-common.obj
 0002:00004710       ?_hb_Null_OT_RangeRecord@@3QBEB 00000001800af710     hb-common.obj
 0002:00004820       ??_C@_0L@PGCGEAJK@HB_OPTIONS@ 00000001800af820     hb-common.obj
 0002:00004830       ??_C@_0BJ@EELCEACD@uniscribe?9bug?9compatible@ 00000001800af830     hb-common.obj
 0002:0000484c       __real@38800000            00000001800af84c     hb-common.obj
 0002:00004850       __real@4f000000            00000001800af850     hb-common.obj
 0002:00004860       __xmm@ff7fffffff7fffff7f7fffff7f7fffff 00000001800af860     hb-common.obj
 0002:00004870       __real@3eaaaaab            00000001800af870     hb-draw.obj
 0002:00004878       ??_C@_0L@LHCHIOPJ@successful@ 00000001800af878     hb-face-builder.obj
 0002:00004888       ??_C@_0N@KIEOCLDL@UNSUCCESSFUL@ 00000001800af888     hb-face-builder.obj
 0002:00004898       ??_C@_0CF@PIDDOBFK@end?5?$FL?$CFp?4?4?$CFp?$FN?5serialized?5?$CFu?5byte@ 00000001800af898     hb-face-builder.obj
 0002:000048c0       ??_C@_09EPPNEDIL@SERIALIZE@ 00000001800af8c0     hb-face-builder.obj
 0002:00005a48       ??_C@_0O@DNAEAGNO@HB_FONT_FUNCS@ 00000001800b0a48     hb-font.obj
 0002:00005a60       __xmm@bf800000bf8000000000000000000000 00000001800b0a60     hb-font.obj
 0002:00005be8       __real@0010000000000000    00000001800b0be8     hb-number.obj
 0002:00005bf0       __real@4024000000000000    00000001800b0bf0     hb-number.obj
 0002:00005bf8       __real@42f9999999999990    00000001800b0bf8     hb-number.obj
 0002:00005c00       __real@7fefffffffffffff    00000001800b0c00     hb-number.obj
 0002:00005c08       __real@8010000000000000    00000001800b0c08     hb-number.obj
 0002:00005c10       __real@bff0000000000000    00000001800b0c10     hb-number.obj
 0002:00005c18       __real@ffefffffffffffff    00000001800b0c18     hb-number.obj
 0002:000072b8       __real@3fe0000000000000    00000001800b22b8     hb-ot-cff1-table.obj
 0002:000072c0       __xmm@41dfffffffc0000041dfffffffc00000 00000001800b22c0     hb-ot-cff1-table.obj
 0002:000072d0       __xmm@7fffffffffffffff7fffffffffffffff 00000001800b22d0     hb-ot-cff1-table.obj
 0002:000072e0       __xmm@c1e0000000000000c1e0000000000000 00000001800b22e0     hb-ot-cff1-table.obj
 0002:0000bfc0       ??_C@_0BB@HNNCONOI@0123456789?4EE?$DP?9?$DP@ 00000001800b6fc0     hb-ot-font.obj
 0002:0000bfd4       __real@30800000            00000001800b6fd4     hb-ot-font.obj
 0002:0000bfd8       __real@40490fdb            00000001800b6fd8     hb-ot-font.obj
 0002:0000bfdc       __real@4e800000            00000001800b6fdc     hb-ot-font.obj
 0002:0000bfe0       __xmm@3f0000003f0000003f0000003f000000 00000001800b6fe0     hb-ot-font.obj
 0002:0000c7f0       ??_C@_0BN@IMAOBAG@recursing?5to?5lookup?5?$CFu?5at?5?$CFu@ 00000001800b77f0     hb-ot-layout.obj
 0002:0000c810       ??_C@_0BG@HECNAHM@recursed?5to?5lookup?5?$CFu@ 00000001800b7810     hb-ot-layout.obj
 0002:0000c828       ??_C@_0BI@LEONKCCB@positioning?5glyph?5at?5?$CFu@ 00000001800b7828     hb-ot-layout.obj
 0002:0000c840       ??_C@_0BH@NHBAIFPO@positioned?5glyph?5at?5?$CFu@ 00000001800b7840     hb-ot-layout.obj
 0002:0000c858       ??_C@_0CN@LEDGNLBP@cursive?5attaching?5glyph?5at?5?$CFu?5t@ 00000001800b7858     hb-ot-layout.obj
 0002:0000c888       ??_C@_0CM@NPOIGCBF@cursive?5attached?5glyph?5at?5?$CFu?5to@ 00000001800b7888     hb-ot-layout.obj
 0002:0000c8b8       ??_C@_0CK@HCENOEA@attaching?5mark?5glyph?5at?5?$CFu?5to?5g@ 00000001800b78b8     hb-ot-layout.obj
 0002:0000c8e8       ??_C@_0CJ@IBLNDIDG@attached?5mark?5glyph?5at?5?$CFu?5to?5gl@ 00000001800b78e8     hb-ot-layout.obj
 0002:0000c918       ??_C@_0DG@CFBMBHJC@replacing?5glyph?5at?5?$CFu?5?$CIreverse?5@ 00000001800b7918     hb-ot-layout.obj
 0002:0000c950       ??_C@_0DF@HANPKIIM@replaced?5glyph?5at?5?$CFu?5?$CIreverse?5c@ 00000001800b7950     hb-ot-layout.obj
 0002:0000c988       ??_C@_0BB@INONMPMF@start?5table?5kern@ 00000001800b7988     hb-ot-layout.obj
 0002:0000c9a0       ??_C@_0P@NNJEDJAO@end?5table?5kern@ 00000001800b79a0     hb-ot-layout.obj
 0002:0000c9b0       ??_C@_0CH@IEHKJJLD@start?5table?5GSUB?5script?5tag?5?8?$CFc@ 00000001800b79b0     hb-ot-layout.obj
 0002:0000c9d8       ??_C@_0CF@EJFPDLF@end?5table?5GSUB?5script?5tag?5?8?$CFc?$CFc@ 00000001800b79d8     hb-ot-layout.obj
 0002:0000ca00       ??_C@_0CH@GMBJPMNF@start?5table?5GPOS?5script?5tag?5?8?$CFc@ 00000001800b7a00     hb-ot-layout.obj
 0002:0000ca28       ??_C@_0CF@OMPGJGND@end?5table?5GPOS?5script?5tag?5?8?$CFc?$CFc@ 00000001800b7a28     hb-ot-layout.obj
 0002:0000ca50       ??_C@_0CD@BOMDBIAK@start?5lookup?5?$CFu?5feature?5?8?$CFc?$CFc?$CFc@ 00000001800b7a50     hb-ot-layout.obj
 0002:0000ca78       ??_C@_0DO@IEOLAPEI@skipped?5lookup?5?$CFu?5feature?5?8?$CFc?$CFc@ 00000001800b7a78     hb-ot-layout.obj
 0002:0000cab8       ??_C@_0CB@CHKBGOD@end?5lookup?5?$CFu?5feature?5?8?$CFc?$CFc?$CFc?$CFc@ 00000001800b7ab8     hb-ot-layout.obj
 0002:0000cae0       ??_C@_0CM@MBFHEMDL@replacing?5glyph?5at?5?$CFu?5?$CIsingle?5s@ 00000001800b7ae0     hb-ot-layout.obj
 0002:0000cb10       ??_C@_0CL@HNJEFGAB@replaced?5glyph?5at?5?$CFu?5?$CIsingle?5su@ 00000001800b7b10     hb-ot-layout.obj
 0002:0000cb40       ??_C@_0CP@EIOKABLL@replacing?5glyph?5at?5?$CFu?5?$CIalternat@ 00000001800b7b40     hb-ot-layout.obj
 0002:0000cb70       ??_C@_0CO@NDFGAIJA@replaced?5glyph?5at?5?$CFu?5?$CIalternate@ 00000001800b7b70     hb-ot-layout.obj
 0002:0000cba0       ??_C@_0CO@BKNPNBH@replacing?5glyph?5at?5?$CFu?5?$CImultiple@ 00000001800b7ba0     hb-ot-layout.obj
 0002:0000cbd0       ??_C@_0CN@NJGGGGNH@replaced?5glyph?5at?5?$CFu?5?$CImultiple?5@ 00000001800b7bd0     hb-ot-layout.obj
 0002:0000cc00       ??_C@_0CN@NDMMJMPC@deleting?5glyph?5at?5?$CFu?5?$CImultiple?5@ 00000001800b7c00     hb-ot-layout.obj
 0002:0000cc30       ??_C@_0CM@LFICHOPB@deleted?5glyph?5at?5?$CFu?5?$CImultiple?5s@ 00000001800b7c30     hb-ot-layout.obj
 0002:0000cc60       ??_C@_0BI@MNHOPBOM@multiplying?5glyph?5at?5?$CFu@ 00000001800b7c60     hb-ot-layout.obj
 0002:0000cc78       ??_C@_0BI@MMDNIBFC@multiplied?5glyphs?5at?5?$CFs@ 00000001800b7c78     hb-ot-layout.obj
 0002:0000cc90       ??_C@_0BM@ILJLMNPF@try?5kerning?5glyphs?5at?5?$CFu?0?$CFu@ 00000001800b7c90     hb-ot-layout.obj
 0002:0000ccb0       ??_C@_0BH@OPPMFNJB@kerned?5glyphs?5at?5?$CFu?0?$CFu@ 00000001800b7cb0     hb-ot-layout.obj
 0002:0000ccc8       ??_C@_0BO@DMMODMBI@tried?5kerning?5glyphs?5at?5?$CFu?0?$CFu@ 00000001800b7cc8     hb-ot-layout.obj
 0002:0000cce8       ??_C@_0CO@NFINLDBE@replacing?5glyph?5at?5?$CFu?5?$CIligature@ 00000001800b7ce8     hb-ot-layout.obj
 0002:0000cd18       ??_C@_0CN@NEGCINE@replaced?5glyph?5at?5?$CFu?5?$CIligature?5@ 00000001800b7d18     hb-ot-layout.obj
 0002:0000cd48       ??_C@_0BG@PELKDOGC@ligating?5glyphs?5at?5?$CFs@ 00000001800b7d48     hb-ot-layout.obj
 0002:0000cd60       ??_C@_0BE@CENOONDG@ligated?5glyph?5at?5?$CFu@ 00000001800b7d60     hb-ot-layout.obj
 0002:0000cd78       __real@3ff8000000000000    00000001800b7d78     hb-ot-layout.obj
 0002:0000cd80       __xmm@ffffffffffffffffffffffffffffffff 00000001800b7d80     hb-ot-layout.obj
 0002:0000dcd0       __xmm@7fffffff7fffffff7fffffff7fffffff 00000001800b8cd0     hb-ot-metrics.obj
 0002:0000dcf0       ??_C@_0BE@JHLPALHA@start?5fallback?5mark@ 00000001800b8cf0     hb-ot-shape-fallback.obj
 0002:0000dd08       ??_C@_0BC@GBHKPNCC@end?5fallback?5mark@ 00000001800b8d08     hb-ot-shape-fallback.obj
 0002:0000dd20       ??_C@_0BE@OKOKJNMC@start?5fallback?5kern@ 00000001800b8d20     hb-ot-shape-fallback.obj
 0002:0000dd38       ??_C@_0BC@BMCPGLJA@end?5fallback?5kern@ 00000001800b8d38     hb-ot-shape-fallback.obj
 0002:0000dd50       ??_C@_0O@PHODME@start?5reorder@ 00000001800b8d50     hb-ot-shape-normalize.obj
 0002:0000dd60       ??_C@_0M@MGJODAHL@end?5reorder@ 00000001800b8d60     hb-ot-shape-normalize.obj
 0002:0000dde0       ??_C@_0BJ@JCPBKLAK@start?5postprocess?9glyphs@ 00000001800b8de0     hb-ot-shape.obj
 0002:0000de00       ??_C@_0BH@KGKNGMEK@end?5postprocess?9glyphs@ 00000001800b8e00     hb-ot-shape.obj
 0002:0000de18       ??_C@_0BG@KEPPLGKM@start?5preprocess?9text@ 00000001800b8e18     hb-ot-shape.obj
 0002:0000de30       ??_C@_0BE@HIKMCIJG@end?5preprocess?9text@ 00000001800b8e30     hb-ot-shape.obj
 0002:0000de44       ??_C@_02IGGBGAC@ot@        00000001800b8e44     hb-ot-shape.obj
 0002:0000de50       __xmm@00000007000000070000000700000007 00000001800b8e50     hb-ot-shape.obj
 0002:0000e050       ?_hb_ot_shaper_arabic@@3Uhb_ot_shaper_t@@B 00000001800b9050     hb-ot-shaper-arabic.obj
 0002:0000f110       ??_C@_09BJHPDKCP@measuring@ 00000001800ba110     hb-ot-shaper-arabic.obj
 0002:0000f120       ??_C@_07MINDNCFJ@cutting@  00000001800ba120     hb-ot-shaper-arabic.obj
 0002:0000f128       ??_C@_0BJ@CMFJBMOA@?$CFs?5stretch?5at?5?$CI?$CFu?0?$CFu?0?$CFu?$CJ@ 00000001800ba128     hb-ot-shaper-arabic.obj
 0002:0000f144       ??_C@_06DBDILMHG@ARABIC@   00000001800ba144     hb-ot-shaper-arabic.obj
 0002:0000f150       ?_hb_ot_shaper_default@@3Uhb_ot_shaper_t@@B 00000001800ba150     hb-ot-shaper-default.obj
 0002:0000f1b0       ?_hb_ot_shaper_dumber@@3Uhb_ot_shaper_t@@B 00000001800ba1b0     hb-ot-shaper-default.obj
 0002:0000f220       ?_hb_ot_shaper_hangul@@3Uhb_ot_shaper_t@@B 00000001800ba220     hb-ot-shaper-hangul.obj
 0002:0000f2a0       ?_hb_ot_shaper_hebrew@@3Uhb_ot_shaper_t@@B 00000001800ba2a0     hb-ot-shaper-hebrew.obj
 0002:00012c70       ?_hb_ot_shaper_indic@@3Uhb_ot_shaper_t@@B 00000001800bdc70     hb-ot-shaper-indic.obj
 0002:00014f08       ??_C@_0BP@PFJNIBAL@start?5reordering?5indic?5initial@ 00000001800bff08     hb-ot-shaper-indic.obj
 0002:00014f28       ??_C@_0BN@DEJECPK@end?5reordering?5indic?5initial@ 00000001800bff28     hb-ot-shaper-indic.obj
 0002:00014f48       ??_C@_0BN@BEFMFOMM@start?5reordering?5indic?5final@ 00000001800bff48     hb-ot-shaper-indic.obj
 0002:00014f68       ??_C@_0BL@CMBCGANJ@end?5reordering?5indic?5final@ 00000001800bff68     hb-ot-shaper-indic.obj
 0002:00014fa0       ?_hb_ot_shaper_khmer@@3Uhb_ot_shaper_t@@B 00000001800bffa0     hb-ot-shaper-khmer.obj
 0002:00015628       ??_C@_0BH@LEEFGPFH@start?5reordering?5khmer@ 00000001800c0628     hb-ot-shaper-khmer.obj
 0002:00015640       ??_C@_0BF@HCJFOFHL@end?5reordering?5khmer@ 00000001800c0640     hb-ot-shaper-khmer.obj
 0002:00015670       ?_hb_ot_shaper_myanmar@@3Uhb_ot_shaper_t@@B 00000001800c0670     hb-ot-shaper-myanmar.obj
 0002:000156d0       ?_hb_ot_shaper_myanmar_zawgyi@@3Uhb_ot_shaper_t@@B 00000001800c06d0     hb-ot-shaper-myanmar.obj
 0002:000164f0       ??_C@_0BJ@HDEFJBCC@start?5reordering?5myanmar@ 00000001800c14f0     hb-ot-shaper-myanmar.obj
 0002:00016510       ??_C@_0BH@EHBJFGGC@end?5reordering?5myanmar@ 00000001800c1510     hb-ot-shaper-myanmar.obj
 0002:00016530       ??_C@_0EG@MEHLKFP@skipped?5inserting?5dotted?9circle@ 00000001800c1530     hb-ot-shaper-syllabic.obj
 0002:00016578       ??_C@_0BP@BAKDHKAL@start?5inserting?5dotted?9circles@ 00000001800c1578     hb-ot-shaper-syllabic.obj
 0002:00016598       ??_C@_0BN@OGHHLJPK@end?5inserting?5dotted?9circles@ 00000001800c1598     hb-ot-shaper-syllabic.obj
 0002:000165d0       ?_hb_ot_shaper_thai@@3Uhb_ot_shaper_t@@B 00000001800c15d0     hb-ot-shaper-thai.obj
 0002:00017be0       ?_hb_ot_shaper_use@@3Uhb_ot_shaper_t@@B 00000001800c2be0     hb-ot-shaper-use.obj
 0002:00019370       ??_C@_0BF@INKMBGAO@start?5reordering?5USE@ 00000001800c4370     hb-ot-shaper-use.obj
 0002:00019388       ??_C@_0BD@IDPODCA@end?5reordering?5USE@ 00000001800c4388     hb-ot-shaper-use.obj
 0002:0001c070       ??_C@_08LOEDBOED@?9fonnapa@ 00000001800c7070     hb-ot-tag.obj
 0002:0001c080       ??_C@_08GMLKJDFJ@?9polyton@ 00000001800c7080     hb-ot-tag.obj
 0002:0001c090       ??_C@_08NJCBHCMA@?9arevmda@ 00000001800c7090     hb-ot-tag.obj
 0002:0001c0a0       ??_C@_08DCLOKPKI@?9provenc@ 00000001800c70a0     hb-ot-tag.obj
 0002:0001c0b0       ??_C@_07KBFBNAFC@?9fonipa@ 00000001800c70b0     hb-ot-tag.obj
 0002:0001c0b8       ??_C@_05BHGHNKKJ@?9geok@   00000001800c70b8     hb-ot-tag.obj
 0002:0001c0c0       ??_C@_05BCLFBOGB@?9syre@   00000001800c70c0     hb-ot-tag.obj
 0002:0001c0c8       ??_C@_05JFCNACKO@?9syrj@   00000001800c70c8     hb-ot-tag.obj
 0002:0001c0d0       ??_C@_05PBEBMHKK@?9syrn@   00000001800c70d0     hb-ot-tag.obj
 0002:0001c0d8       ??_C@_09GEIHALDG@rt?9lojban@ 00000001800c70d8     hb-ot-tag.obj
 0002:0001c0e8       ??_C@_0L@KFNBBKMN@do?9hant?9hk@ 00000001800c70e8     hb-ot-tag.obj
 0002:0001c0f8       ??_C@_0L@MHHGBNCC@do?9hant?9mo@ 00000001800c70f8     hb-ot-tag.obj
 0002:0001c108       ??_C@_0L@NNBHMAGE@jy?9hant?9hk@ 00000001800c7108     hb-ot-tag.obj
 0002:0001c118       ??_C@_0L@LPLAMHIL@jy?9hant?9mo@ 00000001800c7118     hb-ot-tag.obj
 0002:0001c128       ??_C@_0L@DBFOEPHG@mn?9hant?9hk@ 00000001800c7128     hb-ot-tag.obj
 0002:0001c138       ??_C@_0L@FDPJEIJJ@mn?9hant?9mo@ 00000001800c7138     hb-ot-tag.obj
 0002:0001c148       ??_C@_0L@JBNLJICM@np?9hant?9hk@ 00000001800c7148     hb-ot-tag.obj
 0002:0001c158       ??_C@_0L@PDHMJPMD@np?9hant?9mo@ 00000001800c7158     hb-ot-tag.obj
 0002:0001c168       ??_C@_0L@HOIMDHBF@px?9hant?9hk@ 00000001800c7168     hb-ot-tag.obj
 0002:0001c178       ??_C@_0L@BMCLDAPK@px?9hant?9mo@ 00000001800c7178     hb-ot-tag.obj
 0002:0001c188       ??_C@_0L@PELJBBOA@sp?9hant?9hk@ 00000001800c7188     hb-ot-tag.obj
 0002:0001c198       ??_C@_0L@JGBOBGAP@sp?9hant?9mo@ 00000001800c7198     hb-ot-tag.obj
 0002:0001c1a8       ??_C@_0L@LLINOOHJ@zh?9hant?9hk@ 00000001800c71a8     hb-ot-tag.obj
 0002:0001c1b8       ??_C@_0L@NJCKOJJG@zh?9hant?9mo@ 00000001800c71b8     hb-ot-tag.obj
 0002:0001c1c8       ??_C@_0L@FJFBPFAA@zo?9hant?9hk@ 00000001800c71c8     hb-ot-tag.obj
 0002:0001c1d8       ??_C@_0L@DLPGPCOP@zo?9hant?9mo@ 00000001800c71d8     hb-ot-tag.obj
 0002:0001c1e8       ??_C@_07GEDDMEMG@do?9hans@ 00000001800c71e8     hb-ot-tag.obj
 0002:0001c1f0       ??_C@_07CLHCFCAB@do?9hant@ 00000001800c71f0     hb-ot-tag.obj
 0002:0001c1f8       ??_C@_07HFLHHPAA@jy?9hans@ 00000001800c71f8     hb-ot-tag.obj
 0002:0001c200       ??_C@_07DKPGOJMH@jy?9hant@ 00000001800c7200     hb-ot-tag.obj
 0002:0001c208       ??_C@_07NNALNEFJ@mn?9hans@ 00000001800c7208     hb-ot-tag.obj
 0002:0001c210       ??_C@_07JCEKECJO@mn?9hant@ 00000001800c7210     hb-ot-tag.obj
 0002:0001c218       ??_C@_07GEGFDECJ@np?9hans@ 00000001800c7218     hb-ot-tag.obj
 0002:0001c220       ??_C@_07CLCEKCOO@np?9hant@ 00000001800c7220     hb-ot-tag.obj
 0002:0001c228       ??_C@_07DOLLFJFH@px?9hans@ 00000001800c7228     hb-ot-tag.obj
 0002:0001c230       ??_C@_07HBPKMPJA@px?9hant@ 00000001800c7230     hb-ot-tag.obj
 0002:0001c238       ??_C@_07IDNLBAND@sp?9hans@ 00000001800c7238     hb-ot-tag.obj
 0002:0001c240       ??_C@_07MMJKIGBE@sp?9hant@ 00000001800c7240     hb-ot-tag.obj
 0002:0001c248       ??_C@_07MIKFNJFB@zh?9hans@ 00000001800c7248     hb-ot-tag.obj
 0002:0001c250       ??_C@_07IHOEEPJG@zh?9hant@ 00000001800c7250     hb-ot-tag.obj
 0002:0001c258       ??_C@_07NACOHNP@zo?9hans@  00000001800c7258     hb-ot-tag.obj
 0002:0001c260       ??_C@_07ECEDHBBI@zo?9hant@ 00000001800c7260     hb-ot-tag.obj
 0002:0001c268       ??_C@_03JFOJGEF@do?9@      00000001800c7268     hb-ot-tag.obj
 0002:0001c26c       ??_C@_03EMCOHPPE@?9hk@     00000001800c726c     hb-ot-tag.obj
 0002:0001c270       ??_C@_03COIJHIBL@?9mo@     00000001800c7270     hb-ot-tag.obj
 0002:0001c274       ??_C@_03LPGFHILN@?9tw@     00000001800c7274     hb-ot-tag.obj
 0002:0001c278       ??_C@_03PBCKDOLE@jy?9@     00000001800c7278     hb-ot-tag.obj
 0002:0001c27c       ??_C@_03HFJELDPI@mn?9@     00000001800c727c     hb-ot-tag.obj
 0002:0001c280       ??_C@_03HBJJJCGM@np?9@     00000001800c7280     hb-ot-tag.obj
 0002:0001c284       ??_C@_03MPEMODHI@px?9@     00000001800c7284     hb-ot-tag.obj
 0002:0001c288       ??_C@_03NDOKBNCO@sp?9@     00000001800c7288     hb-ot-tag.obj
 0002:0001c28c       ??_C@_03LMNHKAGM@zh?9@     00000001800c728c     hb-ot-tag.obj
 0002:0001c290       ??_C@_03LJJILGOJ@zo?9@     00000001800c7290     hb-ot-tag.obj
 0002:0001c298       ??_C@_0L@DLEENNLB@an?9hant?9hk@ 00000001800c7298     hb-ot-tag.obj
 0002:0001c2a8       ??_C@_0L@FJODNKFO@an?9hant?9mo@ 00000001800c72a8     hb-ot-tag.obj
 0002:0001c2b8       ??_C@_07IKKEMBBG@an?9hans@ 00000001800c72b8     hb-ot-tag.obj
 0002:0001c2c0       ??_C@_07MFOFFHNB@an?9hant@ 00000001800c72c0     hb-ot-tag.obj
 0002:0001c2c8       ??_C@_06FCHMEGPO@a?9latg@  00000001800c72c8     hb-ot-tag.obj
 0002:0001c2d0       ??_C@_03DPECAMEA@an?9@     00000001800c72d0     hb-ot-tag.obj
 0002:0001c2d8       ??_C@_0L@NNGNBGPF@ak?9hant?9hk@ 00000001800c72d8     hb-ot-tag.obj
 0002:0001c2e8       ??_C@_0L@LPMKBBBK@ak?9hant?9mo@ 00000001800c72e8     hb-ot-tag.obj
 0002:0001c2f8       ??_C@_0L@EDILJCHE@nm?9hant?9hk@ 00000001800c72f8     hb-ot-tag.obj
 0002:0001c308       ??_C@_0L@CBCMJFJL@nm?9hant?9mo@ 00000001800c7308     hb-ot-tag.obj
 0002:0001c318       ??_C@_0L@MNNOKALL@sn?9hant?9hk@ 00000001800c7318     hb-ot-tag.obj
 0002:0001c328       ??_C@_0L@KPHJKHFE@sn?9hant?9mo@ 00000001800c7328     hb-ot-tag.obj
 0002:0001c338       ??_C@_07NIJMOOLB@ak?9hans@ 00000001800c7338     hb-ot-tag.obj
 0002:0001c340       ??_C@_07JHNNHIHG@ak?9hant@ 00000001800c7340     hb-ot-tag.obj
 0002:0001c348       ??_C@_07GCGMMJCH@nm?9hans@ 00000001800c7348     hb-ot-tag.obj
 0002:0001c350       ??_C@_07CNCNFPOA@nm?9hant@ 00000001800c7350     hb-ot-tag.obj
 0002:0001c358       ??_C@_07LEDKPHEA@sn?9hans@ 00000001800c7358     hb-ot-tag.obj
 0002:0001c360       ??_C@_07PLHLGBIH@sn?9hant@ 00000001800c7360     hb-ot-tag.obj
 0002:0001c368       ??_C@_03DJIJMOKL@ak?9@     00000001800c7368     hb-ot-tag.obj
 0002:0001c36c       ??_C@_03GFGHKCEP@nm?9@     00000001800c736c     hb-ot-tag.obj
 0002:0001c370       ??_C@_03MFFCJDFE@sn?9@     00000001800c7370     hb-ot-tag.obj
 0002:0001c378       ??_C@_07LCKCAAMB@?9navajo@ 00000001800c7378     hb-ot-tag.obj
 0002:0001c380       ??_C@_04DBACCPMA@?9hak@    00000001800c7380     hb-ot-tag.obj
 0002:0001c388       ??_C@_04MEKAPCKJ@?9lux@    00000001800c7388     hb-ot-tag.obj
 0002:0001c390       ??_C@_0L@CIHFBKLP@uh?9hant?9hk@ 00000001800c7390     hb-ot-tag.obj
 0002:0001c3a0       ??_C@_0L@EKNCBNFA@uh?9hant?9mo@ 00000001800c73a0     hb-ot-tag.obj
 0002:0001c3b0       ??_C@_07BBIFMLPN@uh?9hans@ 00000001800c73b0     hb-ot-tag.obj
 0002:0001c3b8       ??_C@_07FOMEFNDK@uh?9hant@ 00000001800c73b8     hb-ot-tag.obj
 0002:0001c3c0       ??_C@_03OELELADK@uh?9@     00000001800c73c0     hb-ot-tag.obj
 0002:0001c3c4       ??_C@_03HENGIEOJ@nw?9@     00000001800c73c4     hb-ot-tag.obj
 0002:0001c3c8       ??_C@_03HCDPHGCD@?9th@     00000001800c73c8     hb-ot-tag.obj
 0002:0001c3cc       ??_C@_05NKGDAJJP@o?9bok@   00000001800c73cc     hb-ot-tag.obj
 0002:0001c3d4       ??_C@_05PFGJJNKA@o?9nyn@   00000001800c73d4     hb-ot-tag.obj
 0002:0001c3dc       ??_C@_02GDBPPABP@o?9@      00000001800c73dc     hb-ot-tag.obj
 0002:0001c3e0       ??_C@_03MNHNKBNA@?9md@     00000001800c73e0     hb-ot-tag.obj
 0002:0001c3e8       ??_C@_0L@ONJLNBEF@jc?9hant?9hk@ 00000001800c73e8     hb-ot-tag.obj
 0002:0001c3f8       ??_C@_0L@IPDMNGKK@jc?9hant?9mo@ 00000001800c73f8     hb-ot-tag.obj
 0002:0001c408       ??_C@_07LGBJLMIA@jc?9hans@ 00000001800c7408     hb-ot-tag.obj
 0002:0001c410       ??_C@_07PJFICKEH@jc?9hant@ 00000001800c7410     hb-ot-tag.obj
 0002:0001c418       ??_C@_03OAJLBIBC@jc?9@     00000001800c7418     hb-ot-tag.obj
 0002:0001c420       ??_C@_0L@PKCFBAOH@uu?9hant?9hk@ 00000001800c7420     hb-ot-tag.obj
 0002:0001c430       ??_C@_0L@JIICBHAI@uu?9hant?9mo@ 00000001800c7430     hb-ot-tag.obj
 0002:0001c440       ??_C@_07BHIMDGPD@uu?9hans@ 00000001800c7440     hb-ot-tag.obj
 0002:0001c448       ??_C@_07FIMNKADE@uu?9hant@ 00000001800c7448     hb-ot-tag.obj
 0002:0001c450       ??_C@_03PAEKIABJ@uu?9@     00000001800c7450     hb-ot-tag.obj
 0002:0001c458       ??_C@_07HAFCKKDN@ue?9hans@ 00000001800c7458     hb-ot-tag.obj
 0002:0001c460       ??_C@_09CPANDNJE@h?9hant?9hk@ 00000001800c7460     hb-ot-tag.obj
 0002:0001c470       ??_C@_09ENKKDKHL@h?9hant?9mo@ 00000001800c7470     hb-ot-tag.obj
 0002:0001c480       ??_C@_09JKAGOIDE@h?9min?9nan@ 00000001800c7480     hb-ot-tag.obj
 0002:0001c48c       ??_C@_06NHLFEBO@h?9hans@   00000001800c748c     hb-ot-tag.obj
 0002:0001c494       ??_C@_06ECDKMCNJ@h?9hant@  00000001800c7494     hb-ot-tag.obj
 0002:0001c49c       ??_C@_05OGPPKBIG@h?9min@   00000001800c749c     hb-ot-tag.obj
 0002:0001c4a4       ??_C@_02GGFAOGJK@h?9@      00000001800c74a4     hb-ot-tag.obj
 0002:0001c4a8       ??_C@_03FHLPDODD@alt@      00000001800c74a8     hb-ot-tag.obj
 0002:0001c4b0       ??_C@_0M@EFNICDFC@und?9fonnapa@ 00000001800c74b0     hb-ot-tag.obj
 0002:0001c4bc       ??_C@_03OPDALMNL@rki@      00000001800c74bc     hb-ot-tag.obj
 0002:0001c4c0       ??_C@_03KDPNJBKG@ath@      00000001800c74c0     hb-ot-tag.obj
 0002:0001c4c4       ??_C@_03BMIBANNE@ber@      00000001800c74c4     hb-ot-tag.obj
 0002:0001c4c8       ??_C@_03IOJLFNKI@bik@      00000001800c74c8     hb-ot-tag.obj
 0002:0001c4cc       ??_C@_03JKGFGNIL@btk@      00000001800c74cc     hb-ot-tag.obj
 0002:0001c4d0       ??_C@_03IPGCLNMG@crp@      00000001800c74d0     hb-ot-tag.obj
 0002:0001c4d4       ??_C@_03EHLLDHMO@crx@      00000001800c74d4     hb-ot-tag.obj
 0002:0001c4d8       ??_C@_03JNELBMEE@doi@      00000001800c74d8     hb-ot-tag.obj
 0002:0001c4dc       ??_C@_03NGIHPGDB@din@      00000001800c74dc     hb-ot-tag.obj
 0002:0001c4e0       ??_C@_03OGODBGHE@prs@      00000001800c74e0     hb-ot-tag.obj
 0002:0001c4e4       ??_C@_03MALPCFGN@gon@      00000001800c74e4     hb-ot-tag.obj
 0002:0001c4e8       ??_C@_03NPJADACO@mrj@      00000001800c74e8     hb-ot-tag.obj
 0002:0001c4ec       ??_C@_03JLFIOBFF@hmn@      00000001800c74ec     hb-ot-tag.obj
 0002:0001c4f0       ??_C@_03GDPBLHIG@hnd@      00000001800c74f0     hb-ot-tag.obj
 0002:0001c4f4       ??_C@_03BLHHEDOB@hyw@      00000001800c74f4     hb-ot-tag.obj
 0002:0001c4f8       ??_C@_03KPCANNMC@iba@      00000001800c74f8     hb-ot-tag.obj
 0002:0001c4fc       ??_C@_03DPLAKBPE@ijo@      00000001800c74fc     hb-ot-tag.obj
 0002:0001c500       ??_C@_0L@OOCAKEAN@und?9fonipa@ 00000001800c7500     hb-ot-tag.obj
 0002:0001c50c       ??_C@_03HAFOENKF@ghc@      00000001800c750c     hb-ot-tag.obj
 0002:0001c510       ??_C@_02OPKBKFNM@yi@       00000001800c7510     hb-ot-tag.obj
 0002:0001c514       ??_C@_03IICPCEIM@kln@      00000001800c7514     hb-ot-tag.obj
 0002:0001c518       ??_C@_08IBMBBMEF@und?9Geok@ 00000001800c7518     hb-ot-tag.obj
 0002:0001c524       ??_C@_03CJCPPGJN@okm@      00000001800c7524     hb-ot-tag.obj
 0002:0001c528       ??_C@_03PHBOGOJA@kok@      00000001800c7528     hb-ot-tag.obj
 0002:0001c52c       ??_C@_03HOOHKHFD@kpe@      00000001800c752c     hb-ot-tag.obj
 0002:0001c530       ??_C@_03GGIAOKIC@kar@      00000001800c7530     hb-ot-tag.obj
 0002:0001c534       ??_C@_03HCOHIEGC@uki@      00000001800c7534     hb-ot-tag.obj
 0002:0001c538       ??_C@_03EMDKIONB@mhr@      00000001800c7538     hb-ot-tag.obj
 0002:0001c53c       ??_C@_03DIMAAFM@luy@       00000001800c753c     hb-ot-tag.obj
 0002:0001c540       ??_C@_03FLEAGKJM@mwr@      00000001800c7540     hb-ot-tag.obj
 0002:0001c544       ??_C@_02EEKDFEKL@ms@       00000001800c7544     hb-ot-tag.obj
 0002:0001c548       ??_C@_03KFJMOIAD@man@      00000001800c7548     hb-ot-tag.obj
 0002:0001c54c       ??_C@_05KNLKPBHL@ro?9MD@   00000001800c754c     hb-ot-tag.obj
 0002:0001c554       ??_C@_06PALDGLND@mnw?9TH@  00000001800c7554     hb-ot-tag.obj
 0002:0001c55c       ??_C@_03LHKJBKML@myn@      00000001800c755c     hb-ot-tag.obj
 0002:0001c560       ??_C@_03OBHDOAGL@nah@      00000001800c7560     hb-ot-tag.obj
 0002:0001c564       ??_C@_03JFNCHPFJ@njz@      00000001800c7564     hb-ot-tag.obj
 0002:0001c568       ??_C@_02KAJCLHKP@no@       00000001800c7568     hb-ot-tag.obj
 0002:0001c570       ??_C@_0L@LGMOIJP@el?9polyton@ 00000001800c7570     hb-ot-tag.obj
 0002:0001c57c       ??_C@_03JEELCJ@pro@        00000001800c757c     hb-ot-tag.obj
 0002:0001c580       ??_C@_03PCCGKMAO@quh@      00000001800c7580     hb-ot-tag.obj
 0002:0001c584       ??_C@_03OJHLCDBG@qvi@      00000001800c7584     hb-ot-tag.obj
 0002:0001c588       ??_C@_03PBKCHIGA@qwh@      00000001800c7588     hb-ot-tag.obj
 0002:0001c58c       ??_C@_03MJIKGKMO@raj@      00000001800c758c     hb-ot-tag.obj
 0002:0001c590       ??_C@_02LFKOONLL@ro@       00000001800c7590     hb-ot-tag.obj
 0002:0001c594       ??_C@_03IMFFNBAD@rom@      00000001800c7594     hb-ot-tag.obj
 0002:0001c598       ??_C@_03JGEPKINC@sga@      00000001800c7598     hb-ot-tag.obj
 0002:0001c59c       ??_C@_02ELAAOLJA@sr@       00000001800c759c     hb-ot-tag.obj
 0002:0001c5a0       ??_C@_03KNGLMNJH@xnj@      00000001800c75a0     hb-ot-tag.obj
 0002:0001c5a4       ??_C@_03OBBIGHDK@syr@      00000001800c75a4     hb-ot-tag.obj
 0002:0001c5a8       ??_C@_08IEBDNIIN@und?9Syre@ 00000001800c75a8     hb-ot-tag.obj
 0002:0001c5b8       ??_C@_08DILMEEC@und?9Syrj@ 00000001800c75b8     hb-ot-tag.obj
 0002:0001c5c8       ??_C@_08GHOHABEG@und?9Syrn@ 00000001800c75c8     hb-ot-tag.obj
 0002:0001c5d4       ??_C@_03NHMNKOPE@tmh@      00000001800c75d4     hb-ot-tag.obj
 0002:0001c5d8       ??_C@_03MDOLKBCN@xwo@      00000001800c75d8     hb-ot-tag.obj
 0002:0001c5dc       ??_C@_03CMNOGHMI@wdt@      00000001800c75dc     hb-ot-tag.obj
 0002:0001c5e0       ??_C@_03IIANKNDA@wyn@      00000001800c75e0     hb-ot-tag.obj
 0002:0001c5e4       ??_C@_05HCJKHBCC@zh?9HK@   00000001800c75e4     hb-ot-tag.obj
 0002:0001c5f0       ??_C@_07JGEPGFF@zh?9Hans@  00000001800c75f0     hb-ot-tag.obj
 0002:0001c5f8       ??_C@_07EGCFGAJC@zh?9Hant@ 00000001800c75f8     hb-ot-tag.obj
 0002:0001c600       ??_C@_05BADNHGMN@zh?9MO@   00000001800c7600     hb-ot-tag.obj
 0002:0001c608       ??_C@_03PPLJNHHL@zza@      00000001800c7608     hb-ot-tag.obj
 0002:0001c60c       ??_C@_05NFAFKFNN@?9hbsc@   00000001800c760c     hb-ot-tag.obj
 0002:0001c614       ??_C@_05MFLKHLFP@?9hbot@   00000001800c7614     hb-ot-tag.obj
 0002:0001c620       ??_C@_0M@MFILKOCI@x?9hbot?9?$CF08x@ 00000001800c7620     hb-ot-tag.obj
 0002:0001c62c       __real@46800000            00000001800c762c     hb-ot-var.obj
 0002:0001c630       __real@bf700000            00000001800c7630     hb-outline.obj
 0002:0001c634       __real@bf800000            00000001800c7634     hb-paint-extents.obj
 0002:0001c640       ??_C@_08LFBOCJLE@fallback@ 00000001800c7640     hb-shape-plan.obj
 0002:0001c650       ??_C@_0DF@MPFFHONM@face?$DN?$CFp?5num_features?$DN?$CFu?5num_coo@ 00000001800c7650     hb-shape-plan.obj
 0002:0001c690       ??_C@_0MH@MMALGGGN@struct?5hb_shape_plan_t?5?$CK__cdecl@ 00000001800c7690     hb-shape-plan.obj
 0002:0001c758       ??_C@_0L@HJBOBLCO@SHAPE_PLAN@ 00000001800c7758     hb-shape-plan.obj
 0002:0001c768       ??_C@_0CP@GAFDBLDO@num_features?$DN?$CFu?5shaper_func?$DN?$CFp?0@ 00000001800c7768     hb-shape-plan.obj
 0002:0001c7a0       ??_C@_0JI@JOJJJOPA@bool?5__cdecl?5_hb_shape_plan_exe@ 00000001800c77a0     hb-shape-plan.obj
 0002:0001c838       ??_C@_0CH@EAKAEIJM@face?$DN?$CFp?5num_features?$DN?$CFu?5shaper_@ 00000001800c7838     hb-shape-plan.obj
 0002:0001c860       ??_C@_0MO@MGHFPDJG@struct?5hb_shape_plan_t?5?$CK__cdecl@ 00000001800c7860     hb-shape-plan.obj
 0002:0001c968       ??_C@_0P@GEOKODDH@HB_SHAPER_LIST@ 00000001800c7968     hb-shaper.obj
 0002:00028bb0       ?_hb_modified_combining_class@@3QBEB 00000001800d3bb0     hb-unicode.obj
 0002:00028e80       ??_C@_0BG@NKHBBPH@sun?1font?1TrueTypeFont@ 00000001800d3e80     sunFont.obj
 0002:00028e98       ??_C@_0BL@GAAGJDLL@?$CILjava?1nio?1ByteBuffer?$DLII?$CJI@ 00000001800d3e98     sunFont.obj
 0002:00028eb8       ??_C@_09CKAKNPHP@readBlock@ 00000001800d3eb8     sunFont.obj
 0002:00028ec4       ??_C@_06JMOJDKIE@?$CIII?$CJ?$FLB@ 00000001800d3ec4     sunFont.obj
 0002:00028ed0       ??_C@_09IDIEPDPI@readBytes@ 00000001800d3ed0     sunFont.obj
 0002:00028ee0       ??_C@_0BD@OPLCIPMH@sun?1font?1Type1Font@ 00000001800d3ee0     sunFont.obj
 0002:00028ef8       ??_C@_0BJ@LMHMPPKE@?$CILjava?1nio?1ByteBuffer?$DL?$CJV@ 00000001800d3ef8     sunFont.obj
 0002:00028f18       ??_C@_08CJNGBMAG@readFile@ 00000001800d3f18     sunFont.obj
 0002:00028f28       ??_C@_0BM@DGICEJAA@java?1awt?1geom?1Point2D$Float@ 00000001800d3f28     sunFont.obj
 0002:00028f44       ??_C@_05BHHDPELC@?$CIFF?$CJV@ 00000001800d3f44     sunFont.obj
 0002:00028f4c       ??_C@_01BIAFAFID@F@        00000001800d3f4c     sunFont.obj
 0002:00028f50       ??_C@_01FJMABOPO@x@        00000001800d3f50     sunFont.obj
 0002:00028f54       ??_C@_01EANLCPLP@y@        00000001800d3f54     sunFont.obj
 0002:00028f58       ??_C@_0BH@ENELCGL@sun?1font?1StrikeMetrics@ 00000001800d3f58     sunFont.obj
 0002:00028f70       ??_C@_0O@LBAHCNJL@?$CIFFFFFFFFFF?$CJV@ 00000001800d3f70     sunFont.obj
 0002:00028f80       ??_C@_0CA@PDMBNICK@java?1awt?1geom?1Rectangle2D$Float@ 00000001800d3f80     sunFont.obj
 0002:00028fa0       ??_C@_07PMCFNNPC@?$CIFFFF?$CJV@ 00000001800d3fa0     sunFont.obj
 0002:00028fa8       ??_C@_05IGKADHGO@width@    00000001800d3fa8     sunFont.obj
 0002:00028fb0       ??_C@_06LNLHEAAG@height@   00000001800d3fb0     sunFont.obj
 0002:00028fb8       ??_C@_0BK@COJNCHEM@java?1awt?1geom?1GeneralPath@ 00000001800d3fb8     sunFont.obj
 0002:00028fd8       ??_C@_0L@MDPODKN@?$CII?$FLBI?$FLFI?$CJV@ 00000001800d3fd8     sunFont.obj
 0002:00028fe8       ??_C@_0BA@OKNBFGCN@sun?1font?1Font2D@ 00000001800d3fe8     sunFont.obj
 0002:00028ff8       ??_C@_04DIFHPCLD@?$CII?$CJI@ 00000001800d3ff8     sunFont.obj
 0002:00029000       ??_C@_0P@JJDMFJPG@charToGlyphRaw@ 00000001800d4000     sunFont.obj
 0002:00029010       ??_C@_05BKHNKL@?$CIII?$CJI@ 00000001800d4010     sunFont.obj
 0002:00029018       ??_C@_0BI@IPDJMKHN@charToVariationGlyphRaw@ 00000001800d4018     sunFont.obj
 0002:00029030       ??_C@_0BP@CBNLOFNN@?$CI?$CJLsun?1font?1CharToGlyphMapper?$DL@ 00000001800d4030     sunFont.obj
 0002:00029050       ??_C@_09DGCMEJKL@getMapper@ 00000001800d4050     sunFont.obj
 0002:0002905c       ??_C@_05IPLNOPFN@?$CII?$CJ?$FLB@ 00000001800d405c     sunFont.obj
 0002:00029068       ??_C@_0O@DBNIPDIH@getTableBytes@ 00000001800d4068     sunFont.obj
 0002:00029078       ??_C@_04DGAFFDEF@?$CIC?$CJZ@ 00000001800d4078     sunFont.obj
 0002:00029080       ??_C@_0L@PGEPPKMA@canDisplay@ 00000001800d4080     sunFont.obj
 0002:00029090       ??_C@_0BL@GAPGNAAC@sun?1font?1CharToGlyphMapper@ 00000001800d4090     sunFont.obj
 0002:000290b0       ??_C@_0M@NMGOHDEJ@charToGlyph@ 00000001800d40b0     sunFont.obj
 0002:000290c0       ??_C@_0BI@GDBHNKM@sun?1font?1PhysicalStrike@ 00000001800d40c0     sunFont.obj
 0002:000290d8       ??_C@_0CB@IBGFEOCM@?$CII?$CJLjava?1awt?1geom?1Point2D$Float@ 00000001800d40d8     sunFont.obj
 0002:00029100       ??_C@_0BA@FMKHNFIF@getGlyphMetrics@ 00000001800d4100     sunFont.obj
 0002:00029110       ??_C@_0CC@IBLMDHKA@?$CIII?$CJLjava?1awt?1geom?1Point2D$Floa@ 00000001800d4110     sunFont.obj
 0002:00029138       ??_C@_0O@NHLNHECD@getGlyphPoint@ 00000001800d4138     sunFont.obj
 0002:00029148       ??_C@_0CB@CONGGNHA@?$CILjava?1awt?1geom?1Point2D$Float?$DL?$CJ@ 00000001800d4148     sunFont.obj
 0002:00029170       ??_C@_0M@MJABIGBP@adjustPoint@ 00000001800d4170     sunFont.obj
 0002:0002917c       ??_C@_01LELAEKIP@J@        00000001800d417c     sunFont.obj
 0002:00029180       ??_C@_0P@DPIICNJB@pScalerContext@ 00000001800d4180     sunFont.obj
 0002:00029190       ??_C@_0BD@LPHBDEDB@sun?1font?1GlyphList@ 00000001800d4190     sunFont.obj
 0002:000291a4       ??_C@_05HAAKEDND@gposx@    00000001800d41a4     sunFont.obj
 0002:000291ac       ??_C@_05GJBBHCJC@gposy@    00000001800d41ac     sunFont.obj
 0002:000291b4       ??_C@_03BKCJCHLK@len@      00000001800d41b4     sunFont.obj
 0002:000291b8       ??_C@_02GKMBEADD@?$FLJ@    00000001800d41b8     sunFont.obj
 0002:000291bc       ??_C@_06IAHKIHIK@images@   00000001800d41bc     sunFont.obj
 0002:000291c4       ??_C@_01POHCFINO@Z@        00000001800d41c4     sunFont.obj
 0002:000291c8       ??_C@_0N@CLHDJEN@usePositions@ 00000001800d41c8     sunFont.obj
 0002:000291d8       ??_C@_09HEJILCIA@positions@ 00000001800d41d8     sunFont.obj
 0002:000291e8       ??_C@_0M@IOGNPDID@lcdRGBOrder@ 00000001800d41e8     sunFont.obj
 0002:000291f8       ??_C@_0N@OIMCCICM@lcdSubPixPos@ 00000001800d41f8     sunFont.obj
 0002:00029218       _pDefaultRawDllMain        00000001800d4218     MSVCRT:dll_dllmain.obj
 0002:00029218       _pRawDllMain               00000001800d4218     MSVCRT:dll_dllmain.obj
 0002:00029220       _load_config_used          00000001800d4220     MSVCRT:loadcfg.obj
 0002:00029400       __volatile_metadata        00000001800d4400     <linker-defined>
 0002:0002a3f0       __rtc_iaa                  00000001800d53f0     MSVCRT:initsect.obj
 0002:0002a3f8       __rtc_izz                  00000001800d53f8     MSVCRT:initsect.obj
 0002:0002a400       __rtc_taa                  00000001800d5400     MSVCRT:initsect.obj
 0002:0002a408       __rtc_tzz                  00000001800d5408     MSVCRT:initsect.obj
 0002:00034bd0       __IMPORT_DESCRIPTOR_awt    00000001800dfbd0     awt:awt.dll
 0002:00034be4       __IMPORT_DESCRIPTOR_java   00000001800dfbe4     java:java.dll
 0002:00034bf8       __IMPORT_DESCRIPTOR_freetype 00000001800dfbf8     freetype:freetype.dll
 0002:00034c0c       __IMPORT_DESCRIPTOR_ADVAPI32 00000001800dfc0c     advapi32:ADVAPI32.dll
 0002:00034c20       __IMPORT_DESCRIPTOR_GDI32  00000001800dfc20     gdi32:GDI32.dll
 0002:00034c34       __IMPORT_DESCRIPTOR_USER32 00000001800dfc34     user32:USER32.dll
 0002:00034c48       __IMPORT_DESCRIPTOR_KERNEL32 00000001800dfc48     kernel32:KERNEL32.dll
 0002:00034c5c       __IMPORT_DESCRIPTOR_VCRUNTIME140 00000001800dfc5c     vcruntime:VCRUNTIME140.dll
 0002:00034c70       __IMPORT_DESCRIPTOR_api-ms-win-crt-heap-l1-1-0 00000001800dfc70     ucrt:api-ms-win-crt-heap-l1-1-0.dll
 0002:00034c84       __IMPORT_DESCRIPTOR_api-ms-win-crt-math-l1-1-0 00000001800dfc84     ucrt:api-ms-win-crt-math-l1-1-0.dll
 0002:00034c98       __IMPORT_DESCRIPTOR_api-ms-win-crt-environment-l1-1-0 00000001800dfc98     ucrt:api-ms-win-crt-environment-l1-1-0.dll
 0002:00034cac       __IMPORT_DESCRIPTOR_api-ms-win-crt-convert-l1-1-0 00000001800dfcac     ucrt:api-ms-win-crt-convert-l1-1-0.dll
 0002:00034cc0       __IMPORT_DESCRIPTOR_api-ms-win-crt-stdio-l1-1-0 00000001800dfcc0     ucrt:api-ms-win-crt-stdio-l1-1-0.dll
 0002:00034cd4       __IMPORT_DESCRIPTOR_api-ms-win-crt-string-l1-1-0 00000001800dfcd4     ucrt:api-ms-win-crt-string-l1-1-0.dll
 0002:00034ce8       __IMPORT_DESCRIPTOR_api-ms-win-crt-runtime-l1-1-0 00000001800dfce8     ucrt:api-ms-win-crt-runtime-l1-1-0.dll
 0002:00034cfc       __NULL_IMPORT_DESCRIPTOR   00000001800dfcfc     awt:awt.dll
 0003:00000000       defaultGammaLUT            00000001800e1000     DrawGlyphList.obj
 0003:00000100       defaultInvGammaLUT         00000001800e1100     DrawGlyphList.obj
 0003:00000230       ?_hb_Null_hb_buffer_t@@3Uhb_buffer_t@@B 00000001800e1230     hb-buffer.obj
 0003:00000320       ?endchar_str@@3PEBEEB      00000001800e1320     hb-common.obj
 0003:00000330       ?_hb_Null_hb_draw_funcs_t@@3Uhb_draw_funcs_t@@B 00000001800e1330     hb-draw.obj
 0003:00000380       ?_hb_Null_hb_face_t@@3Uhb_face_t@@B 00000001800e1380     hb-face.obj
 0003:00000560       ?_hb_Null_hb_font_funcs_t@@3Uhb_font_funcs_t@@B 00000001800e1560     hb-font.obj
 0003:00000620       ?_hb_Null_hb_font_t@@3Uhb_font_t@@B 00000001800e1620     hb-font.obj
 0003:00000860       ?_hb_Null_hb_paint_funcs_t@@3Uhb_paint_funcs_t@@B 00000001800e1860     hb-paint.obj
 0003:000008f0       ?_hb_Null_hb_unicode_funcs_t@@3Uhb_unicode_funcs_t@@B 00000001800e18f0     hb-unicode.obj
 0003:000009d0       MAX_ICU_SCRIPTCODE         00000001800e19d0     scriptMapping.obj
 0003:000009e0       ICU_to_Harfbuzz_ScriptCode 00000001800e19e0     scriptMapping.obj
 0003:00000aa0       __security_cookie          00000001800e1aa0     MSVCRT:gs_cookie.obj
 0003:00000aa8       __security_cookie_complement 00000001800e1aa8     MSVCRT:gs_cookie.obj
 0003:00000ab0       _fltused                   00000001800e1ab0     MSVCRT:fltused.obj
 0003:00000ac0       __isa_available            00000001800e1ac0     MSVCRT:cpu_disp.obj
 0003:00000ac4       __isa_enabled              00000001800e1ac4     MSVCRT:cpu_disp.obj
 0003:00000ac8       __memset_fast_string_threshold 00000001800e1ac8     MSVCRT:cpu_disp.obj
 0003:00000ad0       __memset_nt_threshold      00000001800e1ad0     MSVCRT:cpu_disp.obj
 0003:00000ae0       __scrt_native_dllmain_reason 00000001800e1ae0     MSVCRT:utility.obj
 0003:00000af0       __scrt_ucrt_dll_is_in_use  00000001800e1af0     MSVCRT:ucrt_stubs.obj
 0003:00000b58       ?_OptionsStorage@?1??__local_stdio_printf_options@@9@4_KA 00000001800e1b58     hb-buffer-serialize.obj
 0003:00000b60       ?_hb_CrapPool@@3PA_KA      00000001800e1b60     hb-common.obj
 0003:00000de0       ?_hb_options@@3U?$hb_atomic_t@I@@A 00000001800e1de0     hb-common.obj
 0003:000017b4       __favor                    00000001800e27b4     MSVCRT:cpu_disp.obj
 0003:000017c0       ?__type_info_root_node@@3U__type_info_node@@A 00000001800e27c0     MSVCRT:tncleanup.obj
 0003:000017d0       ?_OptionsStorage@?1??__local_stdio_scanf_options@@9@4_KA 00000001800e27d0     MSVCRT:default_local_stdio_options.obj
 0003:000017d8       __scrt_current_native_startup_state 00000001800e27d8     MSVCRT:utility.obj
 0003:000017e0       __scrt_native_startup_lock 00000001800e27e0     MSVCRT:utility.obj
 0003:00001820       __scrt_debugger_hook_flag  00000001800e2820     MSVCRT:utility_desktop.obj
 0003:00001840       sunFontIDs                 00000001800e2840     <common>
 0003:00001980       lcdInvGammaLUT             00000001800e2980     <common>
 0003:00001e40       lcdGammaLUT                00000001800e2e40     <common>
 0003:000022f8       __dyn_tls_init_callback    00000001800e32f8     <common>

 entry point at        0001:000a8934

 Static symbols

 0000:fff11000       .debug$S                   0000000180000000     fontmanager.exp
 0000:fff11000       .debug$S                   0000000180000000     advapi32:ADVAPI32.dll
 0000:fff11000       .debug$S                   0000000180000000     advapi32:ADVAPI32.dll
 0000:fff11000       .debug$S                   0000000180000000     advapi32:ADVAPI32.dll
 0000:fff11000       .debug$S                   0000000180000000     advapi32:ADVAPI32.dll
 0000:fff11000       .debug$S                   0000000180000000     gdi32:GDI32.dll
 0000:fff11000       .debug$S                   0000000180000000     gdi32:GDI32.dll
 0000:fff11000       .debug$S                   0000000180000000     gdi32:GDI32.dll
 0000:fff11000       .debug$S                   0000000180000000     gdi32:GDI32.dll
 0000:fff11000       .debug$S                   0000000180000000     gdi32:GDI32.dll
 0000:fff11000       .debug$S                   0000000180000000     gdi32:GDI32.dll
 0000:fff11000       .debug$S                   0000000180000000     gdi32:GDI32.dll
 0000:fff11000       .debug$S                   0000000180000000     gdi32:GDI32.dll
 0000:fff11000       .debug$S                   0000000180000000     gdi32:GDI32.dll
 0000:fff11000       .debug$S                   0000000180000000     gdi32:GDI32.dll
 0000:fff11000       .debug$S                   0000000180000000     gdi32:GDI32.dll
 0000:fff11000       .debug$S                   0000000180000000     gdi32:GDI32.dll
 0000:fff11000       .debug$S                   0000000180000000     gdi32:GDI32.dll
 0000:fff11000       .debug$S                   0000000180000000     gdi32:GDI32.dll
 0000:fff11000       .debug$S                   0000000180000000     gdi32:GDI32.dll
 0000:fff11000       .debug$S                   0000000180000000     gdi32:GDI32.dll
 0000:fff11000       .debug$S                   0000000180000000     kernel32:KERNEL32.dll
 0000:fff11000       .debug$S                   0000000180000000     kernel32:KERNEL32.dll
 0000:fff11000       .debug$S                   0000000180000000     kernel32:KERNEL32.dll
 0000:fff11000       .debug$S                   0000000180000000     kernel32:KERNEL32.dll
 0000:fff11000       .debug$S                   0000000180000000     kernel32:KERNEL32.dll
 0000:fff11000       .debug$S                   0000000180000000     kernel32:KERNEL32.dll
 0000:fff11000       .debug$S                   0000000180000000     kernel32:KERNEL32.dll
 0000:fff11000       .debug$S                   0000000180000000     kernel32:KERNEL32.dll
 0000:fff11000       .debug$S                   0000000180000000     kernel32:KERNEL32.dll
 0000:fff11000       .debug$S                   0000000180000000     kernel32:KERNEL32.dll
 0000:fff11000       .debug$S                   0000000180000000     kernel32:KERNEL32.dll
 0000:fff11000       .debug$S                   0000000180000000     kernel32:KERNEL32.dll
 0000:fff11000       .debug$S                   0000000180000000     kernel32:KERNEL32.dll
 0000:fff11000       .debug$S                   0000000180000000     kernel32:KERNEL32.dll
 0000:fff11000       .debug$S                   0000000180000000     kernel32:KERNEL32.dll
 0000:fff11000       .debug$S                   0000000180000000     kernel32:KERNEL32.dll
 0000:fff11000       .debug$S                   0000000180000000     kernel32:KERNEL32.dll
 0000:fff11000       .debug$S                   0000000180000000     kernel32:KERNEL32.dll
 0000:fff11000       .debug$S                   0000000180000000     kernel32:KERNEL32.dll
 0000:fff11000       .debug$S                   0000000180000000     kernel32:KERNEL32.dll
 0000:fff11000       .debug$S                   0000000180000000     kernel32:KERNEL32.dll
 0000:fff11000       .debug$S                   0000000180000000     kernel32:KERNEL32.dll
 0000:fff11000       .debug$S                   0000000180000000     kernel32:KERNEL32.dll
 0000:fff11000       .debug$S                   0000000180000000     kernel32:KERNEL32.dll
 0000:fff11000       .debug$S                   0000000180000000     kernel32:KERNEL32.dll
 0000:fff11000       .debug$S                   0000000180000000     kernel32:KERNEL32.dll
 0000:fff11000       .debug$S                   0000000180000000     kernel32:KERNEL32.dll
 0000:fff11000       .debug$S                   0000000180000000     kernel32:KERNEL32.dll
 0000:fff11000       .debug$S                   0000000180000000     kernel32:KERNEL32.dll
 0000:fff11000       .debug$S                   0000000180000000     kernel32:KERNEL32.dll
 0000:fff11000       .debug$S                   0000000180000000     ucrt:api-ms-win-crt-convert-l1-1-0.dll
 0000:fff11000       .debug$S                   0000000180000000     ucrt:api-ms-win-crt-convert-l1-1-0.dll
 0000:fff11000       .debug$S                   0000000180000000     ucrt:api-ms-win-crt-convert-l1-1-0.dll
 0000:fff11000       .debug$S                   0000000180000000     ucrt:api-ms-win-crt-environment-l1-1-0.dll
 0000:fff11000       .debug$S                   0000000180000000     ucrt:api-ms-win-crt-heap-l1-1-0.dll
 0000:fff11000       .debug$S                   0000000180000000     ucrt:api-ms-win-crt-heap-l1-1-0.dll
 0000:fff11000       .debug$S                   0000000180000000     ucrt:api-ms-win-crt-heap-l1-1-0.dll
 0000:fff11000       .debug$S                   0000000180000000     ucrt:api-ms-win-crt-heap-l1-1-0.dll
 0000:fff11000       .debug$S                   0000000180000000     ucrt:api-ms-win-crt-math-l1-1-0.dll
 0000:fff11000       .debug$S                   0000000180000000     ucrt:api-ms-win-crt-math-l1-1-0.dll
 0000:fff11000       .debug$S                   0000000180000000     ucrt:api-ms-win-crt-math-l1-1-0.dll
 0000:fff11000       .debug$S                   0000000180000000     ucrt:api-ms-win-crt-math-l1-1-0.dll
 0000:fff11000       .debug$S                   0000000180000000     ucrt:api-ms-win-crt-math-l1-1-0.dll
 0000:fff11000       .debug$S                   0000000180000000     ucrt:api-ms-win-crt-math-l1-1-0.dll
 0000:fff11000       .debug$S                   0000000180000000     ucrt:api-ms-win-crt-math-l1-1-0.dll
 0000:fff11000       .debug$S                   0000000180000000     ucrt:api-ms-win-crt-math-l1-1-0.dll
 0000:fff11000       .debug$S                   0000000180000000     ucrt:api-ms-win-crt-math-l1-1-0.dll
 0000:fff11000       .debug$S                   0000000180000000     ucrt:api-ms-win-crt-runtime-l1-1-0.dll
 0000:fff11000       .debug$S                   0000000180000000     ucrt:api-ms-win-crt-runtime-l1-1-0.dll
 0000:fff11000       .debug$S                   0000000180000000     ucrt:api-ms-win-crt-runtime-l1-1-0.dll
 0000:fff11000       .debug$S                   0000000180000000     ucrt:api-ms-win-crt-runtime-l1-1-0.dll
 0000:fff11000       .debug$S                   0000000180000000     ucrt:api-ms-win-crt-runtime-l1-1-0.dll
 0000:fff11000       .debug$S                   0000000180000000     ucrt:api-ms-win-crt-runtime-l1-1-0.dll
 0000:fff11000       .debug$S                   0000000180000000     ucrt:api-ms-win-crt-runtime-l1-1-0.dll
 0000:fff11000       .debug$S                   0000000180000000     ucrt:api-ms-win-crt-runtime-l1-1-0.dll
 0000:fff11000       .debug$S                   0000000180000000     ucrt:api-ms-win-crt-runtime-l1-1-0.dll
 0000:fff11000       .debug$S                   0000000180000000     ucrt:api-ms-win-crt-runtime-l1-1-0.dll
 0000:fff11000       .debug$S                   0000000180000000     ucrt:api-ms-win-crt-runtime-l1-1-0.dll
 0000:fff11000       .debug$S                   0000000180000000     ucrt:api-ms-win-crt-runtime-l1-1-0.dll
 0000:fff11000       .debug$S                   0000000180000000     ucrt:api-ms-win-crt-runtime-l1-1-0.dll
 0000:fff11000       .debug$S                   0000000180000000     ucrt:api-ms-win-crt-stdio-l1-1-0.dll
 0000:fff11000       .debug$S                   0000000180000000     ucrt:api-ms-win-crt-stdio-l1-1-0.dll
 0000:fff11000       .debug$S                   0000000180000000     ucrt:api-ms-win-crt-stdio-l1-1-0.dll
 0000:fff11000       .debug$S                   0000000180000000     ucrt:api-ms-win-crt-stdio-l1-1-0.dll
 0000:fff11000       .debug$S                   0000000180000000     ucrt:api-ms-win-crt-stdio-l1-1-0.dll
 0000:fff11000       .debug$S                   0000000180000000     ucrt:api-ms-win-crt-stdio-l1-1-0.dll
 0000:fff11000       .debug$S                   0000000180000000     ucrt:api-ms-win-crt-stdio-l1-1-0.dll
 0000:fff11000       .debug$S                   0000000180000000     ucrt:api-ms-win-crt-stdio-l1-1-0.dll
 0000:fff11000       .debug$S                   0000000180000000     ucrt:api-ms-win-crt-string-l1-1-0.dll
 0000:fff11000       .debug$S                   0000000180000000     ucrt:api-ms-win-crt-string-l1-1-0.dll
 0000:fff11000       .debug$S                   0000000180000000     ucrt:api-ms-win-crt-string-l1-1-0.dll
 0000:fff11000       .debug$S                   0000000180000000     ucrt:api-ms-win-crt-string-l1-1-0.dll
 0000:fff11000       .debug$S                   0000000180000000     ucrt:api-ms-win-crt-string-l1-1-0.dll
 0000:fff11000       .debug$S                   0000000180000000     user32:USER32.dll
 0000:fff11000       .debug$S                   0000000180000000     user32:USER32.dll
 0000:fff11000       .debug$S                   0000000180000000     user32:USER32.dll
 0000:fff11000       .debug$S                   0000000180000000     user32:USER32.dll
 0000:fff11000       .debug$S                   0000000180000000     user32:USER32.dll
 0000:fff11000       .debug$S                   0000000180000000     user32:USER32.dll
 0000:fff11000       .debug$S                   0000000180000000     vcruntime:VCRUNTIME140.dll
 0000:fff11000       .debug$S                   0000000180000000     vcruntime:VCRUNTIME140.dll
 0000:fff11000       .debug$S                   0000000180000000     vcruntime:VCRUNTIME140.dll
 0000:fff11000       .debug$S                   0000000180000000     vcruntime:VCRUNTIME140.dll
 0000:fff11000       .debug$S                   0000000180000000     vcruntime:VCRUNTIME140.dll
 0000:fff11000       .debug$S                   0000000180000000     vcruntime:VCRUNTIME140.dll
 0000:fff11000       .debug$S                   0000000180000000     vcruntime:VCRUNTIME140.dll
 0000:fff11000       .debug$S                   0000000180000000     vcruntime:VCRUNTIME140.dll
 0000:fff11000       .debug$S                   0000000180000000     vcruntime:VCRUNTIME140.dll
 0000:fff11000       .debug$S                   0000000180000000     vcruntime:VCRUNTIME140.dll
 0000:fff11000       .debug$S                   0000000180000000     vcruntime:VCRUNTIME140.dll
 0000:fff11000       .debug$S                   0000000180000000     vcruntime:VCRUNTIME140.dll
 0000:fff11000       .debug$S                   0000000180000000     vcruntime:VCRUNTIME140.dll
 0000:fff11000       .debug$S                   0000000180000000     java:java.dll
 0000:fff11000       .debug$S                   0000000180000000     java:java.dll
 0000:fff11000       .debug$S                   0000000180000000     java:java.dll
 0000:fff11000       .debug$S                   0000000180000000     java:java.dll
 0000:fff11000       .debug$S                   0000000180000000     java:java.dll
 0000:fff11000       .debug$S                   0000000180000000     awt:awt.dll
 0000:fff11000       .debug$S                   0000000180000000     awt:awt.dll
 0000:fff11000       .debug$S                   0000000180000000     awt:awt.dll
 0000:fff11000       .debug$S                   0000000180000000     awt:awt.dll
 0000:fff11000       .debug$S                   0000000180000000     awt:awt.dll
 0000:fff11000       .debug$S                   0000000180000000     awt:awt.dll
 0000:fff11000       .debug$S                   0000000180000000     awt:awt.dll
 0000:fff11000       .debug$S                   0000000180000000     awt:awt.dll
 0000:fff11000       .debug$S                   0000000180000000     awt:awt.dll
 0000:fff11000       .debug$S                   0000000180000000     awt:awt.dll
 0000:fff11000       .debug$S                   0000000180000000     freetype:freetype.dll
 0000:fff11000       .debug$S                   0000000180000000     freetype:freetype.dll
 0000:fff11000       .debug$S                   0000000180000000     freetype:freetype.dll
 0000:fff11000       .debug$S                   0000000180000000     freetype:freetype.dll
 0000:fff11000       .debug$S                   0000000180000000     freetype:freetype.dll
 0000:fff11000       .debug$S                   0000000180000000     freetype:freetype.dll
 0000:fff11000       .debug$S                   0000000180000000     freetype:freetype.dll
 0000:fff11000       .debug$S                   0000000180000000     freetype:freetype.dll
 0000:fff11000       .debug$S                   0000000180000000     freetype:freetype.dll
 0000:fff11000       .debug$S                   0000000180000000     freetype:freetype.dll
 0000:fff11000       .debug$S                   0000000180000000     freetype:freetype.dll
 0000:fff11000       .debug$S                   0000000180000000     freetype:freetype.dll
 0000:fff11000       .debug$S                   0000000180000000     freetype:freetype.dll
 0000:fff11000       .debug$S                   0000000180000000     freetype:freetype.dll
 0000:fff11000       .debug$S                   0000000180000000     freetype:freetype.dll
 0000:fff11000       .debug$S                   0000000180000000     freetype:freetype.dll
 0000:fff11000       .debug$S                   0000000180000000     freetype:freetype.dll
 0000:fff11000       .debug$S                   0000000180000000     freetype:freetype.dll
 0000:fff11000       .debug$S                   0000000180000000     freetype:freetype.dll
 0000:fff11000       .debug$S                   0000000180000000     freetype:freetype.dll
 0001:00000000       Glyph_GetRasInfo           0000000180001000 f   ColorGlyphSurfaceData.obj
 0001:00000030       Glyph_Lock                 0000000180001030 f   ColorGlyphSurfaceData.obj
 0001:00000450       drawGlyphList              0000000180001450 f   DrawGlyphList.obj
 0001:00000600       drawGlyphListLCD           0000000180001600 f   DrawGlyphList.obj
 0001:000018a0       euclidianDistance          00000001800028a0 f   HBShaper.obj
 0001:00002540       CheckFontFamilyProcW       0000000180003540 f   fontpath.obj
 0001:00002580       EnumFamilyNamesW           0000000180003580 f   fontpath.obj
 0001:000028c0       EnumFontFacesInFamilyProcW 00000001800038c0 f   fontpath.obj
 0001:000030e0       populateFontFileNameFromRegistryKey 00000001800040e0 f   fontpath.obj
 0001:00003390       registerFontW              0000000180004390 f   fontpath.obj
 0001:00003640       moveTo                     0000000180004640 f   freetypeScaler.obj
 0001:000036c0       lineTo                     00000001800046c0 f   freetypeScaler.obj
 0001:00003720       conicTo                    0000000180004720 f   freetypeScaler.obj
 0001:000037d0       cubicTo                    00000001800047d0 f   freetypeScaler.obj
 0001:000038d0       CopyBW2Grey8               00000001800048d0 f   freetypeScaler.obj
 0001:00003a00       GlyphSlot_Embolden         0000000180004a00 f   freetypeScaler.obj
 0001:00004960       ?hb_font_draw_glyph_or_fail_nil@@YAHPEAUhb_font_t@@PEAXIPEAUhb_draw_funcs_t@@11@Z 0000000180005960 f   hb-font.obj
 0001:00004960       ?hb_font_get_glyph_h_kerning_nil@@YAHPEAUhb_font_t@@PEAXII1@Z 0000000180005960 f   hb-font.obj
 0001:00004960       ?hb_font_get_glyph_v_kerning_nil@@YAHPEAUhb_font_t@@PEAXII1@Z 0000000180005960 f   hb-font.obj
 0001:00004960       ?hb_font_paint_glyph_or_fail_nil@@YAHPEAUhb_font_t@@PEAXIPEAUhb_paint_funcs_t@@1II1@Z 0000000180005960 f   hb-font.obj
 0001:00004960       ?hb_jdk_get_glyph_extents@@YAHPEAUhb_font_t@@PEAXIPEAUhb_glyph_extents_t@@1@Z 0000000180005960 f   hb-jdk-font-p.obj
 0001:00004960       ?hb_jdk_get_glyph_from_name@@YAHPEAUhb_font_t@@PEAXPEBDHPEAI1@Z 0000000180005960 f   hb-jdk-font-p.obj
 0001:00004960       ?hb_jdk_get_glyph_h_kerning@@YAHPEAUhb_font_t@@PEAXII1@Z 0000000180005960 f   hb-jdk-font-p.obj
 0001:00004960       ?hb_jdk_get_glyph_name@@YAHPEAUhb_font_t@@PEAXIPEADI1@Z 0000000180005960 f   hb-jdk-font-p.obj
 0001:00004960       ?hb_jdk_get_glyph_v_kerning@@YAHPEAUhb_font_t@@PEAXII1@Z 0000000180005960 f   hb-jdk-font-p.obj
 0001:00004960       ?hb_jdk_get_glyph_v_origin@@YAHPEAUhb_font_t@@PEAXIPEAH21@Z 0000000180005960 f   hb-jdk-font-p.obj
 0001:00004960       ?hb_jdk_get_glyph_extents@@YAHPEAUhb_font_t@@PEAXIPEAUhb_glyph_extents_t@@1@Z 0000000180005960 f   hb-jdk-font.obj
 0001:00004960       ?hb_jdk_get_glyph_from_name@@YAHPEAUhb_font_t@@PEAXPEBDHPEAI1@Z 0000000180005960 f   hb-jdk-font.obj
 0001:00004960       ?hb_jdk_get_glyph_h_kerning@@YAHPEAUhb_font_t@@PEAXII1@Z 0000000180005960 f   hb-jdk-font.obj
 0001:00004960       ?hb_jdk_get_glyph_name@@YAHPEAUhb_font_t@@PEAXIPEADI1@Z 0000000180005960 f   hb-jdk-font.obj
 0001:00004960       ?hb_jdk_get_glyph_v_kerning@@YAHPEAUhb_font_t@@PEAXII1@Z 0000000180005960 f   hb-jdk-font.obj
 0001:00004960       ?hb_jdk_get_glyph_v_origin@@YAHPEAUhb_font_t@@PEAXIPEAH21@Z 0000000180005960 f   hb-jdk-font.obj
 0001:00004960       ?hb_paint_color_glyph_nil@@YAHPEAUhb_paint_funcs_t@@PEAXIPEAUhb_font_t@@1@Z 0000000180005960 f   hb-paint.obj
 0001:00004960       ?hb_paint_custom_palette_color_nil@@YAHPEAUhb_paint_funcs_t@@PEAXIPEAI1@Z 0000000180005960 f   hb-paint.obj
 0001:00004960       ?hb_paint_image_nil@@YAHPEAUhb_paint_funcs_t@@PEAXPEAUhb_blob_t@@IIIMPEAUhb_glyph_extents_t@@1@Z 0000000180005960 f   hb-paint.obj
 0001:00004960       ?hb_unicode_combining_class_nil@@YA?AW4hb_unicode_combining_class_t@@PEAUhb_unicode_funcs_t@@IPEAX@Z 0000000180005960 f   hb-unicode.obj
 0001:00004960       ?hb_unicode_compose_nil@@YAHPEAUhb_unicode_funcs_t@@IIPEAIPEAX@Z 0000000180005960 f   hb-unicode.obj
 0001:00004960       ?hb_unicode_decompose_compatibility_nil@@YAIPEAUhb_unicode_funcs_t@@IPEAIPEAX@Z 0000000180005960 f   hb-unicode.obj
 0001:00004960       ?hb_unicode_decompose_nil@@YAHPEAUhb_unicode_funcs_t@@IPEAI1PEAX@Z 0000000180005960 f   hb-unicode.obj
 0001:00004d50       ReadTTFontFileFunc         0000000180005d50 f   freetypeScaler.obj
 0001:00004fa0       getFTOutline               0000000180005fa0 f   freetypeScaler.obj
 0001:00005090       getGlyphGeneralPath        0000000180006090 f   freetypeScaler.obj
 0001:00005290       getGlyphImageNativeInternal 0000000180006290 f   freetypeScaler.obj
 0001:000057c0       invalidateJavaScaler       00000001800067c0 f   freetypeScaler.obj
 0001:00005860       setupFTContext             0000000180006860 f   freetypeScaler.obj
 0001:00005950       ??$_hb_debug_msg@$0A@@@YAXPEBDPEBX0_NIH0ZZ 0000000180006950 f   hb-aat-layout.obj
 0001:00005950       ??$_hb_debug_msg@$0A@@@YAXPEBDPEBX0_NIH0ZZ 0000000180006950 f   hb-blob.obj
 0001:00005950       ??$_hb_debug_msg@$0A@@@YAXPEBDPEBX0_NIH0ZZ 0000000180006950 f   hb-common.obj
 0001:00005950       ?hb_draw_close_path_nil@@YAXPEAUhb_draw_funcs_t@@PEAXPEAUhb_draw_state_t@@1@Z 0000000180006950 f   hb-draw.obj
 0001:00005950       ?hb_draw_cubic_to_nil@@YAXPEAUhb_draw_funcs_t@@PEAXPEAUhb_draw_state_t@@MMMMMM1@Z 0000000180006950 f   hb-draw.obj
 0001:00005950       ?hb_draw_line_to_nil@@YAXPEAUhb_draw_funcs_t@@PEAXPEAUhb_draw_state_t@@MM1@Z 0000000180006950 f   hb-draw.obj
 0001:00005950       ?hb_draw_move_to_nil@@YAXPEAUhb_draw_funcs_t@@PEAXPEAUhb_draw_state_t@@MM1@Z 0000000180006950 f   hb-draw.obj
 0001:00005950       ??$_hb_debug_msg@$0A@@@YAXPEBDPEBX0_NIH0ZZ 0000000180006950 f   hb-face.obj
 0001:00005950       ??$_hb_debug_msg@$0A@@@YAXPEBDPEBX0_NIH0ZZ 0000000180006950 f   hb-font.obj
 0001:00005950       ?_do_nothing@@YAXXZ        0000000180006950 f   hb-jdk-font-p.obj
 0001:00005950       ?_do_nothing@@YAXXZ        0000000180006950 f   hb-jdk-font.obj
 0001:00005950       ??$_hb_debug_msg@$0A@@@YAXPEBDPEBX0_NIH0ZZ 0000000180006950 f   hb-ot-color.obj
 0001:00005950       ??$_hb_debug_msg@$0A@@@YAXPEBDPEBX0_NIH0ZZ 0000000180006950 f   hb-ot-font.obj
 0001:00005950       ??$_hb_debug_msg@$0A@@@YAXPEBDPEBX0_NIH0ZZ 0000000180006950 f   hb-ot-layout.obj
 0001:00005950       ??$_hb_debug_msg@$0A@@@YAXPEBDPEBX0_NIH0ZZ 0000000180006950 f   hb-ot-metrics.obj
 0001:00005950       ??$_hb_debug_msg@$0A@@@YAXPEBDPEBX0_NIH0ZZ 0000000180006950 f   hb-ot-shape.obj
 0001:00005950       ??$_hb_debug_msg@$0A@@@YAXPEBDPEBX0_NIH0ZZ 0000000180006950 f   hb-ot-shaper-arabic.obj
 0001:00005950       ??$_hb_debug_msg@$0A@@@YAXPEBDPEBX0_NIH0ZZ 0000000180006950 f   hb-ot-var.obj
 0001:00005950       ?hb_paint_color_nil@@YAXPEAUhb_paint_funcs_t@@PEAXHI1@Z 0000000180006950 f   hb-paint.obj
 0001:00005950       ?hb_paint_linear_gradient_nil@@YAXPEAUhb_paint_funcs_t@@PEAXPEAUhb_color_line_t@@MMMMMM1@Z 0000000180006950 f   hb-paint.obj
 0001:00005950       ?hb_paint_pop_clip_nil@@YAXPEAUhb_paint_funcs_t@@PEAX1@Z 0000000180006950 f   hb-paint.obj
 0001:00005950       ?hb_paint_pop_group_nil@@YAXPEAUhb_paint_funcs_t@@PEAXW4hb_paint_composite_mode_t@@1@Z 0000000180006950 f   hb-paint.obj
 0001:00005950       ?hb_paint_pop_transform_nil@@YAXPEAUhb_paint_funcs_t@@PEAX1@Z 0000000180006950 f   hb-paint.obj
 0001:00005950       ?hb_paint_push_clip_glyph_nil@@YAXPEAUhb_paint_funcs_t@@PEAXIPEAUhb_font_t@@1@Z 0000000180006950 f   hb-paint.obj
 0001:00005950       ?hb_paint_push_clip_rectangle_nil@@YAXPEAUhb_paint_funcs_t@@PEAXMMMM1@Z 0000000180006950 f   hb-paint.obj
 0001:00005950       ?hb_paint_push_group_nil@@YAXPEAUhb_paint_funcs_t@@PEAX1@Z 0000000180006950 f   hb-paint.obj
 0001:00005950       ?hb_paint_push_transform_nil@@YAXPEAUhb_paint_funcs_t@@PEAXMMMMMM1@Z 0000000180006950 f   hb-paint.obj
 0001:00005950       ?hb_paint_radial_gradient_nil@@YAXPEAUhb_paint_funcs_t@@PEAXPEAUhb_color_line_t@@MMMMMM1@Z 0000000180006950 f   hb-paint.obj
 0001:00005950       ?hb_paint_sweep_gradient_nil@@YAXPEAUhb_paint_funcs_t@@PEAXPEAUhb_color_line_t@@MMMM1@Z 0000000180006950 f   hb-paint.obj
 0001:00005950       ??$_hb_debug_msg@$0A@@@YAXPEBDPEBX0_NIH0ZZ 0000000180006950 f   hb-shape-plan.obj
 0001:00006910       $LN174                     0000000180007910     hb-aat-layout.obj
 0001:00006910       $LN174                     0000000180007910     hb-aat-layout.obj
 0001:00006910       $LN174                     0000000180007910     hb-aat-layout.obj
 0001:0000be08       $LN46                      000000018000ce08     hb-aat-layout.obj
 0001:00018090       ?is_deleted_glyph@@YA_NPEBUhb_glyph_info_t@@@Z 0000000180019090 f   hb-aat-layout.obj
 0001:0001b778       $LN251                     000000018001c778     hb-aat-layout.obj
 0001:0001ba38       $LN243                     000000018001ca38     hb-aat-layout.obj
 0001:0001bee4       $LN351                     000000018001cee4     hb-aat-layout.obj
 0001:0001c18c       $LN247                     000000018001d18c     hb-aat-layout.obj
 0001:000241f0       ??$sort_r_simple@$$V@@YAXPEAX_K1P6AHPEBX2@Z@Z 00000001800251f0 f   hb-aat-map.obj
 0001:000241f0       ??$sort_r_simple@$$V@@YAXPEAX_K1P6AHPEBX2@Z@Z 00000001800251f0 f   hb-ot-font.obj
 0001:000241f0       ??$sort_r_simple@$$V@@YAXPEAX_K1P6AHPEBX2@Z@Z 00000001800251f0 f   hb-ot-map.obj
 0001:000241f0       ??$sort_r_simple@$$V@@YAXPEAX_K1P6AHPEBX2@Z@Z 00000001800251f0 f   hb-ot-shaper-arabic.obj
 0001:00025510       ?_hb_blob_destroy@@YAXPEAX@Z 0000000180026510 f   hb-blob.obj
 0001:000255a0       ?_hb_mapped_file_destroy@@YAXPEAX@Z 00000001800265a0 f   hb-blob.obj
 0001:00026270       ?buffer_verify_error@@YAXPEAUhb_buffer_t@@PEAUhb_font_t@@PEBDZZ 0000000180027270 f   hb-buffer-verify.obj
 0001:00026320       ?buffer_verify_unsafe_to_break@@YA_NPEAUhb_buffer_t@@0PEAUhb_font_t@@PEBUhb_feature_t@@IPEBQEBD@Z 0000000180027320 f   hb-buffer-verify.obj
 0001:00026620       ?buffer_verify_unsafe_to_concat@@YA_NPEAUhb_buffer_t@@0PEAUhb_font_t@@PEBUhb_feature_t@@IPEBQEBD@Z 0000000180027620 f   hb-buffer-verify.obj
 0001:00026c90       ??$hb_buffer_add_utf@U?$hb_utf16_xe_t@G@@@@YAXPEAUhb_buffer_t@@PEBGHIH@Z 0000000180027c90 f   hb-buffer.obj
 0001:00030190       ?lang_find_or_insert@@YAPEAUhb_language_item_t@@PEBD@Z 0000000180031190 f   hb-common.obj
 0001:00030370       ?parse_bool@@YA_NPEAPEBDPEBDPEAI@Z 0000000180031370 f   hb-common.obj
 0001:000304a0       ?parse_feature_indices@@YA_NPEAPEBDPEBDPEAUhb_feature_t@@@Z 00000001800314a0 f   hb-common.obj
 0001:00030640       ?parse_one_feature@@YA_NPEAPEBDPEBDPEAUhb_feature_t@@@Z 0000000180031640 f   hb-common.obj
 0001:000307c0       ?parse_tag@@YA_NPEAPEBDPEBDPEAI@Z 00000001800317c0 f   hb-common.obj
 0001:00031ba0       ?hb_draw_quadratic_to_nil@@YAXPEAUhb_draw_funcs_t@@PEAXPEAUhb_draw_state_t@@MMMM1@Z 0000000180032ba0 f   hb-draw.obj
 0001:00031eb0       ?hb_draw_extents_cubic_to@@YAXPEAUhb_draw_funcs_t@@PEAXPEAUhb_draw_state_t@@MMMMMM1@Z 0000000180032eb0 f   hb-draw.obj
 0001:00031f70       ?hb_draw_extents_line_to@@YAXPEAUhb_draw_funcs_t@@PEAXPEAUhb_draw_state_t@@MM1@Z 0000000180032f70 f   hb-draw.obj
 0001:00031f70       ?hb_draw_extents_move_to@@YAXPEAUhb_draw_funcs_t@@PEAXPEAUhb_draw_state_t@@MM1@Z 0000000180032f70 f   hb-draw.obj
 0001:00031f90       ?hb_draw_extents_quadratic_to@@YAXPEAUhb_draw_funcs_t@@PEAXPEAUhb_draw_state_t@@MMMM1@Z 0000000180032f90 f   hb-draw.obj
 0001:00033400       ?fasthash32@@YAIPEBX_KI@Z  0000000180034400 f   hb-face-builder.obj
 0001:00033400       ?fasthash32@@YAIPEBX_KI@Z  0000000180034400 f   hb-ot-shaper-arabic.obj
 0001:00033564       $LN50                      0000000180034564     hb-face-builder.obj
 0001:00033564       $LN50                      0000000180034564     hb-ot-shaper-arabic.obj
 0001:00034850       ??$get_glyph_from_symbol@UCmapSubtable@OT@@$1?_hb_arabic_pua_simp_map@@YAII@Z@accelerator_t@cmap@OT@@KA_NPEBXIPEAI@Z 0000000180035850 f   hb-face.obj
 0001:000348c0       ??$get_glyph_from_symbol@UCmapSubtable@OT@@$1?_hb_arabic_pua_trad_map@@YAII@Z@accelerator_t@cmap@OT@@KA_NPEBXIPEAI@Z 00000001800358c0 f   hb-face.obj
 0001:00034930       ??$get_glyph_from_symbol@UCmapSubtable@OT@@$1?_hb_symbol_pua_map@2@YAII@Z@accelerator_t@cmap@OT@@KA_NPEBXIPEAI@Z 0000000180035930 f   hb-face.obj
 0001:000349a0       ??$hb_object_create@Uhb_face_t@@$$V@@YAPEAUhb_face_t@@XZ 00000001800359a0 f   hb-face.obj
 0001:000357a0       ?_hb_arabic_pua_simp_map@@YAII@Z 00000001800367a0 f   hb-face.obj
 0001:00035840       ?_hb_arabic_pua_trad_map@@YAII@Z 0000000180036840 f   hb-face.obj
 0001:000358e0       ?_hb_face_for_data_closure_destroy@@YAXPEAX@Z 00000001800368e0 f   hb-face.obj
 0001:00035900       ?_hb_face_for_data_get_table_tags@@YAIPEBUhb_face_t@@IPEAI1PEAX@Z 0000000180036900 f   hb-face.obj
 0001:00035a80       ?_hb_face_for_data_reference_table@@YAPEAUhb_blob_t@@PEAUhb_face_t@@IPEAX@Z 0000000180036a80 f   hb-face.obj
 0001:00036bb0       $LN86                      0000000180037bb0     hb-face.obj
 0001:000370c4       $LN214                     00000001800380c4     hb-face.obj
 0001:00039240       ?hb_jdk_get_glyph_h_origin@@YAHPEAUhb_font_t@@PEAXIPEAH21@Z 000000018003a240 f   hb-jdk-font-p.obj
 0001:00039240       ?hb_jdk_get_glyph_h_origin@@YAHPEAUhb_font_t@@PEAXIPEAH21@Z 000000018003a240 f   hb-jdk-font.obj
 0001:00039240       ?hb_unicode_eastasian_width_nil@@YAIPEAUhb_unicode_funcs_t@@IPEAX@Z 000000018003a240 f   hb-unicode.obj
 0001:00039250       ?hb_font_get_font_h_extents_nil@@YAHPEAUhb_font_t@@PEAXPEAUhb_font_extents_t@@1@Z 000000018003a250 f   hb-font.obj
 0001:00039250       ?hb_font_get_font_v_extents_nil@@YAHPEAUhb_font_t@@PEAXPEAUhb_font_extents_t@@1@Z 000000018003a250 f   hb-font.obj
 0001:00039270       ?hb_font_get_font_h_extents_default@@YAHPEAUhb_font_t@@PEAXPEAUhb_font_extents_t@@1@Z 000000018003a270 f   hb-font.obj
 0001:00039370       ?hb_font_get_font_v_extents_default@@YAHPEAUhb_font_t@@PEAXPEAUhb_font_extents_t@@1@Z 000000018003a370 f   hb-font.obj
 0001:00039470       ?hb_font_get_nominal_glyph_nil@@YAHPEAUhb_font_t@@PEAXIPEAI1@Z 000000018003a470 f   hb-font.obj
 0001:00039480       ?hb_font_get_nominal_glyph_default@@YAHPEAUhb_font_t@@PEAXIPEAI1@Z 000000018003a480 f   hb-font.obj
 0001:00039510       ?hb_font_get_nominal_glyphs_default@@YAIPEAUhb_font_t@@PEAXIPEBIIPEAII1@Z 000000018003a510 f   hb-font.obj
 0001:00039620       ?hb_font_get_glyph_from_name_nil@@YAHPEAUhb_font_t@@PEAXPEBDHPEAI1@Z 000000018003a620 f   hb-font.obj
 0001:00039620       ?hb_font_get_variation_glyph_nil@@YAHPEAUhb_font_t@@PEAXIIPEAI1@Z 000000018003a620 f   hb-font.obj
 0001:00039630       ?hb_font_get_variation_glyph_default@@YAHPEAUhb_font_t@@PEAXIIPEAI1@Z 000000018003a630 f   hb-font.obj
 0001:00039670       ?hb_font_get_glyph_h_advance_nil@@YAHPEAUhb_font_t@@PEAXI1@Z 000000018003a670 f   hb-font.obj
 0001:00039680       ?hb_font_get_glyph_h_advance_default@@YAHPEAUhb_font_t@@PEAXI1@Z 000000018003a680 f   hb-font.obj
 0001:00039750       ?hb_font_get_glyph_v_advance_nil@@YAHPEAUhb_font_t@@PEAXI1@Z 000000018003a750 f   hb-font.obj
 0001:00039760       ?hb_font_get_glyph_v_advance_default@@YAHPEAUhb_font_t@@PEAXI1@Z 000000018003a760 f   hb-font.obj
 0001:00039830       ?hb_font_get_glyph_h_advances_default@@YAXPEAUhb_font_t@@PEAXIPEBIIPEAHI1@Z 000000018003a830 f   hb-font.obj
 0001:00039980       ?hb_font_get_glyph_v_advances_default@@YAXPEAUhb_font_t@@PEAXIPEBIIPEAHI1@Z 000000018003a980 f   hb-font.obj
 0001:00039ad0       ?hb_font_get_glyph_h_origin_nil@@YAHPEAUhb_font_t@@PEAXIPEAH21@Z 000000018003aad0 f   hb-font.obj
 0001:00039ae0       ?hb_font_get_glyph_h_origin_default@@YAHPEAUhb_font_t@@PEAXIPEAH21@Z 000000018003aae0 f   hb-font.obj
 0001:00039ba0       ?hb_font_get_glyph_v_origin_nil@@YAHPEAUhb_font_t@@PEAXIPEAH21@Z 000000018003aba0 f   hb-font.obj
 0001:00039bb0       ?hb_font_get_glyph_v_origin_default@@YAHPEAUhb_font_t@@PEAXIPEAH21@Z 000000018003abb0 f   hb-font.obj
 0001:00039c70       ?hb_font_get_glyph_h_kerning_default@@YAHPEAUhb_font_t@@PEAXII1@Z 000000018003ac70 f   hb-font.obj
 0001:00039ce0       ?hb_font_get_glyph_v_kerning_default@@YAHPEAUhb_font_t@@PEAXII1@Z 000000018003ace0 f   hb-font.obj
 0001:00039d50       ?hb_font_get_glyph_extents_nil@@YAHPEAUhb_font_t@@PEAXIPEAUhb_glyph_extents_t@@1@Z 000000018003ad50 f   hb-font.obj
 0001:00039d60       ?hb_font_get_glyph_extents_default@@YAHPEAUhb_font_t@@PEAXIPEAUhb_glyph_extents_t@@1@Z 000000018003ad60 f   hb-font.obj
 0001:00039e80       ?hb_font_get_glyph_contour_point_nil@@YAHPEAUhb_font_t@@PEAXIIPEAH21@Z 000000018003ae80 f   hb-font.obj
 0001:00039ea0       ?hb_font_get_glyph_contour_point_default@@YAHPEAUhb_font_t@@PEAXIIPEAH21@Z 000000018003aea0 f   hb-font.obj
 0001:00039f80       ?hb_font_get_glyph_name_nil@@YAHPEAUhb_font_t@@PEAXIPEADI1@Z 000000018003af80 f   hb-font.obj
 0001:00039f90       ?hb_font_get_glyph_name_default@@YAHPEAUhb_font_t@@PEAXIPEADI1@Z 000000018003af90 f   hb-font.obj
 0001:00039fd0       ?hb_font_get_glyph_from_name_default@@YAHPEAUhb_font_t@@PEAXPEBDHPEAI1@Z 000000018003afd0 f   hb-font.obj
 0001:0003a030       ?hb_draw_move_to_default@@YAXPEAUhb_draw_funcs_t@@PEAXPEAUhb_draw_state_t@@MM1@Z 000000018003b030 f   hb-font.obj
 0001:0003a070       ?hb_draw_line_to_default@@YAXPEAUhb_draw_funcs_t@@PEAXPEAUhb_draw_state_t@@MM1@Z 000000018003b070 f   hb-font.obj
 0001:0003a0d0       ?hb_draw_quadratic_to_default@@YAXPEAUhb_draw_funcs_t@@PEAXPEAUhb_draw_state_t@@MMMM1@Z 000000018003b0d0 f   hb-font.obj
 0001:0003a150       ?hb_draw_cubic_to_default@@YAXPEAUhb_draw_funcs_t@@PEAXPEAUhb_draw_state_t@@MMMMMM1@Z 000000018003b150 f   hb-font.obj
 0001:0003a220       ?hb_draw_close_path_default@@YAXPEAUhb_draw_funcs_t@@PEAXPEAUhb_draw_state_t@@1@Z 000000018003b220 f   hb-font.obj
 0001:0003a250       ?hb_font_draw_glyph_or_fail_default@@YAHPEAUhb_font_t@@PEAXIPEAUhb_draw_funcs_t@@11@Z 000000018003b250 f   hb-font.obj
 0001:0003a320       ?hb_font_paint_glyph_or_fail_default@@YAHPEAUhb_font_t@@PEAXIPEAUhb_paint_funcs_t@@1II1@Z 000000018003b320 f   hb-font.obj
 0001:0003a760       ?_hb_font_adopt_var_coords@@YAXPEAUhb_font_t@@PEAHPEAMI@Z 000000018003b760 f   hb-font.obj
 0001:0003a7d0       ?_hb_font_create@@YAPEAUhb_font_t@@PEAUhb_face_t@@@Z 000000018003b7d0 f   hb-font.obj
 0001:0003e820       ?reference_table@@YAPEAUhb_blob_t@@PEAUhb_face_t@@IPEAX@Z 000000018003f820 f   hb-jdk-font-p.obj
 0001:0003eac0       ?cleanupFontInfo@@YAXPEAX@Z 000000018003fac0 f   hb-jdk-font.obj
 0001:0003eb00       ?hb_jdk_get_glyph_contour_point@@YAHPEAUhb_font_t@@PEAXIIPEAH21@Z 000000018003fb00 f   hb-jdk-font.obj
 0001:0003ebe0       ?hb_jdk_get_glyph_h_advance@@YAHPEAUhb_font_t@@PEAXI1@Z 000000018003fbe0 f   hb-jdk-font.obj
 0001:0003ec90       ?hb_jdk_get_glyph_v_advance@@YAHPEAUhb_font_t@@PEAXI1@Z 000000018003fc90 f   hb-jdk-font.obj
 0001:0003ed30       ?hb_jdk_get_nominal_glyph@@YAHPEAUhb_font_t@@PEAXIPEAI1@Z 000000018003fd30 f   hb-jdk-font.obj
 0001:0003ed90       ?hb_jdk_get_variation_glyph@@YAHPEAUhb_font_t@@PEAXIIPEAI1@Z 000000018003fd90 f   hb-jdk-font.obj
 0001:0003ee00       ?reference_table@@YAPEAUhb_blob_t@@PEAUhb_face_t@@IPEAX@Z 000000018003fe00 f   hb-jdk-font.obj
 0001:0003f320       ?strtod_rl@@YANPEBDPEAPEBD@Z 0000000180040320 f   hb-number.obj
 0001:0003fa00       ?_get_bounds@@YA_NPEBUaccelerator_t@cff1@OT@@IAEAUbounds_t@@_N@Z 0000000180040a00 f   hb-ot-cff1-table.obj
 0001:0003fb70       ?_get_path@@YA_NPEBUaccelerator_t@cff1@OT@@PEAUhb_font_t@@IAEAUhb_draw_session_t@@_NPEAUpoint_t@CFF@@@Z 0000000180040b70 f   hb-ot-cff1-table.obj
 0001:0003fee0       $LN30                      0000000180040ee0     hb-ot-cff1-table.obj
 0001:0003fee0       $LN30                      0000000180040ee0     hb-ot-cff1-table.obj
 0001:0003fef0       $LN29                      0000000180040ef0     hb-ot-cff1-table.obj
 0001:0003fef0       $LN29                      0000000180040ef0     hb-ot-cff1-table.obj
 0001:00044de4       $LN578                     0000000180045de4     hb-ot-cff1-table.obj
 0001:00044e3c       $LN577                     0000000180045e3c     hb-ot-cff1-table.obj
 0001:000453bc       $LN566                     00000001800463bc     hb-ot-cff1-table.obj
 0001:00045414       $LN565                     0000000180046414     hb-ot-cff1-table.obj
 0001:00045714       $LN89                      0000000180046714     hb-ot-cff1-table.obj
 0001:00045724       $LN88                      0000000180046724     hb-ot-cff1-table.obj
 0001:0004fc40       $LN529                     0000000180050c40     hb-ot-cff2-table.obj
 0001:0004fc98       $LN528                     0000000180050c98     hb-ot-cff2-table.obj
 0001:0005016c       $LN410                     000000018005116c     hb-ot-cff2-table.obj
 0001:000501c4       $LN409                     00000001800511c4     hb-ot-cff2-table.obj
 0001:00055854       $LN1029                    0000000180056854     hb-ot-color.obj
 0001:0005a780       ??$StructAtOffsetOrNull@U?$CFFIndex@U?$IntType@G$01@OT@@@OT@@$$V@CFF@@YAAEBU?$CFFIndex@U?$IntType@G$01@OT@@@OT@@PEBXHAEAUhb_sanitize_context_t@@@Z 000000018005b780 f   hb-ot-font.obj
 0001:0005a780       ??$StructAtOffsetOrNull@U?$Subrs@U?$IntType@G$01@OT@@@CFF@@$$V@CFF@@YAAEBU?$Subrs@U?$IntType@G$01@OT@@@0@PEBXHAEAUhb_sanitize_context_t@@@Z 000000018005b780 f   hb-ot-font.obj
 0001:0005a780       ??$StructAtOffsetOrNull@UCFF1StringIndex@CFF@@$$V@CFF@@YAAEBUCFF1StringIndex@0@PEBXHAEAUhb_sanitize_context_t@@@Z 000000018005b780 f   hb-ot-font.obj
 0001:0005a850       ??$StructAtOffsetOrNull@U?$Subrs@U?$IntType@I$03@OT@@@CFF@@$$V@CFF@@YAAEBU?$Subrs@U?$IntType@I$03@OT@@@0@PEBXHAEAUhb_sanitize_context_t@@@Z 000000018005b850 f   hb-ot-font.obj
 0001:0005b03c       $LN414                     000000018005c03c     hb-ot-font.obj
 0001:0005cc90       ??$sort_r_simple@PEAX@@YAXPEAX_K1P6AHPEBX20@Z0@Z 000000018005dc90 f   hb-ot-font.obj
 0001:0005f8c0       ?_hb_ot_font_destroy@@YAXPEAX@Z 00000001800608c0 f   hb-ot-font.obj
 0001:00063130       ?hb_ot_draw_glyph_or_fail@@YAHPEAUhb_font_t@@PEAXIPEAUhb_draw_funcs_t@@11@Z 0000000180064130 f   hb-ot-font.obj
 0001:00063390       ?hb_ot_get_font_h_extents@@YAHPEAUhb_font_t@@PEAXPEAUhb_font_extents_t@@1@Z 0000000180064390 f   hb-ot-font.obj
 0001:00063400       ?hb_ot_get_font_v_extents@@YAHPEAUhb_font_t@@PEAXPEAUhb_font_extents_t@@1@Z 0000000180064400 f   hb-ot-font.obj
 0001:00063470       ?hb_ot_get_glyph_extents@@YAHPEAUhb_font_t@@PEAXIPEAUhb_glyph_extents_t@@1@Z 0000000180064470 f   hb-ot-font.obj
 0001:00063680       ?hb_ot_get_glyph_from_name@@YAHPEAUhb_font_t@@PEAXPEBDHPEAI1@Z 0000000180064680 f   hb-ot-font.obj
 0001:00063710       ?hb_ot_get_glyph_h_advances@@YAXPEAUhb_font_t@@PEAXIPEBIIPEAHI1@Z 0000000180064710 f   hb-ot-font.obj
 0001:00063c30       ?hb_ot_get_glyph_name@@YAHPEAUhb_font_t@@PEAXIPEADI1@Z 0000000180064c30 f   hb-ot-font.obj
 0001:00063d60       ?hb_ot_get_glyph_v_advances@@YAXPEAUhb_font_t@@PEAXIPEBIIPEAHI1@Z 0000000180064d60 f   hb-ot-font.obj
 0001:00064070       ?hb_ot_get_glyph_v_origin@@YAHPEAUhb_font_t@@PEAXIPEAH21@Z 0000000180065070 f   hb-ot-font.obj
 0001:000646b0       ?hb_ot_get_nominal_glyph@@YAHPEAUhb_font_t@@PEAXIPEAI1@Z 00000001800656b0 f   hb-ot-font.obj
 0001:00064700       ?hb_ot_get_nominal_glyphs@@YAIPEAUhb_font_t@@PEAXIPEBIIPEAII1@Z 0000000180065700 f   hb-ot-font.obj
 0001:000647f0       ?hb_ot_get_variation_glyph@@YAHPEAUhb_font_t@@PEAXIIPEAI1@Z 00000001800657f0 f   hb-ot-font.obj
 0001:00064910       ?hb_ot_paint_glyph_or_fail@@YAHPEAUhb_font_t@@PEAXIPEAUhb_paint_funcs_t@@1II1@Z 0000000180065910 f   hb-ot-font.obj
 0001:000652cc       $LN110                     00000001800662cc     hb-ot-font.obj
 0001:0006530c       $LN109                     000000018006630c     hb-ot-font.obj
 0001:00065870       $LN136                     0000000180066870     hb-ot-font.obj
 0001:000658b8       $LN135                     00000001800668b8     hb-ot-font.obj
 0001:00068f5c       $LN280                     0000000180069f5c     hb-ot-font.obj
 0001:00068fa8       $LN279                     0000000180069fa8     hb-ot-font.obj
 0001:00068fc0       $LN278                     0000000180069fc0     hb-ot-font.obj
 0001:0006bed0       ??$apply_string@UGSUBProxy@@@@YA_NPEAUhb_ot_apply_context_t@OT@@AEBUSubstLookup@GSUB_impl@Layout@1@AEBUhb_ot_layout_lookup_accelerator_t@1@@Z 000000018006ced0 f   hb-ot-layout.obj
 0001:0006dfc4       $LN433                     000000018006efc4     hb-ot-layout.obj
 0001:0006e2ec       $LN338                     000000018006f2ec     hb-ot-layout.obj
 0001:0006ee58       $LN217                     000000018006fe58     hb-ot-layout.obj
 0001:0006f5a0       $LN293                     00000001800705a0     hb-ot-layout.obj
 0001:00070410       ??$op_@U<unnamed-type-hb_bitwise_or>@@@hb_bit_set_t@@SA?AU?$hb_vector_size_t@_K$0EA@@@AEBU1@0@Z 0000000180071410 f   hb-ot-layout.obj
 0001:00070ce0       ??$would_match_input@U?$IntType@G$01@OT@@@OT@@YA_NPEAUhb_would_apply_context_t@0@IQEBU?$IntType@G$01@0@P6A_NAEAUhb_glyph_info_t@@IPEBX@Z3@Z 0000000180071ce0 f   hb-ot-layout.obj
 0001:00071e60       ?_hb_allocate_lig_id@@YAEPEAUhb_buffer_t@@@Z 0000000180072e60 f   hb-ot-layout.obj
 0001:00071e90       ?_hb_ot_layout_set_glyph_props@@YAXPEAUhb_font_t@@PEAUhb_buffer_t@@@Z 0000000180072e90 f   hb-ot-layout.obj
 0001:0007a340       ?apply_backward@@YA_NPEAUhb_ot_apply_context_t@OT@@AEBUhb_ot_layout_lookup_accelerator_t@2@I@Z 000000018007b340 f   hb-ot-layout.obj
 0001:0007a500       ?apply_forward@@YA_NPEAUhb_ot_apply_context_t@OT@@AEBUhb_ot_layout_lookup_accelerator_t@2@I@Z 000000018007b500 f   hb-ot-layout.obj
 0001:0007a840       ?apply_lookup@OT@@YAXPEAUhb_ot_apply_context_t@1@IPEAIIQEBULookupRecord@1@I@Z 000000018007b840 f   hb-ot-layout.obj
 0001:0007cc70       ?get_gsubgpos_table@@YAAEBUGSUBGPOS@OT@@PEAUhb_face_t@@I@Z 000000018007dc70 f   hb-ot-layout.obj
 0001:00080210       ?ligate_input@OT@@YA_NPEAUhb_ot_apply_context_t@1@IPEBIIII@Z 0000000180081210 f   hb-ot-layout.obj
 0001:000805c0       ?match_always@OT@@YA_NAEAUhb_glyph_info_t@@IPEBX@Z 00000001800815c0 f   hb-ot-layout.obj
 0001:000805d0       ?match_class@OT@@YA_NAEAUhb_glyph_info_t@@IPEBX@Z 00000001800815d0 f   hb-ot-layout.obj
 0001:000805f0       ?match_class_cached1@OT@@YA_NAEAUhb_glyph_info_t@@IPEBX@Z 00000001800815f0 f   hb-ot-layout.obj
 0001:00080640       ?match_class_cached2@OT@@YA_NAEAUhb_glyph_info_t@@IPEBX@Z 0000000180081640 f   hb-ot-layout.obj
 0001:00080690       ?match_class_cached@OT@@YA_NAEAUhb_glyph_info_t@@IPEBX@Z 0000000180081690 f   hb-ot-layout.obj
 0001:000806d0       ?match_coverage@OT@@YA_NAEAUhb_glyph_info_t@@IPEBX@Z 00000001800816d0 f   hb-ot-layout.obj
 0001:00080770       ?match_glyph@OT@@YA_NAEAUhb_glyph_info_t@@IPEBX@Z 0000000180081770 f   hb-ot-layout.obj
 0001:000812d0       ?propagate_attachment_offsets@Layout@OT@@YAXPEAUhb_glyph_position_t@@IIW4hb_direction_t@@I@Z 00000001800822d0 f   hb-ot-layout.obj
 0001:00081400       ?reverse_cursive_minor_offset@GPOS_impl@Layout@OT@@YAXPEAUhb_glyph_position_t@@IW4hb_direction_t@@I@Z 0000000180082400 f   hb-ot-layout.obj
 0001:00086f70       ?_fix_ascender_descender@@YAMMW4hb_ot_metrics_tag_t@@@Z 0000000180087f70 f   hb-ot-metrics.obj
 0001:00087bfc       $LN94                      0000000180088bfc     hb-ot-shape-fallback.obj
 0001:00087c0c       $LN93                      0000000180088c0c     hb-ot-shape-fallback.obj
 0001:00087cac       $LN92                      0000000180088cac     hb-ot-shape-fallback.obj
 0001:00087cc8       $LN91                      0000000180088cc8     hb-ot-shape-fallback.obj
 0001:000880b4       $LN105                     00000001800890b4     hb-ot-shape-fallback.obj
 0001:000880cc       $LN104                     00000001800890cc     hb-ot-shape-fallback.obj
 0001:000885e0       ?position_around_base@@YAXPEBUhb_ot_shape_plan_t@@PEAUhb_font_t@@PEAUhb_buffer_t@@II_N@Z 00000001800895e0 f   hb-ot-shape-fallback.obj
 0001:00088a30       ?position_cluster@@YAXPEBUhb_ot_shape_plan_t@@PEAUhb_font_t@@PEAUhb_buffer_t@@II_N@Z 0000000180089a30 f   hb-ot-shape-fallback.obj
 0001:00088b30       ?position_mark@@YAXPEBUhb_ot_shape_plan_t@@PEAUhb_font_t@@PEAUhb_buffer_t@@AEAUhb_glyph_extents_t@@II@Z 0000000180089b30 f   hb-ot-shape-fallback.obj
 0001:00088d00       $LN52                      0000000180089d00     hb-ot-shape-fallback.obj
 0001:00088d14       $LN51                      0000000180089d14     hb-ot-shape-fallback.obj
 0001:00088d38       $LN50                      0000000180089d38     hb-ot-shape-fallback.obj
 0001:00088d4c       $LN49                      0000000180089d4c     hb-ot-shape-fallback.obj
 0001:00088d70       ?_hb_glyph_info_set_unicode_props@@YAXPEAUhb_glyph_info_t@@PEAUhb_buffer_t@@@Z 0000000180089d70 f   hb-ot-shape-normalize.obj
 0001:00088d70       ?_hb_glyph_info_set_unicode_props@@YAXPEAUhb_glyph_info_t@@PEAUhb_buffer_t@@@Z 0000000180089d70 f   hb-ot-shape.obj
 0001:000899d4       $LN381                     000000018008a9d4     hb-ot-shape-normalize.obj
 0001:00089a04       $LN380                     000000018008aa04     hb-ot-shape-normalize.obj
 0001:00089a70       ?compare_combining_class@@YAHPEBUhb_glyph_info_t@@0@Z 000000018008aa70 f   hb-ot-shape-normalize.obj
 0001:00089b00       ?decompose@@YAIPEBUhb_ot_shape_normalize_context_t@@_NI@Z 000000018008ab00 f   hb-ot-shape-normalize.obj
 0001:00089c90       ?decompose_current_character@@YAXPEBUhb_ot_shape_normalize_context_t@@_N@Z 000000018008ac90 f   hb-ot-shape-normalize.obj
 0001:00089f78       $LN98                      000000018008af78     hb-ot-shape-normalize.obj
 0001:00089fa8       $LN97                      000000018008afa8     hb-ot-shape-normalize.obj
 0001:0008a040       ?handle_variation_selector_cluster@@YAXPEBUhb_ot_shape_normalize_context_t@@I_N@Z 000000018008b040 f   hb-ot-shape-normalize.obj
 0001:0008a4a0       ?output_char@@YAXPEAUhb_buffer_t@@II@Z 000000018008b4a0 f   hb-ot-shape-normalize.obj
 0001:0008a960       ?_hb_glyph_info_is_default_ignorable@@YA_NPEBUhb_glyph_info_t@@@Z 000000018008b960 f   hb-ot-shape.obj
 0001:0008a980       ?_hb_grapheme_group_func@@YA_NAEBUhb_glyph_info_t@@0@Z 000000018008b980 f   hb-ot-shape.obj
 0001:0008b120       ?hb_form_clusters@@YAXPEAUhb_buffer_t@@@Z 000000018008c120 f   hb-ot-shape.obj
 0001:0008b2b0       ?hb_ot_position_default@@YAXPEBUhb_ot_shape_context_t@@@Z 000000018008c2b0 f   hb-ot-shape.obj
 0001:0008b660       ?hb_ot_position_plan@@YAXPEBUhb_ot_shape_context_t@@@Z 000000018008c660 f   hb-ot-shape.obj
 0001:0008ba40       ?hb_ot_rotate_chars@@YAXPEBUhb_ot_shape_context_t@@@Z 000000018008ca40 f   hb-ot-shape.obj
 0001:0008bd3c       $LN90                      000000018008cd3c     hb-ot-shape.obj
 0001:0008bd70       $LN89                      000000018008cd70     hb-ot-shape.obj
 0001:0008bdd0       $LN88                      000000018008cdd0     hb-ot-shape.obj
 0001:0008be30       ?hb_ot_shape_collect_features@@YAXPEAUhb_ot_shape_planner_t@@PEBUhb_feature_t@@I@Z 000000018008ce30 f   hb-ot-shape.obj
 0001:0008c0d0       ?hb_ot_shape_internal@@YAXPEAUhb_ot_shape_context_t@@@Z 000000018008d0d0 f   hb-ot-shape.obj
 0001:0008c470       ?hb_ot_shape_setup_masks_fraction@@YAXPEBUhb_ot_shape_context_t@@@Z 000000018008d470 f   hb-ot-shape.obj
 0001:0008c720       ?hb_ot_shaper_categorize@@YAPEBUhb_ot_shaper_t@@W4hb_script_t@@W4hb_direction_t@@I@Z 000000018008d720 f   hb-ot-shape.obj
 0001:0008cd40       ?hb_ot_substitute_default@@YAXPEBUhb_ot_shape_context_t@@@Z 000000018008dd40 f   hb-ot-shape.obj
 0001:0008cec0       ?hb_ot_substitute_post@@YAXPEBUhb_ot_shape_context_t@@@Z 000000018008dec0 f   hb-ot-shape.obj
 0001:0008d090       ?hb_propagate_flags@@YAXPEAUhb_buffer_t@@@Z 000000018008e090 f   hb-ot-shape.obj
 0001:0008d330       ?hb_set_unicode_props@@YAXPEAUhb_buffer_t@@@Z 000000018008e330 f   hb-ot-shape.obj
 0001:0008da30       ?zero_mark_widths_by_gdef@@YAXPEAUhb_buffer_t@@_N@Z 000000018008ea30 f   hb-ot-shape.obj
 0001:0008dd10       ?setup_masks_arabic@@YAXPEBUhb_ot_shape_plan_t@@PEAUhb_buffer_t@@PEAUhb_font_t@@@Z 000000018008ed10 f   hb-ot-shaper-arabic.obj
 0001:0008dde0       ?postprocess_glyphs_arabic@@YAXPEBUhb_ot_shape_plan_t@@PEAUhb_buffer_t@@PEAUhb_font_t@@@Z 000000018008ede0 f   hb-ot-shaper-arabic.obj
 0001:0008ddf0       ?reorder_marks_arabic@@YAXPEBUhb_ot_shape_plan_t@@PEAUhb_buffer_t@@II@Z 000000018008edf0 f   hb-ot-shaper-arabic.obj
 0001:0008e230       ?collect_features_arabic@@YAXPEAUhb_ot_shape_planner_t@@@Z 000000018008f230 f   hb-ot-shaper-arabic.obj
 0001:0008e470       ??$arabic_fallback_synthesize_lookup_ligature@$$BY00Uligature_3_set_t@@@@YAPEAUSubstLookup@GSUB_impl@Layout@OT@@PEBUhb_ot_shape_plan_t@@PEAUhb_font_t@@AEAY00$$CBUligature_3_set_t@@I@Z 000000018008f470 f   hb-ot-shaper-arabic.obj
 0001:0008eac0       ??$arabic_fallback_synthesize_lookup_ligature@$$BY00Uligature_mark_set_t@@@@YAPEAUSubstLookup@GSUB_impl@Layout@OT@@PEBUhb_ot_shape_plan_t@@PEAUhb_font_t@@AEAY00$$CBUligature_mark_set_t@@I@Z 000000018008fac0 f   hb-ot-shaper-arabic.obj
 0001:0008f110       ??$arabic_fallback_synthesize_lookup_ligature@$$BY0BC@Uligature_set_t@@@@YAPEAUSubstLookup@GSUB_impl@Layout@OT@@PEBUhb_ot_shape_plan_t@@PEAUhb_font_t@@AEAY0BC@$$CBUligature_set_t@@I@Z 0000000180090110 f   hb-ot-shaper-arabic.obj
 0001:0008faf0       ??$hb_stable_sort@UHBGlyphID16@OT@@U?$IntType@G$01@2@I@@YAXPEAUHBGlyphID16@OT@@IP6AHPEBU?$IntType@G$01@1@1@ZPEAI@Z 0000000180090af0 f   hb-ot-shaper-arabic.obj
 0001:0008fc90       ??$serialize@U?$hb_map_iter_t@U?$hb_zip_iter_t@U?$hb_sorted_array_t@UHBGlyphID16@OT@@@@U?$hb_array_t@UHBGlyphID16@OT@@@@@@AEBU<unnamed-type-hb_first>@@$00$0A@@@$0A@@?$CoverageFormat2_4@USmallTypes@Layout@OT@@@Common@Layout@OT@@AEAA_NPEAUhb_serialize_context_t@@U?$hb_map_iter_t@U?$hb_zip_iter_t@U?$hb_sorted_array_t@UHBGlyphID16@OT@@@@U?$hb_array_t@UHBGlyphID16@OT@@@@@@AEBU<unnamed-type-hb_first>@@$00$0A@@@@Z 0000000180090c90 f   hb-ot-shaper-arabic.obj
 0001:0008ff80       ??$serialize@U?$hb_map_iter_t@U?$hb_zip_iter_t@U?$hb_sorted_array_t@UHBGlyphID16@OT@@@@U?$hb_array_t@UHBGlyphID16@OT@@@@@@AEBU<unnamed-type-hb_first>@@$00$0A@@@$0A@@Coverage@Common@Layout@OT@@QEAA_NPEAUhb_serialize_context_t@@U?$hb_map_iter_t@U?$hb_zip_iter_t@U?$hb_sorted_array_t@UHBGlyphID16@OT@@@@U?$hb_array_t@UHBGlyphID16@OT@@@@@@AEBU<unnamed-type-hb_first>@@$00$0A@@@@Z 0000000180090f80 f   hb-ot-shaper-arabic.obj
 0001:00090ad0       ??$serialize_serialize@AEAU?$hb_map_iter_t@U?$hb_zip_iter_t@U?$hb_sorted_array_t@UHBGlyphID16@OT@@@@U?$hb_array_t@UHBGlyphID16@OT@@@@@@AEBU<unnamed-type-hb_first>@@$00$0A@@@@?$OffsetTo@UCoverage@Common@Layout@OT@@U?$IntType@G$01@4@X$00@OT@@QEAA_NPEAUhb_serialize_context_t@@AEAU?$hb_map_iter_t@U?$hb_zip_iter_t@U?$hb_sorted_array_t@UHBGlyphID16@OT@@@@U?$hb_array_t@UHBGlyphID16@OT@@@@@@AEBU<unnamed-type-hb_first>@@$00$0A@@@@Z 0000000180091ad0 f   hb-ot-shaper-arabic.obj
 0001:00090ce0       ?apply_stch@@YAXPEBUhb_ot_shape_plan_t@@PEAUhb_buffer_t@@PEAUhb_font_t@@@Z 0000000180091ce0 f   hb-ot-shaper-arabic.obj
 0001:000912d0       ?arabic_fallback_plan_destroy@@YAXPEAUarabic_fallback_plan_t@@@Z 00000001800922d0 f   hb-ot-shaper-arabic.obj
 0001:00091370       ?arabic_fallback_plan_init_unicode@@YA_NPEAUarabic_fallback_plan_t@@PEBUhb_ot_shape_plan_t@@PEAUhb_font_t@@@Z 0000000180092370 f   hb-ot-shaper-arabic.obj
 0001:000914e0       ?arabic_fallback_plan_init_win1256@@YA_NPEAUarabic_fallback_plan_t@@PEBUhb_ot_shape_plan_t@@PEAUhb_font_t@@@Z 00000001800924e0 f   hb-ot-shaper-arabic.obj
 0001:00091730       ?arabic_fallback_shape@@YA_NPEBUhb_ot_shape_plan_t@@PEAUhb_font_t@@PEAUhb_buffer_t@@@Z 0000000180092730 f   hb-ot-shaper-arabic.obj
 0001:00091970       ?arabic_fallback_synthesize_lookup_single@@YAPEAUSubstLookup@GSUB_impl@Layout@OT@@PEBUhb_ot_shape_plan_t@@PEAUhb_font_t@@I@Z 0000000180092970 f   hb-ot-shaper-arabic.obj
 0001:00091eb0       ?arabic_joining@@YAXPEAUhb_buffer_t@@@Z 0000000180092eb0 f   hb-ot-shaper-arabic.obj
 0001:00092390       ?deallocate_buffer_var@@YA_NPEBUhb_ot_shape_plan_t@@PEAUhb_font_t@@PEAUhb_buffer_t@@@Z 0000000180093390 f   hb-ot-shaper-arabic.obj
 0001:00092510       ?end@?$hb_iter_t@U?$hb_map_iter_t@U?$hb_zip_iter_t@U?$hb_sorted_array_t@UHBGlyphID16@OT@@@@U?$hb_array_t@UHBGlyphID16@OT@@@@@@AEBU<unnamed-type-hb_first>@@$00$0A@@@AEAUHBGlyphID16@OT@@@@QEBA?AU?$hb_map_iter_t@U?$hb_zip_iter_t@U?$hb_sorted_array_t@UHBGlyphID16@OT@@@@U?$hb_array_t@UHBGlyphID16@OT@@@@@@AEBU<unnamed-type-hb_first>@@$00$0A@@@XZ 0000000180093510 f   hb-ot-shaper-arabic.obj
 0001:000926f0       ?get_joining_type@@YAIIW4hb_unicode_general_category_t@@@Z 00000001800936f0 f   hb-ot-shaper-arabic.obj
 0001:00092840       $LN52                      0000000180093840     hb-ot-shaper-arabic.obj
 0001:00092860       $LN51                      0000000180093860     hb-ot-shaper-arabic.obj
 0001:00092a20       ?record_stch@@YA_NPEBUhb_ot_shape_plan_t@@PEAUhb_font_t@@PEAUhb_buffer_t@@@Z 0000000180093a20 f   hb-ot-shaper-arabic.obj
 0001:000938d0       ?collect_features_hangul@@YAXPEAUhb_ot_shape_planner_t@@@Z 00000001800948d0 f   hb-ot-shaper-hangul.obj
 0001:00093920       ?override_features_hangul@@YAXPEAUhb_ot_shape_planner_t@@@Z 0000000180094920 f   hb-ot-shaper-hangul.obj
 0001:00093940       ?data_create_hangul@@YAPEAXPEBUhb_ot_shape_plan_t@@@Z 0000000180094940 f   hb-ot-shaper-hangul.obj
 0001:00093ac0       ?data_destroy_hangul@@YAXPEAX@Z 0000000180094ac0 f   hb-ot-shaper-hangul.obj
 0001:00093ac0       ?data_destroy_indic@@YAXPEAX@Z 0000000180094ac0 f   hb-ot-shaper-indic.obj
 0001:00093ac0       ?data_destroy_khmer@@YAXPEAX@Z 0000000180094ac0 f   hb-ot-shaper-khmer.obj
 0001:00093ad0       ?preprocess_text_hangul@@YAXPEBUhb_ot_shape_plan_t@@PEAUhb_buffer_t@@PEAUhb_font_t@@@Z 0000000180094ad0 f   hb-ot-shaper-hangul.obj
 0001:00094680       ?setup_masks_hangul@@YAXPEBUhb_ot_shape_plan_t@@PEAUhb_buffer_t@@PEAUhb_font_t@@@Z 0000000180095680 f   hb-ot-shaper-hangul.obj
 0001:000946c0       ?compose_hebrew@@YA_NPEBUhb_ot_shape_normalize_context_t@@IIPEAI@Z 00000001800956c0 f   hb-ot-shaper-hebrew.obj
 0001:00094870       $LN41                      0000000180095870     hb-ot-shaper-hebrew.obj
 0001:000948b0       ?reorder_marks_hebrew@@YAXPEBUhb_ot_shape_plan_t@@PEAUhb_buffer_t@@II@Z 00000001800958b0 f   hb-ot-shaper-hebrew.obj
 0001:00094bb4       $LN62                      0000000180095bb4     hb-ot-shaper-indic-table.obj
 0001:00094c00       ?collect_features_indic@@YAXPEAUhb_ot_shape_planner_t@@@Z 0000000180095c00 f   hb-ot-shaper-indic.obj
 0001:00094cf0       ?override_features_indic@@YAXPEAUhb_ot_shape_planner_t@@@Z 0000000180095cf0 f   hb-ot-shaper-indic.obj
 0001:00094d30       ?data_create_indic@@YAPEAXPEBUhb_ot_shape_plan_t@@@Z 0000000180095d30 f   hb-ot-shaper-indic.obj
 0001:00094f10       ?setup_masks_indic@@YAXPEBUhb_ot_shape_plan_t@@PEAUhb_buffer_t@@PEAUhb_font_t@@@Z 0000000180095f10 f   hb-ot-shaper-indic.obj
 0001:00094f60       ?preprocess_text_indic@@YAXPEBUhb_ot_shape_plan_t@@PEAUhb_buffer_t@@PEAUhb_font_t@@@Z 0000000180095f60 f   hb-ot-shaper-indic.obj
 0001:00094f80       ?decompose_indic@@YA_NPEBUhb_ot_shape_normalize_context_t@@IPEAI1@Z 0000000180095f80 f   hb-ot-shaper-indic.obj
 0001:00094fe0       ?compose_indic@@YA_NPEBUhb_ot_shape_normalize_context_t@@IIPEAI@Z 0000000180095fe0 f   hb-ot-shaper-indic.obj
 0001:000950a0       ?consonant_position_from_face@@YA?AW4ot_position_t@@PEBUindic_shape_plan_t@@IIPEAUhb_face_t@@@Z 00000001800960a0 f   hb-ot-shaper-indic.obj
 0001:000952f0       ?final_reordering_indic@@YA_NPEBUhb_ot_shape_plan_t@@PEAUhb_font_t@@PEAUhb_buffer_t@@@Z 00000001800962f0 f   hb-ot-shaper-indic.obj
 0001:000953f0       ?final_reordering_syllable_indic@@YAXPEBUhb_ot_shape_plan_t@@PEAUhb_buffer_t@@II@Z 00000001800963f0 f   hb-ot-shaper-indic.obj
 0001:000965f0       $LN255                     00000001800975f0     hb-ot-shaper-indic.obj
 0001:00096760       ?initial_reordering_consonant_syllable@@YAXPEBUhb_ot_shape_plan_t@@PEAUhb_face_t@@PEAUhb_buffer_t@@II@Z 0000000180097760 f   hb-ot-shaper-indic.obj
 0001:00097530       ?initial_reordering_indic@@YA_NPEBUhb_ot_shape_plan_t@@PEAUhb_font_t@@PEAUhb_buffer_t@@@Z 0000000180098530 f   hb-ot-shaper-indic.obj
 0001:00097770       ?setup_syllables_indic@@YA_NPEBUhb_ot_shape_plan_t@@PEAUhb_font_t@@PEAUhb_buffer_t@@@Z 0000000180098770 f   hb-ot-shaper-indic.obj
 0001:00097940       ?collect_features_khmer@@YAXPEAUhb_ot_shape_planner_t@@@Z 0000000180098940 f   hb-ot-shaper-khmer.obj
 0001:00097a20       ?override_features_khmer@@YAXPEAUhb_ot_shape_planner_t@@@Z 0000000180098a20 f   hb-ot-shaper-khmer.obj
 0001:00097a90       ?data_create_khmer@@YAPEAXPEBUhb_ot_shape_plan_t@@@Z 0000000180098a90 f   hb-ot-shaper-khmer.obj
 0001:00097c10       ?setup_masks_khmer@@YAXPEBUhb_ot_shape_plan_t@@PEAUhb_buffer_t@@PEAUhb_font_t@@@Z 0000000180098c10 f   hb-ot-shaper-khmer.obj
 0001:00097c50       ?decompose_khmer@@YA_NPEBUhb_ot_shape_normalize_context_t@@IPEAI1@Z 0000000180098c50 f   hb-ot-shaper-khmer.obj
 0001:00097d10       ?compose_khmer@@YA_NPEBUhb_ot_shape_normalize_context_t@@IIPEAI@Z 0000000180098d10 f   hb-ot-shaper-khmer.obj
 0001:00097d10       ?compose_use@@YA_NPEBUhb_ot_shape_normalize_context_t@@IIPEAI@Z 0000000180098d10 f   hb-ot-shaper-use.obj
 0001:00098184       $LN151                     0000000180099184     hb-ot-shaper-khmer.obj
 0001:000981c0       ?reorder_consonant_syllable@@YAXPEBUhb_ot_shape_plan_t@@PEAUhb_face_t@@PEAUhb_buffer_t@@II@Z 00000001800991c0 f   hb-ot-shaper-khmer.obj
 0001:00098470       ?reorder_khmer@@YA_NPEBUhb_ot_shape_plan_t@@PEAUhb_font_t@@PEAUhb_buffer_t@@@Z 0000000180099470 f   hb-ot-shaper-khmer.obj
 0001:000985b0       ?setup_syllables_khmer@@YA_NPEBUhb_ot_shape_plan_t@@PEAUhb_font_t@@PEAUhb_buffer_t@@@Z 00000001800995b0 f   hb-ot-shaper-khmer.obj
 0001:000986f0       ?collect_features_myanmar@@YAXPEAUhb_ot_shape_planner_t@@@Z 00000001800996f0 f   hb-ot-shaper-myanmar.obj
 0001:00098800       ?setup_masks_myanmar@@YAXPEBUhb_ot_shape_plan_t@@PEAUhb_buffer_t@@PEAUhb_font_t@@@Z 0000000180099800 f   hb-ot-shaper-myanmar.obj
 0001:00098840       ?compare_myanmar_order@@YAHPEBUhb_glyph_info_t@@0@Z 0000000180099840 f   hb-ot-shaper-myanmar.obj
 0001:00098c64       $LN163                     0000000180099c64     hb-ot-shaper-myanmar.obj
 0001:00098c90       ?initial_reordering_consonant_syllable@@YAXPEAUhb_buffer_t@@II@Z 0000000180099c90 f   hb-ot-shaper-myanmar.obj
 0001:00099000       ?reorder_myanmar@@YA_NPEBUhb_ot_shape_plan_t@@PEAUhb_font_t@@PEAUhb_buffer_t@@@Z 000000018009a000 f   hb-ot-shaper-myanmar.obj
 0001:00099130       ?setup_syllables_myanmar@@YA_NPEBUhb_ot_shape_plan_t@@PEAUhb_font_t@@PEAUhb_buffer_t@@@Z 000000018009a130 f   hb-ot-shaper-myanmar.obj
 0001:000994c0       ?preprocess_text_thai@@YAXPEBUhb_ot_shape_plan_t@@PEAUhb_buffer_t@@PEAUhb_font_t@@@Z 000000018009a4c0 f   hb-ot-shaper-thai.obj
 0001:000997f0       ?do_thai_pua_shaping@@YAXPEBUhb_ot_shape_plan_t@@PEAUhb_buffer_t@@PEAUhb_font_t@@@Z 000000018009a7f0 f   hb-ot-shaper-thai.obj
 0001:00099aa0       ?thai_pua_shape@@YAIIW4thai_action_t@@PEAUhb_font_t@@@Z 000000018009aaa0 f   hb-ot-shaper-thai.obj
 0001:00099b80       ?collect_features_use@@YAXPEAUhb_ot_shape_planner_t@@@Z 000000018009ab80 f   hb-ot-shaper-use.obj
 0001:00099d40       ?data_create_use@@YAPEAXPEBUhb_ot_shape_plan_t@@@Z 000000018009ad40 f   hb-ot-shaper-use.obj
 0001:00099e50       ?data_destroy_use@@YAXPEAX@Z 000000018009ae50 f   hb-ot-shaper-use.obj
 0001:00099e80       ?setup_masks_use@@YAXPEBUhb_ot_shape_plan_t@@PEAUhb_buffer_t@@PEAUhb_font_t@@@Z 000000018009ae80 f   hb-ot-shaper-use.obj
 0001:00099f90       ?preprocess_text_use@@YAXPEBUhb_ot_shape_plan_t@@PEAUhb_buffer_t@@PEAUhb_font_t@@@Z 000000018009af90 f   hb-ot-shaper-use.obj
 0001:00099fa0       ??4?$machine_index_t@U?$hb_zip_iter_t@U?$hb_iota_iter_t@II@@U?$hb_filter_iter_t@U?$hb_filter_iter_t@U?$hb_zip_iter_t@U?$hb_iota_iter_t@II@@U?$hb_array_t@Uhb_glyph_info_t@@@@@@V<lambda_e52748becc06432fe81365edeb8c4003>@@AEBU<unnamed-type-hb_second>@@$0A@@@V<lambda_a2885d5959499a7c5bcf896c0de144bb>@@AEBU<unnamed-type-hb_identity>@@$0A@@@@@@@QEAAXAEBU0@@Z 000000018009afa0 f   hb-ot-shaper-use.obj
 0001:0009a070       ??D?$hb_iter_t@U?$hb_zip_iter_t@U?$hb_iota_iter_t@II@@U?$hb_filter_iter_t@U?$hb_filter_iter_t@U?$hb_zip_iter_t@U?$hb_iota_iter_t@II@@U?$hb_array_t@Uhb_glyph_info_t@@@@@@V<lambda_e52748becc06432fe81365edeb8c4003>@@AEBU<unnamed-type-hb_second>@@$0A@@@V<lambda_a2885d5959499a7c5bcf896c0de144bb>@@AEBU<unnamed-type-hb_identity>@@$0A@@@@@U?$hb_pair_t@IU?$hb_pair_t@IAEAUhb_glyph_info_t@@@@@@@@QEBA?AU?$hb_pair_t@IU?$hb_pair_t@IAEAUhb_glyph_info_t@@@@@@XZ 000000018009b070 f   hb-ot-shaper-use.obj
 0001:0009a0d0       ??E?$hb_iter_t@U?$hb_filter_iter_t@U?$hb_filter_iter_t@U?$hb_zip_iter_t@U?$hb_iota_iter_t@II@@U?$hb_array_t@Uhb_glyph_info_t@@@@@@V<lambda_e52748becc06432fe81365edeb8c4003>@@AEBU<unnamed-type-hb_second>@@$0A@@@V<lambda_a2885d5959499a7c5bcf896c0de144bb>@@AEBU<unnamed-type-hb_identity>@@$0A@@@U?$hb_pair_t@IAEAUhb_glyph_info_t@@@@@@QEGAAAEAU?$hb_filter_iter_t@U?$hb_filter_iter_t@U?$hb_zip_iter_t@U?$hb_iota_iter_t@II@@U?$hb_array_t@Uhb_glyph_info_t@@@@@@V<lambda_e52748becc06432fe81365edeb8c4003>@@AEBU<unnamed-type-hb_second>@@$0A@@@V<lambda_a2885d5959499a7c5bcf896c0de144bb>@@AEBU<unnamed-type-hb_identity>@@$0A@@@XZ 000000018009b0d0 f   hb-ot-shaper-use.obj
 0001:0009a1d0       ??F?$hb_iter_t@U?$hb_filter_iter_t@U?$hb_filter_iter_t@U?$hb_zip_iter_t@U?$hb_iota_iter_t@II@@U?$hb_array_t@Uhb_glyph_info_t@@@@@@V<lambda_e52748becc06432fe81365edeb8c4003>@@AEBU<unnamed-type-hb_second>@@$0A@@@V<lambda_a2885d5959499a7c5bcf896c0de144bb>@@AEBU<unnamed-type-hb_identity>@@$0A@@@U?$hb_pair_t@IAEAUhb_glyph_info_t@@@@@@QEGAAAEAU?$hb_filter_iter_t@U?$hb_filter_iter_t@U?$hb_zip_iter_t@U?$hb_iota_iter_t@II@@U?$hb_array_t@Uhb_glyph_info_t@@@@@@V<lambda_e52748becc06432fe81365edeb8c4003>@@AEBU<unnamed-type-hb_second>@@$0A@@@V<lambda_a2885d5959499a7c5bcf896c0de144bb>@@AEBU<unnamed-type-hb_identity>@@$0A@@@XZ 000000018009b1d0 f   hb-ot-shaper-use.obj
 0001:0009a2f0       ??G?$hb_iter_t@U?$machine_index_t@U?$hb_zip_iter_t@U?$hb_iota_iter_t@II@@U?$hb_filter_iter_t@U?$hb_filter_iter_t@U?$hb_zip_iter_t@U?$hb_iota_iter_t@II@@U?$hb_array_t@Uhb_glyph_info_t@@@@@@V<lambda_e52748becc06432fe81365edeb8c4003>@@AEBU<unnamed-type-hb_second>@@$0A@@@V<lambda_a2885d5959499a7c5bcf896c0de144bb>@@AEBU<unnamed-type-hb_identity>@@$0A@@@@@@@U?$hb_pair_t@IU?$hb_pair_t@IAEAUhb_glyph_info_t@@@@@@@@QEBA?AU?$machine_index_t@U?$hb_zip_iter_t@U?$hb_iota_iter_t@II@@U?$hb_filter_iter_t@U?$hb_filter_iter_t@U?$hb_zip_iter_t@U?$hb_iota_iter_t@II@@U?$hb_array_t@Uhb_glyph_info_t@@@@@@V<lambda_e52748becc06432fe81365edeb8c4003>@@AEBU<unnamed-type-hb_second>@@$0A@@@V<lambda_a2885d5959499a7c5bcf896c0de144bb>@@AEBU<unnamed-type-hb_identity>@@$0A@@@@@@@I@Z 000000018009b2f0 f   hb-ot-shaper-use.obj
 0001:0009a380       ??H?$hb_iter_t@U?$machine_index_t@U?$hb_zip_iter_t@U?$hb_iota_iter_t@II@@U?$hb_filter_iter_t@U?$hb_filter_iter_t@U?$hb_zip_iter_t@U?$hb_iota_iter_t@II@@U?$hb_array_t@Uhb_glyph_info_t@@@@@@V<lambda_e52748becc06432fe81365edeb8c4003>@@AEBU<unnamed-type-hb_second>@@$0A@@@V<lambda_a2885d5959499a7c5bcf896c0de144bb>@@AEBU<unnamed-type-hb_identity>@@$0A@@@@@@@U?$hb_pair_t@IU?$hb_pair_t@IAEAUhb_glyph_info_t@@@@@@@@QEBA?AU?$machine_index_t@U?$hb_zip_iter_t@U?$hb_iota_iter_t@II@@U?$hb_filter_iter_t@U?$hb_filter_iter_t@U?$hb_zip_iter_t@U?$hb_iota_iter_t@II@@U?$hb_array_t@Uhb_glyph_info_t@@@@@@V<lambda_e52748becc06432fe81365edeb8c4003>@@AEBU<unnamed-type-hb_second>@@$0A@@@V<lambda_a2885d5959499a7c5bcf896c0de144bb>@@AEBU<unnamed-type-hb_identity>@@$0A@@@@@@@I@Z 000000018009b380 f   hb-ot-shaper-use.obj
 0001:0009a410       ??Y?$hb_iter_t@U?$hb_zip_iter_t@U?$hb_iota_iter_t@II@@U?$hb_filter_iter_t@U?$hb_filter_iter_t@U?$hb_zip_iter_t@U?$hb_iota_iter_t@II@@U?$hb_array_t@Uhb_glyph_info_t@@@@@@V<lambda_e52748becc06432fe81365edeb8c4003>@@AEBU<unnamed-type-hb_second>@@$0A@@@V<lambda_a2885d5959499a7c5bcf896c0de144bb>@@AEBU<unnamed-type-hb_identity>@@$0A@@@@@U?$hb_pair_t@IU?$hb_pair_t@IAEAUhb_glyph_info_t@@@@@@@@QEGAAAEAU?$hb_zip_iter_t@U?$hb_iota_iter_t@II@@U?$hb_filter_iter_t@U?$hb_filter_iter_t@U?$hb_zip_iter_t@U?$hb_iota_iter_t@II@@U?$hb_array_t@Uhb_glyph_info_t@@@@@@V<lambda_e52748becc06432fe81365edeb8c4003>@@AEBU<unnamed-type-hb_second>@@$0A@@@V<lambda_a2885d5959499a7c5bcf896c0de144bb>@@AEBU<unnamed-type-hb_identity>@@$0A@@@@@I@Z 000000018009b410 f   hb-ot-shaper-use.obj
 0001:0009a460       ?__forward__@?$hb_iter_fallback_mixin_t@U?$hb_filter_iter_t@U?$hb_filter_iter_t@U?$hb_zip_iter_t@U?$hb_iota_iter_t@II@@U?$hb_array_t@Uhb_glyph_info_t@@@@@@V<lambda_e52748becc06432fe81365edeb8c4003>@@AEBU<unnamed-type-hb_second>@@$0A@@@V<lambda_a2885d5959499a7c5bcf896c0de144bb>@@AEBU<unnamed-type-hb_identity>@@$0A@@@U?$hb_pair_t@IAEAUhb_glyph_info_t@@@@@@QEAAXI@Z 000000018009b460 f   hb-ot-shaper-use.obj
 0001:0009a680       ?__rewind__@?$hb_iter_fallback_mixin_t@U?$hb_filter_iter_t@U?$hb_filter_iter_t@U?$hb_zip_iter_t@U?$hb_iota_iter_t@II@@U?$hb_array_t@Uhb_glyph_info_t@@@@@@V<lambda_e52748becc06432fe81365edeb8c4003>@@AEBU<unnamed-type-hb_second>@@$0A@@@V<lambda_a2885d5959499a7c5bcf896c0de144bb>@@AEBU<unnamed-type-hb_identity>@@$0A@@@U?$hb_pair_t@IAEAUhb_glyph_info_t@@@@@@QEAAXI@Z 000000018009b680 f   hb-ot-shaper-use.obj
 0001:0009a890       ?_hb_clear_substitution_flags@@YA_NPEBUhb_ot_shape_plan_t@@PEAUhb_font_t@@PEAUhb_buffer_t@@@Z 000000018009b890 f   hb-ot-shaper-use.obj
 0001:0009a8c0       ?find_syllables_use@@YAXPEAUhb_buffer_t@@@Z 000000018009b8c0 f   hb-ot-shaper-use.obj
 0001:0009be78       $LN2343                    000000018009ce78     hb-ot-shaper-use.obj
 0001:0009bee0       ?record_pref_use@@YA_NPEBUhb_ot_shape_plan_t@@PEAUhb_font_t@@PEAUhb_buffer_t@@@Z 000000018009cee0 f   hb-ot-shaper-use.obj
 0001:0009bfb0       ?record_rphf_use@@YA_NPEBUhb_ot_shape_plan_t@@PEAUhb_font_t@@PEAUhb_buffer_t@@@Z 000000018009cfb0 f   hb-ot-shaper-use.obj
 0001:0009c0a0       ?reorder_syllable_use@@YAXPEAUhb_buffer_t@@II@Z 000000018009d0a0 f   hb-ot-shaper-use.obj
 0001:0009c2d0       ?reorder_use@@YA_NPEBUhb_ot_shape_plan_t@@PEAUhb_font_t@@PEAUhb_buffer_t@@@Z 000000018009d2d0 f   hb-ot-shaper-use.obj
 0001:0009c3e0       ?setup_syllables_use@@YA_NPEBUhb_ot_shape_plan_t@@PEAUhb_font_t@@PEAUhb_buffer_t@@@Z 000000018009d3e0 f   hb-ot-shaper-use.obj
 0001:0009c5c0       ?setup_topographical_masks@@YAXPEBUhb_ot_shape_plan_t@@PEAUhb_buffer_t@@@Z 000000018009d5c0 f   hb-ot-shaper-use.obj
 0001:0009c938       $LN185                     000000018009d938     hb-ot-shaper-use.obj
 0001:0009d520       $LN454                     000000018009e520     hb-ot-shaper-vowel-constraints.obj
 0001:0009d55c       $LN453                     000000018009e55c     hb-ot-shaper-vowel-constraints.obj
 0001:0009d564       $LN452                     000000018009e564     hb-ot-shaper-vowel-constraints.obj
 0001:0009d584       $LN451                     000000018009e584     hb-ot-shaper-vowel-constraints.obj
 0001:0009d5c4       $LN450                     000000018009e5c4     hb-ot-shaper-vowel-constraints.obj
 0001:0009d5cc       $LN449                     000000018009e5cc     hb-ot-shaper-vowel-constraints.obj
 0001:0009d5f0       ?_output_with_dotted_circle@@YAXPEAUhb_buffer_t@@@Z 000000018009e5f0 f   hb-ot-shaper-vowel-constraints.obj
 0001:0009d690       ?hb_ot_ambiguous_tag_to_language@@YAPEBUhb_language_impl_t@@I@Z 000000018009e690 f   hb-ot-tag.obj
 0001:0009dd60       ?hb_ot_tags_from_complex_language@@YA_NPEBD0PEAI1@Z 000000018009ed60 f   hb-ot-tag.obj
 0001:000a0404       $LN1175                    00000001800a1404     hb-ot-tag.obj
 0001:000a0470       ?hb_ot_tags_from_language@@YAXPEBD0PEAI1@Z 00000001800a1470 f   hb-ot-tag.obj
 0001:000a0680       ?subtag_matches@@YA_NPEBD00I@Z 00000001800a1680 f   hb-ot-tag.obj
 0001:000a2120       ?hb_outline_recording_pen_close_path@@YAXPEAUhb_draw_funcs_t@@PEAXPEAUhb_draw_state_t@@1@Z 00000001800a3120 f   hb-outline.obj
 0001:000a21d0       ?hb_outline_recording_pen_cubic_to@@YAXPEAUhb_draw_funcs_t@@PEAXPEAUhb_draw_state_t@@MMMMMM1@Z 00000001800a31d0 f   hb-outline.obj
 0001:000a2430       ?hb_outline_recording_pen_line_to@@YAXPEAUhb_draw_funcs_t@@PEAXPEAUhb_draw_state_t@@MM1@Z 00000001800a3430 f   hb-outline.obj
 0001:000a24c0       ?hb_outline_recording_pen_move_to@@YAXPEAUhb_draw_funcs_t@@PEAXPEAUhb_draw_state_t@@MM1@Z 00000001800a34c0 f   hb-outline.obj
 0001:000a2550       ?hb_outline_recording_pen_quadratic_to@@YAXPEAUhb_draw_funcs_t@@PEAXPEAUhb_draw_state_t@@MMMM1@Z 00000001800a3550 f   hb-outline.obj
 0001:000a2d50       ?hb_paint_bounded_paint_color@@YAXPEAUhb_paint_funcs_t@@PEAXHI1@Z 00000001800a3d50 f   hb-paint-bounded.obj
 0001:000a2d50       ?hb_paint_bounded_paint_linear_gradient@@YAXPEAUhb_paint_funcs_t@@PEAXPEAUhb_color_line_t@@MMMMMM1@Z 00000001800a3d50 f   hb-paint-bounded.obj
 0001:000a2d50       ?hb_paint_bounded_paint_radial_gradient@@YAXPEAUhb_paint_funcs_t@@PEAXPEAUhb_color_line_t@@MMMMMM1@Z 00000001800a3d50 f   hb-paint-bounded.obj
 0001:000a2d50       ?hb_paint_bounded_paint_sweep_gradient@@YAXPEAUhb_paint_funcs_t@@PEAXPEAUhb_color_line_t@@MMMM1@Z 00000001800a3d50 f   hb-paint-bounded.obj
 0001:000a2d60       ?hb_paint_bounded_paint_image@@YAHPEAUhb_paint_funcs_t@@PEAXPEAUhb_blob_t@@IIIMPEAUhb_glyph_extents_t@@1@Z 00000001800a3d60 f   hb-paint-bounded.obj
 0001:000a2d80       ?hb_paint_bounded_pop_clip@@YAXPEAUhb_paint_funcs_t@@PEAX1@Z 00000001800a3d80 f   hb-paint-bounded.obj
 0001:000a2d80       ?hb_paint_extents_pop_transform@@YAXPEAUhb_paint_funcs_t@@PEAX1@Z 00000001800a3d80 f   hb-paint-extents.obj
 0001:000a2d90       ?hb_paint_bounded_pop_group@@YAXPEAUhb_paint_funcs_t@@PEAXW4hb_paint_composite_mode_t@@1@Z 00000001800a3d90 f   hb-paint-bounded.obj
 0001:000a2e00       $LN22                      00000001800a3e00     hb-paint-bounded.obj
 0001:000a2e30       ?hb_paint_bounded_push_clip_glyph@@YAXPEAUhb_paint_funcs_t@@PEAXIPEAUhb_font_t@@1@Z 00000001800a3e30 f   hb-paint-bounded.obj
 0001:000a2e30       ?hb_paint_bounded_push_clip_rectangle@@YAXPEAUhb_paint_funcs_t@@PEAXMMMM1@Z 00000001800a3e30 f   hb-paint-bounded.obj
 0001:000a2e40       ?hb_paint_bounded_push_group@@YAXPEAUhb_paint_funcs_t@@PEAX1@Z 00000001800a3e40 f   hb-paint-bounded.obj
 0001:000a3080       ?hb_paint_extents_paint_color@@YAXPEAUhb_paint_funcs_t@@PEAXHI1@Z 00000001800a4080 f   hb-paint-extents.obj
 0001:000a3080       ?hb_paint_extents_paint_linear_gradient@@YAXPEAUhb_paint_funcs_t@@PEAXPEAUhb_color_line_t@@MMMMMM1@Z 00000001800a4080 f   hb-paint-extents.obj
 0001:000a3080       ?hb_paint_extents_paint_radial_gradient@@YAXPEAUhb_paint_funcs_t@@PEAXPEAUhb_color_line_t@@MMMMMM1@Z 00000001800a4080 f   hb-paint-extents.obj
 0001:000a3080       ?hb_paint_extents_paint_sweep_gradient@@YAXPEAUhb_paint_funcs_t@@PEAXPEAUhb_color_line_t@@MMMM1@Z 00000001800a4080 f   hb-paint-extents.obj
 0001:000a3090       ?hb_paint_extents_paint_image@@YAHPEAUhb_paint_funcs_t@@PEAXPEAUhb_blob_t@@IIIMPEAUhb_glyph_extents_t@@1@Z 00000001800a4090 f   hb-paint-extents.obj
 0001:000a3120       ?hb_paint_extents_pop_clip@@YAXPEAUhb_paint_funcs_t@@PEAX1@Z 00000001800a4120 f   hb-paint-extents.obj
 0001:000a3130       ?hb_paint_extents_pop_group@@YAXPEAUhb_paint_funcs_t@@PEAXW4hb_paint_composite_mode_t@@1@Z 00000001800a4130 f   hb-paint-extents.obj
 0001:000a3140       ?hb_paint_extents_push_clip_glyph@@YAXPEAUhb_paint_funcs_t@@PEAXIPEAUhb_font_t@@1@Z 00000001800a4140 f   hb-paint-extents.obj
 0001:000a31b0       ?hb_paint_extents_push_clip_rectangle@@YAXPEAUhb_paint_funcs_t@@PEAXMMMM1@Z 00000001800a41b0 f   hb-paint-extents.obj
 0001:000a31f0       ?hb_paint_extents_push_group@@YAXPEAUhb_paint_funcs_t@@PEAX1@Z 00000001800a41f0 f   hb-paint-extents.obj
 0001:000a3270       ?hb_paint_extents_push_transform@@YAXPEAUhb_paint_funcs_t@@PEAXMMMMMM1@Z 00000001800a4270 f   hb-paint-extents.obj
 0001:000a37d8       $LN58                      00000001800a47d8     hb-paint-extents.obj
 0001:000a4ff0       ?_hb_shape_plan_execute_internal@@YA_NPEAUhb_shape_plan_t@@PEAUhb_font_t@@PEAUhb_buffer_t@@PEBUhb_feature_t@@I@Z 00000001800a5ff0 f   hb-shape-plan.obj
 0001:000a60b0       ?hb_ucd_combining_class@@YA?AW4hb_unicode_combining_class_t@@PEAUhb_unicode_funcs_t@@IPEAX@Z 00000001800a70b0 f   hb-ucd.obj
 0001:000a6130       ?hb_ucd_compose@@YAHPEAUhb_unicode_funcs_t@@IIPEAIPEAX@Z 00000001800a7130 f   hb-ucd.obj
 0001:000a62e0       ?hb_ucd_decompose@@YAHPEAUhb_unicode_funcs_t@@IPEAI1PEAX@Z 00000001800a72e0 f   hb-ucd.obj
 0001:000a6490       ?hb_ucd_general_category@@YA?AW4hb_unicode_general_category_t@@PEAUhb_unicode_funcs_t@@IPEAX@Z 00000001800a7490 f   hb-ucd.obj
 0001:000a6520       ?hb_ucd_mirroring@@YAIPEAUhb_unicode_funcs_t@@IPEAX@Z 00000001800a7520 f   hb-ucd.obj
 0001:000a65b0       ?hb_ucd_script@@YA?AW4hb_script_t@@PEAUhb_unicode_funcs_t@@IPEAX@Z 00000001800a75b0 f   hb-ucd.obj
 0001:000a6750       ?hb_unicode_general_category_nil@@YA?AW4hb_unicode_general_category_t@@PEAUhb_unicode_funcs_t@@IPEAX@Z 00000001800a7750 f   hb-unicode.obj
 0001:000a6760       ?hb_unicode_mirroring_nil@@YAIPEAUhb_unicode_funcs_t@@IPEAX@Z 00000001800a7760 f   hb-unicode.obj
 0001:000a6770       ?hb_unicode_script_nil@@YA?AW4hb_script_t@@PEAUhb_unicode_funcs_t@@IPEAX@Z 00000001800a7770 f   hb-unicode.obj
 0001:000a79d0       initFontIDs                00000001800a89d0 f   sunFont.obj
 0001:000a82c0       $$000000                   00000001800a92c0     MSVCRT:amdsecgs.obj
 0001:000a84b0       capture_current_context    00000001800a94b0 f   MSVCRT:gs_report.obj
 0001:000a8520       capture_previous_context   00000001800a9520 f   MSVCRT:gs_report.obj
 0001:000a85a0       $$000000                   00000001800a95a0     MSVCRT:chkstk.obj
 0001:000a8600       $$000000                   00000001800a9600     MSVCRT:svml_sfloorf4_dispatch.obj
 0001:000a8614       ?dllmain_crt_dispatch@@YAHQEAUHINSTANCE__@@KQEAX@Z 00000001800a9614 f   MSVCRT:dll_dllmain.obj
 0001:000a8664       ?dllmain_crt_process_attach@@YAHQEAUHINSTANCE__@@QEAX@Z 00000001800a9664 f   MSVCRT:dll_dllmain.obj
 0001:000a877c       ?dllmain_crt_process_detach@@YAH_N@Z 00000001800a977c f   MSVCRT:dll_dllmain.obj
 0001:000a8800       ?dllmain_dispatch@@YAHQEAUHINSTANCE__@@KQEAX@Z 00000001800a9800 f   MSVCRT:dll_dllmain.obj
 0001:000a8b30       $$000000                   00000001800a9b30     MSVCRT:svml_sfloorf4_sse2.obj
 0001:000a8b80       $$000000                   00000001800a9b80     MSVCRT:svml_sfloorf4_sse4.obj
 0001:000a9270       $$000000                   00000001800aa270     MSVCRT:guard_dispatch.obj
 0001:000a9290       $$000000                   00000001800aa290     MSVCRT:guard_xfg_dispatch.obj
 0001:000a92a6       ?fin$0@?0??dllmain_crt_process_attach@@YAHQEAUHINSTANCE__@@QEAX@Z@4HA 00000001800aa2a6 f   MSVCRT:dll_dllmain.obj
 0001:000a92bd       ?fin$0@?0??dllmain_crt_process_detach@@YAH_N@Z@4HA 00000001800aa2bd f   MSVCRT:dll_dllmain.obj
 0001:000a92d6       ?fin$1@?0??dllmain_crt_process_detach@@YAH_N@Z@4HA 00000001800aa2d6 f   MSVCRT:dll_dllmain.obj
 0001:000a92ea       ?filt$0@?0??dllmain_dispatch@@YAHQEAUHINSTANCE__@@KQEAX@Z@4HA 00000001800aa2ea f   MSVCRT:dll_dllmain.obj
 0001:000a9320       __scrt_is_nonwritable_in_current_image$filt$0 00000001800aa320 f   MSVCRT:utility.obj
 0002:00000690       FONTKEY_NT                 00000001800ab690     fontpath.obj
 0002:000006c8       ?TTSUFFIX@?1??RegistryToBaseTTNameW@@9@9 00000001800ab6c8     fontpath.obj
 0002:000006e0       ?OTSUFFIX@?1??RegistryToBaseTTNameW@@9@9 00000001800ab6e0     fontpath.obj
 0002:00000840       ?outline_funcs@?1??addToGP@@9@9 00000001800ab840     freetypeScaler.obj
 0002:00000940       ?feature_mappings@@3QBUhb_aat_feature_mapping_t@@B 00000001800ab940     hb-aat-layout.obj
 0002:00000e20       ?hb_set_digest_shifts@@3QBIB 00000001800abe20     hb-aat-layout.obj
 0002:00001130       ?_deserialize_json_trans_keys@@3QBEB 00000001800ac130     hb-buffer-serialize.obj
 0002:000011c0       ?_deserialize_json_indicies@@3QBDB 00000001800ac1c0     hb-buffer-serialize.obj
 0002:00002050       ?_deserialize_text_glyphs_trans_keys@@3QBEB 00000001800ad050     hb-buffer-serialize.obj
 0002:000020c0       ?_deserialize_text_glyphs_indicies@@3QBDB 00000001800ad0c0     hb-buffer-serialize.obj
 0002:000028b0       ?_deserialize_text_unicode_trans_keys@@3QBEB 00000001800ad8b0     hb-buffer-serialize.obj
 0002:000028d0       ?_deserialize_text_unicode_indicies@@3QBDB 00000001800ad8d0     hb-buffer-serialize.obj
 0002:00002ab0       ?_deserialize_json_key_spans@@3QBDB 00000001800adab0     hb-buffer-serialize.obj
 0002:00002af0       ?_deserialize_json_index_offsets@@3QBFB 00000001800adaf0     hb-buffer-serialize.obj
 0002:00002b70       ?_deserialize_json_trans_targs@@3QBDB 00000001800adb70     hb-buffer-serialize.obj
 0002:00002be0       ?_deserialize_json_trans_actions@@3QBDB 00000001800adbe0     hb-buffer-serialize.obj
 0002:00002c50       ?_deserialize_text_glyphs_key_spans@@3QBDB 00000001800adc50     hb-buffer-serialize.obj
 0002:00002c88       ?_deserialize_text_glyphs_eof_actions@@3QBDB 00000001800adc88     hb-buffer-serialize.obj
 0002:00002cc0       ?_deserialize_text_glyphs_index_offsets@@3QBFB 00000001800adcc0     hb-buffer-serialize.obj
 0002:00002d30       ?_deserialize_text_glyphs_trans_targs@@3QBDB 00000001800add30     hb-buffer-serialize.obj
 0002:00002d98       ?_deserialize_text_unicode_key_spans@@3QBDB 00000001800add98     hb-buffer-serialize.obj
 0002:00002db0       ?_deserialize_text_glyphs_trans_actions@@3QBDB 00000001800addb0     hb-buffer-serialize.obj
 0002:00002e18       ?_deserialize_text_unicode_index_offsets@@3QBFB 00000001800ade18     hb-buffer-serialize.obj
 0002:00002e30       ?_deserialize_text_unicode_trans_targs@@3QBDB 00000001800ade30     hb-buffer-serialize.obj
 0002:00002e40       ?_deserialize_text_unicode_trans_actions@@3QBDB 00000001800ade40     hb-buffer-serialize.obj
 0002:00002e50       ?_deserialize_text_unicode_eof_actions@@3QBDB 00000001800ade50     hb-buffer-serialize.obj
 0002:00002f60       ?_hb_os2_unicode_ranges@OT@@3QBUOS2Range@1@B 00000001800adf60     hb-common.obj
 0002:00003753       ?static_endchar_str@@3QBEB 00000001800ae753     hb-common.obj
 0002:000039e0       ?_hb_arabic_u8@@3QBEB      00000001800ae9e0     hb-common.obj
 0002:00003bd0       ?_hb_ms_language_map@@3QBUhb_ot_language_map_t@@B 00000001800aebd0     hb-common.obj
 0002:00004350       ?_hb_mac_language_map@@3QBUhb_ot_language_map_t@@B 00000001800af350     hb-common.obj
 0002:00004700       ?direction_strings@@3QAY03$$CBDA 00000001800af700     hb-common.obj
 0002:00004720       ?canon_map@@3QBDB          00000001800af720     hb-common.obj
 0002:00004874       ?hb_identity@@3U<unnamed-type-hb_identity>@@B 00000001800af874     hb-face-builder.obj
 0002:00004875       ?hb_ridentity@@3U<unnamed-type-hb_ridentity>@@B 00000001800af875     hb-face-builder.obj
 0002:000048d0       ?nil_face_loader_list@@3QBQEBDB 00000001800af8d0     hb-face.obj
 0002:000048e0       ?_hb_os2_unicode_ranges@OT@@3QBUOS2Range@1@B 00000001800af8e0     hb-face.obj
 0002:000050d0       ?_hb_arabic_u8@@3QBEB      00000001800b00d0     hb-face.obj
 0002:000052a0       ?_hb_arabic_u16@@3QBGB     00000001800b02a0     hb-face.obj
 0002:00005840       ?mapping@?1??unicode_to_macroman@OT@@YAEI@Z@4QBUunicode_to_macroman_t@?1??12@YAEI@Z@B 00000001800b0840     hb-face.obj
 0002:00005a40       ?nil_font_funcs_list@@3QBQEBDB 00000001800b0a40     hb-font.obj
 0002:00005a70       ?hb_identity@@3U<unnamed-type-hb_identity>@@B 00000001800b0a70     hb-map.obj
 0002:00005a71       ?hb_ridentity@@3U<unnamed-type-hb_ridentity>@@B 00000001800b0a71     hb-map.obj
 0002:00005a80       ?_double_parser_trans_keys@@3QBEB 00000001800b0a80     hb-number.obj
 0002:00005aa0       ?_double_parser_indicies@@3QBDB 00000001800b0aa0     hb-number.obj
 0002:00005b60       ?_double_parser_key_spans@@3QBDB 00000001800b0b60     hb-number.obj
 0002:00005b70       ?_double_parser_index_offsets@@3QBEB 00000001800b0b70     hb-number.obj
 0002:00005b80       ?_double_parser_trans_targs@@3QBDB 00000001800b0b80     hb-number.obj
 0002:00005b90       ?_double_parser_trans_actions@@3QBDB 00000001800b0b90     hb-number.obj
 0002:00005ba0       ?_powers_of_10@?1??_pow10@@YANI@Z@4QBNB 00000001800b0ba0     hb-number.obj
 0002:00005c20       ?standard_encoding_to_code@@3QBEB 00000001800b0c20     hb-ot-cff1-table.obj
 0002:00005cc0       ?expert_encoding_to_code@@3QBEB 00000001800b0cc0     hb-ot-cff1-table.obj
 0002:00005e40       ?expert_charset_to_sid@@3QBGB 00000001800b0e40     hb-ot-cff1-table.obj
 0002:00005f90       ?expert_subset_charset_to_sid@@3QBGB 00000001800b0f90     hb-ot-cff1-table.obj
 0002:00006040       ?expert_charset_sid_to_gid@@3QBUsid_to_gid_t@@B 00000001800b1040     hb-ot-cff1-table.obj
 0002:000062e0       ?expert_subset_charset_sid_to_gid@@3QBUsid_to_gid_t@@B 00000001800b12e0     hb-ot-cff1-table.obj
 0002:00006440       ?standard_encoding_to_sid@@3QBEB 00000001800b1440     hb-ot-cff1-table.obj
 0002:00006540       ?cff1_std_strings_msgstr@@3Tcff1_std_strings_msgstr_t@@B 00000001800b1540     hb-ot-cff1-table.obj
 0002:000072f0       ?format1_names_msgstr@@3Tformat1_names_msgstr_t@@B 00000001800b22f0     hb-ot-face.obj
 0002:00007a30       ?_hb_arabic_u8@@3QBEB      00000001800b2a30     hb-ot-face.obj
 0002:00007c00       ?cff1_std_strings_msgstr@@3Tcff1_std_strings_msgstr_t@@B 00000001800b2c00     hb-ot-face.obj
 0002:00008980       ?_hb_os2_unicode_ranges@OT@@3QBUOS2Range@1@B 00000001800b3980     hb-ot-face.obj
 0002:00009170       ?_hb_arabic_u8@@3QBEB      00000001800b4170     hb-ot-font.obj
 0002:00009340       ?format1_names_msgstr@@3Tformat1_names_msgstr_t@@B 00000001800b4340     hb-ot-font.obj
 0002:00009a80       ?_hb_os2_unicode_ranges@OT@@3QBUOS2Range@1@B 00000001800b4a80     hb-ot-font.obj
 0002:0000a270       ?cff1_std_strings_msgstr@@3Tcff1_std_strings_msgstr_t@@B 00000001800b5270     hb-ot-font.obj
 0002:0000aff0       ?_hb_arabic_u16@@3QBGB     00000001800b5ff0     hb-ot-font.obj
 0002:0000b590       ?cff1_std_strings_msgidx@@3QBIB 00000001800b6590     hb-ot-font.obj
 0002:0000bbb0       ?format1_names_msgidx@@3QBIB 00000001800b6bb0     hb-ot-font.obj
 0002:0000bff0       ?_hb_os2_unicode_ranges@OT@@3QBUOS2Range@1@B 00000001800b6ff0     hb-ot-layout.obj
 0002:0000c7dc       ?hb_first@@3U<unnamed-type-hb_first>@@B 00000001800b77dc     hb-ot-layout.obj
 0002:0000c7dd       ?hb_second@@3U<unnamed-type-hb_second>@@B 00000001800b77dd     hb-ot-layout.obj
 0002:0000c7de       ?hb_add@@3U<unnamed-type-hb_add>@@B 00000001800b77de     hb-ot-layout.obj
 0002:0000c7e0       ?hb_set_digest_shifts@@3QBIB 00000001800b77e0     hb-ot-layout.obj
 0002:0000cd90       ?table_tags@@3QBIB         00000001800b7d90     hb-ot-map.obj
 0002:0000cda0       ?_hb_os2_unicode_ranges@OT@@3QBUOS2Range@1@B 00000001800b7da0     hb-ot-metrics.obj
 0002:0000d590       ?format1_names_msgstr@@3Tformat1_names_msgstr_t@@B 00000001800b8590     hb-ot-metrics.obj
 0002:0000dce0       ?hb_set_digest_shifts@@3QBIB 00000001800b8ce0     hb-ot-shape-fallback.obj
 0002:0000dd70       ?common_features@@3QBUhb_ot_map_feature_t@@B 00000001800b8d70     hb-ot-shape.obj
 0002:0000dda8       ?horizontal_features@@3QBUhb_ot_map_feature_t@@B 00000001800b8da8     hb-ot-shape.obj
 0002:0000de60       ?hb_identity@@3U<unnamed-type-hb_identity>@@B 00000001800b8e60     hb-ot-shaper-arabic.obj
 0002:0000de61       ?hb_hash@@3U<unnamed-type-hb_hash>@@B 00000001800b8e61     hb-ot-shaper-arabic.obj
 0002:0000de62       ?hb_invoke@@3U<unnamed-type-hb_invoke>@@B 00000001800b8e62     hb-ot-shaper-arabic.obj
 0002:0000de63       ?hb_has@@3U<unnamed-type-hb_has>@@B 00000001800b8e63     hb-ot-shaper-arabic.obj
 0002:0000de64       ?hb_match@@3U<unnamed-type-hb_match>@@B 00000001800b8e64     hb-ot-shaper-arabic.obj
 0002:0000de65       ?hb_get@@3U<unnamed-type-hb_get>@@B 00000001800b8e65     hb-ot-shaper-arabic.obj
 0002:0000de66       ?hb_swap@@3U<unnamed-type-hb_swap>@@B 00000001800b8e66     hb-ot-shaper-arabic.obj
 0002:0000de67       ?hb_first@@3U<unnamed-type-hb_first>@@B 00000001800b8e67     hb-ot-shaper-arabic.obj
 0002:0000de68       ?hb_second@@3U<unnamed-type-hb_second>@@B 00000001800b8e68     hb-ot-shaper-arabic.obj
 0002:0000de69       ?hb_min@@3U<unnamed-type-hb_min>@@B 00000001800b8e69     hb-ot-shaper-arabic.obj
 0002:0000de6a       ?hb_max@@3U<unnamed-type-hb_max>@@B 00000001800b8e6a     hb-ot-shaper-arabic.obj
 0002:0000de6b       ?hb_clamp@@3U<unnamed-type-hb_clamp>@@B 00000001800b8e6b     hb-ot-shaper-arabic.obj
 0002:0000de6c       ?hb_add@@3U<unnamed-type-hb_add>@@B 00000001800b8e6c     hb-ot-shaper-arabic.obj
 0002:0000de6d       ?hb_iter@@3U<unnamed-type-hb_iter>@@B 00000001800b8e6d     hb-ot-shaper-arabic.obj
 0002:0000de6e       ?hb_len@@3U<unnamed-type-hb_len>@@B 00000001800b8e6e     hb-ot-shaper-arabic.obj
 0002:0000de6f       ?hb_map@@3U<unnamed-type-hb_map>@@B 00000001800b8e6f     hb-ot-shaper-arabic.obj
 0002:0000de70       ?hb_map_retains_sorting@@3U<unnamed-type-hb_map_retains_sorting>@@B 00000001800b8e70     hb-ot-shaper-arabic.obj
 0002:0000de71       ?hb_filter@@3U<unnamed-type-hb_filter>@@B 00000001800b8e71     hb-ot-shaper-arabic.obj
 0002:0000de72       ?hb_zip@@3U<unnamed-type-hb_zip>@@B 00000001800b8e72     hb-ot-shaper-arabic.obj
 0002:0000de73       ?hb_apply@@3U<unnamed-type-hb_apply>@@B 00000001800b8e73     hb-ot-shaper-arabic.obj
 0002:0000de74       ?hb_all@@3U<unnamed-type-hb_all>@@B 00000001800b8e74     hb-ot-shaper-arabic.obj
 0002:0000de75       ?hb_any@@3U<unnamed-type-hb_any>@@B 00000001800b8e75     hb-ot-shaper-arabic.obj
 0002:0000de76       ?hb_deref@@3U<unnamed-type-hb_deref>@@B 00000001800b8e76     hb-ot-shaper-arabic.obj
 0002:0000de78       ?arabic_fallback_features@@3QBIB 00000001800b8e78     hb-ot-shaper-arabic.obj
 0002:0000dea0       ?arabic_win1256_gsub_lookups@@3U0@B 00000001800b8ea0     hb-ot-shaper-arabic.obj
 0002:0000e038       ?hb_set_digest_shifts@@3QBIB 00000001800b9038     hb-ot-shaper-arabic.obj
 0002:0000e0b0       ?shaping_table@@3QAY03$$CBGA 00000001800b90b0     hb-ot-shaper-arabic.obj
 0002:0000e650       ?ligature_table@@3QBUligature_set_t@@B 00000001800b9650     hb-ot-shaper-arabic.obj
 0002:0000ea68       ?ligature_mark_table@@3QBUligature_mark_set_t@@B 00000001800b9a68     hb-ot-shaper-arabic.obj
 0002:0000ea80       ?ligature_3_table@@3QBUligature_3_set_t@@B 00000001800b9a80     hb-ot-shaper-arabic.obj
 0002:0000ea98       ?arabic_features@@3QBIB    00000001800b9a98     hb-ot-shaper-arabic.obj
 0002:0000eac0       ?arabic_state_table@@3QAY05$$CBUarabic_state_table_entry@@A 00000001800b9ac0     hb-ot-shaper-arabic.obj
 0002:0000eb70       ?joining_table@@3QBEB      00000001800b9b70     hb-ot-shaper-arabic.obj
 0002:0000f210       ?hb_min@@3U<unnamed-type-hb_min>@@B 00000001800ba210     hb-ot-shaper-hangul.obj
 0002:0000f280       ?hangul_features@@3QBIB    00000001800ba280     hb-ot-shaper-hangul.obj
 0002:0000f290       ?hb_swap@@3U<unnamed-type-hb_swap>@@B 00000001800ba290     hb-ot-shaper-hebrew.obj
 0002:0000f300       ?sDageshForms@?1??compose_hebrew@@YA_NPEBUhb_ot_shape_normalize_context_t@@IIPEAI@Z@4QBIB 00000001800ba300     hb-ot-shaper-hebrew.obj
 0002:0000f370       ?_indic_syllable_machine_trans_keys@@3QBEB 00000001800ba370     hb-ot-shaper-indic-table.obj
 0002:0000f490       ?_indic_syllable_machine_indicies@@3QBEB 00000001800ba490     hb-ot-shaper-indic-table.obj
 0002:00010f00       ?_khmer_syllable_machine_trans_keys@@3QBEB 00000001800bbf00     hb-ot-shaper-indic-table.obj
 0002:00010f60       ?_khmer_syllable_machine_indicies@@3QBDB 00000001800bbf60     hb-ot-shaper-indic-table.obj
 0002:00011320       ?_myanmar_syllable_machine_trans_keys@@3QBEB 00000001800bc320     hb-ot-shaper-indic-table.obj
 0002:00011390       ?_myanmar_syllable_machine_indicies@@3QBDB 00000001800bc390     hb-ot-shaper-indic-table.obj
 0002:00011eb0       ?indic_table@@3QBGB        00000001800bceb0     hb-ot-shaper-indic-table.obj
 0002:00012c60       ?hb_swap@@3U<unnamed-type-hb_swap>@@B 00000001800bdc60     hb-ot-shaper-indic.obj
 0002:00012c61       ?hb_min@@3U<unnamed-type-hb_min>@@B 00000001800bdc61     hb-ot-shaper-indic.obj
 0002:00012c62       ?hb_max@@3U<unnamed-type-hb_max>@@B 00000001800bdc62     hb-ot-shaper-indic.obj
 0002:00012cd0       ?_indic_syllable_machine_trans_keys@@3QBEB 00000001800bdcd0     hb-ot-shaper-indic.obj
 0002:00012df0       ?_indic_syllable_machine_key_spans@@3QBDB 00000001800bddf0     hb-ot-shaper-indic.obj
 0002:00012e80       ?_indic_syllable_machine_index_offsets@@3QBFB 00000001800bde80     hb-ot-shaper-indic.obj
 0002:00012fa0       ?_indic_syllable_machine_indicies@@3QBEB 00000001800bdfa0     hb-ot-shaper-indic.obj
 0002:00014a10       ?_indic_syllable_machine_trans_targs@@3QBEB 00000001800bfa10     hb-ot-shaper-indic.obj
 0002:00014ab0       ?_indic_syllable_machine_trans_actions@@3QBDB 00000001800bfab0     hb-ot-shaper-indic.obj
 0002:00014b50       ?_indic_syllable_machine_to_state_actions@@3QBDB 00000001800bfb50     hb-ot-shaper-indic.obj
 0002:00014be0       ?_indic_syllable_machine_from_state_actions@@3QBDB 00000001800bfbe0     hb-ot-shaper-indic.obj
 0002:00014c70       ?_indic_syllable_machine_eof_trans@@3QBFB 00000001800bfc70     hb-ot-shaper-indic.obj
 0002:00014d90       ?indic_configs@@3QBUindic_config_t@@B 00000001800bfd90     hb-ot-shaper-indic.obj
 0002:00014e80       ?indic_features@@3QBUhb_ot_map_feature_t@@B 00000001800bfe80     hb-ot-shaper-indic.obj
 0002:00014f90       ?hb_min@@3U<unnamed-type-hb_min>@@B 00000001800bff90     hb-ot-shaper-khmer.obj
 0002:00015000       ?_khmer_syllable_machine_trans_keys@@3QBEB 00000001800c0000     hb-ot-shaper-khmer.obj
 0002:00015058       ?_khmer_syllable_machine_key_spans@@3QBDB 00000001800c0058     hb-ot-shaper-khmer.obj
 0002:00015090       ?_khmer_syllable_machine_index_offsets@@3QBFB 00000001800c0090     hb-ot-shaper-khmer.obj
 0002:000150f0       ?_khmer_syllable_machine_indicies@@3QBDB 00000001800c00f0     hb-ot-shaper-khmer.obj
 0002:000154b0       ?_khmer_syllable_machine_trans_targs@@3QBDB 00000001800c04b0     hb-ot-shaper-khmer.obj
 0002:000154e8       ?_khmer_syllable_machine_trans_actions@@3QBDB 00000001800c04e8     hb-ot-shaper-khmer.obj
 0002:00015520       ?_khmer_syllable_machine_to_state_actions@@3QBDB 00000001800c0520     hb-ot-shaper-khmer.obj
 0002:00015550       ?_khmer_syllable_machine_from_state_actions@@3QBDB 00000001800c0550     hb-ot-shaper-khmer.obj
 0002:00015580       ?_khmer_syllable_machine_eof_trans@@3QBFB 00000001800c0580     hb-ot-shaper-khmer.obj
 0002:000155e0       ?khmer_features@@3QBUhb_ot_map_feature_t@@B 00000001800c05e0     hb-ot-shaper-khmer.obj
 0002:00015660       ?hb_swap@@3U<unnamed-type-hb_swap>@@B 00000001800c0660     hb-ot-shaper-myanmar.obj
 0002:00015661       ?hb_min@@3U<unnamed-type-hb_min>@@B 00000001800c0661     hb-ot-shaper-myanmar.obj
 0002:00015730       ?_myanmar_syllable_machine_trans_keys@@3QBEB 00000001800c0730     hb-ot-shaper-myanmar.obj
 0002:000157a0       ?_myanmar_syllable_machine_key_spans@@3QBDB 00000001800c07a0     hb-ot-shaper-myanmar.obj
 0002:000157e0       ?_myanmar_syllable_machine_index_offsets@@3QBFB 00000001800c07e0     hb-ot-shaper-myanmar.obj
 0002:00015850       ?_myanmar_syllable_machine_indicies@@3QBDB 00000001800c0850     hb-ot-shaper-myanmar.obj
 0002:00016368       ?_myanmar_syllable_machine_trans_targs@@3QBDB 00000001800c1368     hb-ot-shaper-myanmar.obj
 0002:000163a8       ?_myanmar_syllable_machine_trans_actions@@3QBDB 00000001800c13a8     hb-ot-shaper-myanmar.obj
 0002:000163e8       ?_myanmar_syllable_machine_to_state_actions@@3QBDB 00000001800c13e8     hb-ot-shaper-myanmar.obj
 0002:00016420       ?_myanmar_syllable_machine_from_state_actions@@3QBDB 00000001800c1420     hb-ot-shaper-myanmar.obj
 0002:00016460       ?_myanmar_syllable_machine_eof_trans@@3QBFB 00000001800c1460     hb-ot-shaper-myanmar.obj
 0002:000164d0       ?myanmar_basic_features@@3QBIB 00000001800c14d0     hb-ot-shaper-myanmar.obj
 0002:000164e0       ?myanmar_other_features@@3QBIB 00000001800c14e0     hb-ot-shaper-myanmar.obj
 0002:000165c0       ?hb_min@@3U<unnamed-type-hb_min>@@B 00000001800c15c0     hb-ot-shaper-thai.obj
 0002:00016630       ?thai_above_state_machine@@3QAY02$$CBUthai_above_state_machine_edge_t@@A 00000001800c1630     hb-ot-shaper-thai.obj
 0002:00016690       ?thai_below_state_machine@@3QAY02$$CBUthai_below_state_machine_edge_t@@A 00000001800c1690     hb-ot-shaper-thai.obj
 0002:000166d8       ?SD_mappings@?1??thai_pua_shape@@YAIIW4thai_action_t@@PEAUhb_font_t@@@Z@4QBUthai_pua_mapping_t@?1??1@YAII01@Z@B 00000001800c16d8     hb-ot-shaper-thai.obj
 0002:00016710       ?SDL_mappings@?1??thai_pua_shape@@YAIIW4thai_action_t@@PEAUhb_font_t@@@Z@4QBUthai_pua_mapping_t@?1??1@YAII01@Z@B 00000001800c1710     hb-ot-shaper-thai.obj
 0002:00016740       ?SL_mappings@?1??thai_pua_shape@@YAIIW4thai_action_t@@PEAUhb_font_t@@@Z@4QBUthai_pua_mapping_t@?1??1@YAII01@Z@B 00000001800c1740     hb-ot-shaper-thai.obj
 0002:00016790       ?RD_mappings@?1??thai_pua_shape@@YAIIW4thai_action_t@@PEAUhb_font_t@@@Z@4QBUthai_pua_mapping_t@?1??1@YAII01@Z@B 00000001800c1790     hb-ot-shaper-thai.obj
 0002:000167b0       ?hb_identity@@3U<unnamed-type-hb_identity>@@B 00000001800c17b0     hb-ot-shaper-use.obj
 0002:000167b1       ?hb_ridentity@@3U<unnamed-type-hb_ridentity>@@B 00000001800c17b1     hb-ot-shaper-use.obj
 0002:000167b2       ?hb_invoke@@3U<unnamed-type-hb_invoke>@@B 00000001800c17b2     hb-ot-shaper-use.obj
 0002:000167b3       ?hb_has@@3U<unnamed-type-hb_has>@@B 00000001800c17b3     hb-ot-shaper-use.obj
 0002:000167b4       ?hb_get@@3U<unnamed-type-hb_get>@@B 00000001800c17b4     hb-ot-shaper-use.obj
 0002:000167b5       ?hb_second@@3U<unnamed-type-hb_second>@@B 00000001800c17b5     hb-ot-shaper-use.obj
 0002:000167b6       ?hb_min@@3U<unnamed-type-hb_min>@@B 00000001800c17b6     hb-ot-shaper-use.obj
 0002:000167b7       ?hb_iter@@3U<unnamed-type-hb_iter>@@B 00000001800c17b7     hb-ot-shaper-use.obj
 0002:000167b8       ?hb_filter@@3U<unnamed-type-hb_filter>@@B 00000001800c17b8     hb-ot-shaper-use.obj
 0002:000167b9       ?hb_zip@@3U<unnamed-type-hb_zip>@@B 00000001800c17b9     hb-ot-shaper-use.obj
 0002:000167ba       ?hb_iota@@3U<unnamed-type-hb_iota>@@B 00000001800c17ba     hb-ot-shaper-use.obj
 0002:000167bb       ?hb_enumerate@@3U<unnamed-type-hb_enumerate>@@B 00000001800c17bb     hb-ot-shaper-use.obj
 0002:000167bc       ?hb_deref@@3U<unnamed-type-hb_deref>@@B 00000001800c17bc     hb-ot-shaper-use.obj
 0002:000167bd       ?machine_index@@3U<unnamed-type-machine_index>@@B 00000001800c17bd     hb-ot-shaper-use.obj
 0002:000167c0       ?hb_use_u8@@3QBEB          00000001800c17c0     hb-ot-shaper-use.obj
 0002:000174e0       ?hb_use_u16@@3QBGB         00000001800c24e0     hb-ot-shaper-use.obj
 0002:00017b90       ?use_basic_features@@3QBIB 00000001800c2b90     hb-ot-shaper-use.obj
 0002:00017bb0       ?use_topographical_features@@3QBIB 00000001800c2bb0     hb-ot-shaper-use.obj
 0002:00017bc0       ?use_other_features@@3QBIB 00000001800c2bc0     hb-ot-shaper-use.obj
 0002:00017c40       ?_use_syllable_machine_trans_keys@@3QBEB 00000001800c2c40     hb-ot-shaper-use.obj
 0002:00017d40       ?_use_syllable_machine_key_spans@@3QBDB 00000001800c2d40     hb-ot-shaper-use.obj
 0002:00017dc0       ?_use_syllable_machine_index_offsets@@3QBFB 00000001800c2dc0     hb-ot-shaper-use.obj
 0002:00017ec0       ?_use_syllable_machine_indicies@@3QBEB 00000001800c2ec0     hb-ot-shaper-use.obj
 0002:00019030       ?_use_syllable_machine_trans_targs@@3QBDB 00000001800c4030     hb-ot-shaper-use.obj
 0002:000190d0       ?_use_syllable_machine_trans_actions@@3QBDB 00000001800c40d0     hb-ot-shaper-use.obj
 0002:00019170       ?_use_syllable_machine_to_state_actions@@3QBDB 00000001800c4170     hb-ot-shaper-use.obj
 0002:000191f0       ?_use_syllable_machine_from_state_actions@@3QBDB 00000001800c41f0     hb-ot-shaper-use.obj
 0002:00019270       ?_use_syllable_machine_eof_trans@@3QBFB 00000001800c4270     hb-ot-shaper-use.obj
 0002:000193a0       ?ot_languages3@@3QBULangTag@@B 00000001800c43a0     hb-ot-tag.obj
 0002:0001ba10       ?ot_languages2@@3QBULangTag@@B 00000001800c6a10     hb-ot-tag.obj
 0002:0001c638       ?table_tags@@3QBIB         00000001800c7638     hb-shape-plan.obj
 0002:0001c930       ?nil_shaper_list@@3QBQEBDB 00000001800c7930     hb-shape.obj
 0002:0001c938       ?_hb_all_shapers@@3QBUhb_shaper_entry_t@@B 00000001800c7938     hb-shaper.obj
 0002:0001c980       ?_hb_arabic_u8@@3QBEB      00000001800c7980     hb-static.obj
 0002:0001cb50       ?_hb_os2_unicode_ranges@OT@@3QBUOS2Range@1@B 00000001800c7b50     hb-static.obj
 0002:0001d340       ?_hb_ucd_dm2_u64_map@@3QB_KB 00000001800c8340     hb-ucd.obj
 0002:0001e000       ?_hb_ucd_u8@@3QBEB         00000001800c9000     hb-ucd.obj
 0002:000224d0       ?_hb_ucd_dm1_p0_map@@3QBGB 00000001800cd4d0     hb-ucd.obj
 0002:00022b50       ?_hb_ucd_dm1_p2_map@@3QBGB 00000001800cdb50     hb-ucd.obj
 0002:00022c30       ?_hb_ucd_dm2_u32_map@@3QBIB 00000001800cdc30     hb-ucd.obj
 0002:00023630       ?_hb_ucd_sc_map@@3QBW4hb_script_t@@B 00000001800ce630     hb-ucd.obj
 0002:000238e0       ?_hb_ucd_u16@@3QBGB        00000001800ce8e0     hb-ucd.obj
 0002:00028a20       ?_hb_ucd_i16@@3QBFB        00000001800d3a20     hb-ucd.obj
 0002:00028cb0       ?_hb_emoji_u8@@3QBEB       00000001800d3cb0     hb-unicode.obj
 0002:00029208       GS_ExceptionPointers       00000001800d4208     MSVCRT:gs_report.obj
 0002:0002a410       $unwind$Glyph_Lock         00000001800d5410     ColorGlyphSurfaceData.obj
 0002:0002a420       $unwind$Java_sun_font_ColorGlyphSurfaceData_initOps 00000001800d5420     ColorGlyphSurfaceData.obj
 0002:0002a420       $unwind$Java_sun_font_ColorGlyphSurfaceData_setCurrentGlyph 00000001800d5420     ColorGlyphSurfaceData.obj
 0002:0002a420       $unwind$??1hb_aat_apply_context_t@AAT@@QEAA@XZ 00000001800d5420     hb-aat-layout.obj
 0002:0002a420       $unwind$??1hb_aat_scratch_t@AAT@@QEAA@XZ 00000001800d5420     hb-aat-layout.obj
 0002:0002a420       $unwind$?clear@hb_bit_set_t@@QEAAXXZ 00000001800d5420     hb-aat-layout.obj
 0002:0002a420       $unwind$?create_buffer_glyph_set@hb_aat_scratch_t@AAT@@QEBAPEAUhb_bit_set_t@@XZ 00000001800d5420     hb-aat-layout.obj
 0002:0002a420       $unwind$?get_value_or_null@?$Lookup@U?$IntType@G$01@OT@@@AAT@@QEBA?BGII@Z 00000001800d5420     hb-aat-layout.obj
 0002:0002a420       $unwind$?mark_set_covers@GDEF@OT@@QEBA_NII@Z 00000001800d5420     hb-aat-layout.obj
 0002:0002a420       $unwind$?neuter@?$OffsetTo@U?$AlternateSet@USmallTypes@Layout@OT@@@GSUB_impl@Layout@OT@@U?$IntType@G$01@4@X$00@OT@@QEBA_NPEAUhb_sanitize_context_t@@@Z 00000001800d5420     hb-aat-layout.obj
 0002:0002a420       $unwind$?neuter@?$OffsetTo@U?$ChainRule@USmallTypes@Layout@OT@@@OT@@U?$IntType@G$01@2@X$00@OT@@QEBA_NPEAUhb_sanitize_context_t@@@Z 00000001800d5420     hb-aat-layout.obj
 0002:0002a420       $unwind$?neuter@?$OffsetTo@U?$ChainRuleSet@USmallTypes@Layout@OT@@@OT@@U?$IntType@G$01@2@X$00@OT@@QEBA_NPEAUhb_sanitize_context_t@@@Z 00000001800d5420     hb-aat-layout.obj
 0002:0002a420       $unwind$?neuter@?$OffsetTo@U?$Ligature@USmallTypes@Layout@OT@@@GSUB_impl@Layout@OT@@U?$IntType@G$01@4@X$00@OT@@QEBA_NPEAUhb_sanitize_context_t@@@Z 00000001800d5420     hb-aat-layout.obj
 0002:0002a420       $unwind$?neuter@?$OffsetTo@U?$LigatureSet@USmallTypes@Layout@OT@@@GSUB_impl@Layout@OT@@U?$IntType@G$01@4@X$00@OT@@QEBA_NPEAUhb_sanitize_context_t@@@Z 00000001800d5420     hb-aat-layout.obj
 0002:0002a420       $unwind$?neuter@?$OffsetTo@U?$List16OfOffsetTo@USubstLookup@GSUB_impl@Layout@OT@@U?$IntType@G$01@4@@OT@@U?$IntType@G$01@2@X$00@OT@@QEBA_NPEAUhb_sanitize_context_t@@@Z 00000001800d5420     hb-aat-layout.obj
 0002:0002a420       $unwind$?neuter@?$OffsetTo@U?$Lookup@U?$OffsetTo@U?$ArrayOf@UAnchor@AAT@@U?$IntType@I$03@OT@@@OT@@U?$IntType@G$01@2@X$0A@@OT@@@AAT@@U?$IntType@I$03@OT@@X$00@OT@@QEBA_NPEAUhb_sanitize_context_t@@@Z 00000001800d5420     hb-aat-layout.obj
 0002:0002a420       $unwind$?neuter@?$OffsetTo@U?$RecordListOf@UFeature@OT@@@OT@@U?$IntType@G$01@2@X$00@OT@@QEBA_NPEAUhb_sanitize_context_t@@@Z 00000001800d5420     hb-aat-layout.obj
 0002:0002a420       $unwind$?neuter@?$OffsetTo@U?$Rule@USmallTypes@Layout@OT@@@OT@@U?$IntType@G$01@2@X$00@OT@@QEBA_NPEAUhb_sanitize_context_t@@@Z 00000001800d5420     hb-aat-layout.obj
 0002:0002a420       $unwind$?neuter@?$OffsetTo@U?$RuleSet@USmallTypes@Layout@OT@@@OT@@U?$IntType@G$01@2@X$00@OT@@QEBA_NPEAUhb_sanitize_context_t@@@Z 00000001800d5420     hb-aat-layout.obj
 0002:0002a420       $unwind$?neuter@?$OffsetTo@U?$Sequence@USmallTypes@Layout@OT@@@GSUB_impl@Layout@OT@@U?$IntType@G$01@4@X$00@OT@@QEBA_NPEAUhb_sanitize_context_t@@@Z 00000001800d5420     hb-aat-layout.obj
 0002:0002a420       $unwind$?neuter@?$OffsetTo@UAttachList@OT@@U?$IntType@G$01@2@X$00@OT@@QEBA_NPEAUhb_sanitize_context_t@@@Z 00000001800d5420     hb-aat-layout.obj
 0002:0002a420       $unwind$?neuter@?$OffsetTo@UAttachPoint@OT@@U?$IntType@G$01@2@X$00@OT@@QEBA_NPEAUhb_sanitize_context_t@@@Z 00000001800d5420     hb-aat-layout.obj
 0002:0002a420       $unwind$?neuter@?$OffsetTo@UCaretValue@OT@@U?$IntType@G$01@2@X$00@OT@@QEBA_NPEAUhb_sanitize_context_t@@@Z 00000001800d5420     hb-aat-layout.obj
 0002:0002a420       $unwind$?neuter@?$OffsetTo@UClassDef@OT@@U?$IntType@G$01@2@X$00@OT@@QEBA_NPEAUhb_sanitize_context_t@@@Z 00000001800d5420     hb-aat-layout.obj
 0002:0002a420       $unwind$?neuter@?$OffsetTo@UCondition@OT@@U?$IntType@I$02@2@X$00@OT@@QEBA_NPEAUhb_sanitize_context_t@@@Z 00000001800d5420     hb-aat-layout.obj
 0002:0002a420       $unwind$?neuter@?$OffsetTo@UCondition@OT@@U?$IntType@I$03@2@X$00@OT@@QEBA_NPEAUhb_sanitize_context_t@@@Z 00000001800d5420     hb-aat-layout.obj
 0002:0002a420       $unwind$?neuter@?$OffsetTo@UConditionSet@OT@@U?$IntType@I$03@2@X$00@OT@@QEBA_NPEAUhb_sanitize_context_t@@@Z 00000001800d5420     hb-aat-layout.obj
 0002:0002a420       $unwind$?neuter@?$OffsetTo@UCoverage@Common@Layout@OT@@U?$IntType@G$01@4@X$00@OT@@QEBA_NPEAUhb_sanitize_context_t@@@Z 00000001800d5420     hb-aat-layout.obj
 0002:0002a420       $unwind$?neuter@?$OffsetTo@UCoverage@Common@Layout@OT@@U?$IntType@I$03@4@X$00@OT@@QEBA_NPEAUhb_sanitize_context_t@@@Z 00000001800d5420     hb-aat-layout.obj
 0002:0002a420       $unwind$?neuter@?$OffsetTo@UDevice@OT@@U?$IntType@G$01@2@X$00@OT@@QEBA_NPEAUhb_sanitize_context_t@@@Z 00000001800d5420     hb-aat-layout.obj
 0002:0002a420       $unwind$?neuter@?$OffsetTo@UFeature@OT@@U?$IntType@G$01@2@X$00@OT@@QEBA_NPEAUhb_sanitize_context_t@@@Z 00000001800d5420     hb-aat-layout.obj
 0002:0002a420       $unwind$?neuter@?$OffsetTo@UFeature@OT@@U?$IntType@I$03@2@X$00@OT@@QEBA_NPEAUhb_sanitize_context_t@@@Z 00000001800d5420     hb-aat-layout.obj
 0002:0002a420       $unwind$?neuter@?$OffsetTo@UFeatureParams@OT@@U?$IntType@G$01@2@X$00@OT@@QEBA_NPEAUhb_sanitize_context_t@@@Z 00000001800d5420     hb-aat-layout.obj
 0002:0002a420       $unwind$?neuter@?$OffsetTo@UFeatureTableSubstitution@OT@@U?$IntType@I$03@2@X$00@OT@@QEBA_NPEAUhb_sanitize_context_t@@@Z 00000001800d5420     hb-aat-layout.obj
 0002:0002a420       $unwind$?neuter@?$OffsetTo@UFeatureVariations@OT@@U?$IntType@I$03@2@X$00@OT@@QEBA_NPEAUhb_sanitize_context_t@@@Z 00000001800d5420     hb-aat-layout.obj
 0002:0002a420       $unwind$?neuter@?$OffsetTo@UItemVariationStore@OT@@U?$IntType@I$03@2@X$00@OT@@QEBA_NPEAUhb_sanitize_context_t@@@Z 00000001800d5420     hb-aat-layout.obj
 0002:0002a420       $unwind$?neuter@?$OffsetTo@ULangSys@OT@@U?$IntType@G$01@2@X$00@OT@@QEBA_NPEAUhb_sanitize_context_t@@@Z 00000001800d5420     hb-aat-layout.obj
 0002:0002a420       $unwind$?neuter@?$OffsetTo@ULigCaretList@OT@@U?$IntType@G$01@2@X$00@OT@@QEBA_NPEAUhb_sanitize_context_t@@@Z 00000001800d5420     hb-aat-layout.obj
 0002:0002a420       $unwind$?neuter@?$OffsetTo@ULigGlyph@OT@@U?$IntType@G$01@2@X$00@OT@@QEBA_NPEAUhb_sanitize_context_t@@@Z 00000001800d5420     hb-aat-layout.obj
 0002:0002a420       $unwind$?neuter@?$OffsetTo@UMarkGlyphSets@OT@@U?$IntType@G$01@2@X$00@OT@@QEBA_NPEAUhb_sanitize_context_t@@@Z 00000001800d5420     hb-aat-layout.obj
 0002:0002a420       $unwind$?neuter@?$OffsetTo@URecordListOfScript@OT@@U?$IntType@G$01@2@X$00@OT@@QEBA_NPEAUhb_sanitize_context_t@@@Z 00000001800d5420     hb-aat-layout.obj
 0002:0002a420       $unwind$?neuter@?$OffsetTo@UScript@OT@@U?$IntType@G$01@2@X$00@OT@@QEBA_NPEAUhb_sanitize_context_t@@@Z 00000001800d5420     hb-aat-layout.obj
 0002:0002a420       $unwind$?neuter@?$OffsetTo@USubstLookup@GSUB_impl@Layout@OT@@U?$IntType@G$01@4@X$00@OT@@QEBA_NPEAUhb_sanitize_context_t@@@Z 00000001800d5420     hb-aat-layout.obj
 0002:0002a420       $unwind$?neuter@?$OffsetTo@USubstLookupSubTable@GSUB_impl@Layout@OT@@U?$IntType@G$01@4@X$00@OT@@QEBA_NPEAUhb_sanitize_context_t@@@Z 00000001800d5420     hb-aat-layout.obj
 0002:0002a420       $unwind$?neuter@?$OffsetTo@UTrackData@AAT@@U?$IntType@G$01@OT@@X$00@OT@@QEBA_NPEAUhb_sanitize_context_t@@@Z 00000001800d5420     hb-aat-layout.obj
 0002:0002a420       $unwind$?neuter@?$OffsetTo@UVarData@OT@@U?$IntType@I$03@2@X$00@OT@@QEBA_NPEAUhb_sanitize_context_t@@@Z 00000001800d5420     hb-aat-layout.obj
 0002:0002a420       $unwind$?neuter@?$OffsetTo@UVarRegionList@OT@@U?$IntType@I$03@2@X$00@OT@@QEBA_NPEAUhb_sanitize_context_t@@@Z 00000001800d5420     hb-aat-layout.obj
 0002:0002a420       $unwind$?_hb_mapped_file_destroy@@YAXPEAX@Z 00000001800d5420     hb-blob.obj
 0002:0002a420       $unwind$hb_blob_create_sub_blob 00000001800d5420     hb-blob.obj
 0002:0002a420       $unwind$?reset@hb_buffer_t@@QEAAXXZ 00000001800d5420     hb-buffer.obj
 0002:0002a420       $unwind$hb_buffer_create   00000001800d5420     hb-buffer.obj
 0002:0002a420       $unwind$hb_buffer_get_glyph_positions 00000001800d5420     hb-buffer.obj
 0002:0002a420       $unwind$?load_num_glyphs@hb_face_t@@AEBAIXZ 00000001800d5420     hb-common.obj
 0002:0002a420       $unwind$?load_upem@hb_face_t@@AEBAIXZ 00000001800d5420     hb-common.obj
 0002:0002a420       $unwind$?neuter@?$OffsetTo@UDeltaSetIndexMap@OT@@U?$IntType@I$03@2@X$00@OT@@QEBA_NPEAUhb_sanitize_context_t@@@Z 00000001800d5420     hb-common.obj
 0002:0002a420       $unwind$hb_language_matches 00000001800d5420     hb-common.obj
 0002:0002a420       $unwind$?create@hb_draw_extents_funcs_lazy_loader_t@@SAPEAUhb_draw_funcs_t@@XZ 00000001800d5420     hb-draw.obj
 0002:0002a420       $unwind$?hb_draw_extents_cubic_to@@YAXPEAUhb_draw_funcs_t@@PEAXPEAUhb_draw_state_t@@MMMMMM1@Z 00000001800d5420     hb-draw.obj
 0002:0002a420       $unwind$?hb_draw_extents_quadratic_to@@YAXPEAUhb_draw_funcs_t@@PEAXPEAUhb_draw_state_t@@MMMM1@Z 00000001800d5420     hb-draw.obj
 0002:0002a420       $unwind$??$hb_object_create@Uhb_face_t@@$$V@@YAPEAUhb_face_t@@XZ 00000001800d5420     hb-face.obj
 0002:0002a420       $unwind$?_hb_face_for_data_closure_destroy@@YAXPEAX@Z 00000001800d5420     hb-face.obj
 0002:0002a420       $unwind$?neuter@?$OffsetTo@UCmapSubtable@OT@@U?$IntType@I$03@2@X$00@OT@@QEBA_NPEAUhb_sanitize_context_t@@@Z 00000001800d5420     hb-face.obj
 0002:0002a420       $unwind$?neuter@?$OffsetTo@UDefaultUVS@OT@@U?$IntType@I$03@2@X$00@OT@@QEBA_NPEAUhb_sanitize_context_t@@@Z 00000001800d5420     hb-face.obj
 0002:0002a420       $unwind$?neuter@?$OffsetTo@UNonDefaultUVS@OT@@U?$IntType@I$03@2@X$00@OT@@QEBA_NPEAUhb_sanitize_context_t@@@Z 00000001800d5420     hb-face.obj
 0002:0002a420       $unwind$?neuter@?$OffsetTo@UOpenTypeOffsetTable@OT@@U?$IntType@I$03@2@X$00@OT@@QEBA_NPEAUhb_sanitize_context_t@@@Z 00000001800d5420     hb-face.obj
 0002:0002a420       $unwind$hb_font_funcs_create 00000001800d5420     hb-font.obj
 0002:0002a420       $unwind$?cleanupFontInfo@@YAXPEAX@Z 00000001800d5420     hb-jdk-font.obj
 0002:0002a420       $unwind$?process_op@?$opset_t@Unumber_t@CFF@@@CFF@@SAXIAEAU?$interp_env_t@Unumber_t@CFF@@@2@@Z 00000001800d5420     hb-ot-cff1-table.obj
 0002:0002a420       $unwind$?process_op@?$cs_opset_t@Unumber_t@CFF@@Ucff2_cs_opset_extents_t@@U?$cff2_cs_interp_env_t@Unumber_t@CFF@@@2@Ucff2_extents_param_t@@Ucff2_path_procs_extents_t@@@CFF@@SAXIAEAU?$cff2_cs_interp_env_t@Unumber_t@CFF@@@2@AEAUcff2_extents_param_t@@@Z 00000001800d5420     hb-ot-cff2-table.obj
 0002:0002a420       $unwind$??$sanitize@$$V@Paint@OT@@QEBA_NPEAUhb_sanitize_context_t@@@Z 00000001800d5420     hb-ot-color.obj
 0002:0002a420       $unwind$?neuter@?$OffsetTo@U?$ColorLine@UNoVariable@OT@@@OT@@U?$IntType@I$02@2@X$00@OT@@QEBA_NPEAUhb_sanitize_context_t@@@Z 00000001800d5420     hb-ot-color.obj
 0002:0002a420       $unwind$?neuter@?$OffsetTo@U?$ColorLine@UVariable@OT@@@OT@@U?$IntType@I$02@2@X$00@OT@@QEBA_NPEAUhb_sanitize_context_t@@@Z 00000001800d5420     hb-ot-color.obj
 0002:0002a420       $unwind$?neuter@?$OffsetTo@U?$NoVariable@UAffine2x3@OT@@@OT@@U?$IntType@I$02@2@X$00@OT@@QEBA_NPEAUhb_sanitize_context_t@@@Z 00000001800d5420     hb-ot-color.obj
 0002:0002a420       $unwind$?neuter@?$OffsetTo@U?$Variable@UAffine2x3@OT@@@OT@@U?$IntType@I$02@2@X$00@OT@@QEBA_NPEAUhb_sanitize_context_t@@@Z 00000001800d5420     hb-ot-color.obj
 0002:0002a420       $unwind$?neuter@?$OffsetTo@UBaseGlyphList@OT@@U?$IntType@I$03@2@X$00@OT@@QEBA_NPEAUhb_sanitize_context_t@@@Z 00000001800d5420     hb-ot-color.obj
 0002:0002a420       $unwind$?neuter@?$OffsetTo@UClipBox@OT@@U?$IntType@I$02@2@X$00@OT@@QEBA_NPEAUhb_sanitize_context_t@@@Z 00000001800d5420     hb-ot-color.obj
 0002:0002a420       $unwind$?neuter@?$OffsetTo@UClipList@OT@@U?$IntType@I$03@2@X$00@OT@@QEBA_NPEAUhb_sanitize_context_t@@@Z 00000001800d5420     hb-ot-color.obj
 0002:0002a420       $unwind$?neuter@?$OffsetTo@UIndexSubtable@OT@@U?$IntType@I$03@2@X$00@OT@@QEBA_NPEAUhb_sanitize_context_t@@@Z 00000001800d5420     hb-ot-color.obj
 0002:0002a420       $unwind$?neuter@?$OffsetTo@ULayerList@OT@@U?$IntType@I$03@2@X$00@OT@@QEBA_NPEAUhb_sanitize_context_t@@@Z 00000001800d5420     hb-ot-color.obj
 0002:0002a420       $unwind$?neuter@?$OffsetTo@UPaint@OT@@U?$IntType@I$02@2@X$00@OT@@QEBA_NPEAUhb_sanitize_context_t@@@Z 00000001800d5420     hb-ot-color.obj
 0002:0002a420       $unwind$?neuter@?$OffsetTo@UPaint@OT@@U?$IntType@I$03@2@X$00@OT@@QEBA_NPEAUhb_sanitize_context_t@@@Z 00000001800d5420     hb-ot-color.obj
 0002:0002a420       $unwind$?neuter@?$OffsetTo@USBIXStrike@OT@@U?$IntType@I$03@2@X$00@OT@@QEBA_NPEAUhb_sanitize_context_t@@@Z 00000001800d5420     hb-ot-color.obj
 0002:0002a420       $unwind$?_hb_ot_font_destroy@@YAXPEAX@Z 00000001800d5420     hb-ot-font.obj
 0002:0002a420       $unwind$?process_op@dict_opset_t@CFF@@SAXIAEAU?$interp_env_t@Unumber_t@CFF@@@2@@Z 00000001800d5420     hb-ot-font.obj
 0002:0002a420       $unwind$?recurse@hb_paint_context_t@OT@@QEAAXAEBUPaint@2@@Z 00000001800d5420     hb-ot-font.obj
 0002:0002a420       $unwind$?release_scratch@accelerator_t@COLR@OT@@AEBAXPEAUhb_colr_scratch_t@@@Z 00000001800d5420     hb-ot-font.obj
 0002:0002a420       $unwind$??$dispatch@Uhb_accelerate_subtables_context_t@OT@@$$V@Context@OT@@QEBA?AUhb_empty_t@@PEAUhb_accelerate_subtables_context_t@1@@Z 00000001800d5420     hb-ot-layout.obj
 0002:0002a420       $unwind$??$dispatch@Uhb_accelerate_subtables_context_t@OT@@$$V@SubstLookupSubTable@GSUB_impl@Layout@OT@@QEBA?AUhb_empty_t@@PEAUhb_accelerate_subtables_context_t@3@I@Z 00000001800d5420     hb-ot-layout.obj
 0002:0002a420       $unwind$?match_class@OT@@YA_NAEAUhb_glyph_info_t@@IPEBX@Z 00000001800d5420     hb-ot-layout.obj
 0002:0002a420       $unwind$?neuter@?$OffsetTo@U?$List16OfOffsetTo@UPosLookup@GPOS_impl@Layout@OT@@U?$IntType@G$01@4@@OT@@U?$IntType@G$01@2@X$00@OT@@QEBA_NPEAUhb_sanitize_context_t@@@Z 00000001800d5420     hb-ot-layout.obj
 0002:0002a420       $unwind$?neuter@?$OffsetTo@U?$PairSet@USmallTypes@Layout@OT@@@GPOS_impl@Layout@OT@@U?$IntType@G$01@4@X$00@OT@@QEBA_NPEAUhb_sanitize_context_t@@@Z 00000001800d5420     hb-ot-layout.obj
 0002:0002a420       $unwind$?neuter@?$OffsetTo@UAnchor@GPOS_impl@Layout@OT@@U?$IntType@G$01@4@UAnchorMatrix@234@$00@OT@@QEBA_NPEAUhb_sanitize_context_t@@@Z 00000001800d5420     hb-ot-layout.obj
 0002:0002a420       $unwind$?neuter@?$OffsetTo@UAnchor@GPOS_impl@Layout@OT@@U?$IntType@G$01@4@UCursivePosFormat1@234@$00@OT@@QEBA_NPEAUhb_sanitize_context_t@@@Z 00000001800d5420     hb-ot-layout.obj
 0002:0002a420       $unwind$?neuter@?$OffsetTo@UAnchor@GPOS_impl@Layout@OT@@U?$IntType@G$01@4@X$00@OT@@QEBA_NPEAUhb_sanitize_context_t@@@Z 00000001800d5420     hb-ot-layout.obj
 0002:0002a420       $unwind$?neuter@?$OffsetTo@UAnchorMatrix@GPOS_impl@Layout@OT@@U?$IntType@G$01@4@X$00@OT@@QEBA_NPEAUhb_sanitize_context_t@@@Z 00000001800d5420     hb-ot-layout.obj
 0002:0002a420       $unwind$?neuter@?$OffsetTo@UDevice@OT@@U?$IntType@G$01@2@UValueBase@GPOS_impl@Layout@2@$00@OT@@QEBA_NPEAUhb_sanitize_context_t@@@Z 00000001800d5420     hb-ot-layout.obj
 0002:0002a420       $unwind$?neuter@?$OffsetTo@ULigatureArray@GPOS_impl@Layout@OT@@U?$IntType@G$01@4@X$00@OT@@QEBA_NPEAUhb_sanitize_context_t@@@Z 00000001800d5420     hb-ot-layout.obj
 0002:0002a420       $unwind$?neuter@?$OffsetTo@UMarkArray@GPOS_impl@Layout@OT@@U?$IntType@G$01@4@X$00@OT@@QEBA_NPEAUhb_sanitize_context_t@@@Z 00000001800d5420     hb-ot-layout.obj
 0002:0002a420       $unwind$?neuter@?$OffsetTo@UPosLookup@GPOS_impl@Layout@OT@@U?$IntType@G$01@4@X$00@OT@@QEBA_NPEAUhb_sanitize_context_t@@@Z 00000001800d5420     hb-ot-layout.obj
 0002:0002a420       $unwind$?neuter@?$OffsetTo@UPosLookupSubTable@GPOS_impl@Layout@OT@@U?$IntType@G$01@4@X$00@OT@@QEBA_NPEAUhb_sanitize_context_t@@@Z 00000001800d5420     hb-ot-layout.obj
 0002:0002a420       $unwind$?neuter@?$OffsetTo@UItemVariationStore@OT@@U?$IntType@G$01@2@X$00@OT@@QEBA_NPEAUhb_sanitize_context_t@@@Z 00000001800d5420     hb-ot-metrics.obj
 0002:0002a420       $unwind$?fini@hb_ot_shape_plan_t@@QEAAXXZ 00000001800d5420     hb-ot-shape.obj
 0002:0002a420       $unwind$?neuter@?$OffsetTo@UAxisValue@OT@@U?$IntType@G$01@2@X$00@OT@@QEBA_NPEAUhb_sanitize_context_t@@@Z 00000001800d5420     hb-ot-shape.obj
 0002:0002a420       $unwind$??$push@UCoverage@Common@Layout@OT@@@hb_serialize_context_t@@QEAAPEAUCoverage@Common@Layout@OT@@XZ 00000001800d5420     hb-ot-shaper-arabic.obj
 0002:0002a420       $unwind$?data_destroy_arabic@@YAXPEAX@Z 00000001800d5420     hb-ot-shaper-arabic.obj
 0002:0002a420       $unwind$?override_features_indic@@YAXPEAUhb_ot_shape_planner_t@@@Z 00000001800d5420     hb-ot-shaper-indic.obj
 0002:0002a420       $unwind$?setup_masks_indic@@YAXPEBUhb_ot_shape_plan_t@@PEAUhb_buffer_t@@PEAUhb_font_t@@@Z 00000001800d5420     hb-ot-shaper-indic.obj
 0002:0002a420       $unwind$?override_features_khmer@@YAXPEAUhb_ot_shape_planner_t@@@Z 00000001800d5420     hb-ot-shaper-khmer.obj
 0002:0002a420       $unwind$?setup_masks_khmer@@YAXPEBUhb_ot_shape_plan_t@@PEAUhb_buffer_t@@PEAUhb_font_t@@@Z 00000001800d5420     hb-ot-shaper-khmer.obj
 0002:0002a420       $unwind$?setup_masks_myanmar@@YAXPEBUhb_ot_shape_plan_t@@PEAUhb_buffer_t@@PEAUhb_font_t@@@Z 00000001800d5420     hb-ot-shaper-myanmar.obj
 0002:0002a420       $unwind$??G?$hb_iter_t@U?$machine_index_t@U?$hb_zip_iter_t@U?$hb_iota_iter_t@II@@U?$hb_filter_iter_t@U?$hb_filter_iter_t@U?$hb_zip_iter_t@U?$hb_iota_iter_t@II@@U?$hb_array_t@Uhb_glyph_info_t@@@@@@V<lambda_e52748becc06432fe81365edeb8c4003>@@AEBU<unnamed-type-hb_second>@@$0A@@@V<lambda_a2885d5959499a7c5bcf896c0de144bb>@@AEBU<unnamed-type-hb_identity>@@$0A@@@@@@@U?$hb_pair_t@IU?$hb_pair_t@IAEAUhb_glyph_info_t@@@@@@@@QEBA?AU?$machine_index_t@U?$hb_zip_iter_t@U?$hb_iota_iter_t@II@@U?$hb_filter_iter_t@U?$hb_filter_iter_t@U?$hb_zip_iter_t@U?$hb_iota_iter_t@II@@U?$hb_array_t@Uhb_glyph_info_t@@@@@@V<lambda_e52748becc06432fe81365edeb8c4003>@@AEBU<unnamed-type-hb_second>@@$0A@@@V<lambda_a2885d5959499a7c5bcf896c0de144bb>@@AEBU<unnamed-type-hb_identity>@@$0A@@@@@@@I@Z 00000001800d5420     hb-ot-shaper-use.obj
 0002:0002a420       $unwind$??H?$hb_iter_t@U?$machine_index_t@U?$hb_zip_iter_t@U?$hb_iota_iter_t@II@@U?$hb_filter_iter_t@U?$hb_filter_iter_t@U?$hb_zip_iter_t@U?$hb_iota_iter_t@II@@U?$hb_array_t@Uhb_glyph_info_t@@@@@@V<lambda_e52748becc06432fe81365edeb8c4003>@@AEBU<unnamed-type-hb_second>@@$0A@@@V<lambda_a2885d5959499a7c5bcf896c0de144bb>@@AEBU<unnamed-type-hb_identity>@@$0A@@@@@@@U?$hb_pair_t@IU?$hb_pair_t@IAEAUhb_glyph_info_t@@@@@@@@QEBA?AU?$machine_index_t@U?$hb_zip_iter_t@U?$hb_iota_iter_t@II@@U?$hb_filter_iter_t@U?$hb_filter_iter_t@U?$hb_zip_iter_t@U?$hb_iota_iter_t@II@@U?$hb_array_t@Uhb_glyph_info_t@@@@@@V<lambda_e52748becc06432fe81365edeb8c4003>@@AEBU<unnamed-type-hb_second>@@$0A@@@V<lambda_a2885d5959499a7c5bcf896c0de144bb>@@AEBU<unnamed-type-hb_identity>@@$0A@@@@@@@I@Z 00000001800d5420     hb-ot-shaper-use.obj
 0002:0002a420       $unwind$??Y?$hb_iter_t@U?$hb_zip_iter_t@U?$hb_iota_iter_t@II@@U?$hb_filter_iter_t@U?$hb_filter_iter_t@U?$hb_zip_iter_t@U?$hb_iota_iter_t@II@@U?$hb_array_t@Uhb_glyph_info_t@@@@@@V<lambda_e52748becc06432fe81365edeb8c4003>@@AEBU<unnamed-type-hb_second>@@$0A@@@V<lambda_a2885d5959499a7c5bcf896c0de144bb>@@AEBU<unnamed-type-hb_identity>@@$0A@@@@@U?$hb_pair_t@IU?$hb_pair_t@IAEAUhb_glyph_info_t@@@@@@@@QEGAAAEAU?$hb_zip_iter_t@U?$hb_iota_iter_t@II@@U?$hb_filter_iter_t@U?$hb_filter_iter_t@U?$hb_zip_iter_t@U?$hb_iota_iter_t@II@@U?$hb_array_t@Uhb_glyph_info_t@@@@@@V<lambda_e52748becc06432fe81365edeb8c4003>@@AEBU<unnamed-type-hb_second>@@$0A@@@V<lambda_a2885d5959499a7c5bcf896c0de144bb>@@AEBU<unnamed-type-hb_identity>@@$0A@@@@@I@Z 00000001800d5420     hb-ot-shaper-use.obj
 0002:0002a420       $unwind$?data_destroy_use@@YAXPEAX@Z 00000001800d5420     hb-ot-shaper-use.obj
 0002:0002a420       $unwind$?setup_masks_use@@YAXPEBUhb_ot_shape_plan_t@@PEAUhb_buffer_t@@PEAUhb_font_t@@@Z 00000001800d5420     hb-ot-shaper-use.obj
 0002:0002a420       $unwind$?_hb_preprocess_text_vowel_constraints@@YAXPEBUhb_ot_shape_plan_t@@PEAUhb_buffer_t@@PEAUhb_font_t@@@Z 00000001800d5420     hb-ot-shaper-vowel-constraints.obj
 0002:0002a420       $unwind$?_output_with_dotted_circle@@YAXPEAUhb_buffer_t@@@Z 00000001800d5420     hb-ot-shaper-vowel-constraints.obj
 0002:0002a420       $unwind$?hb_paint_extents_push_group@@YAXPEAUhb_paint_funcs_t@@PEAX1@Z 00000001800d5420     hb-paint-extents.obj
 0002:0002a420       $unwind$initFontIDs        00000001800d5420     sunFont.obj
 0002:0002a420       $unwind$__raise_securityfailure 00000001800d5420     MSVCRT:gs_report.obj
 0002:0002a420       $unwind$__scrt_initialize_crt 00000001800d5420     MSVCRT:utility.obj
 0002:0002a420       $unwind$__scrt_initialize_onexit_tables 00000001800d5420     MSVCRT:utility.obj
 0002:0002a420       $unwind$__scrt_release_startup_lock 00000001800d5420     MSVCRT:utility.obj
 0002:0002a420       $unwind$__scrt_uninitialize_crt 00000001800d5420     MSVCRT:utility.obj
 0002:0002a428       $unwind$RefineBounds       00000001800d5428     DrawGlyphList.obj
 0002:0002a438       $chain$0$RefineBounds      00000001800d5438     DrawGlyphList.obj
 0002:0002a44c       $chain$2$RefineBounds      00000001800d544c     DrawGlyphList.obj
 0002:0002a464       $chain$3$RefineBounds      00000001800d5464     DrawGlyphList.obj
 0002:0002a474       $chain$4$RefineBounds      00000001800d5474     DrawGlyphList.obj
 0002:0002a484       $unwind$setupBlitVector    00000001800d5484     DrawGlyphList.obj
 0002:0002a4a0       $chain$0$setupBlitVector   00000001800d54a0     DrawGlyphList.obj
 0002:0002a4b4       $chain$1$setupBlitVector   00000001800d54b4     DrawGlyphList.obj
 0002:0002a4c8       $chain$2$setupBlitVector   00000001800d54c8     DrawGlyphList.obj
 0002:0002a4dc       $chain$3$setupBlitVector   00000001800d54dc     DrawGlyphList.obj
 0002:0002a4ec       $chain$4$setupBlitVector   00000001800d54ec     DrawGlyphList.obj
 0002:0002a4fc       $chain$5$setupBlitVector   00000001800d54fc     DrawGlyphList.obj
 0002:0002a50c       $unwind$setupLCDBlitVector 00000001800d550c     DrawGlyphList.obj
 0002:0002a530       $chain$5$setupLCDBlitVector 00000001800d5530     DrawGlyphList.obj
 0002:0002a558       $chain$6$setupLCDBlitVector 00000001800d5558     DrawGlyphList.obj
 0002:0002a568       $unwind$Java_sun_java2d_loops_DrawGlyphListAA_DrawGlyphListAA 00000001800d5568     DrawGlyphList.obj
 0002:0002a568       $unwind$Java_sun_java2d_loops_DrawGlyphList_DrawGlyphList 00000001800d5568     DrawGlyphList.obj
 0002:0002a57c       $chain$0$Java_sun_java2d_loops_DrawGlyphListAA_DrawGlyphListAA 00000001800d557c     DrawGlyphList.obj
 0002:0002a57c       $chain$0$Java_sun_java2d_loops_DrawGlyphList_DrawGlyphList 00000001800d557c     DrawGlyphList.obj
 0002:0002a590       $chain$1$Java_sun_java2d_loops_DrawGlyphListAA_DrawGlyphListAA 00000001800d5590     DrawGlyphList.obj
 0002:0002a590       $chain$1$Java_sun_java2d_loops_DrawGlyphList_DrawGlyphList 00000001800d5590     DrawGlyphList.obj
 0002:0002a5a4       $chain$2$Java_sun_java2d_loops_DrawGlyphListAA_DrawGlyphListAA 00000001800d55a4     DrawGlyphList.obj
 0002:0002a5a4       $chain$2$Java_sun_java2d_loops_DrawGlyphList_DrawGlyphList 00000001800d55a4     DrawGlyphList.obj
 0002:0002a5b4       $chain$3$Java_sun_java2d_loops_DrawGlyphListAA_DrawGlyphListAA 00000001800d55b4     DrawGlyphList.obj
 0002:0002a5b4       $chain$3$Java_sun_java2d_loops_DrawGlyphList_DrawGlyphList 00000001800d55b4     DrawGlyphList.obj
 0002:0002a5c4       $unwind$drawGlyphList      00000001800d55c4     DrawGlyphList.obj
 0002:0002a5e4       $unwind$drawGlyphListLCD   00000001800d55e4     DrawGlyphList.obj
 0002:0002a600       $chain$1$drawGlyphListLCD  00000001800d5600     DrawGlyphList.obj
 0002:0002a618       $chain$2$drawGlyphListLCD  00000001800d5618     DrawGlyphList.obj
 0002:0002a628       $unwind$Java_sun_java2d_loops_DrawGlyphListLCD_DrawGlyphListLCD 00000001800d5628     DrawGlyphList.obj
 0002:0002a638       $chain$0$Java_sun_java2d_loops_DrawGlyphListLCD_DrawGlyphListLCD 00000001800d5638     DrawGlyphList.obj
 0002:0002a64c       $chain$2$Java_sun_java2d_loops_DrawGlyphListLCD_DrawGlyphListLCD 00000001800d564c     DrawGlyphList.obj
 0002:0002a664       $chain$3$Java_sun_java2d_loops_DrawGlyphListLCD_DrawGlyphListLCD 00000001800d5664     DrawGlyphList.obj
 0002:0002a674       $chain$4$Java_sun_java2d_loops_DrawGlyphListLCD_DrawGlyphListLCD 00000001800d5674     DrawGlyphList.obj
 0002:0002a684       $unwind$initLUT            00000001800d5684     DrawGlyphList.obj
 0002:0002a6a8       $unwind$initLCDGammaTables 00000001800d56a8     DrawGlyphList.obj
 0002:0002a6a8       $unwind$?get_value_or_null@?$Lookup@U?$IntType@I$03@OT@@@AAT@@QEBA?BIII@Z 00000001800d56a8     hb-aat-layout.obj
 0002:0002a6a8       $unwind$?match_properties_mark@hb_ot_apply_context_t@OT@@QEBA_NIII@Z 00000001800d56a8     hb-aat-layout.obj
 0002:0002a6a8       $unwind$hb_aat_layout_has_positioning 00000001800d56a8     hb-aat-layout.obj
 0002:0002a6a8       $unwind$hb_aat_layout_has_tracking 00000001800d56a8     hb-aat-layout.obj
 0002:0002a6a8       $unwind$hb_tag_from_string 00000001800d56a8     hb-common.obj
 0002:0002a6a8       $unwind$?hb_draw_extents_get_funcs@@YAPEAUhb_draw_funcs_t@@XZ 00000001800d56a8     hb-draw.obj
 0002:0002a6a8       $unwind$hb_draw_funcs_create 00000001800d56a8     hb-draw.obj
 0002:0002a6a8       $unwind$??$get_glyph_from_ascii@UCmapSubtable@OT@@@accelerator_t@cmap@OT@@KA_NPEBXIPEAI@Z 00000001800d56a8     hb-face.obj
 0002:0002a6a8       $unwind$hb_face_reference_table 00000001800d56a8     hb-face.obj
 0002:0002a6a8       $unwind$?has_func@hb_font_t@@QEAA_NI@Z 00000001800d56a8     hb-font.obj
 0002:0002a6a8       $unwind$?glyph_to_sid@?$accelerator_templ_t@Ucff1_private_dict_opset_t@CFF@@U?$cff1_private_dict_values_base_t@Udict_val_t@CFF@@@2@@cff1@OT@@QEBAIIPEAUcode_pair_t@CFF@@@Z 00000001800d56a8     hb-ot-font.obj
 0002:0002a6a8       $unwind$??$cache_func_to@U?$LigatureSubstFormat1_2@USmallTypes@Layout@OT@@@GSUB_impl@Layout@OT@@@hb_accelerate_subtables_context_t@OT@@SAPEAXPEAXW4hb_ot_lookup_cache_op_t@1@@Z 00000001800d56a8     hb-ot-layout.obj
 0002:0002a6a8       $unwind$??$cache_func_to@U?$PairPosFormat1_3@USmallTypes@Layout@OT@@@GPOS_impl@Layout@OT@@@hb_accelerate_subtables_context_t@OT@@SAPEAXPEAXW4hb_ot_lookup_cache_op_t@1@@Z 00000001800d56a8     hb-ot-layout.obj
 0002:0002a6a8       $unwind$??$cache_func_to@U?$PairPosFormat2_4@USmallTypes@Layout@OT@@@GPOS_impl@Layout@OT@@@hb_accelerate_subtables_context_t@OT@@SAPEAXPEAXW4hb_ot_lookup_cache_op_t@1@@Z 00000001800d56a8     hb-ot-layout.obj
 0002:0002a6a8       $unwind$??$dispatch@Uhb_would_apply_context_t@OT@@$$V@SubstLookupSubTable@GSUB_impl@Layout@OT@@QEBA_NPEAUhb_would_apply_context_t@3@I@Z 00000001800d56a8     hb-ot-layout.obj
 0002:0002a6a8       $unwind$?get_gsubgpos_table@@YAAEBUGSUBGPOS@OT@@PEAUhb_face_t@@I@Z 00000001800d56a8     hb-ot-layout.obj
 0002:0002a6a8       $unwind$?hb_ot_layout_has_cross_kerning@@YA_NPEAUhb_face_t@@@Z 00000001800d56a8     hb-ot-layout.obj
 0002:0002a6a8       $unwind$?hb_ot_layout_has_kerning@@YA_NPEAUhb_face_t@@@Z 00000001800d56a8     hb-ot-layout.obj
 0002:0002a6a8       $unwind$?hb_ot_layout_has_machine_kerning@@YA_NPEAUhb_face_t@@@Z 00000001800d56a8     hb-ot-layout.obj
 0002:0002a6a8       $unwind$?match_coverage@OT@@YA_NAEAUhb_glyph_info_t@@IPEBX@Z 00000001800d56a8     hb-ot-layout.obj
 0002:0002a6a8       $unwind$hb_ot_layout_has_glyph_classes 00000001800d56a8     hb-ot-layout.obj
 0002:0002a6a8       $unwind$hb_ot_layout_has_positioning 00000001800d56a8     hb-ot-layout.obj
 0002:0002a6a8       $unwind$hb_ot_layout_has_substitution 00000001800d56a8     hb-ot-layout.obj
 0002:0002a6a8       $unwind$hb_ot_layout_table_get_lookup_count 00000001800d56a8     hb-ot-layout.obj
 0002:0002a6a8       $unwind$?hb_outline_recording_pen_get_funcs@@YAPEAUhb_draw_funcs_t@@XZ 00000001800d56a8     hb-outline.obj
 0002:0002a6a8       $unwind$?hb_paint_bounded_get_funcs@@YAPEAUhb_paint_funcs_t@@XZ 00000001800d56a8     hb-paint-bounded.obj
 0002:0002a6a8       $unwind$?hb_paint_extents_get_funcs@@YAPEAUhb_paint_funcs_t@@XZ 00000001800d56a8     hb-paint-extents.obj
 0002:0002a6a8       $unwind$hb_paint_funcs_create 00000001800d56a8     hb-paint.obj
 0002:0002a6a8       $unwind$hb_ucd_get_unicode_funcs 00000001800d56a8     hb-ucd.obj
 0002:0002a6a8       $unwind$Java_sun_font_NullFontScaler_getNullScalerContext 00000001800d56a8     sunFont.obj
 0002:0002a6a8       $unwind$__scrt_initialize_default_local_stdio_options 00000001800d56a8     MSVCRT:default_local_stdio_options.obj
 0002:0002a6a8       $unwind$?dllmain_crt_dispatch@@YAHQEAUHINSTANCE__@@KQEAX@Z 00000001800d56a8     MSVCRT:dll_dllmain.obj
 0002:0002a6a8       $unwind$DllMain            00000001800d56a8     MSVCRT:dll_dllmain_stub.obj
 0002:0002a6a8       $unwind$__report_rangecheckfailure 00000001800d56a8     MSVCRT:gs_report.obj
 0002:0002a6a8       $unwind$__GSHandlerCheck   00000001800d56a8     MSVCRT:gshandler.obj
 0002:0002a6a8       $unwind$__scrt_acquire_startup_lock 00000001800d56a8     MSVCRT:utility.obj
 0002:0002a6a8       $unwind$__scrt_dllmain_after_initialize_c 00000001800d56a8     MSVCRT:utility.obj
 0002:0002a6a8       $unwind$__scrt_dllmain_before_initialize_c 00000001800d56a8     MSVCRT:utility.obj
 0002:0002a6a8       $unwind$__scrt_dllmain_crt_thread_attach 00000001800d56a8     MSVCRT:utility.obj
 0002:0002a6a8       $unwind$__scrt_dllmain_crt_thread_detach 00000001800d56a8     MSVCRT:utility.obj
 0002:0002a6a8       $unwind$__scrt_dllmain_uninitialize_c 00000001800d56a8     MSVCRT:utility.obj
 0002:0002a6a8       $unwind$__scrt_dllmain_uninitialize_critical 00000001800d56a8     MSVCRT:utility.obj
 0002:0002a6b0       $unwind$storeGVData        00000001800d56b0     HBShaper.obj
 0002:0002a6e0       $unwind$euclidianDistance  00000001800d56e0     HBShaper.obj
 0002:0002a6ec       $unwind$Java_sun_font_SunLayoutEngine_shape 00000001800d56ec     HBShaper.obj
 0002:0002a700       $chain$0$Java_sun_font_SunLayoutEngine_shape 00000001800d5700     HBShaper.obj
 0002:0002a714       $chain$1$Java_sun_font_SunLayoutEngine_shape 00000001800d5714     HBShaper.obj
 0002:0002a714       $chain$5$Java_sun_font_SunLayoutEngine_shape 00000001800d5714     HBShaper.obj
 0002:0002a724       $chain$2$Java_sun_font_SunLayoutEngine_shape 00000001800d5724     HBShaper.obj
 0002:0002a738       $chain$3$Java_sun_font_SunLayoutEngine_shape 00000001800d5738     HBShaper.obj
 0002:0002a74c       $chain$4$Java_sun_font_SunLayoutEngine_shape 00000001800d574c     HBShaper.obj
 0002:0002a75c       $unwind$jdk_hb_shape       00000001800d575c     HBShaper_Panama.obj
 0002:0002a780       $unwind$Java_sun_awt_Win32FontManager_populateFontFileNameMap0 00000001800d5780     fontpath.obj
 0002:0002a79c       $chain$0$Java_sun_awt_Win32FontManager_populateFontFileNameMap0 00000001800d579c     fontpath.obj
 0002:0002a7b0       $chain$1$Java_sun_awt_Win32FontManager_populateFontFileNameMap0 00000001800d57b0     fontpath.obj
 0002:0002a7c0       $unwind$Java_sun_awt_Win32FontManager_getFontPath 00000001800d57c0     fontpath.obj
 0002:0002a7e4       $unwind$EnumFontFacesInFamilyProcW 00000001800d57e4     fontpath.obj
 0002:0002a804       $unwind$EnumFamilyNamesW   00000001800d5804     fontpath.obj
 0002:0002a824       $unwind$registerFontW      00000001800d5824     fontpath.obj
 0002:0002a840       $unwind$populateFontFileNameFromRegistryKey 00000001800d5840     fontpath.obj
 0002:0002a84c       $chain$0$populateFontFileNameFromRegistryKey 00000001800d584c     fontpath.obj
 0002:0002a860       $chain$5$populateFontFileNameFromRegistryKey 00000001800d5860     fontpath.obj
 0002:0002a880       $chain$7$populateFontFileNameFromRegistryKey 00000001800d5880     fontpath.obj
 0002:0002a898       $chain$8$populateFontFileNameFromRegistryKey 00000001800d5898     fontpath.obj
 0002:0002a8a8       $chain$9$populateFontFileNameFromRegistryKey 00000001800d58a8     fontpath.obj
 0002:0002a8b8       $unwind$Java_sun_font_FreetypeFontScaler_initIDs 00000001800d58b8     freetypeScaler.obj
 0002:0002a8b8       $unwind$?hb_font_get_glyph_h_kerning_default@@YAHPEAUhb_font_t@@PEAXII1@Z 00000001800d58b8     hb-font.obj
 0002:0002a8b8       $unwind$?hb_font_get_glyph_v_kerning_default@@YAHPEAUhb_font_t@@PEAXII1@Z 00000001800d58b8     hb-font.obj
 0002:0002a8b8       $unwind$hb_font_get_glyph  00000001800d58b8     hb-font.obj
 0002:0002a8b8       $unwind$?process_op@?$cs_opset_t@Unumber_t@CFF@@Ucff2_cs_opset_path_t@@U?$cff2_cs_interp_env_t@Unumber_t@CFF@@@2@Ucff2_path_param_t@@Ucff2_path_procs_path_t@@@CFF@@SAXIAEAU?$cff2_cs_interp_env_t@Unumber_t@CFF@@@2@AEAUcff2_path_param_t@@@Z 00000001800d58b8     hb-ot-cff2-table.obj
 0002:0002a8b8       $unwind$?hb_paint_extents_paint_image@@YAHPEAUhb_paint_funcs_t@@PEAXPEAUhb_blob_t@@IIIMPEAUhb_glyph_extents_t@@1@Z 00000001800d58b8     hb-paint-extents.obj
 0002:0002a8b8       $unwind$hb_shape_plan_execute 00000001800d58b8     hb-shape-plan.obj
 0002:0002a8c0       $unwind$Java_sun_font_FreetypeFontScaler_initNativeScaler 00000001800d58c0     freetypeScaler.obj
 0002:0002a8d8       $chain$2$Java_sun_font_FreetypeFontScaler_initNativeScaler 00000001800d58d8     freetypeScaler.obj
 0002:0002a8ec       $chain$3$Java_sun_font_FreetypeFontScaler_initNativeScaler 00000001800d58ec     freetypeScaler.obj
 0002:0002a8fc       $unwind$Java_sun_font_FreetypeFontScaler_getFontMetricsNative 00000001800d58fc     freetypeScaler.obj
 0002:0002a918       $chain$9$Java_sun_font_FreetypeFontScaler_getFontMetricsNative 00000001800d5918     freetypeScaler.obj
 0002:0002a950       $chain$10$Java_sun_font_FreetypeFontScaler_getFontMetricsNative 00000001800d5950     freetypeScaler.obj
 0002:0002a960       $unwind$Java_sun_font_FreetypeFontScaler_getGlyphAdvanceNative 00000001800d5960     freetypeScaler.obj
 0002:0002a960       $unwind$?start_processing@hb_sanitize_context_t@@QEAAXXZ 00000001800d5960     hb-aat-layout.obj
 0002:0002a960       $unwind$?hhcurveto@?$path_procs_t@Ucff2_path_procs_extents_t@@U?$cff2_cs_interp_env_t@Unumber_t@CFF@@@CFF@@Ucff2_extents_param_t@@@CFF@@SAXAEAU?$cff2_cs_interp_env_t@Unumber_t@CFF@@@2@AEAUcff2_extents_param_t@@@Z 00000001800d5960     hb-ot-cff2-table.obj
 0002:0002a960       $unwind$?vvcurveto@?$path_procs_t@Ucff2_path_procs_extents_t@@U?$cff2_cs_interp_env_t@Unumber_t@CFF@@@CFF@@Ucff2_extents_param_t@@@CFF@@SAXAEAU?$cff2_cs_interp_env_t@Unumber_t@CFF@@@2@AEAUcff2_extents_param_t@@@Z 00000001800d5960     hb-ot-cff2-table.obj
 0002:0002a960       $unwind$_hb_ot_shape       00000001800d5960     hb-ot-shape.obj
 0002:0002a960       $unwind$?pop_group@hb_paint_extents_context_t@@QEAAXW4hb_paint_composite_mode_t@@@Z 00000001800d5960     hb-paint-extents.obj
 0002:0002a960       $unwind$hb_paint_push_transform 00000001800d5960     hb-paint.obj
 0002:0002a968       $chain$0$Java_sun_font_FreetypeFontScaler_getGlyphAdvanceNative 00000001800d5968     freetypeScaler.obj
 0002:0002a97c       $chain$1$Java_sun_font_FreetypeFontScaler_getGlyphAdvanceNative 00000001800d597c     freetypeScaler.obj
 0002:0002a98c       $unwind$Java_sun_font_FreetypeFontScaler_getGlyphMetricsNative 00000001800d598c     freetypeScaler.obj
 0002:0002a998       $unwind$Java_sun_font_FreetypeFontScaler_getGlyphImageNative 00000001800d5998     freetypeScaler.obj
 0002:0002a998       $unwind$?rcurveline@?$path_procs_t@Ucff1_path_procs_extents_t@@Ucff1_cs_interp_env_t@CFF@@Ucff1_extents_param_t@@@CFF@@SAXAEAUcff1_cs_interp_env_t@2@AEAUcff1_extents_param_t@@@Z 00000001800d5998     hb-ot-cff1-table.obj
 0002:0002a998       $unwind$?rlinecurve@?$path_procs_t@Ucff1_path_procs_extents_t@@Ucff1_cs_interp_env_t@CFF@@Ucff1_extents_param_t@@@CFF@@SAXAEAUcff1_cs_interp_env_t@2@AEAUcff1_extents_param_t@@@Z 00000001800d5998     hb-ot-cff1-table.obj
 0002:0002a998       $unwind$?rrcurveto@?$path_procs_t@Ucff1_path_procs_extents_t@@Ucff1_cs_interp_env_t@CFF@@Ucff1_extents_param_t@@@CFF@@SAXAEAUcff1_cs_interp_env_t@2@AEAUcff1_extents_param_t@@@Z 00000001800d5998     hb-ot-cff1-table.obj
 0002:0002a998       $unwind$?end@?$hb_iter_t@U?$hb_map_iter_t@U?$hb_zip_iter_t@U?$hb_sorted_array_t@UHBGlyphID16@OT@@@@U?$hb_array_t@UHBGlyphID16@OT@@@@@@AEBU<unnamed-type-hb_first>@@$00$0A@@@AEAUHBGlyphID16@OT@@@@QEBA?AU?$hb_map_iter_t@U?$hb_zip_iter_t@U?$hb_sorted_array_t@UHBGlyphID16@OT@@@@U?$hb_array_t@UHBGlyphID16@OT@@@@@@AEBU<unnamed-type-hb_first>@@$00$0A@@@XZ 00000001800d5998     hb-ot-shaper-arabic.obj
 0002:0002a9a0       $unwind$Java_sun_font_FreetypeFontScaler_getGlyphOutlineBoundsNative 00000001800d59a0     freetypeScaler.obj
 0002:0002a9a0       $unwind$?parse_bcd@dict_opset_t@CFF@@SANAEAUbyte_str_ref_t@2@@Z 00000001800d59a0     hb-ot-font.obj
 0002:0002a9b0       $unwind$Java_sun_font_FreetypeFontScaler_getGlyphOutlineNative 00000001800d59b0     freetypeScaler.obj
 0002:0002a9b8       $unwind$Java_sun_font_FreetypeFontScaler_getGlyphVectorOutlineNative 00000001800d59b8     freetypeScaler.obj
 0002:0002a9d0       $chain$1$Java_sun_font_FreetypeFontScaler_getGlyphVectorOutlineNative 00000001800d59d0     freetypeScaler.obj
 0002:0002a9e4       $chain$4$Java_sun_font_FreetypeFontScaler_getGlyphVectorOutlineNative 00000001800d59e4     freetypeScaler.obj
 0002:0002aa00       $chain$5$Java_sun_font_FreetypeFontScaler_getGlyphVectorOutlineNative 00000001800d5a00     freetypeScaler.obj
 0002:0002aa10       $chain$6$Java_sun_font_FreetypeFontScaler_getGlyphVectorOutlineNative 00000001800d5a10     freetypeScaler.obj
 0002:0002aa20       $unwind$Java_sun_font_FreetypeFontScaler_getGlyphPointNative 00000001800d5a20     freetypeScaler.obj
 0002:0002aa30       $unwind$Java_sun_font_FreetypeFontScaler_disposeNativeScaler 00000001800d5a30     freetypeScaler.obj
 0002:0002aa30       $unwind$?get@hb_bit_set_t@@QEBA_NI@Z 00000001800d5a30     hb-aat-layout.obj
 0002:0002aa30       $unwind$?move_to@hb_buffer_t@@QEAA_NI@Z 00000001800d5a30     hb-buffer.obj
 0002:0002aa30       $unwind$?clear@advance_cache_t@hb_ot_font_t@@QEBAXXZ 00000001800d5a30     hb-ot-font.obj
 0002:0002aa3c       $unwind$Java_sun_font_FreetypeFontScaler_getGlyphCodeNative 00000001800d5a3c     freetypeScaler.obj
 0002:0002aa48       $unwind$Java_sun_font_FreetypeFontScaler_getNumGlyphsNative 00000001800d5a48     freetypeScaler.obj
 0002:0002aa48       $unwind$invalidateJavaScaler 00000001800d5a48     freetypeScaler.obj
 0002:0002aa48       $unwind$??1accelerator_t@?$KerxTable@Ukerx@AAT@@@AAT@@QEAA@XZ 00000001800d5a48     hb-aat-layout.obj
 0002:0002aa48       $unwind$?fini@hb_bit_set_t@@QEAAXXZ 00000001800d5a48     hb-aat-layout.obj
 0002:0002aa48       $unwind$?next_glyph@hb_buffer_t@@QEAA_NXZ 00000001800d5a48     hb-aat-layout.obj
 0002:0002aa48       $unwind$?replace_glyph_inplace@hb_aat_apply_context_t@AAT@@QEAAXII@Z 00000001800d5a48     hb-aat-layout.obj
 0002:0002aa48       $unwind$?resize@?$hb_vector_t@Upage_map_t@hb_bit_set_t@@$00@@QEAA_NH_N0@Z 00000001800d5a48     hb-aat-layout.obj
 0002:0002aa48       $unwind$hb_aat_layout_has_substitution 00000001800d5a48     hb-aat-layout.obj
 0002:0002aa48       $unwind$?make_room_for@hb_buffer_t@@QEAA_NII@Z 00000001800d5a48     hb-buffer.obj
 0002:0002aa48       $unwind$??1hb_glyf_scratch_t@@QEAA@XZ 00000001800d5a48     hb-common.obj
 0002:0002aa48       $unwind$?_glyf_get_advance_with_var_unscaled@@YAIPEAUhb_font_t@@I_N@Z 00000001800d5a48     hb-common.obj
 0002:0002aa48       $unwind$?resize@?$hb_vector_t@Ucontour_point_t@@$0A@@@QEAA_NH_N0@Z 00000001800d5a48     hb-common.obj
 0002:0002aa48       $unwind$?sanitize@VVAR@OT@@QEBA_NPEAUhb_sanitize_context_t@@@Z 00000001800d5a48     hb-common.obj
 0002:0002aa48       $unwind$?alloc@?$hb_pool_t@Uobject_t@hb_serialize_context_t@@$0CA@@@QEAAPEAUobject_t@hb_serialize_context_t@@XZ 00000001800d5a48     hb-face-builder.obj
 0002:0002aa48       $unwind$?fini@object_t@hb_serialize_context_t@@QEAAXXZ 00000001800d5a48     hb-face-builder.obj
 0002:0002aa48       $unwind$??$get_glyph_from_macroman@UCmapSubtable@OT@@@accelerator_t@cmap@OT@@KA_NPEBXIPEAI@Z 00000001800d5a48     hb-face.obj
 0002:0002aa48       $unwind$??$get_glyph_from_symbol@UCmapSubtable@OT@@$1?_hb_arabic_pua_simp_map@@YAII@Z@accelerator_t@cmap@OT@@KA_NPEBXIPEAI@Z 00000001800d5a48     hb-face.obj
 0002:0002aa48       $unwind$??$get_glyph_from_symbol@UCmapSubtable@OT@@$1?_hb_arabic_pua_trad_map@@YAII@Z@accelerator_t@cmap@OT@@KA_NPEBXIPEAI@Z 00000001800d5a48     hb-face.obj
 0002:0002aa48       $unwind$??$get_glyph_from_symbol@UCmapSubtable@OT@@$1?_hb_symbol_pua_map@2@YAII@Z@accelerator_t@cmap@OT@@KA_NPEBXIPEAI@Z 00000001800d5a48     hb-face.obj
 0002:0002aa48       $unwind$?hb_font_get_font_h_extents_default@@YAHPEAUhb_font_t@@PEAXPEAUhb_font_extents_t@@1@Z 00000001800d5a48     hb-font.obj
 0002:0002aa48       $unwind$?hb_font_get_font_v_extents_default@@YAHPEAUhb_font_t@@PEAXPEAUhb_font_extents_t@@1@Z 00000001800d5a48     hb-font.obj
 0002:0002aa48       $unwind$hb_jdk_font_create 00000001800d5a48     hb-jdk-font.obj
 0002:0002aa48       $unwind$?process_op@?$cs_opset_t@Unumber_t@CFF@@Ucff1_cs_opset_extents_t@@Ucff1_cs_interp_env_t@2@Ucff1_extents_param_t@@Ucff1_path_procs_extents_t@@@CFF@@SAXIAEAUcff1_cs_interp_env_t@2@AEAUcff1_extents_param_t@@@Z 00000001800d5a48     hb-ot-cff1-table.obj
 0002:0002aa48       $unwind$??1hb_paint_extents_context_t@@QEAA@XZ 00000001800d5a48     hb-ot-color.obj
 0002:0002aa48       $unwind$?hb_ot_get_glyph_from_name@@YAHPEAUhb_font_t@@PEAXPEBDHPEAI1@Z 00000001800d5a48     hb-ot-font.obj
 0002:0002aa48       $unwind$?paint_glyph@PaintRotate@OT@@QEBAXPEAUhb_paint_context_t@2@I@Z 00000001800d5a48     hb-ot-font.obj
 0002:0002aa48       $unwind$?push@?$hb_vector_t@Ucff1_font_dict_values_t@CFF@@$0A@@@QEAAPEAUcff1_font_dict_values_t@CFF@@XZ 00000001800d5a48     hb-ot-font.obj
 0002:0002aa48       $unwind$?push@?$hb_vector_t@Ucff2_font_dict_values_t@CFF@@$0A@@@QEAAPEAUcff2_font_dict_values_t@CFF@@XZ 00000001800d5a48     hb-ot-font.obj
 0002:0002aa48       $unwind$??$dispatch@Uhb_accelerate_subtables_context_t@OT@@$$V@PosLookupSubTable@GPOS_impl@Layout@OT@@QEBA?AUhb_empty_t@@PEAUhb_accelerate_subtables_context_t@3@I@Z 00000001800d5a48     hb-ot-layout.obj
 0002:0002aa48       $unwind$??1accelerator_t@kern@OT@@QEAA@XZ 00000001800d5a48     hb-ot-layout.obj
 0002:0002aa48       $unwind$?get_class@ClassDef@OT@@QEBAIIPEAU?$hb_cache_t@$0P@$07$06$00@@@Z 00000001800d5a48     hb-ot-layout.obj
 0002:0002aa48       $unwind$??$extend@ULookup@OT@@$$V@hb_serialize_context_t@@QEAAPEAULookup@OT@@PEAU12@@Z 00000001800d5a48     hb-ot-shaper-arabic.obj
 0002:0002aa48       $unwind$??$extend_size@U?$ArrayOf@UHBGlyphID16@OT@@U?$IntType@G$01@2@@OT@@@hb_serialize_context_t@@QEAAPEAU?$ArrayOf@UHBGlyphID16@OT@@U?$IntType@G$01@2@@OT@@PEAU12@_K_N@Z 00000001800d5a48     hb-ot-shaper-arabic.obj
 0002:0002aa48       $unwind$??$extend_size@U?$HeadlessArrayOf@UHBGlyphID16@OT@@U?$IntType@G$01@2@@OT@@@hb_serialize_context_t@@QEAAPEAU?$HeadlessArrayOf@UHBGlyphID16@OT@@U?$IntType@G$01@2@@OT@@PEAU12@_K_N@Z 00000001800d5a48     hb-ot-shaper-arabic.obj
 0002:0002aa48       $unwind$?setup_masks_arabic@@YAXPEBUhb_ot_shape_plan_t@@PEAUhb_buffer_t@@PEAUhb_font_t@@@Z 00000001800d5a48     hb-ot-shaper-arabic.obj
 0002:0002aa48       $unwind$?setup_masks_arabic_plan@@YAXPEBUarabic_shape_plan_t@@PEAUhb_buffer_t@@W4hb_script_t@@@Z 00000001800d5a48     hb-ot-shaper-arabic.obj
 0002:0002aa48       $unwind$?collect_features_hangul@@YAXPEAUhb_ot_shape_planner_t@@@Z 00000001800d5a48     hb-ot-shaper-hangul.obj
 0002:0002aa48       $unwind$?collect_features_indic@@YAXPEAUhb_ot_shape_planner_t@@@Z 00000001800d5a48     hb-ot-shaper-indic.obj
 0002:0002aa48       $unwind$?init@hb_indic_would_substitute_feature_t@@QEAAXPEBUhb_ot_map_t@@I_N@Z 00000001800d5a48     hb-ot-shaper-indic.obj
 0002:0002aa48       $unwind$?collect_features_khmer@@YAXPEAUhb_ot_shape_planner_t@@@Z 00000001800d5a48     hb-ot-shaper-khmer.obj
 0002:0002aa48       $unwind$?collect_features_use@@YAXPEAUhb_ot_shape_planner_t@@@Z 00000001800d5a48     hb-ot-shaper-use.obj
 0002:0002aa48       $unwind$?subtag_matches@@YA_NPEBD00I@Z 00000001800d5a48     hb-ot-tag.obj
 0002:0002aa48       $unwind$hb_unicode_funcs_create 00000001800d5a48     hb-unicode.obj
 0002:0002aa48       $unwind$_DllMainCRTStartup 00000001800d5a48     MSVCRT:dll_dllmain.obj
 0002:0002aa58       $unwind$Java_sun_font_FreetypeFontScaler_createScalerContextNative 00000001800d5a58     freetypeScaler.obj
 0002:0002aa70       $unwind$ReadTTFontFileFunc 00000001800d5a70     freetypeScaler.obj
 0002:0002aa70       $unwind$?end_path@cff1_path_param_t@@QEAAXXZ 00000001800d5a70     hb-ot-cff1-table.obj
 0002:0002aa70       $unwind$??$dispatch@Uhb_paint_context_t@OT@@$$V@Paint@OT@@QEBA?AUhb_empty_t@@PEAUhb_paint_context_t@1@@Z 00000001800d5a70     hb-ot-font.obj
 0002:0002aa70       $unwind$?apply@?$ContextFormat1_4@USmallTypes@Layout@OT@@@OT@@QEBA_NPEAUhb_ot_apply_context_t@2@@Z 00000001800d5a70     hb-ot-layout.obj
 0002:0002aa70       $unwind$?serialize@Lookup@OT@@QEAA_NPEAUhb_serialize_context_t@@III@Z 00000001800d5a70     hb-ot-shaper-arabic.obj
 0002:0002aa88       $unwind$GlyphSlot_Embolden 00000001800d5a88     freetypeScaler.obj
 0002:0002aa94       $chain$0$GlyphSlot_Embolden 00000001800d5a94     freetypeScaler.obj
 0002:0002aaa8       $chain$1$GlyphSlot_Embolden 00000001800d5aa8     freetypeScaler.obj
 0002:0002aab8       $unwind$setupFTContext     00000001800d5ab8     freetypeScaler.obj
 0002:0002aacc       $unwind$getGlyphImageNativeInternal 00000001800d5acc     freetypeScaler.obj
 0002:0002aae8       $chain$0$getGlyphImageNativeInternal 00000001800d5ae8     freetypeScaler.obj
 0002:0002aafc       $chain$1$getGlyphImageNativeInternal 00000001800d5afc     freetypeScaler.obj
 0002:0002ab0c       $unwind$CopyBW2Grey8       00000001800d5b0c     freetypeScaler.obj
 0002:0002ab1c       $chain$1$CopyBW2Grey8      00000001800d5b1c     freetypeScaler.obj
 0002:0002ab34       $chain$2$CopyBW2Grey8      00000001800d5b34     freetypeScaler.obj
 0002:0002ab44       $unwind$getFTOutline       00000001800d5b44     freetypeScaler.obj
 0002:0002ab58       $unwind$getGlyphGeneralPath 00000001800d5b58     freetypeScaler.obj
 0002:0002ab6c       $chain$0$getGlyphGeneralPath 00000001800d5b6c     freetypeScaler.obj
 0002:0002ab80       $chain$1$getGlyphGeneralPath 00000001800d5b80     freetypeScaler.obj
 0002:0002ab90       $unwind$?reverse_range@hb_buffer_t@@QEAAXII@Z 00000001800d5b90     hb-aat-layout.obj
 0002:0002ab90       $unwind$?find_lang_sys_index@Script@OT@@QEBA_NIPEAI@Z 00000001800d5b90     hb-ot-layout.obj
 0002:0002ab90       $unwind$?find_script_index@GSUBGPOS@OT@@QEBA_NIPEAI@Z 00000001800d5b90     hb-ot-layout.obj
 0002:0002ab90       $unwind$?get_kerning@?$KerxSubTableFormat0@UKernAATSubTableHeader@OT@@@AAT@@QEBAHIIPEAUhb_aat_apply_context_t@2@@Z 00000001800d5b90     hb-ot-layout.obj
 0002:0002ab90       $unwind$?get_kerning@?$KerxSubTableFormat0@UKernOTSubTableHeader@OT@@@AAT@@QEBAHIIPEAUhb_aat_apply_context_t@2@@Z 00000001800d5b90     hb-ot-layout.obj
 0002:0002ab90       $unwind$?record_pref_use@@YA_NPEBUhb_ot_shape_plan_t@@PEAUhb_font_t@@PEAUhb_buffer_t@@@Z 00000001800d5b90     hb-ot-shaper-use.obj
 0002:0002aba0       $unwind$??$dispatch@Uhb_accelerate_subtables_context_t@AAT@@$$V@?$ChainSubtable@UExtendedTypes@AAT@@@AAT@@QEBA?AUhb_empty_t@@PEAUhb_accelerate_subtables_context_t@1@@Z 00000001800d5ba0     hb-aat-layout.obj
 0002:0002aba0       $unwind$??$dispatch@Uhb_accelerate_subtables_context_t@AAT@@$$V@?$ChainSubtable@UObsoleteTypes@AAT@@@AAT@@QEBA?AUhb_empty_t@@PEAUhb_accelerate_subtables_context_t@1@@Z 00000001800d5ba0     hb-aat-layout.obj
 0002:0002aba0       $unwind$?get_anchor@ankr@AAT@@QEBAAEBUAnchor@2@III@Z 00000001800d5ba0     hb-aat-layout.obj
 0002:0002aba0       $unwind$?replace_glyph@hb_buffer_t@@QEAA_NI@Z 00000001800d5ba0     hb-aat-layout.obj
 0002:0002aba0       $unwind$hb_blob_get_data_writable 00000001800d5ba0     hb-blob.obj
 0002:0002aba0       $unwind$?delete_glyph@hb_buffer_t@@QEAAXXZ 00000001800d5ba0     hb-buffer.obj
 0002:0002aba0       $unwind$hb_buffer_create_similar 00000001800d5ba0     hb-buffer.obj
 0002:0002aba0       $unwind$hb_buffer_set_length 00000001800d5ba0     hb-buffer.obj
 0002:0002aba0       $unwind$??$get_glyph_from@UCmapSubtableFormat12@OT@@@accelerator_t@cmap@OT@@KA_NPEBXIPEAI@Z 00000001800d5ba0     hb-face.obj
 0002:0002aba0       $unwind$?_hb_font_create@@YAPEAUhb_font_t@@PEAUhb_face_t@@@Z 00000001800d5ba0     hb-font.obj
 0002:0002aba0       $unwind$?get_h_extents_with_fallback@hb_font_t@@QEAAXPEAUhb_font_extents_t@@@Z 00000001800d5ba0     hb-font.obj
 0002:0002aba0       $unwind$hb_font_get_glyph_h_advance 00000001800d5ba0     hb-font.obj
 0002:0002aba0       $unwind$?hb_jdk_get_nominal_glyph@@YAHPEAUhb_font_t@@PEAXIPEAI1@Z 00000001800d5ba0     hb-jdk-font.obj
 0002:0002aba0       $unwind$??1kern_accelerator_data_t@AAT@@QEAA@XZ 00000001800d5ba0     hb-ot-face.obj
 0002:0002aba0       $unwind$?cmp@gname_t@accelerator_t@cff1@OT@@SAHPEBX0@Z 00000001800d5ba0     hb-ot-font.obj
 0002:0002aba0       $unwind$?hb_ot_get_font_h_extents@@YAHPEAUhb_font_t@@PEAXPEAUhb_font_extents_t@@1@Z 00000001800d5ba0     hb-ot-font.obj
 0002:0002aba0       $unwind$?hb_ot_get_font_v_extents@@YAHPEAUhb_font_t@@PEAXPEAUhb_font_extents_t@@1@Z 00000001800d5ba0     hb-ot-font.obj
 0002:0002aba0       $unwind$?hb_ot_get_nominal_glyph@@YAHPEAUhb_font_t@@PEAXIPEAI1@Z 00000001800d5ba0     hb-ot-font.obj
 0002:0002aba0       $unwind$?interpret@?$dict_interpreter_t@Ucff1_top_dict_opset_t@CFF@@Ucff1_top_dict_values_t@2@Ucff1_top_dict_interp_env_t@2@@CFF@@QEAA_NAEAUcff1_top_dict_values_t@2@@Z 00000001800d5ba0     hb-ot-font.obj
 0002:0002aba0       $unwind$?interpret@?$dict_interpreter_t@Ucff2_top_dict_opset_t@CFF@@Ucff2_top_dict_values_t@2@U?$interp_env_t@Unumber_t@CFF@@@2@@CFF@@QEAA_NAEAUcff2_top_dict_values_t@2@@Z 00000001800d5ba0     hb-ot-font.obj
 0002:0002aba0       $unwind$?match_class_cached1@OT@@YA_NAEAUhb_glyph_info_t@@IPEBX@Z 00000001800d5ba0     hb-ot-layout.obj
 0002:0002aba0       $unwind$?match_class_cached2@OT@@YA_NAEAUhb_glyph_info_t@@IPEBX@Z 00000001800d5ba0     hb-ot-layout.obj
 0002:0002aba0       $unwind$?match_class_cached@OT@@YA_NAEAUhb_glyph_info_t@@IPEBX@Z 00000001800d5ba0     hb-ot-layout.obj
 0002:0002aba0       $unwind$hb_ot_layout_feature_with_variations_get_lookups 00000001800d5ba0     hb-ot-layout.obj
 0002:0002aba0       $unwind$?output_char@@YAXPEAUhb_buffer_t@@II@Z 00000001800d5ba0     hb-ot-shape-normalize.obj
 0002:0002aba0       $unwind$?pop_discard@hb_serialize_context_t@@QEAAXXZ 00000001800d5ba0     hb-ot-shaper-arabic.obj
 0002:0002aba0       $unwind$?data_create_use@@YAPEAXPEBUhb_ot_shape_plan_t@@@Z 00000001800d5ba0     hb-ot-shaper-use.obj
 0002:0002aba0       $unwind$?hb_outline_recording_pen_close_path@@YAXPEAUhb_draw_funcs_t@@PEAXPEAUhb_draw_state_t@@1@Z 00000001800d5ba0     hb-outline.obj
 0002:0002aba0       $unwind$?hb_paint_bounded_push_group@@YAXPEAUhb_paint_funcs_t@@PEAX1@Z 00000001800d5ba0     hb-paint-bounded.obj
 0002:0002aba0       $unwind$_RTC_Initialize    00000001800d5ba0     MSVCRT:initsect.obj
 0002:0002aba0       $unwind$_RTC_Terminate     00000001800d5ba0     MSVCRT:initsect.obj
 0002:0002abac       $unwind$?copy_glyph@hb_buffer_t@@QEAA_NXZ 00000001800d5bac     hb-aat-layout.obj
 0002:0002abac       $unwind$?hb_font_get_glyph_extents_default@@YAHPEAUhb_font_t@@PEAXIPEAUhb_glyph_extents_t@@1@Z 00000001800d5bac     hb-font.obj
 0002:0002abac       $unwind$?hb_jdk_get_glyph_contour_point@@YAHPEAUhb_font_t@@PEAXIIPEAH21@Z 00000001800d5bac     hb-jdk-font.obj
 0002:0002abac       $unwind$?hb_jdk_get_glyph_v_advance@@YAHPEAUhb_font_t@@PEAXI1@Z 00000001800d5bac     hb-jdk-font.obj
 0002:0002abac       $unwind$?hb_jdk_get_variation_glyph@@YAHPEAUhb_font_t@@PEAXIIPEAI1@Z 00000001800d5bac     hb-jdk-font.obj
 0002:0002abac       $unwind$?get_x_delta@Device@OT@@QEBAHPEAUhb_font_t@@AEBUItemVariationStore@2@PEAU?$hb_atomic_t@H@@@Z 00000001800d5bac     hb-ot-layout.obj
 0002:0002abac       $unwind$?get_y_delta@Device@OT@@QEBAHPEAUhb_font_t@@AEBUItemVariationStore@2@PEAU?$hb_atomic_t@H@@@Z 00000001800d5bac     hb-ot-layout.obj
 0002:0002abb8       $unwind$?unsafe_to_break@hb_buffer_t@@QEAAXII@Z 00000001800d5bb8     hb-aat-layout.obj
 0002:0002abc8       $unwind$?unsafe_to_break_from_outbuffer@hb_buffer_t@@QEAAXII@Z 00000001800d5bc8     hb-aat-layout.obj
 0002:0002abd8       $chain$0$?unsafe_to_break_from_outbuffer@hb_buffer_t@@QEAAXII@Z 00000001800d5bd8     hb-aat-layout.obj
 0002:0002abec       $chain$1$?unsafe_to_break_from_outbuffer@hb_buffer_t@@QEAAXII@Z 00000001800d5bec     hb-aat-layout.obj
 0002:0002abfc       $unwind$?message@hb_buffer_t@@QEAA_NPEAUhb_font_t@@PEBDZZ 00000001800d5bfc     hb-aat-layout.obj
 0002:0002abfc       $unwind$?CallIntMethod@JNIEnv_@@QEAAHPEAV_jobject@@PEAU_jmethodID@@ZZ 00000001800d5bfc     hb-jdk-font.obj
 0002:0002abfc       $unwind$?CallObjectMethod@JNIEnv_@@QEAAPEAV_jobject@@PEAV2@PEAU_jmethodID@@ZZ 00000001800d5bfc     hb-jdk-font.obj
 0002:0002ac04       $unwind$?_infos_set_glyph_flags@hb_buffer_t@@QEAAXPEAUhb_glyph_info_t@@IIII@Z 00000001800d5c04     hb-aat-layout.obj
 0002:0002ac04       $unwind$?merge_out_clusters@hb_buffer_t@@QEAAXII@Z 00000001800d5c04     hb-buffer.obj
 0002:0002ac04       $unwind$?get_glyph@Charset@CFF@@QEBAIII@Z 00000001800d5c04     hb-ot-cff1-table.obj
 0002:0002ac04       $unwind$?get_fd@CFF2FDSelect@CFF@@QEBAII@Z 00000001800d5c04     hb-ot-cff2-table.obj
 0002:0002ac04       $unwind$??4?$machine_index_t@U?$hb_zip_iter_t@U?$hb_iota_iter_t@II@@U?$hb_filter_iter_t@U?$hb_filter_iter_t@U?$hb_zip_iter_t@U?$hb_iota_iter_t@II@@U?$hb_array_t@Uhb_glyph_info_t@@@@@@V<lambda_e52748becc06432fe81365edeb8c4003>@@AEBU<unnamed-type-hb_second>@@$0A@@@V<lambda_a2885d5959499a7c5bcf896c0de144bb>@@AEBU<unnamed-type-hb_identity>@@$0A@@@@@@@QEAAXAEBU0@@Z 00000001800d5c04     hb-ot-shaper-use.obj
 0002:0002ac04       $unwind$?hb_ucd_compose@@YAHPEAUhb_unicode_funcs_t@@IIPEAIPEAX@Z 00000001800d5c04     hb-ucd.obj
 0002:0002ac04       $unwind$__GSHandlerCheckCommon 00000001800d5c04     MSVCRT:gshandler.obj
 0002:0002ac0c       $chain$0$?_infos_set_glyph_flags@hb_buffer_t@@QEAAXPEAUhb_glyph_info_t@@IIII@Z 00000001800d5c0c     hb-aat-layout.obj
 0002:0002ac20       $chain$2$?_infos_set_glyph_flags@hb_buffer_t@@QEAAXPEAUhb_glyph_info_t@@IIII@Z 00000001800d5c20     hb-aat-layout.obj
 0002:0002ac20       $chain$4$?_infos_set_glyph_flags@hb_buffer_t@@QEAAXPEAUhb_glyph_info_t@@IIII@Z 00000001800d5c20     hb-aat-layout.obj
 0002:0002ac34       $chain$5$?_infos_set_glyph_flags@hb_buffer_t@@QEAAXPEAUhb_glyph_info_t@@IIII@Z 00000001800d5c34     hb-aat-layout.obj
 0002:0002ac44       $unwind$?shrink_vector@?$hb_vector_t@U?$hb_vector_t@Urange_flags_t@hb_aat_map_t@@$00@@$0A@@@QEAAXI@Z 00000001800d5c44     hb-aat-layout.obj
 0002:0002ac44       $unwind$?shrink_vector@?$hb_vector_t@Ukern_subtable_accelerator_data_t@AAT@@$0A@@@QEAAXI@Z 00000001800d5c44     hb-aat-layout.obj
 0002:0002ac44       $unwind$?shrink_vector@?$hb_vector_t@U?$cff1_private_dict_values_base_t@Udict_val_t@CFF@@@CFF@@$0A@@@QEAAXI@Z 00000001800d5c44     hb-ot-face.obj
 0002:0002ac44       $unwind$?shrink_vector@?$hb_vector_t@U?$cff2_private_dict_values_base_t@Udict_val_t@CFF@@@CFF@@$0A@@@QEAAXI@Z 00000001800d5c44     hb-ot-face.obj
 0002:0002ac44       $unwind$?shrink_vector@?$hb_vector_t@Ucff1_font_dict_values_t@CFF@@$0A@@@QEAAXI@Z 00000001800d5c44     hb-ot-face.obj
 0002:0002ac44       $unwind$?shrink_vector@?$hb_vector_t@Ucff2_font_dict_values_t@CFF@@$0A@@@QEAAXI@Z 00000001800d5c44     hb-ot-face.obj
 0002:0002ac54       $chain$2$?shrink_vector@?$hb_vector_t@U?$hb_vector_t@Urange_flags_t@hb_aat_map_t@@$00@@$0A@@@QEAAXI@Z 00000001800d5c54     hb-aat-layout.obj
 0002:0002ac70       $chain$3$?shrink_vector@?$hb_vector_t@U?$hb_vector_t@Urange_flags_t@hb_aat_map_t@@$00@@$0A@@@QEAAXI@Z 00000001800d5c70     hb-aat-layout.obj
 0002:0002ac80       $unwind$?end_processing@hb_sanitize_context_t@@QEAAXXZ 00000001800d5c80     hb-aat-layout.obj
 0002:0002ac8c       $unwind$??$check_array@U?$Entry@X@AAT@@@hb_sanitize_context_t@@QEBA_NPEBU?$Entry@X@AAT@@I@Z 00000001800d5c8c     hb-aat-layout.obj
 0002:0002ac8c       $unwind$??$check_array@UFeature@AAT@@@hb_sanitize_context_t@@QEBA_NPEBUFeature@AAT@@I@Z 00000001800d5c8c     hb-aat-layout.obj
 0002:0002ac8c       $unwind$??$check_array@UHBGlyphID16@OT@@@hb_sanitize_context_t@@QEBA_NPEBUHBGlyphID16@OT@@I@Z 00000001800d5c8c     hb-aat-layout.obj
 0002:0002ac8c       $unwind$?may_edit@hb_sanitize_context_t@@QEAA_NPEBXI@Z 00000001800d5c8c     hb-aat-layout.obj
 0002:0002ac8c       $unwind$?sanitize_shallow@?$UnsizedArrayOf@U?$HBFixed@U?$IntType@H$03@OT@@$0BA@@OT@@@OT@@QEBA_NPEAUhb_sanitize_context_t@@I@Z 00000001800d5c8c     hb-aat-layout.obj
 0002:0002ac8c       $unwind$?sanitize_shallow@?$UnsizedArrayOf@U?$IntType@I$03@OT@@@OT@@QEBA_NPEAUhb_sanitize_context_t@@I@Z 00000001800d5c8c     hb-aat-layout.obj
 0002:0002ac8c       $unwind$?sanitize_shallow@?$UnsizedArrayOf@U?$OffsetTo@U?$ArrayOf@UAnchor@AAT@@U?$IntType@I$03@OT@@@OT@@U?$IntType@G$01@2@X$0A@@OT@@@OT@@QEBA_NPEAUhb_sanitize_context_t@@I@Z 00000001800d5c8c     hb-aat-layout.obj
 0002:0002ac8c       $unwind$?sanitize_shallow@?$UnsizedArrayOf@U?$OffsetTo@U?$Lookup@UHBGlyphID16@OT@@@AAT@@U?$IntType@G$01@OT@@X$0A@@OT@@@OT@@QEBA_NPEAUhb_sanitize_context_t@@I@Z 00000001800d5c8c     hb-aat-layout.obj
 0002:0002ac8c       $unwind$?sanitize_shallow@?$UnsizedArrayOf@U?$OffsetTo@U?$Lookup@UHBGlyphID16@OT@@@AAT@@U?$IntType@I$03@OT@@X$0A@@OT@@@OT@@QEBA_NPEAUhb_sanitize_context_t@@I@Z 00000001800d5c8c     hb-aat-layout.obj
 0002:0002ac8c       $unwind$?sanitize_shallow@?$UnsizedArrayOf@UFeatureName@AAT@@@OT@@QEBA_NPEAUhb_sanitize_context_t@@I@Z 00000001800d5c8c     hb-aat-layout.obj
 0002:0002ac8c       $unwind$?sanitize_shallow@?$UnsizedArrayOf@USettingName@AAT@@@OT@@QEBA_NPEAUhb_sanitize_context_t@@I@Z 00000001800d5c8c     hb-aat-layout.obj
 0002:0002ac8c       $unwind$?sanitize_shallow@?$UnsizedArrayOf@UTrackTableEntry@AAT@@@OT@@QEBA_NPEAUhb_sanitize_context_t@@I@Z 00000001800d5c8c     hb-aat-layout.obj
 0002:0002ac8c       $unwind$?sanitize_shallow@?$UnsizedArrayOf@UVarRegionAxis@OT@@@OT@@QEBA_NPEAUhb_sanitize_context_t@@I@Z 00000001800d5c8c     hb-aat-layout.obj
 0002:0002ac8c       $unwind$??$check_array@U?$IntType@G$01@OT@@@hb_sanitize_context_t@@QEBA_NPEBU?$IntType@G$01@OT@@I@Z 00000001800d5c8c     hb-common.obj
 0002:0002ac8c       $unwind$??$check_array@U?$IntType@I$03@OT@@@hb_sanitize_context_t@@QEBA_NPEBU?$IntType@I$03@OT@@I@Z 00000001800d5c8c     hb-common.obj
 0002:0002ac8c       $unwind$?sanitize_shallow@?$UnsizedArrayOf@U?$HBFixed@U?$IntType@F$01@OT@@$0O@@OT@@@OT@@QEBA_NPEAUhb_sanitize_context_t@@I@Z 00000001800d5c8c     hb-common.obj
 0002:0002ac8c       $unwind$?sanitize_shallow@?$UnsizedArrayOf@UResourceRecord@OT@@@OT@@QEBA_NPEAUhb_sanitize_context_t@@I@Z 00000001800d5c8c     hb-face.obj
 0002:0002ac8c       $unwind$?get_extents@accelerator_t@cff2@OT@@QEBA_NPEAUhb_font_t@@IPEAUhb_glyph_extents_t@@@Z 00000001800d5c8c     hb-ot-cff2-table.obj
 0002:0002ac8c       $unwind$?get_path@accelerator_t@cff2@OT@@QEBA_NPEAUhb_font_t@@IAEAUhb_draw_session_t@@@Z 00000001800d5c8c     hb-ot-cff2-table.obj
 0002:0002ac8c       $unwind$?sanitize_shallow@?$UnsizedArrayOf@U?$IntType@G$01@OT@@@OT@@QEBA_NPEAUhb_sanitize_context_t@@I@Z 00000001800d5c8c     hb-ot-color.obj
 0002:0002ac8c       $unwind$?sanitize_shallow@?$UnsizedArrayOf@U?$Offset@U?$IntType@G$01@OT@@$00@OT@@@OT@@QEBA_NPEAUhb_sanitize_context_t@@I@Z 00000001800d5c8c     hb-ot-color.obj
 0002:0002ac8c       $unwind$?sanitize_shallow@?$UnsizedArrayOf@U?$Offset@U?$IntType@I$03@OT@@$00@OT@@@OT@@QEBA_NPEAUhb_sanitize_context_t@@I@Z 00000001800d5c8c     hb-ot-color.obj
 0002:0002ac8c       $unwind$?sanitize_shallow@?$UnsizedArrayOf@UBaseGlyphRecord@OT@@@OT@@QEBA_NPEAUhb_sanitize_context_t@@I@Z 00000001800d5c8c     hb-ot-color.obj
 0002:0002ac8c       $unwind$?sanitize_shallow@?$UnsizedArrayOf@UIndex@OT@@@OT@@QEBA_NPEAUhb_sanitize_context_t@@I@Z 00000001800d5c8c     hb-ot-color.obj
 0002:0002ac8c       $unwind$?sanitize_shallow@?$UnsizedArrayOf@UIndexSubtableRecord@OT@@@OT@@QEBA_NPEAUhb_sanitize_context_t@@I@Z 00000001800d5c8c     hb-ot-color.obj
 0002:0002ac8c       $unwind$?sanitize_shallow@?$UnsizedArrayOf@ULayerRecord@OT@@@OT@@QEBA_NPEAUhb_sanitize_context_t@@I@Z 00000001800d5c8c     hb-ot-color.obj
 0002:0002ac8c       $unwind$??$sanitize@Uhb_sanitize_context_t@@@?$hb_array_t@$$CBE@@QEBA_NPEAUhb_sanitize_context_t@@@Z 00000001800d5c8c     hb-ot-font.obj
 0002:0002ac8c       $unwind$?sanitize_shallow@?$UnsizedArrayOf@U?$OffsetTo@UAxisValue@OT@@U?$IntType@G$01@2@X$00@OT@@@OT@@QEBA_NPEAUhb_sanitize_context_t@@I@Z 00000001800d5c8c     hb-ot-shape.obj
 0002:0002ac8c       $unwind$?sanitize_shallow@?$UnsizedArrayOf@UAxisValueRecord@OT@@@OT@@QEBA_NPEAUhb_sanitize_context_t@@I@Z 00000001800d5c8c     hb-ot-shape.obj
 0002:0002ac8c       $unwind$?sanitize_shallow@?$UnsizedArrayOf@UStatAxisRecord@OT@@@OT@@QEBA_NPEAUhb_sanitize_context_t@@I@Z 00000001800d5c8c     hb-ot-shape.obj
 0002:0002ac94       $unwind$?get@?$hb_lazy_loader_t@UGDEF_accelerator_t@OT@@U?$hb_face_lazy_loader_t@UGDEF_accelerator_t@OT@@$0BI@@@Uhb_face_t@@$0BI@U12@@@QEBAPEBUGDEF_accelerator_t@OT@@XZ 00000001800d5c94     hb-aat-layout.obj
 0002:0002ac94       $unwind$??C?$hb_lazy_loader_t@Uglyf_accelerator_t@OT@@U?$hb_face_lazy_loader_t@Uglyf_accelerator_t@OT@@$0P@@@Uhb_face_t@@$0P@U12@@@QEBAPEBUglyf_accelerator_t@OT@@XZ 00000001800d5c94     hb-common.obj
 0002:0002ac94       $unwind$?get@?$hb_lazy_loader_t@Uhmtx_accelerator_t@OT@@U?$hb_face_lazy_loader_t@Uhmtx_accelerator_t@OT@@$04@@Uhb_face_t@@$04U12@@@QEBAPEBUhmtx_accelerator_t@OT@@XZ 00000001800d5c94     hb-common.obj
 0002:0002ac94       $unwind$?get@?$hb_lazy_loader_t@Uvmtx_accelerator_t@OT@@U?$hb_face_lazy_loader_t@Uvmtx_accelerator_t@OT@@$0M@@@Uhb_face_t@@$0M@U12@@@QEBAPEBUvmtx_accelerator_t@OT@@XZ 00000001800d5c94     hb-common.obj
 0002:0002ac94       $unwind$?parse_tag@@YA_NPEAPEBDPEBDPEAI@Z 00000001800d5c94     hb-common.obj
 0002:0002ac94       $unwind$??C?$hb_lazy_loader_t@Ucmap_accelerator_t@OT@@U?$hb_face_lazy_loader_t@Ucmap_accelerator_t@OT@@$02@@Uhb_face_t@@$02U12@@@QEBAPEBUcmap_accelerator_t@OT@@XZ 00000001800d5c94     hb-face.obj
 0002:0002ac94       $unwind$??C?$hb_lazy_loader_t@Ucff1_accelerator_t@OT@@U?$hb_face_lazy_loader_t@Ucff1_accelerator_t@OT@@$0BA@@@Uhb_face_t@@$0BA@U12@@@QEBAPEBUcff1_accelerator_t@OT@@XZ 00000001800d5c94     hb-ot-font.obj
 0002:0002ac94       $unwind$??C?$hb_lazy_loader_t@Upost_accelerator_t@OT@@U?$hb_face_lazy_loader_t@Upost_accelerator_t@OT@@$06@@Uhb_face_t@@$06U12@@@QEBAPEBUpost_accelerator_t@OT@@XZ 00000001800d5c94     hb-ot-font.obj
 0002:0002ac94       $unwind$??$apply_string@UGSUBProxy@@@@YA_NPEAUhb_ot_apply_context_t@OT@@AEBUSubstLookup@GSUB_impl@Layout@1@AEBUhb_ot_layout_lookup_accelerator_t@1@@Z 00000001800d5c94     hb-ot-layout.obj
 0002:0002ac94       $unwind$?get_accel@?$accelerator_t@UGPOS@Layout@OT@@@GSUBGPOS@OT@@QEBAPEAUhb_ot_layout_lookup_accelerator_t@3@I@Z 00000001800d5c94     hb-ot-layout.obj
 0002:0002ac94       $unwind$?get_accel@?$accelerator_t@UGSUB@Layout@OT@@@GSUBGPOS@OT@@QEBAPEAUhb_ot_layout_lookup_accelerator_t@3@I@Z 00000001800d5c94     hb-ot-layout.obj
 0002:0002aca8       $unwind$??$collect_glyphs@Uhb_bit_set_t@@@KerxSubTable@AAT@@QEBAXAEAUhb_bit_set_t@@0I@Z 00000001800d5ca8     hb-aat-layout.obj
 0002:0002aca8       $unwind$?get@?$hb_lazy_loader_t@Ukerx_accelerator_t@AAT@@U?$hb_face_lazy_loader_t@Ukerx_accelerator_t@AAT@@$0BO@@@Uhb_face_t@@$0BO@U12@@@QEBAPEBUkerx_accelerator_t@AAT@@XZ 00000001800d5ca8     hb-aat-layout.obj
 0002:0002aca8       $unwind$?get@?$hb_lazy_loader_t@Umorx_accelerator_t@AAT@@U?$hb_face_lazy_loader_t@Umorx_accelerator_t@AAT@@$0BM@@@Uhb_face_t@@$0BM@U12@@@QEBAPEBUmorx_accelerator_t@AAT@@XZ 00000001800d5ca8     hb-aat-layout.obj
 0002:0002aca8       $unwind$?resize@hb_bit_set_t@@QEAA_NI_N0@Z 00000001800d5ca8     hb-aat-layout.obj
 0002:0002aca8       $unwind$?hb_parse_double@@YA_NPEAPEBDPEBDPEAN_N@Z 00000001800d5ca8     hb-number.obj
 0002:0002aca8       $unwind$??A?$CFFIndex@U?$IntType@I$03@OT@@@OT@@QEBA?AU?$hb_array_t@$$CBE@@I@Z 00000001800d5ca8     hb-ot-cff2-table.obj
 0002:0002aca8       $unwind$?_fini@?$accelerator_templ_t@Ucff2_private_dict_opset_t@CFF@@U?$cff2_private_dict_values_base_t@Udict_val_t@CFF@@@2@@cff2@OT@@QEAAXXZ 00000001800d5ca8     hb-ot-face.obj
 0002:0002aca8       $unwind$??C?$hb_lazy_loader_t@Ucff2_accelerator_t@OT@@U?$hb_face_lazy_loader_t@Ucff2_accelerator_t@OT@@$0BB@@@Uhb_face_t@@$0BB@U12@@@QEBAPEBUcff2_accelerator_t@OT@@XZ 00000001800d5ca8     hb-ot-font.obj
 0002:0002aca8       $unwind$?get@?$hb_lazy_loader_t@Ukern_accelerator_t@OT@@U?$hb_face_lazy_loader_t@Ukern_accelerator_t@OT@@$0BH@@@Uhb_face_t@@$0BH@U12@@@QEBAPEBUkern_accelerator_t@OT@@XZ 00000001800d5ca8     hb-ot-layout.obj
 0002:0002acbc       $unwind$?get_stored@?$hb_lazy_loader_t@Umort_accelerator_t@AAT@@U?$hb_face_lazy_loader_t@Umort_accelerator_t@AAT@@$0BN@@@Uhb_face_t@@$0BN@U12@@@QEBAPEAUmort_accelerator_t@AAT@@XZ 00000001800d5cbc     hb-aat-layout.obj
 0002:0002acbc       $unwind$??C?$hb_lazy_loader_t@UCOLR_accelerator_t@OT@@U?$hb_face_lazy_loader_t@UCOLR_accelerator_t@OT@@$0CD@@@Uhb_face_t@@$0CD@U12@@@QEBAPEBUCOLR_accelerator_t@OT@@XZ 00000001800d5cbc     hb-ot-color.obj
 0002:0002acbc       $unwind$??C?$hb_lazy_loader_t@Usbix_accelerator_t@OT@@U?$hb_face_lazy_loader_t@Usbix_accelerator_t@OT@@$0CG@@@Uhb_face_t@@$0CG@U12@@@QEBAPEBUsbix_accelerator_t@OT@@XZ 00000001800d5cbc     hb-ot-color.obj
 0002:0002acd8       $unwind$??C?$hb_lazy_loader_t@Ufeat@AAT@@U?$hb_table_lazy_loader_t@Ufeat@AAT@@$0CC@$0A@@@Uhb_face_t@@$0CC@Uhb_blob_t@@@@QEBAPEBUfeat@AAT@@XZ 00000001800d5cd8     hb-aat-layout.obj
 0002:0002acd8       $unwind$??C?$hb_lazy_loader_t@Ultag@AAT@@U?$hb_table_lazy_loader_t@Ultag@AAT@@$0CB@$0A@@@Uhb_face_t@@$0CB@Uhb_blob_t@@@@QEBAPEBUltag@AAT@@XZ 00000001800d5cd8     hb-aat-layout.obj
 0002:0002acd8       $unwind$?get@?$hb_lazy_loader_t@Utrak@AAT@@U?$hb_table_lazy_loader_t@Utrak@AAT@@$0CA@$0A@@@Uhb_face_t@@$0CA@Uhb_blob_t@@@@QEBAPEBUtrak@AAT@@XZ 00000001800d5cd8     hb-aat-layout.obj
 0002:0002acd8       $unwind$??C?$hb_lazy_loader_t@Uhhea@OT@@U?$hb_table_lazy_loader_t@Uhhea@OT@@$03$00@@Uhb_face_t@@$03Uhb_blob_t@@@@QEBAPEBUhhea@OT@@XZ 00000001800d5cd8     hb-common.obj
 0002:0002acd8       $unwind$??C?$hb_lazy_loader_t@Umaxp@OT@@U?$hb_table_lazy_loader_t@Umaxp@OT@@$01$00@@Uhb_face_t@@$01Uhb_blob_t@@@@QEBAPEBUmaxp@OT@@XZ 00000001800d5cd8     hb-common.obj
 0002:0002acd8       $unwind$??C?$hb_lazy_loader_t@Uvhea@OT@@U?$hb_table_lazy_loader_t@Uvhea@OT@@$0L@$00@@Uhb_face_t@@$0L@Uhb_blob_t@@@@QEBAPEBUvhea@OT@@XZ 00000001800d5cd8     hb-common.obj
 0002:0002acd8       $unwind$?get@?$hb_lazy_loader_t@Uhead@OT@@U?$hb_table_lazy_loader_t@Uhead@OT@@$00$00@@Uhb_face_t@@$00Uhb_blob_t@@@@QEBAPEBUhead@OT@@XZ 00000001800d5cd8     hb-common.obj
 0002:0002acd8       $unwind$?get@?$hb_lazy_loader_t@Ufvar@OT@@U?$hb_table_lazy_loader_t@Ufvar@OT@@$0BC@$00@@Uhb_face_t@@$0BC@Uhb_blob_t@@@@QEBAPEBUfvar@OT@@XZ 00000001800d5cd8     hb-font.obj
 0002:0002acd8       $unwind$??C?$hb_lazy_loader_t@UCPAL@OT@@U?$hb_table_lazy_loader_t@UCPAL@OT@@$0CE@$00@@Uhb_face_t@@$0CE@Uhb_blob_t@@@@QEBAPEBUCPAL@OT@@XZ 00000001800d5cd8     hb-ot-color.obj
 0002:0002acd8       $unwind$??C?$hb_lazy_loader_t@UOS2@OT@@U?$hb_table_lazy_loader_t@UOS2@OT@@$05$00@@Uhb_face_t@@$05Uhb_blob_t@@@@QEBAPEBUOS2@OT@@XZ 00000001800d5cd8     hb-ot-metrics.obj
 0002:0002acd8       $unwind$?get@?$hb_lazy_loader_t@UMVAR@OT@@U?$hb_table_lazy_loader_t@UMVAR@OT@@$0BG@$00@@Uhb_face_t@@$0BG@Uhb_blob_t@@@@QEBAPEBUMVAR@OT@@XZ 00000001800d5cd8     hb-ot-metrics.obj
 0002:0002acd8       $unwind$??C?$hb_lazy_loader_t@Uavar@OT@@U?$hb_table_lazy_loader_t@Uavar@OT@@$0BD@$00@@Uhb_face_t@@$0BD@Uhb_blob_t@@@@QEBAPEBUavar@OT@@XZ 00000001800d5cd8     hb-ot-var.obj
 0002:0002ace8       $chain$1$?get@?$hb_lazy_loader_t@Utrak@AAT@@U?$hb_table_lazy_loader_t@Utrak@AAT@@$0CA@$0A@@@Uhb_face_t@@$0CA@Uhb_blob_t@@@@QEBAPEBUtrak@AAT@@XZ 00000001800d5ce8     hb-aat-layout.obj
 0002:0002ad00       $chain$2$?get@?$hb_lazy_loader_t@Utrak@AAT@@U?$hb_table_lazy_loader_t@Utrak@AAT@@$0CA@$0A@@@Uhb_face_t@@$0CA@Uhb_blob_t@@@@QEBAPEBUtrak@AAT@@XZ 00000001800d5d00     hb-aat-layout.obj
 0002:0002ad10       $chain$1$??C?$hb_lazy_loader_t@Ultag@AAT@@U?$hb_table_lazy_loader_t@Ultag@AAT@@$0CB@$0A@@@Uhb_face_t@@$0CB@Uhb_blob_t@@@@QEBAPEBUltag@AAT@@XZ 00000001800d5d10     hb-aat-layout.obj
 0002:0002ad28       $chain$2$??C?$hb_lazy_loader_t@Ultag@AAT@@U?$hb_table_lazy_loader_t@Ultag@AAT@@$0CB@$0A@@@Uhb_face_t@@$0CB@Uhb_blob_t@@@@QEBAPEBUltag@AAT@@XZ 00000001800d5d28     hb-aat-layout.obj
 0002:0002ad38       $chain$1$??C?$hb_lazy_loader_t@Ufeat@AAT@@U?$hb_table_lazy_loader_t@Ufeat@AAT@@$0CC@$0A@@@Uhb_face_t@@$0CC@Uhb_blob_t@@@@QEBAPEBUfeat@AAT@@XZ 00000001800d5d38     hb-aat-layout.obj
 0002:0002ad50       $chain$2$??C?$hb_lazy_loader_t@Ufeat@AAT@@U?$hb_table_lazy_loader_t@Ufeat@AAT@@$0CC@$0A@@@Uhb_face_t@@$0CC@Uhb_blob_t@@@@QEBAPEBUfeat@AAT@@XZ 00000001800d5d50     hb-aat-layout.obj
 0002:0002ad60       $unwind$?add_range@hb_bit_page_t@@QEAAXII@Z 00000001800d5d60     hb-aat-layout.obj
 0002:0002ad60       $unwind$?_cached_get@accelerator_t@cmap@OT@@QEBA_NIPEAI@Z 00000001800d5d60     hb-ot-font.obj
 0002:0002ad74       $unwind$?alloc@?$hb_vector_t@Uhb_bit_page_t@@$0A@@@QEAA_NI_N@Z 00000001800d5d74     hb-aat-layout.obj
 0002:0002ad74       $unwind$?alloc@?$hb_vector_t@Upage_map_t@hb_bit_set_t@@$00@@QEAA_NI_N@Z 00000001800d5d74     hb-aat-layout.obj
 0002:0002ad74       $unwind$?setup_buffer_glyph_set@hb_aat_apply_context_t@AAT@@QEAAXXZ 00000001800d5d74     hb-aat-layout.obj
 0002:0002ad74       $unwind$?alloc@?$hb_vector_t@Ufeature_info_t@hb_aat_map_builder_t@@$00@@QEAA_NI_N@Z 00000001800d5d74     hb-aat-map.obj
 0002:0002ad74       $unwind$?alloc@?$hb_vector_t@Ucontour_point_t@@$0A@@@QEAA_NI_N@Z 00000001800d5d74     hb-common.obj
 0002:0002ad74       $unwind$?alloc@?$hb_vector_t@Uhb_bounds_t@@$0A@@@QEAA_NI_N@Z 00000001800d5d74     hb-font.obj
 0002:0002ad74       $unwind$?alloc@?$hb_vector_t@Uhb_transform_t@@$0A@@@QEAA_NI_N@Z 00000001800d5d74     hb-font.obj
 0002:0002ad74       $unwind$?acquire_varStore_cache@advance_cache_t@hb_ot_font_t@@QEBAPEAU?$hb_atomic_t@H@@AEBUItemVariationStore@OT@@@Z 00000001800d5d74     hb-ot-font.obj
 0002:0002ad74       $unwind$?alloc@?$hb_vector_t@Ufeature_info_t@hb_ot_map_builder_t@@$0A@@@QEAA_NI_N@Z 00000001800d5d74     hb-ot-map.obj
 0002:0002ad74       $unwind$?alloc@?$hb_vector_t@Ulookup_map_t@hb_ot_map_t@@$0A@@@QEAA_NI_N@Z 00000001800d5d74     hb-ot-map.obj
 0002:0002ad74       $unwind$?alloc@?$hb_vector_t@Uhb_outline_point_t@@$0A@@@QEAA_NI_N@Z 00000001800d5d74     hb-outline.obj
 0002:0002ad7c       $chain$0$?alloc@?$hb_vector_t@Upage_map_t@hb_bit_set_t@@$00@@QEAA_NI_N@Z 00000001800d5d7c     hb-aat-layout.obj
 0002:0002ad90       $chain$2$?alloc@?$hb_vector_t@Upage_map_t@hb_bit_set_t@@$00@@QEAA_NI_N@Z 00000001800d5d90     hb-aat-layout.obj
 0002:0002ad90       $chain$4$?alloc@?$hb_vector_t@Upage_map_t@hb_bit_set_t@@$00@@QEAA_NI_N@Z 00000001800d5d90     hb-aat-layout.obj
 0002:0002ada4       $chain$0$?alloc@?$hb_vector_t@Uhb_bit_page_t@@$0A@@@QEAA_NI_N@Z 00000001800d5da4     hb-aat-layout.obj
 0002:0002adb8       $chain$2$?alloc@?$hb_vector_t@Uhb_bit_page_t@@$0A@@@QEAA_NI_N@Z 00000001800d5db8     hb-aat-layout.obj
 0002:0002adb8       $chain$4$?alloc@?$hb_vector_t@Uhb_bit_page_t@@$0A@@@QEAA_NI_N@Z 00000001800d5db8     hb-aat-layout.obj
 0002:0002adcc       $unwind$??0hb_aat_apply_context_t@AAT@@QEAA@PEBUhb_ot_shape_plan_t@@PEAUhb_font_t@@PEAUhb_buffer_t@@PEAUhb_blob_t@@@Z 00000001800d5dcc     hb-aat-layout.obj
 0002:0002adcc       $unwind$??0hb_ot_apply_context_t@OT@@QEAA@IPEAUhb_font_t@@PEAUhb_buffer_t@@PEAUhb_blob_t@@PEAU?$hb_atomic_t@H@@@Z 00000001800d5dcc     hb-aat-layout.obj
 0002:0002adcc       $unwind$?get_kerning@?$KerxSubTableFormat0@UKerxSubTableHeader@AAT@@@AAT@@QEBAHIIPEAUhb_aat_apply_context_t@2@@Z 00000001800d5dcc     hb-aat-layout.obj
 0002:0002adcc       $unwind$?hb_aat_layout_compile_map@@YAXPEBUhb_aat_map_builder_t@@PEAUhb_aat_map_t@@@Z 00000001800d5dcc     hb-aat-layout.obj
 0002:0002adcc       $unwind$?resize@?$hb_vector_t@Uhb_bit_page_t@@$0A@@@QEAA_NH_N0@Z 00000001800d5dcc     hb-aat-layout.obj
 0002:0002adcc       $unwind$hb_face_create_for_tables 00000001800d5dcc     hb-face.obj
 0002:0002adcc       $unwind$?_hb_font_adopt_var_coords@@YAXPEAUhb_font_t@@PEAHPEAMI@Z 00000001800d5dcc     hb-font.obj
 0002:0002adcc       $unwind$??1?$accelerator_templ_t@Ucff1_private_dict_opset_t@CFF@@U?$cff1_private_dict_values_base_t@Udict_val_t@CFF@@@2@@cff1@OT@@QEAA@XZ 00000001800d5dcc     hb-ot-face.obj
 0002:0002adcc       $unwind$??1?$accelerator_templ_t@Ucff2_private_dict_opset_t@CFF@@U?$cff2_private_dict_values_base_t@Udict_val_t@CFF@@@2@@cff2@OT@@QEAA@XZ 00000001800d5dcc     hb-ot-face.obj
 0002:0002adcc       $unwind$??_Ghb_colr_scratch_t@@QEAAPEAXI@Z 00000001800d5dcc     hb-ot-face.obj
 0002:0002adcc       $unwind$?_fini@?$accelerator_templ_t@Ucff1_private_dict_opset_t@CFF@@U?$cff1_private_dict_values_base_t@Udict_val_t@CFF@@@2@@cff1@OT@@QEAAXXZ 00000001800d5dcc     hb-ot-face.obj
 0002:0002adcc       $unwind$?hb_ot_get_variation_glyph@@YAHPEAUhb_font_t@@PEAXIIPEAI1@Z 00000001800d5dcc     hb-ot-font.obj
 0002:0002adcc       $unwind$?_set_glyph_class@hb_ot_apply_context_t@OT@@QEAAXII_N0@Z 00000001800d5dcc     hb-ot-layout.obj
 0002:0002adcc       $unwind$?is_blocklisted@GDEF@OT@@QEBA_NPEAUhb_blob_t@@PEAUhb_face_t@@@Z 00000001800d5dcc     hb-ot-layout.obj
 0002:0002adcc       $unwind$?fini@hb_ot_map_t@@QEAAXXZ 00000001800d5dcc     hb-ot-shape.obj
 0002:0002adcc       $unwind$??$add_link@U?$OffsetTo@U?$Ligature@USmallTypes@Layout@OT@@@GSUB_impl@Layout@OT@@U?$IntType@G$01@4@X$00@OT@@@hb_serialize_context_t@@QEAAXAEAU?$OffsetTo@U?$Ligature@USmallTypes@Layout@OT@@@GSUB_impl@Layout@OT@@U?$IntType@G$01@4@X$00@OT@@IW4whence_t@0@I@Z 00000001800d5dcc     hb-ot-shaper-arabic.obj
 0002:0002adcc       $unwind$??$add_link@U?$OffsetTo@U?$LigatureSet@USmallTypes@Layout@OT@@@GSUB_impl@Layout@OT@@U?$IntType@G$01@4@X$00@OT@@@hb_serialize_context_t@@QEAAXAEAU?$OffsetTo@U?$LigatureSet@USmallTypes@Layout@OT@@@GSUB_impl@Layout@OT@@U?$IntType@G$01@4@X$00@OT@@IW4whence_t@0@I@Z 00000001800d5dcc     hb-ot-shaper-arabic.obj
 0002:0002adcc       $unwind$??$add_link@U?$OffsetTo@UCoverage@Common@Layout@OT@@U?$IntType@G$01@4@X$00@OT@@@hb_serialize_context_t@@QEAAXAEAU?$OffsetTo@UCoverage@Common@Layout@OT@@U?$IntType@G$01@4@X$00@OT@@IW4whence_t@0@I@Z 00000001800d5dcc     hb-ot-shaper-arabic.obj
 0002:0002adcc       $unwind$?collect_features_arabic@@YAXPEAUhb_ot_shape_planner_t@@@Z 00000001800d5dcc     hb-ot-shaper-arabic.obj
 0002:0002adcc       $unwind$?collect_features_myanmar@@YAXPEAUhb_ot_shape_planner_t@@@Z 00000001800d5dcc     hb-ot-shaper-myanmar.obj
 0002:0002adcc       $unwind$hb_ot_var_named_instance_get_design_coords 00000001800d5dcc     hb-ot-var.obj
 0002:0002adcc       $unwind$hb_unicode_funcs_set_combining_class_func 00000001800d5dcc     hb-unicode.obj
 0002:0002adcc       $unwind$hb_unicode_funcs_set_compose_func 00000001800d5dcc     hb-unicode.obj
 0002:0002adcc       $unwind$hb_unicode_funcs_set_decompose_func 00000001800d5dcc     hb-unicode.obj
 0002:0002adcc       $unwind$hb_unicode_funcs_set_general_category_func 00000001800d5dcc     hb-unicode.obj
 0002:0002adcc       $unwind$hb_unicode_funcs_set_mirroring_func 00000001800d5dcc     hb-unicode.obj
 0002:0002adcc       $unwind$hb_unicode_funcs_set_script_func 00000001800d5dcc     hb-unicode.obj
 0002:0002adcc       $unwind$__scrt_dllmain_exception_filter 00000001800d5dcc     MSVCRT:utility.obj
 0002:0002ade0       $chain$0$?resize@hb_bit_set_t@@QEAA_NI_N0@Z 00000001800d5de0     hb-aat-layout.obj
 0002:0002adf4       $chain$1$?resize@hb_bit_set_t@@QEAA_NI_N0@Z 00000001800d5df4     hb-aat-layout.obj
 0002:0002ae04       $chain$1$?clear@hb_bit_set_t@@QEAAXXZ 00000001800d5e04     hb-aat-layout.obj
 0002:0002ae1c       $chain$4$?clear@hb_bit_set_t@@QEAAXXZ 00000001800d5e1c     hb-aat-layout.obj
 0002:0002ae30       $chain$3$?clear@hb_bit_set_t@@QEAAXXZ 00000001800d5e30     hb-aat-layout.obj
 0002:0002ae48       $chain$5$?clear@hb_bit_set_t@@QEAAXXZ 00000001800d5e48     hb-aat-layout.obj
 0002:0002ae58       $unwind$?add_range@hb_bit_set_t@@QEAA_NII@Z 00000001800d5e58     hb-aat-layout.obj
 0002:0002ae68       $chain$1$?add_range@hb_bit_set_t@@QEAA_NII@Z 00000001800d5e68     hb-aat-layout.obj
 0002:0002ae80       $chain$3$?add_range@hb_bit_set_t@@QEAA_NII@Z 00000001800d5e80     hb-aat-layout.obj
 0002:0002ae98       $unwind$?page_for@hb_bit_set_t@@IEAAPEAUhb_bit_page_t@@I_N@Z 00000001800d5e98     hb-aat-layout.obj
 0002:0002aeb4       $unwind$?guess_v_origin_minus_h_origin@hb_font_t@@QEAAXIPEAH0@Z 00000001800d5eb4     hb-aat-layout.obj
 0002:0002aecc       $unwind$?get_glyph_contour_point_for_origin@hb_font_t@@QEAAHIIW4hb_direction_t@@PEAH1@Z 00000001800d5ecc     hb-aat-layout.obj
 0002:0002aee8       $unwind$??$dispatch@Uhb_sanitize_context_t@@$$V@?$ChainSubtable@UObsoleteTypes@AAT@@@AAT@@QEBA_NPEAUhb_sanitize_context_t@@@Z 00000001800d5ee8     hb-aat-layout.obj
 0002:0002aee8       $unwind$?sanitize@?$IntType@G$01@OT@@QEBA_NPEAUhb_sanitize_context_t@@@Z 00000001800d5ee8     hb-aat-layout.obj
 0002:0002aee8       $unwind$?sanitize@?$IntType@H$03@OT@@QEBA_NPEAUhb_sanitize_context_t@@@Z 00000001800d5ee8     hb-aat-layout.obj
 0002:0002aee8       $unwind$?sanitize@?$IntType@I$03@OT@@QEBA_NPEAUhb_sanitize_context_t@@@Z 00000001800d5ee8     hb-aat-layout.obj
 0002:0002aee8       $unwind$?sanitize@FDSelect0@CFF@@QEBA_NPEAUhb_sanitize_context_t@@I@Z 00000001800d5ee8     hb-ot-font.obj
 0002:0002aee8       $unwind$?end_serialize@hb_serialize_context_t@@QEAAXXZ 00000001800d5ee8     hb-ot-shaper-arabic.obj
 0002:0002aef0       $unwind$??$sanitize@USubstLookupSubTable@GSUB_impl@Layout@OT@@@Lookup@OT@@QEBA_NPEAUhb_sanitize_context_t@@@Z 00000001800d5ef0     hb-aat-layout.obj
 0002:0002aef0       $unwind$??$sanitize_blob@Ufeat@AAT@@@hb_sanitize_context_t@@QEAAPEAUhb_blob_t@@PEAU1@@Z 00000001800d5ef0     hb-aat-layout.obj
 0002:0002aef0       $unwind$??$sanitize_blob@Ultag@AAT@@@hb_sanitize_context_t@@QEAAPEAUhb_blob_t@@PEAU1@@Z 00000001800d5ef0     hb-aat-layout.obj
 0002:0002aef0       $unwind$??$sanitize_blob@Umorx@AAT@@@hb_sanitize_context_t@@QEAAPEAUhb_blob_t@@PEAU1@@Z 00000001800d5ef0     hb-aat-layout.obj
 0002:0002aef0       $unwind$?sanitize@?$KerxTable@Ukerx@AAT@@@AAT@@QEBA_NPEAUhb_sanitize_context_t@@@Z 00000001800d5ef0     hb-aat-layout.obj
 0002:0002aef0       $unwind$?sanitize@?$Lookup@U?$OffsetTo@U?$ArrayOf@UAnchor@AAT@@U?$IntType@I$03@OT@@@OT@@U?$IntType@G$01@2@X$0A@@OT@@@AAT@@QEBA_NPEAUhb_sanitize_context_t@@PEBX@Z 00000001800d5ef0     hb-aat-layout.obj
 0002:0002aef0       $unwind$?sanitize@FeatureTableSubstitution@OT@@QEBA_NPEAUhb_sanitize_context_t@@@Z 00000001800d5ef0     hb-aat-layout.obj
 0002:0002aef0       $unwind$?sanitize@feat@AAT@@QEBA_NPEAUhb_sanitize_context_t@@@Z 00000001800d5ef0     hb-aat-layout.obj
 0002:0002aef0       $unwind$?sanitize@ltag@AAT@@QEBA_NPEAUhb_sanitize_context_t@@@Z 00000001800d5ef0     hb-aat-layout.obj
 0002:0002aef0       $unwind$?sanitize_shallow@?$gvar_GVAR@U?$IntType@G$01@OT@@$0GHHGGBHC@@OT@@QEBA_NPEAUhb_sanitize_context_t@@@Z 00000001800d5ef0     hb-common.obj
 0002:0002aef0       $unwind$?sanitize@CmapSubtableFormat14@OT@@QEBA_NPEAUhb_sanitize_context_t@@@Z 00000001800d5ef0     hb-face.obj
 0002:0002aef0       $unwind$?sanitize@cmap@OT@@QEBA_NPEAUhb_sanitize_context_t@@@Z 00000001800d5ef0     hb-face.obj
 0002:0002aef0       $unwind$?sanitize@avar@OT@@QEBA_NPEAUhb_sanitize_context_t@@@Z 00000001800d5ef0     hb-font.obj
 0002:0002aef0       $unwind$??$sanitize_blob@UCBLC@OT@@@hb_sanitize_context_t@@QEAAPEAUhb_blob_t@@PEAU1@@Z 00000001800d5ef0     hb-ot-color.obj
 0002:0002aef0       $unwind$??$sanitize_blob@Usbix@OT@@@hb_sanitize_context_t@@QEAAPEAUhb_blob_t@@PEAU1@@Z 00000001800d5ef0     hb-ot-color.obj
 0002:0002aef0       $unwind$?sanitize@ClipList@OT@@QEBA_NPEAUhb_sanitize_context_t@@@Z 00000001800d5ef0     hb-ot-color.obj
 0002:0002aef0       $unwind$?sanitize@?$FDSelect3_4@U?$IntType@G$01@OT@@U?$IntType@E$00@2@@CFF@@QEBA_NPEAUhb_sanitize_context_t@@I@Z 00000001800d5ef0     hb-ot-font.obj
 0002:0002aef0       $unwind$?sanitize@?$FDSelect3_4@U?$IntType@I$03@OT@@U?$IntType@G$01@2@@CFF@@QEBA_NPEAUhb_sanitize_context_t@@I@Z 00000001800d5ef0     hb-ot-font.obj
 0002:0002aef0       $unwind$??$sanitize@UPosLookupSubTable@GPOS_impl@Layout@OT@@@Lookup@OT@@QEBA_NPEAUhb_sanitize_context_t@@@Z 00000001800d5ef0     hb-ot-layout.obj
 0002:0002aef0       $unwind$?sanitize@MVAR@OT@@QEBA_NPEAUhb_sanitize_context_t@@@Z 00000001800d5ef0     hb-ot-metrics.obj
 0002:0002af0c       $unwind$?sanitize@?$ChainSubtable@UObsoleteTypes@AAT@@@AAT@@QEBA_NPEAUhb_sanitize_context_t@@@Z 00000001800d5f0c     hb-aat-layout.obj
 0002:0002af0c       $unwind$?sanitize_shallow@?$ArrayOf@U?$IntType@G$01@OT@@U12@@OT@@QEBA_NPEAUhb_sanitize_context_t@@@Z 00000001800d5f0c     hb-aat-layout.obj
 0002:0002af0c       $unwind$?sanitize_shallow@?$ArrayOf@U?$IntType@I$02@OT@@U?$IntType@G$01@2@@OT@@QEBA_NPEAUhb_sanitize_context_t@@@Z 00000001800d5f0c     hb-aat-layout.obj
 0002:0002af0c       $unwind$?sanitize_shallow@?$ArrayOf@U?$Offset@U?$IntType@G$01@OT@@$00@OT@@U?$IntType@G$01@2@@OT@@QEBA_NPEAUhb_sanitize_context_t@@@Z 00000001800d5f0c     hb-aat-layout.obj
 0002:0002af0c       $unwind$?sanitize_shallow@?$ArrayOf@U?$OffsetTo@U?$AlternateSet@USmallTypes@Layout@OT@@@GSUB_impl@Layout@OT@@U?$IntType@G$01@4@X$00@OT@@U?$IntType@G$01@2@@OT@@QEBA_NPEAUhb_sanitize_context_t@@@Z 00000001800d5f0c     hb-aat-layout.obj
 0002:0002af0c       $unwind$?sanitize_shallow@?$ArrayOf@U?$OffsetTo@U?$ChainRule@USmallTypes@Layout@OT@@@OT@@U?$IntType@G$01@2@X$00@OT@@U?$IntType@G$01@2@@OT@@QEBA_NPEAUhb_sanitize_context_t@@@Z 00000001800d5f0c     hb-aat-layout.obj
 0002:0002af0c       $unwind$?sanitize_shallow@?$ArrayOf@U?$OffsetTo@U?$ChainRuleSet@USmallTypes@Layout@OT@@@OT@@U?$IntType@G$01@2@X$00@OT@@U?$IntType@G$01@2@@OT@@QEBA_NPEAUhb_sanitize_context_t@@@Z 00000001800d5f0c     hb-aat-layout.obj
 0002:0002af0c       $unwind$?sanitize_shallow@?$ArrayOf@U?$OffsetTo@U?$Ligature@USmallTypes@Layout@OT@@@GSUB_impl@Layout@OT@@U?$IntType@G$01@4@X$00@OT@@U?$IntType@G$01@2@@OT@@QEBA_NPEAUhb_sanitize_context_t@@@Z 00000001800d5f0c     hb-aat-layout.obj
 0002:0002af0c       $unwind$?sanitize_shallow@?$ArrayOf@U?$OffsetTo@U?$LigatureSet@USmallTypes@Layout@OT@@@GSUB_impl@Layout@OT@@U?$IntType@G$01@4@X$00@OT@@U?$IntType@G$01@2@@OT@@QEBA_NPEAUhb_sanitize_context_t@@@Z 00000001800d5f0c     hb-aat-layout.obj
 0002:0002af0c       $unwind$?sanitize_shallow@?$ArrayOf@U?$OffsetTo@U?$Rule@USmallTypes@Layout@OT@@@OT@@U?$IntType@G$01@2@X$00@OT@@U?$IntType@G$01@2@@OT@@QEBA_NPEAUhb_sanitize_context_t@@@Z 00000001800d5f0c     hb-aat-layout.obj
 0002:0002af0c       $unwind$?sanitize_shallow@?$ArrayOf@U?$OffsetTo@U?$RuleSet@USmallTypes@Layout@OT@@@OT@@U?$IntType@G$01@2@X$00@OT@@U?$IntType@G$01@2@@OT@@QEBA_NPEAUhb_sanitize_context_t@@@Z 00000001800d5f0c     hb-aat-layout.obj
 0002:0002af0c       $unwind$?sanitize_shallow@?$ArrayOf@U?$OffsetTo@U?$Sequence@USmallTypes@Layout@OT@@@GSUB_impl@Layout@OT@@U?$IntType@G$01@4@X$00@OT@@U?$IntType@G$01@2@@OT@@QEBA_NPEAUhb_sanitize_context_t@@@Z 00000001800d5f0c     hb-aat-layout.obj
 0002:0002af0c       $unwind$?sanitize_shallow@?$ArrayOf@U?$OffsetTo@UAttachPoint@OT@@U?$IntType@G$01@2@X$00@OT@@U?$IntType@G$01@2@@OT@@QEBA_NPEAUhb_sanitize_context_t@@@Z 00000001800d5f0c     hb-aat-layout.obj
 0002:0002af0c       $unwind$?sanitize_shallow@?$ArrayOf@U?$OffsetTo@UCaretValue@OT@@U?$IntType@G$01@2@X$00@OT@@U?$IntType@G$01@2@@OT@@QEBA_NPEAUhb_sanitize_context_t@@@Z 00000001800d5f0c     hb-aat-layout.obj
 0002:0002af0c       $unwind$?sanitize_shallow@?$ArrayOf@U?$OffsetTo@UCondition@OT@@U?$IntType@I$02@2@X$00@OT@@U?$IntType@E$00@2@@OT@@QEBA_NPEAUhb_sanitize_context_t@@@Z 00000001800d5f0c     hb-aat-layout.obj
 0002:0002af0c       $unwind$?sanitize_shallow@?$ArrayOf@U?$OffsetTo@UCondition@OT@@U?$IntType@I$03@2@X$00@OT@@U?$IntType@G$01@2@@OT@@QEBA_NPEAUhb_sanitize_context_t@@@Z 00000001800d5f0c     hb-aat-layout.obj
 0002:0002af0c       $unwind$?sanitize_shallow@?$ArrayOf@U?$OffsetTo@UCoverage@Common@Layout@OT@@U?$IntType@G$01@4@X$00@OT@@U?$IntType@G$01@2@@OT@@QEBA_NPEAUhb_sanitize_context_t@@@Z 00000001800d5f0c     hb-aat-layout.obj
 0002:0002af0c       $unwind$?sanitize_shallow@?$ArrayOf@U?$OffsetTo@UCoverage@Common@Layout@OT@@U?$IntType@I$03@4@X$00@OT@@U?$IntType@G$01@2@@OT@@QEBA_NPEAUhb_sanitize_context_t@@@Z 00000001800d5f0c     hb-aat-layout.obj
 0002:0002af0c       $unwind$?sanitize_shallow@?$ArrayOf@U?$OffsetTo@ULigGlyph@OT@@U?$IntType@G$01@2@X$00@OT@@U?$IntType@G$01@2@@OT@@QEBA_NPEAUhb_sanitize_context_t@@@Z 00000001800d5f0c     hb-aat-layout.obj
 0002:0002af0c       $unwind$?sanitize_shallow@?$ArrayOf@U?$OffsetTo@USubstLookup@GSUB_impl@Layout@OT@@U?$IntType@G$01@4@X$00@OT@@U?$IntType@G$01@2@@OT@@QEBA_NPEAUhb_sanitize_context_t@@@Z 00000001800d5f0c     hb-aat-layout.obj
 0002:0002af0c       $unwind$?sanitize_shallow@?$ArrayOf@U?$OffsetTo@USubstLookupSubTable@GSUB_impl@Layout@OT@@U?$IntType@G$01@4@X$00@OT@@U?$IntType@G$01@2@@OT@@QEBA_NPEAUhb_sanitize_context_t@@@Z 00000001800d5f0c     hb-aat-layout.obj
 0002:0002af0c       $unwind$?sanitize_shallow@?$ArrayOf@U?$OffsetTo@UVarData@OT@@U?$IntType@I$03@2@X$00@OT@@U?$IntType@G$01@2@@OT@@QEBA_NPEAUhb_sanitize_context_t@@@Z 00000001800d5f0c     hb-aat-layout.obj
 0002:0002af0c       $unwind$?sanitize_shallow@?$ArrayOf@UAnchor@AAT@@U?$IntType@I$03@OT@@@OT@@QEBA_NPEAUhb_sanitize_context_t@@@Z 00000001800d5f0c     hb-aat-layout.obj
 0002:0002af0c       $unwind$?sanitize_shallow@?$ArrayOf@UFTStringRange@AAT@@U?$IntType@I$03@OT@@@OT@@QEBA_NPEAUhb_sanitize_context_t@@@Z 00000001800d5f0c     hb-aat-layout.obj
 0002:0002af0c       $unwind$?sanitize_shallow@?$ArrayOf@UFeatureVariationRecord@OT@@U?$IntType@I$03@2@@OT@@QEBA_NPEAUhb_sanitize_context_t@@@Z 00000001800d5f0c     hb-aat-layout.obj
 0002:0002af0c       $unwind$?sanitize_shallow@?$ArrayOf@UHBGlyphID16@OT@@U?$IntType@G$01@2@@OT@@QEBA_NPEAUhb_sanitize_context_t@@@Z 00000001800d5f0c     hb-aat-layout.obj
 0002:0002af0c       $unwind$?sanitize_shallow@?$ArrayOf@UIndex@OT@@U?$IntType@G$01@2@@OT@@QEBA_NPEAUhb_sanitize_context_t@@@Z 00000001800d5f0c     hb-aat-layout.obj
 0002:0002af0c       $unwind$?sanitize_shallow@?$ArrayOf@UKernPair@AAT@@U?$BinSearchHeader@U?$IntType@I$03@OT@@@OT@@@OT@@QEBA_NPEAUhb_sanitize_context_t@@@Z 00000001800d5f0c     hb-aat-layout.obj
 0002:0002af0c       $unwind$?sanitize_shallow@?$ArrayOf@ULookupRecord@OT@@U?$IntType@G$01@2@@OT@@QEBA_NPEAUhb_sanitize_context_t@@@Z 00000001800d5f0c     hb-aat-layout.obj
 0002:0002af0c       $unwind$?sanitize_shallow@?$ArrayOf@U?$OffsetTo@UOpenTypeOffsetTable@OT@@U?$IntType@I$03@2@X$00@OT@@U?$IntType@I$03@2@@OT@@QEBA_NPEAUhb_sanitize_context_t@@@Z 00000001800d5f0c     hb-face.obj
 0002:0002af0c       $unwind$?sanitize_shallow@?$ArrayOf@UEncodingRecord@OT@@U?$IntType@G$01@2@@OT@@QEBA_NPEAUhb_sanitize_context_t@@@Z 00000001800d5f0c     hb-face.obj
 0002:0002af0c       $unwind$?sanitize_shallow@?$ArrayOf@UHBGlyphID16@OT@@U?$IntType@I$03@2@@OT@@QEBA_NPEAUhb_sanitize_context_t@@@Z 00000001800d5f0c     hb-face.obj
 0002:0002af0c       $unwind$?sanitize_shallow@?$ArrayOf@UUVSMapping@OT@@U?$IntType@I$03@2@@OT@@QEBA_NPEAUhb_sanitize_context_t@@@Z 00000001800d5f0c     hb-face.obj
 0002:0002af0c       $unwind$?sanitize_shallow@?$ArrayOf@UUnicodeValueRange@OT@@U?$IntType@I$03@2@@OT@@QEBA_NPEAUhb_sanitize_context_t@@@Z 00000001800d5f0c     hb-face.obj
 0002:0002af0c       $unwind$?sanitize_shallow@?$ArrayOf@UVariationSelectorRecord@OT@@U?$IntType@I$03@2@@OT@@QEBA_NPEAUhb_sanitize_context_t@@@Z 00000001800d5f0c     hb-face.obj
 0002:0002af0c       $unwind$?sanitize_shallow@?$ArrayOfM1@UResourceTypeRecord@OT@@U?$IntType@G$01@2@@OT@@AEBA_NPEAUhb_sanitize_context_t@@@Z 00000001800d5f0c     hb-face.obj
 0002:0002af0c       $unwind$?sanitize_shallow@?$ArrayOf@UAxisValueMap@OT@@U?$IntType@G$01@2@@OT@@QEBA_NPEAUhb_sanitize_context_t@@@Z 00000001800d5f0c     hb-font.obj
 0002:0002af0c       $unwind$??$dispatch@USBIXStrike@OT@@$$V@hb_sanitize_context_t@@QEAA_NAEBUSBIXStrike@OT@@@Z 00000001800d5f0c     hb-ot-color.obj
 0002:0002af0c       $unwind$?sanitize_shallow@?$ArrayOf@U?$OffsetTo@UPaint@OT@@U?$IntType@I$03@2@X$00@OT@@U?$IntType@I$03@2@@OT@@QEBA_NPEAUhb_sanitize_context_t@@@Z 00000001800d5f0c     hb-ot-color.obj
 0002:0002af0c       $unwind$?sanitize_shallow@?$ArrayOf@U?$OffsetTo@USBIXStrike@OT@@U?$IntType@I$03@2@X$00@OT@@U?$IntType@I$03@2@@OT@@QEBA_NPEAUhb_sanitize_context_t@@@Z 00000001800d5f0c     hb-ot-color.obj
 0002:0002af0c       $unwind$?sanitize_shallow@?$ArrayOf@UClipRecord@OT@@U?$IntType@I$03@2@@OT@@QEBA_NPEAUhb_sanitize_context_t@@@Z 00000001800d5f0c     hb-ot-color.obj
 0002:0002af0c       $unwind$?sanitize_shallow@?$ArrayOf@U?$FDSelect3_4_Range@U?$IntType@G$01@OT@@U?$IntType@E$00@2@@CFF@@U?$IntType@G$01@OT@@@OT@@QEBA_NPEAUhb_sanitize_context_t@@@Z 00000001800d5f0c     hb-ot-font.obj
 0002:0002af0c       $unwind$?sanitize_shallow@?$ArrayOf@U?$IntType@E$00@OT@@U12@@OT@@QEBA_NPEAUhb_sanitize_context_t@@@Z 00000001800d5f0c     hb-ot-font.obj
 0002:0002af0c       $unwind$?sanitize_shallow@?$ArrayOf@UEncoding1_Range@CFF@@U?$IntType@E$00@OT@@@OT@@QEBA_NPEAUhb_sanitize_context_t@@@Z 00000001800d5f0c     hb-ot-font.obj
 0002:0002af0c       $unwind$?sanitize_shallow@?$ArrayOf@USuppEncoding@CFF@@U?$IntType@E$00@OT@@@OT@@QEBA_NPEAUhb_sanitize_context_t@@@Z 00000001800d5f0c     hb-ot-font.obj
 0002:0002af0c       $unwind$?sanitize_shallow@?$ArrayOf@UVertOriginMetric@OT@@U?$IntType@G$01@2@@OT@@QEBA_NPEAUhb_sanitize_context_t@@@Z 00000001800d5f0c     hb-ot-font.obj
 0002:0002af0c       $unwind$?sanitize_shallow@?$ArrayOf@U?$OffsetTo@U?$PairSet@USmallTypes@Layout@OT@@@GPOS_impl@Layout@OT@@U?$IntType@G$01@4@X$00@OT@@U?$IntType@G$01@2@@OT@@QEBA_NPEAUhb_sanitize_context_t@@@Z 00000001800d5f0c     hb-ot-layout.obj
 0002:0002af0c       $unwind$?sanitize_shallow@?$ArrayOf@U?$OffsetTo@UAnchorMatrix@GPOS_impl@Layout@OT@@U?$IntType@G$01@4@X$00@OT@@U?$IntType@G$01@2@@OT@@QEBA_NPEAUhb_sanitize_context_t@@@Z 00000001800d5f0c     hb-ot-layout.obj
 0002:0002af0c       $unwind$?sanitize_shallow@?$ArrayOf@U?$OffsetTo@UPosLookup@GPOS_impl@Layout@OT@@U?$IntType@G$01@4@X$00@OT@@U?$IntType@G$01@2@@OT@@QEBA_NPEAUhb_sanitize_context_t@@@Z 00000001800d5f0c     hb-ot-layout.obj
 0002:0002af0c       $unwind$?sanitize_shallow@?$ArrayOf@U?$OffsetTo@UPosLookupSubTable@GPOS_impl@Layout@OT@@U?$IntType@G$01@4@X$00@OT@@U?$IntType@G$01@2@@OT@@QEBA_NPEAUhb_sanitize_context_t@@@Z 00000001800d5f0c     hb-ot-layout.obj
 0002:0002af0c       $unwind$?sanitize_shallow@?$ArrayOf@UEntryExitRecord@GPOS_impl@Layout@OT@@U?$IntType@G$01@4@@OT@@QEBA_NPEAUhb_sanitize_context_t@@@Z 00000001800d5f0c     hb-ot-layout.obj
 0002:0002af0c       $unwind$?sanitize_shallow@?$ArrayOf@UMarkRecord@GPOS_impl@Layout@OT@@U?$IntType@G$01@4@@OT@@QEBA_NPEAUhb_sanitize_context_t@@@Z 00000001800d5f0c     hb-ot-layout.obj
 0002:0002af20       $unwind$?get_coverage@?$CoverageFormat1_3@USmallTypes@Layout@OT@@@Common@Layout@OT@@AEBAII@Z 00000001800d5f20     hb-aat-layout.obj
 0002:0002af20       $unwind$?get_feature@feat@AAT@@QEBAAEBUFeatureName@2@W4hb_aat_layout_feature_type_t@@@Z 00000001800d5f20     hb-aat-layout.obj
 0002:0002af20       $unwind$?hb_aat_layout_find_feature_mapping@@YAPEBUhb_aat_feature_mapping_t@@I@Z 00000001800d5f20     hb-aat-layout.obj
 0002:0002af20       $unwind$?parse_bool@@YA_NPEAPEBDPEBDPEAI@Z 00000001800d5f20     hb-common.obj
 0002:0002af20       $unwind$?get_base_glyph_record@COLR@OT@@QEBAPEBUBaseGlyphRecord@2@I@Z 00000001800d5f20     hb-ot-font.obj
 0002:0002af20       $unwind$?get_script@GSUBGPOS@OT@@QEBAAEBUScript@2@I@Z 00000001800d5f20     hb-ot-layout.obj
 0002:0002af20       $unwind$?cmp_range@?$RangeRecord@USmallTypes@Layout@OT@@@Common@Layout@OT@@SAHPEBX0@Z 00000001800d5f20     hb-ot-shaper-arabic.obj
 0002:0002af20       $unwind$??E?$hb_iter_t@U?$hb_filter_iter_t@U?$hb_filter_iter_t@U?$hb_zip_iter_t@U?$hb_iota_iter_t@II@@U?$hb_array_t@Uhb_glyph_info_t@@@@@@V<lambda_e52748becc06432fe81365edeb8c4003>@@AEBU<unnamed-type-hb_second>@@$0A@@@V<lambda_a2885d5959499a7c5bcf896c0de144bb>@@AEBU<unnamed-type-hb_identity>@@$0A@@@U?$hb_pair_t@IAEAUhb_glyph_info_t@@@@@@QEGAAAEAU?$hb_filter_iter_t@U?$hb_filter_iter_t@U?$hb_zip_iter_t@U?$hb_iota_iter_t@II@@U?$hb_array_t@Uhb_glyph_info_t@@@@@@V<lambda_e52748becc06432fe81365edeb8c4003>@@AEBU<unnamed-type-hb_second>@@$0A@@@V<lambda_a2885d5959499a7c5bcf896c0de144bb>@@AEBU<unnamed-type-hb_identity>@@$0A@@@XZ 00000001800d5f20     hb-ot-shaper-use.obj
 0002:0002af20       $unwind$??F?$hb_iter_t@U?$hb_filter_iter_t@U?$hb_filter_iter_t@U?$hb_zip_iter_t@U?$hb_iota_iter_t@II@@U?$hb_array_t@Uhb_glyph_info_t@@@@@@V<lambda_e52748becc06432fe81365edeb8c4003>@@AEBU<unnamed-type-hb_second>@@$0A@@@V<lambda_a2885d5959499a7c5bcf896c0de144bb>@@AEBU<unnamed-type-hb_identity>@@$0A@@@U?$hb_pair_t@IAEAUhb_glyph_info_t@@@@@@QEGAAAEAU?$hb_filter_iter_t@U?$hb_filter_iter_t@U?$hb_zip_iter_t@U?$hb_iota_iter_t@II@@U?$hb_array_t@Uhb_glyph_info_t@@@@@@V<lambda_e52748becc06432fe81365edeb8c4003>@@AEBU<unnamed-type-hb_second>@@$0A@@@V<lambda_a2885d5959499a7c5bcf896c0de144bb>@@AEBU<unnamed-type-hb_identity>@@$0A@@@XZ 00000001800d5f20     hb-ot-shaper-use.obj
 0002:0002af28       $unwind$?hb_aat_layout_substitute@@YAXPEBUhb_ot_shape_plan_t@@PEAUhb_font_t@@PEAUhb_buffer_t@@PEBUhb_feature_t@@I@Z 00000001800d5f28     hb-aat-layout.obj
 0002:0002af48       $unwind$?hb_aat_layout_position@@YAXPEBUhb_ot_shape_plan_t@@PEAUhb_font_t@@PEAUhb_buffer_t@@@Z 00000001800d5f48     hb-aat-layout.obj
 0002:0002af54       $chain$3$?hb_aat_layout_position@@YAXPEBUhb_ot_shape_plan_t@@PEAUhb_font_t@@PEAUhb_buffer_t@@@Z 00000001800d5f54     hb-aat-layout.obj
 0002:0002af74       $chain$4$?hb_aat_layout_position@@YAXPEBUhb_ot_shape_plan_t@@PEAUhb_font_t@@PEAUhb_buffer_t@@@Z 00000001800d5f74     hb-aat-layout.obj
 0002:0002af88       $chain$6$?hb_aat_layout_position@@YAXPEBUhb_ot_shape_plan_t@@PEAUhb_font_t@@PEAUhb_buffer_t@@@Z 00000001800d5f88     hb-aat-layout.obj
 0002:0002afa0       $chain$7$?hb_aat_layout_position@@YAXPEBUhb_ot_shape_plan_t@@PEAUhb_font_t@@PEAUhb_buffer_t@@@Z 00000001800d5fa0     hb-aat-layout.obj
 0002:0002afb4       $chain$8$?hb_aat_layout_position@@YAXPEBUhb_ot_shape_plan_t@@PEAUhb_font_t@@PEAUhb_buffer_t@@@Z 00000001800d5fb4     hb-aat-layout.obj
 0002:0002afc4       $chain$9$?hb_aat_layout_position@@YAXPEBUhb_ot_shape_plan_t@@PEAUhb_font_t@@PEAUhb_buffer_t@@@Z 00000001800d5fc4     hb-aat-layout.obj
 0002:0002afd4       $unwind$?hb_aat_layout_track@@YAXPEBUhb_ot_shape_plan_t@@PEAUhb_font_t@@PEAUhb_buffer_t@@@Z 00000001800d5fd4     hb-aat-layout.obj
 0002:0002afec       $unwind$??$dispatch@U?$Rule@USmallTypes@Layout@OT@@@OT@@$$V@hb_sanitize_context_t@@QEAA_NAEBU?$Rule@USmallTypes@Layout@OT@@@OT@@@Z 00000001800d5fec     hb-aat-layout.obj
 0002:0002afec       $unwind$?sanitize@?$KerxSubTableFormat2@UKerxSubTableHeader@AAT@@@AAT@@QEBA_NPEAUhb_sanitize_context_t@@@Z 00000001800d5fec     hb-aat-layout.obj
 0002:0002afec       $unwind$?sanitize_shallow@?$ArrayOf@U?$IntType@E$00@OT@@U?$IntType@G$01@2@@OT@@QEBA_NPEAUhb_sanitize_context_t@@@Z 00000001800d5fec     hb-aat-layout.obj
 0002:0002afec       $unwind$?sanitize_shallow@?$ArrayOf@U?$RangeRecord@USmallTypes@Layout@OT@@@Common@Layout@OT@@U?$IntType@G$01@4@@OT@@QEBA_NPEAUhb_sanitize_context_t@@@Z 00000001800d5fec     hb-aat-layout.obj
 0002:0002afec       $unwind$?sanitize_shallow@?$ArrayOf@U?$Record@UFeature@OT@@@OT@@U?$IntType@G$01@2@@OT@@QEBA_NPEAUhb_sanitize_context_t@@@Z 00000001800d5fec     hb-aat-layout.obj
 0002:0002afec       $unwind$?sanitize_shallow@?$ArrayOf@U?$Record@ULangSys@OT@@@OT@@U?$IntType@G$01@2@@OT@@QEBA_NPEAUhb_sanitize_context_t@@@Z 00000001800d5fec     hb-aat-layout.obj
 0002:0002afec       $unwind$?sanitize_shallow@?$ArrayOf@U?$Record@UScript@OT@@@OT@@U?$IntType@G$01@2@@OT@@QEBA_NPEAUhb_sanitize_context_t@@@Z 00000001800d5fec     hb-aat-layout.obj
 0002:0002afec       $unwind$?sanitize_shallow@?$ArrayOf@UFeatureTableSubstitutionRecord@OT@@U?$IntType@G$01@2@@OT@@QEBA_NPEAUhb_sanitize_context_t@@@Z 00000001800d5fec     hb-aat-layout.obj
 0002:0002afec       $unwind$?sanitize_shallow@?$HeadlessArrayOf@UHBGlyphID16@OT@@U?$IntType@G$01@2@@OT@@AEBA_NPEAUhb_sanitize_context_t@@@Z 00000001800d5fec     hb-aat-layout.obj
 0002:0002afec       $unwind$?sanitize_shallow@?$ArrayOf@U?$IntType@E$00@OT@@U?$IntType@I$03@2@@OT@@QEBA_NPEAUhb_sanitize_context_t@@@Z 00000001800d5fec     hb-face.obj
 0002:0002afec       $unwind$?sanitize_shallow@?$ArrayOf@UCmapSubtableLongGroup@OT@@U?$IntType@I$03@2@@OT@@QEBA_NPEAUhb_sanitize_context_t@@@Z 00000001800d5fec     hb-face.obj
 0002:0002afec       $unwind$?sanitize_shallow@?$ArrayOf@UTableRecord@OT@@U?$BinSearchHeader@U?$IntType@G$01@OT@@@2@@OT@@QEBA_NPEAUhb_sanitize_context_t@@@Z 00000001800d5fec     hb-face.obj
 0002:0002afec       $unwind$?sanitize_shallow@?$ArrayOf@U?$NoVariable@UColorStop@OT@@@OT@@U?$IntType@G$01@2@@OT@@QEBA_NPEAUhb_sanitize_context_t@@@Z 00000001800d5fec     hb-ot-color.obj
 0002:0002afec       $unwind$?sanitize_shallow@?$ArrayOf@U?$Variable@UColorStop@OT@@@OT@@U?$IntType@G$01@2@@OT@@QEBA_NPEAUhb_sanitize_context_t@@@Z 00000001800d5fec     hb-ot-color.obj
 0002:0002afec       $unwind$?sanitize_shallow@?$ArrayOf@UBaseGlyphPaintRecord@OT@@U?$IntType@I$03@2@@OT@@QEBA_NPEAUhb_sanitize_context_t@@@Z 00000001800d5fec     hb-ot-color.obj
 0002:0002afec       $unwind$?sanitize_shallow@?$ArrayOf@UBitmapSizeTable@OT@@U?$IntType@I$03@2@@OT@@QEBA_NPEAUhb_sanitize_context_t@@@Z 00000001800d5fec     hb-ot-color.obj
 0002:0002afec       $unwind$?sanitize_shallow@?$ArrayOf@U?$FDSelect3_4_Range@U?$IntType@I$03@OT@@U?$IntType@G$01@2@@CFF@@U?$IntType@I$03@OT@@@OT@@QEBA_NPEAUhb_sanitize_context_t@@@Z 00000001800d5fec     hb-ot-font.obj
 0002:0002afec       $unwind$?sanitize@?$KerxSubTableFormat2@UKernAATSubTableHeader@OT@@@AAT@@QEBA_NPEAUhb_sanitize_context_t@@@Z 00000001800d5fec     hb-ot-layout.obj
 0002:0002afec       $unwind$?sanitize@?$KerxSubTableFormat2@UKernOTSubTableHeader@OT@@@AAT@@QEBA_NPEAUhb_sanitize_context_t@@@Z 00000001800d5fec     hb-ot-layout.obj
 0002:0002afec       $unwind$?sanitize_shallow@?$ArrayOf@UKernPair@AAT@@U?$BinSearchHeader@U?$IntType@G$01@OT@@@OT@@@OT@@QEBA_NPEAUhb_sanitize_context_t@@@Z 00000001800d5fec     hb-ot-layout.obj
 0002:0002b004       $unwind$?get_coverage@?$CoverageFormat2_4@USmallTypes@Layout@OT@@@Common@Layout@OT@@AEBAII@Z 00000001800d6004     hb-aat-layout.obj
 0002:0002b004       $unwind$?interpolate_at@TrackTableEntry@AAT@@QEBAMIMPEBXU?$hb_array_t@$$CBU?$HBFixed@U?$IntType@H$03@OT@@$0BA@@OT@@@@@Z 00000001800d6004     hb-aat-layout.obj
 0002:0002b004       $unwind$?fasthash32@@YAIPEBX_KI@Z 00000001800d6004     hb-face-builder.obj
 0002:0002b004       $unwind$??$bsearch@I@?$SortedArrayOf@UCmapSubtableLongGroup@OT@@U?$IntType@I$03@2@@OT@@QEBAAEBUCmapSubtableLongGroup@1@AEBIAEBU21@@Z 00000001800d6004     hb-face.obj
 0002:0002b004       $unwind$?group_get_glyph@CmapSubtableFormat12@OT@@SAIAEBUCmapSubtableLongGroup@2@I@Z 00000001800d6004     hb-face.obj
 0002:0002b004       $unwind$?fetch_item@?$hb_hashmap_t@II$00@@QEBAPEAUitem_t@1@AEBII@Z 00000001800d6004     hb-map.obj
 0002:0002b004       $unwind$?hlineto@?$path_procs_t@Ucff1_path_procs_extents_t@@Ucff1_cs_interp_env_t@CFF@@Ucff1_extents_param_t@@@CFF@@SAXAEAUcff1_cs_interp_env_t@2@AEAUcff1_extents_param_t@@@Z 00000001800d6004     hb-ot-cff1-table.obj
 0002:0002b004       $unwind$?vlineto@?$path_procs_t@Ucff1_path_procs_extents_t@@Ucff1_cs_interp_env_t@CFF@@Ucff1_extents_param_t@@@CFF@@SAXAEAUcff1_cs_interp_env_t@2@AEAUcff1_extents_param_t@@@Z 00000001800d6004     hb-ot-cff1-table.obj
 0002:0002b004       $unwind$?find_table@IndexSubtableArray@OT@@QEBAPEBUIndexSubtableRecord@2@II@Z 00000001800d6004     hb-ot-color.obj
 0002:0002b004       $unwind$?get_feature@GSUBGPOS@OT@@QEBAAEBUFeature@2@I@Z 00000001800d6004     hb-ot-layout.obj
 0002:0002b004       $unwind$?fasthash32@@YAIPEBX_KI@Z 00000001800d6004     hb-ot-shaper-arabic.obj
 0002:0002b010       $unwind$?get_class@ClassDef@OT@@QEBAII@Z 00000001800d6010     hb-aat-layout.obj
 0002:0002b010       $unwind$?get_population@Coverage@Common@Layout@OT@@QEBAIXZ 00000001800d6010     hb-aat-layout.obj
 0002:0002b010       $unwind$?get_face_count@OpenTypeFontFile@OT@@QEBAIXZ 00000001800d6010     hb-face.obj
 0002:0002b010       $unwind$?blend_deltas@?$cff2_cs_interp_env_t@Unumber_t@CFF@@@CFF@@QEBANU?$hb_array_t@$$CBUnumber_t@CFF@@@@@Z 00000001800d6010     hb-ot-cff2-table.obj
 0002:0002b010       $unwind$?_hb_ot_shape_fallback_mark_position_recategorize_marks@@YAXPEBUhb_ot_shape_plan_t@@PEAUhb_font_t@@PEAUhb_buffer_t@@@Z 00000001800d6010     hb-ot-shape-fallback.obj
 0002:0002b010       $unwind$?intersect@hb_bounds_t@@QEAAXAEBU1@@Z 00000001800d6010     hb-paint-extents.obj
 0002:0002b018       $chain$0$?get_population@Coverage@Common@Layout@OT@@QEBAIXZ 00000001800d6018     hb-aat-layout.obj
 0002:0002b02c       $chain$1$?get_population@Coverage@Common@Layout@OT@@QEBAIXZ 00000001800d602c     hb-aat-layout.obj
 0002:0002b03c       $unwind$??$dispatch@U?$ClassTable@U?$IntType@E$00@OT@@@AAT@@$$V@hb_sanitize_context_t@@QEAA_NAEBU?$ClassTable@U?$IntType@E$00@OT@@@AAT@@@Z 00000001800d603c     hb-aat-layout.obj
 0002:0002b03c       $unwind$??$dispatch@U?$Ligature@USmallTypes@Layout@OT@@@GSUB_impl@Layout@OT@@$$V@hb_sanitize_context_t@@QEAA_NAEBU?$Ligature@USmallTypes@Layout@OT@@@GSUB_impl@Layout@OT@@@Z 00000001800d603c     hb-aat-layout.obj
 0002:0002b03c       $unwind$??$dispatch@Uhb_sanitize_context_t@@$$V@SubstLookupSubTable@GSUB_impl@Layout@OT@@QEBA_NPEAUhb_sanitize_context_t@@I@Z 00000001800d603c     hb-aat-layout.obj
 0002:0002b03c       $unwind$?sanitize@FeatureParams@OT@@QEBA_NPEAUhb_sanitize_context_t@@I@Z 00000001800d603c     hb-aat-layout.obj
 0002:0002b03c       $unwind$?sanitize@GDEF@OT@@QEBA_NPEAUhb_sanitize_context_t@@@Z 00000001800d603c     hb-aat-layout.obj
 0002:0002b03c       $unwind$?sanitize@GSUB@Layout@OT@@QEBA_NPEAUhb_sanitize_context_t@@@Z 00000001800d603c     hb-aat-layout.obj
 0002:0002b03c       $unwind$?sanitize@LangSys@OT@@QEBA_NPEAUhb_sanitize_context_t@@PEBURecord_sanitize_closure_t@2@@Z 00000001800d603c     hb-aat-layout.obj
 0002:0002b03c       $unwind$?sanitize@?$_hea@Uhhea@OT@@@OT@@QEBA_NPEAUhb_sanitize_context_t@@@Z 00000001800d603c     hb-common.obj
 0002:0002b03c       $unwind$?sanitize@?$_hea@Uvhea@OT@@@OT@@QEBA_NPEAUhb_sanitize_context_t@@@Z 00000001800d603c     hb-common.obj
 0002:0002b03c       $unwind$?sanitize@head@OT@@QEBA_NPEAUhb_sanitize_context_t@@@Z 00000001800d603c     hb-common.obj
 0002:0002b03c       $unwind$?sanitize@OpenTypeOffsetTable@OT@@QEBA_NPEAUhb_sanitize_context_t@@@Z 00000001800d603c     hb-face.obj
 0002:0002b03c       $unwind$??$dispatch@U?$ColorLine@UNoVariable@OT@@@OT@@$$V@hb_sanitize_context_t@@QEAA_NAEBU?$ColorLine@UNoVariable@OT@@@OT@@@Z 00000001800d603c     hb-ot-color.obj
 0002:0002b03c       $unwind$??$dispatch@U?$ColorLine@UVariable@OT@@@OT@@$$V@hb_sanitize_context_t@@QEAA_NAEBU?$ColorLine@UVariable@OT@@@OT@@@Z 00000001800d603c     hb-ot-color.obj
 0002:0002b03c       $unwind$?sanitize@CBDT@OT@@QEBA_NPEAUhb_sanitize_context_t@@@Z 00000001800d603c     hb-ot-color.obj
 0002:0002b03c       $unwind$??$StructAtOffsetOrNull@U?$CFFIndex@U?$IntType@G$01@OT@@@OT@@$$V@CFF@@YAAEBU?$CFFIndex@U?$IntType@G$01@OT@@@OT@@PEBXHAEAUhb_sanitize_context_t@@@Z 00000001800d603c     hb-ot-font.obj
 0002:0002b03c       $unwind$??$StructAtOffsetOrNull@U?$Subrs@U?$IntType@G$01@OT@@@CFF@@$$V@CFF@@YAAEBU?$Subrs@U?$IntType@G$01@OT@@@0@PEBXHAEAUhb_sanitize_context_t@@@Z 00000001800d603c     hb-ot-font.obj
 0002:0002b03c       $unwind$??$StructAtOffsetOrNull@U?$Subrs@U?$IntType@I$03@OT@@@CFF@@$$V@CFF@@YAAEBU?$Subrs@U?$IntType@I$03@OT@@@0@PEBXHAEAUhb_sanitize_context_t@@@Z 00000001800d603c     hb-ot-font.obj
 0002:0002b03c       $unwind$??$StructAtOffsetOrNull@UCFF1StringIndex@CFF@@$$V@CFF@@YAAEBUCFF1StringIndex@0@PEBXHAEAUhb_sanitize_context_t@@@Z 00000001800d603c     hb-ot-font.obj
 0002:0002b03c       $unwind$?sanitize@VORG@OT@@QEBA_NPEAUhb_sanitize_context_t@@@Z 00000001800d603c     hb-ot-font.obj
 0002:0002b03c       $unwind$?sanitize@cff1@OT@@QEBA_NPEAUhb_sanitize_context_t@@@Z 00000001800d603c     hb-ot-font.obj
 0002:0002b03c       $unwind$?sanitize@cff2@OT@@QEBA_NPEAUhb_sanitize_context_t@@@Z 00000001800d603c     hb-ot-font.obj
 0002:0002b03c       $unwind$??$dispatch@U?$ClassTable@U?$IntType@G$01@OT@@@AAT@@$$V@hb_sanitize_context_t@@QEAA_NAEBU?$ClassTable@U?$IntType@G$01@OT@@@AAT@@@Z 00000001800d603c     hb-ot-layout.obj
 0002:0002b03c       $unwind$??$dispatch@Uhb_sanitize_context_t@@$$V@PosLookupSubTable@GPOS_impl@Layout@OT@@QEBA_NPEAUhb_sanitize_context_t@@I@Z 00000001800d603c     hb-ot-layout.obj
 0002:0002b03c       $unwind$?get_kerning@?$KerxSubTableFormat2@UKernAATSubTableHeader@OT@@@AAT@@QEBAHIIPEAUhb_aat_apply_context_t@2@@Z 00000001800d603c     hb-ot-layout.obj
 0002:0002b03c       $unwind$?get_kerning@?$KerxSubTableFormat2@UKernOTSubTableHeader@OT@@@AAT@@QEBAHIIPEAUhb_aat_apply_context_t@2@@Z 00000001800d603c     hb-ot-layout.obj
 0002:0002b03c       $unwind$?sanitize@GPOS@Layout@OT@@QEBA_NPEAUhb_sanitize_context_t@@@Z 00000001800d603c     hb-ot-layout.obj
 0002:0002b03c       $unwind$?sanitize@kern@OT@@QEBA_NPEAUhb_sanitize_context_t@@@Z 00000001800d603c     hb-ot-layout.obj
 0002:0002b048       $unwind$?sanitize@Feature@OT@@QEBA_NPEAUhb_sanitize_context_t@@PEBURecord_sanitize_closure_t@2@@Z 00000001800d6048     hb-aat-layout.obj
 0002:0002b060       $unwind$??$dispatch@UCoverage@Common@Layout@OT@@$$V@hb_sanitize_context_t@@QEAA_NAEBUCoverage@Common@Layout@OT@@@Z 00000001800d6060     hb-aat-layout.obj
 0002:0002b060       $unwind$??$dispatch@UVarData@OT@@$$V@hb_sanitize_context_t@@QEAA_NAEBUVarData@OT@@@Z 00000001800d6060     hb-aat-layout.obj
 0002:0002b060       $unwind$??$dispatch@UVarRegionList@OT@@$$V@hb_sanitize_context_t@@QEAA_NAEBUVarRegionList@OT@@@Z 00000001800d6060     hb-aat-layout.obj
 0002:0002b060       $unwind$?sanitize_shallow@?$OffsetTo@U?$AlternateSet@USmallTypes@Layout@OT@@@GSUB_impl@Layout@OT@@U?$IntType@G$01@4@X$00@OT@@QEBA_NPEAUhb_sanitize_context_t@@PEBX@Z 00000001800d6060     hb-aat-layout.obj
 0002:0002b060       $unwind$?sanitize_shallow@?$OffsetTo@U?$ArrayOf@UAnchor@AAT@@U?$IntType@I$03@OT@@@OT@@U?$IntType@G$01@2@X$0A@@OT@@QEBA_NPEAUhb_sanitize_context_t@@PEBX@Z 00000001800d6060     hb-aat-layout.obj
 0002:0002b060       $unwind$?sanitize_shallow@?$OffsetTo@U?$ChainRule@USmallTypes@Layout@OT@@@OT@@U?$IntType@G$01@2@X$00@OT@@QEBA_NPEAUhb_sanitize_context_t@@PEBX@Z 00000001800d6060     hb-aat-layout.obj
 0002:0002b060       $unwind$?sanitize_shallow@?$OffsetTo@U?$ChainRuleSet@USmallTypes@Layout@OT@@@OT@@U?$IntType@G$01@2@X$00@OT@@QEBA_NPEAUhb_sanitize_context_t@@PEBX@Z 00000001800d6060     hb-aat-layout.obj
 0002:0002b060       $unwind$?sanitize_shallow@?$OffsetTo@U?$ClassTable@U?$IntType@E$00@OT@@@AAT@@U?$IntType@G$01@OT@@X$0A@@OT@@QEBA_NPEAUhb_sanitize_context_t@@PEBX@Z 00000001800d6060     hb-aat-layout.obj
 0002:0002b060       $unwind$?sanitize_shallow@?$OffsetTo@U?$Ligature@USmallTypes@Layout@OT@@@GSUB_impl@Layout@OT@@U?$IntType@G$01@4@X$00@OT@@QEBA_NPEAUhb_sanitize_context_t@@PEBX@Z 00000001800d6060     hb-aat-layout.obj
 0002:0002b060       $unwind$?sanitize_shallow@?$OffsetTo@U?$LigatureSet@USmallTypes@Layout@OT@@@GSUB_impl@Layout@OT@@U?$IntType@G$01@4@X$00@OT@@QEBA_NPEAUhb_sanitize_context_t@@PEBX@Z 00000001800d6060     hb-aat-layout.obj
 0002:0002b060       $unwind$?sanitize_shallow@?$OffsetTo@U?$List16OfOffsetTo@USubstLookup@GSUB_impl@Layout@OT@@U?$IntType@G$01@4@@OT@@U?$IntType@G$01@2@X$00@OT@@QEBA_NPEAUhb_sanitize_context_t@@PEBX@Z 00000001800d6060     hb-aat-layout.obj
 0002:0002b060       $unwind$?sanitize_shallow@?$OffsetTo@U?$Lookup@U?$IntType@G$01@OT@@@AAT@@U?$IntType@I$03@OT@@X$0A@@OT@@QEBA_NPEAUhb_sanitize_context_t@@PEBX@Z 00000001800d6060     hb-aat-layout.obj
 0002:0002b060       $unwind$?sanitize_shallow@?$OffsetTo@U?$Lookup@U?$IntType@I$03@OT@@@AAT@@U?$IntType@I$03@OT@@X$0A@@OT@@QEBA_NPEAUhb_sanitize_context_t@@PEBX@Z 00000001800d6060     hb-aat-layout.obj
 0002:0002b060       $unwind$?sanitize_shallow@?$OffsetTo@U?$Lookup@U?$OffsetTo@U?$ArrayOf@UAnchor@AAT@@U?$IntType@I$03@OT@@@OT@@U?$IntType@G$01@2@X$0A@@OT@@@AAT@@U?$IntType@I$03@OT@@X$00@OT@@QEBA_NPEAUhb_sanitize_context_t@@PEBX@Z 00000001800d6060     hb-aat-layout.obj
 0002:0002b060       $unwind$?sanitize_shallow@?$OffsetTo@U?$Lookup@UHBGlyphID16@OT@@@AAT@@U?$IntType@G$01@OT@@X$0A@@OT@@QEBA_NPEAUhb_sanitize_context_t@@PEBX@Z 00000001800d6060     hb-aat-layout.obj
 0002:0002b060       $unwind$?sanitize_shallow@?$OffsetTo@U?$Lookup@UHBGlyphID16@OT@@@AAT@@U?$IntType@I$03@OT@@X$0A@@OT@@QEBA_NPEAUhb_sanitize_context_t@@PEBX@Z 00000001800d6060     hb-aat-layout.obj
 0002:0002b060       $unwind$?sanitize_shallow@?$OffsetTo@U?$RecordListOf@UFeature@OT@@@OT@@U?$IntType@G$01@2@X$00@OT@@QEBA_NPEAUhb_sanitize_context_t@@PEBX@Z 00000001800d6060     hb-aat-layout.obj
 0002:0002b060       $unwind$?sanitize_shallow@?$OffsetTo@U?$Rule@USmallTypes@Layout@OT@@@OT@@U?$IntType@G$01@2@X$00@OT@@QEBA_NPEAUhb_sanitize_context_t@@PEBX@Z 00000001800d6060     hb-aat-layout.obj
 0002:0002b060       $unwind$?sanitize_shallow@?$OffsetTo@U?$RuleSet@USmallTypes@Layout@OT@@@OT@@U?$IntType@G$01@2@X$00@OT@@QEBA_NPEAUhb_sanitize_context_t@@PEBX@Z 00000001800d6060     hb-aat-layout.obj
 0002:0002b060       $unwind$?sanitize_shallow@?$OffsetTo@U?$Sequence@USmallTypes@Layout@OT@@@GSUB_impl@Layout@OT@@U?$IntType@G$01@4@X$00@OT@@QEBA_NPEAUhb_sanitize_context_t@@PEBX@Z 00000001800d6060     hb-aat-layout.obj
 0002:0002b060       $unwind$?sanitize_shallow@?$OffsetTo@U?$UnsizedArrayOf@U?$HBFixed@U?$IntType@H$03@OT@@$0BA@@OT@@@OT@@U?$IntType@I$03@2@X$0A@@OT@@QEBA_NPEAUhb_sanitize_context_t@@PEBX@Z 00000001800d6060     hb-aat-layout.obj
 0002:0002b060       $unwind$?sanitize_shallow@?$OffsetTo@U?$UnsizedArrayOf@U?$IntType@E$00@OT@@@OT@@U?$IntType@I$03@2@X$0A@@OT@@QEBA_NPEAUhb_sanitize_context_t@@PEBX@Z 00000001800d6060     hb-aat-layout.obj
 0002:0002b060       $unwind$?sanitize_shallow@?$OffsetTo@U?$UnsizedArrayOf@U?$IntType@F$01@OT@@@OT@@U?$IntType@G$01@2@X$0A@@OT@@QEBA_NPEAUhb_sanitize_context_t@@PEBX@Z 00000001800d6060     hb-aat-layout.obj
 0002:0002b060       $unwind$?sanitize_shallow@?$OffsetTo@U?$UnsizedArrayOf@U?$IntType@G$01@OT@@@OT@@U?$IntType@G$01@2@X$0A@@OT@@QEBA_NPEAUhb_sanitize_context_t@@PEBX@Z 00000001800d6060     hb-aat-layout.obj
 0002:0002b060       $unwind$?sanitize_shallow@?$OffsetTo@U?$UnsizedArrayOf@U?$IntType@I$03@OT@@@OT@@U?$IntType@G$01@2@X$0A@@OT@@QEBA_NPEAUhb_sanitize_context_t@@PEBX@Z 00000001800d6060     hb-aat-layout.obj
 0002:0002b060       $unwind$?sanitize_shallow@?$OffsetTo@U?$UnsizedArrayOf@U?$OffsetTo@U?$ArrayOf@UAnchor@AAT@@U?$IntType@I$03@OT@@@OT@@U?$IntType@G$01@2@X$0A@@OT@@@OT@@U?$IntType@G$01@2@X$0A@@OT@@QEBA_NPEAUhb_sanitize_context_t@@PEBX@Z 00000001800d6060     hb-aat-layout.obj
 0002:0002b060       $unwind$?sanitize_shallow@?$OffsetTo@U?$UnsizedArrayOf@UHBGlyphID16@OT@@@OT@@U?$IntType@G$01@2@X$0A@@OT@@QEBA_NPEAUhb_sanitize_context_t@@PEBX@Z 00000001800d6060     hb-aat-layout.obj
 0002:0002b060       $unwind$?sanitize_shallow@?$OffsetTo@U?$UnsizedListOfOffset16To@U?$Lookup@UHBGlyphID16@OT@@@AAT@@U?$IntType@G$01@OT@@X$0A@@OT@@U?$IntType@G$01@2@X$0A@@OT@@QEBA_NPEAUhb_sanitize_context_t@@PEBX@Z 00000001800d6060     hb-aat-layout.obj
 0002:0002b060       $unwind$?sanitize_shallow@?$OffsetTo@U?$UnsizedListOfOffset16To@U?$Lookup@UHBGlyphID16@OT@@@AAT@@U?$IntType@I$03@OT@@X$0A@@OT@@U?$IntType@I$03@2@X$0A@@OT@@QEBA_NPEAUhb_sanitize_context_t@@PEBX@Z 00000001800d6060     hb-aat-layout.obj
 0002:0002b060       $unwind$?sanitize_shallow@?$OffsetTo@UAttachList@OT@@U?$IntType@G$01@2@X$00@OT@@QEBA_NPEAUhb_sanitize_context_t@@PEBX@Z 00000001800d6060     hb-aat-layout.obj
 0002:0002b060       $unwind$?sanitize_shallow@?$OffsetTo@UAttachPoint@OT@@U?$IntType@G$01@2@X$00@OT@@QEBA_NPEAUhb_sanitize_context_t@@PEBX@Z 00000001800d6060     hb-aat-layout.obj
 0002:0002b060       $unwind$?sanitize_shallow@?$OffsetTo@UCaretValue@OT@@U?$IntType@G$01@2@X$00@OT@@QEBA_NPEAUhb_sanitize_context_t@@PEBX@Z 00000001800d6060     hb-aat-layout.obj
 0002:0002b060       $unwind$?sanitize_shallow@?$OffsetTo@UClassDef@OT@@U?$IntType@G$01@2@X$00@OT@@QEBA_NPEAUhb_sanitize_context_t@@PEBX@Z 00000001800d6060     hb-aat-layout.obj
 0002:0002b060       $unwind$?sanitize_shallow@?$OffsetTo@UCondition@OT@@U?$IntType@I$02@2@X$00@OT@@QEBA_NPEAUhb_sanitize_context_t@@PEBX@Z 00000001800d6060     hb-aat-layout.obj
 0002:0002b060       $unwind$?sanitize_shallow@?$OffsetTo@UCondition@OT@@U?$IntType@I$03@2@X$00@OT@@QEBA_NPEAUhb_sanitize_context_t@@PEBX@Z 00000001800d6060     hb-aat-layout.obj
 0002:0002b060       $unwind$?sanitize_shallow@?$OffsetTo@UConditionSet@OT@@U?$IntType@I$03@2@X$00@OT@@QEBA_NPEAUhb_sanitize_context_t@@PEBX@Z 00000001800d6060     hb-aat-layout.obj
 0002:0002b060       $unwind$?sanitize_shallow@?$OffsetTo@UCoverage@Common@Layout@OT@@U?$IntType@G$01@4@X$00@OT@@QEBA_NPEAUhb_sanitize_context_t@@PEBX@Z 00000001800d6060     hb-aat-layout.obj
 0002:0002b060       $unwind$?sanitize_shallow@?$OffsetTo@UCoverage@Common@Layout@OT@@U?$IntType@I$03@4@X$00@OT@@QEBA_NPEAUhb_sanitize_context_t@@PEBX@Z 00000001800d6060     hb-aat-layout.obj
 0002:0002b060       $unwind$?sanitize_shallow@?$OffsetTo@UDevice@OT@@U?$IntType@G$01@2@X$00@OT@@QEBA_NPEAUhb_sanitize_context_t@@PEBX@Z 00000001800d6060     hb-aat-layout.obj
 0002:0002b060       $unwind$?sanitize_shallow@?$OffsetTo@UFeature@OT@@U?$IntType@G$01@2@X$00@OT@@QEBA_NPEAUhb_sanitize_context_t@@PEBX@Z 00000001800d6060     hb-aat-layout.obj
 0002:0002b060       $unwind$?sanitize_shallow@?$OffsetTo@UFeature@OT@@U?$IntType@I$03@2@X$00@OT@@QEBA_NPEAUhb_sanitize_context_t@@PEBX@Z 00000001800d6060     hb-aat-layout.obj
 0002:0002b060       $unwind$?sanitize_shallow@?$OffsetTo@UFeatureParams@OT@@U?$IntType@G$01@2@X$00@OT@@QEBA_NPEAUhb_sanitize_context_t@@PEBX@Z 00000001800d6060     hb-aat-layout.obj
 0002:0002b060       $unwind$?sanitize_shallow@?$OffsetTo@UFeatureTableSubstitution@OT@@U?$IntType@I$03@2@X$00@OT@@QEBA_NPEAUhb_sanitize_context_t@@PEBX@Z 00000001800d6060     hb-aat-layout.obj
 0002:0002b060       $unwind$?sanitize_shallow@?$OffsetTo@UFeatureVariations@OT@@U?$IntType@I$03@2@X$00@OT@@QEBA_NPEAUhb_sanitize_context_t@@PEBX@Z 00000001800d6060     hb-aat-layout.obj
 0002:0002b060       $unwind$?sanitize_shallow@?$OffsetTo@UItemVariationStore@OT@@U?$IntType@I$03@2@X$00@OT@@QEBA_NPEAUhb_sanitize_context_t@@PEBX@Z 00000001800d6060     hb-aat-layout.obj
 0002:0002b060       $unwind$?sanitize_shallow@?$OffsetTo@ULangSys@OT@@U?$IntType@G$01@2@X$00@OT@@QEBA_NPEAUhb_sanitize_context_t@@PEBX@Z 00000001800d6060     hb-aat-layout.obj
 0002:0002b060       $unwind$?sanitize_shallow@?$OffsetTo@ULigCaretList@OT@@U?$IntType@G$01@2@X$00@OT@@QEBA_NPEAUhb_sanitize_context_t@@PEBX@Z 00000001800d6060     hb-aat-layout.obj
 0002:0002b060       $unwind$?sanitize_shallow@?$OffsetTo@ULigGlyph@OT@@U?$IntType@G$01@2@X$00@OT@@QEBA_NPEAUhb_sanitize_context_t@@PEBX@Z 00000001800d6060     hb-aat-layout.obj
 0002:0002b060       $unwind$?sanitize_shallow@?$OffsetTo@UMarkGlyphSets@OT@@U?$IntType@G$01@2@X$00@OT@@QEBA_NPEAUhb_sanitize_context_t@@PEBX@Z 00000001800d6060     hb-aat-layout.obj
 0002:0002b060       $unwind$?sanitize_shallow@?$OffsetTo@URecordListOfScript@OT@@U?$IntType@G$01@2@X$00@OT@@QEBA_NPEAUhb_sanitize_context_t@@PEBX@Z 00000001800d6060     hb-aat-layout.obj
 0002:0002b060       $unwind$?sanitize_shallow@?$OffsetTo@UScript@OT@@U?$IntType@G$01@2@X$00@OT@@QEBA_NPEAUhb_sanitize_context_t@@PEBX@Z 00000001800d6060     hb-aat-layout.obj
 0002:0002b060       $unwind$?sanitize_shallow@?$OffsetTo@USubstLookup@GSUB_impl@Layout@OT@@U?$IntType@G$01@4@X$00@OT@@QEBA_NPEAUhb_sanitize_context_t@@PEBX@Z 00000001800d6060     hb-aat-layout.obj
 0002:0002b060       $unwind$?sanitize_shallow@?$OffsetTo@USubstLookupSubTable@GSUB_impl@Layout@OT@@U?$IntType@G$01@4@X$00@OT@@QEBA_NPEAUhb_sanitize_context_t@@PEBX@Z 00000001800d6060     hb-aat-layout.obj
 0002:0002b060       $unwind$?sanitize_shallow@?$OffsetTo@UTrackData@AAT@@U?$IntType@G$01@OT@@X$00@OT@@QEBA_NPEAUhb_sanitize_context_t@@PEBX@Z 00000001800d6060     hb-aat-layout.obj
 0002:0002b060       $unwind$?sanitize_shallow@?$OffsetTo@UVarData@OT@@U?$IntType@I$03@2@X$00@OT@@QEBA_NPEAUhb_sanitize_context_t@@PEBX@Z 00000001800d6060     hb-aat-layout.obj
 0002:0002b060       $unwind$?sanitize_shallow@?$OffsetTo@UVarRegionList@OT@@U?$IntType@I$03@2@X$00@OT@@QEBA_NPEAUhb_sanitize_context_t@@PEBX@Z 00000001800d6060     hb-aat-layout.obj
 0002:0002b060       $unwind$?sanitize_shallow@?$VarSizedBinSearchArrayOf@U?$LookupSegmentArray@U?$IntType@G$01@OT@@@AAT@@@OT@@AEBA_NPEAUhb_sanitize_context_t@@@Z 00000001800d6060     hb-aat-layout.obj
 0002:0002b060       $unwind$?sanitize_shallow@?$VarSizedBinSearchArrayOf@U?$LookupSegmentArray@U?$IntType@I$03@OT@@@AAT@@@OT@@AEBA_NPEAUhb_sanitize_context_t@@@Z 00000001800d6060     hb-aat-layout.obj
 0002:0002b060       $unwind$?sanitize_shallow@?$VarSizedBinSearchArrayOf@U?$LookupSegmentArray@U?$OffsetTo@U?$ArrayOf@UAnchor@AAT@@U?$IntType@I$03@OT@@@OT@@U?$IntType@G$01@2@X$0A@@OT@@@AAT@@@OT@@AEBA_NPEAUhb_sanitize_context_t@@@Z 00000001800d6060     hb-aat-layout.obj
 0002:0002b060       $unwind$?sanitize_shallow@?$VarSizedBinSearchArrayOf@U?$LookupSegmentArray@UHBGlyphID16@OT@@@AAT@@@OT@@AEBA_NPEAUhb_sanitize_context_t@@@Z 00000001800d6060     hb-aat-layout.obj
 0002:0002b060       $unwind$?sanitize_shallow@?$VarSizedBinSearchArrayOf@U?$LookupSegmentSingle@U?$IntType@G$01@OT@@@AAT@@@OT@@AEBA_NPEAUhb_sanitize_context_t@@@Z 00000001800d6060     hb-aat-layout.obj
 0002:0002b060       $unwind$?sanitize_shallow@?$VarSizedBinSearchArrayOf@U?$LookupSegmentSingle@U?$IntType@I$03@OT@@@AAT@@@OT@@AEBA_NPEAUhb_sanitize_context_t@@@Z 00000001800d6060     hb-aat-layout.obj
 0002:0002b060       $unwind$?sanitize_shallow@?$VarSizedBinSearchArrayOf@U?$LookupSegmentSingle@U?$OffsetTo@U?$ArrayOf@UAnchor@AAT@@U?$IntType@I$03@OT@@@OT@@U?$IntType@G$01@2@X$0A@@OT@@@AAT@@@OT@@AEBA_NPEAUhb_sanitize_context_t@@@Z 00000001800d6060     hb-aat-layout.obj
 0002:0002b060       $unwind$?sanitize_shallow@?$VarSizedBinSearchArrayOf@U?$LookupSegmentSingle@UHBGlyphID16@OT@@@AAT@@@OT@@AEBA_NPEAUhb_sanitize_context_t@@@Z 00000001800d6060     hb-aat-layout.obj
 0002:0002b060       $unwind$?sanitize_shallow@?$VarSizedBinSearchArrayOf@U?$LookupSingle@U?$IntType@G$01@OT@@@AAT@@@OT@@AEBA_NPEAUhb_sanitize_context_t@@@Z 00000001800d6060     hb-aat-layout.obj
 0002:0002b060       $unwind$?sanitize_shallow@?$VarSizedBinSearchArrayOf@U?$LookupSingle@U?$IntType@I$03@OT@@@AAT@@@OT@@AEBA_NPEAUhb_sanitize_context_t@@@Z 00000001800d6060     hb-aat-layout.obj
 0002:0002b060       $unwind$?sanitize_shallow@?$VarSizedBinSearchArrayOf@U?$LookupSingle@U?$OffsetTo@U?$ArrayOf@UAnchor@AAT@@U?$IntType@I$03@OT@@@OT@@U?$IntType@G$01@2@X$0A@@OT@@@AAT@@@OT@@AEBA_NPEAUhb_sanitize_context_t@@@Z 00000001800d6060     hb-aat-layout.obj
 0002:0002b060       $unwind$?sanitize_shallow@?$VarSizedBinSearchArrayOf@U?$LookupSingle@UHBGlyphID16@OT@@@AAT@@@OT@@AEBA_NPEAUhb_sanitize_context_t@@@Z 00000001800d6060     hb-aat-layout.obj
 0002:0002b060       $unwind$?sanitize@HVARVVAR@OT@@QEBA_NPEAUhb_sanitize_context_t@@@Z 00000001800d6060     hb-common.obj
 0002:0002b060       $unwind$?sanitize_shallow@?$OffsetTo@U?$UnsizedArrayOf@U?$HBFixed@U?$IntType@F$01@OT@@$0O@@OT@@@OT@@U?$IntType@I$03@2@X$0A@@OT@@QEBA_NPEAUhb_sanitize_context_t@@PEBX@Z 00000001800d6060     hb-common.obj
 0002:0002b060       $unwind$?sanitize_shallow@?$OffsetTo@UDeltaSetIndexMap@OT@@U?$IntType@I$03@2@X$00@OT@@QEBA_NPEAUhb_sanitize_context_t@@PEBX@Z 00000001800d6060     hb-common.obj
 0002:0002b060       $unwind$?sanitize_shallow@?$OffsetTo@U?$ArrayOf@U?$IntType@E$00@OT@@U?$IntType@I$03@2@@OT@@U?$IntType@I$02@2@X$0A@@OT@@QEBA_NPEAUhb_sanitize_context_t@@PEBX@Z 00000001800d6060     hb-face.obj
 0002:0002b060       $unwind$?sanitize_shallow@?$OffsetTo@U?$ArrayOfM1@UResourceTypeRecord@OT@@U?$IntType@G$01@2@@OT@@U?$IntType@G$01@2@X$0A@@OT@@QEBA_NPEAUhb_sanitize_context_t@@PEBX@Z 00000001800d6060     hb-face.obj
 0002:0002b060       $unwind$?sanitize_shallow@?$OffsetTo@U?$UnsizedArrayOf@UResourceRecord@OT@@@OT@@U?$IntType@G$01@2@X$0A@@OT@@QEBA_NPEAUhb_sanitize_context_t@@PEBX@Z 00000001800d6060     hb-face.obj
 0002:0002b060       $unwind$?sanitize_shallow@?$OffsetTo@UCmapSubtable@OT@@U?$IntType@I$03@2@X$00@OT@@QEBA_NPEAUhb_sanitize_context_t@@PEBX@Z 00000001800d6060     hb-face.obj
 0002:0002b060       $unwind$?sanitize_shallow@?$OffsetTo@UDefaultUVS@OT@@U?$IntType@I$03@2@X$00@OT@@QEBA_NPEAUhb_sanitize_context_t@@PEBX@Z 00000001800d6060     hb-face.obj
 0002:0002b060       $unwind$?sanitize_shallow@?$OffsetTo@UNonDefaultUVS@OT@@U?$IntType@I$03@2@X$00@OT@@QEBA_NPEAUhb_sanitize_context_t@@PEBX@Z 00000001800d6060     hb-face.obj
 0002:0002b060       $unwind$?sanitize_shallow@?$OffsetTo@UOpenTypeOffsetTable@OT@@U?$IntType@I$03@2@X$00@OT@@QEBA_NPEAUhb_sanitize_context_t@@PEBX@Z 00000001800d6060     hb-face.obj
 0002:0002b060       $unwind$?sanitize_shallow@?$OffsetTo@UResourceMap@OT@@U?$IntType@I$03@2@X$0A@@OT@@QEBA_NPEAUhb_sanitize_context_t@@PEBX@Z 00000001800d6060     hb-face.obj
 0002:0002b060       $unwind$?sanitize@COLR@OT@@QEBA_NPEAUhb_sanitize_context_t@@@Z 00000001800d6060     hb-ot-color.obj
 0002:0002b060       $unwind$?sanitize@PaintRotate@OT@@QEBA_NPEAUhb_sanitize_context_t@@@Z 00000001800d6060     hb-ot-color.obj
 0002:0002b060       $unwind$?sanitize@PaintRotateAroundCenter@OT@@QEBA_NPEAUhb_sanitize_context_t@@@Z 00000001800d6060     hb-ot-color.obj
 0002:0002b060       $unwind$?sanitize@PaintScale@OT@@QEBA_NPEAUhb_sanitize_context_t@@@Z 00000001800d6060     hb-ot-color.obj
 0002:0002b060       $unwind$?sanitize@PaintScaleAroundCenter@OT@@QEBA_NPEAUhb_sanitize_context_t@@@Z 00000001800d6060     hb-ot-color.obj
 0002:0002b060       $unwind$?sanitize@PaintScaleUniform@OT@@QEBA_NPEAUhb_sanitize_context_t@@@Z 00000001800d6060     hb-ot-color.obj
 0002:0002b060       $unwind$?sanitize@PaintScaleUniformAroundCenter@OT@@QEBA_NPEAUhb_sanitize_context_t@@@Z 00000001800d6060     hb-ot-color.obj
 0002:0002b060       $unwind$?sanitize@PaintSkew@OT@@QEBA_NPEAUhb_sanitize_context_t@@@Z 00000001800d6060     hb-ot-color.obj
 0002:0002b060       $unwind$?sanitize@PaintSkewAroundCenter@OT@@QEBA_NPEAUhb_sanitize_context_t@@@Z 00000001800d6060     hb-ot-color.obj
 0002:0002b060       $unwind$?sanitize@PaintTranslate@OT@@QEBA_NPEAUhb_sanitize_context_t@@@Z 00000001800d6060     hb-ot-color.obj
 0002:0002b060       $unwind$?sanitize_shallow@?$OffsetTo@U?$ColorLine@UNoVariable@OT@@@OT@@U?$IntType@I$02@2@X$00@OT@@QEBA_NPEAUhb_sanitize_context_t@@PEBX@Z 00000001800d6060     hb-ot-color.obj
 0002:0002b060       $unwind$?sanitize_shallow@?$OffsetTo@U?$ColorLine@UVariable@OT@@@OT@@U?$IntType@I$02@2@X$00@OT@@QEBA_NPEAUhb_sanitize_context_t@@PEBX@Z 00000001800d6060     hb-ot-color.obj
 0002:0002b060       $unwind$?sanitize_shallow@?$OffsetTo@U?$NoVariable@UAffine2x3@OT@@@OT@@U?$IntType@I$02@2@X$00@OT@@QEBA_NPEAUhb_sanitize_context_t@@PEBX@Z 00000001800d6060     hb-ot-color.obj
 0002:0002b060       $unwind$?sanitize_shallow@?$OffsetTo@U?$Variable@UAffine2x3@OT@@@OT@@U?$IntType@I$02@2@X$00@OT@@QEBA_NPEAUhb_sanitize_context_t@@PEBX@Z 00000001800d6060     hb-ot-color.obj
 0002:0002b060       $unwind$?sanitize_shallow@?$OffsetTo@UBaseGlyphList@OT@@U?$IntType@I$03@2@X$00@OT@@QEBA_NPEAUhb_sanitize_context_t@@PEBX@Z 00000001800d6060     hb-ot-color.obj
 0002:0002b060       $unwind$?sanitize_shallow@?$OffsetTo@UClipBox@OT@@U?$IntType@I$02@2@X$00@OT@@QEBA_NPEAUhb_sanitize_context_t@@PEBX@Z 00000001800d6060     hb-ot-color.obj
 0002:0002b060       $unwind$?sanitize_shallow@?$OffsetTo@UClipList@OT@@U?$IntType@I$03@2@X$00@OT@@QEBA_NPEAUhb_sanitize_context_t@@PEBX@Z 00000001800d6060     hb-ot-color.obj
 0002:0002b060       $unwind$?sanitize_shallow@?$OffsetTo@UIndexSubtable@OT@@U?$IntType@I$03@2@X$00@OT@@QEBA_NPEAUhb_sanitize_context_t@@PEBX@Z 00000001800d6060     hb-ot-color.obj
 0002:0002b060       $unwind$?sanitize_shallow@?$OffsetTo@UIndexSubtableArray@OT@@U?$IntType@I$03@2@X$0A@@OT@@QEBA_NPEAUhb_sanitize_context_t@@PEBX@Z 00000001800d6060     hb-ot-color.obj
 0002:0002b060       $unwind$?sanitize_shallow@?$OffsetTo@ULayerList@OT@@U?$IntType@I$03@2@X$00@OT@@QEBA_NPEAUhb_sanitize_context_t@@PEBX@Z 00000001800d6060     hb-ot-color.obj
 0002:0002b060       $unwind$?sanitize_shallow@?$OffsetTo@UPaint@OT@@U?$IntType@I$02@2@X$00@OT@@QEBA_NPEAUhb_sanitize_context_t@@PEBX@Z 00000001800d6060     hb-ot-color.obj
 0002:0002b060       $unwind$?sanitize_shallow@?$OffsetTo@UPaint@OT@@U?$IntType@I$03@2@X$00@OT@@QEBA_NPEAUhb_sanitize_context_t@@PEBX@Z 00000001800d6060     hb-ot-color.obj
 0002:0002b060       $unwind$?sanitize_shallow@?$OffsetTo@USBIXStrike@OT@@U?$IntType@I$03@2@X$00@OT@@QEBA_NPEAUhb_sanitize_context_t@@PEBX@Z 00000001800d6060     hb-ot-color.obj
 0002:0002b060       $unwind$?sanitize@post@OT@@QEBA_NPEAUhb_sanitize_context_t@@@Z 00000001800d6060     hb-ot-font.obj
 0002:0002b060       $unwind$?sanitize_shallow@?$OffsetTo@U?$ClassTable@U?$IntType@G$01@OT@@@AAT@@U?$IntType@G$01@OT@@X$0A@@OT@@QEBA_NPEAUhb_sanitize_context_t@@PEBX@Z 00000001800d6060     hb-ot-layout.obj
 0002:0002b060       $unwind$?sanitize_shallow@?$OffsetTo@U?$List16OfOffsetTo@UPosLookup@GPOS_impl@Layout@OT@@U?$IntType@G$01@4@@OT@@U?$IntType@G$01@2@X$00@OT@@QEBA_NPEAUhb_sanitize_context_t@@PEBX@Z 00000001800d6060     hb-ot-layout.obj
 0002:0002b060       $unwind$?sanitize_shallow@?$OffsetTo@U?$PairSet@USmallTypes@Layout@OT@@@GPOS_impl@Layout@OT@@U?$IntType@G$01@4@X$00@OT@@QEBA_NPEAUhb_sanitize_context_t@@PEBX@Z 00000001800d6060     hb-ot-layout.obj
 0002:0002b060       $unwind$?sanitize_shallow@?$OffsetTo@UAnchor@GPOS_impl@Layout@OT@@U?$IntType@G$01@4@UAnchorMatrix@234@$00@OT@@QEBA_NPEAUhb_sanitize_context_t@@PEBUAnchorMatrix@GPOS_impl@Layout@2@@Z 00000001800d6060     hb-ot-layout.obj
 0002:0002b060       $unwind$?sanitize_shallow@?$OffsetTo@UAnchor@GPOS_impl@Layout@OT@@U?$IntType@G$01@4@UCursivePosFormat1@234@$00@OT@@QEBA_NPEAUhb_sanitize_context_t@@PEBUCursivePosFormat1@GPOS_impl@Layout@2@@Z 00000001800d6060     hb-ot-layout.obj
 0002:0002b060       $unwind$?sanitize_shallow@?$OffsetTo@UAnchor@GPOS_impl@Layout@OT@@U?$IntType@G$01@4@X$00@OT@@QEBA_NPEAUhb_sanitize_context_t@@PEBX@Z 00000001800d6060     hb-ot-layout.obj
 0002:0002b060       $unwind$?sanitize_shallow@?$OffsetTo@UAnchorMatrix@GPOS_impl@Layout@OT@@U?$IntType@G$01@4@X$00@OT@@QEBA_NPEAUhb_sanitize_context_t@@PEBX@Z 00000001800d6060     hb-ot-layout.obj
 0002:0002b060       $unwind$?sanitize_shallow@?$OffsetTo@UDevice@OT@@U?$IntType@G$01@2@UValueBase@GPOS_impl@Layout@2@$00@OT@@QEBA_NPEAUhb_sanitize_context_t@@PEBUValueBase@GPOS_impl@Layout@2@@Z 00000001800d6060     hb-ot-layout.obj
 0002:0002b060       $unwind$?sanitize_shallow@?$OffsetTo@ULigatureArray@GPOS_impl@Layout@OT@@U?$IntType@G$01@4@X$00@OT@@QEBA_NPEAUhb_sanitize_context_t@@PEBX@Z 00000001800d6060     hb-ot-layout.obj
 0002:0002b060       $unwind$?sanitize_shallow@?$OffsetTo@UMarkArray@GPOS_impl@Layout@OT@@U?$IntType@G$01@4@X$00@OT@@QEBA_NPEAUhb_sanitize_context_t@@PEBX@Z 00000001800d6060     hb-ot-layout.obj
 0002:0002b060       $unwind$?sanitize_shallow@?$OffsetTo@UPosLookup@GPOS_impl@Layout@OT@@U?$IntType@G$01@4@X$00@OT@@QEBA_NPEAUhb_sanitize_context_t@@PEBX@Z 00000001800d6060     hb-ot-layout.obj
 0002:0002b060       $unwind$?sanitize_shallow@?$OffsetTo@UPosLookupSubTable@GPOS_impl@Layout@OT@@U?$IntType@G$01@4@X$00@OT@@QEBA_NPEAUhb_sanitize_context_t@@PEBX@Z 00000001800d6060     hb-ot-layout.obj
 0002:0002b060       $unwind$?sanitize_shallow@?$OffsetTo@UItemVariationStore@OT@@U?$IntType@G$01@2@X$00@OT@@QEBA_NPEAUhb_sanitize_context_t@@PEBX@Z 00000001800d6060     hb-ot-metrics.obj
 0002:0002b060       $unwind$?sanitize_shallow@?$OffsetTo@U?$UnsizedArrayOf@UStatAxisRecord@OT@@@OT@@U?$IntType@I$03@2@X$0A@@OT@@QEBA_NPEAUhb_sanitize_context_t@@PEBX@Z 00000001800d6060     hb-ot-shape.obj
 0002:0002b060       $unwind$?sanitize_shallow@?$OffsetTo@UAxisValue@OT@@U?$IntType@G$01@2@X$00@OT@@QEBA_NPEAUhb_sanitize_context_t@@PEBX@Z 00000001800d6060     hb-ot-shape.obj
 0002:0002b060       $unwind$?sanitize_shallow@?$OffsetTo@UAxisValueOffsetArray@OT@@U?$IntType@I$03@2@X$0A@@OT@@QEBA_NPEAUhb_sanitize_context_t@@PEBX@Z 00000001800d6060     hb-ot-shape.obj
 0002:0002b070       $unwind$?sanitize@?$Chain@UExtendedTypes@AAT@@@AAT@@QEBA_NPEAUhb_sanitize_context_t@@I@Z 00000001800d6070     hb-aat-layout.obj
 0002:0002b070       $unwind$?sanitize@ContextFormat3@OT@@QEBA_NPEAUhb_sanitize_context_t@@@Z 00000001800d6070     hb-aat-layout.obj
 0002:0002b070       $unwind$?sanitize@Script@OT@@QEBA_NPEAUhb_sanitize_context_t@@PEBURecord_sanitize_closure_t@2@@Z 00000001800d6070     hb-aat-layout.obj
 0002:0002b070       $unwind$?sanitize@fvar@OT@@QEBA_NPEAUhb_sanitize_context_t@@@Z 00000001800d6070     hb-font.obj
 0002:0002b070       $unwind$?sanitize@?$KerxTable@UKernAAT@OT@@@AAT@@QEBA_NPEAUhb_sanitize_context_t@@@Z 00000001800d6070     hb-ot-layout.obj
 0002:0002b070       $unwind$?sanitize@?$KerxTable@UKernOT@OT@@@AAT@@QEBA_NPEAUhb_sanitize_context_t@@@Z 00000001800d6070     hb-ot-layout.obj
 0002:0002b070       $unwind$?sanitize@AnchorMatrix@GPOS_impl@Layout@OT@@QEBA_NPEAUhb_sanitize_context_t@@I@Z 00000001800d6070     hb-ot-layout.obj
 0002:0002b070       $unwind$?sanitize@SinglePosFormat1@GPOS_impl@Layout@OT@@QEBA_NPEAUhb_sanitize_context_t@@@Z 00000001800d6070     hb-ot-layout.obj
 0002:0002b08c       $chain$0$?get_class@ClassDef@OT@@QEBAII@Z 00000001800d608c     hb-aat-layout.obj
 0002:0002b0a0       $chain$1$?get_class@ClassDef@OT@@QEBAII@Z 00000001800d60a0     hb-aat-layout.obj
 0002:0002b0b0       $chain$1$?sanitize_shallow@?$UnsizedArrayOf@UVarRegionAxis@OT@@@OT@@QEBA_NPEAUhb_sanitize_context_t@@I@Z 00000001800d60b0     hb-aat-layout.obj
 0002:0002b0b0       $chain$1$?sanitize_shallow@?$UnsizedArrayOf@UBaseGlyphRecord@OT@@@OT@@QEBA_NPEAUhb_sanitize_context_t@@I@Z 00000001800d60b0     hb-ot-color.obj
 0002:0002b0b0       $chain$1$?sanitize_shallow@?$UnsizedArrayOf@UAxisValueRecord@OT@@@OT@@QEBA_NPEAUhb_sanitize_context_t@@I@Z 00000001800d60b0     hb-ot-shape.obj
 0002:0002b0c8       $chain$2$?sanitize_shallow@?$UnsizedArrayOf@UVarRegionAxis@OT@@@OT@@QEBA_NPEAUhb_sanitize_context_t@@I@Z 00000001800d60c8     hb-aat-layout.obj
 0002:0002b0c8       $chain$2$?sanitize_shallow@?$UnsizedArrayOf@UBaseGlyphRecord@OT@@@OT@@QEBA_NPEAUhb_sanitize_context_t@@I@Z 00000001800d60c8     hb-ot-color.obj
 0002:0002b0c8       $chain$2$?sanitize_shallow@?$UnsizedArrayOf@UAxisValueRecord@OT@@@OT@@QEBA_NPEAUhb_sanitize_context_t@@I@Z 00000001800d60c8     hb-ot-shape.obj
 0002:0002b0d8       $unwind$??$check_range@U?$IntType@E$00@OT@@@hb_sanitize_context_t@@QEBA_NPEBU?$IntType@E$00@OT@@II@Z 00000001800d60d8     hb-aat-layout.obj
 0002:0002b0d8       $unwind$??$check_range@U?$IntType@F$01@OT@@@hb_sanitize_context_t@@QEBA_NPEBU?$IntType@F$01@OT@@II@Z 00000001800d60d8     hb-aat-layout.obj
 0002:0002b0d8       $unwind$??$check_range@U?$IntType@G$01@OT@@@hb_sanitize_context_t@@QEBA_NPEBU?$IntType@G$01@OT@@II@Z 00000001800d60d8     hb-aat-layout.obj
 0002:0002b0e0       $chain$0$??$check_range@U?$IntType@E$00@OT@@@hb_sanitize_context_t@@QEBA_NPEBU?$IntType@E$00@OT@@II@Z 00000001800d60e0     hb-aat-layout.obj
 0002:0002b0e0       $chain$0$??$check_range@U?$IntType@F$01@OT@@@hb_sanitize_context_t@@QEBA_NPEBU?$IntType@F$01@OT@@II@Z 00000001800d60e0     hb-aat-layout.obj
 0002:0002b0e0       $chain$0$??$check_range@U?$IntType@G$01@OT@@@hb_sanitize_context_t@@QEBA_NPEBU?$IntType@G$01@OT@@II@Z 00000001800d60e0     hb-aat-layout.obj
 0002:0002b0f4       $chain$1$??$check_range@U?$IntType@E$00@OT@@@hb_sanitize_context_t@@QEBA_NPEBU?$IntType@E$00@OT@@II@Z 00000001800d60f4     hb-aat-layout.obj
 0002:0002b0f4       $chain$1$??$check_range@U?$IntType@F$01@OT@@@hb_sanitize_context_t@@QEBA_NPEBU?$IntType@F$01@OT@@II@Z 00000001800d60f4     hb-aat-layout.obj
 0002:0002b0f4       $chain$1$??$check_range@U?$IntType@G$01@OT@@@hb_sanitize_context_t@@QEBA_NPEBU?$IntType@G$01@OT@@II@Z 00000001800d60f4     hb-aat-layout.obj
 0002:0002b104       $unwind$?sanitize@?$GDEFVersion1_2@USmallTypes@Layout@OT@@@OT@@QEBA_NPEAUhb_sanitize_context_t@@@Z 00000001800d6104     hb-aat-layout.obj
 0002:0002b104       $unwind$?sanitize@ItemVariationStore@OT@@QEBA_NPEAUhb_sanitize_context_t@@@Z 00000001800d6104     hb-aat-layout.obj
 0002:0002b104       $unwind$?sanitize@trak@AAT@@QEBA_NPEAUhb_sanitize_context_t@@@Z 00000001800d6104     hb-aat-layout.obj
 0002:0002b104       $unwind$?sanitize@CBLC@OT@@QEBA_NPEAUhb_sanitize_context_t@@@Z 00000001800d6104     hb-ot-color.obj
 0002:0002b104       $unwind$?sanitize@sbix@OT@@QEBA_NPEAUhb_sanitize_context_t@@@Z 00000001800d6104     hb-ot-color.obj
 0002:0002b104       $unwind$?hb_ot_shape_internal@@YAXPEAUhb_ot_shape_context_t@@@Z 00000001800d6104     hb-ot-shape.obj
 0002:0002b11c       $unwind$?get_kerning@?$KerxSubTableFormat6@UKerxSubTableHeader@AAT@@@AAT@@QEBAHIIPEAUhb_aat_apply_context_t@2@@Z 00000001800d611c     hb-aat-layout.obj
 0002:0002b11c       $unwind$?sanitize@Condition@OT@@QEBA_NPEAUhb_sanitize_context_t@@@Z 00000001800d611c     hb-aat-layout.obj
 0002:0002b11c       $unwind$?sanitize@OS2@OT@@QEBA_NPEAUhb_sanitize_context_t@@@Z 00000001800d611c     hb-face.obj
 0002:0002b11c       $unwind$?sanitize@CPAL@OT@@QEBA_NPEAUhb_sanitize_context_t@@@Z 00000001800d611c     hb-ot-color.obj
 0002:0002b11c       $unwind$?sanitize@?$MarkBasePosFormat1_2@USmallTypes@Layout@OT@@@GPOS_impl@Layout@OT@@QEBA_NPEAUhb_sanitize_context_t@@@Z 00000001800d611c     hb-ot-layout.obj
 0002:0002b11c       $unwind$?sanitize@?$MarkMarkPosFormat1_2@USmallTypes@Layout@OT@@@GPOS_impl@Layout@OT@@QEBA_NPEAUhb_sanitize_context_t@@@Z 00000001800d611c     hb-ot-layout.obj
 0002:0002b11c       $unwind$?sanitize@AxisValue@OT@@QEBA_NPEAUhb_sanitize_context_t@@@Z 00000001800d611c     hb-ot-shape.obj
 0002:0002b138       $unwind$?get_kerning@?$KerxSubTableFormat2@UKerxSubTableHeader@AAT@@@AAT@@QEBAHIIPEAUhb_aat_apply_context_t@2@@Z 00000001800d6138     hb-aat-layout.obj
 0002:0002b138       $unwind$?sanitize@?$mortmorx@Umort@AAT@@UObsoleteTypes@2@$0GNGPHCHE@@AAT@@QEBA_NPEAUhb_sanitize_context_t@@@Z 00000001800d6138     hb-aat-layout.obj
 0002:0002b138       $unwind$?sanitize@?$mortmorx@Umorx@AAT@@UExtendedTypes@2@$0GNGPHCHI@@AAT@@QEBA_NPEAUhb_sanitize_context_t@@@Z 00000001800d6138     hb-aat-layout.obj
 0002:0002b138       $unwind$?sanitize@FeatureVariations@OT@@QEBA_NPEAUhb_sanitize_context_t@@@Z 00000001800d6138     hb-aat-layout.obj
 0002:0002b138       $unwind$?sanitize@CmapSubtable@OT@@QEBA_NPEAUhb_sanitize_context_t@@@Z 00000001800d6138     hb-face.obj
 0002:0002b138       $unwind$??$dispatch@Uhb_sanitize_context_t@@$$V@ClipBox@OT@@QEBA_NPEAUhb_sanitize_context_t@@@Z 00000001800d6138     hb-ot-color.obj
 0002:0002b138       $unwind$?sanitize@SinglePosFormat2@GPOS_impl@Layout@OT@@QEBA_NPEAUhb_sanitize_context_t@@@Z 00000001800d6138     hb-ot-layout.obj
 0002:0002b150       $unwind$?sanitize@?$Chain@UObsoleteTypes@AAT@@@AAT@@QEBA_NPEAUhb_sanitize_context_t@@I@Z 00000001800d6150     hb-aat-layout.obj
 0002:0002b150       $unwind$?sanitize@?$KerxSubTableFormat6@UKerxSubTableHeader@AAT@@@AAT@@QEBA_NPEAUhb_sanitize_context_t@@@Z 00000001800d6150     hb-aat-layout.obj
 0002:0002b150       $unwind$?sanitize@Device@OT@@QEBA_NPEAUhb_sanitize_context_t@@@Z 00000001800d6150     hb-aat-layout.obj
 0002:0002b150       $unwind$?sanitize@KerxSubTable@AAT@@QEBA_NPEAUhb_sanitize_context_t@@@Z 00000001800d6150     hb-aat-layout.obj
 0002:0002b150       $unwind$?sanitize@SubtableGlyphCoverage@AAT@@QEBA_NPEAUhb_sanitize_context_t@@I@Z 00000001800d6150     hb-aat-layout.obj
 0002:0002b16c       $unwind$?sanitize@CaretValue@OT@@QEBA_NPEAUhb_sanitize_context_t@@@Z 00000001800d616c     hb-aat-layout.obj
 0002:0002b16c       $unwind$?sanitize@Anchor@GPOS_impl@Layout@OT@@QEBA_NPEAUhb_sanitize_context_t@@@Z 00000001800d616c     hb-ot-layout.obj
 0002:0002b184       $chain$0$?sanitize@CaretValue@OT@@QEBA_NPEAUhb_sanitize_context_t@@@Z 00000001800d6184     hb-aat-layout.obj
 0002:0002b198       $chain$2$?sanitize@CaretValue@OT@@QEBA_NPEAUhb_sanitize_context_t@@@Z 00000001800d6198     hb-aat-layout.obj
 0002:0002b1ac       $chain$3$?sanitize@CaretValue@OT@@QEBA_NPEAUhb_sanitize_context_t@@@Z 00000001800d61ac     hb-aat-layout.obj
 0002:0002b1bc       $unwind$??$sanitize@USubstLookup@GSUB_impl@Layout@OT@@@?$GSUBGPOSVersion1_2@USmallTypes@Layout@OT@@@OT@@QEBA_NPEAUhb_sanitize_context_t@@@Z 00000001800d61bc     hb-aat-layout.obj
 0002:0002b1bc       $unwind$?get_glyph_props@GDEF@OT@@QEBAII@Z 00000001800d61bc     hb-aat-layout.obj
 0002:0002b1bc       $unwind$?push@?$hb_vector_t@Ufeature_event_t@hb_aat_map_builder_t@@$0A@@@QEAAPEAUfeature_event_t@hb_aat_map_builder_t@@XZ 00000001800d61bc     hb-aat-map.obj
 0002:0002b1bc       $unwind$?push@?$hb_vector_t@Ufeature_range_t@hb_aat_map_builder_t@@$00@@QEAAPEAUfeature_range_t@hb_aat_map_builder_t@@XZ 00000001800d61bc     hb-aat-map.obj
 0002:0002b1bc       $unwind$hb_blob_create_or_fail 00000001800d61bc     hb-blob.obj
 0002:0002b1bc       $unwind$?clear@hb_paint_extents_context_t@@QEAAXXZ 00000001800d61bc     hb-font.obj
 0002:0002b1bc       $unwind$HBCreateFontFuncs  00000001800d61bc     hb-jdk-font-p.obj
 0002:0002b1bc       $unwind$??$sanitize@UPosLookup@GPOS_impl@Layout@OT@@@?$GSUBGPOSVersion1_2@USmallTypes@Layout@OT@@@OT@@QEBA_NPEAUhb_sanitize_context_t@@@Z 00000001800d61bc     hb-ot-layout.obj
 0002:0002b1bc       $unwind$?apply@?$AlternateSubstFormat1_2@USmallTypes@Layout@OT@@@GSUB_impl@Layout@OT@@QEBA_NPEAUhb_ot_apply_context_t@4@@Z 00000001800d61bc     hb-ot-layout.obj
 0002:0002b1bc       $unwind$?apply@?$MultipleSubstFormat1_2@USmallTypes@Layout@OT@@@GSUB_impl@Layout@OT@@QEBA_NPEAUhb_ot_apply_context_t@4@@Z 00000001800d61bc     hb-ot-layout.obj
 0002:0002b1bc       $unwind$?hb_ot_layout_table_find_feature@@YA_NPEAUhb_face_t@@IIPEAI@Z 00000001800d61bc     hb-ot-layout.obj
 0002:0002b1bc       $unwind$hb_ot_layout_language_get_required_feature 00000001800d61bc     hb-ot-layout.obj
 0002:0002b1bc       $unwind$hb_ot_layout_script_select_language 00000001800d61bc     hb-ot-layout.obj
 0002:0002b1bc       $unwind$?_hb_glyph_info_set_unicode_props@@YAXPEAUhb_glyph_info_t@@PEAUhb_buffer_t@@@Z 00000001800d61bc     hb-ot-shape-normalize.obj
 0002:0002b1bc       $unwind$?_hb_glyph_info_set_unicode_props@@YAXPEAUhb_glyph_info_t@@PEAUhb_buffer_t@@@Z 00000001800d61bc     hb-ot-shape.obj
 0002:0002b1bc       $unwind$?push@?$hb_vector_t@Ulink_t@object_t@hb_serialize_context_t@@$0A@@@QEAAPEAUlink_t@object_t@hb_serialize_context_t@@XZ 00000001800d61bc     hb-ot-shaper-arabic.obj
 0002:0002b1d4       $unwind$??0accelerator_t@GDEF@OT@@QEAA@PEAUhb_face_t@@@Z 00000001800d61d4     hb-aat-layout.obj
 0002:0002b1f4       $chain$1$??1hb_aat_scratch_t@AAT@@QEAA@XZ 00000001800d61f4     hb-aat-layout.obj
 0002:0002b20c       $chain$2$??1hb_aat_scratch_t@AAT@@QEAA@XZ 00000001800d620c     hb-aat-layout.obj
 0002:0002b21c       $chain$0$?setup_buffer_glyph_set@hb_aat_apply_context_t@AAT@@QEAAXXZ 00000001800d621c     hb-aat-layout.obj
 0002:0002b230       $chain$1$?setup_buffer_glyph_set@hb_aat_apply_context_t@AAT@@QEAAXXZ 00000001800d6230     hb-aat-layout.obj
 0002:0002b240       $unwind$?replace_glyph@hb_aat_apply_context_t@AAT@@QEAA_NI@Z 00000001800d6240     hb-aat-layout.obj
 0002:0002b250       $chain$0$?replace_glyph@hb_aat_apply_context_t@AAT@@QEAA_NI@Z 00000001800d6250     hb-aat-layout.obj
 0002:0002b264       $chain$1$?replace_glyph@hb_aat_apply_context_t@AAT@@QEAA_NI@Z 00000001800d6264     hb-aat-layout.obj
 0002:0002b274       $unwind$?sanitize@ankr@AAT@@QEBA_NPEAUhb_sanitize_context_t@@@Z 00000001800d6274     hb-aat-layout.obj
 0002:0002b28c       $chain$1$?sanitize_shallow@?$UnsizedArrayOf@U?$OffsetTo@U?$ArrayOf@UAnchor@AAT@@U?$IntType@I$03@OT@@@OT@@U?$IntType@G$01@2@X$0A@@OT@@@OT@@QEBA_NPEAUhb_sanitize_context_t@@I@Z 00000001800d628c     hb-aat-layout.obj
 0002:0002b28c       $chain$1$?sanitize_shallow@?$UnsizedArrayOf@U?$OffsetTo@U?$Lookup@UHBGlyphID16@OT@@@AAT@@U?$IntType@G$01@OT@@X$0A@@OT@@@OT@@QEBA_NPEAUhb_sanitize_context_t@@I@Z 00000001800d628c     hb-aat-layout.obj
 0002:0002b28c       $chain$1$?sanitize_shallow@?$UnsizedArrayOf@U?$HBFixed@U?$IntType@F$01@OT@@$0O@@OT@@@OT@@QEBA_NPEAUhb_sanitize_context_t@@I@Z 00000001800d628c     hb-common.obj
 0002:0002b28c       $chain$1$?sanitize_shallow@?$UnsizedArrayOf@U?$IntType@G$01@OT@@@OT@@QEBA_NPEAUhb_sanitize_context_t@@I@Z 00000001800d628c     hb-ot-color.obj
 0002:0002b28c       $chain$1$?sanitize_shallow@?$UnsizedArrayOf@U?$Offset@U?$IntType@G$01@OT@@$00@OT@@@OT@@QEBA_NPEAUhb_sanitize_context_t@@I@Z 00000001800d628c     hb-ot-color.obj
 0002:0002b28c       $chain$1$?sanitize_shallow@?$UnsizedArrayOf@UIndex@OT@@@OT@@QEBA_NPEAUhb_sanitize_context_t@@I@Z 00000001800d628c     hb-ot-color.obj
 0002:0002b28c       $chain$1$?sanitize_shallow@?$UnsizedArrayOf@U?$OffsetTo@UAxisValue@OT@@U?$IntType@G$01@2@X$00@OT@@@OT@@QEBA_NPEAUhb_sanitize_context_t@@I@Z 00000001800d628c     hb-ot-shape.obj
 0002:0002b2a4       $chain$2$?sanitize_shallow@?$UnsizedArrayOf@U?$OffsetTo@U?$ArrayOf@UAnchor@AAT@@U?$IntType@I$03@OT@@@OT@@U?$IntType@G$01@2@X$0A@@OT@@@OT@@QEBA_NPEAUhb_sanitize_context_t@@I@Z 00000001800d62a4     hb-aat-layout.obj
 0002:0002b2a4       $chain$2$?sanitize_shallow@?$UnsizedArrayOf@U?$OffsetTo@U?$Lookup@UHBGlyphID16@OT@@@AAT@@U?$IntType@G$01@OT@@X$0A@@OT@@@OT@@QEBA_NPEAUhb_sanitize_context_t@@I@Z 00000001800d62a4     hb-aat-layout.obj
 0002:0002b2a4       $chain$2$?sanitize_shallow@?$UnsizedArrayOf@U?$HBFixed@U?$IntType@F$01@OT@@$0O@@OT@@@OT@@QEBA_NPEAUhb_sanitize_context_t@@I@Z 00000001800d62a4     hb-common.obj
 0002:0002b2a4       $chain$2$?sanitize_shallow@?$UnsizedArrayOf@U?$IntType@G$01@OT@@@OT@@QEBA_NPEAUhb_sanitize_context_t@@I@Z 00000001800d62a4     hb-ot-color.obj
 0002:0002b2a4       $chain$2$?sanitize_shallow@?$UnsizedArrayOf@U?$Offset@U?$IntType@G$01@OT@@$00@OT@@@OT@@QEBA_NPEAUhb_sanitize_context_t@@I@Z 00000001800d62a4     hb-ot-color.obj
 0002:0002b2a4       $chain$2$?sanitize_shallow@?$UnsizedArrayOf@UIndex@OT@@@OT@@QEBA_NPEAUhb_sanitize_context_t@@I@Z 00000001800d62a4     hb-ot-color.obj
 0002:0002b2a4       $chain$2$?sanitize_shallow@?$UnsizedArrayOf@U?$OffsetTo@UAxisValue@OT@@U?$IntType@G$01@2@X$00@OT@@@OT@@QEBA_NPEAUhb_sanitize_context_t@@I@Z 00000001800d62a4     hb-ot-shape.obj
 0002:0002b2b4       $unwind$?get_value@?$LookupFormat2@U?$IntType@G$01@OT@@@AAT@@AEBAPEBU?$IntType@G$01@OT@@I@Z 00000001800d62b4     hb-aat-layout.obj
 0002:0002b2b4       $unwind$?get_value@?$LookupFormat2@U?$IntType@I$03@OT@@@AAT@@AEBAPEBU?$IntType@I$03@OT@@I@Z 00000001800d62b4     hb-aat-layout.obj
 0002:0002b2b4       $unwind$?get_value@?$LookupFormat2@U?$OffsetTo@U?$ArrayOf@UAnchor@AAT@@U?$IntType@I$03@OT@@@OT@@U?$IntType@G$01@2@X$0A@@OT@@@AAT@@AEBAPEBU?$OffsetTo@U?$ArrayOf@UAnchor@AAT@@U?$IntType@I$03@OT@@@OT@@U?$IntType@G$01@2@X$0A@@OT@@I@Z 00000001800d62b4     hb-aat-layout.obj
 0002:0002b2b4       $unwind$?get_value@?$LookupFormat2@UHBGlyphID16@OT@@@AAT@@AEBAPEBUHBGlyphID16@OT@@I@Z 00000001800d62b4     hb-aat-layout.obj
 0002:0002b2b4       $unwind$?get_value@?$LookupFormat6@U?$IntType@G$01@OT@@@AAT@@AEBAPEBU?$IntType@G$01@OT@@I@Z 00000001800d62b4     hb-aat-layout.obj
 0002:0002b2b4       $unwind$?get_value@?$LookupFormat6@U?$IntType@I$03@OT@@@AAT@@AEBAPEBU?$IntType@I$03@OT@@I@Z 00000001800d62b4     hb-aat-layout.obj
 0002:0002b2b4       $unwind$?get_value@?$LookupFormat6@U?$OffsetTo@U?$ArrayOf@UAnchor@AAT@@U?$IntType@I$03@OT@@@OT@@U?$IntType@G$01@2@X$0A@@OT@@@AAT@@AEBAPEBU?$OffsetTo@U?$ArrayOf@UAnchor@AAT@@U?$IntType@I$03@OT@@@OT@@U?$IntType@G$01@2@X$0A@@OT@@I@Z 00000001800d62b4     hb-aat-layout.obj
 0002:0002b2b4       $unwind$?get_value@?$LookupFormat6@UHBGlyphID16@OT@@@AAT@@AEBAPEBUHBGlyphID16@OT@@I@Z 00000001800d62b4     hb-aat-layout.obj
 0002:0002b2c8       $chain$0$?get_value@?$LookupFormat2@U?$IntType@G$01@OT@@@AAT@@AEBAPEBU?$IntType@G$01@OT@@I@Z 00000001800d62c8     hb-aat-layout.obj
 0002:0002b2c8       $chain$0$?get_value@?$LookupFormat2@U?$IntType@I$03@OT@@@AAT@@AEBAPEBU?$IntType@I$03@OT@@I@Z 00000001800d62c8     hb-aat-layout.obj
 0002:0002b2c8       $chain$0$?get_value@?$LookupFormat2@U?$OffsetTo@U?$ArrayOf@UAnchor@AAT@@U?$IntType@I$03@OT@@@OT@@U?$IntType@G$01@2@X$0A@@OT@@@AAT@@AEBAPEBU?$OffsetTo@U?$ArrayOf@UAnchor@AAT@@U?$IntType@I$03@OT@@@OT@@U?$IntType@G$01@2@X$0A@@OT@@I@Z 00000001800d62c8     hb-aat-layout.obj
 0002:0002b2c8       $chain$0$?get_value@?$LookupFormat2@UHBGlyphID16@OT@@@AAT@@AEBAPEBUHBGlyphID16@OT@@I@Z 00000001800d62c8     hb-aat-layout.obj
 0002:0002b2dc       $chain$1$?get_value@?$LookupFormat2@U?$IntType@G$01@OT@@@AAT@@AEBAPEBU?$IntType@G$01@OT@@I@Z 00000001800d62dc     hb-aat-layout.obj
 0002:0002b2dc       $chain$1$?get_value@?$LookupFormat2@U?$IntType@I$03@OT@@@AAT@@AEBAPEBU?$IntType@I$03@OT@@I@Z 00000001800d62dc     hb-aat-layout.obj
 0002:0002b2dc       $chain$1$?get_value@?$LookupFormat2@U?$OffsetTo@U?$ArrayOf@UAnchor@AAT@@U?$IntType@I$03@OT@@@OT@@U?$IntType@G$01@2@X$0A@@OT@@@AAT@@AEBAPEBU?$OffsetTo@U?$ArrayOf@UAnchor@AAT@@U?$IntType@I$03@OT@@@OT@@U?$IntType@G$01@2@X$0A@@OT@@I@Z 00000001800d62dc     hb-aat-layout.obj
 0002:0002b2dc       $chain$1$?get_value@?$LookupFormat2@UHBGlyphID16@OT@@@AAT@@AEBAPEBUHBGlyphID16@OT@@I@Z 00000001800d62dc     hb-aat-layout.obj
 0002:0002b2f0       $chain$2$?get_value@?$LookupFormat2@U?$IntType@G$01@OT@@@AAT@@AEBAPEBU?$IntType@G$01@OT@@I@Z 00000001800d62f0     hb-aat-layout.obj
 0002:0002b2f0       $chain$2$?get_value@?$LookupFormat2@U?$IntType@I$03@OT@@@AAT@@AEBAPEBU?$IntType@I$03@OT@@I@Z 00000001800d62f0     hb-aat-layout.obj
 0002:0002b2f0       $chain$2$?get_value@?$LookupFormat2@U?$OffsetTo@U?$ArrayOf@UAnchor@AAT@@U?$IntType@I$03@OT@@@OT@@U?$IntType@G$01@2@X$0A@@OT@@@AAT@@AEBAPEBU?$OffsetTo@U?$ArrayOf@UAnchor@AAT@@U?$IntType@I$03@OT@@@OT@@U?$IntType@G$01@2@X$0A@@OT@@I@Z 00000001800d62f0     hb-aat-layout.obj
 0002:0002b2f0       $chain$2$?get_value@?$LookupFormat2@UHBGlyphID16@OT@@@AAT@@AEBAPEBUHBGlyphID16@OT@@I@Z 00000001800d62f0     hb-aat-layout.obj
 0002:0002b300       $chain$3$?get_value@?$LookupFormat2@U?$IntType@G$01@OT@@@AAT@@AEBAPEBU?$IntType@G$01@OT@@I@Z 00000001800d6300     hb-aat-layout.obj
 0002:0002b300       $chain$3$?get_value@?$LookupFormat2@U?$IntType@I$03@OT@@@AAT@@AEBAPEBU?$IntType@I$03@OT@@I@Z 00000001800d6300     hb-aat-layout.obj
 0002:0002b300       $chain$3$?get_value@?$LookupFormat2@U?$OffsetTo@U?$ArrayOf@UAnchor@AAT@@U?$IntType@I$03@OT@@@OT@@U?$IntType@G$01@2@X$0A@@OT@@@AAT@@AEBAPEBU?$OffsetTo@U?$ArrayOf@UAnchor@AAT@@U?$IntType@I$03@OT@@@OT@@U?$IntType@G$01@2@X$0A@@OT@@I@Z 00000001800d6300     hb-aat-layout.obj
 0002:0002b300       $chain$3$?get_value@?$LookupFormat2@UHBGlyphID16@OT@@@AAT@@AEBAPEBUHBGlyphID16@OT@@I@Z 00000001800d6300     hb-aat-layout.obj
 0002:0002b310       $unwind$?get_length@?$VarSizedBinSearchArrayOf@U?$LookupSegmentArray@U?$IntType@G$01@OT@@@AAT@@@OT@@QEBAIXZ 00000001800d6310     hb-aat-layout.obj
 0002:0002b310       $unwind$?get_length@?$VarSizedBinSearchArrayOf@U?$LookupSegmentArray@U?$IntType@I$03@OT@@@AAT@@@OT@@QEBAIXZ 00000001800d6310     hb-aat-layout.obj
 0002:0002b310       $unwind$?get_length@?$VarSizedBinSearchArrayOf@U?$LookupSegmentArray@U?$OffsetTo@U?$ArrayOf@UAnchor@AAT@@U?$IntType@I$03@OT@@@OT@@U?$IntType@G$01@2@X$0A@@OT@@@AAT@@@OT@@QEBAIXZ 00000001800d6310     hb-aat-layout.obj
 0002:0002b310       $unwind$?get_length@?$VarSizedBinSearchArrayOf@U?$LookupSegmentArray@UHBGlyphID16@OT@@@AAT@@@OT@@QEBAIXZ 00000001800d6310     hb-aat-layout.obj
 0002:0002b310       $unwind$?get_length@?$VarSizedBinSearchArrayOf@U?$LookupSegmentSingle@U?$IntType@G$01@OT@@@AAT@@@OT@@QEBAIXZ 00000001800d6310     hb-aat-layout.obj
 0002:0002b310       $unwind$?get_length@?$VarSizedBinSearchArrayOf@U?$LookupSegmentSingle@U?$IntType@I$03@OT@@@AAT@@@OT@@QEBAIXZ 00000001800d6310     hb-aat-layout.obj
 0002:0002b310       $unwind$?get_length@?$VarSizedBinSearchArrayOf@U?$LookupSegmentSingle@U?$OffsetTo@U?$ArrayOf@UAnchor@AAT@@U?$IntType@I$03@OT@@@OT@@U?$IntType@G$01@2@X$0A@@OT@@@AAT@@@OT@@QEBAIXZ 00000001800d6310     hb-aat-layout.obj
 0002:0002b310       $unwind$?get_length@?$VarSizedBinSearchArrayOf@U?$LookupSegmentSingle@UHBGlyphID16@OT@@@AAT@@@OT@@QEBAIXZ 00000001800d6310     hb-aat-layout.obj
 0002:0002b310       $unwind$?get_length@?$VarSizedBinSearchArrayOf@U?$LookupSingle@U?$IntType@G$01@OT@@@AAT@@@OT@@QEBAIXZ 00000001800d6310     hb-aat-layout.obj
 0002:0002b310       $unwind$?get_length@?$VarSizedBinSearchArrayOf@U?$LookupSingle@U?$IntType@I$03@OT@@@AAT@@@OT@@QEBAIXZ 00000001800d6310     hb-aat-layout.obj
 0002:0002b310       $unwind$?get_length@?$VarSizedBinSearchArrayOf@U?$LookupSingle@U?$OffsetTo@U?$ArrayOf@UAnchor@AAT@@U?$IntType@I$03@OT@@@OT@@U?$IntType@G$01@2@X$0A@@OT@@@AAT@@@OT@@QEBAIXZ 00000001800d6310     hb-aat-layout.obj
 0002:0002b310       $unwind$?get_length@?$VarSizedBinSearchArrayOf@U?$LookupSingle@UHBGlyphID16@OT@@@AAT@@@OT@@QEBAIXZ 00000001800d6310     hb-aat-layout.obj
 0002:0002b31c       $unwind$?get_value@?$LookupFormat4@U?$IntType@G$01@OT@@@AAT@@AEBAPEBU?$IntType@G$01@OT@@I@Z 00000001800d631c     hb-aat-layout.obj
 0002:0002b31c       $unwind$?get_value@?$LookupFormat4@U?$IntType@I$03@OT@@@AAT@@AEBAPEBU?$IntType@I$03@OT@@I@Z 00000001800d631c     hb-aat-layout.obj
 0002:0002b31c       $unwind$?get_value@?$LookupFormat4@U?$OffsetTo@U?$ArrayOf@UAnchor@AAT@@U?$IntType@I$03@OT@@@OT@@U?$IntType@G$01@2@X$0A@@OT@@@AAT@@AEBAPEBU?$OffsetTo@U?$ArrayOf@UAnchor@AAT@@U?$IntType@I$03@OT@@@OT@@U?$IntType@G$01@2@X$0A@@OT@@I@Z 00000001800d631c     hb-aat-layout.obj
 0002:0002b31c       $unwind$?get_value@?$LookupFormat4@UHBGlyphID16@OT@@@AAT@@AEBAPEBUHBGlyphID16@OT@@I@Z 00000001800d631c     hb-aat-layout.obj
 0002:0002b32c       $chain$0$?get_value@?$LookupFormat4@U?$IntType@G$01@OT@@@AAT@@AEBAPEBU?$IntType@G$01@OT@@I@Z 00000001800d632c     hb-aat-layout.obj
 0002:0002b32c       $chain$0$?get_value@?$LookupFormat4@U?$OffsetTo@U?$ArrayOf@UAnchor@AAT@@U?$IntType@I$03@OT@@@OT@@U?$IntType@G$01@2@X$0A@@OT@@@AAT@@AEBAPEBU?$OffsetTo@U?$ArrayOf@UAnchor@AAT@@U?$IntType@I$03@OT@@@OT@@U?$IntType@G$01@2@X$0A@@OT@@I@Z 00000001800d632c     hb-aat-layout.obj
 0002:0002b32c       $chain$0$?get_value@?$LookupFormat4@UHBGlyphID16@OT@@@AAT@@AEBAPEBUHBGlyphID16@OT@@I@Z 00000001800d632c     hb-aat-layout.obj
 0002:0002b340       $chain$1$?get_value@?$LookupFormat4@U?$IntType@G$01@OT@@@AAT@@AEBAPEBU?$IntType@G$01@OT@@I@Z 00000001800d6340     hb-aat-layout.obj
 0002:0002b340       $chain$1$?get_value@?$LookupFormat4@U?$OffsetTo@U?$ArrayOf@UAnchor@AAT@@U?$IntType@I$03@OT@@@OT@@U?$IntType@G$01@2@X$0A@@OT@@@AAT@@AEBAPEBU?$OffsetTo@U?$ArrayOf@UAnchor@AAT@@U?$IntType@I$03@OT@@@OT@@U?$IntType@G$01@2@X$0A@@OT@@I@Z 00000001800d6340     hb-aat-layout.obj
 0002:0002b340       $chain$1$?get_value@?$LookupFormat4@UHBGlyphID16@OT@@@AAT@@AEBAPEBUHBGlyphID16@OT@@I@Z 00000001800d6340     hb-aat-layout.obj
 0002:0002b354       $chain$2$?get_value@?$LookupFormat4@U?$IntType@G$01@OT@@@AAT@@AEBAPEBU?$IntType@G$01@OT@@I@Z 00000001800d6354     hb-aat-layout.obj
 0002:0002b354       $chain$2$?get_value@?$LookupFormat4@U?$OffsetTo@U?$ArrayOf@UAnchor@AAT@@U?$IntType@I$03@OT@@@OT@@U?$IntType@G$01@2@X$0A@@OT@@@AAT@@AEBAPEBU?$OffsetTo@U?$ArrayOf@UAnchor@AAT@@U?$IntType@I$03@OT@@@OT@@U?$IntType@G$01@2@X$0A@@OT@@I@Z 00000001800d6354     hb-aat-layout.obj
 0002:0002b354       $chain$2$?get_value@?$LookupFormat4@UHBGlyphID16@OT@@@AAT@@AEBAPEBUHBGlyphID16@OT@@I@Z 00000001800d6354     hb-aat-layout.obj
 0002:0002b364       $chain$3$?get_value@?$LookupFormat4@U?$IntType@G$01@OT@@@AAT@@AEBAPEBU?$IntType@G$01@OT@@I@Z 00000001800d6364     hb-aat-layout.obj
 0002:0002b364       $chain$3$?get_value@?$LookupFormat4@U?$OffsetTo@U?$ArrayOf@UAnchor@AAT@@U?$IntType@I$03@OT@@@OT@@U?$IntType@G$01@2@X$0A@@OT@@@AAT@@AEBAPEBU?$OffsetTo@U?$ArrayOf@UAnchor@AAT@@U?$IntType@I$03@OT@@@OT@@U?$IntType@G$01@2@X$0A@@OT@@I@Z 00000001800d6364     hb-aat-layout.obj
 0002:0002b364       $chain$3$?get_value@?$LookupFormat4@UHBGlyphID16@OT@@@AAT@@AEBAPEBUHBGlyphID16@OT@@I@Z 00000001800d6364     hb-aat-layout.obj
 0002:0002b374       $unwind$?sanitize@?$LookupFormat4@U?$OffsetTo@U?$ArrayOf@UAnchor@AAT@@U?$IntType@I$03@OT@@@OT@@U?$IntType@G$01@2@X$0A@@OT@@@AAT@@AEBA_NPEAUhb_sanitize_context_t@@PEBX@Z 00000001800d6374     hb-aat-layout.obj
 0002:0002b380       $chain$4$?sanitize@?$LookupFormat4@U?$OffsetTo@U?$ArrayOf@UAnchor@AAT@@U?$IntType@I$03@OT@@@OT@@U?$IntType@G$01@2@X$0A@@OT@@@AAT@@AEBA_NPEAUhb_sanitize_context_t@@PEBX@Z 00000001800d6380     hb-aat-layout.obj
 0002:0002b3a4       $chain$6$?sanitize@?$LookupFormat4@U?$OffsetTo@U?$ArrayOf@UAnchor@AAT@@U?$IntType@I$03@OT@@@OT@@U?$IntType@G$01@2@X$0A@@OT@@@AAT@@AEBA_NPEAUhb_sanitize_context_t@@PEBX@Z 00000001800d63a4     hb-aat-layout.obj
 0002:0002b3c8       $chain$0$?get_value@?$LookupFormat6@U?$IntType@G$01@OT@@@AAT@@AEBAPEBU?$IntType@G$01@OT@@I@Z 00000001800d63c8     hb-aat-layout.obj
 0002:0002b3c8       $chain$0$?get_value@?$LookupFormat6@U?$IntType@I$03@OT@@@AAT@@AEBAPEBU?$IntType@I$03@OT@@I@Z 00000001800d63c8     hb-aat-layout.obj
 0002:0002b3c8       $chain$0$?get_value@?$LookupFormat6@U?$OffsetTo@U?$ArrayOf@UAnchor@AAT@@U?$IntType@I$03@OT@@@OT@@U?$IntType@G$01@2@X$0A@@OT@@@AAT@@AEBAPEBU?$OffsetTo@U?$ArrayOf@UAnchor@AAT@@U?$IntType@I$03@OT@@@OT@@U?$IntType@G$01@2@X$0A@@OT@@I@Z 00000001800d63c8     hb-aat-layout.obj
 0002:0002b3c8       $chain$0$?get_value@?$LookupFormat6@UHBGlyphID16@OT@@@AAT@@AEBAPEBUHBGlyphID16@OT@@I@Z 00000001800d63c8     hb-aat-layout.obj
 0002:0002b3dc       $chain$1$?get_value@?$LookupFormat6@U?$IntType@G$01@OT@@@AAT@@AEBAPEBU?$IntType@G$01@OT@@I@Z 00000001800d63dc     hb-aat-layout.obj
 0002:0002b3dc       $chain$1$?get_value@?$LookupFormat6@U?$IntType@I$03@OT@@@AAT@@AEBAPEBU?$IntType@I$03@OT@@I@Z 00000001800d63dc     hb-aat-layout.obj
 0002:0002b3dc       $chain$1$?get_value@?$LookupFormat6@U?$OffsetTo@U?$ArrayOf@UAnchor@AAT@@U?$IntType@I$03@OT@@@OT@@U?$IntType@G$01@2@X$0A@@OT@@@AAT@@AEBAPEBU?$OffsetTo@U?$ArrayOf@UAnchor@AAT@@U?$IntType@I$03@OT@@@OT@@U?$IntType@G$01@2@X$0A@@OT@@I@Z 00000001800d63dc     hb-aat-layout.obj
 0002:0002b3dc       $chain$1$?get_value@?$LookupFormat6@UHBGlyphID16@OT@@@AAT@@AEBAPEBUHBGlyphID16@OT@@I@Z 00000001800d63dc     hb-aat-layout.obj
 0002:0002b3f0       $chain$2$?get_value@?$LookupFormat6@U?$IntType@G$01@OT@@@AAT@@AEBAPEBU?$IntType@G$01@OT@@I@Z 00000001800d63f0     hb-aat-layout.obj
 0002:0002b3f0       $chain$2$?get_value@?$LookupFormat6@U?$IntType@I$03@OT@@@AAT@@AEBAPEBU?$IntType@I$03@OT@@I@Z 00000001800d63f0     hb-aat-layout.obj
 0002:0002b3f0       $chain$2$?get_value@?$LookupFormat6@U?$OffsetTo@U?$ArrayOf@UAnchor@AAT@@U?$IntType@I$03@OT@@@OT@@U?$IntType@G$01@2@X$0A@@OT@@@AAT@@AEBAPEBU?$OffsetTo@U?$ArrayOf@UAnchor@AAT@@U?$IntType@I$03@OT@@@OT@@U?$IntType@G$01@2@X$0A@@OT@@I@Z 00000001800d63f0     hb-aat-layout.obj
 0002:0002b3f0       $chain$2$?get_value@?$LookupFormat6@UHBGlyphID16@OT@@@AAT@@AEBAPEBUHBGlyphID16@OT@@I@Z 00000001800d63f0     hb-aat-layout.obj
 0002:0002b400       $chain$3$?get_value@?$LookupFormat6@U?$IntType@G$01@OT@@@AAT@@AEBAPEBU?$IntType@G$01@OT@@I@Z 00000001800d6400     hb-aat-layout.obj
 0002:0002b400       $chain$3$?get_value@?$LookupFormat6@U?$IntType@I$03@OT@@@AAT@@AEBAPEBU?$IntType@I$03@OT@@I@Z 00000001800d6400     hb-aat-layout.obj
 0002:0002b400       $chain$3$?get_value@?$LookupFormat6@U?$OffsetTo@U?$ArrayOf@UAnchor@AAT@@U?$IntType@I$03@OT@@@OT@@U?$IntType@G$01@2@X$0A@@OT@@@AAT@@AEBAPEBU?$OffsetTo@U?$ArrayOf@UAnchor@AAT@@U?$IntType@I$03@OT@@@OT@@U?$IntType@G$01@2@X$0A@@OT@@I@Z 00000001800d6400     hb-aat-layout.obj
 0002:0002b400       $chain$3$?get_value@?$LookupFormat6@UHBGlyphID16@OT@@@AAT@@AEBAPEBUHBGlyphID16@OT@@I@Z 00000001800d6400     hb-aat-layout.obj
 0002:0002b410       $unwind$?sanitize@?$Lookup@U?$IntType@G$01@OT@@@AAT@@QEBA_NPEAUhb_sanitize_context_t@@@Z 00000001800d6410     hb-aat-layout.obj
 0002:0002b410       $unwind$?sanitize@?$Lookup@U?$IntType@I$03@OT@@@AAT@@QEBA_NPEAUhb_sanitize_context_t@@@Z 00000001800d6410     hb-aat-layout.obj
 0002:0002b410       $unwind$?sanitize@?$Lookup@UHBGlyphID16@OT@@@AAT@@QEBA_NPEAUhb_sanitize_context_t@@@Z 00000001800d6410     hb-aat-layout.obj
 0002:0002b428       $chain$0$?sanitize@?$Lookup@U?$IntType@G$01@OT@@@AAT@@QEBA_NPEAUhb_sanitize_context_t@@@Z 00000001800d6428     hb-aat-layout.obj
 0002:0002b43c       $chain$2$?sanitize@?$Lookup@U?$IntType@G$01@OT@@@AAT@@QEBA_NPEAUhb_sanitize_context_t@@@Z 00000001800d643c     hb-aat-layout.obj
 0002:0002b450       $chain$3$?sanitize@?$Lookup@U?$IntType@G$01@OT@@@AAT@@QEBA_NPEAUhb_sanitize_context_t@@@Z 00000001800d6450     hb-aat-layout.obj
 0002:0002b460       $unwind$?sanitize@?$LookupFormat4@U?$IntType@G$01@OT@@@AAT@@AEBA_NPEAUhb_sanitize_context_t@@@Z 00000001800d6460     hb-aat-layout.obj
 0002:0002b460       $unwind$?sanitize@?$LookupFormat4@U?$IntType@I$03@OT@@@AAT@@AEBA_NPEAUhb_sanitize_context_t@@@Z 00000001800d6460     hb-aat-layout.obj
 0002:0002b460       $unwind$?sanitize@?$LookupFormat4@UHBGlyphID16@OT@@@AAT@@AEBA_NPEAUhb_sanitize_context_t@@@Z 00000001800d6460     hb-aat-layout.obj
 0002:0002b46c       $chain$4$?sanitize@?$LookupFormat4@U?$IntType@G$01@OT@@@AAT@@AEBA_NPEAUhb_sanitize_context_t@@@Z 00000001800d646c     hb-aat-layout.obj
 0002:0002b490       $chain$6$?sanitize@?$LookupFormat4@U?$IntType@G$01@OT@@@AAT@@AEBA_NPEAUhb_sanitize_context_t@@@Z 00000001800d6490     hb-aat-layout.obj
 0002:0002b4b4       $chain$1$?sanitize_shallow@?$UnsizedArrayOf@U?$HBFixed@U?$IntType@H$03@OT@@$0BA@@OT@@@OT@@QEBA_NPEAUhb_sanitize_context_t@@I@Z 00000001800d64b4     hb-aat-layout.obj
 0002:0002b4b4       $chain$1$?sanitize_shallow@?$UnsizedArrayOf@U?$IntType@I$03@OT@@@OT@@QEBA_NPEAUhb_sanitize_context_t@@I@Z 00000001800d64b4     hb-aat-layout.obj
 0002:0002b4b4       $chain$1$?sanitize_shallow@?$UnsizedArrayOf@U?$OffsetTo@U?$Lookup@UHBGlyphID16@OT@@@AAT@@U?$IntType@I$03@OT@@X$0A@@OT@@@OT@@QEBA_NPEAUhb_sanitize_context_t@@I@Z 00000001800d64b4     hb-aat-layout.obj
 0002:0002b4b4       $chain$1$?sanitize_shallow@?$UnsizedArrayOf@USettingName@AAT@@@OT@@QEBA_NPEAUhb_sanitize_context_t@@I@Z 00000001800d64b4     hb-aat-layout.obj
 0002:0002b4b4       $chain$1$?sanitize_shallow@?$UnsizedArrayOf@U?$Offset@U?$IntType@I$03@OT@@$00@OT@@@OT@@QEBA_NPEAUhb_sanitize_context_t@@I@Z 00000001800d64b4     hb-ot-color.obj
 0002:0002b4b4       $chain$1$?sanitize_shallow@?$UnsizedArrayOf@ULayerRecord@OT@@@OT@@QEBA_NPEAUhb_sanitize_context_t@@I@Z 00000001800d64b4     hb-ot-color.obj
 0002:0002b4cc       $chain$2$?sanitize_shallow@?$UnsizedArrayOf@U?$HBFixed@U?$IntType@H$03@OT@@$0BA@@OT@@@OT@@QEBA_NPEAUhb_sanitize_context_t@@I@Z 00000001800d64cc     hb-aat-layout.obj
 0002:0002b4cc       $chain$2$?sanitize_shallow@?$UnsizedArrayOf@U?$IntType@I$03@OT@@@OT@@QEBA_NPEAUhb_sanitize_context_t@@I@Z 00000001800d64cc     hb-aat-layout.obj
 0002:0002b4cc       $chain$2$?sanitize_shallow@?$UnsizedArrayOf@U?$OffsetTo@U?$Lookup@UHBGlyphID16@OT@@@AAT@@U?$IntType@I$03@OT@@X$0A@@OT@@@OT@@QEBA_NPEAUhb_sanitize_context_t@@I@Z 00000001800d64cc     hb-aat-layout.obj
 0002:0002b4cc       $chain$2$?sanitize_shallow@?$UnsizedArrayOf@USettingName@AAT@@@OT@@QEBA_NPEAUhb_sanitize_context_t@@I@Z 00000001800d64cc     hb-aat-layout.obj
 0002:0002b4cc       $chain$2$?sanitize_shallow@?$UnsizedArrayOf@U?$Offset@U?$IntType@I$03@OT@@$00@OT@@@OT@@QEBA_NPEAUhb_sanitize_context_t@@I@Z 00000001800d64cc     hb-ot-color.obj
 0002:0002b4cc       $chain$2$?sanitize_shallow@?$UnsizedArrayOf@ULayerRecord@OT@@@OT@@QEBA_NPEAUhb_sanitize_context_t@@I@Z 00000001800d64cc     hb-ot-color.obj
 0002:0002b4dc       $chain$1$?sanitize_shallow@?$UnsizedArrayOf@UFeatureName@AAT@@@OT@@QEBA_NPEAUhb_sanitize_context_t@@I@Z 00000001800d64dc     hb-aat-layout.obj
 0002:0002b4dc       $chain$1$?sanitize_shallow@?$UnsizedArrayOf@UResourceRecord@OT@@@OT@@QEBA_NPEAUhb_sanitize_context_t@@I@Z 00000001800d64dc     hb-face.obj
 0002:0002b4f4       $chain$2$?sanitize_shallow@?$UnsizedArrayOf@UFeatureName@AAT@@@OT@@QEBA_NPEAUhb_sanitize_context_t@@I@Z 00000001800d64f4     hb-aat-layout.obj
 0002:0002b4f4       $chain$2$?sanitize_shallow@?$UnsizedArrayOf@UResourceRecord@OT@@@OT@@QEBA_NPEAUhb_sanitize_context_t@@I@Z 00000001800d64f4     hb-face.obj
 0002:0002b504       $chain$0$?sanitize@?$Lookup@UHBGlyphID16@OT@@@AAT@@QEBA_NPEAUhb_sanitize_context_t@@@Z 00000001800d6504     hb-aat-layout.obj
 0002:0002b518       $chain$2$?sanitize@?$Lookup@UHBGlyphID16@OT@@@AAT@@QEBA_NPEAUhb_sanitize_context_t@@@Z 00000001800d6518     hb-aat-layout.obj
 0002:0002b52c       $chain$3$?sanitize@?$Lookup@UHBGlyphID16@OT@@@AAT@@QEBA_NPEAUhb_sanitize_context_t@@@Z 00000001800d652c     hb-aat-layout.obj
 0002:0002b53c       $chain$4$?sanitize@?$LookupFormat4@UHBGlyphID16@OT@@@AAT@@AEBA_NPEAUhb_sanitize_context_t@@@Z 00000001800d653c     hb-aat-layout.obj
 0002:0002b560       $chain$6$?sanitize@?$LookupFormat4@UHBGlyphID16@OT@@@AAT@@AEBA_NPEAUhb_sanitize_context_t@@@Z 00000001800d6560     hb-aat-layout.obj
 0002:0002b584       $unwind$?compile_flags@?$mortmorx@Umort@AAT@@UObsoleteTypes@2@$0GNGPHCHE@@AAT@@QEBAXPEBUhb_aat_map_builder_t@@PEAUhb_aat_map_t@@@Z 00000001800d6584     hb-aat-layout.obj
 0002:0002b584       $unwind$?compile_flags@?$mortmorx@Umorx@AAT@@UExtendedTypes@2@$0GNGPHCHI@@AAT@@QEBAXPEBUhb_aat_map_builder_t@@PEAUhb_aat_map_t@@@Z 00000001800d6584     hb-aat-layout.obj
 0002:0002b598       $chain$0$?compile_flags@?$mortmorx@Umorx@AAT@@UExtendedTypes@2@$0GNGPHCHI@@AAT@@QEBAXPEBUhb_aat_map_builder_t@@PEAUhb_aat_map_t@@@Z 00000001800d6598     hb-aat-layout.obj
 0002:0002b5ac       $chain$1$?compile_flags@?$mortmorx@Umorx@AAT@@UExtendedTypes@2@$0GNGPHCHI@@AAT@@QEBAXPEBUhb_aat_map_builder_t@@PEAUhb_aat_map_t@@@Z 00000001800d65ac     hb-aat-layout.obj
 0002:0002b5c0       $chain$3$?compile_flags@?$mortmorx@Umorx@AAT@@UExtendedTypes@2@$0GNGPHCHI@@AAT@@QEBAXPEBUhb_aat_map_builder_t@@PEAUhb_aat_map_t@@@Z 00000001800d65c0     hb-aat-layout.obj
 0002:0002b5d4       $chain$4$?compile_flags@?$mortmorx@Umorx@AAT@@UExtendedTypes@2@$0GNGPHCHI@@AAT@@QEBAXPEBUhb_aat_map_builder_t@@PEAUhb_aat_map_t@@@Z 00000001800d65d4     hb-aat-layout.obj
 0002:0002b5e4       $chain$5$?compile_flags@?$mortmorx@Umorx@AAT@@UExtendedTypes@2@$0GNGPHCHI@@AAT@@QEBAXPEBUhb_aat_map_builder_t@@PEAUhb_aat_map_t@@@Z 00000001800d65e4     hb-aat-layout.obj
 0002:0002b5f4       $unwind$?apply@?$mortmorx@Umorx@AAT@@UExtendedTypes@2@$0GNGPHCHI@@AAT@@QEBAXPEAUhb_aat_apply_context_t@2@AEBUhb_aat_map_t@@AEBUaccelerator_t@12@@Z 00000001800d65f4     hb-aat-layout.obj
 0002:0002b600       $chain$3$?apply@?$mortmorx@Umorx@AAT@@UExtendedTypes@2@$0GNGPHCHI@@AAT@@QEBAXPEAUhb_aat_apply_context_t@2@AEBUhb_aat_map_t@@AEBUaccelerator_t@12@@Z 00000001800d6600     hb-aat-layout.obj
 0002:0002b620       $chain$4$?apply@?$mortmorx@Umorx@AAT@@UExtendedTypes@2@$0GNGPHCHI@@AAT@@QEBAXPEAUhb_aat_apply_context_t@2@AEBUhb_aat_map_t@@AEBUaccelerator_t@12@@Z 00000001800d6620     hb-aat-layout.obj
 0002:0002b634       $chain$5$?apply@?$mortmorx@Umorx@AAT@@UExtendedTypes@2@$0GNGPHCHI@@AAT@@QEBAXPEAUhb_aat_apply_context_t@2@AEBUhb_aat_map_t@@AEBUaccelerator_t@12@@Z 00000001800d6634     hb-aat-layout.obj
 0002:0002b644       $chain$6$?apply@?$mortmorx@Umorx@AAT@@UExtendedTypes@2@$0GNGPHCHI@@AAT@@QEBAXPEAUhb_aat_apply_context_t@2@AEBUhb_aat_map_t@@AEBUaccelerator_t@12@@Z 00000001800d6644     hb-aat-layout.obj
 0002:0002b654       $unwind$?compile_flags@?$Chain@UExtendedTypes@AAT@@@AAT@@QEBAIPEBUhb_aat_map_builder_t@@@Z 00000001800d6654     hb-aat-layout.obj
 0002:0002b654       $unwind$?compile_flags@?$Chain@UObsoleteTypes@AAT@@@AAT@@QEBAIPEBUhb_aat_map_builder_t@@@Z 00000001800d6654     hb-aat-layout.obj
 0002:0002b660       $chain$5$?compile_flags@?$Chain@UExtendedTypes@AAT@@@AAT@@QEBAIPEBUhb_aat_map_builder_t@@@Z 00000001800d6660     hb-aat-layout.obj
 0002:0002b688       $chain$6$?compile_flags@?$Chain@UExtendedTypes@AAT@@@AAT@@QEBAIPEBUhb_aat_map_builder_t@@@Z 00000001800d6688     hb-aat-layout.obj
 0002:0002b698       $unwind$?apply@?$Chain@UExtendedTypes@AAT@@@AAT@@QEBAXPEAUhb_aat_apply_context_t@2@PEBUhb_aat_layout_chain_accelerator_t@2@@Z 00000001800d6698     hb-aat-layout.obj
 0002:0002b698       $unwind$?apply@?$Chain@UObsoleteTypes@AAT@@@AAT@@QEBAXPEAUhb_aat_apply_context_t@2@PEBUhb_aat_layout_chain_accelerator_t@2@@Z 00000001800d6698     hb-aat-layout.obj
 0002:0002b6a8       $chain$3$?apply@?$Chain@UExtendedTypes@AAT@@@AAT@@QEBAXPEAUhb_aat_apply_context_t@2@PEBUhb_aat_layout_chain_accelerator_t@2@@Z 00000001800d66a8     hb-aat-layout.obj
 0002:0002b6c8       $chain$4$?apply@?$Chain@UExtendedTypes@AAT@@@AAT@@QEBAXPEAUhb_aat_apply_context_t@2@PEBUhb_aat_layout_chain_accelerator_t@2@@Z 00000001800d66c8     hb-aat-layout.obj
 0002:0002b6d8       $chain$5$?apply@?$Chain@UExtendedTypes@AAT@@@AAT@@QEBAXPEAUhb_aat_apply_context_t@2@PEBUhb_aat_layout_chain_accelerator_t@2@@Z 00000001800d66d8     hb-aat-layout.obj
 0002:0002b6f8       $chain$0$?compile_flags@?$mortmorx@Umort@AAT@@UObsoleteTypes@2@$0GNGPHCHE@@AAT@@QEBAXPEBUhb_aat_map_builder_t@@PEAUhb_aat_map_t@@@Z 00000001800d66f8     hb-aat-layout.obj
 0002:0002b70c       $chain$1$?compile_flags@?$mortmorx@Umort@AAT@@UObsoleteTypes@2@$0GNGPHCHE@@AAT@@QEBAXPEBUhb_aat_map_builder_t@@PEAUhb_aat_map_t@@@Z 00000001800d670c     hb-aat-layout.obj
 0002:0002b720       $chain$3$?compile_flags@?$mortmorx@Umort@AAT@@UObsoleteTypes@2@$0GNGPHCHE@@AAT@@QEBAXPEBUhb_aat_map_builder_t@@PEAUhb_aat_map_t@@@Z 00000001800d6720     hb-aat-layout.obj
 0002:0002b734       $chain$4$?compile_flags@?$mortmorx@Umort@AAT@@UObsoleteTypes@2@$0GNGPHCHE@@AAT@@QEBAXPEBUhb_aat_map_builder_t@@PEAUhb_aat_map_t@@@Z 00000001800d6734     hb-aat-layout.obj
 0002:0002b744       $chain$5$?compile_flags@?$mortmorx@Umort@AAT@@UObsoleteTypes@2@$0GNGPHCHE@@AAT@@QEBAXPEBUhb_aat_map_builder_t@@PEAUhb_aat_map_t@@@Z 00000001800d6744     hb-aat-layout.obj
 0002:0002b754       $unwind$?apply@?$mortmorx@Umort@AAT@@UObsoleteTypes@2@$0GNGPHCHE@@AAT@@QEBAXPEAUhb_aat_apply_context_t@2@AEBUhb_aat_map_t@@AEBUaccelerator_t@12@@Z 00000001800d6754     hb-aat-layout.obj
 0002:0002b760       $chain$3$?apply@?$mortmorx@Umort@AAT@@UObsoleteTypes@2@$0GNGPHCHE@@AAT@@QEBAXPEAUhb_aat_apply_context_t@2@AEBUhb_aat_map_t@@AEBUaccelerator_t@12@@Z 00000001800d6760     hb-aat-layout.obj
 0002:0002b780       $chain$4$?apply@?$mortmorx@Umort@AAT@@UObsoleteTypes@2@$0GNGPHCHE@@AAT@@QEBAXPEAUhb_aat_apply_context_t@2@AEBUhb_aat_map_t@@AEBUaccelerator_t@12@@Z 00000001800d6780     hb-aat-layout.obj
 0002:0002b794       $chain$5$?apply@?$mortmorx@Umort@AAT@@UObsoleteTypes@2@$0GNGPHCHE@@AAT@@QEBAXPEAUhb_aat_apply_context_t@2@AEBUhb_aat_map_t@@AEBUaccelerator_t@12@@Z 00000001800d6794     hb-aat-layout.obj
 0002:0002b7a4       $chain$6$?apply@?$mortmorx@Umort@AAT@@UObsoleteTypes@2@$0GNGPHCHE@@AAT@@QEBAXPEAUhb_aat_apply_context_t@2@AEBUhb_aat_map_t@@AEBUaccelerator_t@12@@Z 00000001800d67a4     hb-aat-layout.obj
 0002:0002b7b4       $chain$5$?compile_flags@?$Chain@UObsoleteTypes@AAT@@@AAT@@QEBAIPEBUhb_aat_map_builder_t@@@Z 00000001800d67b4     hb-aat-layout.obj
 0002:0002b7dc       $chain$6$?compile_flags@?$Chain@UObsoleteTypes@AAT@@@AAT@@QEBAIPEBUhb_aat_map_builder_t@@@Z 00000001800d67dc     hb-aat-layout.obj
 0002:0002b7ec       $chain$3$?apply@?$Chain@UObsoleteTypes@AAT@@@AAT@@QEBAXPEAUhb_aat_apply_context_t@2@PEBUhb_aat_layout_chain_accelerator_t@2@@Z 00000001800d67ec     hb-aat-layout.obj
 0002:0002b80c       $chain$4$?apply@?$Chain@UObsoleteTypes@AAT@@@AAT@@QEBAXPEAUhb_aat_apply_context_t@2@PEBUhb_aat_layout_chain_accelerator_t@2@@Z 00000001800d680c     hb-aat-layout.obj
 0002:0002b81c       $chain$5$?apply@?$Chain@UObsoleteTypes@AAT@@@AAT@@QEBAXPEAUhb_aat_apply_context_t@2@PEBUhb_aat_layout_chain_accelerator_t@2@@Z 00000001800d681c     hb-aat-layout.obj
 0002:0002b83c       $unwind$??0accelerator_t@?$mortmorx@Umorx@AAT@@UExtendedTypes@2@$0GNGPHCHI@@AAT@@QEAA@PEAUhb_face_t@@@Z 00000001800d683c     hb-aat-layout.obj
 0002:0002b848       $chain$3$??0accelerator_t@?$mortmorx@Umorx@AAT@@UExtendedTypes@2@$0GNGPHCHI@@AAT@@QEAA@PEAUhb_face_t@@@Z 00000001800d6848     hb-aat-layout.obj
 0002:0002b868       $chain$4$??0accelerator_t@?$mortmorx@Umorx@AAT@@UExtendedTypes@2@$0GNGPHCHI@@AAT@@QEAA@PEAUhb_face_t@@@Z 00000001800d6868     hb-aat-layout.obj
 0002:0002b87c       $chain$5$??0accelerator_t@?$mortmorx@Umorx@AAT@@UExtendedTypes@2@$0GNGPHCHI@@AAT@@QEAA@PEAUhb_face_t@@@Z 00000001800d687c     hb-aat-layout.obj
 0002:0002b88c       $chain$6$??0accelerator_t@?$mortmorx@Umorx@AAT@@UExtendedTypes@2@$0GNGPHCHI@@AAT@@QEAA@PEAUhb_face_t@@@Z 00000001800d688c     hb-aat-layout.obj
 0002:0002b8a0       $chain$7$??0accelerator_t@?$mortmorx@Umorx@AAT@@UExtendedTypes@2@$0GNGPHCHI@@AAT@@QEAA@PEAUhb_face_t@@@Z 00000001800d68a0     hb-aat-layout.obj
 0002:0002b8b0       $unwind$??1accelerator_t@?$mortmorx@Umort@AAT@@UObsoleteTypes@2@$0GNGPHCHE@@AAT@@QEAA@XZ 00000001800d68b0     hb-aat-layout.obj
 0002:0002b8b0       $unwind$??1accelerator_t@?$mortmorx@Umorx@AAT@@UExtendedTypes@2@$0GNGPHCHI@@AAT@@QEAA@XZ 00000001800d68b0     hb-aat-layout.obj
 0002:0002b8bc       $chain$4$??1accelerator_t@?$mortmorx@Umort@AAT@@UObsoleteTypes@2@$0GNGPHCHE@@AAT@@QEAA@XZ 00000001800d68bc     hb-aat-layout.obj
 0002:0002b8bc       $chain$4$??1accelerator_t@?$mortmorx@Umorx@AAT@@UExtendedTypes@2@$0GNGPHCHI@@AAT@@QEAA@XZ 00000001800d68bc     hb-aat-layout.obj
 0002:0002b8e0       $chain$5$??1accelerator_t@?$mortmorx@Umort@AAT@@UObsoleteTypes@2@$0GNGPHCHE@@AAT@@QEAA@XZ 00000001800d68e0     hb-aat-layout.obj
 0002:0002b8e0       $chain$5$??1accelerator_t@?$mortmorx@Umorx@AAT@@UExtendedTypes@2@$0GNGPHCHI@@AAT@@QEAA@XZ 00000001800d68e0     hb-aat-layout.obj
 0002:0002b8f0       $unwind$?sanitize@?$StateTable@UObsoleteTypes@AAT@@X@AAT@@QEBA_NPEAUhb_sanitize_context_t@@PEAI@Z 00000001800d68f0     hb-aat-layout.obj
 0002:0002b908       $unwind$?sanitize@?$StateTable@UObsoleteTypes@AAT@@UEntryData@?$ContextualSubtable@UObsoleteTypes@AAT@@@2@@AAT@@QEBA_NPEAUhb_sanitize_context_t@@PEAI@Z 00000001800d6908     hb-aat-layout.obj
 0002:0002b908       $unwind$?sanitize@?$StateTable@UObsoleteTypes@AAT@@UEntryData@?$InsertionSubtable@UObsoleteTypes@AAT@@@2@@AAT@@QEBA_NPEAUhb_sanitize_context_t@@PEAI@Z 00000001800d6908     hb-aat-layout.obj
 0002:0002b920       $unwind$?apply@?$NoncontextualSubtable@UExtendedTypes@AAT@@@AAT@@QEBA_NPEAUhb_aat_apply_context_t@2@@Z 00000001800d6920     hb-aat-layout.obj
 0002:0002b920       $unwind$?apply@?$NoncontextualSubtable@UObsoleteTypes@AAT@@@AAT@@QEBA_NPEAUhb_aat_apply_context_t@2@@Z 00000001800d6920     hb-aat-layout.obj
 0002:0002b934       $chain$2$?apply@?$NoncontextualSubtable@UExtendedTypes@AAT@@@AAT@@QEBA_NPEAUhb_aat_apply_context_t@2@@Z 00000001800d6934     hb-aat-layout.obj
 0002:0002b934       $chain$2$?apply@?$NoncontextualSubtable@UObsoleteTypes@AAT@@@AAT@@QEBA_NPEAUhb_aat_apply_context_t@2@@Z 00000001800d6934     hb-aat-layout.obj
 0002:0002b94c       $chain$3$?apply@?$NoncontextualSubtable@UExtendedTypes@AAT@@@AAT@@QEBA_NPEAUhb_aat_apply_context_t@2@@Z 00000001800d694c     hb-aat-layout.obj
 0002:0002b94c       $chain$3$?apply@?$NoncontextualSubtable@UObsoleteTypes@AAT@@@AAT@@QEBA_NPEAUhb_aat_apply_context_t@2@@Z 00000001800d694c     hb-aat-layout.obj
 0002:0002b95c       $chain$1$?match_properties_mark@hb_ot_apply_context_t@OT@@QEBA_NIII@Z 00000001800d695c     hb-aat-layout.obj
 0002:0002b974       $chain$3$?match_properties_mark@hb_ot_apply_context_t@OT@@QEBA_NIII@Z 00000001800d6974     hb-aat-layout.obj
 0002:0002b98c       $chain$4$?match_properties_mark@hb_ot_apply_context_t@OT@@QEBA_NIII@Z 00000001800d698c     hb-aat-layout.obj
 0002:0002b99c       $unwind$??$dispatch@UAttachList@OT@@$$V@hb_sanitize_context_t@@QEAA_NAEBUAttachList@OT@@@Z 00000001800d699c     hb-aat-layout.obj
 0002:0002b99c       $unwind$??$dispatch@ULigCaretList@OT@@$$V@hb_sanitize_context_t@@QEAA_NAEBULigCaretList@OT@@@Z 00000001800d699c     hb-aat-layout.obj
 0002:0002b99c       $unwind$?sanitize@?$ChainContextFormat2_5@USmallTypes@Layout@OT@@@OT@@QEBA_NPEAUhb_sanitize_context_t@@@Z 00000001800d699c     hb-aat-layout.obj
 0002:0002b99c       $unwind$?sanitize@?$ContextFormat2_5@USmallTypes@Layout@OT@@@OT@@QEBA_NPEAUhb_sanitize_context_t@@@Z 00000001800d699c     hb-aat-layout.obj
 0002:0002b99c       $unwind$??$get_extents_without_var_scaled@Uglyf_accelerator_t@OT@@@GlyphHeader@glyf_impl@OT@@QEBA_NPEAUhb_font_t@@AEBUglyf_accelerator_t@2@IPEAUhb_glyph_extents_t@@@Z 00000001800d699c     hb-ot-font.obj
 0002:0002b99c       $unwind$?_apply@?$LigatureSubstFormat1_2@USmallTypes@Layout@OT@@@GSUB_impl@Layout@OT@@QEBA_NPEAUhb_ot_apply_context_t@4@_N@Z 00000001800d699c     hb-ot-layout.obj
 0002:0002b99c       $unwind$?sanitize_value_devices@ValueFormat@GPOS_impl@Layout@OT@@AEBA_NPEAUhb_sanitize_context_t@@PEBUValueBase@234@PEBU?$IntType@G$01@4@@Z 00000001800d699c     hb-ot-layout.obj
 0002:0002b99c       $unwind$??1hb_ot_map_builder_t@@QEAA@XZ 00000001800d699c     hb-ot-map.obj
 0002:0002b9b8       $unwind$??$dispatch@UClassDef@OT@@$$V@hb_sanitize_context_t@@QEAA_NAEBUClassDef@OT@@@Z 00000001800d69b8     hb-aat-layout.obj
 0002:0002b9b8       $unwind$?sanitize@?$ChainRule@USmallTypes@Layout@OT@@@OT@@QEBA_NPEAUhb_sanitize_context_t@@@Z 00000001800d69b8     hb-aat-layout.obj
 0002:0002b9d0       $unwind$?sanitize@ChainContextFormat3@OT@@QEBA_NPEAUhb_sanitize_context_t@@@Z 00000001800d69d0     hb-aat-layout.obj
 0002:0002b9d0       $unwind$?sanitize@ReverseChainSingleSubstFormat1@GSUB_impl@Layout@OT@@QEBA_NPEAUhb_sanitize_context_t@@@Z 00000001800d69d0     hb-aat-layout.obj
 0002:0002b9d0       $unwind$?get_anchor@AnchorFormat3@GPOS_impl@Layout@OT@@QEBAXPEAUhb_ot_apply_context_t@4@IPEAM1@Z 00000001800d69d0     hb-ot-layout.obj
 0002:0002b9d0       $unwind$hb_ot_layout_language_find_feature 00000001800d69d0     hb-ot-layout.obj
 0002:0002b9d0       $unwind$hb_ot_layout_table_select_script 00000001800d69d0     hb-ot-layout.obj
 0002:0002b9d0       $unwind$?add_pause@hb_ot_map_builder_t@@AEAAXIP6A_NPEBUhb_ot_shape_plan_t@@PEAUhb_font_t@@PEAUhb_buffer_t@@@Z@Z 00000001800d69d0     hb-ot-map.obj
 0002:0002b9d0       $unwind$??$serialize@U?$hb_sorted_array_t@$$CBUHBGlyphID16@OT@@@@$0A@@?$CoverageFormat2_4@USmallTypes@Layout@OT@@@Common@Layout@OT@@AEAA_NPEAUhb_serialize_context_t@@U?$hb_sorted_array_t@$$CBUHBGlyphID16@OT@@@@@Z 00000001800d69d0     hb-ot-shaper-arabic.obj
 0002:0002b9ec       $chain$0$?sanitize@?$Lookup@U?$IntType@I$03@OT@@@AAT@@QEBA_NPEAUhb_sanitize_context_t@@@Z 00000001800d69ec     hb-aat-layout.obj
 0002:0002ba00       $chain$2$?sanitize@?$Lookup@U?$IntType@I$03@OT@@@AAT@@QEBA_NPEAUhb_sanitize_context_t@@@Z 00000001800d6a00     hb-aat-layout.obj
 0002:0002ba14       $chain$3$?sanitize@?$Lookup@U?$IntType@I$03@OT@@@AAT@@QEBA_NPEAUhb_sanitize_context_t@@@Z 00000001800d6a14     hb-aat-layout.obj
 0002:0002ba24       $chain$0$?get_value@?$LookupFormat4@U?$IntType@I$03@OT@@@AAT@@AEBAPEBU?$IntType@I$03@OT@@I@Z 00000001800d6a24     hb-aat-layout.obj
 0002:0002ba38       $chain$1$?get_value@?$LookupFormat4@U?$IntType@I$03@OT@@@AAT@@AEBAPEBU?$IntType@I$03@OT@@I@Z 00000001800d6a38     hb-aat-layout.obj
 0002:0002ba4c       $chain$2$?get_value@?$LookupFormat4@U?$IntType@I$03@OT@@@AAT@@AEBAPEBU?$IntType@I$03@OT@@I@Z 00000001800d6a4c     hb-aat-layout.obj
 0002:0002ba5c       $chain$3$?get_value@?$LookupFormat4@U?$IntType@I$03@OT@@@AAT@@AEBAPEBU?$IntType@I$03@OT@@I@Z 00000001800d6a5c     hb-aat-layout.obj
 0002:0002ba6c       $chain$4$?sanitize@?$LookupFormat4@U?$IntType@I$03@OT@@@AAT@@AEBA_NPEAUhb_sanitize_context_t@@@Z 00000001800d6a6c     hb-aat-layout.obj
 0002:0002ba90       $chain$6$?sanitize@?$LookupFormat4@U?$IntType@I$03@OT@@@AAT@@AEBA_NPEAUhb_sanitize_context_t@@@Z 00000001800d6a90     hb-aat-layout.obj
 0002:0002bab4       $unwind$?sanitize@?$StateTable@UExtendedTypes@AAT@@UEntryData@?$ContextualSubtable@UExtendedTypes@AAT@@@2@@AAT@@QEBA_NPEAUhb_sanitize_context_t@@PEAI@Z 00000001800d6ab4     hb-aat-layout.obj
 0002:0002bab4       $unwind$?sanitize@?$StateTable@UExtendedTypes@AAT@@UEntryData@?$Format1Entry@$00@2@@AAT@@QEBA_NPEAUhb_sanitize_context_t@@PEAI@Z 00000001800d6ab4     hb-aat-layout.obj
 0002:0002bab4       $unwind$?sanitize@?$StateTable@UExtendedTypes@AAT@@UEntryData@?$InsertionSubtable@UExtendedTypes@AAT@@@2@@AAT@@QEBA_NPEAUhb_sanitize_context_t@@PEAI@Z 00000001800d6ab4     hb-aat-layout.obj
 0002:0002bab4       $unwind$?sanitize@?$StateTable@UExtendedTypes@AAT@@UEntryData@?$KerxSubTableFormat4@UKerxSubTableHeader@AAT@@@2@@AAT@@QEBA_NPEAUhb_sanitize_context_t@@PEAI@Z 00000001800d6ab4     hb-aat-layout.obj
 0002:0002bab4       $unwind$?sanitize@?$StateTable@UExtendedTypes@AAT@@UEntryData@?$LigatureEntry@$00@2@@AAT@@QEBA_NPEAUhb_sanitize_context_t@@PEAI@Z 00000001800d6ab4     hb-aat-layout.obj
 0002:0002bacc       $chain$2$?shrink_vector@?$hb_vector_t@Ukern_subtable_accelerator_data_t@AAT@@$0A@@@QEAAXI@Z 00000001800d6acc     hb-aat-layout.obj
 0002:0002bae8       $chain$3$?shrink_vector@?$hb_vector_t@Ukern_subtable_accelerator_data_t@AAT@@$0A@@@QEAAXI@Z 00000001800d6ae8     hb-aat-layout.obj
 0002:0002baf8       $unwind$?apply@?$KerxTable@Ukerx@AAT@@@AAT@@QEBA_NPEAUhb_aat_apply_context_t@2@AEBUkern_accelerator_data_t@2@@Z 00000001800d6af8     hb-aat-layout.obj
 0002:0002bb0c       $chain$0$?apply@?$KerxTable@Ukerx@AAT@@@AAT@@QEBA_NPEAUhb_aat_apply_context_t@2@AEBUkern_accelerator_data_t@2@@Z 00000001800d6b0c     hb-aat-layout.obj
 0002:0002bb20       $chain$1$?apply@?$KerxTable@Ukerx@AAT@@@AAT@@QEBA_NPEAUhb_aat_apply_context_t@2@AEBUkern_accelerator_data_t@2@@Z 00000001800d6b20     hb-aat-layout.obj
 0002:0002bb30       $chain$2$?apply@?$KerxTable@Ukerx@AAT@@@AAT@@QEBA_NPEAUhb_aat_apply_context_t@2@AEBUkern_accelerator_data_t@2@@Z 00000001800d6b30     hb-aat-layout.obj
 0002:0002bb44       $unwind$?create_accelerator_data@?$KerxTable@Ukerx@AAT@@@AAT@@QEBA?AUkern_accelerator_data_t@2@I@Z 00000001800d6b44     hb-aat-layout.obj
 0002:0002bb44       $unwind$?create_accelerator_data@?$KerxTable@UKernAAT@OT@@@AAT@@QEBA?AUkern_accelerator_data_t@2@I@Z 00000001800d6b44     hb-ot-layout.obj
 0002:0002bb44       $unwind$?create_accelerator_data@?$KerxTable@UKernOT@OT@@@AAT@@QEBA?AUkern_accelerator_data_t@2@I@Z 00000001800d6b44     hb-ot-layout.obj
 0002:0002bb5c       $unwind$??0accelerator_t@?$KerxTable@Ukerx@AAT@@@AAT@@QEAA@PEAUhb_face_t@@@Z 00000001800d6b5c     hb-aat-layout.obj
 0002:0002bb70       $unwind$?get_value@TrackTableEntry@AAT@@QEBAMMPEBXU?$hb_array_t@$$CBU?$HBFixed@U?$IntType@H$03@OT@@$0BA@@OT@@@@@Z 00000001800d6b70     hb-aat-layout.obj
 0002:0002bb70       $unwind$?cmp_gids@accelerator_t@post@OT@@KAHPEBX0PEAX@Z 00000001800d6b70     hb-ot-font.obj
 0002:0002bb70       $unwind$?push_font_transform@hb_paint_funcs_t@@QEAAXPEAXPEBUhb_font_t@@@Z 00000001800d6b70     hb-ot-font.obj
 0002:0002bb70       $unwind$?push_inverse_font_transform@hb_paint_funcs_t@@QEAAXPEAXPEBUhb_font_t@@@Z 00000001800d6b70     hb-ot-font.obj
 0002:0002bb80       $unwind$?get_tracking@TrackData@AAT@@QEBAMPEBXMM@Z 00000001800d6b80     hb-aat-layout.obj
 0002:0002bb98       $chain$1$?get_tracking@TrackData@AAT@@QEBAMPEBXMM@Z 00000001800d6b98     hb-aat-layout.obj
 0002:0002bbb0       $chain$5$?get_tracking@TrackData@AAT@@QEBAMPEBXMM@Z 00000001800d6bb0     hb-aat-layout.obj
 0002:0002bbd0       $chain$6$?get_tracking@TrackData@AAT@@QEBAMPEBXMM@Z 00000001800d6bd0     hb-aat-layout.obj
 0002:0002bbe0       $chain$7$?get_tracking@TrackData@AAT@@QEBAMPEBXMM@Z 00000001800d6be0     hb-aat-layout.obj
 0002:0002bbf0       $unwind$?sanitize@TrackData@AAT@@QEBA_NPEAUhb_sanitize_context_t@@PEBX@Z 00000001800d6bf0     hb-aat-layout.obj
 0002:0002bc0c       $chain$1$?sanitize_shallow@?$UnsizedArrayOf@UTrackTableEntry@AAT@@@OT@@QEBA_NPEAUhb_sanitize_context_t@@I@Z 00000001800d6c0c     hb-aat-layout.obj
 0002:0002bc0c       $chain$1$?sanitize_shallow@?$UnsizedArrayOf@UIndexSubtableRecord@OT@@@OT@@QEBA_NPEAUhb_sanitize_context_t@@I@Z 00000001800d6c0c     hb-ot-color.obj
 0002:0002bc0c       $chain$1$?sanitize_shallow@?$UnsizedArrayOf@UStatAxisRecord@OT@@@OT@@QEBA_NPEAUhb_sanitize_context_t@@I@Z 00000001800d6c0c     hb-ot-shape.obj
 0002:0002bc24       $chain$2$?sanitize_shallow@?$UnsizedArrayOf@UTrackTableEntry@AAT@@@OT@@QEBA_NPEAUhb_sanitize_context_t@@I@Z 00000001800d6c24     hb-aat-layout.obj
 0002:0002bc24       $chain$2$?sanitize_shallow@?$UnsizedArrayOf@UIndexSubtableRecord@OT@@@OT@@QEBA_NPEAUhb_sanitize_context_t@@I@Z 00000001800d6c24     hb-ot-color.obj
 0002:0002bc24       $chain$2$?sanitize_shallow@?$UnsizedArrayOf@UStatAxisRecord@OT@@@OT@@QEBA_NPEAUhb_sanitize_context_t@@I@Z 00000001800d6c24     hb-ot-shape.obj
 0002:0002bc34       $unwind$?apply@trak@AAT@@QEBA_NPEAUhb_aat_apply_context_t@2@M@Z 00000001800d6c34     hb-aat-layout.obj
 0002:0002bc34       $unwind$?thai_pua_shape@@YAIIW4thai_action_t@@PEAUhb_font_t@@@Z 00000001800d6c34     hb-ot-shaper-thai.obj
 0002:0002bc44       $unwind$??0?$accelerator_t@UGSUB@Layout@OT@@@GSUBGPOS@OT@@QEAA@PEAUhb_face_t@@@Z 00000001800d6c44     hb-aat-layout.obj
 0002:0002bc44       $unwind$hb_face_create_or_fail 00000001800d6c44     hb-face.obj
 0002:0002bc5c       $unwind$??1?$accelerator_t@UGSUB@Layout@OT@@@GSUBGPOS@OT@@QEAA@XZ 00000001800d6c5c     hb-aat-layout.obj
 0002:0002bc5c       $unwind$??1?$accelerator_t@UGPOS@Layout@OT@@@GSUBGPOS@OT@@QEAA@XZ 00000001800d6c5c     hb-ot-layout.obj
 0002:0002bc5c       $unwind$??$extend_min@U?$CoverageFormat2_4@USmallTypes@Layout@OT@@@Common@Layout@OT@@@hb_serialize_context_t@@QEAAPEAU?$CoverageFormat2_4@USmallTypes@Layout@OT@@@Common@Layout@OT@@PEAU1234@@Z 00000001800d6c5c     hb-ot-shaper-arabic.obj
 0002:0002bc5c       $unwind$??$extend_min@U?$IntType@G$01@OT@@@hb_serialize_context_t@@QEAAPEAU?$IntType@G$01@OT@@AEAU12@@Z 00000001800d6c5c     hb-ot-shaper-arabic.obj
 0002:0002bc5c       $unwind$??$extend_min@U?$Ligature@USmallTypes@Layout@OT@@@GSUB_impl@Layout@OT@@@hb_serialize_context_t@@QEAAPEAU?$Ligature@USmallTypes@Layout@OT@@@GSUB_impl@Layout@OT@@PEAU1234@@Z 00000001800d6c5c     hb-ot-shaper-arabic.obj
 0002:0002bc5c       $unwind$??$extend_min@U?$LigatureSet@USmallTypes@Layout@OT@@@GSUB_impl@Layout@OT@@@hb_serialize_context_t@@QEAAPEAU?$LigatureSet@USmallTypes@Layout@OT@@@GSUB_impl@Layout@OT@@PEAU1234@@Z 00000001800d6c5c     hb-ot-shaper-arabic.obj
 0002:0002bc5c       $unwind$??$extend_min@U?$LigatureSubstFormat1_2@USmallTypes@Layout@OT@@@GSUB_impl@Layout@OT@@@hb_serialize_context_t@@QEAAPEAU?$LigatureSubstFormat1_2@USmallTypes@Layout@OT@@@GSUB_impl@Layout@OT@@PEAU1234@@Z 00000001800d6c5c     hb-ot-shaper-arabic.obj
 0002:0002bc5c       $unwind$??$extend_min@U?$SingleSubstFormat1_3@USmallTypes@Layout@OT@@@GSUB_impl@Layout@OT@@@hb_serialize_context_t@@QEAAPEAU?$SingleSubstFormat1_3@USmallTypes@Layout@OT@@@GSUB_impl@Layout@OT@@PEAU1234@@Z 00000001800d6c5c     hb-ot-shaper-arabic.obj
 0002:0002bc5c       $unwind$??$extend_min@U?$SingleSubstFormat2_4@USmallTypes@Layout@OT@@@GSUB_impl@Layout@OT@@@hb_serialize_context_t@@QEAAPEAU?$SingleSubstFormat2_4@USmallTypes@Layout@OT@@@GSUB_impl@Layout@OT@@PEAU1234@@Z 00000001800d6c5c     hb-ot-shaper-arabic.obj
 0002:0002bc5c       $unwind$??$extend_min@UCoverage@Common@Layout@OT@@@hb_serialize_context_t@@QEAAPEAUCoverage@Common@Layout@OT@@PEAU1234@@Z 00000001800d6c5c     hb-ot-shaper-arabic.obj
 0002:0002bc5c       $unwind$??$extend_min@ULookup@OT@@@hb_serialize_context_t@@QEAAPEAULookup@OT@@PEAU12@@Z 00000001800d6c5c     hb-ot-shaper-arabic.obj
 0002:0002bc68       $chain$0$??1?$accelerator_t@UGSUB@Layout@OT@@@GSUBGPOS@OT@@QEAA@XZ 00000001800d6c68     hb-aat-layout.obj
 0002:0002bc68       $chain$0$??1?$accelerator_t@UGPOS@Layout@OT@@@GSUBGPOS@OT@@QEAA@XZ 00000001800d6c68     hb-ot-layout.obj
 0002:0002bc7c       $chain$1$??1?$accelerator_t@UGSUB@Layout@OT@@@GSUBGPOS@OT@@QEAA@XZ 00000001800d6c7c     hb-aat-layout.obj
 0002:0002bc7c       $chain$1$??1?$accelerator_t@UGPOS@Layout@OT@@@GSUBGPOS@OT@@QEAA@XZ 00000001800d6c7c     hb-ot-layout.obj
 0002:0002bc8c       $chain$1$??$check_array@U?$Entry@X@AAT@@@hb_sanitize_context_t@@QEBA_NPEBU?$Entry@X@AAT@@I@Z 00000001800d6c8c     hb-aat-layout.obj
 0002:0002bc8c       $chain$1$??$check_array@U?$IntType@I$03@OT@@@hb_sanitize_context_t@@QEBA_NPEBU?$IntType@I$03@OT@@I@Z 00000001800d6c8c     hb-common.obj
 0002:0002bca4       $chain$2$??$check_array@U?$Entry@X@AAT@@@hb_sanitize_context_t@@QEBA_NPEBU?$Entry@X@AAT@@I@Z 00000001800d6ca4     hb-aat-layout.obj
 0002:0002bca4       $chain$2$??$check_array@U?$IntType@I$03@OT@@@hb_sanitize_context_t@@QEBA_NPEBU?$IntType@I$03@OT@@I@Z 00000001800d6ca4     hb-common.obj
 0002:0002bcb4       $chain$0$??$dispatch@Uhb_sanitize_context_t@@$$V@?$ChainSubtable@UObsoleteTypes@AAT@@@AAT@@QEBA_NPEAUhb_sanitize_context_t@@@Z 00000001800d6cb4     hb-aat-layout.obj
 0002:0002bcc8       $chain$2$??$dispatch@Uhb_sanitize_context_t@@$$V@?$ChainSubtable@UObsoleteTypes@AAT@@@AAT@@QEBA_NPEAUhb_sanitize_context_t@@@Z 00000001800d6cc8     hb-aat-layout.obj
 0002:0002bcc8       $chain$4$??$dispatch@Uhb_sanitize_context_t@@$$V@?$ChainSubtable@UObsoleteTypes@AAT@@@AAT@@QEBA_NPEAUhb_sanitize_context_t@@@Z 00000001800d6cc8     hb-aat-layout.obj
 0002:0002bcdc       $chain$7$??$dispatch@Uhb_sanitize_context_t@@$$V@?$ChainSubtable@UObsoleteTypes@AAT@@@AAT@@QEBA_NPEAUhb_sanitize_context_t@@@Z 00000001800d6cdc     hb-aat-layout.obj
 0002:0002bcf4       $chain$9$??$dispatch@Uhb_sanitize_context_t@@$$V@?$ChainSubtable@UObsoleteTypes@AAT@@@AAT@@QEBA_NPEAUhb_sanitize_context_t@@@Z 00000001800d6cf4     hb-aat-layout.obj
 0002:0002bd0c       $chain$10$??$dispatch@Uhb_sanitize_context_t@@$$V@?$ChainSubtable@UObsoleteTypes@AAT@@@AAT@@QEBA_NPEAUhb_sanitize_context_t@@@Z 00000001800d6d0c     hb-aat-layout.obj
 0002:0002bd1c       $chain$0$??$collect_glyphs@Uhb_bit_set_t@@@KerxSubTable@AAT@@QEBAXAEAUhb_bit_set_t@@0I@Z 00000001800d6d1c     hb-aat-layout.obj
 0002:0002bd30       $chain$1$??$collect_glyphs@Uhb_bit_set_t@@@KerxSubTable@AAT@@QEBAXAEAUhb_bit_set_t@@0I@Z 00000001800d6d30     hb-aat-layout.obj
 0002:0002bd40       $unwind$??$dispatch@Uhb_aat_apply_context_t@AAT@@$$V@KerxSubTable@AAT@@QEBA_NPEAUhb_aat_apply_context_t@1@@Z 00000001800d6d40     hb-aat-layout.obj
 0002:0002bd40       $unwind$??$dispatch@Uhb_aat_apply_context_t@AAT@@$$V@?$KernSubTable@UKernAATSubTableHeader@OT@@@OT@@QEBA_NPEAUhb_aat_apply_context_t@AAT@@@Z 00000001800d6d40     hb-ot-layout.obj
 0002:0002bd40       $unwind$??$dispatch@Uhb_aat_apply_context_t@AAT@@$$V@?$KernSubTable@UKernOTSubTableHeader@OT@@@OT@@QEBA_NPEAUhb_aat_apply_context_t@AAT@@@Z 00000001800d6d40     hb-ot-layout.obj
 0002:0002bd58       $unwind$?sanitize@?$StateTable@UExtendedTypes@AAT@@X@AAT@@QEBA_NPEAUhb_sanitize_context_t@@PEAI@Z 00000001800d6d58     hb-aat-layout.obj
 0002:0002bd70       $unwind$??$dispatch@Uhb_aat_apply_context_t@AAT@@$$V@?$ChainSubtable@UExtendedTypes@AAT@@@AAT@@QEBA_NPEAUhb_aat_apply_context_t@1@@Z 00000001800d6d70     hb-aat-layout.obj
 0002:0002bd70       $unwind$??$dispatch@Uhb_aat_apply_context_t@AAT@@$$V@?$ChainSubtable@UObsoleteTypes@AAT@@@AAT@@QEBA_NPEAUhb_aat_apply_context_t@1@@Z 00000001800d6d70     hb-aat-layout.obj
 0002:0002bd88       $unwind$??$realloc_vector@Ukern_subtable_accelerator_data_t@AAT@@$0A@@?$hb_vector_t@Ukern_subtable_accelerator_data_t@AAT@@$0A@@@QEAAPEAUkern_subtable_accelerator_data_t@AAT@@IU?$hb_priority@$0A@@@@Z 00000001800d6d88     hb-aat-layout.obj
 0002:0002bd94       $chain$2$??$realloc_vector@Ukern_subtable_accelerator_data_t@AAT@@$0A@@?$hb_vector_t@Ukern_subtable_accelerator_data_t@AAT@@$0A@@@QEAAPEAUkern_subtable_accelerator_data_t@AAT@@IU?$hb_priority@$0A@@@@Z 00000001800d6d94     hb-aat-layout.obj
 0002:0002bdac       $chain$6$??$realloc_vector@Ukern_subtable_accelerator_data_t@AAT@@$0A@@?$hb_vector_t@Ukern_subtable_accelerator_data_t@AAT@@$0A@@@QEAAPEAUkern_subtable_accelerator_data_t@AAT@@IU?$hb_priority@$0A@@@@Z 00000001800d6dac     hb-aat-layout.obj
 0002:0002bdcc       $chain$7$??$realloc_vector@Ukern_subtable_accelerator_data_t@AAT@@$0A@@?$hb_vector_t@Ukern_subtable_accelerator_data_t@AAT@@$0A@@@QEAAPEAUkern_subtable_accelerator_data_t@AAT@@IU?$hb_priority@$0A@@@@Z 00000001800d6dcc     hb-aat-layout.obj
 0002:0002bddc       $chain$8$??$realloc_vector@Ukern_subtable_accelerator_data_t@AAT@@$0A@@?$hb_vector_t@Ukern_subtable_accelerator_data_t@AAT@@$0A@@@QEAAPEAUkern_subtable_accelerator_data_t@AAT@@IU?$hb_priority@$0A@@@@Z 00000001800d6ddc     hb-aat-layout.obj
 0002:0002bdec       $unwind$??$dispatch@UConditionSet@OT@@$$V@hb_sanitize_context_t@@QEAA_NAEBUConditionSet@OT@@@Z 00000001800d6dec     hb-aat-layout.obj
 0002:0002bdf8       $chain$2$??$dispatch@UConditionSet@OT@@$$V@hb_sanitize_context_t@@QEAA_NAEBUConditionSet@OT@@@Z 00000001800d6df8     hb-aat-layout.obj
 0002:0002be14       $chain$4$??$dispatch@UConditionSet@OT@@$$V@hb_sanitize_context_t@@QEAA_NAEBUConditionSet@OT@@@Z 00000001800d6e14     hb-aat-layout.obj
 0002:0002be30       $unwind$??$sanitize_blob@UGDEF@OT@@@hb_sanitize_context_t@@QEAAPEAUhb_blob_t@@PEAU1@@Z 00000001800d6e30     hb-aat-layout.obj
 0002:0002be4c       $unwind$??$collect_coverage@Uhb_set_digest_t@@@MarkGlyphSetsFormat1@OT@@QEBAXAEAU?$hb_vector_t@Uhb_set_digest_t@@$0A@@@@Z 00000001800d6e4c     hb-aat-layout.obj
 0002:0002be5c       $chain$3$??$collect_coverage@Uhb_set_digest_t@@@MarkGlyphSetsFormat1@OT@@QEBAXAEAU?$hb_vector_t@Uhb_set_digest_t@@$0A@@@@Z 00000001800d6e5c     hb-aat-layout.obj
 0002:0002be7c       $chain$4$??$collect_coverage@Uhb_set_digest_t@@@MarkGlyphSetsFormat1@OT@@QEBAXAEAU?$hb_vector_t@Uhb_set_digest_t@@$0A@@@@Z 00000001800d6e7c     hb-aat-layout.obj
 0002:0002be8c       $unwind$??$add_array@I@hb_bit_set_t@@QEAAXPEBIII@Z 00000001800d6e8c     hb-aat-layout.obj
 0002:0002be8c       $unwind$??$add_array@UHBGlyphID16@OT@@@hb_bit_set_t@@QEAAXPEBUHBGlyphID16@OT@@II@Z 00000001800d6e8c     hb-aat-layout.obj
 0002:0002be9c       $chain$3$??$add_array@I@hb_bit_set_t@@QEAAXPEBIII@Z 00000001800d6e9c     hb-aat-layout.obj
 0002:0002bebc       $chain$4$??$add_array@I@hb_bit_set_t@@QEAAXPEBIII@Z 00000001800d6ebc     hb-aat-layout.obj
 0002:0002becc       $unwind$??$sanitize_blob@UGSUB@Layout@OT@@@hb_sanitize_context_t@@QEAAPEAUhb_blob_t@@PEAU1@@Z 00000001800d6ecc     hb-aat-layout.obj
 0002:0002becc       $unwind$??$sanitize_blob@Utrak@AAT@@@hb_sanitize_context_t@@QEAAPEAUhb_blob_t@@PEAU1@@Z 00000001800d6ecc     hb-aat-layout.obj
 0002:0002becc       $unwind$??$sanitize_blob@UGPOS@Layout@OT@@@hb_sanitize_context_t@@QEAAPEAUhb_blob_t@@PEAU1@@Z 00000001800d6ecc     hb-ot-layout.obj
 0002:0002bee8       $unwind$??$sanitize_blob@Ukerx@AAT@@@hb_sanitize_context_t@@QEAAPEAUhb_blob_t@@PEAU1@@Z 00000001800d6ee8     hb-aat-layout.obj
 0002:0002bee8       $unwind$??$sanitize_blob@U?$gvar_GVAR@U?$IntType@G$01@OT@@$0GHHGGBHC@@OT@@@hb_sanitize_context_t@@QEAAPEAUhb_blob_t@@PEAU1@@Z 00000001800d6ee8     hb-common.obj
 0002:0002bee8       $unwind$??$sanitize_blob@UHVAR@OT@@@hb_sanitize_context_t@@QEAAPEAUhb_blob_t@@PEAU1@@Z 00000001800d6ee8     hb-common.obj
 0002:0002bee8       $unwind$??$sanitize_blob@UOS2@OT@@@hb_sanitize_context_t@@QEAAPEAUhb_blob_t@@PEAU1@@Z 00000001800d6ee8     hb-face.obj
 0002:0002bee8       $unwind$??$sanitize_blob@UOpenTypeFontFile@OT@@@hb_sanitize_context_t@@QEAAPEAUhb_blob_t@@PEAU1@@Z 00000001800d6ee8     hb-face.obj
 0002:0002bee8       $unwind$??$sanitize_blob@Ucmap@OT@@@hb_sanitize_context_t@@QEAAPEAUhb_blob_t@@PEAU1@@Z 00000001800d6ee8     hb-face.obj
 0002:0002bee8       $unwind$??$sanitize_blob@Uavar@OT@@@hb_sanitize_context_t@@QEAAPEAUhb_blob_t@@PEAU1@@Z 00000001800d6ee8     hb-font.obj
 0002:0002bee8       $unwind$??$sanitize_blob@Ufvar@OT@@@hb_sanitize_context_t@@QEAAPEAUhb_blob_t@@PEAU1@@Z 00000001800d6ee8     hb-font.obj
 0002:0002bee8       $unwind$??$sanitize_blob@UCOLR@OT@@@hb_sanitize_context_t@@QEAAPEAUhb_blob_t@@PEAU1@@Z 00000001800d6ee8     hb-ot-color.obj
 0002:0002bee8       $unwind$??$sanitize_blob@UCPAL@OT@@@hb_sanitize_context_t@@QEAAPEAUhb_blob_t@@PEAU1@@Z 00000001800d6ee8     hb-ot-color.obj
 0002:0002bf00       $unwind$??$sanitize_blob@Umort@AAT@@@hb_sanitize_context_t@@QEAAPEAUhb_blob_t@@PEAU1@@Z 00000001800d6f00     hb-aat-layout.obj
 0002:0002bf18       $unwind$??$dispatch@UMarkGlyphSets@OT@@$$V@hb_sanitize_context_t@@QEAA_NAEBUMarkGlyphSets@OT@@@Z 00000001800d6f18     hb-aat-layout.obj
 0002:0002bf18       $unwind$??$collect_glyphs@Uhb_bit_set_t@@@?$KernSubTable@UKernAATSubTableHeader@OT@@@OT@@QEBAXAEAUhb_bit_set_t@@0I@Z 00000001800d6f18     hb-ot-layout.obj
 0002:0002bf18       $unwind$??$collect_glyphs@Uhb_bit_set_t@@@?$KernSubTable@UKernOTSubTableHeader@OT@@@OT@@QEBAXAEAUhb_bit_set_t@@0I@Z 00000001800d6f18     hb-ot-layout.obj
 0002:0002bf2c       $chain$0$??$dispatch@UMarkGlyphSets@OT@@$$V@hb_sanitize_context_t@@QEAA_NAEBUMarkGlyphSets@OT@@@Z 00000001800d6f2c     hb-aat-layout.obj
 0002:0002bf40       $chain$1$??$dispatch@UMarkGlyphSets@OT@@$$V@hb_sanitize_context_t@@QEAA_NAEBUMarkGlyphSets@OT@@@Z 00000001800d6f40     hb-aat-layout.obj
 0002:0002bf50       $chain$2$??$dispatch@UMarkGlyphSets@OT@@$$V@hb_sanitize_context_t@@QEAA_NAEBUMarkGlyphSets@OT@@@Z 00000001800d6f50     hb-aat-layout.obj
 0002:0002bf64       $chain$3$??$add_array@UHBGlyphID16@OT@@@hb_bit_set_t@@QEAAXPEBUHBGlyphID16@OT@@II@Z 00000001800d6f64     hb-aat-layout.obj
 0002:0002bf84       $chain$4$??$add_array@UHBGlyphID16@OT@@@hb_bit_set_t@@QEAAXPEBUHBGlyphID16@OT@@II@Z 00000001800d6f84     hb-aat-layout.obj
 0002:0002bf94       $unwind$??$collect_initial_glyphs@Uhb_bit_set_t@@U?$ContextualSubtable@UExtendedTypes@AAT@@@AAT@@@?$StateTable@UExtendedTypes@AAT@@UEntryData@?$ContextualSubtable@UExtendedTypes@AAT@@@2@@AAT@@QEBAXAEAUhb_bit_set_t@@IAEBU?$ContextualSubtable@UExtendedTypes@AAT@@@1@@Z 00000001800d6f94     hb-aat-layout.obj
 0002:0002bf94       $unwind$??$collect_initial_glyphs@Uhb_bit_set_t@@U?$KerxSubTableFormat1@UKerxSubTableHeader@AAT@@@AAT@@@?$StateTable@UExtendedTypes@AAT@@UEntryData@?$Format1Entry@$00@2@@AAT@@QEBAXAEAUhb_bit_set_t@@IAEBU?$KerxSubTableFormat1@UKerxSubTableHeader@AAT@@@1@@Z 00000001800d6f94     hb-aat-layout.obj
 0002:0002bf94       $unwind$??$collect_initial_glyphs@Uhb_bit_set_t@@U?$KerxSubTableFormat4@UKerxSubTableHeader@AAT@@@AAT@@@?$StateTable@UExtendedTypes@AAT@@UEntryData@?$KerxSubTableFormat4@UKerxSubTableHeader@AAT@@@2@@AAT@@QEBAXAEAUhb_bit_set_t@@IAEBU?$KerxSubTableFormat4@UKerxSubTableHeader@AAT@@@1@@Z 00000001800d6f94     hb-aat-layout.obj
 0002:0002bf94       $unwind$??$collect_initial_glyphs@Uhb_bit_set_t@@U?$LigatureSubtable@UExtendedTypes@AAT@@@AAT@@@?$StateTable@UExtendedTypes@AAT@@UEntryData@?$LigatureEntry@$00@2@@AAT@@QEBAXAEAUhb_bit_set_t@@IAEBU?$LigatureSubtable@UExtendedTypes@AAT@@@1@@Z 00000001800d6f94     hb-aat-layout.obj
 0002:0002bfac       $chain$0$??$collect_initial_glyphs@Uhb_bit_set_t@@U?$KerxSubTableFormat1@UKerxSubTableHeader@AAT@@@AAT@@@?$StateTable@UExtendedTypes@AAT@@UEntryData@?$Format1Entry@$00@2@@AAT@@QEBAXAEAUhb_bit_set_t@@IAEBU?$KerxSubTableFormat1@UKerxSubTableHeader@AAT@@@1@@Z 00000001800d6fac     hb-aat-layout.obj
 0002:0002bfac       $chain$0$??$collect_initial_glyphs@Uhb_bit_set_t@@U?$KerxSubTableFormat4@UKerxSubTableHeader@AAT@@@AAT@@@?$StateTable@UExtendedTypes@AAT@@UEntryData@?$KerxSubTableFormat4@UKerxSubTableHeader@AAT@@@2@@AAT@@QEBAXAEAUhb_bit_set_t@@IAEBU?$KerxSubTableFormat4@UKerxSubTableHeader@AAT@@@1@@Z 00000001800d6fac     hb-aat-layout.obj
 0002:0002bfc0       $chain$4$??$collect_initial_glyphs@Uhb_bit_set_t@@U?$KerxSubTableFormat1@UKerxSubTableHeader@AAT@@@AAT@@@?$StateTable@UExtendedTypes@AAT@@UEntryData@?$Format1Entry@$00@2@@AAT@@QEBAXAEAUhb_bit_set_t@@IAEBU?$KerxSubTableFormat1@UKerxSubTableHeader@AAT@@@1@@Z 00000001800d6fc0     hb-aat-layout.obj
 0002:0002bfc0       $chain$4$??$collect_initial_glyphs@Uhb_bit_set_t@@U?$KerxSubTableFormat4@UKerxSubTableHeader@AAT@@@AAT@@@?$StateTable@UExtendedTypes@AAT@@UEntryData@?$KerxSubTableFormat4@UKerxSubTableHeader@AAT@@@2@@AAT@@QEBAXAEAUhb_bit_set_t@@IAEBU?$KerxSubTableFormat4@UKerxSubTableHeader@AAT@@@1@@Z 00000001800d6fc0     hb-aat-layout.obj
 0002:0002bfe0       $chain$5$??$collect_initial_glyphs@Uhb_bit_set_t@@U?$KerxSubTableFormat1@UKerxSubTableHeader@AAT@@@AAT@@@?$StateTable@UExtendedTypes@AAT@@UEntryData@?$Format1Entry@$00@2@@AAT@@QEBAXAEAUhb_bit_set_t@@IAEBU?$KerxSubTableFormat1@UKerxSubTableHeader@AAT@@@1@@Z 00000001800d6fe0     hb-aat-layout.obj
 0002:0002bfe0       $chain$5$??$collect_initial_glyphs@Uhb_bit_set_t@@U?$KerxSubTableFormat4@UKerxSubTableHeader@AAT@@@AAT@@@?$StateTable@UExtendedTypes@AAT@@UEntryData@?$KerxSubTableFormat4@UKerxSubTableHeader@AAT@@@2@@AAT@@QEBAXAEAUhb_bit_set_t@@IAEBU?$KerxSubTableFormat4@UKerxSubTableHeader@AAT@@@1@@Z 00000001800d6fe0     hb-aat-layout.obj
 0002:0002bff0       $chain$6$??$collect_initial_glyphs@Uhb_bit_set_t@@U?$KerxSubTableFormat1@UKerxSubTableHeader@AAT@@@AAT@@@?$StateTable@UExtendedTypes@AAT@@UEntryData@?$Format1Entry@$00@2@@AAT@@QEBAXAEAUhb_bit_set_t@@IAEBU?$KerxSubTableFormat1@UKerxSubTableHeader@AAT@@@1@@Z 00000001800d6ff0     hb-aat-layout.obj
 0002:0002bff0       $chain$6$??$collect_initial_glyphs@Uhb_bit_set_t@@U?$KerxSubTableFormat4@UKerxSubTableHeader@AAT@@@AAT@@@?$StateTable@UExtendedTypes@AAT@@UEntryData@?$KerxSubTableFormat4@UKerxSubTableHeader@AAT@@@2@@AAT@@QEBAXAEAUhb_bit_set_t@@IAEBU?$KerxSubTableFormat4@UKerxSubTableHeader@AAT@@@1@@Z 00000001800d6ff0     hb-aat-layout.obj
 0002:0002c000       $unwind$??$collect_glyphs@Uhb_bit_set_t@@@?$Lookup@U?$IntType@G$01@OT@@@AAT@@QEBAXAEAUhb_bit_set_t@@I@Z 00000001800d7000     hb-aat-layout.obj
 0002:0002c000       $unwind$??$collect_glyphs@Uhb_bit_set_t@@@?$Lookup@U?$IntType@I$03@OT@@@AAT@@QEBAXAEAUhb_bit_set_t@@I@Z 00000001800d7000     hb-aat-layout.obj
 0002:0002c000       $unwind$??$collect_glyphs@Uhb_bit_set_t@@@?$Lookup@UHBGlyphID16@OT@@@AAT@@QEBAXAEAUhb_bit_set_t@@I@Z 00000001800d7000     hb-aat-layout.obj
 0002:0002c000       $unwind$?hb_form_clusters@@YAXPEAUhb_buffer_t@@@Z 00000001800d7000     hb-ot-shape.obj
 0002:0002c000       $unwind$?hb_ot_substitute_default@@YAXPEBUhb_ot_shape_context_t@@@Z 00000001800d7000     hb-ot-shape.obj
 0002:0002c008       $chain$5$??$collect_glyphs@Uhb_bit_set_t@@@?$Lookup@U?$IntType@G$01@OT@@@AAT@@QEBAXAEAUhb_bit_set_t@@I@Z 00000001800d7008     hb-aat-layout.obj
 0002:0002c008       $chain$5$??$collect_glyphs@Uhb_bit_set_t@@@?$Lookup@U?$IntType@I$03@OT@@@AAT@@QEBAXAEAUhb_bit_set_t@@I@Z 00000001800d7008     hb-aat-layout.obj
 0002:0002c008       $chain$5$??$collect_glyphs@Uhb_bit_set_t@@@?$Lookup@UHBGlyphID16@OT@@@AAT@@QEBAXAEAUhb_bit_set_t@@I@Z 00000001800d7008     hb-aat-layout.obj
 0002:0002c030       $chain$6$??$collect_glyphs@Uhb_bit_set_t@@@?$Lookup@U?$IntType@G$01@OT@@@AAT@@QEBAXAEAUhb_bit_set_t@@I@Z 00000001800d7030     hb-aat-layout.obj
 0002:0002c030       $chain$6$??$collect_glyphs@Uhb_bit_set_t@@@?$Lookup@U?$IntType@I$03@OT@@@AAT@@QEBAXAEAUhb_bit_set_t@@I@Z 00000001800d7030     hb-aat-layout.obj
 0002:0002c030       $chain$6$??$collect_glyphs@Uhb_bit_set_t@@@?$Lookup@UHBGlyphID16@OT@@@AAT@@QEBAXAEAUhb_bit_set_t@@I@Z 00000001800d7030     hb-aat-layout.obj
 0002:0002c044       $chain$7$??$collect_glyphs@Uhb_bit_set_t@@@?$Lookup@U?$IntType@G$01@OT@@@AAT@@QEBAXAEAUhb_bit_set_t@@I@Z 00000001800d7044     hb-aat-layout.obj
 0002:0002c044       $chain$7$??$collect_glyphs@Uhb_bit_set_t@@@?$Lookup@U?$IntType@I$03@OT@@@AAT@@QEBAXAEAUhb_bit_set_t@@I@Z 00000001800d7044     hb-aat-layout.obj
 0002:0002c044       $chain$7$??$collect_glyphs@Uhb_bit_set_t@@@?$Lookup@UHBGlyphID16@OT@@@AAT@@QEBAXAEAUhb_bit_set_t@@I@Z 00000001800d7044     hb-aat-layout.obj
 0002:0002c054       $chain$8$??$collect_glyphs@Uhb_bit_set_t@@@?$Lookup@U?$IntType@G$01@OT@@@AAT@@QEBAXAEAUhb_bit_set_t@@I@Z 00000001800d7054     hb-aat-layout.obj
 0002:0002c054       $chain$8$??$collect_glyphs@Uhb_bit_set_t@@@?$Lookup@U?$IntType@I$03@OT@@@AAT@@QEBAXAEAUhb_bit_set_t@@I@Z 00000001800d7054     hb-aat-layout.obj
 0002:0002c054       $chain$8$??$collect_glyphs@Uhb_bit_set_t@@@?$Lookup@UHBGlyphID16@OT@@@AAT@@QEBAXAEAUhb_bit_set_t@@I@Z 00000001800d7054     hb-aat-layout.obj
 0002:0002c064       $chain$9$??$collect_glyphs@Uhb_bit_set_t@@@?$Lookup@U?$IntType@G$01@OT@@@AAT@@QEBAXAEAUhb_bit_set_t@@I@Z 00000001800d7064     hb-aat-layout.obj
 0002:0002c064       $chain$9$??$collect_glyphs@Uhb_bit_set_t@@@?$Lookup@U?$IntType@I$03@OT@@@AAT@@QEBAXAEAUhb_bit_set_t@@I@Z 00000001800d7064     hb-aat-layout.obj
 0002:0002c064       $chain$9$??$collect_glyphs@Uhb_bit_set_t@@@?$Lookup@UHBGlyphID16@OT@@@AAT@@QEBAXAEAUhb_bit_set_t@@I@Z 00000001800d7064     hb-aat-layout.obj
 0002:0002c08c       $unwind$??$sanitize_blob@Uankr@AAT@@@hb_sanitize_context_t@@QEAAPEAUhb_blob_t@@PEAU1@@Z 00000001800d708c     hb-aat-layout.obj
 0002:0002c0a8       $unwind$?transition@driver_context_t@?$InsertionSubtable@UExtendedTypes@AAT@@@AAT@@QEAAXPEAUhb_buffer_t@@PEAU?$StateTableDriver@UExtendedTypes@AAT@@UEntryData@?$InsertionSubtable@UExtendedTypes@AAT@@@2@W4Flags@42@@3@AEBU?$Entry@UEntryData@?$InsertionSubtable@UExtendedTypes@AAT@@@AAT@@@3@@Z 00000001800d70a8     hb-aat-layout.obj
 0002:0002c0a8       $unwind$?transition@driver_context_t@?$InsertionSubtable@UObsoleteTypes@AAT@@@AAT@@QEAAXPEAUhb_buffer_t@@PEAU?$StateTableDriver@UObsoleteTypes@AAT@@UEntryData@?$InsertionSubtable@UObsoleteTypes@AAT@@@2@W4Flags@42@@3@AEBU?$Entry@UEntryData@?$InsertionSubtable@UObsoleteTypes@AAT@@@AAT@@@3@@Z 00000001800d70a8     hb-aat-layout.obj
 0002:0002c0c0       $unwind$??$drive@Udriver_context_t@?$InsertionSubtable@UExtendedTypes@AAT@@@AAT@@@?$StateTableDriver@UExtendedTypes@AAT@@UEntryData@?$InsertionSubtable@UExtendedTypes@AAT@@@2@W4Flags@42@@AAT@@QEAAXPEAUdriver_context_t@?$InsertionSubtable@UExtendedTypes@AAT@@@1@PEAUhb_aat_apply_context_t@1@@Z 00000001800d70c0     hb-aat-layout.obj
 0002:0002c0d0       $chain$2$??$drive@Udriver_context_t@?$InsertionSubtable@UExtendedTypes@AAT@@@AAT@@@?$StateTableDriver@UExtendedTypes@AAT@@UEntryData@?$InsertionSubtable@UExtendedTypes@AAT@@@2@W4Flags@42@@AAT@@QEAAXPEAUdriver_context_t@?$InsertionSubtable@UExtendedTypes@AAT@@@1@PEAUhb_aat_apply_context_t@1@@Z 00000001800d70d0     hb-aat-layout.obj
 0002:0002c0ec       $chain$3$??$drive@Udriver_context_t@?$InsertionSubtable@UExtendedTypes@AAT@@@AAT@@@?$StateTableDriver@UExtendedTypes@AAT@@UEntryData@?$InsertionSubtable@UExtendedTypes@AAT@@@2@W4Flags@42@@AAT@@QEAAXPEAUdriver_context_t@?$InsertionSubtable@UExtendedTypes@AAT@@@1@PEAUhb_aat_apply_context_t@1@@Z 00000001800d70ec     hb-aat-layout.obj
 0002:0002c0fc       $unwind$?transition@driver_context_t@?$LigatureSubtable@UExtendedTypes@AAT@@@AAT@@QEAAXPEAUhb_buffer_t@@PEAU?$StateTableDriver@UExtendedTypes@AAT@@UEntryData@?$LigatureEntry@$00@2@W4Flags@?$LigatureSubtable@UExtendedTypes@AAT@@@2@@3@AEBU?$Entry@UEntryData@?$LigatureEntry@$00@AAT@@@3@@Z 00000001800d70fc     hb-aat-layout.obj
 0002:0002c0fc       $unwind$?transition@driver_context_t@?$LigatureSubtable@UObsoleteTypes@AAT@@@AAT@@QEAAXPEAUhb_buffer_t@@PEAU?$StateTableDriver@UObsoleteTypes@AAT@@XW4Flags@?$LigatureSubtable@UObsoleteTypes@AAT@@@2@@3@AEBU?$Entry@X@3@@Z 00000001800d70fc     hb-aat-layout.obj
 0002:0002c10c       $chain$0$?transition@driver_context_t@?$LigatureSubtable@UExtendedTypes@AAT@@@AAT@@QEAAXPEAUhb_buffer_t@@PEAU?$StateTableDriver@UExtendedTypes@AAT@@UEntryData@?$LigatureEntry@$00@2@W4Flags@?$LigatureSubtable@UExtendedTypes@AAT@@@2@@3@AEBU?$Entry@UEntryData@?$LigatureEntry@$00@AAT@@@3@@Z 00000001800d710c     hb-aat-layout.obj
 0002:0002c120       $chain$4$?transition@driver_context_t@?$LigatureSubtable@UExtendedTypes@AAT@@@AAT@@QEAAXPEAUhb_buffer_t@@PEAU?$StateTableDriver@UExtendedTypes@AAT@@UEntryData@?$LigatureEntry@$00@2@W4Flags@?$LigatureSubtable@UExtendedTypes@AAT@@@2@@3@AEBU?$Entry@UEntryData@?$LigatureEntry@$00@AAT@@@3@@Z 00000001800d7120     hb-aat-layout.obj
 0002:0002c140       $chain$5$?transition@driver_context_t@?$LigatureSubtable@UExtendedTypes@AAT@@@AAT@@QEAAXPEAUhb_buffer_t@@PEAU?$StateTableDriver@UExtendedTypes@AAT@@UEntryData@?$LigatureEntry@$00@2@W4Flags@?$LigatureSubtable@UExtendedTypes@AAT@@@2@@3@AEBU?$Entry@UEntryData@?$LigatureEntry@$00@AAT@@@3@@Z 00000001800d7140     hb-aat-layout.obj
 0002:0002c150       $chain$6$?transition@driver_context_t@?$LigatureSubtable@UExtendedTypes@AAT@@@AAT@@QEAAXPEAUhb_buffer_t@@PEAU?$StateTableDriver@UExtendedTypes@AAT@@UEntryData@?$LigatureEntry@$00@2@W4Flags@?$LigatureSubtable@UExtendedTypes@AAT@@@2@@3@AEBU?$Entry@UEntryData@?$LigatureEntry@$00@AAT@@@3@@Z 00000001800d7150     hb-aat-layout.obj
 0002:0002c160       $unwind$??$drive@Udriver_context_t@?$LigatureSubtable@UExtendedTypes@AAT@@@AAT@@@?$StateTableDriver@UExtendedTypes@AAT@@UEntryData@?$LigatureEntry@$00@2@W4Flags@?$LigatureSubtable@UExtendedTypes@AAT@@@2@@AAT@@QEAAXPEAUdriver_context_t@?$LigatureSubtable@UExtendedTypes@AAT@@@1@PEAUhb_aat_apply_context_t@1@@Z 00000001800d7160     hb-aat-layout.obj
 0002:0002c170       $chain$2$??$drive@Udriver_context_t@?$LigatureSubtable@UExtendedTypes@AAT@@@AAT@@@?$StateTableDriver@UExtendedTypes@AAT@@UEntryData@?$LigatureEntry@$00@2@W4Flags@?$LigatureSubtable@UExtendedTypes@AAT@@@2@@AAT@@QEAAXPEAUdriver_context_t@?$LigatureSubtable@UExtendedTypes@AAT@@@1@PEAUhb_aat_apply_context_t@1@@Z 00000001800d7170     hb-aat-layout.obj
 0002:0002c18c       $chain$3$??$drive@Udriver_context_t@?$LigatureSubtable@UExtendedTypes@AAT@@@AAT@@@?$StateTableDriver@UExtendedTypes@AAT@@UEntryData@?$LigatureEntry@$00@2@W4Flags@?$LigatureSubtable@UExtendedTypes@AAT@@@2@@AAT@@QEAAXPEAUdriver_context_t@?$LigatureSubtable@UExtendedTypes@AAT@@@1@PEAUhb_aat_apply_context_t@1@@Z 00000001800d718c     hb-aat-layout.obj
 0002:0002c19c       $unwind$??$drive@Udriver_context_t@?$ContextualSubtable@UExtendedTypes@AAT@@@AAT@@@?$StateTableDriver@UExtendedTypes@AAT@@UEntryData@?$ContextualSubtable@UExtendedTypes@AAT@@@2@W4Flags@42@@AAT@@QEAAXPEAUdriver_context_t@?$ContextualSubtable@UExtendedTypes@AAT@@@1@PEAUhb_aat_apply_context_t@1@@Z 00000001800d719c     hb-aat-layout.obj
 0002:0002c1ac       $chain$2$??$drive@Udriver_context_t@?$ContextualSubtable@UExtendedTypes@AAT@@@AAT@@@?$StateTableDriver@UExtendedTypes@AAT@@UEntryData@?$ContextualSubtable@UExtendedTypes@AAT@@@2@W4Flags@42@@AAT@@QEAAXPEAUdriver_context_t@?$ContextualSubtable@UExtendedTypes@AAT@@@1@PEAUhb_aat_apply_context_t@1@@Z 00000001800d71ac     hb-aat-layout.obj
 0002:0002c1c8       $chain$3$??$drive@Udriver_context_t@?$ContextualSubtable@UExtendedTypes@AAT@@@AAT@@@?$StateTableDriver@UExtendedTypes@AAT@@UEntryData@?$ContextualSubtable@UExtendedTypes@AAT@@@2@W4Flags@42@@AAT@@QEAAXPEAUdriver_context_t@?$ContextualSubtable@UExtendedTypes@AAT@@@1@PEAUhb_aat_apply_context_t@1@@Z 00000001800d71c8     hb-aat-layout.obj
 0002:0002c1d8       $unwind$?transition@driver_context_t@?$RearrangementSubtable@UExtendedTypes@AAT@@@AAT@@QEAAXPEAUhb_buffer_t@@PEAU?$StateTableDriver@UExtendedTypes@AAT@@XW4Flags@?$RearrangementSubtable@UExtendedTypes@AAT@@@2@@3@AEBU?$Entry@X@3@@Z 00000001800d71d8     hb-aat-layout.obj
 0002:0002c1d8       $unwind$?transition@driver_context_t@?$RearrangementSubtable@UObsoleteTypes@AAT@@@AAT@@QEAAXPEAUhb_buffer_t@@PEAU?$StateTableDriver@UObsoleteTypes@AAT@@XW4Flags@?$RearrangementSubtable@UObsoleteTypes@AAT@@@2@@3@AEBU?$Entry@X@3@@Z 00000001800d71d8     hb-aat-layout.obj
 0002:0002c1d8       $unwind$?apply@ChainContextFormat3@OT@@QEBA_NPEAUhb_ot_apply_context_t@2@@Z 00000001800d71d8     hb-ot-layout.obj
 0002:0002c1f0       $chain$1$?transition@driver_context_t@?$RearrangementSubtable@UExtendedTypes@AAT@@@AAT@@QEAAXPEAUhb_buffer_t@@PEAU?$StateTableDriver@UExtendedTypes@AAT@@XW4Flags@?$RearrangementSubtable@UExtendedTypes@AAT@@@2@@3@AEBU?$Entry@X@3@@Z 00000001800d71f0     hb-aat-layout.obj
 0002:0002c1f0       $chain$1$?transition@driver_context_t@?$RearrangementSubtable@UObsoleteTypes@AAT@@@AAT@@QEAAXPEAUhb_buffer_t@@PEAU?$StateTableDriver@UObsoleteTypes@AAT@@XW4Flags@?$RearrangementSubtable@UObsoleteTypes@AAT@@@2@@3@AEBU?$Entry@X@3@@Z 00000001800d71f0     hb-aat-layout.obj
 0002:0002c208       $chain$4$?transition@driver_context_t@?$RearrangementSubtable@UExtendedTypes@AAT@@@AAT@@QEAAXPEAUhb_buffer_t@@PEAU?$StateTableDriver@UExtendedTypes@AAT@@XW4Flags@?$RearrangementSubtable@UExtendedTypes@AAT@@@2@@3@AEBU?$Entry@X@3@@Z 00000001800d7208     hb-aat-layout.obj
 0002:0002c208       $chain$4$?transition@driver_context_t@?$RearrangementSubtable@UObsoleteTypes@AAT@@@AAT@@QEAAXPEAUhb_buffer_t@@PEAU?$StateTableDriver@UObsoleteTypes@AAT@@XW4Flags@?$RearrangementSubtable@UObsoleteTypes@AAT@@@2@@3@AEBU?$Entry@X@3@@Z 00000001800d7208     hb-aat-layout.obj
 0002:0002c224       $chain$5$?transition@driver_context_t@?$RearrangementSubtable@UExtendedTypes@AAT@@@AAT@@QEAAXPEAUhb_buffer_t@@PEAU?$StateTableDriver@UExtendedTypes@AAT@@XW4Flags@?$RearrangementSubtable@UExtendedTypes@AAT@@@2@@3@AEBU?$Entry@X@3@@Z 00000001800d7224     hb-aat-layout.obj
 0002:0002c224       $chain$5$?transition@driver_context_t@?$RearrangementSubtable@UObsoleteTypes@AAT@@@AAT@@QEAAXPEAUhb_buffer_t@@PEAU?$StateTableDriver@UObsoleteTypes@AAT@@XW4Flags@?$RearrangementSubtable@UObsoleteTypes@AAT@@@2@@3@AEBU?$Entry@X@3@@Z 00000001800d7224     hb-aat-layout.obj
 0002:0002c23c       $chain$6$?transition@driver_context_t@?$RearrangementSubtable@UExtendedTypes@AAT@@@AAT@@QEAAXPEAUhb_buffer_t@@PEAU?$StateTableDriver@UExtendedTypes@AAT@@XW4Flags@?$RearrangementSubtable@UExtendedTypes@AAT@@@2@@3@AEBU?$Entry@X@3@@Z 00000001800d723c     hb-aat-layout.obj
 0002:0002c23c       $chain$6$?transition@driver_context_t@?$RearrangementSubtable@UObsoleteTypes@AAT@@@AAT@@QEAAXPEAUhb_buffer_t@@PEAU?$StateTableDriver@UObsoleteTypes@AAT@@XW4Flags@?$RearrangementSubtable@UObsoleteTypes@AAT@@@2@@3@AEBU?$Entry@X@3@@Z 00000001800d723c     hb-aat-layout.obj
 0002:0002c24c       $chain$7$?transition@driver_context_t@?$RearrangementSubtable@UExtendedTypes@AAT@@@AAT@@QEAAXPEAUhb_buffer_t@@PEAU?$StateTableDriver@UExtendedTypes@AAT@@XW4Flags@?$RearrangementSubtable@UExtendedTypes@AAT@@@2@@3@AEBU?$Entry@X@3@@Z 00000001800d724c     hb-aat-layout.obj
 0002:0002c24c       $chain$7$?transition@driver_context_t@?$RearrangementSubtable@UObsoleteTypes@AAT@@@AAT@@QEAAXPEAUhb_buffer_t@@PEAU?$StateTableDriver@UObsoleteTypes@AAT@@XW4Flags@?$RearrangementSubtable@UObsoleteTypes@AAT@@@2@@3@AEBU?$Entry@X@3@@Z 00000001800d724c     hb-aat-layout.obj
 0002:0002c25c       $unwind$??$drive@Udriver_context_t@?$RearrangementSubtable@UExtendedTypes@AAT@@@AAT@@@?$StateTableDriver@UExtendedTypes@AAT@@XW4Flags@?$RearrangementSubtable@UExtendedTypes@AAT@@@2@@AAT@@QEAAXPEAUdriver_context_t@?$RearrangementSubtable@UExtendedTypes@AAT@@@1@PEAUhb_aat_apply_context_t@1@@Z 00000001800d725c     hb-aat-layout.obj
 0002:0002c26c       $chain$3$??$drive@Udriver_context_t@?$RearrangementSubtable@UExtendedTypes@AAT@@@AAT@@@?$StateTableDriver@UExtendedTypes@AAT@@XW4Flags@?$RearrangementSubtable@UExtendedTypes@AAT@@@2@@AAT@@QEAAXPEAUdriver_context_t@?$RearrangementSubtable@UExtendedTypes@AAT@@@1@PEAUhb_aat_apply_context_t@1@@Z 00000001800d726c     hb-aat-layout.obj
 0002:0002c28c       $chain$4$??$drive@Udriver_context_t@?$RearrangementSubtable@UExtendedTypes@AAT@@@AAT@@@?$StateTableDriver@UExtendedTypes@AAT@@XW4Flags@?$RearrangementSubtable@UExtendedTypes@AAT@@@2@@AAT@@QEAAXPEAUdriver_context_t@?$RearrangementSubtable@UExtendedTypes@AAT@@@1@PEAUhb_aat_apply_context_t@1@@Z 00000001800d728c     hb-aat-layout.obj
 0002:0002c29c       $unwind$?kern@?$hb_kern_machine_t@Uaccelerator_t@?$KerxSubTableFormat0@UKerxSubTableHeader@AAT@@@AAT@@@OT@@QEBAXPEAUhb_font_t@@PEAUhb_buffer_t@@I_N@Z 00000001800d729c     hb-aat-layout.obj
 0002:0002c29c       $unwind$?kern@?$hb_kern_machine_t@Uaccelerator_t@?$KerxSubTableFormat2@UKerxSubTableHeader@AAT@@@AAT@@@OT@@QEBAXPEAUhb_font_t@@PEAUhb_buffer_t@@I_N@Z 00000001800d729c     hb-aat-layout.obj
 0002:0002c29c       $unwind$?kern@?$hb_kern_machine_t@Uaccelerator_t@?$KerxSubTableFormat6@UKerxSubTableHeader@AAT@@@AAT@@@OT@@QEBAXPEAUhb_font_t@@PEAUhb_buffer_t@@I_N@Z 00000001800d729c     hb-aat-layout.obj
 0002:0002c29c       $unwind$?kern@?$hb_kern_machine_t@Uaccelerator_t@?$KerxSubTableFormat0@UKernAATSubTableHeader@OT@@@AAT@@@OT@@QEBAXPEAUhb_font_t@@PEAUhb_buffer_t@@I_N@Z 00000001800d729c     hb-ot-layout.obj
 0002:0002c29c       $unwind$?kern@?$hb_kern_machine_t@Uaccelerator_t@?$KerxSubTableFormat0@UKernOTSubTableHeader@OT@@@AAT@@@OT@@QEBAXPEAUhb_font_t@@PEAUhb_buffer_t@@I_N@Z 00000001800d729c     hb-ot-layout.obj
 0002:0002c29c       $unwind$?kern@?$hb_kern_machine_t@Uaccelerator_t@?$KerxSubTableFormat2@UKernAATSubTableHeader@OT@@@AAT@@@OT@@QEBAXPEAUhb_font_t@@PEAUhb_buffer_t@@I_N@Z 00000001800d729c     hb-ot-layout.obj
 0002:0002c29c       $unwind$?kern@?$hb_kern_machine_t@Uaccelerator_t@?$KerxSubTableFormat2@UKernOTSubTableHeader@OT@@@AAT@@@OT@@QEBAXPEAUhb_font_t@@PEAUhb_buffer_t@@I_N@Z 00000001800d729c     hb-ot-layout.obj
 0002:0002c2b4       $chain$0$?kern@?$hb_kern_machine_t@Uaccelerator_t@?$KerxSubTableFormat6@UKerxSubTableHeader@AAT@@@AAT@@@OT@@QEBAXPEAUhb_font_t@@PEAUhb_buffer_t@@I_N@Z 00000001800d72b4     hb-aat-layout.obj
 0002:0002c2c8       $chain$3$?kern@?$hb_kern_machine_t@Uaccelerator_t@?$KerxSubTableFormat6@UKerxSubTableHeader@AAT@@@AAT@@@OT@@QEBAXPEAUhb_font_t@@PEAUhb_buffer_t@@I_N@Z 00000001800d72c8     hb-aat-layout.obj
 0002:0002c2e4       $chain$4$?kern@?$hb_kern_machine_t@Uaccelerator_t@?$KerxSubTableFormat6@UKerxSubTableHeader@AAT@@@AAT@@@OT@@QEBAXPEAUhb_font_t@@PEAUhb_buffer_t@@I_N@Z 00000001800d72e4     hb-aat-layout.obj
 0002:0002c2f4       $chain$5$?kern@?$hb_kern_machine_t@Uaccelerator_t@?$KerxSubTableFormat6@UKerxSubTableHeader@AAT@@@AAT@@@OT@@QEBAXPEAUhb_font_t@@PEAUhb_buffer_t@@I_N@Z 00000001800d72f4     hb-aat-layout.obj
 0002:0002c304       $unwind$?transition@driver_context_t@?$KerxSubTableFormat4@UKerxSubTableHeader@AAT@@@AAT@@QEAAXPEAUhb_buffer_t@@PEAU?$StateTableDriver@UExtendedTypes@AAT@@UEntryData@?$KerxSubTableFormat4@UKerxSubTableHeader@AAT@@@2@W4Flags@42@@3@AEBU?$Entry@UEntryData@?$KerxSubTableFormat4@UKerxSubTableHeader@AAT@@@AAT@@@3@@Z 00000001800d7304     hb-aat-layout.obj
 0002:0002c31c       $unwind$??$drive@Udriver_context_t@?$KerxSubTableFormat1@UKerxSubTableHeader@AAT@@@AAT@@@?$StateTableDriver@UExtendedTypes@AAT@@UEntryData@?$Format1Entry@$00@2@W4Flags@?$KerxSubTableFormat1@UKerxSubTableHeader@AAT@@@2@@AAT@@QEAAXPEAUdriver_context_t@?$KerxSubTableFormat1@UKerxSubTableHeader@AAT@@@1@PEAUhb_aat_apply_context_t@1@@Z 00000001800d731c     hb-aat-layout.obj
 0002:0002c31c       $unwind$??$drive@Udriver_context_t@?$KerxSubTableFormat4@UKerxSubTableHeader@AAT@@@AAT@@@?$StateTableDriver@UExtendedTypes@AAT@@UEntryData@?$KerxSubTableFormat4@UKerxSubTableHeader@AAT@@@2@W4Flags@42@@AAT@@QEAAXPEAUdriver_context_t@?$KerxSubTableFormat4@UKerxSubTableHeader@AAT@@@1@PEAUhb_aat_apply_context_t@1@@Z 00000001800d731c     hb-aat-layout.obj
 0002:0002c32c       $chain$3$??$drive@Udriver_context_t@?$KerxSubTableFormat4@UKerxSubTableHeader@AAT@@@AAT@@@?$StateTableDriver@UExtendedTypes@AAT@@UEntryData@?$KerxSubTableFormat4@UKerxSubTableHeader@AAT@@@2@W4Flags@42@@AAT@@QEAAXPEAUdriver_context_t@?$KerxSubTableFormat4@UKerxSubTableHeader@AAT@@@1@PEAUhb_aat_apply_context_t@1@@Z 00000001800d732c     hb-aat-layout.obj
 0002:0002c34c       $chain$4$??$drive@Udriver_context_t@?$KerxSubTableFormat4@UKerxSubTableHeader@AAT@@@AAT@@@?$StateTableDriver@UExtendedTypes@AAT@@UEntryData@?$KerxSubTableFormat4@UKerxSubTableHeader@AAT@@@2@W4Flags@42@@AAT@@QEAAXPEAUdriver_context_t@?$KerxSubTableFormat4@UKerxSubTableHeader@AAT@@@1@PEAUhb_aat_apply_context_t@1@@Z 00000001800d734c     hb-aat-layout.obj
 0002:0002c35c       $chain$0$?kern@?$hb_kern_machine_t@Uaccelerator_t@?$KerxSubTableFormat2@UKerxSubTableHeader@AAT@@@AAT@@@OT@@QEBAXPEAUhb_font_t@@PEAUhb_buffer_t@@I_N@Z 00000001800d735c     hb-aat-layout.obj
 0002:0002c370       $chain$3$?kern@?$hb_kern_machine_t@Uaccelerator_t@?$KerxSubTableFormat2@UKerxSubTableHeader@AAT@@@AAT@@@OT@@QEBAXPEAUhb_font_t@@PEAUhb_buffer_t@@I_N@Z 00000001800d7370     hb-aat-layout.obj
 0002:0002c38c       $chain$4$?kern@?$hb_kern_machine_t@Uaccelerator_t@?$KerxSubTableFormat2@UKerxSubTableHeader@AAT@@@AAT@@@OT@@QEBAXPEAUhb_font_t@@PEAUhb_buffer_t@@I_N@Z 00000001800d738c     hb-aat-layout.obj
 0002:0002c39c       $chain$5$?kern@?$hb_kern_machine_t@Uaccelerator_t@?$KerxSubTableFormat2@UKerxSubTableHeader@AAT@@@AAT@@@OT@@QEBAXPEAUhb_font_t@@PEAUhb_buffer_t@@I_N@Z 00000001800d739c     hb-aat-layout.obj
 0002:0002c3ac       $unwind$?transition@driver_context_t@?$KerxSubTableFormat1@UKerxSubTableHeader@AAT@@@AAT@@QEAAXPEAUhb_buffer_t@@PEAU?$StateTableDriver@UExtendedTypes@AAT@@UEntryData@?$Format1Entry@$00@2@W4Flags@?$KerxSubTableFormat1@UKerxSubTableHeader@AAT@@@2@@3@AEBU?$Entry@UEntryData@?$Format1Entry@$00@AAT@@@3@@Z 00000001800d73ac     hb-aat-layout.obj
 0002:0002c3c0       $chain$1$?transition@driver_context_t@?$KerxSubTableFormat1@UKerxSubTableHeader@AAT@@@AAT@@QEAAXPEAUhb_buffer_t@@PEAU?$StateTableDriver@UExtendedTypes@AAT@@UEntryData@?$Format1Entry@$00@2@W4Flags@?$KerxSubTableFormat1@UKerxSubTableHeader@AAT@@@2@@3@AEBU?$Entry@UEntryData@?$Format1Entry@$00@AAT@@@3@@Z 00000001800d73c0     hb-aat-layout.obj
 0002:0002c3d8       $chain$2$?transition@driver_context_t@?$KerxSubTableFormat1@UKerxSubTableHeader@AAT@@@AAT@@QEAAXPEAUhb_buffer_t@@PEAU?$StateTableDriver@UExtendedTypes@AAT@@UEntryData@?$Format1Entry@$00@2@W4Flags@?$KerxSubTableFormat1@UKerxSubTableHeader@AAT@@@2@@3@AEBU?$Entry@UEntryData@?$Format1Entry@$00@AAT@@@3@@Z 00000001800d73d8     hb-aat-layout.obj
 0002:0002c3e8       $chain$3$??$drive@Udriver_context_t@?$KerxSubTableFormat1@UKerxSubTableHeader@AAT@@@AAT@@@?$StateTableDriver@UExtendedTypes@AAT@@UEntryData@?$Format1Entry@$00@2@W4Flags@?$KerxSubTableFormat1@UKerxSubTableHeader@AAT@@@2@@AAT@@QEAAXPEAUdriver_context_t@?$KerxSubTableFormat1@UKerxSubTableHeader@AAT@@@1@PEAUhb_aat_apply_context_t@1@@Z 00000001800d73e8     hb-aat-layout.obj
 0002:0002c408       $chain$4$??$drive@Udriver_context_t@?$KerxSubTableFormat1@UKerxSubTableHeader@AAT@@@AAT@@@?$StateTableDriver@UExtendedTypes@AAT@@UEntryData@?$Format1Entry@$00@2@W4Flags@?$KerxSubTableFormat1@UKerxSubTableHeader@AAT@@@2@@AAT@@QEAAXPEAUdriver_context_t@?$KerxSubTableFormat1@UKerxSubTableHeader@AAT@@@1@PEAUhb_aat_apply_context_t@1@@Z 00000001800d7408     hb-aat-layout.obj
 0002:0002c418       $chain$0$?kern@?$hb_kern_machine_t@Uaccelerator_t@?$KerxSubTableFormat0@UKerxSubTableHeader@AAT@@@AAT@@@OT@@QEBAXPEAUhb_font_t@@PEAUhb_buffer_t@@I_N@Z 00000001800d7418     hb-aat-layout.obj
 0002:0002c42c       $chain$3$?kern@?$hb_kern_machine_t@Uaccelerator_t@?$KerxSubTableFormat0@UKerxSubTableHeader@AAT@@@AAT@@@OT@@QEBAXPEAUhb_font_t@@PEAUhb_buffer_t@@I_N@Z 00000001800d742c     hb-aat-layout.obj
 0002:0002c448       $chain$4$?kern@?$hb_kern_machine_t@Uaccelerator_t@?$KerxSubTableFormat0@UKerxSubTableHeader@AAT@@@AAT@@@OT@@QEBAXPEAUhb_font_t@@PEAUhb_buffer_t@@I_N@Z 00000001800d7448     hb-aat-layout.obj
 0002:0002c458       $chain$5$?kern@?$hb_kern_machine_t@Uaccelerator_t@?$KerxSubTableFormat0@UKerxSubTableHeader@AAT@@@AAT@@@OT@@QEBAXPEAUhb_font_t@@PEAUhb_buffer_t@@I_N@Z 00000001800d7458     hb-aat-layout.obj
 0002:0002c468       $unwind$??$drive@Udriver_context_t@?$InsertionSubtable@UObsoleteTypes@AAT@@@AAT@@@?$StateTableDriver@UObsoleteTypes@AAT@@UEntryData@?$InsertionSubtable@UObsoleteTypes@AAT@@@2@W4Flags@42@@AAT@@QEAAXPEAUdriver_context_t@?$InsertionSubtable@UObsoleteTypes@AAT@@@1@PEAUhb_aat_apply_context_t@1@@Z 00000001800d7468     hb-aat-layout.obj
 0002:0002c478       $chain$2$??$drive@Udriver_context_t@?$InsertionSubtable@UObsoleteTypes@AAT@@@AAT@@@?$StateTableDriver@UObsoleteTypes@AAT@@UEntryData@?$InsertionSubtable@UObsoleteTypes@AAT@@@2@W4Flags@42@@AAT@@QEAAXPEAUdriver_context_t@?$InsertionSubtable@UObsoleteTypes@AAT@@@1@PEAUhb_aat_apply_context_t@1@@Z 00000001800d7478     hb-aat-layout.obj
 0002:0002c494       $chain$3$??$drive@Udriver_context_t@?$InsertionSubtable@UObsoleteTypes@AAT@@@AAT@@@?$StateTableDriver@UObsoleteTypes@AAT@@UEntryData@?$InsertionSubtable@UObsoleteTypes@AAT@@@2@W4Flags@42@@AAT@@QEAAXPEAUdriver_context_t@?$InsertionSubtable@UObsoleteTypes@AAT@@@1@PEAUhb_aat_apply_context_t@1@@Z 00000001800d7494     hb-aat-layout.obj
 0002:0002c4a4       $chain$0$?transition@driver_context_t@?$LigatureSubtable@UObsoleteTypes@AAT@@@AAT@@QEAAXPEAUhb_buffer_t@@PEAU?$StateTableDriver@UObsoleteTypes@AAT@@XW4Flags@?$LigatureSubtable@UObsoleteTypes@AAT@@@2@@3@AEBU?$Entry@X@3@@Z 00000001800d74a4     hb-aat-layout.obj
 0002:0002c4b8       $chain$4$?transition@driver_context_t@?$LigatureSubtable@UObsoleteTypes@AAT@@@AAT@@QEAAXPEAUhb_buffer_t@@PEAU?$StateTableDriver@UObsoleteTypes@AAT@@XW4Flags@?$LigatureSubtable@UObsoleteTypes@AAT@@@2@@3@AEBU?$Entry@X@3@@Z 00000001800d74b8     hb-aat-layout.obj
 0002:0002c4d8       $chain$5$?transition@driver_context_t@?$LigatureSubtable@UObsoleteTypes@AAT@@@AAT@@QEAAXPEAUhb_buffer_t@@PEAU?$StateTableDriver@UObsoleteTypes@AAT@@XW4Flags@?$LigatureSubtable@UObsoleteTypes@AAT@@@2@@3@AEBU?$Entry@X@3@@Z 00000001800d74d8     hb-aat-layout.obj
 0002:0002c4e8       $chain$6$?transition@driver_context_t@?$LigatureSubtable@UObsoleteTypes@AAT@@@AAT@@QEAAXPEAUhb_buffer_t@@PEAU?$StateTableDriver@UObsoleteTypes@AAT@@XW4Flags@?$LigatureSubtable@UObsoleteTypes@AAT@@@2@@3@AEBU?$Entry@X@3@@Z 00000001800d74e8     hb-aat-layout.obj
 0002:0002c4f8       $unwind$??$drive@Udriver_context_t@?$LigatureSubtable@UObsoleteTypes@AAT@@@AAT@@@?$StateTableDriver@UObsoleteTypes@AAT@@XW4Flags@?$LigatureSubtable@UObsoleteTypes@AAT@@@2@@AAT@@QEAAXPEAUdriver_context_t@?$LigatureSubtable@UObsoleteTypes@AAT@@@1@PEAUhb_aat_apply_context_t@1@@Z 00000001800d74f8     hb-aat-layout.obj
 0002:0002c508       $chain$2$??$drive@Udriver_context_t@?$LigatureSubtable@UObsoleteTypes@AAT@@@AAT@@@?$StateTableDriver@UObsoleteTypes@AAT@@XW4Flags@?$LigatureSubtable@UObsoleteTypes@AAT@@@2@@AAT@@QEAAXPEAUdriver_context_t@?$LigatureSubtable@UObsoleteTypes@AAT@@@1@PEAUhb_aat_apply_context_t@1@@Z 00000001800d7508     hb-aat-layout.obj
 0002:0002c524       $chain$3$??$drive@Udriver_context_t@?$LigatureSubtable@UObsoleteTypes@AAT@@@AAT@@@?$StateTableDriver@UObsoleteTypes@AAT@@XW4Flags@?$LigatureSubtable@UObsoleteTypes@AAT@@@2@@AAT@@QEAAXPEAUdriver_context_t@?$LigatureSubtable@UObsoleteTypes@AAT@@@1@PEAUhb_aat_apply_context_t@1@@Z 00000001800d7524     hb-aat-layout.obj
 0002:0002c534       $unwind$?transition@driver_context_t@?$ContextualSubtable@UObsoleteTypes@AAT@@@AAT@@QEAAXPEAUhb_buffer_t@@PEAU?$StateTableDriver@UObsoleteTypes@AAT@@UEntryData@?$ContextualSubtable@UObsoleteTypes@AAT@@@2@W4Flags@42@@3@AEBU?$Entry@UEntryData@?$ContextualSubtable@UObsoleteTypes@AAT@@@AAT@@@3@@Z 00000001800d7534     hb-aat-layout.obj
 0002:0002c540       $chain$4$?transition@driver_context_t@?$ContextualSubtable@UObsoleteTypes@AAT@@@AAT@@QEAAXPEAUhb_buffer_t@@PEAU?$StateTableDriver@UObsoleteTypes@AAT@@UEntryData@?$ContextualSubtable@UObsoleteTypes@AAT@@@2@W4Flags@42@@3@AEBU?$Entry@UEntryData@?$ContextualSubtable@UObsoleteTypes@AAT@@@AAT@@@3@@Z 00000001800d7540     hb-aat-layout.obj
 0002:0002c564       $chain$5$?transition@driver_context_t@?$ContextualSubtable@UObsoleteTypes@AAT@@@AAT@@QEAAXPEAUhb_buffer_t@@PEAU?$StateTableDriver@UObsoleteTypes@AAT@@UEntryData@?$ContextualSubtable@UObsoleteTypes@AAT@@@2@W4Flags@42@@3@AEBU?$Entry@UEntryData@?$ContextualSubtable@UObsoleteTypes@AAT@@@AAT@@@3@@Z 00000001800d7564     hb-aat-layout.obj
 0002:0002c580       $chain$6$?transition@driver_context_t@?$ContextualSubtable@UObsoleteTypes@AAT@@@AAT@@QEAAXPEAUhb_buffer_t@@PEAU?$StateTableDriver@UObsoleteTypes@AAT@@UEntryData@?$ContextualSubtable@UObsoleteTypes@AAT@@@2@W4Flags@42@@3@AEBU?$Entry@UEntryData@?$ContextualSubtable@UObsoleteTypes@AAT@@@AAT@@@3@@Z 00000001800d7580     hb-aat-layout.obj
 0002:0002c590       $unwind$??$drive@Udriver_context_t@?$ContextualSubtable@UObsoleteTypes@AAT@@@AAT@@@?$StateTableDriver@UObsoleteTypes@AAT@@UEntryData@?$ContextualSubtable@UObsoleteTypes@AAT@@@2@W4Flags@42@@AAT@@QEAAXPEAUdriver_context_t@?$ContextualSubtable@UObsoleteTypes@AAT@@@1@PEAUhb_aat_apply_context_t@1@@Z 00000001800d7590     hb-aat-layout.obj
 0002:0002c5a0       $chain$3$??$drive@Udriver_context_t@?$ContextualSubtable@UObsoleteTypes@AAT@@@AAT@@@?$StateTableDriver@UObsoleteTypes@AAT@@UEntryData@?$ContextualSubtable@UObsoleteTypes@AAT@@@2@W4Flags@42@@AAT@@QEAAXPEAUdriver_context_t@?$ContextualSubtable@UObsoleteTypes@AAT@@@1@PEAUhb_aat_apply_context_t@1@@Z 00000001800d75a0     hb-aat-layout.obj
 0002:0002c5c0       $chain$4$??$drive@Udriver_context_t@?$ContextualSubtable@UObsoleteTypes@AAT@@@AAT@@@?$StateTableDriver@UObsoleteTypes@AAT@@UEntryData@?$ContextualSubtable@UObsoleteTypes@AAT@@@2@W4Flags@42@@AAT@@QEAAXPEAUdriver_context_t@?$ContextualSubtable@UObsoleteTypes@AAT@@@1@PEAUhb_aat_apply_context_t@1@@Z 00000001800d75c0     hb-aat-layout.obj
 0002:0002c5d0       $unwind$??$drive@Udriver_context_t@?$RearrangementSubtable@UObsoleteTypes@AAT@@@AAT@@@?$StateTableDriver@UObsoleteTypes@AAT@@XW4Flags@?$RearrangementSubtable@UObsoleteTypes@AAT@@@2@@AAT@@QEAAXPEAUdriver_context_t@?$RearrangementSubtable@UObsoleteTypes@AAT@@@1@PEAUhb_aat_apply_context_t@1@@Z 00000001800d75d0     hb-aat-layout.obj
 0002:0002c5e0       $chain$3$??$drive@Udriver_context_t@?$RearrangementSubtable@UObsoleteTypes@AAT@@@AAT@@@?$StateTableDriver@UObsoleteTypes@AAT@@XW4Flags@?$RearrangementSubtable@UObsoleteTypes@AAT@@@2@@AAT@@QEAAXPEAUdriver_context_t@?$RearrangementSubtable@UObsoleteTypes@AAT@@@1@PEAUhb_aat_apply_context_t@1@@Z 00000001800d75e0     hb-aat-layout.obj
 0002:0002c600       $chain$4$??$drive@Udriver_context_t@?$RearrangementSubtable@UObsoleteTypes@AAT@@@AAT@@@?$StateTableDriver@UObsoleteTypes@AAT@@XW4Flags@?$RearrangementSubtable@UObsoleteTypes@AAT@@@2@@AAT@@QEAAXPEAUdriver_context_t@?$RearrangementSubtable@UObsoleteTypes@AAT@@@1@PEAUhb_aat_apply_context_t@1@@Z 00000001800d7600     hb-aat-layout.obj
 0002:0002c610       $chain$1$??$check_array@UFeature@AAT@@@hb_sanitize_context_t@@QEBA_NPEBUFeature@AAT@@I@Z 00000001800d7610     hb-aat-layout.obj
 0002:0002c628       $chain$2$??$check_array@UFeature@AAT@@@hb_sanitize_context_t@@QEBA_NPEBUFeature@AAT@@I@Z 00000001800d7628     hb-aat-layout.obj
 0002:0002c638       $unwind$??$dispatch@Uhb_sanitize_context_t@@$$V@?$ChainSubtable@UExtendedTypes@AAT@@@AAT@@QEBA_NPEAUhb_sanitize_context_t@@@Z 00000001800d7638     hb-aat-layout.obj
 0002:0002c640       $chain$1$??$dispatch@Uhb_sanitize_context_t@@$$V@?$ChainSubtable@UExtendedTypes@AAT@@@AAT@@QEBA_NPEAUhb_sanitize_context_t@@@Z 00000001800d7640     hb-aat-layout.obj
 0002:0002c658       $chain$3$??$dispatch@Uhb_sanitize_context_t@@$$V@?$ChainSubtable@UExtendedTypes@AAT@@@AAT@@QEBA_NPEAUhb_sanitize_context_t@@@Z 00000001800d7658     hb-aat-layout.obj
 0002:0002c658       $chain$5$??$dispatch@Uhb_sanitize_context_t@@$$V@?$ChainSubtable@UExtendedTypes@AAT@@@AAT@@QEBA_NPEAUhb_sanitize_context_t@@@Z 00000001800d7658     hb-aat-layout.obj
 0002:0002c670       $chain$8$??$dispatch@Uhb_sanitize_context_t@@$$V@?$ChainSubtable@UExtendedTypes@AAT@@@AAT@@QEBA_NPEAUhb_sanitize_context_t@@@Z 00000001800d7670     hb-aat-layout.obj
 0002:0002c68c       $chain$10$??$dispatch@Uhb_sanitize_context_t@@$$V@?$ChainSubtable@UExtendedTypes@AAT@@@AAT@@QEBA_NPEAUhb_sanitize_context_t@@@Z 00000001800d768c     hb-aat-layout.obj
 0002:0002c6a8       $chain$11$??$dispatch@Uhb_sanitize_context_t@@$$V@?$ChainSubtable@UExtendedTypes@AAT@@@AAT@@QEBA_NPEAUhb_sanitize_context_t@@@Z 00000001800d76a8     hb-aat-layout.obj
 0002:0002c6b8       $unwind$??$collect_coverage@Uhb_set_digest_t@@@?$CoverageFormat2_4@USmallTypes@Layout@OT@@@Common@Layout@OT@@AEBA_NPEAUhb_set_digest_t@@@Z 00000001800d76b8     hb-aat-layout.obj
 0002:0002c6b8       $unwind$?read_points@SimpleGlyph@glyf_impl@OT@@SA_NAEAPEBU?$IntType@E$00@3@U?$hb_array_t@Ucontour_point_t@@@@PEBU43@PEQcontour_point_t@@MW4simple_glyph_flag_t@123@4@Z 00000001800d76b8     hb-common.obj
 0002:0002c6d4       $unwind$??$dispatch@URecordListOfScript@OT@@$$V@hb_sanitize_context_t@@QEAA_NAEBURecordListOfScript@OT@@@Z 00000001800d76d4     hb-aat-layout.obj
 0002:0002c6e0       $chain$5$??$dispatch@URecordListOfScript@OT@@$$V@hb_sanitize_context_t@@QEAA_NAEBURecordListOfScript@OT@@@Z 00000001800d76e0     hb-aat-layout.obj
 0002:0002c708       $chain$7$??$dispatch@URecordListOfScript@OT@@$$V@hb_sanitize_context_t@@QEAA_NAEBURecordListOfScript@OT@@@Z 00000001800d7708     hb-aat-layout.obj
 0002:0002c730       $unwind$??$dispatch@U?$RecordListOf@UFeature@OT@@@OT@@$$V@hb_sanitize_context_t@@QEAA_NAEBU?$RecordListOf@UFeature@OT@@@OT@@@Z 00000001800d7730     hb-aat-layout.obj
 0002:0002c73c       $chain$5$??$dispatch@U?$RecordListOf@UFeature@OT@@@OT@@$$V@hb_sanitize_context_t@@QEAA_NAEBU?$RecordListOf@UFeature@OT@@@OT@@@Z 00000001800d773c     hb-aat-layout.obj
 0002:0002c764       $chain$7$??$dispatch@U?$RecordListOf@UFeature@OT@@@OT@@$$V@hb_sanitize_context_t@@QEAA_NAEBU?$RecordListOf@UFeature@OT@@@OT@@@Z 00000001800d7764     hb-aat-layout.obj
 0002:0002c78c       $unwind$??$dispatch@U?$ChainRuleSet@USmallTypes@Layout@OT@@@OT@@$$V@hb_sanitize_context_t@@QEAA_NAEBU?$ChainRuleSet@USmallTypes@Layout@OT@@@OT@@@Z 00000001800d778c     hb-aat-layout.obj
 0002:0002c78c       $unwind$??$dispatch@U?$LigatureSet@USmallTypes@Layout@OT@@@GSUB_impl@Layout@OT@@$$V@hb_sanitize_context_t@@QEAA_NAEBU?$LigatureSet@USmallTypes@Layout@OT@@@GSUB_impl@Layout@OT@@@Z 00000001800d778c     hb-aat-layout.obj
 0002:0002c78c       $unwind$??$dispatch@U?$List16OfOffsetTo@USubstLookup@GSUB_impl@Layout@OT@@U?$IntType@G$01@4@@OT@@$$V@hb_sanitize_context_t@@QEAA_NAEBU?$List16OfOffsetTo@USubstLookup@GSUB_impl@Layout@OT@@U?$IntType@G$01@4@@OT@@@Z 00000001800d778c     hb-aat-layout.obj
 0002:0002c78c       $unwind$??$dispatch@U?$RuleSet@USmallTypes@Layout@OT@@@OT@@$$V@hb_sanitize_context_t@@QEAA_NAEBU?$RuleSet@USmallTypes@Layout@OT@@@OT@@@Z 00000001800d778c     hb-aat-layout.obj
 0002:0002c78c       $unwind$??$dispatch@ULigGlyph@OT@@$$V@hb_sanitize_context_t@@QEAA_NAEBULigGlyph@OT@@@Z 00000001800d778c     hb-aat-layout.obj
 0002:0002c78c       $unwind$??$dispatch@U?$List16OfOffsetTo@UPosLookup@GPOS_impl@Layout@OT@@U?$IntType@G$01@4@@OT@@$$V@hb_sanitize_context_t@@QEAA_NAEBU?$List16OfOffsetTo@UPosLookup@GPOS_impl@Layout@OT@@U?$IntType@G$01@4@@OT@@@Z 00000001800d778c     hb-ot-layout.obj
 0002:0002c798       $chain$4$??$dispatch@U?$List16OfOffsetTo@USubstLookup@GSUB_impl@Layout@OT@@U?$IntType@G$01@4@@OT@@$$V@hb_sanitize_context_t@@QEAA_NAEBU?$List16OfOffsetTo@USubstLookup@GSUB_impl@Layout@OT@@U?$IntType@G$01@4@@OT@@@Z 00000001800d7798     hb-aat-layout.obj
 0002:0002c7bc       $chain$6$??$dispatch@U?$List16OfOffsetTo@USubstLookup@GSUB_impl@Layout@OT@@U?$IntType@G$01@4@@OT@@$$V@hb_sanitize_context_t@@QEAA_NAEBU?$List16OfOffsetTo@USubstLookup@GSUB_impl@Layout@OT@@U?$IntType@G$01@4@@OT@@@Z 00000001800d77bc     hb-aat-layout.obj
 0002:0002c7e0       $unwind$??$collect_glyphs_filtered@Uhb_bit_set_t@@Uhb_bit_page_t@@@?$Lookup@U?$IntType@G$01@OT@@@AAT@@QEBAXAEAUhb_bit_set_t@@IAEBUhb_bit_page_t@@@Z 00000001800d77e0     hb-aat-layout.obj
 0002:0002c7fc       $chain$1$??$check_array@UHBGlyphID16@OT@@@hb_sanitize_context_t@@QEBA_NPEBUHBGlyphID16@OT@@I@Z 00000001800d77fc     hb-aat-layout.obj
 0002:0002c7fc       $chain$1$??$check_array@U?$IntType@G$01@OT@@@hb_sanitize_context_t@@QEBA_NPEBU?$IntType@G$01@OT@@I@Z 00000001800d77fc     hb-common.obj
 0002:0002c814       $chain$2$??$check_array@UHBGlyphID16@OT@@@hb_sanitize_context_t@@QEBA_NPEBUHBGlyphID16@OT@@I@Z 00000001800d7814     hb-aat-layout.obj
 0002:0002c814       $chain$2$??$check_array@U?$IntType@G$01@OT@@@hb_sanitize_context_t@@QEBA_NPEBU?$IntType@G$01@OT@@I@Z 00000001800d7814     hb-common.obj
 0002:0002c824       $unwind$??$output_glyphs@UHBGlyphID16@OT@@@hb_aat_apply_context_t@AAT@@QEAA_NIPEBUHBGlyphID16@OT@@@Z 00000001800d7824     hb-aat-layout.obj
 0002:0002c844       $chain$4$??$dispatch@ULigGlyph@OT@@$$V@hb_sanitize_context_t@@QEAA_NAEBULigGlyph@OT@@@Z 00000001800d7844     hb-aat-layout.obj
 0002:0002c868       $chain$6$??$dispatch@ULigGlyph@OT@@$$V@hb_sanitize_context_t@@QEAA_NAEBULigGlyph@OT@@@Z 00000001800d7868     hb-aat-layout.obj
 0002:0002c88c       $unwind$??$collect_glyphs_filtered@Uhb_bit_set_t@@Uhb_bit_page_t@@@?$LookupFormat4@U?$IntType@G$01@OT@@@AAT@@AEBAXAEAUhb_bit_set_t@@AEBUhb_bit_page_t@@@Z 00000001800d788c     hb-aat-layout.obj
 0002:0002c8a0       $chain$1$??$collect_glyphs_filtered@Uhb_bit_set_t@@Uhb_bit_page_t@@@?$LookupFormat4@U?$IntType@G$01@OT@@@AAT@@AEBAXAEAUhb_bit_set_t@@AEBUhb_bit_page_t@@@Z 00000001800d78a0     hb-aat-layout.obj
 0002:0002c8b8       $chain$2$??$collect_glyphs_filtered@Uhb_bit_set_t@@Uhb_bit_page_t@@@?$LookupFormat4@U?$IntType@G$01@OT@@@AAT@@AEBAXAEAUhb_bit_set_t@@AEBUhb_bit_page_t@@@Z 00000001800d78b8     hb-aat-layout.obj
 0002:0002c8c8       $unwind$??$sanitize@$$V@?$UnsizedListOfOffset16To@U?$Lookup@UHBGlyphID16@OT@@@AAT@@U?$IntType@G$01@OT@@X$0A@@OT@@QEBA_NPEAUhb_sanitize_context_t@@I@Z 00000001800d78c8     hb-aat-layout.obj
 0002:0002c8d8       $chain$1$??$sanitize@$$V@?$UnsizedListOfOffset16To@U?$Lookup@UHBGlyphID16@OT@@@AAT@@U?$IntType@G$01@OT@@X$0A@@OT@@QEBA_NPEAUhb_sanitize_context_t@@I@Z 00000001800d78d8     hb-aat-layout.obj
 0002:0002c8f0       $chain$3$??$sanitize@$$V@?$UnsizedListOfOffset16To@U?$Lookup@UHBGlyphID16@OT@@@AAT@@U?$IntType@G$01@OT@@X$0A@@OT@@QEBA_NPEAUhb_sanitize_context_t@@I@Z 00000001800d78f0     hb-aat-layout.obj
 0002:0002c908       $unwind$??$collect_initial_glyphs@Uhb_bit_set_t@@U?$RearrangementSubtable@UObsoleteTypes@AAT@@@AAT@@@?$StateTable@UObsoleteTypes@AAT@@X@AAT@@QEBAXAEAUhb_bit_set_t@@IAEBU?$RearrangementSubtable@UObsoleteTypes@AAT@@@1@@Z 00000001800d7908     hb-aat-layout.obj
 0002:0002c920       $chain$2$??$collect_initial_glyphs@Uhb_bit_set_t@@U?$RearrangementSubtable@UObsoleteTypes@AAT@@@AAT@@@?$StateTable@UObsoleteTypes@AAT@@X@AAT@@QEBAXAEAUhb_bit_set_t@@IAEBU?$RearrangementSubtable@UObsoleteTypes@AAT@@@1@@Z 00000001800d7920     hb-aat-layout.obj
 0002:0002c93c       $chain$3$??$collect_initial_glyphs@Uhb_bit_set_t@@U?$RearrangementSubtable@UObsoleteTypes@AAT@@@AAT@@@?$StateTable@UObsoleteTypes@AAT@@X@AAT@@QEBAXAEAUhb_bit_set_t@@IAEBU?$RearrangementSubtable@UObsoleteTypes@AAT@@@1@@Z 00000001800d793c     hb-aat-layout.obj
 0002:0002c94c       $unwind$??$collect_initial_glyphs@Uhb_bit_set_t@@U?$ContextualSubtable@UObsoleteTypes@AAT@@@AAT@@@?$StateTable@UObsoleteTypes@AAT@@UEntryData@?$ContextualSubtable@UObsoleteTypes@AAT@@@2@@AAT@@QEBAXAEAUhb_bit_set_t@@IAEBU?$ContextualSubtable@UObsoleteTypes@AAT@@@1@@Z 00000001800d794c     hb-aat-layout.obj
 0002:0002c94c       $unwind$??$collect_initial_glyphs@Uhb_bit_set_t@@U?$LigatureSubtable@UObsoleteTypes@AAT@@@AAT@@@?$StateTable@UObsoleteTypes@AAT@@X@AAT@@QEBAXAEAUhb_bit_set_t@@IAEBU?$LigatureSubtable@UObsoleteTypes@AAT@@@1@@Z 00000001800d794c     hb-aat-layout.obj
 0002:0002c94c       $unwind$??$collect_initial_glyphs@Uhb_bit_set_t@@U?$KerxSubTableFormat1@UKernAATSubTableHeader@OT@@@AAT@@@?$StateTable@UObsoleteTypes@AAT@@X@AAT@@QEBAXAEAUhb_bit_set_t@@IAEBU?$KerxSubTableFormat1@UKernAATSubTableHeader@OT@@@1@@Z 00000001800d794c     hb-ot-layout.obj
 0002:0002c94c       $unwind$??$collect_initial_glyphs@Uhb_bit_set_t@@U?$KerxSubTableFormat1@UKernOTSubTableHeader@OT@@@AAT@@@?$StateTable@UObsoleteTypes@AAT@@X@AAT@@QEBAXAEAUhb_bit_set_t@@IAEBU?$KerxSubTableFormat1@UKernOTSubTableHeader@OT@@@1@@Z 00000001800d794c     hb-ot-layout.obj
 0002:0002c964       $chain$0$??$collect_initial_glyphs@Uhb_bit_set_t@@U?$ContextualSubtable@UObsoleteTypes@AAT@@@AAT@@@?$StateTable@UObsoleteTypes@AAT@@UEntryData@?$ContextualSubtable@UObsoleteTypes@AAT@@@2@@AAT@@QEBAXAEAUhb_bit_set_t@@IAEBU?$ContextualSubtable@UObsoleteTypes@AAT@@@1@@Z 00000001800d7964     hb-aat-layout.obj
 0002:0002c978       $chain$3$??$collect_initial_glyphs@Uhb_bit_set_t@@U?$ContextualSubtable@UObsoleteTypes@AAT@@@AAT@@@?$StateTable@UObsoleteTypes@AAT@@UEntryData@?$ContextualSubtable@UObsoleteTypes@AAT@@@2@@AAT@@QEBAXAEAUhb_bit_set_t@@IAEBU?$ContextualSubtable@UObsoleteTypes@AAT@@@1@@Z 00000001800d7978     hb-aat-layout.obj
 0002:0002c994       $chain$4$??$collect_initial_glyphs@Uhb_bit_set_t@@U?$ContextualSubtable@UObsoleteTypes@AAT@@@AAT@@@?$StateTable@UObsoleteTypes@AAT@@UEntryData@?$ContextualSubtable@UObsoleteTypes@AAT@@@2@@AAT@@QEBAXAEAUhb_bit_set_t@@IAEBU?$ContextualSubtable@UObsoleteTypes@AAT@@@1@@Z 00000001800d7994     hb-aat-layout.obj
 0002:0002c9a4       $chain$5$??$collect_initial_glyphs@Uhb_bit_set_t@@U?$ContextualSubtable@UObsoleteTypes@AAT@@@AAT@@@?$StateTable@UObsoleteTypes@AAT@@UEntryData@?$ContextualSubtable@UObsoleteTypes@AAT@@@2@@AAT@@QEBAXAEAUhb_bit_set_t@@IAEBU?$ContextualSubtable@UObsoleteTypes@AAT@@@1@@Z 00000001800d79a4     hb-aat-layout.obj
 0002:0002c9b4       $chain$3$??$collect_initial_glyphs@Uhb_bit_set_t@@U?$LigatureSubtable@UObsoleteTypes@AAT@@@AAT@@@?$StateTable@UObsoleteTypes@AAT@@X@AAT@@QEBAXAEAUhb_bit_set_t@@IAEBU?$LigatureSubtable@UObsoleteTypes@AAT@@@1@@Z 00000001800d79b4     hb-aat-layout.obj
 0002:0002c9b4       $chain$3$??$collect_initial_glyphs@Uhb_bit_set_t@@U?$KerxSubTableFormat1@UKernAATSubTableHeader@OT@@@AAT@@@?$StateTable@UObsoleteTypes@AAT@@X@AAT@@QEBAXAEAUhb_bit_set_t@@IAEBU?$KerxSubTableFormat1@UKernAATSubTableHeader@OT@@@1@@Z 00000001800d79b4     hb-ot-layout.obj
 0002:0002c9b4       $chain$3$??$collect_initial_glyphs@Uhb_bit_set_t@@U?$KerxSubTableFormat1@UKernOTSubTableHeader@OT@@@AAT@@@?$StateTable@UObsoleteTypes@AAT@@X@AAT@@QEBAXAEAUhb_bit_set_t@@IAEBU?$KerxSubTableFormat1@UKernOTSubTableHeader@OT@@@1@@Z 00000001800d79b4     hb-ot-layout.obj
 0002:0002c9d4       $chain$4$??$collect_initial_glyphs@Uhb_bit_set_t@@U?$LigatureSubtable@UObsoleteTypes@AAT@@@AAT@@@?$StateTable@UObsoleteTypes@AAT@@X@AAT@@QEBAXAEAUhb_bit_set_t@@IAEBU?$LigatureSubtable@UObsoleteTypes@AAT@@@1@@Z 00000001800d79d4     hb-aat-layout.obj
 0002:0002c9d4       $chain$4$??$collect_initial_glyphs@Uhb_bit_set_t@@U?$KerxSubTableFormat1@UKernAATSubTableHeader@OT@@@AAT@@@?$StateTable@UObsoleteTypes@AAT@@X@AAT@@QEBAXAEAUhb_bit_set_t@@IAEBU?$KerxSubTableFormat1@UKernAATSubTableHeader@OT@@@1@@Z 00000001800d79d4     hb-ot-layout.obj
 0002:0002c9d4       $chain$4$??$collect_initial_glyphs@Uhb_bit_set_t@@U?$KerxSubTableFormat1@UKernOTSubTableHeader@OT@@@AAT@@@?$StateTable@UObsoleteTypes@AAT@@X@AAT@@QEBAXAEAUhb_bit_set_t@@IAEBU?$KerxSubTableFormat1@UKernOTSubTableHeader@OT@@@1@@Z 00000001800d79d4     hb-ot-layout.obj
 0002:0002c9e4       $unwind$??$collect_initial_glyphs@Uhb_bit_set_t@@U?$InsertionSubtable@UObsoleteTypes@AAT@@@AAT@@@?$StateTable@UObsoleteTypes@AAT@@UEntryData@?$InsertionSubtable@UObsoleteTypes@AAT@@@2@@AAT@@QEBAXAEAUhb_bit_set_t@@IAEBU?$InsertionSubtable@UObsoleteTypes@AAT@@@1@@Z 00000001800d79e4     hb-aat-layout.obj
 0002:0002c9fc       $chain$0$??$collect_initial_glyphs@Uhb_bit_set_t@@U?$InsertionSubtable@UObsoleteTypes@AAT@@@AAT@@@?$StateTable@UObsoleteTypes@AAT@@UEntryData@?$InsertionSubtable@UObsoleteTypes@AAT@@@2@@AAT@@QEBAXAEAUhb_bit_set_t@@IAEBU?$InsertionSubtable@UObsoleteTypes@AAT@@@1@@Z 00000001800d79fc     hb-aat-layout.obj
 0002:0002ca10       $chain$3$??$collect_initial_glyphs@Uhb_bit_set_t@@U?$InsertionSubtable@UObsoleteTypes@AAT@@@AAT@@@?$StateTable@UObsoleteTypes@AAT@@UEntryData@?$InsertionSubtable@UObsoleteTypes@AAT@@@2@@AAT@@QEBAXAEAUhb_bit_set_t@@IAEBU?$InsertionSubtable@UObsoleteTypes@AAT@@@1@@Z 00000001800d7a10     hb-aat-layout.obj
 0002:0002ca2c       $chain$4$??$collect_initial_glyphs@Uhb_bit_set_t@@U?$InsertionSubtable@UObsoleteTypes@AAT@@@AAT@@@?$StateTable@UObsoleteTypes@AAT@@UEntryData@?$InsertionSubtable@UObsoleteTypes@AAT@@@2@@AAT@@QEBAXAEAUhb_bit_set_t@@IAEBU?$InsertionSubtable@UObsoleteTypes@AAT@@@1@@Z 00000001800d7a2c     hb-aat-layout.obj
 0002:0002ca3c       $chain$5$??$collect_initial_glyphs@Uhb_bit_set_t@@U?$InsertionSubtable@UObsoleteTypes@AAT@@@AAT@@@?$StateTable@UObsoleteTypes@AAT@@UEntryData@?$InsertionSubtable@UObsoleteTypes@AAT@@@2@@AAT@@QEBAXAEAUhb_bit_set_t@@IAEBU?$InsertionSubtable@UObsoleteTypes@AAT@@@1@@Z 00000001800d7a3c     hb-aat-layout.obj
 0002:0002ca4c       $unwind$??$collect_initial_glyphs@Uhb_bit_set_t@@U?$RearrangementSubtable@UExtendedTypes@AAT@@@AAT@@@?$StateTable@UExtendedTypes@AAT@@X@AAT@@QEBAXAEAUhb_bit_set_t@@IAEBU?$RearrangementSubtable@UExtendedTypes@AAT@@@1@@Z 00000001800d7a4c     hb-aat-layout.obj
 0002:0002ca64       $chain$4$??$collect_initial_glyphs@Uhb_bit_set_t@@U?$RearrangementSubtable@UExtendedTypes@AAT@@@AAT@@@?$StateTable@UExtendedTypes@AAT@@X@AAT@@QEBAXAEAUhb_bit_set_t@@IAEBU?$RearrangementSubtable@UExtendedTypes@AAT@@@1@@Z 00000001800d7a64     hb-aat-layout.obj
 0002:0002ca88       $chain$5$??$collect_initial_glyphs@Uhb_bit_set_t@@U?$RearrangementSubtable@UExtendedTypes@AAT@@@AAT@@@?$StateTable@UExtendedTypes@AAT@@X@AAT@@QEBAXAEAUhb_bit_set_t@@IAEBU?$RearrangementSubtable@UExtendedTypes@AAT@@@1@@Z 00000001800d7a88     hb-aat-layout.obj
 0002:0002ca98       $chain$0$??$collect_initial_glyphs@Uhb_bit_set_t@@U?$ContextualSubtable@UExtendedTypes@AAT@@@AAT@@@?$StateTable@UExtendedTypes@AAT@@UEntryData@?$ContextualSubtable@UExtendedTypes@AAT@@@2@@AAT@@QEBAXAEAUhb_bit_set_t@@IAEBU?$ContextualSubtable@UExtendedTypes@AAT@@@1@@Z 00000001800d7a98     hb-aat-layout.obj
 0002:0002caac       $chain$4$??$collect_initial_glyphs@Uhb_bit_set_t@@U?$ContextualSubtable@UExtendedTypes@AAT@@@AAT@@@?$StateTable@UExtendedTypes@AAT@@UEntryData@?$ContextualSubtable@UExtendedTypes@AAT@@@2@@AAT@@QEBAXAEAUhb_bit_set_t@@IAEBU?$ContextualSubtable@UExtendedTypes@AAT@@@1@@Z 00000001800d7aac     hb-aat-layout.obj
 0002:0002cacc       $chain$5$??$collect_initial_glyphs@Uhb_bit_set_t@@U?$ContextualSubtable@UExtendedTypes@AAT@@@AAT@@@?$StateTable@UExtendedTypes@AAT@@UEntryData@?$ContextualSubtable@UExtendedTypes@AAT@@@2@@AAT@@QEBAXAEAUhb_bit_set_t@@IAEBU?$ContextualSubtable@UExtendedTypes@AAT@@@1@@Z 00000001800d7acc     hb-aat-layout.obj
 0002:0002cadc       $chain$6$??$collect_initial_glyphs@Uhb_bit_set_t@@U?$ContextualSubtable@UExtendedTypes@AAT@@@AAT@@@?$StateTable@UExtendedTypes@AAT@@UEntryData@?$ContextualSubtable@UExtendedTypes@AAT@@@2@@AAT@@QEBAXAEAUhb_bit_set_t@@IAEBU?$ContextualSubtable@UExtendedTypes@AAT@@@1@@Z 00000001800d7adc     hb-aat-layout.obj
 0002:0002caec       $chain$4$??$collect_initial_glyphs@Uhb_bit_set_t@@U?$LigatureSubtable@UExtendedTypes@AAT@@@AAT@@@?$StateTable@UExtendedTypes@AAT@@UEntryData@?$LigatureEntry@$00@2@@AAT@@QEBAXAEAUhb_bit_set_t@@IAEBU?$LigatureSubtable@UExtendedTypes@AAT@@@1@@Z 00000001800d7aec     hb-aat-layout.obj
 0002:0002cb10       $chain$5$??$collect_initial_glyphs@Uhb_bit_set_t@@U?$LigatureSubtable@UExtendedTypes@AAT@@@AAT@@@?$StateTable@UExtendedTypes@AAT@@UEntryData@?$LigatureEntry@$00@2@@AAT@@QEBAXAEAUhb_bit_set_t@@IAEBU?$LigatureSubtable@UExtendedTypes@AAT@@@1@@Z 00000001800d7b10     hb-aat-layout.obj
 0002:0002cb20       $unwind$??$collect_initial_glyphs@Uhb_bit_set_t@@U?$InsertionSubtable@UExtendedTypes@AAT@@@AAT@@@?$StateTable@UExtendedTypes@AAT@@UEntryData@?$InsertionSubtable@UExtendedTypes@AAT@@@2@@AAT@@QEBAXAEAUhb_bit_set_t@@IAEBU?$InsertionSubtable@UExtendedTypes@AAT@@@1@@Z 00000001800d7b20     hb-aat-layout.obj
 0002:0002cb38       $chain$3$??$collect_initial_glyphs@Uhb_bit_set_t@@U?$InsertionSubtable@UExtendedTypes@AAT@@@AAT@@@?$StateTable@UExtendedTypes@AAT@@UEntryData@?$InsertionSubtable@UExtendedTypes@AAT@@@2@@AAT@@QEBAXAEAUhb_bit_set_t@@IAEBU?$InsertionSubtable@UExtendedTypes@AAT@@@1@@Z 00000001800d7b38     hb-aat-layout.obj
 0002:0002cb58       $chain$4$??$collect_initial_glyphs@Uhb_bit_set_t@@U?$InsertionSubtable@UExtendedTypes@AAT@@@AAT@@@?$StateTable@UExtendedTypes@AAT@@UEntryData@?$InsertionSubtable@UExtendedTypes@AAT@@@2@@AAT@@QEBAXAEAUhb_bit_set_t@@IAEBU?$InsertionSubtable@UExtendedTypes@AAT@@@1@@Z 00000001800d7b58     hb-aat-layout.obj
 0002:0002cb68       $unwind$??$dispatch@U?$UnsizedArrayOf@U?$OffsetTo@U?$ArrayOf@UAnchor@AAT@@U?$IntType@I$03@OT@@@OT@@U?$IntType@G$01@2@X$0A@@OT@@@OT@@IAEAPEBX@hb_sanitize_context_t@@QEAA_NAEBU?$UnsizedArrayOf@U?$OffsetTo@U?$ArrayOf@UAnchor@AAT@@U?$IntType@I$03@OT@@@OT@@U?$IntType@G$01@2@X$0A@@OT@@@OT@@$$QEAIAEAPEBX@Z 00000001800d7b68     hb-aat-layout.obj
 0002:0002cb78       $chain$1$??$dispatch@U?$UnsizedArrayOf@U?$OffsetTo@U?$ArrayOf@UAnchor@AAT@@U?$IntType@I$03@OT@@@OT@@U?$IntType@G$01@2@X$0A@@OT@@@OT@@IAEAPEBX@hb_sanitize_context_t@@QEAA_NAEBU?$UnsizedArrayOf@U?$OffsetTo@U?$ArrayOf@UAnchor@AAT@@U?$IntType@I$03@OT@@@OT@@U?$IntType@G$01@2@X$0A@@OT@@@OT@@$$QEAIAEAPEBX@Z 00000001800d7b78     hb-aat-layout.obj
 0002:0002cb90       $chain$3$??$dispatch@U?$UnsizedArrayOf@U?$OffsetTo@U?$ArrayOf@UAnchor@AAT@@U?$IntType@I$03@OT@@@OT@@U?$IntType@G$01@2@X$0A@@OT@@@OT@@IAEAPEBX@hb_sanitize_context_t@@QEAA_NAEBU?$UnsizedArrayOf@U?$OffsetTo@U?$ArrayOf@UAnchor@AAT@@U?$IntType@I$03@OT@@@OT@@U?$IntType@G$01@2@X$0A@@OT@@@OT@@$$QEAIAEAPEBX@Z 00000001800d7b90     hb-aat-layout.obj
 0002:0002cba8       $unwind$??$sanitize@$$V@?$UnsizedListOfOffset16To@U?$Lookup@UHBGlyphID16@OT@@@AAT@@U?$IntType@I$03@OT@@X$0A@@OT@@QEBA_NPEAUhb_sanitize_context_t@@I@Z 00000001800d7ba8     hb-aat-layout.obj
 0002:0002cbb4       $chain$2$??$sanitize@$$V@?$UnsizedListOfOffset16To@U?$Lookup@UHBGlyphID16@OT@@@AAT@@U?$IntType@I$03@OT@@X$0A@@OT@@QEBA_NPEAUhb_sanitize_context_t@@I@Z 00000001800d7bb4     hb-aat-layout.obj
 0002:0002cbd0       $chain$4$??$sanitize@$$V@?$UnsizedListOfOffset16To@U?$Lookup@UHBGlyphID16@OT@@@AAT@@U?$IntType@I$03@OT@@X$0A@@OT@@QEBA_NPEAUhb_sanitize_context_t@@I@Z 00000001800d7bd0     hb-aat-layout.obj
 0002:0002cbec       $unwind$??$dispatch@Uhb_sanitize_context_t@@$$V@ChainContext@OT@@QEBA_NPEAUhb_sanitize_context_t@@@Z 00000001800d7bec     hb-aat-layout.obj
 0002:0002cbec       $unwind$??$dispatch@Uhb_sanitize_context_t@@$$V@Context@OT@@QEBA_NPEAUhb_sanitize_context_t@@@Z 00000001800d7bec     hb-aat-layout.obj
 0002:0002cbfc       $chain$2$??$dispatch@Uhb_sanitize_context_t@@$$V@Context@OT@@QEBA_NPEAUhb_sanitize_context_t@@@Z 00000001800d7bfc     hb-aat-layout.obj
 0002:0002cc18       $chain$3$??$dispatch@Uhb_sanitize_context_t@@$$V@Context@OT@@QEBA_NPEAUhb_sanitize_context_t@@@Z 00000001800d7c18     hb-aat-layout.obj
 0002:0002cc28       $chain$2$??$dispatch@Uhb_sanitize_context_t@@$$V@ChainContext@OT@@QEBA_NPEAUhb_sanitize_context_t@@@Z 00000001800d7c28     hb-aat-layout.obj
 0002:0002cc44       $chain$3$??$dispatch@Uhb_sanitize_context_t@@$$V@ChainContext@OT@@QEBA_NPEAUhb_sanitize_context_t@@@Z 00000001800d7c44     hb-aat-layout.obj
 0002:0002cc54       $unwind$??$dispatch@Uhb_sanitize_context_t@@$$V@SingleSubst@GSUB_impl@Layout@OT@@QEBA_NPEAUhb_sanitize_context_t@@@Z 00000001800d7c54     hb-aat-layout.obj
 0002:0002cc54       $unwind$?sanitize@OpenTypeFontFile@OT@@QEBA_NPEAUhb_sanitize_context_t@@@Z 00000001800d7c54     hb-face.obj
 0002:0002cc6c       $chain$0$??$dispatch@Uhb_sanitize_context_t@@$$V@SingleSubst@GSUB_impl@Layout@OT@@QEBA_NPEAUhb_sanitize_context_t@@@Z 00000001800d7c6c     hb-aat-layout.obj
 0002:0002cc80       $chain$1$??$dispatch@Uhb_sanitize_context_t@@$$V@SingleSubst@GSUB_impl@Layout@OT@@QEBA_NPEAUhb_sanitize_context_t@@@Z 00000001800d7c80     hb-aat-layout.obj
 0002:0002cc90       $unwind$??$dispatch@Uhb_sanitize_context_t@@$$V@AlternateSubst@GSUB_impl@Layout@OT@@QEBA_NPEAUhb_sanitize_context_t@@@Z 00000001800d7c90     hb-aat-layout.obj
 0002:0002cc90       $unwind$??$dispatch@Uhb_sanitize_context_t@@$$V@LigatureSubst@GSUB_impl@Layout@OT@@QEBA_NPEAUhb_sanitize_context_t@@@Z 00000001800d7c90     hb-aat-layout.obj
 0002:0002cc90       $unwind$??$dispatch@Uhb_sanitize_context_t@@$$V@MultipleSubst@GSUB_impl@Layout@OT@@QEBA_NPEAUhb_sanitize_context_t@@@Z 00000001800d7c90     hb-aat-layout.obj
 0002:0002cca0       $chain$2$??$dispatch@Uhb_sanitize_context_t@@$$V@AlternateSubst@GSUB_impl@Layout@OT@@QEBA_NPEAUhb_sanitize_context_t@@@Z 00000001800d7ca0     hb-aat-layout.obj
 0002:0002cca0       $chain$2$??$dispatch@Uhb_sanitize_context_t@@$$V@MultipleSubst@GSUB_impl@Layout@OT@@QEBA_NPEAUhb_sanitize_context_t@@@Z 00000001800d7ca0     hb-aat-layout.obj
 0002:0002ccbc       $chain$3$??$dispatch@Uhb_sanitize_context_t@@$$V@AlternateSubst@GSUB_impl@Layout@OT@@QEBA_NPEAUhb_sanitize_context_t@@@Z 00000001800d7cbc     hb-aat-layout.obj
 0002:0002ccbc       $chain$3$??$dispatch@Uhb_sanitize_context_t@@$$V@MultipleSubst@GSUB_impl@Layout@OT@@QEBA_NPEAUhb_sanitize_context_t@@@Z 00000001800d7cbc     hb-aat-layout.obj
 0002:0002cccc       $chain$2$??$dispatch@Uhb_sanitize_context_t@@$$V@LigatureSubst@GSUB_impl@Layout@OT@@QEBA_NPEAUhb_sanitize_context_t@@@Z 00000001800d7ccc     hb-aat-layout.obj
 0002:0002cce8       $chain$3$??$dispatch@Uhb_sanitize_context_t@@$$V@LigatureSubst@GSUB_impl@Layout@OT@@QEBA_NPEAUhb_sanitize_context_t@@@Z 00000001800d7ce8     hb-aat-layout.obj
 0002:0002ccf8       $unwind$??$dispatch@Uhb_sanitize_context_t@@$$V@?$Extension@UExtensionSubst@GSUB_impl@Layout@OT@@@OT@@QEBA_NPEAUhb_sanitize_context_t@@@Z 00000001800d7cf8     hb-aat-layout.obj
 0002:0002ccf8       $unwind$??$dispatch@Uhb_sanitize_context_t@@$$V@?$Extension@UExtensionPos@GPOS_impl@Layout@OT@@@OT@@QEBA_NPEAUhb_sanitize_context_t@@@Z 00000001800d7cf8     hb-ot-layout.obj
 0002:0002cd10       $chain$0$??$dispatch@Uhb_sanitize_context_t@@$$V@?$Extension@UExtensionSubst@GSUB_impl@Layout@OT@@@OT@@QEBA_NPEAUhb_sanitize_context_t@@@Z 00000001800d7d10     hb-aat-layout.obj
 0002:0002cd24       $chain$1$??$dispatch@Uhb_sanitize_context_t@@$$V@?$Extension@UExtensionSubst@GSUB_impl@Layout@OT@@@OT@@QEBA_NPEAUhb_sanitize_context_t@@@Z 00000001800d7d24     hb-aat-layout.obj
 0002:0002cd34       $unwind$??$collect_glyphs@Uhb_bit_set_t@@@?$ClassTable@U?$IntType@E$00@OT@@@AAT@@QEBAXAEAUhb_bit_set_t@@I@Z 00000001800d7d34     hb-aat-layout.obj
 0002:0002cd44       $chain$0$??$collect_glyphs@Uhb_bit_set_t@@@?$ClassTable@U?$IntType@E$00@OT@@@AAT@@QEBAXAEAUhb_bit_set_t@@I@Z 00000001800d7d44     hb-aat-layout.obj
 0002:0002cd58       $chain$1$??$collect_glyphs@Uhb_bit_set_t@@@?$ClassTable@U?$IntType@E$00@OT@@@AAT@@QEBAXAEAUhb_bit_set_t@@I@Z 00000001800d7d58     hb-aat-layout.obj
 0002:0002cd68       $unwind$??$collect_glyphs_filtered@Uhb_bit_set_t@@Uhb_bit_page_t@@@?$ClassTable@U?$IntType@E$00@OT@@@AAT@@QEBAXAEAUhb_bit_set_t@@IAEBUhb_bit_page_t@@@Z 00000001800d7d68     hb-aat-layout.obj
 0002:0002cd7c       $chain$0$??$collect_glyphs_filtered@Uhb_bit_set_t@@Uhb_bit_page_t@@@?$ClassTable@U?$IntType@E$00@OT@@@AAT@@QEBAXAEAUhb_bit_set_t@@IAEBUhb_bit_page_t@@@Z 00000001800d7d7c     hb-aat-layout.obj
 0002:0002cd90       $chain$1$??$collect_glyphs_filtered@Uhb_bit_set_t@@Uhb_bit_page_t@@@?$ClassTable@U?$IntType@E$00@OT@@@AAT@@QEBAXAEAUhb_bit_set_t@@IAEBUhb_bit_page_t@@@Z 00000001800d7d90     hb-aat-layout.obj
 0002:0002cda0       $chain$4$??$dispatch@U?$LigatureSet@USmallTypes@Layout@OT@@@GSUB_impl@Layout@OT@@$$V@hb_sanitize_context_t@@QEAA_NAEBU?$LigatureSet@USmallTypes@Layout@OT@@@GSUB_impl@Layout@OT@@@Z 00000001800d7da0     hb-aat-layout.obj
 0002:0002cdc4       $chain$6$??$dispatch@U?$LigatureSet@USmallTypes@Layout@OT@@@GSUB_impl@Layout@OT@@$$V@hb_sanitize_context_t@@QEAA_NAEBU?$LigatureSet@USmallTypes@Layout@OT@@@GSUB_impl@Layout@OT@@@Z 00000001800d7dc4     hb-aat-layout.obj
 0002:0002cde8       $chain$4$??$dispatch@U?$ChainRuleSet@USmallTypes@Layout@OT@@@OT@@$$V@hb_sanitize_context_t@@QEAA_NAEBU?$ChainRuleSet@USmallTypes@Layout@OT@@@OT@@@Z 00000001800d7de8     hb-aat-layout.obj
 0002:0002ce0c       $chain$6$??$dispatch@U?$ChainRuleSet@USmallTypes@Layout@OT@@@OT@@$$V@hb_sanitize_context_t@@QEAA_NAEBU?$ChainRuleSet@USmallTypes@Layout@OT@@@OT@@@Z 00000001800d7e0c     hb-aat-layout.obj
 0002:0002ce30       $chain$4$??$dispatch@U?$RuleSet@USmallTypes@Layout@OT@@@OT@@$$V@hb_sanitize_context_t@@QEAA_NAEBU?$RuleSet@USmallTypes@Layout@OT@@@OT@@@Z 00000001800d7e30     hb-aat-layout.obj
 0002:0002ce54       $chain$6$??$dispatch@U?$RuleSet@USmallTypes@Layout@OT@@@OT@@$$V@hb_sanitize_context_t@@QEAA_NAEBU?$RuleSet@USmallTypes@Layout@OT@@@OT@@@Z 00000001800d7e54     hb-aat-layout.obj
 0002:0002ce78       $unwind$??$sort_r_simple@$$V@@YAXPEAX_K1P6AHPEBX2@Z@Z 00000001800d7e78     hb-aat-map.obj
 0002:0002ce78       $unwind$??$sort_r_simple@$$V@@YAXPEAX_K1P6AHPEBX2@Z@Z 00000001800d7e78     hb-ot-font.obj
 0002:0002ce78       $unwind$??$sort_r_simple@$$V@@YAXPEAX_K1P6AHPEBX2@Z@Z 00000001800d7e78     hb-ot-map.obj
 0002:0002ce78       $unwind$??$sort_r_simple@$$V@@YAXPEAX_K1P6AHPEBX2@Z@Z 00000001800d7e78     hb-ot-shaper-arabic.obj
 0002:0002ce8c       $chain$0$??$sort_r_simple@$$V@@YAXPEAX_K1P6AHPEBX2@Z@Z 00000001800d7e8c     hb-aat-map.obj
 0002:0002ce8c       $chain$0$??$sort_r_simple@$$V@@YAXPEAX_K1P6AHPEBX2@Z@Z 00000001800d7e8c     hb-ot-font.obj
 0002:0002ce8c       $chain$0$??$sort_r_simple@$$V@@YAXPEAX_K1P6AHPEBX2@Z@Z 00000001800d7e8c     hb-ot-map.obj
 0002:0002ce8c       $chain$0$??$sort_r_simple@$$V@@YAXPEAX_K1P6AHPEBX2@Z@Z 00000001800d7e8c     hb-ot-shaper-arabic.obj
 0002:0002cea0       $chain$1$??$sort_r_simple@$$V@@YAXPEAX_K1P6AHPEBX2@Z@Z 00000001800d7ea0     hb-aat-map.obj
 0002:0002cea0       $chain$1$??$sort_r_simple@$$V@@YAXPEAX_K1P6AHPEBX2@Z@Z 00000001800d7ea0     hb-ot-font.obj
 0002:0002cea0       $chain$1$??$sort_r_simple@$$V@@YAXPEAX_K1P6AHPEBX2@Z@Z 00000001800d7ea0     hb-ot-map.obj
 0002:0002cea0       $chain$1$??$sort_r_simple@$$V@@YAXPEAX_K1P6AHPEBX2@Z@Z 00000001800d7ea0     hb-ot-shaper-arabic.obj
 0002:0002ceb0       $unwind$?add_feature@hb_aat_map_builder_t@@QEAAXAEBUhb_feature_t@@@Z 00000001800d7eb0     hb-aat-map.obj
 0002:0002ceb0       $unwind$?_hb_options_init@@YAXXZ 00000001800d7eb0     hb-common.obj
 0002:0002cebc       $chain$0$?add_feature@hb_aat_map_builder_t@@QEAAXAEBUhb_feature_t@@@Z 00000001800d7ebc     hb-aat-map.obj
 0002:0002ced0       $chain$3$?add_feature@hb_aat_map_builder_t@@QEAAXAEBUhb_feature_t@@@Z 00000001800d7ed0     hb-aat-map.obj
 0002:0002cee4       $chain$4$?add_feature@hb_aat_map_builder_t@@QEAAXAEBUhb_feature_t@@@Z 00000001800d7ee4     hb-aat-map.obj
 0002:0002cef8       $chain$5$?add_feature@hb_aat_map_builder_t@@QEAAXAEBUhb_feature_t@@@Z 00000001800d7ef8     hb-aat-map.obj
 0002:0002cf08       $chain$2$?add_feature@hb_aat_map_builder_t@@QEAAXAEBUhb_feature_t@@@Z 00000001800d7f08     hb-aat-map.obj
 0002:0002cf1c       $chain$6$?add_feature@hb_aat_map_builder_t@@QEAAXAEBUhb_feature_t@@@Z 00000001800d7f1c     hb-aat-map.obj
 0002:0002cf2c       $unwind$?compile@hb_aat_map_builder_t@@QEAAXAEAUhb_aat_map_t@@@Z 00000001800d7f2c     hb-aat-map.obj
 0002:0002cf38       $chain$0$?compile@hb_aat_map_builder_t@@QEAAXAEAUhb_aat_map_t@@@Z 00000001800d7f38     hb-aat-map.obj
 0002:0002cf4c       $chain$5$?compile@hb_aat_map_builder_t@@QEAAXAEAUhb_aat_map_t@@@Z 00000001800d7f4c     hb-aat-map.obj
 0002:0002cf70       $chain$6$?compile@hb_aat_map_builder_t@@QEAAXAEAUhb_aat_map_t@@@Z 00000001800d7f70     hb-aat-map.obj
 0002:0002cf84       $chain$7$?compile@hb_aat_map_builder_t@@QEAAXAEAUhb_aat_map_t@@@Z 00000001800d7f84     hb-aat-map.obj
 0002:0002cf98       $chain$8$?compile@hb_aat_map_builder_t@@QEAAXAEAUhb_aat_map_t@@@Z 00000001800d7f98     hb-aat-map.obj
 0002:0002cfa8       $chain$0$?alloc@?$hb_vector_t@Ufeature_info_t@hb_aat_map_builder_t@@$00@@QEAA_NI_N@Z 00000001800d7fa8     hb-aat-map.obj
 0002:0002cfbc       $chain$2$?alloc@?$hb_vector_t@Ufeature_info_t@hb_aat_map_builder_t@@$00@@QEAA_NI_N@Z 00000001800d7fbc     hb-aat-map.obj
 0002:0002cfbc       $chain$4$?alloc@?$hb_vector_t@Ufeature_info_t@hb_aat_map_builder_t@@$00@@QEAA_NI_N@Z 00000001800d7fbc     hb-aat-map.obj
 0002:0002cfd0       $unwind$hb_blob_create     00000001800d7fd0     hb-blob.obj
 0002:0002cfd0       $unwind$?resolve_links@hb_serialize_context_t@@QEAAXXZ 00000001800d7fd0     hb-face-builder.obj
 0002:0002cfd0       $unwind$hb_font_draw_glyph 00000001800d7fd0     hb-font.obj
 0002:0002cfd0       $unwind$hb_font_get_nominal_glyph 00000001800d7fd0     hb-font.obj
 0002:0002cfd0       $unwind$?reference_table@@YAPEAUhb_blob_t@@PEAUhb_face_t@@IPEAX@Z 00000001800d7fd0     hb-jdk-font-p.obj
 0002:0002cfd0       $unwind$?get_path@accelerator_t@cff1@OT@@QEBA_NPEAUhb_font_t@@IAEAUhb_draw_session_t@@@Z 00000001800d7fd0     hb-ot-cff1-table.obj
 0002:0002cfd0       $unwind$?hhcurveto@?$path_procs_t@Ucff1_path_procs_extents_t@@Ucff1_cs_interp_env_t@CFF@@Ucff1_extents_param_t@@@CFF@@SAXAEAUcff1_cs_interp_env_t@2@AEAUcff1_extents_param_t@@@Z 00000001800d7fd0     hb-ot-cff1-table.obj
 0002:0002cfd0       $unwind$?vvcurveto@?$path_procs_t@Ucff1_path_procs_extents_t@@Ucff1_cs_interp_env_t@CFF@@Ucff1_extents_param_t@@@CFF@@SAXAEAUcff1_cs_interp_env_t@2@AEAUcff1_extents_param_t@@@Z 00000001800d7fd0     hb-ot-cff1-table.obj
 0002:0002cfd0       $unwind$?compose_unicode@hb_ot_shape_normalize_context_t@@SA_NPEBU1@IIPEAI@Z 00000001800d7fd0     hb-ot-shape-normalize.obj
 0002:0002cfd0       $unwind$?decompose_unicode@hb_ot_shape_normalize_context_t@@SA_NPEBU1@IPEAI1@Z 00000001800d7fd0     hb-ot-shape-normalize.obj
 0002:0002cfd0       $unwind$?has_glyph@hb_font_t@@QEAA_NI@Z 00000001800d7fd0     hb-ot-shape.obj
 0002:0002cfd0       $unwind$?decompose_indic@@YA_NPEBUhb_ot_shape_normalize_context_t@@IPEAI1@Z 00000001800d7fd0     hb-ot-shaper-indic.obj
 0002:0002cfd0       $unwind$?decompose_khmer@@YA_NPEBUhb_ot_shape_normalize_context_t@@IPEAI1@Z 00000001800d7fd0     hb-ot-shaper-khmer.obj
 0002:0002cfd0       $unwind$?hb_paint_extents_push_clip_rectangle@@YAXPEAUhb_paint_funcs_t@@PEAXMMMM1@Z 00000001800d7fd0     hb-paint-extents.obj
 0002:0002cfd8       $unwind$hb_blob_create_from_file_or_fail 00000001800d7fd8     hb-blob.obj
 0002:0002cfd8       $unwind$?process_op@cff1_top_dict_opset_t@CFF@@SAXIAEAUcff1_top_dict_interp_env_t@2@AEAUcff1_top_dict_values_t@2@@Z 00000001800d7fd8     hb-ot-font.obj
 0002:0002cff0       $chain$2$hb_blob_create_sub_blob 00000001800d7ff0     hb-blob.obj
 0002:0002d00c       $chain$3$hb_blob_create_sub_blob 00000001800d800c     hb-blob.obj
 0002:0002d01c       $unwind$?_hb_blob_destroy@@YAXPEAX@Z 00000001800d801c     hb-blob.obj
 0002:0002d01c       $unwind$hb_blob_destroy    00000001800d801c     hb-blob.obj
 0002:0002d024       $chain$0$hb_blob_destroy   00000001800d8024     hb-blob.obj
 0002:0002d038       $chain$1$hb_blob_destroy   00000001800d8038     hb-blob.obj
 0002:0002d048       $unwind$?fini@hb_user_data_array_t@@QEAAXXZ 00000001800d8048     hb-blob.obj
 0002:0002d048       $unwind$?hb_font_get_glyph_contour_point_default@@YAHPEAUhb_font_t@@PEAXIIPEAH21@Z 00000001800d8048     hb-font.obj
 0002:0002d05c       $unwind$?try_make_writable@hb_blob_t@@QEAA_NXZ 00000001800d805c     hb-blob.obj
 0002:0002d068       $chain$1$?try_make_writable@hb_blob_t@@QEAA_NXZ 00000001800d8068     hb-blob.obj
 0002:0002d080       $chain$3$?try_make_writable@hb_blob_t@@QEAA_NXZ 00000001800d8080     hb-blob.obj
 0002:0002d098       $chain$4$?try_make_writable@hb_blob_t@@QEAA_NXZ 00000001800d8098     hb-blob.obj
 0002:0002d0a8       $chain$0$?_hb_blob_destroy@@YAXPEAX@Z 00000001800d80a8     hb-blob.obj
 0002:0002d0bc       $chain$1$?_hb_blob_destroy@@YAXPEAX@Z 00000001800d80bc     hb-blob.obj
 0002:0002d0cc       $unwind$hb_buffer_serialize_unicode 00000001800d80cc     hb-buffer-serialize.obj
 0002:0002d0f0       $unwind$snprintf           00000001800d80f0     hb-buffer-serialize.obj
 0002:0002d100       $unwind$fprintf            00000001800d8100     hb-buffer-verify.obj
 0002:0002d10c       $unwind$?verify@hb_buffer_t@@QEAA_NPEAU1@PEAUhb_font_t@@PEBUhb_feature_t@@IPEBQEBD@Z 00000001800d810c     hb-buffer-verify.obj
 0002:0002d124       $unwind$?buffer_verify_error@@YAXPEAUhb_buffer_t@@PEAUhb_font_t@@PEBDZZ 00000001800d8124     hb-buffer-verify.obj
 0002:0002d134       $unwind$?buffer_verify_unsafe_to_break@@YA_NPEAUhb_buffer_t@@0PEAUhb_font_t@@PEBUhb_feature_t@@IPEBQEBD@Z 00000001800d8134     hb-buffer-verify.obj
 0002:0002d140       $chain$5$?buffer_verify_unsafe_to_break@@YA_NPEAUhb_buffer_t@@0PEAUhb_font_t@@PEBUhb_feature_t@@IPEBQEBD@Z 00000001800d8140     hb-buffer-verify.obj
 0002:0002d168       $chain$7$?buffer_verify_unsafe_to_break@@YA_NPEAUhb_buffer_t@@0PEAUhb_font_t@@PEBUhb_feature_t@@IPEBQEBD@Z 00000001800d8168     hb-buffer-verify.obj
 0002:0002d190       $unwind$?buffer_verify_unsafe_to_concat@@YA_NPEAUhb_buffer_t@@0PEAUhb_font_t@@PEBUhb_feature_t@@IPEBQEBD@Z 00000001800d8190     hb-buffer-verify.obj
 0002:0002d1b4       $unwind$hb_buffer_destroy  00000001800d81b4     hb-buffer.obj
 0002:0002d1b4       $unwind$hb_draw_funcs_destroy 00000001800d81b4     hb-draw.obj
 0002:0002d1b4       $unwind$hb_font_destroy    00000001800d81b4     hb-font.obj
 0002:0002d1b4       $unwind$hb_font_funcs_destroy 00000001800d81b4     hb-font.obj
 0002:0002d1b4       $unwind$?arabic_fallback_plan_destroy@@YAXPEAUarabic_fallback_plan_t@@@Z 00000001800d81b4     hb-ot-shaper-arabic.obj
 0002:0002d1b4       $unwind$hb_paint_funcs_destroy 00000001800d81b4     hb-paint.obj
 0002:0002d1b4       $unwind$hb_unicode_funcs_destroy 00000001800d81b4     hb-unicode.obj
 0002:0002d1bc       $chain$0$hb_buffer_destroy 00000001800d81bc     hb-buffer.obj
 0002:0002d1d0       $chain$1$hb_buffer_destroy 00000001800d81d0     hb-buffer.obj
 0002:0002d1e0       $unwind$hb_buffer_append   00000001800d81e0     hb-buffer.obj
 0002:0002d1ec       $chain$0$hb_buffer_append  00000001800d81ec     hb-buffer.obj
 0002:0002d200       $chain$6$hb_buffer_append  00000001800d8200     hb-buffer.obj
 0002:0002d224       $chain$7$hb_buffer_append  00000001800d8224     hb-buffer.obj
 0002:0002d234       $unwind$hb_buffer_diff     00000001800d8234     hb-buffer.obj
 0002:0002d244       $chain$0$hb_buffer_diff    00000001800d8244     hb-buffer.obj
 0002:0002d258       $chain$2$hb_buffer_diff    00000001800d8258     hb-buffer.obj
 0002:0002d26c       $chain$3$hb_buffer_diff    00000001800d826c     hb-buffer.obj
 0002:0002d280       $chain$4$hb_buffer_diff    00000001800d8280     hb-buffer.obj
 0002:0002d290       $unwind$?sync@hb_buffer_t@@QEAA_NXZ 00000001800d8290     hb-buffer.obj
 0002:0002d29c       $chain$1$?sync@hb_buffer_t@@QEAA_NXZ 00000001800d829c     hb-buffer.obj
 0002:0002d2b4       $chain$2$?sync@hb_buffer_t@@QEAA_NXZ 00000001800d82b4     hb-buffer.obj
 0002:0002d2c4       $unwind$?sync_so_far@hb_buffer_t@@QEAAHXZ 00000001800d82c4     hb-buffer.obj
 0002:0002d2d0       $chain$1$?sync_so_far@hb_buffer_t@@QEAAHXZ 00000001800d82d0     hb-buffer.obj
 0002:0002d2e8       $chain$4$?sync_so_far@hb_buffer_t@@QEAAHXZ 00000001800d82e8     hb-buffer.obj
 0002:0002d304       $chain$5$?sync_so_far@hb_buffer_t@@QEAAHXZ 00000001800d8304     hb-buffer.obj
 0002:0002d314       $chain$6$?sync_so_far@hb_buffer_t@@QEAAHXZ 00000001800d8314     hb-buffer.obj
 0002:0002d324       $unwind$?set_masks@hb_buffer_t@@QEAAXIIII@Z 00000001800d8324     hb-buffer.obj
 0002:0002d330       $unwind$?merge_clusters_impl@hb_buffer_t@@QEAAXII@Z 00000001800d8330     hb-buffer.obj
 0002:0002d330       $unwind$?_glyf_get_leading_bearing_with_var_unscaled@@YA_NPEAUhb_font_t@@I_NPEAH@Z 00000001800d8330     hb-common.obj
 0002:0002d330       $unwind$?get_advance_delta_unscaled@HVARVVAR@OT@@QEBAMIPEBHIPEAU?$hb_atomic_t@H@@@Z 00000001800d8330     hb-ot-font.obj
 0002:0002d330       $unwind$?get_extents@ClipList@OT@@QEBA_NIPEAUhb_glyph_extents_t@@AEBUItemVarStoreInstancer@2@@Z 00000001800d8330     hb-ot-font.obj
 0002:0002d330       $unwind$?process_op@cff2_top_dict_opset_t@CFF@@SAXIAEAU?$interp_env_t@Unumber_t@CFF@@@2@AEAUcff2_top_dict_values_t@2@@Z 00000001800d8330     hb-ot-font.obj
 0002:0002d330       $unwind$?compose_indic@@YA_NPEBUhb_ot_shape_normalize_context_t@@IIPEAI@Z 00000001800d8330     hb-ot-shaper-indic.obj
 0002:0002d344       $chain$1$?merge_out_clusters@hb_buffer_t@@QEAAXII@Z 00000001800d8344     hb-buffer.obj
 0002:0002d35c       $chain$2$?merge_out_clusters@hb_buffer_t@@QEAAXII@Z 00000001800d835c     hb-buffer.obj
 0002:0002d370       $chain$3$?merge_out_clusters@hb_buffer_t@@QEAAXII@Z 00000001800d8370     hb-buffer.obj
 0002:0002d380       $unwind$?delete_glyphs_inplace@hb_buffer_t@@QEAAXP6A_NPEBUhb_glyph_info_t@@@Z@Z 00000001800d8380     hb-buffer.obj
 0002:0002d390       $chain$2$?delete_glyphs_inplace@hb_buffer_t@@QEAAXP6A_NPEBUhb_glyph_info_t@@@Z@Z 00000001800d8390     hb-buffer.obj
 0002:0002d3ac       $chain$3$?delete_glyphs_inplace@hb_buffer_t@@QEAAXP6A_NPEBUhb_glyph_info_t@@@Z@Z 00000001800d83ac     hb-buffer.obj
 0002:0002d3bc       $chain$0$?move_to@hb_buffer_t@@QEAA_NI@Z 00000001800d83bc     hb-buffer.obj
 0002:0002d3d0       $chain$2$?move_to@hb_buffer_t@@QEAA_NI@Z 00000001800d83d0     hb-buffer.obj
 0002:0002d3d0       $chain$4$?move_to@hb_buffer_t@@QEAA_NI@Z 00000001800d83d0     hb-buffer.obj
 0002:0002d3e4       $unwind$?enlarge@hb_buffer_t@@QEAA_NI@Z 00000001800d83e4     hb-buffer.obj
 0002:0002d3e4       $unwind$?alloc@?$hb_vector_t@U?$cff1_private_dict_values_base_t@Udict_val_t@CFF@@@CFF@@$0A@@@QEAA_NI_N@Z 00000001800d83e4     hb-ot-font.obj
 0002:0002d3e4       $unwind$?alloc@?$hb_vector_t@U?$cff2_private_dict_values_base_t@Udict_val_t@CFF@@@CFF@@$0A@@@QEAA_NI_N@Z 00000001800d83e4     hb-ot-font.obj
 0002:0002d3e4       $unwind$?alloc@?$hb_vector_t@Ucff1_font_dict_values_t@CFF@@$0A@@@QEAA_NI_N@Z 00000001800d83e4     hb-ot-font.obj
 0002:0002d3e4       $unwind$?alloc@?$hb_vector_t@Ucff2_font_dict_values_t@CFF@@$0A@@@QEAA_NI_N@Z 00000001800d83e4     hb-ot-font.obj
 0002:0002d3e4       $unwind$?discard_stale_objects@hb_serialize_context_t@@QEAAXXZ 00000001800d83e4     hb-ot-shaper-arabic.obj
 0002:0002d3ec       $chain$4$?enlarge@hb_buffer_t@@QEAA_NI@Z 00000001800d83ec     hb-buffer.obj
 0002:0002d410       $chain$5$?enlarge@hb_buffer_t@@QEAA_NI@Z 00000001800d8410     hb-buffer.obj
 0002:0002d424       $chain$6$?enlarge@hb_buffer_t@@QEAA_NI@Z 00000001800d8424     hb-buffer.obj
 0002:0002d434       $chain$7$?enlarge@hb_buffer_t@@QEAA_NI@Z 00000001800d8434     hb-buffer.obj
 0002:0002d454       $chain$8$?enlarge@hb_buffer_t@@QEAA_NI@Z 00000001800d8454     hb-buffer.obj
 0002:0002d46c       $chain$9$?enlarge@hb_buffer_t@@QEAA_NI@Z 00000001800d846c     hb-buffer.obj
 0002:0002d480       $unwind$?ensure@hb_buffer_t@@QEAA_NI@Z 00000001800d8480     hb-buffer.obj
 0002:0002d48c       $chain$3$?ensure@hb_buffer_t@@QEAA_NI@Z 00000001800d848c     hb-buffer.obj
 0002:0002d4ac       $chain$4$?ensure@hb_buffer_t@@QEAA_NI@Z 00000001800d84ac     hb-buffer.obj
 0002:0002d4c0       $chain$5$?ensure@hb_buffer_t@@QEAA_NI@Z 00000001800d84c0     hb-buffer.obj
 0002:0002d4d0       $chain$6$?ensure@hb_buffer_t@@QEAA_NI@Z 00000001800d84d0     hb-buffer.obj
 0002:0002d4ec       $chain$7$?ensure@hb_buffer_t@@QEAA_NI@Z 00000001800d84ec     hb-buffer.obj
 0002:0002d500       $chain$8$?ensure@hb_buffer_t@@QEAA_NI@Z 00000001800d8500     hb-buffer.obj
 0002:0002d510       $unwind$?sort@hb_buffer_t@@QEAAXIIP6AHPEBUhb_glyph_info_t@@0@Z@Z 00000001800d8510     hb-buffer.obj
 0002:0002d51c       $chain$4$?sort@hb_buffer_t@@QEAAXIIP6AHPEBUhb_glyph_info_t@@0@Z@Z 00000001800d851c     hb-buffer.obj
 0002:0002d540       $chain$5$?sort@hb_buffer_t@@QEAAXIIP6AHPEBUhb_glyph_info_t@@0@Z@Z 00000001800d8540     hb-buffer.obj
 0002:0002d550       $unwind$?message_impl@hb_buffer_t@@QEAA_NPEAUhb_font_t@@PEBDPEAD@Z 00000001800d8550     hb-buffer.obj
 0002:0002d568       $unwind$??$reverse_groups@$$A6A_NAEBUhb_glyph_info_t@@0@Z@hb_buffer_t@@QEAAXA6A_NAEBUhb_glyph_info_t@@0@Z_N@Z 00000001800d8568     hb-buffer.obj
 0002:0002d574       $chain$1$??$reverse_groups@$$A6A_NAEBUhb_glyph_info_t@@0@Z@hb_buffer_t@@QEAAXA6A_NAEBUhb_glyph_info_t@@0@Z_N@Z 00000001800d8574     hb-buffer.obj
 0002:0002d58c       $chain$2$??$reverse_groups@$$A6A_NAEBUhb_glyph_info_t@@0@Z@hb_buffer_t@@QEAAXA6A_NAEBUhb_glyph_info_t@@0@Z_N@Z 00000001800d858c     hb-buffer.obj
 0002:0002d5a0       $chain$3$??$reverse_groups@$$A6A_NAEBUhb_glyph_info_t@@0@Z@hb_buffer_t@@QEAAXA6A_NAEBUhb_glyph_info_t@@0@Z_N@Z 00000001800d85a0     hb-buffer.obj
 0002:0002d5b0       $chain$4$??$reverse_groups@$$A6A_NAEBUhb_glyph_info_t@@0@Z@hb_buffer_t@@QEAAXA6A_NAEBUhb_glyph_info_t@@0@Z_N@Z 00000001800d85b0     hb-buffer.obj
 0002:0002d5c0       $unwind$??$hb_buffer_add_utf@U?$hb_utf16_xe_t@G@@@@YAXPEAUhb_buffer_t@@PEBGHIH@Z 00000001800d85c0     hb-buffer.obj
 0002:0002d5d0       $chain$0$??$hb_buffer_add_utf@U?$hb_utf16_xe_t@G@@@@YAXPEAUhb_buffer_t@@PEBGHIH@Z 00000001800d85d0     hb-buffer.obj
 0002:0002d5e4       $chain$1$??$hb_buffer_add_utf@U?$hb_utf16_xe_t@G@@@@YAXPEAUhb_buffer_t@@PEBGHIH@Z 00000001800d85e4     hb-buffer.obj
 0002:0002d5f8       $chain$2$??$hb_buffer_add_utf@U?$hb_utf16_xe_t@G@@@@YAXPEAUhb_buffer_t@@PEBGHIH@Z 00000001800d85f8     hb-buffer.obj
 0002:0002d60c       $chain$3$??$hb_buffer_add_utf@U?$hb_utf16_xe_t@G@@@@YAXPEAUhb_buffer_t@@PEBGHIH@Z 00000001800d860c     hb-buffer.obj
 0002:0002d61c       $chain$4$??$hb_buffer_add_utf@U?$hb_utf16_xe_t@G@@@@YAXPEAUhb_buffer_t@@PEBGHIH@Z 00000001800d861c     hb-buffer.obj
 0002:0002d62c       $chain$5$??$hb_buffer_add_utf@U?$hb_utf16_xe_t@G@@@@YAXPEAUhb_buffer_t@@PEBGHIH@Z 00000001800d862c     hb-buffer.obj
 0002:0002d63c       $unwind$hb_language_from_string 00000001800d863c     hb-common.obj
 0002:0002d64c       $chain$0$hb_language_from_string 00000001800d864c     hb-common.obj
 0002:0002d660       $chain$2$hb_language_from_string 00000001800d8660     hb-common.obj
 0002:0002d660       $chain$4$hb_language_from_string 00000001800d8660     hb-common.obj
 0002:0002d674       $chain$3$hb_language_from_string 00000001800d8674     hb-common.obj
 0002:0002d684       $chain$0$hb_language_matches 00000001800d8684     hb-common.obj
 0002:0002d698       $chain$2$hb_language_matches 00000001800d8698     hb-common.obj
 0002:0002d6ac       $chain$3$hb_language_matches 00000001800d86ac     hb-common.obj
 0002:0002d6bc       $unwind$hb_feature_from_string 00000001800d86bc     hb-common.obj
 0002:0002d6c4       $chain$1$?_hb_options_init@@YAXXZ 00000001800d86c4     hb-common.obj
 0002:0002d6dc       $chain$2$?_hb_options_init@@YAXXZ 00000001800d86dc     hb-common.obj
 0002:0002d6ec       $unwind$?lang_find_or_insert@@YAPEAUhb_language_item_t@@PEBD@Z 00000001800d86ec     hb-common.obj
 0002:0002d700       $unwind$?parse_feature_indices@@YA_NPEAPEBDPEBDPEAUhb_feature_t@@@Z 00000001800d8700     hb-common.obj
 0002:0002d710       $unwind$?parse_one_feature@@YA_NPEAPEBDPEBDPEAUhb_feature_t@@@Z 00000001800d8710     hb-common.obj
 0002:0002d710       $unwind$hb_draw_funcs_set_close_path_func 00000001800d8710     hb-draw.obj
 0002:0002d710       $unwind$hb_draw_funcs_set_cubic_to_func 00000001800d8710     hb-draw.obj
 0002:0002d710       $unwind$hb_draw_funcs_set_line_to_func 00000001800d8710     hb-draw.obj
 0002:0002d710       $unwind$hb_draw_funcs_set_move_to_func 00000001800d8710     hb-draw.obj
 0002:0002d710       $unwind$hb_draw_funcs_set_quadratic_to_func 00000001800d8710     hb-draw.obj
 0002:0002d710       $unwind$hb_font_funcs_set_draw_glyph_or_fail_func 00000001800d8710     hb-font.obj
 0002:0002d710       $unwind$hb_font_funcs_set_font_h_extents_func 00000001800d8710     hb-font.obj
 0002:0002d710       $unwind$hb_font_funcs_set_font_v_extents_func 00000001800d8710     hb-font.obj
 0002:0002d710       $unwind$hb_font_funcs_set_glyph_contour_point_func 00000001800d8710     hb-font.obj
 0002:0002d710       $unwind$hb_font_funcs_set_glyph_extents_func 00000001800d8710     hb-font.obj
 0002:0002d710       $unwind$hb_font_funcs_set_glyph_from_name_func 00000001800d8710     hb-font.obj
 0002:0002d710       $unwind$hb_font_funcs_set_glyph_h_advance_func 00000001800d8710     hb-font.obj
 0002:0002d710       $unwind$hb_font_funcs_set_glyph_h_advances_func 00000001800d8710     hb-font.obj
 0002:0002d710       $unwind$hb_font_funcs_set_glyph_h_kerning_func 00000001800d8710     hb-font.obj
 0002:0002d710       $unwind$hb_font_funcs_set_glyph_h_origin_func 00000001800d8710     hb-font.obj
 0002:0002d710       $unwind$hb_font_funcs_set_glyph_name_func 00000001800d8710     hb-font.obj
 0002:0002d710       $unwind$hb_font_funcs_set_glyph_v_advance_func 00000001800d8710     hb-font.obj
 0002:0002d710       $unwind$hb_font_funcs_set_glyph_v_advances_func 00000001800d8710     hb-font.obj
 0002:0002d710       $unwind$hb_font_funcs_set_glyph_v_kerning_func 00000001800d8710     hb-font.obj
 0002:0002d710       $unwind$hb_font_funcs_set_glyph_v_origin_func 00000001800d8710     hb-font.obj
 0002:0002d710       $unwind$hb_font_funcs_set_nominal_glyph_func 00000001800d8710     hb-font.obj
 0002:0002d710       $unwind$hb_font_funcs_set_nominal_glyphs_func 00000001800d8710     hb-font.obj
 0002:0002d710       $unwind$hb_font_funcs_set_paint_glyph_or_fail_func 00000001800d8710     hb-font.obj
 0002:0002d710       $unwind$hb_font_funcs_set_variation_glyph_func 00000001800d8710     hb-font.obj
 0002:0002d710       $unwind$hb_paint_funcs_set_color_func 00000001800d8710     hb-paint.obj
 0002:0002d710       $unwind$hb_paint_funcs_set_image_func 00000001800d8710     hb-paint.obj
 0002:0002d710       $unwind$hb_paint_funcs_set_linear_gradient_func 00000001800d8710     hb-paint.obj
 0002:0002d710       $unwind$hb_paint_funcs_set_pop_clip_func 00000001800d8710     hb-paint.obj
 0002:0002d710       $unwind$hb_paint_funcs_set_pop_group_func 00000001800d8710     hb-paint.obj
 0002:0002d710       $unwind$hb_paint_funcs_set_pop_transform_func 00000001800d8710     hb-paint.obj
 0002:0002d710       $unwind$hb_paint_funcs_set_push_clip_glyph_func 00000001800d8710     hb-paint.obj
 0002:0002d710       $unwind$hb_paint_funcs_set_push_clip_rectangle_func 00000001800d8710     hb-paint.obj
 0002:0002d710       $unwind$hb_paint_funcs_set_push_group_func 00000001800d8710     hb-paint.obj
 0002:0002d710       $unwind$hb_paint_funcs_set_push_transform_func 00000001800d8710     hb-paint.obj
 0002:0002d710       $unwind$hb_paint_funcs_set_radial_gradient_func 00000001800d8710     hb-paint.obj
 0002:0002d710       $unwind$hb_paint_funcs_set_sweep_gradient_func 00000001800d8710     hb-paint.obj
 0002:0002d724       $chain$1$?get@?$hb_lazy_loader_t@Uhead@OT@@U?$hb_table_lazy_loader_t@Uhead@OT@@$00$00@@Uhb_face_t@@$00Uhb_blob_t@@@@QEBAPEBUhead@OT@@XZ 00000001800d8724     hb-common.obj
 0002:0002d73c       $chain$2$?get@?$hb_lazy_loader_t@Uhead@OT@@U?$hb_table_lazy_loader_t@Uhead@OT@@$00$00@@Uhb_face_t@@$00Uhb_blob_t@@@@QEBAPEBUhead@OT@@XZ 00000001800d873c     hb-common.obj
 0002:0002d74c       $chain$1$??C?$hb_lazy_loader_t@Umaxp@OT@@U?$hb_table_lazy_loader_t@Umaxp@OT@@$01$00@@Uhb_face_t@@$01Uhb_blob_t@@@@QEBAPEBUmaxp@OT@@XZ 00000001800d874c     hb-common.obj
 0002:0002d764       $chain$2$??C?$hb_lazy_loader_t@Umaxp@OT@@U?$hb_table_lazy_loader_t@Umaxp@OT@@$01$00@@Uhb_face_t@@$01Uhb_blob_t@@@@QEBAPEBUmaxp@OT@@XZ 00000001800d8764     hb-common.obj
 0002:0002d774       $chain$1$??C?$hb_lazy_loader_t@Uhhea@OT@@U?$hb_table_lazy_loader_t@Uhhea@OT@@$03$00@@Uhb_face_t@@$03Uhb_blob_t@@@@QEBAPEBUhhea@OT@@XZ 00000001800d8774     hb-common.obj
 0002:0002d78c       $chain$2$??C?$hb_lazy_loader_t@Uhhea@OT@@U?$hb_table_lazy_loader_t@Uhhea@OT@@$03$00@@Uhb_face_t@@$03Uhb_blob_t@@@@QEBAPEBUhhea@OT@@XZ 00000001800d878c     hb-common.obj
 0002:0002d79c       $chain$1$??C?$hb_lazy_loader_t@Uvhea@OT@@U?$hb_table_lazy_loader_t@Uvhea@OT@@$0L@$00@@Uhb_face_t@@$0L@Uhb_blob_t@@@@QEBAPEBUvhea@OT@@XZ 00000001800d879c     hb-common.obj
 0002:0002d7b4       $chain$2$??C?$hb_lazy_loader_t@Uvhea@OT@@U?$hb_table_lazy_loader_t@Uvhea@OT@@$0L@$00@@Uhb_face_t@@$0L@Uhb_blob_t@@@@QEBAPEBUvhea@OT@@XZ 00000001800d87b4     hb-common.obj
 0002:0002d7c4       $unwind$?scale_glyph_extents@hb_font_t@@QEAAXPEAUhb_glyph_extents_t@@@Z 00000001800d87c4     hb-common.obj
 0002:0002d7e4       $unwind$?extend@?$hb_vector_t@Ucontour_point_t@@$0A@@@QEAAXU?$hb_array_t@Ucontour_point_t@@@@@Z 00000001800d87e4     hb-common.obj
 0002:0002d7e4       $unwind$?hb_paint_extents_push_clip_glyph@@YAXPEAUhb_paint_funcs_t@@PEAXIPEAUhb_font_t@@1@Z 00000001800d87e4     hb-paint-extents.obj
 0002:0002d7e4       $unwind$?push_clip@hb_paint_extents_context_t@@QEAAXUhb_extents_t@@@Z 00000001800d87e4     hb-paint-extents.obj
 0002:0002d7f4       $chain$0$?alloc@?$hb_vector_t@Ucontour_point_t@@$0A@@@QEAA_NI_N@Z 00000001800d87f4     hb-common.obj
 0002:0002d808       $chain$2$?alloc@?$hb_vector_t@Ucontour_point_t@@$0A@@@QEAA_NI_N@Z 00000001800d8808     hb-common.obj
 0002:0002d808       $chain$4$?alloc@?$hb_vector_t@Ucontour_point_t@@$0A@@@QEAA_NI_N@Z 00000001800d8808     hb-common.obj
 0002:0002d81c       $unwind$?sanitize@DeltaSetIndexMap@OT@@QEBA_NPEAUhb_sanitize_context_t@@@Z 00000001800d881c     hb-common.obj
 0002:0002d834       $chain$0$?sanitize@DeltaSetIndexMap@OT@@QEBA_NPEAUhb_sanitize_context_t@@@Z 00000001800d8834     hb-common.obj
 0002:0002d848       $chain$1$?sanitize@DeltaSetIndexMap@OT@@QEBA_NPEAUhb_sanitize_context_t@@@Z 00000001800d8848     hb-common.obj
 0002:0002d858       $unwind$?calculate_scalar@TupleVariationHeader@OT@@QEBANU?$hb_array_t@$$CBH@@IU?$hb_array_t@$$CBU?$HBFixed@U?$IntType@F$01@OT@@$0O@@OT@@@@PEBU?$hb_vector_t@U?$hb_pair_t@HH@@$0A@@@@Z 00000001800d8858     hb-common.obj
 0002:0002d874       $unwind$?decompile_points@?$TupleVariationData@U?$IntType@G$01@OT@@@OT@@SA_NAEAPEBU?$IntType@E$00@2@AEAU?$hb_vector_t@I$0A@@@PEBU32@@Z 00000001800d8874     hb-common.obj
 0002:0002d874       $unwind$?add_op@?$parsed_values_t@Udict_val_t@CFF@@@CFF@@QEAAXIAEBUbyte_str_ref_t@2@AEBUdict_val_t@2@@Z 00000001800d8874     hb-ot-font.obj
 0002:0002d874       $unwind$?add_op@?$parsed_values_t@Uop_str_t@CFF@@@CFF@@QEAAXIAEBUbyte_str_ref_t@2@AEBUop_str_t@2@@Z 00000001800d8874     hb-ot-font.obj
 0002:0002d874       $unwind$?_hb_ot_metrics_get_position_common@@YA_NPEAUhb_font_t@@W4hb_ot_metrics_tag_t@@PEAH@Z 00000001800d8874     hb-ot-metrics.obj
 0002:0002d874       $unwind$?initial_reordering_consonant_syllable@@YAXPEAUhb_buffer_t@@II@Z 00000001800d8874     hb-ot-shaper-myanmar.obj
 0002:0002d874       $unwind$??1hb_ot_map_t@@QEAA@XZ 00000001800d8874     hb-shape-plan.obj
 0002:0002d88c       $unwind$?sanitize@maxp@OT@@QEBA_NPEAUhb_sanitize_context_t@@@Z 00000001800d888c     hb-common.obj
 0002:0002d88c       $unwind$??$dispatch@U?$Variable@UAffine2x3@OT@@@OT@@$$V@hb_sanitize_context_t@@QEAA_NAEBU?$Variable@UAffine2x3@OT@@@OT@@@Z 00000001800d888c     hb-ot-color.obj
 0002:0002d8a4       $unwind$??0accelerator_t@?$hmtxvmtx@Uhmtx@OT@@Uhhea@2@UHVAR@2@@OT@@QEAA@PEAUhb_face_t@@@Z 00000001800d88a4     hb-common.obj
 0002:0002d8a4       $unwind$??0accelerator_t@?$hmtxvmtx@Uvmtx@OT@@Uvhea@2@UVVAR@2@@OT@@QEAA@PEAUhb_face_t@@@Z 00000001800d88a4     hb-common.obj
 0002:0002d8bc       $unwind$?get_glyph_var_data_bytes@?$gvar_GVAR@U?$IntType@G$01@OT@@$0GHHGGBHC@@OT@@IEBA?BU?$hb_array_t@$$CBD@@PEAUhb_blob_t@@II@Z 00000001800d88bc     hb-common.obj
 0002:0002d8c8       $chain$0$?get_glyph_var_data_bytes@?$gvar_GVAR@U?$IntType@G$01@OT@@$0GHHGGBHC@@OT@@IEBA?BU?$hb_array_t@$$CBD@@PEAUhb_blob_t@@II@Z 00000001800d88c8     hb-common.obj
 0002:0002d8dc       $chain$1$?get_glyph_var_data_bytes@?$gvar_GVAR@U?$IntType@G$01@OT@@$0GHHGGBHC@@OT@@IEBA?BU?$hb_array_t@$$CBD@@PEAUhb_blob_t@@II@Z 00000001800d88dc     hb-common.obj
 0002:0002d8ec       $unwind$??0accelerator_t@?$gvar_GVAR@U?$IntType@G$01@OT@@$0GHHGGBHC@@OT@@QEAA@PEAUhb_face_t@@@Z 00000001800d88ec     hb-common.obj
 0002:0002d908       $chain$0$??0accelerator_t@?$gvar_GVAR@U?$IntType@G$01@OT@@$0GHHGGBHC@@OT@@QEAA@PEAUhb_face_t@@@Z 00000001800d8908     hb-common.obj
 0002:0002d91c       $chain$1$??0accelerator_t@?$gvar_GVAR@U?$IntType@G$01@OT@@$0GHHGGBHC@@OT@@QEAA@PEAUhb_face_t@@@Z 00000001800d891c     hb-common.obj
 0002:0002d91c       $chain$3$??0accelerator_t@?$gvar_GVAR@U?$IntType@G$01@OT@@$0GHHGGBHC@@OT@@QEAA@PEAUhb_face_t@@@Z 00000001800d891c     hb-common.obj
 0002:0002d92c       $chain$2$??0accelerator_t@?$gvar_GVAR@U?$IntType@G$01@OT@@$0GHHGGBHC@@OT@@QEAA@PEAUhb_face_t@@@Z 00000001800d892c     hb-common.obj
 0002:0002d940       $unwind$?apply_deltas_to_points@accelerator_t@?$gvar_GVAR@U?$IntType@G$01@OT@@$0GHHGGBHC@@OT@@QEBA_NIU?$hb_array_t@$$CBH@@U?$hb_array_t@Ucontour_point_t@@@@AEAUhb_glyf_scratch_t@@_N@Z 00000001800d8940     hb-common.obj
 0002:0002d96c       $unwind$?trim_padding@SimpleGlyph@glyf_impl@OT@@QEBA?BU?$hb_array_t@$$CBD@@XZ 00000001800d896c     hb-common.obj
 0002:0002d984       $unwind$?get_contour_points@SimpleGlyph@glyf_impl@OT@@QEBA_NAEAUcontour_point_vector_t@@_N@Z 00000001800d8984     hb-common.obj
 0002:0002d9a0       $unwind$?get_transformation@CompositeGlyphRecord@glyf_impl@OT@@QEBA_NAEAY03MAEAUcontour_point_t@@@Z 00000001800d89a0     hb-common.obj
 0002:0002d9b4       $unwind$??$get_points@Uglyf_accelerator_t@OT@@@Glyph@glyf_impl@OT@@QEBA_NPEAUhb_font_t@@AEBUglyf_accelerator_t@2@AEAUcontour_point_vector_t@@AEAUhb_glyf_scratch_t@@PEAU5@PEAUhead_maxp_info_t@@PEAI_N77U?$hb_array_t@$$CBH@@I6@Z 00000001800d89b4     hb-common.obj
 0002:0002d9cc       $chain$1$??$get_points@Uglyf_accelerator_t@OT@@@Glyph@glyf_impl@OT@@QEBA_NPEAUhb_font_t@@AEBUglyf_accelerator_t@2@AEAUcontour_point_vector_t@@AEAUhb_glyf_scratch_t@@PEAU5@PEAUhead_maxp_info_t@@PEAI_N77U?$hb_array_t@$$CBH@@I6@Z 00000001800d89cc     hb-common.obj
 0002:0002d9e4       $chain$11$??$get_points@Uglyf_accelerator_t@OT@@@Glyph@glyf_impl@OT@@QEBA_NPEAUhb_font_t@@AEBUglyf_accelerator_t@2@AEAUcontour_point_vector_t@@AEAUhb_glyf_scratch_t@@PEAU5@PEAUhead_maxp_info_t@@PEAI_N77U?$hb_array_t@$$CBH@@I6@Z 00000001800d89e4     hb-common.obj
 0002:0002d9e4       $chain$2$??$get_points@Uglyf_accelerator_t@OT@@@Glyph@glyf_impl@OT@@QEBA_NPEAUhb_font_t@@AEBUglyf_accelerator_t@2@AEAUcontour_point_vector_t@@AEAUhb_glyf_scratch_t@@PEAU5@PEAUhead_maxp_info_t@@PEAI_N77U?$hb_array_t@$$CBH@@I6@Z 00000001800d89e4     hb-common.obj
 0002:0002d9e4       $chain$9$??$get_points@Uglyf_accelerator_t@OT@@@Glyph@glyf_impl@OT@@QEBA_NPEAUhb_font_t@@AEBUglyf_accelerator_t@2@AEAUcontour_point_vector_t@@AEAUhb_glyf_scratch_t@@PEAU5@PEAUhead_maxp_info_t@@PEAI_N77U?$hb_array_t@$$CBH@@I6@Z 00000001800d89e4     hb-common.obj
 0002:0002d9f4       $chain$3$??$get_points@Uglyf_accelerator_t@OT@@@Glyph@glyf_impl@OT@@QEBA_NPEAUhb_font_t@@AEBUglyf_accelerator_t@2@AEAUcontour_point_vector_t@@AEAUhb_glyf_scratch_t@@PEAU5@PEAUhead_maxp_info_t@@PEAI_N77U?$hb_array_t@$$CBH@@I6@Z 00000001800d89f4     hb-common.obj
 0002:0002da0c       $chain$8$??$get_points@Uglyf_accelerator_t@OT@@@Glyph@glyf_impl@OT@@QEBA_NPEAUhb_font_t@@AEBUglyf_accelerator_t@2@AEAUcontour_point_vector_t@@AEAUhb_glyf_scratch_t@@PEAU5@PEAUhead_maxp_info_t@@PEAI_N77U?$hb_array_t@$$CBH@@I6@Z 00000001800d8a0c     hb-common.obj
 0002:0002da30       $chain$10$??$get_points@Uglyf_accelerator_t@OT@@@Glyph@glyf_impl@OT@@QEBA_NPEAUhb_font_t@@AEBUglyf_accelerator_t@2@AEAUcontour_point_vector_t@@AEAUhb_glyf_scratch_t@@PEAU5@PEAUhead_maxp_info_t@@PEAI_N77U?$hb_array_t@$$CBH@@I6@Z 00000001800d8a30     hb-common.obj
 0002:0002da5c       $unwind$??0glyf_accelerator_t@OT@@QEAA@PEAUhb_face_t@@@Z 00000001800d8a5c     hb-common.obj
 0002:0002da6c       $chain$1$??0glyf_accelerator_t@OT@@QEAA@PEAUhb_face_t@@@Z 00000001800d8a6c     hb-common.obj
 0002:0002da84       $chain$2$??0glyf_accelerator_t@OT@@QEAA@PEAUhb_face_t@@@Z 00000001800d8a84     hb-common.obj
 0002:0002da94       $unwind$?get_advance_with_var_unscaled@glyf_accelerator_t@OT@@QEBAIPEAUhb_font_t@@I_N@Z 00000001800d8a94     hb-common.obj
 0002:0002daac       $chain$1$?get_advance_with_var_unscaled@glyf_accelerator_t@OT@@QEBAIPEAUhb_font_t@@I_N@Z 00000001800d8aac     hb-common.obj
 0002:0002dac4       $chain$3$?get_advance_with_var_unscaled@glyf_accelerator_t@OT@@QEBAIPEAUhb_font_t@@I_N@Z 00000001800d8ac4     hb-common.obj
 0002:0002dad8       $chain$2$?get_advance_with_var_unscaled@glyf_accelerator_t@OT@@QEBAIPEAUhb_font_t@@I_N@Z 00000001800d8ad8     hb-common.obj
 0002:0002dae8       $unwind$?get_leading_bearing_with_var_unscaled@glyf_accelerator_t@OT@@QEBA_NPEAUhb_font_t@@I_NPEAH@Z 00000001800d8ae8     hb-common.obj
 0002:0002db00       $chain$0$?get_leading_bearing_with_var_unscaled@glyf_accelerator_t@OT@@QEBA_NPEAUhb_font_t@@I_NPEAH@Z 00000001800d8b00     hb-common.obj
 0002:0002db14       $chain$1$?get_leading_bearing_with_var_unscaled@glyf_accelerator_t@OT@@QEBA_NPEAUhb_font_t@@I_NPEAH@Z 00000001800d8b14     hb-common.obj
 0002:0002db24       $unwind$?glyph_for_gid@glyf_accelerator_t@OT@@QEBA?BUGlyph@glyf_impl@2@I_N@Z 00000001800d8b24     hb-common.obj
 0002:0002db38       $chain$1$?glyph_for_gid@glyf_accelerator_t@OT@@QEBA?BUGlyph@glyf_impl@2@I_N@Z 00000001800d8b38     hb-common.obj
 0002:0002db50       $chain$2$?glyph_for_gid@glyf_accelerator_t@OT@@QEBA?BUGlyph@glyf_impl@2@I_N@Z 00000001800d8b50     hb-common.obj
 0002:0002db60       $unwind$??$get_points@Upoints_aggregator_t@glyf_accelerator_t@OT@@@glyf_accelerator_t@OT@@IEBA_NPEAUhb_font_t@@IUpoints_aggregator_t@01@U?$hb_array_t@$$CBH@@AEAUhb_glyf_scratch_t@@@Z 00000001800d8b60     hb-common.obj
 0002:0002db80       $chain$1$??$get_points@Upoints_aggregator_t@glyf_accelerator_t@OT@@@glyf_accelerator_t@OT@@IEBA_NPEAUhb_font_t@@IUpoints_aggregator_t@01@U?$hb_array_t@$$CBH@@AEAUhb_glyf_scratch_t@@@Z 00000001800d8b80     hb-common.obj
 0002:0002db98       $chain$2$??$get_points@Upoints_aggregator_t@glyf_accelerator_t@OT@@@glyf_accelerator_t@OT@@IEBA_NPEAUhb_font_t@@IUpoints_aggregator_t@01@U?$hb_array_t@$$CBH@@AEAUhb_glyf_scratch_t@@@Z 00000001800d8b98     hb-common.obj
 0002:0002dba8       $unwind$??$sanitize_blob@Uhead@OT@@@hb_sanitize_context_t@@QEAAPEAUhb_blob_t@@PEAU1@@Z 00000001800d8ba8     hb-common.obj
 0002:0002dba8       $unwind$??$sanitize_blob@Uhhea@OT@@@hb_sanitize_context_t@@QEAAPEAUhb_blob_t@@PEAU1@@Z 00000001800d8ba8     hb-common.obj
 0002:0002dba8       $unwind$??$sanitize_blob@Uvhea@OT@@@hb_sanitize_context_t@@QEAAPEAUhb_blob_t@@PEAU1@@Z 00000001800d8ba8     hb-common.obj
 0002:0002dba8       $unwind$??$sanitize_blob@UCBDT@OT@@@hb_sanitize_context_t@@QEAAPEAUhb_blob_t@@PEAU1@@Z 00000001800d8ba8     hb-ot-color.obj
 0002:0002dbc4       $unwind$??$sanitize_blob@UVVAR@OT@@@hb_sanitize_context_t@@QEAAPEAUhb_blob_t@@PEAU1@@Z 00000001800d8bc4     hb-common.obj
 0002:0002dbe0       $unwind$??$decompile@H@TupleValues@OT@@SA_NAEAPEBU?$IntType@E$00@1@AEAU?$hb_vector_t@H$0A@@@PEBU21@_N@Z 00000001800d8be0     hb-common.obj
 0002:0002dbfc       $unwind$??$sanitize_blob@Umaxp@OT@@@hb_sanitize_context_t@@QEAAPEAUhb_blob_t@@PEAU1@@Z 00000001800d8bfc     hb-common.obj
 0002:0002dbfc       $unwind$??$sanitize_blob@UVORG@OT@@@hb_sanitize_context_t@@QEAAPEAUhb_blob_t@@PEAU1@@Z 00000001800d8bfc     hb-ot-font.obj
 0002:0002dbfc       $unwind$??$sanitize_blob@Upost@OT@@@hb_sanitize_context_t@@QEAAPEAUhb_blob_t@@PEAU1@@Z 00000001800d8bfc     hb-ot-font.obj
 0002:0002dbfc       $unwind$??$sanitize_blob@Ukern@OT@@@hb_sanitize_context_t@@QEAAPEAUhb_blob_t@@PEAU1@@Z 00000001800d8bfc     hb-ot-layout.obj
 0002:0002dc18       $chain$0$hb_draw_funcs_set_move_to_func 00000001800d8c18     hb-draw.obj
 0002:0002dc2c       $chain$1$hb_draw_funcs_set_move_to_func 00000001800d8c2c     hb-draw.obj
 0002:0002dc3c       $chain$0$hb_draw_funcs_set_line_to_func 00000001800d8c3c     hb-draw.obj
 0002:0002dc50       $chain$1$hb_draw_funcs_set_line_to_func 00000001800d8c50     hb-draw.obj
 0002:0002dc60       $chain$0$hb_draw_funcs_set_quadratic_to_func 00000001800d8c60     hb-draw.obj
 0002:0002dc74       $chain$1$hb_draw_funcs_set_quadratic_to_func 00000001800d8c74     hb-draw.obj
 0002:0002dc84       $chain$0$hb_draw_funcs_set_cubic_to_func 00000001800d8c84     hb-draw.obj
 0002:0002dc98       $chain$1$hb_draw_funcs_set_cubic_to_func 00000001800d8c98     hb-draw.obj
 0002:0002dca8       $chain$0$hb_draw_funcs_set_close_path_func 00000001800d8ca8     hb-draw.obj
 0002:0002dcbc       $chain$1$hb_draw_funcs_set_close_path_func 00000001800d8cbc     hb-draw.obj
 0002:0002dccc       $chain$1$hb_draw_funcs_destroy 00000001800d8ccc     hb-draw.obj
 0002:0002dce4       $chain$2$hb_draw_funcs_destroy 00000001800d8ce4     hb-draw.obj
 0002:0002dcf8       $chain$3$hb_draw_funcs_destroy 00000001800d8cf8     hb-draw.obj
 0002:0002dd08       $chain$0$?hb_draw_extents_get_funcs@@YAPEAUhb_draw_funcs_t@@XZ 00000001800d8d08     hb-draw.obj
 0002:0002dd1c       $chain$2$?hb_draw_extents_get_funcs@@YAPEAUhb_draw_funcs_t@@XZ 00000001800d8d1c     hb-draw.obj
 0002:0002dd30       $chain$3$?hb_draw_extents_get_funcs@@YAPEAUhb_draw_funcs_t@@XZ 00000001800d8d30     hb-draw.obj
 0002:0002dd40       $unwind$?hb_draw_quadratic_to_nil@@YAXPEAUhb_draw_funcs_t@@PEAXPEAUhb_draw_state_t@@MMMM1@Z 00000001800d8d40     hb-draw.obj
 0002:0002dd4c       $chain$2$?create@hb_draw_extents_funcs_lazy_loader_t@@SAPEAUhb_draw_funcs_t@@XZ 00000001800d8d4c     hb-draw.obj
 0002:0002dd68       $chain$3$?create@hb_draw_extents_funcs_lazy_loader_t@@SAPEAUhb_draw_funcs_t@@XZ 00000001800d8d68     hb-draw.obj
 0002:0002dd78       $unwind$??0hb_serialize_context_t@@QEAA@PEAXI@Z 00000001800d8d78     hb-face-builder.obj
 0002:0002dd84       $chain$2$??0hb_serialize_context_t@@QEAA@PEAXI@Z 00000001800d8d84     hb-face-builder.obj
 0002:0002dda0       $chain$3$??0hb_serialize_context_t@@QEAA@PEAXI@Z 00000001800d8da0     hb-face-builder.obj
 0002:0002ddb4       $chain$4$??0hb_serialize_context_t@@QEAA@PEAXI@Z 00000001800d8db4     hb-face-builder.obj
 0002:0002ddc4       $unwind$?fini@hb_serialize_context_t@@QEAAXXZ 00000001800d8dc4     hb-face-builder.obj
 0002:0002ddd4       $chain$0$?fini@hb_serialize_context_t@@QEAAXXZ 00000001800d8dd4     hb-face-builder.obj
 0002:0002dde8       $chain$1$?fini@hb_serialize_context_t@@QEAAXXZ 00000001800d8de8     hb-face-builder.obj
 0002:0002ddfc       $chain$2$?fini@hb_serialize_context_t@@QEAAXXZ 00000001800d8dfc     hb-face-builder.obj
 0002:0002de0c       $chain$3$?fini@hb_serialize_context_t@@QEAAXXZ 00000001800d8e0c     hb-face-builder.obj
 0002:0002de1c       $unwind$?pop_pack@hb_serialize_context_t@@QEAAI_N@Z 00000001800d8e1c     hb-face-builder.obj
 0002:0002de30       $chain$1$?pop_pack@hb_serialize_context_t@@QEAAI_N@Z 00000001800d8e30     hb-face-builder.obj
 0002:0002de48       $chain$3$?pop_pack@hb_serialize_context_t@@QEAAI_N@Z 00000001800d8e48     hb-face-builder.obj
 0002:0002de60       $chain$4$?pop_pack@hb_serialize_context_t@@QEAAI_N@Z 00000001800d8e60     hb-face-builder.obj
 0002:0002de70       $chain$1$?resolve_links@hb_serialize_context_t@@QEAAXXZ 00000001800d8e70     hb-face-builder.obj
 0002:0002de88       $chain$5$?resolve_links@hb_serialize_context_t@@QEAAXXZ 00000001800d8e88     hb-face-builder.obj
 0002:0002dea8       $chain$6$?resolve_links@hb_serialize_context_t@@QEAAXXZ 00000001800d8ea8     hb-face-builder.obj
 0002:0002deb8       $chain$7$?resolve_links@hb_serialize_context_t@@QEAAXXZ 00000001800d8eb8     hb-face-builder.obj
 0002:0002dec8       $unwind$??1?$hb_pool_t@Uobject_t@hb_serialize_context_t@@$0CA@@@QEAA@XZ 00000001800d8ec8     hb-face-builder.obj
 0002:0002dedc       $unwind$?alloc@?$hb_hashmap_t@PEBUobject_t@hb_serialize_context_t@@I$0A@@@QEAA_NI@Z 00000001800d8edc     hb-face-builder.obj
 0002:0002def0       $chain$0$?alloc@?$hb_hashmap_t@PEBUobject_t@hb_serialize_context_t@@I$0A@@@QEAA_NI@Z 00000001800d8ef0     hb-face-builder.obj
 0002:0002df04       $chain$3$?alloc@?$hb_hashmap_t@PEBUobject_t@hb_serialize_context_t@@I$0A@@@QEAA_NI@Z 00000001800d8f04     hb-face-builder.obj
 0002:0002df20       $chain$5$?alloc@?$hb_hashmap_t@PEBUobject_t@hb_serialize_context_t@@I$0A@@@QEAA_NI@Z 00000001800d8f20     hb-face-builder.obj
 0002:0002df38       $chain$6$?alloc@?$hb_hashmap_t@PEBUobject_t@hb_serialize_context_t@@I$0A@@@QEAA_NI@Z 00000001800d8f38     hb-face-builder.obj
 0002:0002df48       $chain$7$?alloc@?$hb_hashmap_t@PEBUobject_t@hb_serialize_context_t@@I$0A@@@QEAA_NI@Z 00000001800d8f48     hb-face-builder.obj
 0002:0002df58       $chain$8$?alloc@?$hb_hashmap_t@PEBUobject_t@hb_serialize_context_t@@I$0A@@@QEAA_NI@Z 00000001800d8f58     hb-face-builder.obj
 0002:0002df68       $unwind$?fetch_item@?$hb_hashmap_t@PEBUobject_t@hb_serialize_context_t@@I$0A@@@QEBAPEAUitem_t@1@AEBQEBUobject_t@hb_serialize_context_t@@I@Z 00000001800d8f68     hb-face-builder.obj
 0002:0002df80       $unwind$??$set_with_hash@AEAPEAUobject_t@hb_serialize_context_t@@AEAI@?$hb_hashmap_t@PEBUobject_t@hb_serialize_context_t@@I$0A@@@QEAA_NAEAPEAUobject_t@hb_serialize_context_t@@IAEAI_N@Z 00000001800d8f80     hb-face-builder.obj
 0002:0002df98       $unwind$hb_face_create     00000001800d8f98     hb-face.obj
 0002:0002dfb0       $chain$0$hb_face_create    00000001800d8fb0     hb-face.obj
 0002:0002dfc4       $chain$1$hb_face_create    00000001800d8fc4     hb-face.obj
 0002:0002dfd4       $unwind$hb_face_create_from_file_or_fail 00000001800d8fd4     hb-face.obj
 0002:0002dfec       $unwind$hb_face_destroy    00000001800d8fec     hb-face.obj
 0002:0002dfec       $unwind$hb_shape_plan_destroy 00000001800d8fec     hb-shape-plan.obj
 0002:0002dff4       $chain$1$hb_face_destroy   00000001800d8ff4     hb-face.obj
 0002:0002e00c       $chain$2$hb_face_destroy   00000001800d900c     hb-face.obj
 0002:0002e01c       $unwind$?compact@hb_bit_set_t@@AEAAXAEAU?$hb_vector_t@I$0A@@@I@Z 00000001800d901c     hb-face.obj
 0002:0002e01c       $unwind$?paint_glyph@PaintSolid@OT@@QEBAXPEAUhb_paint_context_t@2@I@Z 00000001800d901c     hb-ot-font.obj
 0002:0002e028       $chain$0$?compact@hb_bit_set_t@@AEAAXAEAU?$hb_vector_t@I$0A@@@I@Z 00000001800d9028     hb-face.obj
 0002:0002e03c       $chain$1$?compact@hb_bit_set_t@@AEAAXAEAU?$hb_vector_t@I$0A@@@I@Z 00000001800d903c     hb-face.obj
 0002:0002e04c       $unwind$?alloc@?$hb_hashmap_t@II$00@@QEAA_NI@Z 00000001800d904c     hb-face.obj
 0002:0002e060       $chain$0$?alloc@?$hb_hashmap_t@II$00@@QEAA_NI@Z 00000001800d9060     hb-face.obj
 0002:0002e074       $chain$3$?alloc@?$hb_hashmap_t@II$00@@QEAA_NI@Z 00000001800d9074     hb-face.obj
 0002:0002e090       $chain$4$?alloc@?$hb_hashmap_t@II$00@@QEAA_NI@Z 00000001800d9090     hb-face.obj
 0002:0002e0a4       $chain$5$?alloc@?$hb_hashmap_t@II$00@@QEAA_NI@Z 00000001800d90a4     hb-face.obj
 0002:0002e0b8       $chain$6$?alloc@?$hb_hashmap_t@II$00@@QEAA_NI@Z 00000001800d90b8     hb-face.obj
 0002:0002e0c8       $chain$7$?alloc@?$hb_hashmap_t@II$00@@QEAA_NI@Z 00000001800d90c8     hb-face.obj
 0002:0002e0d8       $chain$8$?alloc@?$hb_hashmap_t@II$00@@QEAA_NI@Z 00000001800d90d8     hb-face.obj
 0002:0002e0e8       $chain$9$?alloc@?$hb_hashmap_t@II$00@@QEAA_NI@Z 00000001800d90e8     hb-face.obj
 0002:0002e0f8       $unwind$?find_table_index@OpenTypeOffsetTable@OT@@QEBA_NIPEAI@Z 00000001800d90f8     hb-face.obj
 0002:0002e104       $chain$0$?find_table_index@OpenTypeOffsetTable@OT@@QEBA_NIPEAI@Z 00000001800d9104     hb-face.obj
 0002:0002e118       $chain$2$?find_table_index@OpenTypeOffsetTable@OT@@QEBA_NIPEAI@Z 00000001800d9118     hb-face.obj
 0002:0002e12c       $unwind$?get_face@ResourceForkHeader@OT@@QEBAAEBUOpenTypeOffsetTable@2@IPEAI@Z 00000001800d912c     hb-face.obj
 0002:0002e144       $unwind$?sanitize@ResourceForkHeader@OT@@QEBA_NPEAUhb_sanitize_context_t@@@Z 00000001800d9144     hb-face.obj
 0002:0002e144       $unwind$?sanitize@STAT@OT@@QEBA_NPEAUhb_sanitize_context_t@@@Z 00000001800d9144     hb-ot-shape.obj
 0002:0002e154       $chain$1$?get_face_count@OpenTypeFontFile@OT@@QEBAIXZ 00000001800d9154     hb-face.obj
 0002:0002e16c       $chain$3$?get_face_count@OpenTypeFontFile@OT@@QEBAIXZ 00000001800d916c     hb-face.obj
 0002:0002e184       $chain$4$?get_face_count@OpenTypeFontFile@OT@@QEBAIXZ 00000001800d9184     hb-face.obj
 0002:0002e198       $chain$5$?get_face_count@OpenTypeFontFile@OT@@QEBAIXZ 00000001800d9198     hb-face.obj
 0002:0002e1a8       $chain$0$?sanitize@OpenTypeFontFile@OT@@QEBA_NPEAUhb_sanitize_context_t@@@Z 00000001800d91a8     hb-face.obj
 0002:0002e1bc       $chain$1$?sanitize@OpenTypeFontFile@OT@@QEBA_NPEAUhb_sanitize_context_t@@@Z 00000001800d91bc     hb-face.obj
 0002:0002e1cc       $unwind$?get_glyph@accelerator_t@CmapSubtableFormat4@OT@@QEBA_NIPEAI@Z 00000001800d91cc     hb-face.obj
 0002:0002e1e4       $unwind$?sanitize@CmapSubtableFormat4@OT@@QEBA_NPEAUhb_sanitize_context_t@@@Z 00000001800d91e4     hb-face.obj
 0002:0002e1f8       $unwind$?get_glyph@?$CmapSubtableLongSegmented@UCmapSubtableFormat12@OT@@@OT@@QEBA_NIPEAI@Z 00000001800d91f8     hb-face.obj
 0002:0002e200       $unwind$?get_glyph@CmapSubtable@OT@@QEBA_NIPEAI@Z 00000001800d9200     hb-face.obj
 0002:0002e200       $unwind$?hb_font_draw_glyph_or_fail_default@@YAHPEAUhb_font_t@@PEAXIPEAUhb_draw_funcs_t@@11@Z 00000001800d9200     hb-font.obj
 0002:0002e200       $unwind$??RItemVarStoreInstancer@OT@@QEBAMIG@Z 00000001800d9200     hb-ot-font.obj
 0002:0002e200       $unwind$??$start_serialize@USubstLookup@GSUB_impl@Layout@OT@@@hb_serialize_context_t@@QEAAPEAUSubstLookup@GSUB_impl@Layout@OT@@XZ 00000001800d9200     hb-ot-shaper-arabic.obj
 0002:0002e208       $unwind$??0accelerator_t@cmap@OT@@QEAA@PEAUhb_face_t@@@Z 00000001800d9208     hb-face.obj
 0002:0002e228       $unwind$?find_subtable@cmap@OT@@IEBAPEBUCmapSubtable@2@II@Z 00000001800d9228     hb-face.obj
 0002:0002e230       $chain$6$?find_subtable@cmap@OT@@IEBAPEBUCmapSubtable@2@II@Z 00000001800d9230     hb-face.obj
 0002:0002e25c       $chain$7$?find_subtable@cmap@OT@@IEBAPEBUCmapSubtable@2@II@Z 00000001800d925c     hb-face.obj
 0002:0002e26c       $unwind$?_hb_face_for_data_reference_table@@YAPEAUhb_blob_t@@PEAUhb_face_t@@IPEAX@Z 00000001800d926c     hb-face.obj
 0002:0002e27c       $unwind$?_hb_face_for_data_get_table_tags@@YAIPEBUhb_face_t@@IPEAI1PEAX@Z 00000001800d927c     hb-face.obj
 0002:0002e298       $unwind$??$set_with_hash@AEBIAEAI@?$hb_hashmap_t@II$00@@QEAA_NAEBIIAEAI_N@Z 00000001800d9298     hb-face.obj
 0002:0002e2b0       $unwind$??$dispatch@U?$UnsizedArrayOf@UResourceRecord@OT@@@OT@@IAEAPEBX@hb_sanitize_context_t@@QEAA_NAEBU?$UnsizedArrayOf@UResourceRecord@OT@@@OT@@$$QEAIAEAPEBX@Z 00000001800d92b0     hb-face.obj
 0002:0002e2c0       $chain$3$??$dispatch@U?$UnsizedArrayOf@UResourceRecord@OT@@@OT@@IAEAPEBX@hb_sanitize_context_t@@QEAA_NAEBU?$UnsizedArrayOf@UResourceRecord@OT@@@OT@@$$QEAIAEAPEBX@Z 00000001800d92c0     hb-face.obj
 0002:0002e2e0       $chain$5$??$dispatch@U?$UnsizedArrayOf@UResourceRecord@OT@@@OT@@IAEAPEBX@hb_sanitize_context_t@@QEAA_NAEBU?$UnsizedArrayOf@UResourceRecord@OT@@@OT@@$$QEAIAEAPEBX@Z 00000001800d92e0     hb-face.obj
 0002:0002e300       $unwind$??$dispatch@U?$ArrayOfM1@UResourceTypeRecord@OT@@U?$IntType@G$01@2@@OT@@PEBU12@AEAPEBX@hb_sanitize_context_t@@QEAA_NAEBU?$ArrayOfM1@UResourceTypeRecord@OT@@U?$IntType@G$01@2@@OT@@$$QEAPEBU12@AEAPEBX@Z 00000001800d9300     hb-face.obj
 0002:0002e320       $unwind$??$dispatch@UResourceMap@OT@@PEBU?$UnsizedArrayOf@U?$IntType@E$00@OT@@@2@@hb_sanitize_context_t@@QEAA_NAEBUResourceMap@OT@@$$QEAPEBU?$UnsizedArrayOf@U?$IntType@E$00@OT@@@2@@Z 00000001800d9320     hb-face.obj
 0002:0002e330       $unwind$_hb_fallback_shape 00000001800d9330     hb-fallback-shape.obj
 0002:0002e33c       $chain$1$_hb_fallback_shape 00000001800d933c     hb-fallback-shape.obj
 0002:0002e354       $chain$4$_hb_fallback_shape 00000001800d9354     hb-fallback-shape.obj
 0002:0002e370       $chain$5$_hb_fallback_shape 00000001800d9370     hb-fallback-shape.obj
 0002:0002e380       $chain$6$_hb_fallback_shape 00000001800d9380     hb-fallback-shape.obj
 0002:0002e390       $chain$1$hb_font_funcs_destroy 00000001800d9390     hb-font.obj
 0002:0002e3a8       $chain$2$hb_font_funcs_destroy 00000001800d93a8     hb-font.obj
 0002:0002e3bc       $chain$3$hb_font_funcs_destroy 00000001800d93bc     hb-font.obj
 0002:0002e3cc       $chain$0$hb_font_funcs_set_font_h_extents_func 00000001800d93cc     hb-font.obj
 0002:0002e3e0       $chain$1$hb_font_funcs_set_font_h_extents_func 00000001800d93e0     hb-font.obj
 0002:0002e3f0       $chain$0$hb_font_funcs_set_font_v_extents_func 00000001800d93f0     hb-font.obj
 0002:0002e404       $chain$1$hb_font_funcs_set_font_v_extents_func 00000001800d9404     hb-font.obj
 0002:0002e414       $chain$0$hb_font_funcs_set_nominal_glyph_func 00000001800d9414     hb-font.obj
 0002:0002e428       $chain$1$hb_font_funcs_set_nominal_glyph_func 00000001800d9428     hb-font.obj
 0002:0002e438       $chain$0$hb_font_funcs_set_nominal_glyphs_func 00000001800d9438     hb-font.obj
 0002:0002e44c       $chain$1$hb_font_funcs_set_nominal_glyphs_func 00000001800d944c     hb-font.obj
 0002:0002e45c       $chain$0$hb_font_funcs_set_variation_glyph_func 00000001800d945c     hb-font.obj
 0002:0002e470       $chain$1$hb_font_funcs_set_variation_glyph_func 00000001800d9470     hb-font.obj
 0002:0002e480       $chain$0$hb_font_funcs_set_glyph_h_advance_func 00000001800d9480     hb-font.obj
 0002:0002e494       $chain$1$hb_font_funcs_set_glyph_h_advance_func 00000001800d9494     hb-font.obj
 0002:0002e4a4       $chain$0$hb_font_funcs_set_glyph_v_advance_func 00000001800d94a4     hb-font.obj
 0002:0002e4b8       $chain$1$hb_font_funcs_set_glyph_v_advance_func 00000001800d94b8     hb-font.obj
 0002:0002e4c8       $chain$0$hb_font_funcs_set_glyph_h_advances_func 00000001800d94c8     hb-font.obj
 0002:0002e4dc       $chain$1$hb_font_funcs_set_glyph_h_advances_func 00000001800d94dc     hb-font.obj
 0002:0002e4ec       $chain$0$hb_font_funcs_set_glyph_v_advances_func 00000001800d94ec     hb-font.obj
 0002:0002e500       $chain$1$hb_font_funcs_set_glyph_v_advances_func 00000001800d9500     hb-font.obj
 0002:0002e510       $chain$0$hb_font_funcs_set_glyph_h_origin_func 00000001800d9510     hb-font.obj
 0002:0002e524       $chain$1$hb_font_funcs_set_glyph_h_origin_func 00000001800d9524     hb-font.obj
 0002:0002e534       $chain$0$hb_font_funcs_set_glyph_v_origin_func 00000001800d9534     hb-font.obj
 0002:0002e548       $chain$1$hb_font_funcs_set_glyph_v_origin_func 00000001800d9548     hb-font.obj
 0002:0002e558       $chain$0$hb_font_funcs_set_glyph_h_kerning_func 00000001800d9558     hb-font.obj
 0002:0002e56c       $chain$1$hb_font_funcs_set_glyph_h_kerning_func 00000001800d956c     hb-font.obj
 0002:0002e57c       $chain$0$hb_font_funcs_set_glyph_extents_func 00000001800d957c     hb-font.obj
 0002:0002e590       $chain$1$hb_font_funcs_set_glyph_extents_func 00000001800d9590     hb-font.obj
 0002:0002e5a0       $chain$0$hb_font_funcs_set_glyph_contour_point_func 00000001800d95a0     hb-font.obj
 0002:0002e5b4       $chain$1$hb_font_funcs_set_glyph_contour_point_func 00000001800d95b4     hb-font.obj
 0002:0002e5c4       $chain$0$hb_font_funcs_set_glyph_name_func 00000001800d95c4     hb-font.obj
 0002:0002e5d8       $chain$1$hb_font_funcs_set_glyph_name_func 00000001800d95d8     hb-font.obj
 0002:0002e5e8       $chain$0$hb_font_funcs_set_glyph_from_name_func 00000001800d95e8     hb-font.obj
 0002:0002e5fc       $chain$1$hb_font_funcs_set_glyph_from_name_func 00000001800d95fc     hb-font.obj
 0002:0002e60c       $chain$0$hb_font_funcs_set_draw_glyph_or_fail_func 00000001800d960c     hb-font.obj
 0002:0002e620       $chain$1$hb_font_funcs_set_draw_glyph_or_fail_func 00000001800d9620     hb-font.obj
 0002:0002e630       $chain$0$hb_font_funcs_set_paint_glyph_or_fail_func 00000001800d9630     hb-font.obj
 0002:0002e644       $chain$1$hb_font_funcs_set_paint_glyph_or_fail_func 00000001800d9644     hb-font.obj
 0002:0002e654       $unwind$hb_font_create     00000001800d9654     hb-font.obj
 0002:0002e670       $unwind$hb_font_create_sub_font 00000001800d9670     hb-font.obj
 0002:0002e67c       $chain$0$hb_font_create_sub_font 00000001800d967c     hb-font.obj
 0002:0002e690       $chain$3$hb_font_create_sub_font 00000001800d9690     hb-font.obj
 0002:0002e6ac       $chain$4$hb_font_create_sub_font 00000001800d96ac     hb-font.obj
 0002:0002e6bc       $chain$5$hb_font_create_sub_font 00000001800d96bc     hb-font.obj
 0002:0002e6cc       $chain$0$hb_font_destroy   00000001800d96cc     hb-font.obj
 0002:0002e6e0       $chain$1$hb_font_destroy   00000001800d96e0     hb-font.obj
 0002:0002e6f0       $unwind$hb_font_set_funcs  00000001800d96f0     hb-font.obj
 0002:0002e700       $chain$1$hb_font_set_funcs 00000001800d9700     hb-font.obj
 0002:0002e718       $chain$2$hb_font_set_funcs 00000001800d9718     hb-font.obj
 0002:0002e728       $unwind$hb_font_set_variations 00000001800d9728     hb-font.obj
 0002:0002e734       $chain$4$hb_font_set_variations 00000001800d9734     hb-font.obj
 0002:0002e758       $chain$5$hb_font_set_variations 00000001800d9758     hb-font.obj
 0002:0002e768       $unwind$hb_font_set_var_coords_normalized 00000001800d9768     hb-font.obj
 0002:0002e778       $chain$4$hb_font_set_var_coords_normalized 00000001800d9778     hb-font.obj
 0002:0002e79c       $chain$7$hb_font_set_var_coords_normalized 00000001800d979c     hb-font.obj
 0002:0002e7b8       $chain$8$hb_font_set_var_coords_normalized 00000001800d97b8     hb-font.obj
 0002:0002e7c8       $chain$9$hb_font_set_var_coords_normalized 00000001800d97c8     hb-font.obj
 0002:0002e7d8       $chain$0$hb_font_funcs_set_glyph_v_kerning_func 00000001800d97d8     hb-font.obj
 0002:0002e7ec       $chain$1$hb_font_funcs_set_glyph_v_kerning_func 00000001800d97ec     hb-font.obj
 0002:0002e7fc       $chain$1$?get@?$hb_lazy_loader_t@Ufvar@OT@@U?$hb_table_lazy_loader_t@Ufvar@OT@@$0BC@$00@@Uhb_face_t@@$0BC@Uhb_blob_t@@@@QEBAPEBUfvar@OT@@XZ 00000001800d97fc     hb-font.obj
 0002:0002e814       $chain$2$?get@?$hb_lazy_loader_t@Ufvar@OT@@U?$hb_table_lazy_loader_t@Ufvar@OT@@$0BC@$00@@Uhb_face_t@@$0BC@Uhb_blob_t@@@@QEBAPEBUfvar@OT@@XZ 00000001800d9814     hb-font.obj
 0002:0002e824       $chain$0$?alloc@?$hb_vector_t@Uhb_transform_t@@$0A@@@QEAA_NI_N@Z 00000001800d9824     hb-font.obj
 0002:0002e838       $chain$2$?alloc@?$hb_vector_t@Uhb_transform_t@@$0A@@@QEAA_NI_N@Z 00000001800d9838     hb-font.obj
 0002:0002e838       $chain$4$?alloc@?$hb_vector_t@Uhb_transform_t@@$0A@@@QEAA_NI_N@Z 00000001800d9838     hb-font.obj
 0002:0002e84c       $chain$0$?alloc@?$hb_vector_t@Uhb_bounds_t@@$0A@@@QEAA_NI_N@Z 00000001800d984c     hb-font.obj
 0002:0002e860       $chain$2$?alloc@?$hb_vector_t@Uhb_bounds_t@@$0A@@@QEAA_NI_N@Z 00000001800d9860     hb-font.obj
 0002:0002e860       $chain$4$?alloc@?$hb_vector_t@Uhb_bounds_t@@$0A@@@QEAA_NI_N@Z 00000001800d9860     hb-font.obj
 0002:0002e874       $unwind$?get_glyph_extents@hb_font_t@@QEAAHIPEAUhb_glyph_extents_t@@_N@Z 00000001800d9874     hb-font.obj
 0002:0002e88c       $chain$0$?get_glyph_extents@hb_font_t@@QEAAHIPEAUhb_glyph_extents_t@@_N@Z 00000001800d988c     hb-font.obj
 0002:0002e8a0       $chain$3$?get_glyph_extents@hb_font_t@@QEAAHIPEAUhb_glyph_extents_t@@_N@Z 00000001800d98a0     hb-font.obj
 0002:0002e8bc       $chain$4$?get_glyph_extents@hb_font_t@@QEAAHIPEAUhb_glyph_extents_t@@_N@Z 00000001800d98bc     hb-font.obj
 0002:0002e8cc       $chain$5$?get_glyph_extents@hb_font_t@@QEAAHIPEAUhb_glyph_extents_t@@_N@Z 00000001800d98cc     hb-font.obj
 0002:0002e8dc       $unwind$?draw_glyph_or_fail@hb_font_t@@QEAA_NIPEAUhb_draw_funcs_t@@PEAX_N@Z 00000001800d98dc     hb-font.obj
 0002:0002e8f8       $chain$3$?draw_glyph_or_fail@hb_font_t@@QEAA_NIPEAUhb_draw_funcs_t@@PEAX_N@Z 00000001800d98f8     hb-font.obj
 0002:0002e910       $chain$4$?draw_glyph_or_fail@hb_font_t@@QEAA_NIPEAUhb_draw_funcs_t@@PEAX_N@Z 00000001800d9910     hb-font.obj
 0002:0002e920       $unwind$?paint_glyph_or_fail@hb_font_t@@QEAA_NIPEAUhb_paint_funcs_t@@PEAXII_N@Z 00000001800d9920     hb-font.obj
 0002:0002e938       $unwind$?changed@hb_font_t@@QEAAXXZ 00000001800d9938     hb-font.obj
 0002:0002e94c       $unwind$?map@SegmentMaps@OT@@QEBAHHII@Z 00000001800d994c     hb-font.obj
 0002:0002e958       $chain$0$?map@SegmentMaps@OT@@QEBAHHII@Z 00000001800d9958     hb-font.obj
 0002:0002e96c       $chain$5$?map@SegmentMaps@OT@@QEBAHHII@Z 00000001800d996c     hb-font.obj
 0002:0002e98c       $unwind$?hb_font_get_nominal_glyph_default@@YAHPEAUhb_font_t@@PEAXIPEAI1@Z 00000001800d998c     hb-font.obj
 0002:0002e994       $unwind$?hb_font_get_nominal_glyphs_default@@YAIPEAUhb_font_t@@PEAXIPEBIIPEAII1@Z 00000001800d9994     hb-font.obj
 0002:0002e9a4       $chain$3$?hb_font_get_nominal_glyphs_default@@YAIPEAUhb_font_t@@PEAXIPEBIIPEAII1@Z 00000001800d99a4     hb-font.obj
 0002:0002e9c4       $chain$5$?hb_font_get_nominal_glyphs_default@@YAIPEAUhb_font_t@@PEAXIPEBIIPEAII1@Z 00000001800d99c4     hb-font.obj
 0002:0002e9e4       $chain$6$?hb_font_get_nominal_glyphs_default@@YAIPEAUhb_font_t@@PEAXIPEBIIPEAII1@Z 00000001800d99e4     hb-font.obj
 0002:0002e9f4       $unwind$?hb_font_get_glyph_h_advance_default@@YAHPEAUhb_font_t@@PEAXI1@Z 00000001800d99f4     hb-font.obj
 0002:0002e9f4       $unwind$?hb_font_get_glyph_v_advance_default@@YAHPEAUhb_font_t@@PEAXI1@Z 00000001800d99f4     hb-font.obj
 0002:0002e9fc       $unwind$?hb_font_get_glyph_h_advances_default@@YAXPEAUhb_font_t@@PEAXIPEBIIPEAHI1@Z 00000001800d99fc     hb-font.obj
 0002:0002e9fc       $unwind$?hb_font_get_glyph_v_advances_default@@YAXPEAUhb_font_t@@PEAXIPEBIIPEAHI1@Z 00000001800d99fc     hb-font.obj
 0002:0002ea10       $chain$1$?hb_font_get_glyph_h_advances_default@@YAXPEAUhb_font_t@@PEAXIPEBIIPEAHI1@Z 00000001800d9a10     hb-font.obj
 0002:0002ea28       $chain$2$?hb_font_get_glyph_h_advances_default@@YAXPEAUhb_font_t@@PEAXIPEBIIPEAHI1@Z 00000001800d9a28     hb-font.obj
 0002:0002ea38       $chain$1$?hb_font_get_glyph_v_advances_default@@YAXPEAUhb_font_t@@PEAXIPEBIIPEAHI1@Z 00000001800d9a38     hb-font.obj
 0002:0002ea50       $chain$2$?hb_font_get_glyph_v_advances_default@@YAXPEAUhb_font_t@@PEAXIPEBIIPEAHI1@Z 00000001800d9a50     hb-font.obj
 0002:0002ea60       $unwind$?hb_font_get_glyph_h_origin_default@@YAHPEAUhb_font_t@@PEAXIPEAH21@Z 00000001800d9a60     hb-font.obj
 0002:0002ea60       $unwind$?hb_font_get_glyph_v_origin_default@@YAHPEAUhb_font_t@@PEAXIPEAH21@Z 00000001800d9a60     hb-font.obj
 0002:0002ea60       $unwind$?hb_jdk_get_glyph_h_advance@@YAHPEAUhb_font_t@@PEAXI1@Z 00000001800d9a60     hb-jdk-font.obj
 0002:0002ea60       $unwind$?reference_table@@YAPEAUhb_blob_t@@PEAUhb_face_t@@IPEAX@Z 00000001800d9a60     hb-jdk-font.obj
 0002:0002ea60       $unwind$Java_sun_font_SunLayoutEngine_createFace 00000001800d9a60     hb-jdk-font.obj
 0002:0002ea60       $unwind$?process_op@?$cs_opset_t@Unumber_t@CFF@@Ucff1_cs_opset_path_t@@Ucff1_cs_interp_env_t@2@Ucff1_path_param_t@@Ucff1_path_procs_path_t@@@CFF@@SAXIAEAUcff1_cs_interp_env_t@2@AEAUcff1_path_param_t@@@Z 00000001800d9a60     hb-ot-cff1-table.obj
 0002:0002ea60       $unwind$?get_clip_box@ClipBoxFormat2@OT@@QEBAXAEAUClipBoxData@2@AEBUItemVarStoreInstancer@2@@Z 00000001800d9a60     hb-ot-font.obj
 0002:0002ea60       $unwind$?get_delta@ItemVariationStore@OT@@QEBAMIPEBHIPEAU?$hb_atomic_t@H@@@Z 00000001800d9a60     hb-ot-font.obj
 0002:0002ea60       $unwind$?apply@?$SingleSubstFormat1_3@USmallTypes@Layout@OT@@@GSUB_impl@Layout@OT@@QEBA_NPEAUhb_ot_apply_context_t@4@@Z 00000001800d9a60     hb-ot-layout.obj
 0002:0002ea60       $unwind$?apply@SinglePosFormat1@GPOS_impl@Layout@OT@@QEBA_NPEAUhb_ot_apply_context_t@4@@Z 00000001800d9a60     hb-ot-layout.obj
 0002:0002ea70       $unwind$?hb_draw_cubic_to_default@@YAXPEAUhb_draw_funcs_t@@PEAXPEAUhb_draw_state_t@@MMMMMM1@Z 00000001800d9a70     hb-font.obj
 0002:0002ea7c       $unwind$?hb_font_paint_glyph_or_fail_default@@YAHPEAUhb_font_t@@PEAXIPEAUhb_paint_funcs_t@@1II1@Z 00000001800d9a7c     hb-font.obj
 0002:0002ea90       $unwind$jdk_font_create_hbp 00000001800d9a90     hb-jdk-font-p.obj
 0002:0002eaa0       $chain$0$?hb_jdk_get_glyph_h_advance@@YAHPEAUhb_font_t@@PEAXI1@Z 00000001800d9aa0     hb-jdk-font.obj
 0002:0002eab4       $chain$1$?hb_jdk_get_glyph_h_advance@@YAHPEAUhb_font_t@@PEAXI1@Z 00000001800d9ab4     hb-jdk-font.obj
 0002:0002eac4       $chain$0$?hb_jdk_get_glyph_v_advance@@YAHPEAUhb_font_t@@PEAXI1@Z 00000001800d9ac4     hb-jdk-font.obj
 0002:0002ead8       $chain$1$?hb_jdk_get_glyph_v_advance@@YAHPEAUhb_font_t@@PEAXI1@Z 00000001800d9ad8     hb-jdk-font.obj
 0002:0002eae8       $unwind$?hb_parse_int@@YA_NPEAPEBDPEBDPEAH_N@Z 00000001800d9ae8     hb-number.obj
 0002:0002eb00       $unwind$?strtod_rl@@YANPEBDPEAPEBD@Z 00000001800d9b00     hb-number.obj
 0002:0002eb10       $chain$6$?strtod_rl@@YANPEBDPEAPEBD@Z 00000001800d9b10     hb-number.obj
 0002:0002eb3c       $chain$7$?strtod_rl@@YANPEBDPEAPEBD@Z 00000001800d9b3c     hb-number.obj
 0002:0002eb50       $chain$8$?strtod_rl@@YANPEBDPEAPEBD@Z 00000001800d9b50     hb-number.obj
 0002:0002eb60       $unwind$?get_fd@FDSelect@CFF@@QEBAII@Z 00000001800d9b60     hb-ot-cff1-table.obj
 0002:0002eb60       $unwind$__scrt_is_nonwritable_in_current_image$filt$0 00000001800d9b60     MSVCRT:utility.obj
 0002:0002eb68       $chain$2$?get_fd@FDSelect@CFF@@QEBAII@Z 00000001800d9b68     hb-ot-cff1-table.obj
 0002:0002eb84       $chain$3$?get_fd@FDSelect@CFF@@QEBAII@Z 00000001800d9b84     hb-ot-cff1-table.obj
 0002:0002eb94       $chain$0$?get_glyph@Charset@CFF@@QEBAIII@Z 00000001800d9b94     hb-ot-cff1-table.obj
 0002:0002eba8       $chain$1$?get_glyph@Charset@CFF@@QEBAIII@Z 00000001800d9ba8     hb-ot-cff1-table.obj
 0002:0002eba8       $chain$11$?get_glyph@Charset@CFF@@QEBAIII@Z 00000001800d9ba8     hb-ot-cff1-table.obj
 0002:0002ebb8       $chain$4$?get_glyph@Charset@CFF@@QEBAIII@Z 00000001800d9bb8     hb-ot-cff1-table.obj
 0002:0002ebd4       $chain$6$?get_glyph@Charset@CFF@@QEBAIII@Z 00000001800d9bd4     hb-ot-cff1-table.obj
 0002:0002ebf0       $chain$10$?get_glyph@Charset@CFF@@QEBAIII@Z 00000001800d9bf0     hb-ot-cff1-table.obj
 0002:0002ebf0       $chain$8$?get_glyph@Charset@CFF@@QEBAIII@Z 00000001800d9bf0     hb-ot-cff1-table.obj
 0002:0002ec04       $unwind$??A?$CFFIndex@U?$IntType@G$01@OT@@@OT@@QEBA?AU?$hb_array_t@$$CBE@@I@Z 00000001800d9c04     hb-ot-cff1-table.obj
 0002:0002ec1c       $chain$0$??A?$CFFIndex@U?$IntType@G$01@OT@@@OT@@QEBA?AU?$hb_array_t@$$CBE@@I@Z 00000001800d9c1c     hb-ot-cff1-table.obj
 0002:0002ec30       $chain$1$??A?$CFFIndex@U?$IntType@G$01@OT@@@OT@@QEBA?AU?$hb_array_t@$$CBE@@I@Z 00000001800d9c30     hb-ot-cff1-table.obj
 0002:0002ec40       $unwind$?get_extents@accelerator_t@cff1@OT@@QEBA_NPEAUhb_font_t@@IPEAUhb_glyph_extents_t@@@Z 00000001800d9c40     hb-ot-cff1-table.obj
 0002:0002ec6c       $unwind$??0?$cs_interp_env_t@Unumber_t@CFF@@U?$Subrs@U?$IntType@G$01@OT@@@2@@CFF@@QEAA@AEBU?$hb_array_t@$$CBE@@PEBU?$Subrs@U?$IntType@G$01@OT@@@1@1@Z 00000001800d9c6c     hb-ot-cff1-table.obj
 0002:0002ec84       $unwind$?call_subr@?$cs_interp_env_t@Unumber_t@CFF@@U?$Subrs@U?$IntType@G$01@OT@@@2@@CFF@@QEAAXAEBU?$biased_subrs_t@U?$Subrs@U?$IntType@G$01@OT@@@CFF@@@2@W4cs_type_t@2@@Z 00000001800d9c84     hb-ot-cff1-table.obj
 0002:0002ec84       $unwind$?call_subr@?$cs_interp_env_t@Unumber_t@CFF@@U?$Subrs@U?$IntType@I$03@OT@@@2@@CFF@@QEAAXAEBU?$biased_subrs_t@U?$Subrs@U?$IntType@I$03@OT@@@CFF@@@2@W4cs_type_t@2@@Z 00000001800d9c84     hb-ot-cff2-table.obj
 0002:0002ec94       $chain$0$?call_subr@?$cs_interp_env_t@Unumber_t@CFF@@U?$Subrs@U?$IntType@G$01@OT@@@2@@CFF@@QEAAXAEBU?$biased_subrs_t@U?$Subrs@U?$IntType@G$01@OT@@@CFF@@@2@W4cs_type_t@2@@Z 00000001800d9c94     hb-ot-cff1-table.obj
 0002:0002eca8       $chain$1$?call_subr@?$cs_interp_env_t@Unumber_t@CFF@@U?$Subrs@U?$IntType@G$01@OT@@@2@@CFF@@QEAAXAEBU?$biased_subrs_t@U?$Subrs@U?$IntType@G$01@OT@@@CFF@@@2@W4cs_type_t@2@@Z 00000001800d9ca8     hb-ot-cff1-table.obj
 0002:0002ecb8       $chain$1$?rrcurveto@?$path_procs_t@Ucff1_path_procs_extents_t@@Ucff1_cs_interp_env_t@CFF@@Ucff1_extents_param_t@@@CFF@@SAXAEAUcff1_cs_interp_env_t@2@AEAUcff1_extents_param_t@@@Z 00000001800d9cb8     hb-ot-cff1-table.obj
 0002:0002ecd0       $chain$2$?rrcurveto@?$path_procs_t@Ucff1_path_procs_extents_t@@Ucff1_cs_interp_env_t@CFF@@Ucff1_extents_param_t@@@CFF@@SAXAEAUcff1_cs_interp_env_t@2@AEAUcff1_extents_param_t@@@Z 00000001800d9cd0     hb-ot-cff1-table.obj
 0002:0002ece0       $chain$0$?rcurveline@?$path_procs_t@Ucff1_path_procs_extents_t@@Ucff1_cs_interp_env_t@CFF@@Ucff1_extents_param_t@@@CFF@@SAXAEAUcff1_cs_interp_env_t@2@AEAUcff1_extents_param_t@@@Z 00000001800d9ce0     hb-ot-cff1-table.obj
 0002:0002ecf4       $chain$2$?rcurveline@?$path_procs_t@Ucff1_path_procs_extents_t@@Ucff1_cs_interp_env_t@CFF@@Ucff1_extents_param_t@@@CFF@@SAXAEAUcff1_cs_interp_env_t@2@AEAUcff1_extents_param_t@@@Z 00000001800d9cf4     hb-ot-cff1-table.obj
 0002:0002ed0c       $chain$3$?rcurveline@?$path_procs_t@Ucff1_path_procs_extents_t@@Ucff1_cs_interp_env_t@CFF@@Ucff1_extents_param_t@@@CFF@@SAXAEAUcff1_cs_interp_env_t@2@AEAUcff1_extents_param_t@@@Z 00000001800d9d0c     hb-ot-cff1-table.obj
 0002:0002ed1c       $chain$4$?rcurveline@?$path_procs_t@Ucff1_path_procs_extents_t@@Ucff1_cs_interp_env_t@CFF@@Ucff1_extents_param_t@@@CFF@@SAXAEAUcff1_cs_interp_env_t@2@AEAUcff1_extents_param_t@@@Z 00000001800d9d1c     hb-ot-cff1-table.obj
 0002:0002ed2c       $chain$2$?rlinecurve@?$path_procs_t@Ucff1_path_procs_extents_t@@Ucff1_cs_interp_env_t@CFF@@Ucff1_extents_param_t@@@CFF@@SAXAEAUcff1_cs_interp_env_t@2@AEAUcff1_extents_param_t@@@Z 00000001800d9d2c     hb-ot-cff1-table.obj
 0002:0002ed48       $chain$3$?rlinecurve@?$path_procs_t@Ucff1_path_procs_extents_t@@Ucff1_cs_interp_env_t@CFF@@Ucff1_extents_param_t@@@CFF@@SAXAEAUcff1_cs_interp_env_t@2@AEAUcff1_extents_param_t@@@Z 00000001800d9d48     hb-ot-cff1-table.obj
 0002:0002ed60       $chain$4$?rlinecurve@?$path_procs_t@Ucff1_path_procs_extents_t@@Ucff1_cs_interp_env_t@CFF@@Ucff1_extents_param_t@@@CFF@@SAXAEAUcff1_cs_interp_env_t@2@AEAUcff1_extents_param_t@@@Z 00000001800d9d60     hb-ot-cff1-table.obj
 0002:0002ed74       $chain$5$?rlinecurve@?$path_procs_t@Ucff1_path_procs_extents_t@@Ucff1_cs_interp_env_t@CFF@@Ucff1_extents_param_t@@@CFF@@SAXAEAUcff1_cs_interp_env_t@2@AEAUcff1_extents_param_t@@@Z 00000001800d9d74     hb-ot-cff1-table.obj
 0002:0002ed84       $chain$0$?vvcurveto@?$path_procs_t@Ucff1_path_procs_extents_t@@Ucff1_cs_interp_env_t@CFF@@Ucff1_extents_param_t@@@CFF@@SAXAEAUcff1_cs_interp_env_t@2@AEAUcff1_extents_param_t@@@Z 00000001800d9d84     hb-ot-cff1-table.obj
 0002:0002ed98       $chain$1$?vvcurveto@?$path_procs_t@Ucff1_path_procs_extents_t@@Ucff1_cs_interp_env_t@CFF@@Ucff1_extents_param_t@@@CFF@@SAXAEAUcff1_cs_interp_env_t@2@AEAUcff1_extents_param_t@@@Z 00000001800d9d98     hb-ot-cff1-table.obj
 0002:0002eda8       $chain$0$?hhcurveto@?$path_procs_t@Ucff1_path_procs_extents_t@@Ucff1_cs_interp_env_t@CFF@@Ucff1_extents_param_t@@@CFF@@SAXAEAUcff1_cs_interp_env_t@2@AEAUcff1_extents_param_t@@@Z 00000001800d9da8     hb-ot-cff1-table.obj
 0002:0002edbc       $chain$1$?hhcurveto@?$path_procs_t@Ucff1_path_procs_extents_t@@Ucff1_cs_interp_env_t@CFF@@Ucff1_extents_param_t@@@CFF@@SAXAEAUcff1_cs_interp_env_t@2@AEAUcff1_extents_param_t@@@Z 00000001800d9dbc     hb-ot-cff1-table.obj
 0002:0002edcc       $unwind$?hvcurveto@?$path_procs_t@Ucff1_path_procs_extents_t@@Ucff1_cs_interp_env_t@CFF@@Ucff1_extents_param_t@@@CFF@@SAXAEAUcff1_cs_interp_env_t@2@AEAUcff1_extents_param_t@@@Z 00000001800d9dcc     hb-ot-cff1-table.obj
 0002:0002edcc       $unwind$?vhcurveto@?$path_procs_t@Ucff1_path_procs_extents_t@@Ucff1_cs_interp_env_t@CFF@@Ucff1_extents_param_t@@@CFF@@SAXAEAUcff1_cs_interp_env_t@2@AEAUcff1_extents_param_t@@@Z 00000001800d9dcc     hb-ot-cff1-table.obj
 0002:0002ede0       $chain$0$?vhcurveto@?$path_procs_t@Ucff1_path_procs_extents_t@@Ucff1_cs_interp_env_t@CFF@@Ucff1_extents_param_t@@@CFF@@SAXAEAUcff1_cs_interp_env_t@2@AEAUcff1_extents_param_t@@@Z 00000001800d9de0     hb-ot-cff1-table.obj
 0002:0002edf4       $chain$1$?vhcurveto@?$path_procs_t@Ucff1_path_procs_extents_t@@Ucff1_cs_interp_env_t@CFF@@Ucff1_extents_param_t@@@CFF@@SAXAEAUcff1_cs_interp_env_t@2@AEAUcff1_extents_param_t@@@Z 00000001800d9df4     hb-ot-cff1-table.obj
 0002:0002ee04       $chain$2$?vhcurveto@?$path_procs_t@Ucff1_path_procs_extents_t@@Ucff1_cs_interp_env_t@CFF@@Ucff1_extents_param_t@@@CFF@@SAXAEAUcff1_cs_interp_env_t@2@AEAUcff1_extents_param_t@@@Z 00000001800d9e04     hb-ot-cff1-table.obj
 0002:0002ee18       $chain$3$?vhcurveto@?$path_procs_t@Ucff1_path_procs_extents_t@@Ucff1_cs_interp_env_t@CFF@@Ucff1_extents_param_t@@@CFF@@SAXAEAUcff1_cs_interp_env_t@2@AEAUcff1_extents_param_t@@@Z 00000001800d9e18     hb-ot-cff1-table.obj
 0002:0002ee28       $chain$0$?hvcurveto@?$path_procs_t@Ucff1_path_procs_extents_t@@Ucff1_cs_interp_env_t@CFF@@Ucff1_extents_param_t@@@CFF@@SAXAEAUcff1_cs_interp_env_t@2@AEAUcff1_extents_param_t@@@Z 00000001800d9e28     hb-ot-cff1-table.obj
 0002:0002ee3c       $chain$1$?hvcurveto@?$path_procs_t@Ucff1_path_procs_extents_t@@Ucff1_cs_interp_env_t@CFF@@Ucff1_extents_param_t@@@CFF@@SAXAEAUcff1_cs_interp_env_t@2@AEAUcff1_extents_param_t@@@Z 00000001800d9e3c     hb-ot-cff1-table.obj
 0002:0002ee4c       $chain$2$?hvcurveto@?$path_procs_t@Ucff1_path_procs_extents_t@@Ucff1_cs_interp_env_t@CFF@@Ucff1_extents_param_t@@@CFF@@SAXAEAUcff1_cs_interp_env_t@2@AEAUcff1_extents_param_t@@@Z 00000001800d9e4c     hb-ot-cff1-table.obj
 0002:0002ee60       $chain$3$?hvcurveto@?$path_procs_t@Ucff1_path_procs_extents_t@@Ucff1_cs_interp_env_t@CFF@@Ucff1_extents_param_t@@@CFF@@SAXAEAUcff1_cs_interp_env_t@2@AEAUcff1_extents_param_t@@@Z 00000001800d9e60     hb-ot-cff1-table.obj
 0002:0002ee70       $unwind$?flex1@?$path_procs_t@Ucff1_path_procs_extents_t@@Ucff1_cs_interp_env_t@CFF@@Ucff1_extents_param_t@@@CFF@@SAXAEAUcff1_cs_interp_env_t@2@AEAUcff1_extents_param_t@@@Z 00000001800d9e70     hb-ot-cff1-table.obj
 0002:0002ee70       $unwind$?flex1@?$path_procs_t@Ucff1_path_procs_path_t@@Ucff1_cs_interp_env_t@CFF@@Ucff1_path_param_t@@@CFF@@SAXAEAUcff1_cs_interp_env_t@2@AEAUcff1_path_param_t@@@Z 00000001800d9e70     hb-ot-cff1-table.obj
 0002:0002ee70       $unwind$?flex@?$path_procs_t@Ucff1_path_procs_extents_t@@Ucff1_cs_interp_env_t@CFF@@Ucff1_extents_param_t@@@CFF@@SAXAEAUcff1_cs_interp_env_t@2@AEAUcff1_extents_param_t@@@Z 00000001800d9e70     hb-ot-cff1-table.obj
 0002:0002ee70       $unwind$?flex@?$path_procs_t@Ucff1_path_procs_path_t@@Ucff1_cs_interp_env_t@CFF@@Ucff1_path_param_t@@@CFF@@SAXAEAUcff1_cs_interp_env_t@2@AEAUcff1_path_param_t@@@Z 00000001800d9e70     hb-ot-cff1-table.obj
 0002:0002ee70       $unwind$?hflex1@?$path_procs_t@Ucff1_path_procs_extents_t@@Ucff1_cs_interp_env_t@CFF@@Ucff1_extents_param_t@@@CFF@@SAXAEAUcff1_cs_interp_env_t@2@AEAUcff1_extents_param_t@@@Z 00000001800d9e70     hb-ot-cff1-table.obj
 0002:0002ee70       $unwind$?hflex1@?$path_procs_t@Ucff1_path_procs_path_t@@Ucff1_cs_interp_env_t@CFF@@Ucff1_path_param_t@@@CFF@@SAXAEAUcff1_cs_interp_env_t@2@AEAUcff1_path_param_t@@@Z 00000001800d9e70     hb-ot-cff1-table.obj
 0002:0002ee70       $unwind$?hflex@?$path_procs_t@Ucff1_path_procs_extents_t@@Ucff1_cs_interp_env_t@CFF@@Ucff1_extents_param_t@@@CFF@@SAXAEAUcff1_cs_interp_env_t@2@AEAUcff1_extents_param_t@@@Z 00000001800d9e70     hb-ot-cff1-table.obj
 0002:0002ee70       $unwind$?hflex@?$path_procs_t@Ucff1_path_procs_path_t@@Ucff1_cs_interp_env_t@CFF@@Ucff1_path_param_t@@@CFF@@SAXAEAUcff1_cs_interp_env_t@2@AEAUcff1_path_param_t@@@Z 00000001800d9e70     hb-ot-cff1-table.obj
 0002:0002ee70       $unwind$?flex1@?$path_procs_t@Ucff2_path_procs_extents_t@@U?$cff2_cs_interp_env_t@Unumber_t@CFF@@@CFF@@Ucff2_extents_param_t@@@CFF@@SAXAEAU?$cff2_cs_interp_env_t@Unumber_t@CFF@@@2@AEAUcff2_extents_param_t@@@Z 00000001800d9e70     hb-ot-cff2-table.obj
 0002:0002ee70       $unwind$?flex1@?$path_procs_t@Ucff2_path_procs_path_t@@U?$cff2_cs_interp_env_t@Unumber_t@CFF@@@CFF@@Ucff2_path_param_t@@@CFF@@SAXAEAU?$cff2_cs_interp_env_t@Unumber_t@CFF@@@2@AEAUcff2_path_param_t@@@Z 00000001800d9e70     hb-ot-cff2-table.obj
 0002:0002ee70       $unwind$?flex@?$path_procs_t@Ucff2_path_procs_extents_t@@U?$cff2_cs_interp_env_t@Unumber_t@CFF@@@CFF@@Ucff2_extents_param_t@@@CFF@@SAXAEAU?$cff2_cs_interp_env_t@Unumber_t@CFF@@@2@AEAUcff2_extents_param_t@@@Z 00000001800d9e70     hb-ot-cff2-table.obj
 0002:0002ee70       $unwind$?flex@?$path_procs_t@Ucff2_path_procs_path_t@@U?$cff2_cs_interp_env_t@Unumber_t@CFF@@@CFF@@Ucff2_path_param_t@@@CFF@@SAXAEAU?$cff2_cs_interp_env_t@Unumber_t@CFF@@@2@AEAUcff2_path_param_t@@@Z 00000001800d9e70     hb-ot-cff2-table.obj
 0002:0002ee70       $unwind$?hflex1@?$path_procs_t@Ucff2_path_procs_extents_t@@U?$cff2_cs_interp_env_t@Unumber_t@CFF@@@CFF@@Ucff2_extents_param_t@@@CFF@@SAXAEAU?$cff2_cs_interp_env_t@Unumber_t@CFF@@@2@AEAUcff2_extents_param_t@@@Z 00000001800d9e70     hb-ot-cff2-table.obj
 0002:0002ee70       $unwind$?hflex1@?$path_procs_t@Ucff2_path_procs_path_t@@U?$cff2_cs_interp_env_t@Unumber_t@CFF@@@CFF@@Ucff2_path_param_t@@@CFF@@SAXAEAU?$cff2_cs_interp_env_t@Unumber_t@CFF@@@2@AEAUcff2_path_param_t@@@Z 00000001800d9e70     hb-ot-cff2-table.obj
 0002:0002ee70       $unwind$?hflex@?$path_procs_t@Ucff2_path_procs_extents_t@@U?$cff2_cs_interp_env_t@Unumber_t@CFF@@@CFF@@Ucff2_extents_param_t@@@CFF@@SAXAEAU?$cff2_cs_interp_env_t@Unumber_t@CFF@@@2@AEAUcff2_extents_param_t@@@Z 00000001800d9e70     hb-ot-cff2-table.obj
 0002:0002ee70       $unwind$?hflex@?$path_procs_t@Ucff2_path_procs_path_t@@U?$cff2_cs_interp_env_t@Unumber_t@CFF@@@CFF@@Ucff2_path_param_t@@@CFF@@SAXAEAU?$cff2_cs_interp_env_t@Unumber_t@CFF@@@2@AEAUcff2_path_param_t@@@Z 00000001800d9e70     hb-ot-cff2-table.obj
 0002:0002ee80       $unwind$?_get_bounds@@YA_NPEBUaccelerator_t@cff1@OT@@IAEAUbounds_t@@_N@Z 00000001800d9e80     hb-ot-cff1-table.obj
 0002:0002ee9c       $unwind$?process_seac@cff1_cs_opset_extents_t@@SAXAEAUcff1_cs_interp_env_t@CFF@@AEAUcff1_extents_param_t@@@Z 00000001800d9e9c     hb-ot-cff1-table.obj
 0002:0002eeac       $chain$1$?process_seac@cff1_cs_opset_extents_t@@SAXAEAUcff1_cs_interp_env_t@CFF@@AEAUcff1_extents_param_t@@@Z 00000001800d9eac     hb-ot-cff1-table.obj
 0002:0002eec4       $chain$3$?process_seac@cff1_cs_opset_extents_t@@SAXAEAUcff1_cs_interp_env_t@CFF@@AEAUcff1_extents_param_t@@@Z 00000001800d9ec4     hb-ot-cff1-table.obj
 0002:0002eedc       $chain$4$?process_seac@cff1_cs_opset_extents_t@@SAXAEAUcff1_cs_interp_env_t@CFF@@AEAUcff1_extents_param_t@@@Z 00000001800d9edc     hb-ot-cff1-table.obj
 0002:0002eef0       $chain$5$?process_seac@cff1_cs_opset_extents_t@@SAXAEAUcff1_cs_interp_env_t@CFF@@AEAUcff1_extents_param_t@@@Z 00000001800d9ef0     hb-ot-cff1-table.obj
 0002:0002ef04       $unwind$?interpret@?$cs_interpreter_t@Ucff1_cs_interp_env_t@CFF@@Ucff1_cs_opset_extents_t@@Ucff1_extents_param_t@@@CFF@@QEAA_NAEAUcff1_extents_param_t@@@Z 00000001800d9f04     hb-ot-cff1-table.obj
 0002:0002ef04       $unwind$?interpret@?$cs_interpreter_t@Ucff1_cs_interp_env_t@CFF@@Ucff1_cs_opset_path_t@@Ucff1_path_param_t@@@CFF@@QEAA_NAEAUcff1_path_param_t@@@Z 00000001800d9f04     hb-ot-cff1-table.obj
 0002:0002ef1c       $unwind$?rlineto@?$path_procs_t@Ucff1_path_procs_path_t@@Ucff1_cs_interp_env_t@CFF@@Ucff1_path_param_t@@@CFF@@SAXAEAUcff1_cs_interp_env_t@2@AEAUcff1_path_param_t@@@Z 00000001800d9f1c     hb-ot-cff1-table.obj
 0002:0002ef1c       $unwind$?rlineto@?$path_procs_t@Ucff2_path_procs_path_t@@U?$cff2_cs_interp_env_t@Unumber_t@CFF@@@CFF@@Ucff2_path_param_t@@@CFF@@SAXAEAU?$cff2_cs_interp_env_t@Unumber_t@CFF@@@2@AEAUcff2_path_param_t@@@Z 00000001800d9f1c     hb-ot-cff2-table.obj
 0002:0002ef28       $chain$8$?rlineto@?$path_procs_t@Ucff1_path_procs_path_t@@Ucff1_cs_interp_env_t@CFF@@Ucff1_path_param_t@@@CFF@@SAXAEAUcff1_cs_interp_env_t@2@AEAUcff1_path_param_t@@@Z 00000001800d9f28     hb-ot-cff1-table.obj
 0002:0002ef5c       $chain$9$?rlineto@?$path_procs_t@Ucff1_path_procs_path_t@@Ucff1_cs_interp_env_t@CFF@@Ucff1_path_param_t@@@CFF@@SAXAEAUcff1_cs_interp_env_t@2@AEAUcff1_path_param_t@@@Z 00000001800d9f5c     hb-ot-cff1-table.obj
 0002:0002ef6c       $unwind$?hlineto@?$path_procs_t@Ucff1_path_procs_path_t@@Ucff1_cs_interp_env_t@CFF@@Ucff1_path_param_t@@@CFF@@SAXAEAUcff1_cs_interp_env_t@2@AEAUcff1_path_param_t@@@Z 00000001800d9f6c     hb-ot-cff1-table.obj
 0002:0002ef6c       $unwind$?vlineto@?$path_procs_t@Ucff1_path_procs_path_t@@Ucff1_cs_interp_env_t@CFF@@Ucff1_path_param_t@@@CFF@@SAXAEAUcff1_cs_interp_env_t@2@AEAUcff1_path_param_t@@@Z 00000001800d9f6c     hb-ot-cff1-table.obj
 0002:0002ef7c       $chain$7$?hlineto@?$path_procs_t@Ucff1_path_procs_path_t@@Ucff1_cs_interp_env_t@CFF@@Ucff1_path_param_t@@@CFF@@SAXAEAUcff1_cs_interp_env_t@2@AEAUcff1_path_param_t@@@Z 00000001800d9f7c     hb-ot-cff1-table.obj
 0002:0002efac       $chain$8$?hlineto@?$path_procs_t@Ucff1_path_procs_path_t@@Ucff1_cs_interp_env_t@CFF@@Ucff1_path_param_t@@@CFF@@SAXAEAUcff1_cs_interp_env_t@2@AEAUcff1_path_param_t@@@Z 00000001800d9fac     hb-ot-cff1-table.obj
 0002:0002efbc       $chain$7$?vlineto@?$path_procs_t@Ucff1_path_procs_path_t@@Ucff1_cs_interp_env_t@CFF@@Ucff1_path_param_t@@@CFF@@SAXAEAUcff1_cs_interp_env_t@2@AEAUcff1_path_param_t@@@Z 00000001800d9fbc     hb-ot-cff1-table.obj
 0002:0002efec       $chain$8$?vlineto@?$path_procs_t@Ucff1_path_procs_path_t@@Ucff1_cs_interp_env_t@CFF@@Ucff1_path_param_t@@@CFF@@SAXAEAUcff1_cs_interp_env_t@2@AEAUcff1_path_param_t@@@Z 00000001800d9fec     hb-ot-cff1-table.obj
 0002:0002effc       $unwind$?rrcurveto@?$path_procs_t@Ucff1_path_procs_path_t@@Ucff1_cs_interp_env_t@CFF@@Ucff1_path_param_t@@@CFF@@SAXAEAUcff1_cs_interp_env_t@2@AEAUcff1_path_param_t@@@Z 00000001800d9ffc     hb-ot-cff1-table.obj
 0002:0002effc       $unwind$?rrcurveto@?$path_procs_t@Ucff2_path_procs_path_t@@U?$cff2_cs_interp_env_t@Unumber_t@CFF@@@CFF@@Ucff2_path_param_t@@@CFF@@SAXAEAU?$cff2_cs_interp_env_t@Unumber_t@CFF@@@2@AEAUcff2_path_param_t@@@Z 00000001800d9ffc     hb-ot-cff2-table.obj
 0002:0002f008       $chain$12$?rrcurveto@?$path_procs_t@Ucff1_path_procs_path_t@@Ucff1_cs_interp_env_t@CFF@@Ucff1_path_param_t@@@CFF@@SAXAEAUcff1_cs_interp_env_t@2@AEAUcff1_path_param_t@@@Z 00000001800da008     hb-ot-cff1-table.obj
 0002:0002f04c       $chain$13$?rrcurveto@?$path_procs_t@Ucff1_path_procs_path_t@@Ucff1_cs_interp_env_t@CFF@@Ucff1_path_param_t@@@CFF@@SAXAEAUcff1_cs_interp_env_t@2@AEAUcff1_path_param_t@@@Z 00000001800da04c     hb-ot-cff1-table.obj
 0002:0002f05c       $unwind$?rcurveline@?$path_procs_t@Ucff1_path_procs_path_t@@Ucff1_cs_interp_env_t@CFF@@Ucff1_path_param_t@@@CFF@@SAXAEAUcff1_cs_interp_env_t@2@AEAUcff1_path_param_t@@@Z 00000001800da05c     hb-ot-cff1-table.obj
 0002:0002f068       $chain$1$?rcurveline@?$path_procs_t@Ucff1_path_procs_path_t@@Ucff1_cs_interp_env_t@CFF@@Ucff1_path_param_t@@@CFF@@SAXAEAUcff1_cs_interp_env_t@2@AEAUcff1_path_param_t@@@Z 00000001800da068     hb-ot-cff1-table.obj
 0002:0002f080       $chain$13$?rcurveline@?$path_procs_t@Ucff1_path_procs_path_t@@Ucff1_cs_interp_env_t@CFF@@Ucff1_path_param_t@@@CFF@@SAXAEAUcff1_cs_interp_env_t@2@AEAUcff1_path_param_t@@@Z 00000001800da080     hb-ot-cff1-table.obj
 0002:0002f0c0       $chain$14$?rcurveline@?$path_procs_t@Ucff1_path_procs_path_t@@Ucff1_cs_interp_env_t@CFF@@Ucff1_path_param_t@@@CFF@@SAXAEAUcff1_cs_interp_env_t@2@AEAUcff1_path_param_t@@@Z 00000001800da0c0     hb-ot-cff1-table.obj
 0002:0002f0d0       $chain$15$?rcurveline@?$path_procs_t@Ucff1_path_procs_path_t@@Ucff1_cs_interp_env_t@CFF@@Ucff1_path_param_t@@@CFF@@SAXAEAUcff1_cs_interp_env_t@2@AEAUcff1_path_param_t@@@Z 00000001800da0d0     hb-ot-cff1-table.obj
 0002:0002f0e0       $unwind$?rlinecurve@?$path_procs_t@Ucff1_path_procs_path_t@@Ucff1_cs_interp_env_t@CFF@@Ucff1_path_param_t@@@CFF@@SAXAEAUcff1_cs_interp_env_t@2@AEAUcff1_path_param_t@@@Z 00000001800da0e0     hb-ot-cff1-table.obj
 0002:0002f0ec       $chain$1$?rlinecurve@?$path_procs_t@Ucff1_path_procs_path_t@@Ucff1_cs_interp_env_t@CFF@@Ucff1_path_param_t@@@CFF@@SAXAEAUcff1_cs_interp_env_t@2@AEAUcff1_path_param_t@@@Z 00000001800da0ec     hb-ot-cff1-table.obj
 0002:0002f104       $chain$9$?rlinecurve@?$path_procs_t@Ucff1_path_procs_path_t@@Ucff1_cs_interp_env_t@CFF@@Ucff1_path_param_t@@@CFF@@SAXAEAUcff1_cs_interp_env_t@2@AEAUcff1_path_param_t@@@Z 00000001800da104     hb-ot-cff1-table.obj
 0002:0002f134       $chain$10$?rlinecurve@?$path_procs_t@Ucff1_path_procs_path_t@@Ucff1_cs_interp_env_t@CFF@@Ucff1_path_param_t@@@CFF@@SAXAEAUcff1_cs_interp_env_t@2@AEAUcff1_path_param_t@@@Z 00000001800da134     hb-ot-cff1-table.obj
 0002:0002f144       $chain$11$?rlinecurve@?$path_procs_t@Ucff1_path_procs_path_t@@Ucff1_cs_interp_env_t@CFF@@Ucff1_path_param_t@@@CFF@@SAXAEAUcff1_cs_interp_env_t@2@AEAUcff1_path_param_t@@@Z 00000001800da144     hb-ot-cff1-table.obj
 0002:0002f154       $unwind$?hhcurveto@?$path_procs_t@Ucff1_path_procs_path_t@@Ucff1_cs_interp_env_t@CFF@@Ucff1_path_param_t@@@CFF@@SAXAEAUcff1_cs_interp_env_t@2@AEAUcff1_path_param_t@@@Z 00000001800da154     hb-ot-cff1-table.obj
 0002:0002f154       $unwind$?vvcurveto@?$path_procs_t@Ucff1_path_procs_path_t@@Ucff1_cs_interp_env_t@CFF@@Ucff1_path_param_t@@@CFF@@SAXAEAUcff1_cs_interp_env_t@2@AEAUcff1_path_param_t@@@Z 00000001800da154     hb-ot-cff1-table.obj
 0002:0002f154       $unwind$?hhcurveto@?$path_procs_t@Ucff2_path_procs_path_t@@U?$cff2_cs_interp_env_t@Unumber_t@CFF@@@CFF@@Ucff2_path_param_t@@@CFF@@SAXAEAU?$cff2_cs_interp_env_t@Unumber_t@CFF@@@2@AEAUcff2_path_param_t@@@Z 00000001800da154     hb-ot-cff2-table.obj
 0002:0002f154       $unwind$?vvcurveto@?$path_procs_t@Ucff2_path_procs_path_t@@U?$cff2_cs_interp_env_t@Unumber_t@CFF@@@CFF@@Ucff2_path_param_t@@@CFF@@SAXAEAU?$cff2_cs_interp_env_t@Unumber_t@CFF@@@2@AEAUcff2_path_param_t@@@Z 00000001800da154     hb-ot-cff2-table.obj
 0002:0002f16c       $chain$8$?vvcurveto@?$path_procs_t@Ucff1_path_procs_path_t@@Ucff1_cs_interp_env_t@CFF@@Ucff1_path_param_t@@@CFF@@SAXAEAUcff1_cs_interp_env_t@2@AEAUcff1_path_param_t@@@Z 00000001800da16c     hb-ot-cff1-table.obj
 0002:0002f1a0       $chain$9$?vvcurveto@?$path_procs_t@Ucff1_path_procs_path_t@@Ucff1_cs_interp_env_t@CFF@@Ucff1_path_param_t@@@CFF@@SAXAEAUcff1_cs_interp_env_t@2@AEAUcff1_path_param_t@@@Z 00000001800da1a0     hb-ot-cff1-table.obj
 0002:0002f1b0       $chain$8$?hhcurveto@?$path_procs_t@Ucff1_path_procs_path_t@@Ucff1_cs_interp_env_t@CFF@@Ucff1_path_param_t@@@CFF@@SAXAEAUcff1_cs_interp_env_t@2@AEAUcff1_path_param_t@@@Z 00000001800da1b0     hb-ot-cff1-table.obj
 0002:0002f1e4       $chain$9$?hhcurveto@?$path_procs_t@Ucff1_path_procs_path_t@@Ucff1_cs_interp_env_t@CFF@@Ucff1_path_param_t@@@CFF@@SAXAEAUcff1_cs_interp_env_t@2@AEAUcff1_path_param_t@@@Z 00000001800da1e4     hb-ot-cff1-table.obj
 0002:0002f1f4       $unwind$?hvcurveto@?$path_procs_t@Ucff1_path_procs_path_t@@Ucff1_cs_interp_env_t@CFF@@Ucff1_path_param_t@@@CFF@@SAXAEAUcff1_cs_interp_env_t@2@AEAUcff1_path_param_t@@@Z 00000001800da1f4     hb-ot-cff1-table.obj
 0002:0002f1f4       $unwind$?vhcurveto@?$path_procs_t@Ucff1_path_procs_path_t@@Ucff1_cs_interp_env_t@CFF@@Ucff1_path_param_t@@@CFF@@SAXAEAUcff1_cs_interp_env_t@2@AEAUcff1_path_param_t@@@Z 00000001800da1f4     hb-ot-cff1-table.obj
 0002:0002f1f4       $unwind$?hvcurveto@?$path_procs_t@Ucff2_path_procs_path_t@@U?$cff2_cs_interp_env_t@Unumber_t@CFF@@@CFF@@Ucff2_path_param_t@@@CFF@@SAXAEAU?$cff2_cs_interp_env_t@Unumber_t@CFF@@@2@AEAUcff2_path_param_t@@@Z 00000001800da1f4     hb-ot-cff2-table.obj
 0002:0002f1f4       $unwind$?vhcurveto@?$path_procs_t@Ucff2_path_procs_path_t@@U?$cff2_cs_interp_env_t@Unumber_t@CFF@@@CFF@@Ucff2_path_param_t@@@CFF@@SAXAEAU?$cff2_cs_interp_env_t@Unumber_t@CFF@@@2@AEAUcff2_path_param_t@@@Z 00000001800da1f4     hb-ot-cff2-table.obj
 0002:0002f230       $unwind$?moveto@cff1_path_procs_path_t@@SAXAEAUcff1_cs_interp_env_t@CFF@@AEAUcff1_path_param_t@@AEBUpoint_t@3@@Z 00000001800da230     hb-ot-cff1-table.obj
 0002:0002f24c       $chain$1$?moveto@cff1_path_procs_path_t@@SAXAEAUcff1_cs_interp_env_t@CFF@@AEAUcff1_path_param_t@@AEBUpoint_t@3@@Z 00000001800da24c     hb-ot-cff1-table.obj
 0002:0002f264       $chain$2$?moveto@cff1_path_procs_path_t@@SAXAEAUcff1_cs_interp_env_t@CFF@@AEAUcff1_path_param_t@@AEBUpoint_t@3@@Z 00000001800da264     hb-ot-cff1-table.obj
 0002:0002f274       $unwind$?line@cff1_path_procs_path_t@@SAXAEAUcff1_cs_interp_env_t@CFF@@AEAUcff1_path_param_t@@AEBUpoint_t@3@@Z 00000001800da274     hb-ot-cff1-table.obj
 0002:0002f294       $unwind$?curve@cff1_path_procs_path_t@@SAXAEAUcff1_cs_interp_env_t@CFF@@AEAUcff1_path_param_t@@AEBUpoint_t@3@22@Z 00000001800da294     hb-ot-cff1-table.obj
 0002:0002f2c8       $unwind$?_get_path@@YA_NPEBUaccelerator_t@cff1@OT@@PEAUhb_font_t@@IAEAUhb_draw_session_t@@_NPEAUpoint_t@CFF@@@Z 00000001800da2c8     hb-ot-cff1-table.obj
 0002:0002f2e4       $unwind$?process_seac@cff1_cs_opset_path_t@@SAXAEAUcff1_cs_interp_env_t@CFF@@AEAUcff1_path_param_t@@@Z 00000001800da2e4     hb-ot-cff1-table.obj
 0002:0002f2f4       $chain$1$?process_seac@cff1_cs_opset_path_t@@SAXAEAUcff1_cs_interp_env_t@CFF@@AEAUcff1_path_param_t@@@Z 00000001800da2f4     hb-ot-cff1-table.obj
 0002:0002f30c       $chain$3$?process_seac@cff1_cs_opset_path_t@@SAXAEAUcff1_cs_interp_env_t@CFF@@AEAUcff1_path_param_t@@@Z 00000001800da30c     hb-ot-cff1-table.obj
 0002:0002f324       $chain$4$?process_seac@cff1_cs_opset_path_t@@SAXAEAUcff1_cs_interp_env_t@CFF@@AEAUcff1_path_param_t@@@Z 00000001800da324     hb-ot-cff1-table.obj
 0002:0002f338       $chain$5$?process_seac@cff1_cs_opset_path_t@@SAXAEAUcff1_cs_interp_env_t@CFF@@AEAUcff1_path_param_t@@@Z 00000001800da338     hb-ot-cff1-table.obj
 0002:0002f34c       $chain$0$??A?$CFFIndex@U?$IntType@I$03@OT@@@OT@@QEBA?AU?$hb_array_t@$$CBE@@I@Z 00000001800da34c     hb-ot-cff2-table.obj
 0002:0002f360       $chain$1$??A?$CFFIndex@U?$IntType@I$03@OT@@@OT@@QEBA?AU?$hb_array_t@$$CBE@@I@Z 00000001800da360     hb-ot-cff2-table.obj
 0002:0002f370       $unwind$?get_region_scalars@VarData@OT@@QEBAXPEBHIAEBUVarRegionList@2@PEAMI@Z 00000001800da370     hb-ot-cff2-table.obj
 0002:0002f378       $chain$1$?get_region_scalars@VarData@OT@@QEBAXPEBHIAEBUVarRegionList@2@PEAMI@Z 00000001800da378     hb-ot-cff2-table.obj
 0002:0002f390       $chain$6$?get_region_scalars@VarData@OT@@QEBAXPEBHIAEBUVarRegionList@2@PEAMI@Z 00000001800da390     hb-ot-cff2-table.obj
 0002:0002f3b4       $chain$7$?get_region_scalars@VarData@OT@@QEBAXPEBHIAEBUVarRegionList@2@PEAMI@Z 00000001800da3b4     hb-ot-cff2-table.obj
 0002:0002f3c4       $chain$8$?get_region_scalars@VarData@OT@@QEBAXPEBHIAEBUVarRegionList@2@PEAMI@Z 00000001800da3c4     hb-ot-cff2-table.obj
 0002:0002f3d4       $chain$9$?get_region_scalars@VarData@OT@@QEBAXPEBHIAEBUVarRegionList@2@PEAMI@Z 00000001800da3d4     hb-ot-cff2-table.obj
 0002:0002f400       $chain$1$?get_fd@CFF2FDSelect@CFF@@QEBAII@Z 00000001800da400     hb-ot-cff2-table.obj
 0002:0002f418       $chain$3$?get_fd@CFF2FDSelect@CFF@@QEBAII@Z 00000001800da418     hb-ot-cff2-table.obj
 0002:0002f418       $chain$5$?get_fd@CFF2FDSelect@CFF@@QEBAII@Z 00000001800da418     hb-ot-cff2-table.obj
 0002:0002f418       $chain$7$?get_fd@CFF2FDSelect@CFF@@QEBAII@Z 00000001800da418     hb-ot-cff2-table.obj
 0002:0002f430       $chain$10$?get_fd@CFF2FDSelect@CFF@@QEBAII@Z 00000001800da430     hb-ot-cff2-table.obj
 0002:0002f44c       $chain$12$?get_fd@CFF2FDSelect@CFF@@QEBAII@Z 00000001800da44c     hb-ot-cff2-table.obj
 0002:0002f468       $chain$13$?get_fd@CFF2FDSelect@CFF@@QEBAII@Z 00000001800da468     hb-ot-cff2-table.obj
 0002:0002f478       $unwind$?get_extents_at@accelerator_t@cff2@OT@@QEBA_NPEAUhb_font_t@@IPEAUhb_glyph_extents_t@@U?$hb_array_t@$$CBH@@@Z 00000001800da478     hb-ot-cff2-table.obj
 0002:0002f490       $chain$0$?get_extents_at@accelerator_t@cff2@OT@@QEBA_NPEAUhb_font_t@@IPEAUhb_glyph_extents_t@@U?$hb_array_t@$$CBH@@@Z 00000001800da490     hb-ot-cff2-table.obj
 0002:0002f4a4       $chain$3$?get_extents_at@accelerator_t@cff2@OT@@QEBA_NPEAUhb_font_t@@IPEAUhb_glyph_extents_t@@U?$hb_array_t@$$CBH@@@Z 00000001800da4a4     hb-ot-cff2-table.obj
 0002:0002f4c0       $chain$5$?get_extents_at@accelerator_t@cff2@OT@@QEBA_NPEAUhb_font_t@@IPEAUhb_glyph_extents_t@@U?$hb_array_t@$$CBH@@@Z 00000001800da4c0     hb-ot-cff2-table.obj
 0002:0002f4d8       $chain$6$?get_extents_at@accelerator_t@cff2@OT@@QEBA_NPEAUhb_font_t@@IPEAUhb_glyph_extents_t@@U?$hb_array_t@$$CBH@@@Z 00000001800da4d8     hb-ot-cff2-table.obj
 0002:0002f4e8       $chain$7$?get_extents_at@accelerator_t@cff2@OT@@QEBA_NPEAUhb_font_t@@IPEAUhb_glyph_extents_t@@U?$hb_array_t@$$CBH@@@Z 00000001800da4e8     hb-ot-cff2-table.obj
 0002:0002f4fc       $chain$8$?get_extents_at@accelerator_t@cff2@OT@@QEBA_NPEAUhb_font_t@@IPEAUhb_glyph_extents_t@@U?$hb_array_t@$$CBH@@@Z 00000001800da4fc     hb-ot-cff2-table.obj
 0002:0002f50c       $unwind$?get_path_at@accelerator_t@cff2@OT@@QEBA_NPEAUhb_font_t@@IAEAUhb_draw_session_t@@U?$hb_array_t@$$CBH@@@Z 00000001800da50c     hb-ot-cff2-table.obj
 0002:0002f528       $chain$0$?get_path_at@accelerator_t@cff2@OT@@QEBA_NPEAUhb_font_t@@IAEAUhb_draw_session_t@@U?$hb_array_t@$$CBH@@@Z 00000001800da528     hb-ot-cff2-table.obj
 0002:0002f53c       $chain$2$?get_path_at@accelerator_t@cff2@OT@@QEBA_NPEAUhb_font_t@@IAEAUhb_draw_session_t@@U?$hb_array_t@$$CBH@@@Z 00000001800da53c     hb-ot-cff2-table.obj
 0002:0002f554       $chain$3$?get_path_at@accelerator_t@cff2@OT@@QEBA_NPEAUhb_font_t@@IAEAUhb_draw_session_t@@U?$hb_array_t@$$CBH@@@Z 00000001800da554     hb-ot-cff2-table.obj
 0002:0002f568       $chain$4$?get_path_at@accelerator_t@cff2@OT@@QEBA_NPEAUhb_font_t@@IAEAUhb_draw_session_t@@U?$hb_array_t@$$CBH@@@Z 00000001800da568     hb-ot-cff2-table.obj
 0002:0002f578       $unwind$?hlineto@?$path_procs_t@Ucff2_path_procs_extents_t@@U?$cff2_cs_interp_env_t@Unumber_t@CFF@@@CFF@@Ucff2_extents_param_t@@@CFF@@SAXAEAU?$cff2_cs_interp_env_t@Unumber_t@CFF@@@2@AEAUcff2_extents_param_t@@@Z 00000001800da578     hb-ot-cff2-table.obj
 0002:0002f578       $unwind$?vlineto@?$path_procs_t@Ucff2_path_procs_extents_t@@U?$cff2_cs_interp_env_t@Unumber_t@CFF@@@CFF@@Ucff2_extents_param_t@@@CFF@@SAXAEAU?$cff2_cs_interp_env_t@Unumber_t@CFF@@@2@AEAUcff2_extents_param_t@@@Z 00000001800da578     hb-ot-cff2-table.obj
 0002:0002f584       $chain$0$?hlineto@?$path_procs_t@Ucff2_path_procs_extents_t@@U?$cff2_cs_interp_env_t@Unumber_t@CFF@@@CFF@@Ucff2_extents_param_t@@@CFF@@SAXAEAU?$cff2_cs_interp_env_t@Unumber_t@CFF@@@2@AEAUcff2_extents_param_t@@@Z 00000001800da584     hb-ot-cff2-table.obj
 0002:0002f598       $chain$1$?hlineto@?$path_procs_t@Ucff2_path_procs_extents_t@@U?$cff2_cs_interp_env_t@Unumber_t@CFF@@@CFF@@Ucff2_extents_param_t@@@CFF@@SAXAEAU?$cff2_cs_interp_env_t@Unumber_t@CFF@@@2@AEAUcff2_extents_param_t@@@Z 00000001800da598     hb-ot-cff2-table.obj
 0002:0002f5ac       $chain$2$?hlineto@?$path_procs_t@Ucff2_path_procs_extents_t@@U?$cff2_cs_interp_env_t@Unumber_t@CFF@@@CFF@@Ucff2_extents_param_t@@@CFF@@SAXAEAU?$cff2_cs_interp_env_t@Unumber_t@CFF@@@2@AEAUcff2_extents_param_t@@@Z 00000001800da5ac     hb-ot-cff2-table.obj
 0002:0002f5bc       $chain$3$?hlineto@?$path_procs_t@Ucff2_path_procs_extents_t@@U?$cff2_cs_interp_env_t@Unumber_t@CFF@@@CFF@@Ucff2_extents_param_t@@@CFF@@SAXAEAU?$cff2_cs_interp_env_t@Unumber_t@CFF@@@2@AEAUcff2_extents_param_t@@@Z 00000001800da5bc     hb-ot-cff2-table.obj
 0002:0002f5cc       $chain$0$?vlineto@?$path_procs_t@Ucff2_path_procs_extents_t@@U?$cff2_cs_interp_env_t@Unumber_t@CFF@@@CFF@@Ucff2_extents_param_t@@@CFF@@SAXAEAU?$cff2_cs_interp_env_t@Unumber_t@CFF@@@2@AEAUcff2_extents_param_t@@@Z 00000001800da5cc     hb-ot-cff2-table.obj
 0002:0002f5e0       $chain$1$?vlineto@?$path_procs_t@Ucff2_path_procs_extents_t@@U?$cff2_cs_interp_env_t@Unumber_t@CFF@@@CFF@@Ucff2_extents_param_t@@@CFF@@SAXAEAU?$cff2_cs_interp_env_t@Unumber_t@CFF@@@2@AEAUcff2_extents_param_t@@@Z 00000001800da5e0     hb-ot-cff2-table.obj
 0002:0002f5f4       $chain$2$?vlineto@?$path_procs_t@Ucff2_path_procs_extents_t@@U?$cff2_cs_interp_env_t@Unumber_t@CFF@@@CFF@@Ucff2_extents_param_t@@@CFF@@SAXAEAU?$cff2_cs_interp_env_t@Unumber_t@CFF@@@2@AEAUcff2_extents_param_t@@@Z 00000001800da5f4     hb-ot-cff2-table.obj
 0002:0002f604       $chain$3$?vlineto@?$path_procs_t@Ucff2_path_procs_extents_t@@U?$cff2_cs_interp_env_t@Unumber_t@CFF@@@CFF@@Ucff2_extents_param_t@@@CFF@@SAXAEAU?$cff2_cs_interp_env_t@Unumber_t@CFF@@@2@AEAUcff2_extents_param_t@@@Z 00000001800da604     hb-ot-cff2-table.obj
 0002:0002f614       $unwind$?rcurveline@?$path_procs_t@Ucff2_path_procs_extents_t@@U?$cff2_cs_interp_env_t@Unumber_t@CFF@@@CFF@@Ucff2_extents_param_t@@@CFF@@SAXAEAU?$cff2_cs_interp_env_t@Unumber_t@CFF@@@2@AEAUcff2_extents_param_t@@@Z 00000001800da614     hb-ot-cff2-table.obj
 0002:0002f614       $unwind$?rlinecurve@?$path_procs_t@Ucff2_path_procs_extents_t@@U?$cff2_cs_interp_env_t@Unumber_t@CFF@@@CFF@@Ucff2_extents_param_t@@@CFF@@SAXAEAU?$cff2_cs_interp_env_t@Unumber_t@CFF@@@2@AEAUcff2_extents_param_t@@@Z 00000001800da614     hb-ot-cff2-table.obj
 0002:0002f614       $unwind$?rrcurveto@?$path_procs_t@Ucff2_path_procs_extents_t@@U?$cff2_cs_interp_env_t@Unumber_t@CFF@@@CFF@@Ucff2_extents_param_t@@@CFF@@SAXAEAU?$cff2_cs_interp_env_t@Unumber_t@CFF@@@2@AEAUcff2_extents_param_t@@@Z 00000001800da614     hb-ot-cff2-table.obj
 0002:0002f61c       $chain$3$?rrcurveto@?$path_procs_t@Ucff2_path_procs_extents_t@@U?$cff2_cs_interp_env_t@Unumber_t@CFF@@@CFF@@Ucff2_extents_param_t@@@CFF@@SAXAEAU?$cff2_cs_interp_env_t@Unumber_t@CFF@@@2@AEAUcff2_extents_param_t@@@Z 00000001800da61c     hb-ot-cff2-table.obj
 0002:0002f63c       $chain$4$?rrcurveto@?$path_procs_t@Ucff2_path_procs_extents_t@@U?$cff2_cs_interp_env_t@Unumber_t@CFF@@@CFF@@Ucff2_extents_param_t@@@CFF@@SAXAEAU?$cff2_cs_interp_env_t@Unumber_t@CFF@@@2@AEAUcff2_extents_param_t@@@Z 00000001800da63c     hb-ot-cff2-table.obj
 0002:0002f64c       $chain$0$?rcurveline@?$path_procs_t@Ucff2_path_procs_extents_t@@U?$cff2_cs_interp_env_t@Unumber_t@CFF@@@CFF@@Ucff2_extents_param_t@@@CFF@@SAXAEAU?$cff2_cs_interp_env_t@Unumber_t@CFF@@@2@AEAUcff2_extents_param_t@@@Z 00000001800da64c     hb-ot-cff2-table.obj
 0002:0002f660       $chain$4$?rcurveline@?$path_procs_t@Ucff2_path_procs_extents_t@@U?$cff2_cs_interp_env_t@Unumber_t@CFF@@@CFF@@Ucff2_extents_param_t@@@CFF@@SAXAEAU?$cff2_cs_interp_env_t@Unumber_t@CFF@@@2@AEAUcff2_extents_param_t@@@Z 00000001800da660     hb-ot-cff2-table.obj
 0002:0002f680       $chain$5$?rcurveline@?$path_procs_t@Ucff2_path_procs_extents_t@@U?$cff2_cs_interp_env_t@Unumber_t@CFF@@@CFF@@Ucff2_extents_param_t@@@CFF@@SAXAEAU?$cff2_cs_interp_env_t@Unumber_t@CFF@@@2@AEAUcff2_extents_param_t@@@Z 00000001800da680     hb-ot-cff2-table.obj
 0002:0002f690       $chain$6$?rcurveline@?$path_procs_t@Ucff2_path_procs_extents_t@@U?$cff2_cs_interp_env_t@Unumber_t@CFF@@@CFF@@Ucff2_extents_param_t@@@CFF@@SAXAEAU?$cff2_cs_interp_env_t@Unumber_t@CFF@@@2@AEAUcff2_extents_param_t@@@Z 00000001800da690     hb-ot-cff2-table.obj
 0002:0002f6a0       $chain$4$?rlinecurve@?$path_procs_t@Ucff2_path_procs_extents_t@@U?$cff2_cs_interp_env_t@Unumber_t@CFF@@@CFF@@Ucff2_extents_param_t@@@CFF@@SAXAEAU?$cff2_cs_interp_env_t@Unumber_t@CFF@@@2@AEAUcff2_extents_param_t@@@Z 00000001800da6a0     hb-ot-cff2-table.obj
 0002:0002f6c4       $chain$5$?rlinecurve@?$path_procs_t@Ucff2_path_procs_extents_t@@U?$cff2_cs_interp_env_t@Unumber_t@CFF@@@CFF@@Ucff2_extents_param_t@@@CFF@@SAXAEAU?$cff2_cs_interp_env_t@Unumber_t@CFF@@@2@AEAUcff2_extents_param_t@@@Z 00000001800da6c4     hb-ot-cff2-table.obj
 0002:0002f6e4       $chain$6$?rlinecurve@?$path_procs_t@Ucff2_path_procs_extents_t@@U?$cff2_cs_interp_env_t@Unumber_t@CFF@@@CFF@@Ucff2_extents_param_t@@@CFF@@SAXAEAU?$cff2_cs_interp_env_t@Unumber_t@CFF@@@2@AEAUcff2_extents_param_t@@@Z 00000001800da6e4     hb-ot-cff2-table.obj
 0002:0002f700       $chain$7$?rlinecurve@?$path_procs_t@Ucff2_path_procs_extents_t@@U?$cff2_cs_interp_env_t@Unumber_t@CFF@@@CFF@@Ucff2_extents_param_t@@@CFF@@SAXAEAU?$cff2_cs_interp_env_t@Unumber_t@CFF@@@2@AEAUcff2_extents_param_t@@@Z 00000001800da700     hb-ot-cff2-table.obj
 0002:0002f718       $chain$8$?rlinecurve@?$path_procs_t@Ucff2_path_procs_extents_t@@U?$cff2_cs_interp_env_t@Unumber_t@CFF@@@CFF@@Ucff2_extents_param_t@@@CFF@@SAXAEAU?$cff2_cs_interp_env_t@Unumber_t@CFF@@@2@AEAUcff2_extents_param_t@@@Z 00000001800da718     hb-ot-cff2-table.obj
 0002:0002f72c       $chain$9$?rlinecurve@?$path_procs_t@Ucff2_path_procs_extents_t@@U?$cff2_cs_interp_env_t@Unumber_t@CFF@@@CFF@@Ucff2_extents_param_t@@@CFF@@SAXAEAU?$cff2_cs_interp_env_t@Unumber_t@CFF@@@2@AEAUcff2_extents_param_t@@@Z 00000001800da72c     hb-ot-cff2-table.obj
 0002:0002f73c       $chain$2$?vvcurveto@?$path_procs_t@Ucff2_path_procs_extents_t@@U?$cff2_cs_interp_env_t@Unumber_t@CFF@@@CFF@@Ucff2_extents_param_t@@@CFF@@SAXAEAU?$cff2_cs_interp_env_t@Unumber_t@CFF@@@2@AEAUcff2_extents_param_t@@@Z 00000001800da73c     hb-ot-cff2-table.obj
 0002:0002f758       $chain$3$?vvcurveto@?$path_procs_t@Ucff2_path_procs_extents_t@@U?$cff2_cs_interp_env_t@Unumber_t@CFF@@@CFF@@Ucff2_extents_param_t@@@CFF@@SAXAEAU?$cff2_cs_interp_env_t@Unumber_t@CFF@@@2@AEAUcff2_extents_param_t@@@Z 00000001800da758     hb-ot-cff2-table.obj
 0002:0002f768       $chain$2$?hhcurveto@?$path_procs_t@Ucff2_path_procs_extents_t@@U?$cff2_cs_interp_env_t@Unumber_t@CFF@@@CFF@@Ucff2_extents_param_t@@@CFF@@SAXAEAU?$cff2_cs_interp_env_t@Unumber_t@CFF@@@2@AEAUcff2_extents_param_t@@@Z 00000001800da768     hb-ot-cff2-table.obj
 0002:0002f784       $chain$3$?hhcurveto@?$path_procs_t@Ucff2_path_procs_extents_t@@U?$cff2_cs_interp_env_t@Unumber_t@CFF@@@CFF@@Ucff2_extents_param_t@@@CFF@@SAXAEAU?$cff2_cs_interp_env_t@Unumber_t@CFF@@@2@AEAUcff2_extents_param_t@@@Z 00000001800da784     hb-ot-cff2-table.obj
 0002:0002f794       $unwind$?hvcurveto@?$path_procs_t@Ucff2_path_procs_extents_t@@U?$cff2_cs_interp_env_t@Unumber_t@CFF@@@CFF@@Ucff2_extents_param_t@@@CFF@@SAXAEAU?$cff2_cs_interp_env_t@Unumber_t@CFF@@@2@AEAUcff2_extents_param_t@@@Z 00000001800da794     hb-ot-cff2-table.obj
 0002:0002f794       $unwind$?vhcurveto@?$path_procs_t@Ucff2_path_procs_extents_t@@U?$cff2_cs_interp_env_t@Unumber_t@CFF@@@CFF@@Ucff2_extents_param_t@@@CFF@@SAXAEAU?$cff2_cs_interp_env_t@Unumber_t@CFF@@@2@AEAUcff2_extents_param_t@@@Z 00000001800da794     hb-ot-cff2-table.obj
 0002:0002f7b0       $chain$0$?call_subr@?$cs_interp_env_t@Unumber_t@CFF@@U?$Subrs@U?$IntType@I$03@OT@@@2@@CFF@@QEAAXAEBU?$biased_subrs_t@U?$Subrs@U?$IntType@I$03@OT@@@CFF@@@2@W4cs_type_t@2@@Z 00000001800da7b0     hb-ot-cff2-table.obj
 0002:0002f7c4       $chain$1$?call_subr@?$cs_interp_env_t@Unumber_t@CFF@@U?$Subrs@U?$IntType@I$03@OT@@@2@@CFF@@QEAAXAEBU?$biased_subrs_t@U?$Subrs@U?$IntType@I$03@OT@@@CFF@@@2@W4cs_type_t@2@@Z 00000001800da7c4     hb-ot-cff2-table.obj
 0002:0002f7d4       $unwind$?process_blend@?$cff2_cs_interp_env_t@Unumber_t@CFF@@@CFF@@QEAAXXZ 00000001800da7d4     hb-ot-cff2-table.obj
 0002:0002f7dc       $chain$1$?process_blend@?$cff2_cs_interp_env_t@Unumber_t@CFF@@@CFF@@QEAAXXZ 00000001800da7dc     hb-ot-cff2-table.obj
 0002:0002f7f4       $chain$4$?process_blend@?$cff2_cs_interp_env_t@Unumber_t@CFF@@@CFF@@QEAAXXZ 00000001800da7f4     hb-ot-cff2-table.obj
 0002:0002f810       $chain$6$?process_blend@?$cff2_cs_interp_env_t@Unumber_t@CFF@@@CFF@@QEAAXXZ 00000001800da810     hb-ot-cff2-table.obj
 0002:0002f828       $chain$7$?process_blend@?$cff2_cs_interp_env_t@Unumber_t@CFF@@@CFF@@QEAAXXZ 00000001800da828     hb-ot-cff2-table.obj
 0002:0002f838       $chain$8$?process_blend@?$cff2_cs_interp_env_t@Unumber_t@CFF@@@CFF@@QEAAXXZ 00000001800da838     hb-ot-cff2-table.obj
 0002:0002f848       $chain$9$?process_blend@?$cff2_cs_interp_env_t@Unumber_t@CFF@@@CFF@@QEAAXXZ 00000001800da848     hb-ot-cff2-table.obj
 0002:0002f858       $chain$10$?process_blend@?$cff2_cs_interp_env_t@Unumber_t@CFF@@@CFF@@QEAAXXZ 00000001800da858     hb-ot-cff2-table.obj
 0002:0002f884       $chain$1$?blend_deltas@?$cff2_cs_interp_env_t@Unumber_t@CFF@@@CFF@@QEBANU?$hb_array_t@$$CBUnumber_t@CFF@@@@@Z 00000001800da884     hb-ot-cff2-table.obj
 0002:0002f89c       $chain$3$?blend_deltas@?$cff2_cs_interp_env_t@Unumber_t@CFF@@@CFF@@QEBANU?$hb_array_t@$$CBUnumber_t@CFF@@@@@Z 00000001800da89c     hb-ot-cff2-table.obj
 0002:0002f89c       $chain$5$?blend_deltas@?$cff2_cs_interp_env_t@Unumber_t@CFF@@@CFF@@QEBANU?$hb_array_t@$$CBUnumber_t@CFF@@@@@Z 00000001800da89c     hb-ot-cff2-table.obj
 0002:0002f8b4       $chain$6$?blend_deltas@?$cff2_cs_interp_env_t@Unumber_t@CFF@@@CFF@@QEBANU?$hb_array_t@$$CBUnumber_t@CFF@@@@@Z 00000001800da8b4     hb-ot-cff2-table.obj
 0002:0002f8c4       $unwind$??$?0$$CBUaccelerator_t@cff2@OT@@@?$cff2_cs_interp_env_t@Unumber_t@CFF@@@CFF@@QEAA@AEBU?$hb_array_t@$$CBE@@AEBUaccelerator_t@cff2@OT@@IPEBHI@Z 00000001800da8c4     hb-ot-cff2-table.obj
 0002:0002f8e0       $chain$8$?rlineto@?$path_procs_t@Ucff2_path_procs_path_t@@U?$cff2_cs_interp_env_t@Unumber_t@CFF@@@CFF@@Ucff2_path_param_t@@@CFF@@SAXAEAU?$cff2_cs_interp_env_t@Unumber_t@CFF@@@2@AEAUcff2_path_param_t@@@Z 00000001800da8e0     hb-ot-cff2-table.obj
 0002:0002f914       $chain$9$?rlineto@?$path_procs_t@Ucff2_path_procs_path_t@@U?$cff2_cs_interp_env_t@Unumber_t@CFF@@@CFF@@Ucff2_path_param_t@@@CFF@@SAXAEAU?$cff2_cs_interp_env_t@Unumber_t@CFF@@@2@AEAUcff2_path_param_t@@@Z 00000001800da914     hb-ot-cff2-table.obj
 0002:0002f924       $unwind$?hlineto@?$path_procs_t@Ucff2_path_procs_path_t@@U?$cff2_cs_interp_env_t@Unumber_t@CFF@@@CFF@@Ucff2_path_param_t@@@CFF@@SAXAEAU?$cff2_cs_interp_env_t@Unumber_t@CFF@@@2@AEAUcff2_path_param_t@@@Z 00000001800da924     hb-ot-cff2-table.obj
 0002:0002f924       $unwind$?vlineto@?$path_procs_t@Ucff2_path_procs_path_t@@U?$cff2_cs_interp_env_t@Unumber_t@CFF@@@CFF@@Ucff2_path_param_t@@@CFF@@SAXAEAU?$cff2_cs_interp_env_t@Unumber_t@CFF@@@2@AEAUcff2_path_param_t@@@Z 00000001800da924     hb-ot-cff2-table.obj
 0002:0002f934       $chain$8$?hlineto@?$path_procs_t@Ucff2_path_procs_path_t@@U?$cff2_cs_interp_env_t@Unumber_t@CFF@@@CFF@@Ucff2_path_param_t@@@CFF@@SAXAEAU?$cff2_cs_interp_env_t@Unumber_t@CFF@@@2@AEAUcff2_path_param_t@@@Z 00000001800da934     hb-ot-cff2-table.obj
 0002:0002f968       $chain$9$?hlineto@?$path_procs_t@Ucff2_path_procs_path_t@@U?$cff2_cs_interp_env_t@Unumber_t@CFF@@@CFF@@Ucff2_path_param_t@@@CFF@@SAXAEAU?$cff2_cs_interp_env_t@Unumber_t@CFF@@@2@AEAUcff2_path_param_t@@@Z 00000001800da968     hb-ot-cff2-table.obj
 0002:0002f978       $chain$8$?vlineto@?$path_procs_t@Ucff2_path_procs_path_t@@U?$cff2_cs_interp_env_t@Unumber_t@CFF@@@CFF@@Ucff2_path_param_t@@@CFF@@SAXAEAU?$cff2_cs_interp_env_t@Unumber_t@CFF@@@2@AEAUcff2_path_param_t@@@Z 00000001800da978     hb-ot-cff2-table.obj
 0002:0002f9ac       $chain$9$?vlineto@?$path_procs_t@Ucff2_path_procs_path_t@@U?$cff2_cs_interp_env_t@Unumber_t@CFF@@@CFF@@Ucff2_path_param_t@@@CFF@@SAXAEAU?$cff2_cs_interp_env_t@Unumber_t@CFF@@@2@AEAUcff2_path_param_t@@@Z 00000001800da9ac     hb-ot-cff2-table.obj
 0002:0002f9bc       $chain$12$?rrcurveto@?$path_procs_t@Ucff2_path_procs_path_t@@U?$cff2_cs_interp_env_t@Unumber_t@CFF@@@CFF@@Ucff2_path_param_t@@@CFF@@SAXAEAU?$cff2_cs_interp_env_t@Unumber_t@CFF@@@2@AEAUcff2_path_param_t@@@Z 00000001800da9bc     hb-ot-cff2-table.obj
 0002:0002fa00       $chain$13$?rrcurveto@?$path_procs_t@Ucff2_path_procs_path_t@@U?$cff2_cs_interp_env_t@Unumber_t@CFF@@@CFF@@Ucff2_path_param_t@@@CFF@@SAXAEAU?$cff2_cs_interp_env_t@Unumber_t@CFF@@@2@AEAUcff2_path_param_t@@@Z 00000001800daa00     hb-ot-cff2-table.obj
 0002:0002fa10       $unwind$?rcurveline@?$path_procs_t@Ucff2_path_procs_path_t@@U?$cff2_cs_interp_env_t@Unumber_t@CFF@@@CFF@@Ucff2_path_param_t@@@CFF@@SAXAEAU?$cff2_cs_interp_env_t@Unumber_t@CFF@@@2@AEAUcff2_path_param_t@@@Z 00000001800daa10     hb-ot-cff2-table.obj
 0002:0002fa1c       $chain$0$?rcurveline@?$path_procs_t@Ucff2_path_procs_path_t@@U?$cff2_cs_interp_env_t@Unumber_t@CFF@@@CFF@@Ucff2_path_param_t@@@CFF@@SAXAEAU?$cff2_cs_interp_env_t@Unumber_t@CFF@@@2@AEAUcff2_path_param_t@@@Z 00000001800daa1c     hb-ot-cff2-table.obj
 0002:0002fa30       $chain$2$?rcurveline@?$path_procs_t@Ucff2_path_procs_path_t@@U?$cff2_cs_interp_env_t@Unumber_t@CFF@@@CFF@@Ucff2_path_param_t@@@CFF@@SAXAEAU?$cff2_cs_interp_env_t@Unumber_t@CFF@@@2@AEAUcff2_path_param_t@@@Z 00000001800daa30     hb-ot-cff2-table.obj
 0002:0002fa48       $chain$14$?rcurveline@?$path_procs_t@Ucff2_path_procs_path_t@@U?$cff2_cs_interp_env_t@Unumber_t@CFF@@@CFF@@Ucff2_path_param_t@@@CFF@@SAXAEAU?$cff2_cs_interp_env_t@Unumber_t@CFF@@@2@AEAUcff2_path_param_t@@@Z 00000001800daa48     hb-ot-cff2-table.obj
 0002:0002fa88       $chain$15$?rcurveline@?$path_procs_t@Ucff2_path_procs_path_t@@U?$cff2_cs_interp_env_t@Unumber_t@CFF@@@CFF@@Ucff2_path_param_t@@@CFF@@SAXAEAU?$cff2_cs_interp_env_t@Unumber_t@CFF@@@2@AEAUcff2_path_param_t@@@Z 00000001800daa88     hb-ot-cff2-table.obj
 0002:0002fa98       $chain$16$?rcurveline@?$path_procs_t@Ucff2_path_procs_path_t@@U?$cff2_cs_interp_env_t@Unumber_t@CFF@@@CFF@@Ucff2_path_param_t@@@CFF@@SAXAEAU?$cff2_cs_interp_env_t@Unumber_t@CFF@@@2@AEAUcff2_path_param_t@@@Z 00000001800daa98     hb-ot-cff2-table.obj
 0002:0002faac       $chain$17$?rcurveline@?$path_procs_t@Ucff2_path_procs_path_t@@U?$cff2_cs_interp_env_t@Unumber_t@CFF@@@CFF@@Ucff2_path_param_t@@@CFF@@SAXAEAU?$cff2_cs_interp_env_t@Unumber_t@CFF@@@2@AEAUcff2_path_param_t@@@Z 00000001800daaac     hb-ot-cff2-table.obj
 0002:0002fabc       $unwind$?rlinecurve@?$path_procs_t@Ucff2_path_procs_path_t@@U?$cff2_cs_interp_env_t@Unumber_t@CFF@@@CFF@@Ucff2_path_param_t@@@CFF@@SAXAEAU?$cff2_cs_interp_env_t@Unumber_t@CFF@@@2@AEAUcff2_path_param_t@@@Z 00000001800daabc     hb-ot-cff2-table.obj
 0002:0002fac8       $chain$1$?rlinecurve@?$path_procs_t@Ucff2_path_procs_path_t@@U?$cff2_cs_interp_env_t@Unumber_t@CFF@@@CFF@@Ucff2_path_param_t@@@CFF@@SAXAEAU?$cff2_cs_interp_env_t@Unumber_t@CFF@@@2@AEAUcff2_path_param_t@@@Z 00000001800daac8     hb-ot-cff2-table.obj
 0002:0002fae0       $chain$2$?rlinecurve@?$path_procs_t@Ucff2_path_procs_path_t@@U?$cff2_cs_interp_env_t@Unumber_t@CFF@@@CFF@@Ucff2_path_param_t@@@CFF@@SAXAEAU?$cff2_cs_interp_env_t@Unumber_t@CFF@@@2@AEAUcff2_path_param_t@@@Z 00000001800daae0     hb-ot-cff2-table.obj
 0002:0002faf4       $chain$10$?rlinecurve@?$path_procs_t@Ucff2_path_procs_path_t@@U?$cff2_cs_interp_env_t@Unumber_t@CFF@@@CFF@@Ucff2_path_param_t@@@CFF@@SAXAEAU?$cff2_cs_interp_env_t@Unumber_t@CFF@@@2@AEAUcff2_path_param_t@@@Z 00000001800daaf4     hb-ot-cff2-table.obj
 0002:0002fb24       $chain$11$?rlinecurve@?$path_procs_t@Ucff2_path_procs_path_t@@U?$cff2_cs_interp_env_t@Unumber_t@CFF@@@CFF@@Ucff2_path_param_t@@@CFF@@SAXAEAU?$cff2_cs_interp_env_t@Unumber_t@CFF@@@2@AEAUcff2_path_param_t@@@Z 00000001800dab24     hb-ot-cff2-table.obj
 0002:0002fb34       $chain$12$?rlinecurve@?$path_procs_t@Ucff2_path_procs_path_t@@U?$cff2_cs_interp_env_t@Unumber_t@CFF@@@CFF@@Ucff2_path_param_t@@@CFF@@SAXAEAU?$cff2_cs_interp_env_t@Unumber_t@CFF@@@2@AEAUcff2_path_param_t@@@Z 00000001800dab34     hb-ot-cff2-table.obj
 0002:0002fb44       $chain$13$?rlinecurve@?$path_procs_t@Ucff2_path_procs_path_t@@U?$cff2_cs_interp_env_t@Unumber_t@CFF@@@CFF@@Ucff2_path_param_t@@@CFF@@SAXAEAU?$cff2_cs_interp_env_t@Unumber_t@CFF@@@2@AEAUcff2_path_param_t@@@Z 00000001800dab44     hb-ot-cff2-table.obj
 0002:0002fb54       $chain$8$?vvcurveto@?$path_procs_t@Ucff2_path_procs_path_t@@U?$cff2_cs_interp_env_t@Unumber_t@CFF@@@CFF@@Ucff2_path_param_t@@@CFF@@SAXAEAU?$cff2_cs_interp_env_t@Unumber_t@CFF@@@2@AEAUcff2_path_param_t@@@Z 00000001800dab54     hb-ot-cff2-table.obj
 0002:0002fb88       $chain$9$?vvcurveto@?$path_procs_t@Ucff2_path_procs_path_t@@U?$cff2_cs_interp_env_t@Unumber_t@CFF@@@CFF@@Ucff2_path_param_t@@@CFF@@SAXAEAU?$cff2_cs_interp_env_t@Unumber_t@CFF@@@2@AEAUcff2_path_param_t@@@Z 00000001800dab88     hb-ot-cff2-table.obj
 0002:0002fb98       $chain$8$?hhcurveto@?$path_procs_t@Ucff2_path_procs_path_t@@U?$cff2_cs_interp_env_t@Unumber_t@CFF@@@CFF@@Ucff2_path_param_t@@@CFF@@SAXAEAU?$cff2_cs_interp_env_t@Unumber_t@CFF@@@2@AEAUcff2_path_param_t@@@Z 00000001800dab98     hb-ot-cff2-table.obj
 0002:0002fbcc       $chain$9$?hhcurveto@?$path_procs_t@Ucff2_path_procs_path_t@@U?$cff2_cs_interp_env_t@Unumber_t@CFF@@@CFF@@Ucff2_path_param_t@@@CFF@@SAXAEAU?$cff2_cs_interp_env_t@Unumber_t@CFF@@@2@AEAUcff2_path_param_t@@@Z 00000001800dabcc     hb-ot-cff2-table.obj
 0002:0002fbdc       $unwind$?moveto@cff2_path_procs_path_t@@SAXAEAU?$cff2_cs_interp_env_t@Unumber_t@CFF@@@CFF@@AEAUcff2_path_param_t@@AEBUpoint_t@3@@Z 00000001800dabdc     hb-ot-cff2-table.obj
 0002:0002fbf8       $chain$1$?moveto@cff2_path_procs_path_t@@SAXAEAU?$cff2_cs_interp_env_t@Unumber_t@CFF@@@CFF@@AEAUcff2_path_param_t@@AEBUpoint_t@3@@Z 00000001800dabf8     hb-ot-cff2-table.obj
 0002:0002fc10       $chain$2$?moveto@cff2_path_procs_path_t@@SAXAEAU?$cff2_cs_interp_env_t@Unumber_t@CFF@@@CFF@@AEAUcff2_path_param_t@@AEBUpoint_t@3@@Z 00000001800dac10     hb-ot-cff2-table.obj
 0002:0002fc20       $unwind$?line@cff2_path_procs_path_t@@SAXAEAU?$cff2_cs_interp_env_t@Unumber_t@CFF@@@CFF@@AEAUcff2_path_param_t@@AEBUpoint_t@3@@Z 00000001800dac20     hb-ot-cff2-table.obj
 0002:0002fc40       $unwind$?curve@cff2_path_procs_path_t@@SAXAEAU?$cff2_cs_interp_env_t@Unumber_t@CFF@@@CFF@@AEAUcff2_path_param_t@@AEBUpoint_t@3@22@Z 00000001800dac40     hb-ot-cff2-table.obj
 0002:0002fc74       $chain$1$??C?$hb_lazy_loader_t@UCPAL@OT@@U?$hb_table_lazy_loader_t@UCPAL@OT@@$0CE@$00@@Uhb_face_t@@$0CE@Uhb_blob_t@@@@QEBAPEBUCPAL@OT@@XZ 00000001800dac74     hb-ot-color.obj
 0002:0002fc8c       $chain$2$??C?$hb_lazy_loader_t@UCPAL@OT@@U?$hb_table_lazy_loader_t@UCPAL@OT@@$0CE@$00@@Uhb_face_t@@$0CE@Uhb_blob_t@@@@QEBAPEBUCPAL@OT@@XZ 00000001800dac8c     hb-ot-color.obj
 0002:0002fc9c       $unwind$?get_stored@?$hb_lazy_loader_t@UCBDT_accelerator_t@OT@@U?$hb_face_lazy_loader_t@UCBDT_accelerator_t@OT@@$0CF@@@Uhb_face_t@@$0CF@U12@@@QEBAPEAUCBDT_accelerator_t@OT@@XZ 00000001800dac9c     hb-ot-color.obj
 0002:0002fcb8       $unwind$?sanitize@IndexSubtable@OT@@QEBA_NPEAUhb_sanitize_context_t@@I@Z 00000001800dacb8     hb-ot-color.obj
 0002:0002fcd4       $unwind$?get_image_data@IndexSubtable@OT@@QEBA_NIPEAI00@Z 00000001800dacd4     hb-ot-color.obj
 0002:0002fce8       $chain$2$?get_image_data@IndexSubtable@OT@@QEBA_NIPEAI00@Z 00000001800dace8     hb-ot-color.obj
 0002:0002fcfc       $unwind$?sanitize@BitmapSizeTable@OT@@QEBA_NPEAUhb_sanitize_context_t@@PEBX@Z 00000001800dacfc     hb-ot-color.obj
 0002:0002fd14       $unwind$?choose_strike@CBLC@OT@@IEBAAEBUBitmapSizeTable@2@PEAUhb_font_t@@@Z 00000001800dad14     hb-ot-color.obj
 0002:0002fd20       $chain$1$?choose_strike@CBLC@OT@@IEBAAEBUBitmapSizeTable@2@PEAUhb_font_t@@@Z 00000001800dad20     hb-ot-color.obj
 0002:0002fd38       $chain$3$?choose_strike@CBLC@OT@@IEBAAEBUBitmapSizeTable@2@PEAUhb_font_t@@@Z 00000001800dad38     hb-ot-color.obj
 0002:0002fd50       $unwind$?reference_png@accelerator_t@CBDT@OT@@QEBAPEAUhb_blob_t@@PEAUhb_font_t@@I@Z 00000001800dad50     hb-ot-color.obj
 0002:0002fd64       $unwind$?sanitize@BaseGlyphList@OT@@QEBA_NPEAUhb_sanitize_context_t@@@Z 00000001800dad64     hb-ot-color.obj
 0002:0002fd70       $chain$5$?sanitize@BaseGlyphList@OT@@QEBA_NPEAUhb_sanitize_context_t@@@Z 00000001800dad70     hb-ot-color.obj
 0002:0002fd98       $chain$7$?sanitize@BaseGlyphList@OT@@QEBA_NPEAUhb_sanitize_context_t@@@Z 00000001800dad98     hb-ot-color.obj
 0002:0002fdc0       $unwind$??1accelerator_t@COLR@OT@@QEAA@XZ 00000001800dadc0     hb-ot-color.obj
 0002:0002fdd0       $chain$0$??1accelerator_t@COLR@OT@@QEAA@XZ 00000001800dadd0     hb-ot-color.obj
 0002:0002fde4       $chain$1$??1accelerator_t@COLR@OT@@QEAA@XZ 00000001800dade4     hb-ot-color.obj
 0002:0002fdf4       $unwind$?get_base_glyph_paint@COLR@OT@@QEBAPEBUPaint@2@I@Z 00000001800dadf4     hb-ot-color.obj
 0002:0002fe08       $unwind$?get_glyph_blob@SBIXStrike@OT@@QEBAPEAUhb_blob_t@@IPEAU3@IPEAH1IPEAI@Z 00000001800dae08     hb-ot-color.obj
 0002:0002fe14       $chain$4$?get_glyph_blob@SBIXStrike@OT@@QEBAPEAUhb_blob_t@@IPEAU3@IPEAH1IPEAI@Z 00000001800dae14     hb-ot-color.obj
 0002:0002fe38       $chain$6$?get_glyph_blob@SBIXStrike@OT@@QEBAPEAUhb_blob_t@@IPEAU3@IPEAH1IPEAI@Z 00000001800dae38     hb-ot-color.obj
 0002:0002fe5c       $unwind$?choose_strike@accelerator_t@sbix@OT@@AEBAAEBUSBIXStrike@3@PEAUhb_font_t@@@Z 00000001800dae5c     hb-ot-color.obj
 0002:0002fe70       $chain$4$?choose_strike@accelerator_t@sbix@OT@@AEBAAEBUSBIXStrike@3@PEAUhb_font_t@@@Z 00000001800dae70     hb-ot-color.obj
 0002:0002fe8c       $chain$5$?choose_strike@accelerator_t@sbix@OT@@AEBAAEBUSBIXStrike@3@PEAUhb_font_t@@@Z 00000001800dae8c     hb-ot-color.obj
 0002:0002fe9c       $unwind$?reference_blob_for_glyph@accelerator_t@SVG@OT@@QEBAPEAUhb_blob_t@@I@Z 00000001800dae9c     hb-ot-color.obj
 0002:0002feb0       $unwind$?sanitize@SVG@OT@@QEBA_NPEAUhb_sanitize_context_t@@@Z 00000001800daeb0     hb-ot-color.obj
 0002:0002fec8       $unwind$??$_dispatch@UIndexSubtableArray@OT@@AEBU?$IntType@I$03@2@@hb_sanitize_context_t@@AEAA_NAEBUIndexSubtableArray@OT@@U?$hb_priority@$00@@AEBU?$IntType@I$03@2@@Z 00000001800daec8     hb-ot-color.obj
 0002:0002fed4       $chain$4$??$_dispatch@UIndexSubtableArray@OT@@AEBU?$IntType@I$03@2@@hb_sanitize_context_t@@AEAA_NAEBUIndexSubtableArray@OT@@U?$hb_priority@$00@@AEBU?$IntType@I$03@2@@Z 00000001800daed4     hb-ot-color.obj
 0002:0002fef8       $chain$6$??$_dispatch@UIndexSubtableArray@OT@@AEBU?$IntType@I$03@2@@hb_sanitize_context_t@@AEAA_NAEBUIndexSubtableArray@OT@@U?$hb_priority@$00@@AEBU?$IntType@I$03@2@@Z 00000001800daef8     hb-ot-color.obj
 0002:0002ff1c       $unwind$??$dispatch@Uhb_sanitize_context_t@@$$V@Paint@OT@@QEBA_NPEAUhb_sanitize_context_t@@@Z 00000001800daf1c     hb-ot-color.obj
 0002:0002ff34       $chain$0$??$dispatch@Uhb_sanitize_context_t@@$$V@Paint@OT@@QEBA_NPEAUhb_sanitize_context_t@@@Z 00000001800daf34     hb-ot-color.obj
 0002:0002ff48       $chain$1$??$dispatch@Uhb_sanitize_context_t@@$$V@Paint@OT@@QEBA_NPEAUhb_sanitize_context_t@@@Z 00000001800daf48     hb-ot-color.obj
 0002:0002ff58       $chain$2$??$dispatch@Uhb_sanitize_context_t@@$$V@Paint@OT@@QEBA_NPEAUhb_sanitize_context_t@@@Z 00000001800daf58     hb-ot-color.obj
 0002:0002ff6c       $unwind$??$dispatch@ULayerList@OT@@$$V@hb_sanitize_context_t@@QEAA_NAEBULayerList@OT@@@Z 00000001800daf6c     hb-ot-color.obj
 0002:0002ff78       $chain$2$??$dispatch@ULayerList@OT@@$$V@hb_sanitize_context_t@@QEAA_NAEBULayerList@OT@@@Z 00000001800daf78     hb-ot-color.obj
 0002:0002ff94       $chain$4$??$dispatch@ULayerList@OT@@$$V@hb_sanitize_context_t@@QEAA_NAEBULayerList@OT@@@Z 00000001800daf94     hb-ot-color.obj
 0002:0002ffb0       $unwind$??$sanitize_blob@USVG@OT@@@hb_sanitize_context_t@@QEAAPEAUhb_blob_t@@PEAU1@@Z 00000001800dafb0     hb-ot-color.obj
 0002:0002ffcc       $unwind$??$dispatch@U?$NoVariable@UAffine2x3@OT@@@OT@@$$V@hb_sanitize_context_t@@QEAA_NAEBU?$NoVariable@UAffine2x3@OT@@@OT@@@Z 00000001800dafcc     hb-ot-color.obj
 0002:0002ffe0       $chain$0$??$dispatch@U?$NoVariable@UAffine2x3@OT@@@OT@@$$V@hb_sanitize_context_t@@QEAA_NAEBU?$NoVariable@UAffine2x3@OT@@@OT@@@Z 00000001800dafe0     hb-ot-color.obj
 0002:0002fff4       $chain$1$??$dispatch@U?$NoVariable@UAffine2x3@OT@@@OT@@$$V@hb_sanitize_context_t@@QEAA_NAEBU?$NoVariable@UAffine2x3@OT@@@OT@@@Z 00000001800daff4     hb-ot-color.obj
 0002:00030004       $unwind$?fini@hb_ot_face_t@@QEAAXXZ 00000001800db004     hb-ot-face.obj
 0002:00030010       $chain$0$?fini@hb_ot_face_t@@QEAAXXZ 00000001800db010     hb-ot-face.obj
 0002:00030024       $chain$2$?fini@hb_ot_face_t@@QEAAXXZ 00000001800db024     hb-ot-face.obj
 0002:0003003c       $chain$3$?fini@hb_ot_face_t@@QEAAXXZ 00000001800db03c     hb-ot-face.obj
 0002:00030050       $chain$4$?fini@hb_ot_face_t@@QEAAXXZ 00000001800db050     hb-ot-face.obj
 0002:00030064       $chain$5$?fini@hb_ot_face_t@@QEAAXXZ 00000001800db064     hb-ot-face.obj
 0002:00030074       $chain$6$?fini@hb_ot_face_t@@QEAAXXZ 00000001800db074     hb-ot-face.obj
 0002:00030084       $chain$7$?fini@hb_ot_face_t@@QEAAXXZ 00000001800db084     hb-ot-face.obj
 0002:00030094       $chain$2$?shrink_vector@?$hb_vector_t@U?$cff1_private_dict_values_base_t@Udict_val_t@CFF@@@CFF@@$0A@@@QEAAXI@Z 00000001800db094     hb-ot-face.obj
 0002:00030094       $chain$2$?shrink_vector@?$hb_vector_t@Ucff1_font_dict_values_t@CFF@@$0A@@@QEAAXI@Z 00000001800db094     hb-ot-face.obj
 0002:00030094       $chain$2$?shrink_vector@?$hb_vector_t@Ucff2_font_dict_values_t@CFF@@$0A@@@QEAAXI@Z 00000001800db094     hb-ot-face.obj
 0002:000300b0       $chain$3$?shrink_vector@?$hb_vector_t@U?$cff1_private_dict_values_base_t@Udict_val_t@CFF@@@CFF@@$0A@@@QEAAXI@Z 00000001800db0b0     hb-ot-face.obj
 0002:000300b0       $chain$3$?shrink_vector@?$hb_vector_t@Ucff1_font_dict_values_t@CFF@@$0A@@@QEAAXI@Z 00000001800db0b0     hb-ot-face.obj
 0002:000300b0       $chain$3$?shrink_vector@?$hb_vector_t@Ucff2_font_dict_values_t@CFF@@$0A@@@QEAAXI@Z 00000001800db0b0     hb-ot-face.obj
 0002:000300c0       $chain$2$?shrink_vector@?$hb_vector_t@U?$cff2_private_dict_values_base_t@Udict_val_t@CFF@@@CFF@@$0A@@@QEAAXI@Z 00000001800db0c0     hb-ot-face.obj
 0002:000300dc       $chain$3$?shrink_vector@?$hb_vector_t@U?$cff2_private_dict_values_base_t@Udict_val_t@CFF@@@CFF@@$0A@@@QEAAXI@Z 00000001800db0dc     hb-ot-face.obj
 0002:000300ec       $unwind$hb_ot_font_set_funcs 00000001800db0ec     hb-ot-font.obj
 0002:000300f8       $chain$0$hb_ot_font_set_funcs 00000001800db0f8     hb-ot-font.obj
 0002:0003010c       $chain$1$hb_ot_font_set_funcs 00000001800db10c     hb-ot-font.obj
 0002:0003011c       $unwind$??$sort_r_simple@PEAX@@YAXPEAX_K1P6AHPEBX20@Z0@Z 00000001800db11c     hb-ot-font.obj
 0002:00030134       $unwind$?sanitize@?$CFFIndex@U?$IntType@G$01@OT@@@OT@@QEBA_NPEAUhb_sanitize_context_t@@@Z 00000001800db134     hb-ot-font.obj
 0002:00030134       $unwind$?sanitize@?$CFFIndex@U?$IntType@I$03@OT@@@OT@@QEBA_NPEAUhb_sanitize_context_t@@@Z 00000001800db134     hb-ot-font.obj
 0002:00030150       $unwind$?get_delta@VarData@OT@@QEBAMIPEBHIAEBUVarRegionList@2@PEAU?$hb_atomic_t@H@@@Z 00000001800db150     hb-ot-font.obj
 0002:00030158       $chain$8$?get_delta@VarData@OT@@QEBAMIPEBHIAEBUVarRegionList@2@PEAU?$hb_atomic_t@H@@@Z 00000001800db158     hb-ot-font.obj
 0002:0003018c       $chain$10$?get_delta@VarData@OT@@QEBAMIPEBHIAEBUVarRegionList@2@PEAU?$hb_atomic_t@H@@@Z 00000001800db18c     hb-ot-font.obj
 0002:000301c0       $unwind$?get_glyph@VariationSelectorRecord@OT@@QEBA?AW4glyph_variant_t@2@IPEAIPEBX@Z 00000001800db1c0     hb-ot-font.obj
 0002:000301d4       $unwind$?push_rotate@hb_paint_funcs_t@@QEAA_NPEAXM@Z 00000001800db1d4     hb-ot-font.obj
 0002:000301e8       $chain$0$?push_rotate@hb_paint_funcs_t@@QEAA_NPEAXM@Z 00000001800db1e8     hb-ot-font.obj
 0002:000301fc       $chain$1$?push_rotate@hb_paint_funcs_t@@QEAA_NPEAXM@Z 00000001800db1fc     hb-ot-font.obj
 0002:0003020c       $unwind$?push_skew@hb_paint_funcs_t@@QEAA_NPEAXMM@Z 00000001800db20c     hb-ot-font.obj
 0002:00030220       $chain$0$?push_skew@hb_paint_funcs_t@@QEAA_NPEAXMM@Z 00000001800db220     hb-ot-font.obj
 0002:00030234       $chain$1$?push_skew@hb_paint_funcs_t@@QEAA_NPEAXMM@Z 00000001800db234     hb-ot-font.obj
 0002:00030244       $unwind$?contour_end@path_builder_t@glyf_impl@OT@@QEAAXXZ 00000001800db244     hb-ot-font.obj
 0002:00030258       $chain$6$?contour_end@path_builder_t@glyf_impl@OT@@QEAAXXZ 00000001800db258     hb-ot-font.obj
 0002:00030284       $chain$7$?contour_end@path_builder_t@glyf_impl@OT@@QEAAXXZ 00000001800db284     hb-ot-font.obj
 0002:00030298       $chain$8$?contour_end@path_builder_t@glyf_impl@OT@@QEAAXXZ 00000001800db298     hb-ot-font.obj
 0002:000302ac       $chain$9$?contour_end@path_builder_t@glyf_impl@OT@@QEAAXXZ 00000001800db2ac     hb-ot-font.obj
 0002:000302bc       $chain$10$?contour_end@path_builder_t@glyf_impl@OT@@QEAAXXZ 00000001800db2bc     hb-ot-font.obj
 0002:000302cc       $chain$11$?contour_end@path_builder_t@glyf_impl@OT@@QEAAXXZ 00000001800db2cc     hb-ot-font.obj
 0002:000302dc       $unwind$?get_extents_at@glyf_accelerator_t@OT@@QEBA_NPEAUhb_font_t@@IPEAUhb_glyph_extents_t@@U?$hb_array_t@$$CBH@@@Z 00000001800db2dc     hb-ot-font.obj
 0002:000302f4       $chain$0$?get_extents_at@glyf_accelerator_t@OT@@QEBA_NPEAUhb_font_t@@IPEAUhb_glyph_extents_t@@U?$hb_array_t@$$CBH@@@Z 00000001800db2f4     hb-ot-font.obj
 0002:00030308       $chain$1$?get_extents_at@glyf_accelerator_t@OT@@QEBA_NPEAUhb_font_t@@IPEAUhb_glyph_extents_t@@U?$hb_array_t@$$CBH@@@Z 00000001800db308     hb-ot-font.obj
 0002:00030318       $unwind$??$get_points@Upath_builder_t@glyf_impl@OT@@@glyf_accelerator_t@OT@@IEBA_NPEAUhb_font_t@@IUpath_builder_t@glyf_impl@1@U?$hb_array_t@$$CBH@@AEAUhb_glyf_scratch_t@@@Z 00000001800db318     hb-ot-font.obj
 0002:0003032c       $chain$7$??$get_points@Upath_builder_t@glyf_impl@OT@@@glyf_accelerator_t@OT@@IEBA_NPEAUhb_font_t@@IUpath_builder_t@glyf_impl@1@U?$hb_array_t@$$CBH@@AEAUhb_glyf_scratch_t@@@Z 00000001800db32c     hb-ot-font.obj
 0002:0003035c       $chain$10$??$get_points@Upath_builder_t@glyf_impl@OT@@@glyf_accelerator_t@OT@@IEBA_NPEAUhb_font_t@@IUpath_builder_t@glyf_impl@1@U?$hb_array_t@$$CBH@@AEAUhb_glyf_scratch_t@@@Z 00000001800db35c     hb-ot-font.obj
 0002:0003035c       $chain$8$??$get_points@Upath_builder_t@glyf_impl@OT@@@glyf_accelerator_t@OT@@IEBA_NPEAUhb_font_t@@IUpath_builder_t@glyf_impl@1@U?$hb_array_t@$$CBH@@AEAUhb_glyf_scratch_t@@@Z 00000001800db35c     hb-ot-font.obj
 0002:0003036c       $chain$9$??$get_points@Upath_builder_t@glyf_impl@OT@@@glyf_accelerator_t@OT@@IEBA_NPEAUhb_font_t@@IUpath_builder_t@glyf_impl@1@U?$hb_array_t@$$CBH@@AEAUhb_glyf_scratch_t@@@Z 00000001800db36c     hb-ot-font.obj
 0002:0003039c       $chain$1$?parse_bcd@dict_opset_t@CFF@@SANAEAUbyte_str_ref_t@2@@Z 00000001800db39c     hb-ot-font.obj
 0002:000303b4       $chain$2$?parse_bcd@dict_opset_t@CFF@@SANAEAUbyte_str_ref_t@2@@Z 00000001800db3b4     hb-ot-font.obj
 0002:000303c4       $chain$3$?parse_bcd@dict_opset_t@CFF@@SANAEAUbyte_str_ref_t@2@@Z 00000001800db3c4     hb-ot-font.obj
 0002:000303dc       $chain$3$?alloc@?$hb_vector_t@Ucff2_font_dict_values_t@CFF@@$0A@@@QEAA_NI_N@Z 00000001800db3dc     hb-ot-font.obj
 0002:000303fc       $chain$5$?alloc@?$hb_vector_t@Ucff2_font_dict_values_t@CFF@@$0A@@@QEAA_NI_N@Z 00000001800db3fc     hb-ot-font.obj
 0002:0003041c       $chain$6$?alloc@?$hb_vector_t@Ucff2_font_dict_values_t@CFF@@$0A@@@QEAA_NI_N@Z 00000001800db41c     hb-ot-font.obj
 0002:00030430       $chain$7$?alloc@?$hb_vector_t@Ucff2_font_dict_values_t@CFF@@$0A@@@QEAA_NI_N@Z 00000001800db430     hb-ot-font.obj
 0002:00030444       $chain$8$?alloc@?$hb_vector_t@Ucff2_font_dict_values_t@CFF@@$0A@@@QEAA_NI_N@Z 00000001800db444     hb-ot-font.obj
 0002:00030454       $chain$9$?alloc@?$hb_vector_t@Ucff2_font_dict_values_t@CFF@@$0A@@@QEAA_NI_N@Z 00000001800db454     hb-ot-font.obj
 0002:00030464       $unwind$??0?$accelerator_templ_t@Ucff2_private_dict_opset_t@CFF@@U?$cff2_private_dict_values_base_t@Udict_val_t@CFF@@@2@@cff2@OT@@QEAA@PEAUhb_face_t@@@Z 00000001800db464     hb-ot-font.obj
 0002:00030480       $chain$1$??0?$accelerator_templ_t@Ucff2_private_dict_opset_t@CFF@@U?$cff2_private_dict_values_base_t@Udict_val_t@CFF@@@2@@cff2@OT@@QEAA@PEAUhb_face_t@@@Z 00000001800db480     hb-ot-font.obj
 0002:00030498       $chain$2$??0?$accelerator_templ_t@Ucff2_private_dict_opset_t@CFF@@U?$cff2_private_dict_values_base_t@Udict_val_t@CFF@@@2@@cff2@OT@@QEAA@PEAUhb_face_t@@@Z 00000001800db498     hb-ot-font.obj
 0002:000304a8       $chain$3$?alloc@?$hb_vector_t@U?$cff2_private_dict_values_base_t@Udict_val_t@CFF@@@CFF@@$0A@@@QEAA_NI_N@Z 00000001800db4a8     hb-ot-font.obj
 0002:000304c8       $chain$5$?alloc@?$hb_vector_t@U?$cff2_private_dict_values_base_t@Udict_val_t@CFF@@@CFF@@$0A@@@QEAA_NI_N@Z 00000001800db4c8     hb-ot-font.obj
 0002:000304e8       $chain$6$?alloc@?$hb_vector_t@U?$cff2_private_dict_values_base_t@Udict_val_t@CFF@@@CFF@@$0A@@@QEAA_NI_N@Z 00000001800db4e8     hb-ot-font.obj
 0002:000304fc       $chain$7$?alloc@?$hb_vector_t@U?$cff2_private_dict_values_base_t@Udict_val_t@CFF@@@CFF@@$0A@@@QEAA_NI_N@Z 00000001800db4fc     hb-ot-font.obj
 0002:00030510       $chain$8$?alloc@?$hb_vector_t@U?$cff2_private_dict_values_base_t@Udict_val_t@CFF@@@CFF@@$0A@@@QEAA_NI_N@Z 00000001800db510     hb-ot-font.obj
 0002:00030520       $chain$9$?alloc@?$hb_vector_t@U?$cff2_private_dict_values_base_t@Udict_val_t@CFF@@@CFF@@$0A@@@QEAA_NI_N@Z 00000001800db520     hb-ot-font.obj
 0002:00030530       $unwind$?get_sid@Charset@CFF@@QEBAIIIPEAUcode_pair_t@2@@Z 00000001800db530     hb-ot-font.obj
 0002:00030538       $unwind$?sanitize@Charset@CFF@@QEBA_NPEAUhb_sanitize_context_t@@PEAI@Z 00000001800db538     hb-ot-font.obj
 0002:0003054c       $chain$1$?sanitize@Charset@CFF@@QEBA_NPEAUhb_sanitize_context_t@@PEAI@Z 00000001800db54c     hb-ot-font.obj
 0002:00030564       $chain$2$?sanitize@Charset@CFF@@QEBA_NPEAUhb_sanitize_context_t@@PEAI@Z 00000001800db564     hb-ot-font.obj
 0002:00030564       $chain$4$?sanitize@Charset@CFF@@QEBA_NPEAUhb_sanitize_context_t@@PEAI@Z 00000001800db564     hb-ot-font.obj
 0002:00030574       $chain$3$?sanitize@Charset@CFF@@QEBA_NPEAUhb_sanitize_context_t@@PEAI@Z 00000001800db574     hb-ot-font.obj
 0002:0003058c       $chain$3$?alloc@?$hb_vector_t@Ucff1_font_dict_values_t@CFF@@$0A@@@QEAA_NI_N@Z 00000001800db58c     hb-ot-font.obj
 0002:000305ac       $chain$5$?alloc@?$hb_vector_t@Ucff1_font_dict_values_t@CFF@@$0A@@@QEAA_NI_N@Z 00000001800db5ac     hb-ot-font.obj
 0002:000305cc       $chain$6$?alloc@?$hb_vector_t@Ucff1_font_dict_values_t@CFF@@$0A@@@QEAA_NI_N@Z 00000001800db5cc     hb-ot-font.obj
 0002:000305e0       $chain$7$?alloc@?$hb_vector_t@Ucff1_font_dict_values_t@CFF@@$0A@@@QEAA_NI_N@Z 00000001800db5e0     hb-ot-font.obj
 0002:000305f4       $chain$8$?alloc@?$hb_vector_t@Ucff1_font_dict_values_t@CFF@@$0A@@@QEAA_NI_N@Z 00000001800db5f4     hb-ot-font.obj
 0002:00030604       $chain$9$?alloc@?$hb_vector_t@Ucff1_font_dict_values_t@CFF@@$0A@@@QEAA_NI_N@Z 00000001800db604     hb-ot-font.obj
 0002:00030614       $unwind$??0?$accelerator_templ_t@Ucff1_private_dict_opset_t@CFF@@U?$cff1_private_dict_values_base_t@Udict_val_t@CFF@@@2@@cff1@OT@@QEAA@PEAUhb_face_t@@@Z 00000001800db614     hb-ot-font.obj
 0002:00030634       $chain$0$??0?$accelerator_templ_t@Ucff1_private_dict_opset_t@CFF@@U?$cff1_private_dict_values_base_t@Udict_val_t@CFF@@@2@@cff1@OT@@QEAA@PEAUhb_face_t@@@Z 00000001800db634     hb-ot-font.obj
 0002:00030648       $chain$1$??0?$accelerator_templ_t@Ucff1_private_dict_opset_t@CFF@@U?$cff1_private_dict_values_base_t@Udict_val_t@CFF@@@2@@cff1@OT@@QEAA@PEAUhb_face_t@@@Z 00000001800db648     hb-ot-font.obj
 0002:00030658       $chain$3$?alloc@?$hb_vector_t@U?$cff1_private_dict_values_base_t@Udict_val_t@CFF@@@CFF@@$0A@@@QEAA_NI_N@Z 00000001800db658     hb-ot-font.obj
 0002:00030678       $chain$5$?alloc@?$hb_vector_t@U?$cff1_private_dict_values_base_t@Udict_val_t@CFF@@@CFF@@$0A@@@QEAA_NI_N@Z 00000001800db678     hb-ot-font.obj
 0002:00030698       $chain$6$?alloc@?$hb_vector_t@U?$cff1_private_dict_values_base_t@Udict_val_t@CFF@@@CFF@@$0A@@@QEAA_NI_N@Z 00000001800db698     hb-ot-font.obj
 0002:000306ac       $chain$7$?alloc@?$hb_vector_t@U?$cff1_private_dict_values_base_t@Udict_val_t@CFF@@@CFF@@$0A@@@QEAA_NI_N@Z 00000001800db6ac     hb-ot-font.obj
 0002:000306c0       $chain$8$?alloc@?$hb_vector_t@U?$cff1_private_dict_values_base_t@Udict_val_t@CFF@@@CFF@@$0A@@@QEAA_NI_N@Z 00000001800db6c0     hb-ot-font.obj
 0002:000306d0       $chain$9$?alloc@?$hb_vector_t@U?$cff1_private_dict_values_base_t@Udict_val_t@CFF@@@CFF@@$0A@@@QEAA_NI_N@Z 00000001800db6d0     hb-ot-font.obj
 0002:000306e0       $unwind$??1accelerator_t@cff1@OT@@QEAA@XZ 00000001800db6e0     hb-ot-font.obj
 0002:000306ec       $chain$1$??1accelerator_t@cff1@OT@@QEAA@XZ 00000001800db6ec     hb-ot-font.obj
 0002:00030704       $chain$2$??1accelerator_t@cff1@OT@@QEAA@XZ 00000001800db704     hb-ot-font.obj
 0002:00030714       $unwind$?get_glyph_from_name@accelerator_t@cff1@OT@@QEBA_NPEBDHPEAI@Z 00000001800db714     hb-ot-font.obj
 0002:00030730       $unwind$??0accelerator_t@post@OT@@QEAA@PEAUhb_face_t@@@Z 00000001800db730     hb-ot-font.obj
 0002:00030744       $chain$1$??0accelerator_t@post@OT@@QEAA@PEAUhb_face_t@@@Z 00000001800db744     hb-ot-font.obj
 0002:00030758       $chain$2$??0accelerator_t@post@OT@@QEAA@PEAUhb_face_t@@@Z 00000001800db758     hb-ot-font.obj
 0002:0003076c       $chain$3$??0accelerator_t@post@OT@@QEAA@PEAUhb_face_t@@@Z 00000001800db76c     hb-ot-font.obj
 0002:0003077c       $chain$4$??0accelerator_t@post@OT@@QEAA@PEAUhb_face_t@@@Z 00000001800db77c     hb-ot-font.obj
 0002:0003077c       $chain$7$??0accelerator_t@post@OT@@QEAA@PEAUhb_face_t@@@Z 00000001800db77c     hb-ot-font.obj
 0002:0003078c       $chain$5$??0accelerator_t@post@OT@@QEAA@PEAUhb_face_t@@@Z 00000001800db78c     hb-ot-font.obj
 0002:000307a4       $chain$6$??0accelerator_t@post@OT@@QEAA@PEAUhb_face_t@@@Z 00000001800db7a4     hb-ot-font.obj
 0002:000307b8       $unwind$?get_glyph_from_name@accelerator_t@post@OT@@QEBA_NPEBDHPEAI@Z 00000001800db7b8     hb-ot-font.obj
 0002:000307d0       $unwind$?get_extents@accelerator_t@CBDT@OT@@QEBA_NPEAUhb_font_t@@IPEAUhb_glyph_extents_t@@_N@Z 00000001800db7d0     hb-ot-font.obj
 0002:000307d0       $unwind$?sanitize@?$PairPosFormat2_4@USmallTypes@Layout@OT@@@GPOS_impl@Layout@OT@@QEBA_NPEAUhb_sanitize_context_t@@@Z 00000001800db7d0     hb-ot-layout.obj
 0002:000307e8       $chain$2$?get_extents@accelerator_t@CBDT@OT@@QEBA_NPEAUhb_font_t@@IPEAUhb_glyph_extents_t@@_N@Z 00000001800db7e8     hb-ot-font.obj
 0002:00030804       $chain$3$?get_extents@accelerator_t@CBDT@OT@@QEBA_NPEAUhb_font_t@@IPEAUhb_glyph_extents_t@@_N@Z 00000001800db804     hb-ot-font.obj
 0002:00030814       $unwind$??0hb_paint_context_t@OT@@QEAA@PEBXPEAUhb_paint_funcs_t@@PEAXPEAUhb_font_t@@IIAEAUItemVarStoreInstancer@1@@Z 00000001800db814     hb-ot-font.obj
 0002:00030828       $unwind$?get_color@hb_paint_context_t@OT@@QEAAIIMPEAH@Z 00000001800db828     hb-ot-font.obj
 0002:0003083c       $unwind$?get_color_stop@ColorStop@OT@@QEBAXPEAUhb_paint_context_t@2@PEAUhb_color_stop_t@@IAEBUItemVarStoreInstancer@2@@Z 00000001800db83c     hb-ot-font.obj
 0002:00030854       $unwind$?paint_glyph@Affine2x3@OT@@QEBAXPEAUhb_paint_context_t@2@I@Z 00000001800db854     hb-ot-font.obj
 0002:00030880       $unwind$?paint_glyph@PaintColrLayers@OT@@QEBAXPEAUhb_paint_context_t@2@@Z 00000001800db880     hb-ot-font.obj
 0002:00030888       $chain$4$?paint_glyph@PaintColrLayers@OT@@QEBAXPEAUhb_paint_context_t@2@@Z 00000001800db888     hb-ot-font.obj
 0002:000308ac       $chain$7$?paint_glyph@PaintColrLayers@OT@@QEBAXPEAUhb_paint_context_t@2@@Z 00000001800db8ac     hb-ot-font.obj
 0002:000308c8       $chain$8$?paint_glyph@PaintColrLayers@OT@@QEBAXPEAUhb_paint_context_t@2@@Z 00000001800db8c8     hb-ot-font.obj
 0002:000308d8       $chain$9$?paint_glyph@PaintColrLayers@OT@@QEBAXPEAUhb_paint_context_t@2@@Z 00000001800db8d8     hb-ot-font.obj
 0002:000308e8       $unwind$?paint_glyph@PaintColrGlyph@OT@@QEBAXPEAUhb_paint_context_t@2@@Z 00000001800db8e8     hb-ot-font.obj
 0002:000308f0       $chain$2$?paint_glyph@PaintColrGlyph@OT@@QEBAXPEAUhb_paint_context_t@2@@Z 00000001800db8f0     hb-ot-font.obj
 0002:0003090c       $chain$4$?paint_glyph@PaintColrGlyph@OT@@QEBAXPEAUhb_paint_context_t@2@@Z 00000001800db90c     hb-ot-font.obj
 0002:00030924       $chain$5$?paint_glyph@PaintColrGlyph@OT@@QEBAXPEAUhb_paint_context_t@2@@Z 00000001800db924     hb-ot-font.obj
 0002:00030934       $chain$6$?paint_glyph@PaintColrGlyph@OT@@QEBAXPEAUhb_paint_context_t@2@@Z 00000001800db934     hb-ot-font.obj
 0002:00030944       $unwind$?paint_glyph@PaintTranslate@OT@@QEBAXPEAUhb_paint_context_t@2@I@Z 00000001800db944     hb-ot-font.obj
 0002:00030960       $unwind$?paint_glyph@PaintScale@OT@@QEBAXPEAUhb_paint_context_t@2@I@Z 00000001800db960     hb-ot-font.obj
 0002:00030978       $unwind$?paint_glyph@PaintScaleAroundCenter@OT@@QEBAXPEAUhb_paint_context_t@2@I@Z 00000001800db978     hb-ot-font.obj
 0002:00030978       $unwind$?paint_glyph@PaintSkewAroundCenter@OT@@QEBAXPEAUhb_paint_context_t@2@I@Z 00000001800db978     hb-ot-font.obj
 0002:000309ac       $unwind$?paint_glyph@PaintScaleUniform@OT@@QEBAXPEAUhb_paint_context_t@2@I@Z 00000001800db9ac     hb-ot-font.obj
 0002:000309c0       $unwind$?paint_glyph@PaintRotateAroundCenter@OT@@QEBAXPEAUhb_paint_context_t@2@I@Z 00000001800db9c0     hb-ot-font.obj
 0002:000309c0       $unwind$?paint_glyph@PaintScaleUniformAroundCenter@OT@@QEBAXPEAUhb_paint_context_t@2@I@Z 00000001800db9c0     hb-ot-font.obj
 0002:000309f0       $unwind$?paint_glyph@PaintSkew@OT@@QEBAXPEAUhb_paint_context_t@2@I@Z 00000001800db9f0     hb-ot-font.obj
 0002:00030a08       $chain$0$?get_clip_box@ClipBoxFormat2@OT@@QEBAXAEAUClipBoxData@2@AEBUItemVarStoreInstancer@2@@Z 00000001800dba08     hb-ot-font.obj
 0002:00030a1c       $chain$1$?get_clip_box@ClipBoxFormat2@OT@@QEBAXAEAUClipBoxData@2@AEBUItemVarStoreInstancer@2@@Z 00000001800dba1c     hb-ot-font.obj
 0002:00030a2c       $unwind$?paint_glyph@?$PaintLinearGradient@UNoVariable@OT@@@OT@@QEBAXPEAUhb_paint_context_t@2@I@Z 00000001800dba2c     hb-ot-font.obj
 0002:00030a2c       $unwind$?paint_glyph@?$PaintLinearGradient@UVariable@OT@@@OT@@QEBAXPEAUhb_paint_context_t@2@I@Z 00000001800dba2c     hb-ot-font.obj
 0002:00030a60       $unwind$?static_get_color_stops@?$ColorLine@UNoVariable@OT@@@OT@@SAIPEAUhb_color_line_t@@PEAXIPEAIPEAUhb_color_stop_t@@1@Z 00000001800dba60     hb-ot-font.obj
 0002:00030a60       $unwind$?static_get_color_stops@?$ColorLine@UVariable@OT@@@OT@@SAIPEAUhb_color_line_t@@PEAXIPEAIPEAUhb_color_stop_t@@1@Z 00000001800dba60     hb-ot-font.obj
 0002:00030a74       $chain$0$?static_get_color_stops@?$ColorLine@UNoVariable@OT@@@OT@@SAIPEAUhb_color_line_t@@PEAXIPEAIPEAUhb_color_stop_t@@1@Z 00000001800dba74     hb-ot-font.obj
 0002:00030a88       $chain$1$?static_get_color_stops@?$ColorLine@UNoVariable@OT@@@OT@@SAIPEAUhb_color_line_t@@PEAXIPEAIPEAUhb_color_stop_t@@1@Z 00000001800dba88     hb-ot-font.obj
 0002:00030a9c       $chain$2$?static_get_color_stops@?$ColorLine@UNoVariable@OT@@@OT@@SAIPEAUhb_color_line_t@@PEAXIPEAIPEAUhb_color_stop_t@@1@Z 00000001800dba9c     hb-ot-font.obj
 0002:00030aac       $chain$4$?static_get_color_stops@?$ColorLine@UNoVariable@OT@@@OT@@SAIPEAUhb_color_line_t@@PEAXIPEAIPEAUhb_color_stop_t@@1@Z 00000001800dbaac     hb-ot-font.obj
 0002:00030ac0       $chain$5$?static_get_color_stops@?$ColorLine@UNoVariable@OT@@@OT@@SAIPEAUhb_color_line_t@@PEAXIPEAIPEAUhb_color_stop_t@@1@Z 00000001800dbac0     hb-ot-font.obj
 0002:00030ad0       $chain$0$?static_get_color_stops@?$ColorLine@UVariable@OT@@@OT@@SAIPEAUhb_color_line_t@@PEAXIPEAIPEAUhb_color_stop_t@@1@Z 00000001800dbad0     hb-ot-font.obj
 0002:00030ae4       $chain$1$?static_get_color_stops@?$ColorLine@UVariable@OT@@@OT@@SAIPEAUhb_color_line_t@@PEAXIPEAIPEAUhb_color_stop_t@@1@Z 00000001800dbae4     hb-ot-font.obj
 0002:00030af8       $chain$2$?static_get_color_stops@?$ColorLine@UVariable@OT@@@OT@@SAIPEAUhb_color_line_t@@PEAXIPEAIPEAUhb_color_stop_t@@1@Z 00000001800dbaf8     hb-ot-font.obj
 0002:00030b08       $chain$4$?static_get_color_stops@?$ColorLine@UVariable@OT@@@OT@@SAIPEAUhb_color_line_t@@PEAXIPEAIPEAUhb_color_stop_t@@1@Z 00000001800dbb08     hb-ot-font.obj
 0002:00030b1c       $chain$5$?static_get_color_stops@?$ColorLine@UVariable@OT@@@OT@@SAIPEAUhb_color_line_t@@PEAXIPEAIPEAUhb_color_stop_t@@1@Z 00000001800dbb1c     hb-ot-font.obj
 0002:00030b2c       $unwind$?paint_glyph@?$PaintRadialGradient@UNoVariable@OT@@@OT@@QEBAXPEAUhb_paint_context_t@2@I@Z 00000001800dbb2c     hb-ot-font.obj
 0002:00030b2c       $unwind$?paint_glyph@?$PaintRadialGradient@UVariable@OT@@@OT@@QEBAXPEAUhb_paint_context_t@2@I@Z 00000001800dbb2c     hb-ot-font.obj
 0002:00030b5c       $unwind$?paint_glyph@?$PaintSweepGradient@UNoVariable@OT@@@OT@@QEBAXPEAUhb_paint_context_t@2@I@Z 00000001800dbb5c     hb-ot-font.obj
 0002:00030b5c       $unwind$?paint_glyph@?$PaintSweepGradient@UVariable@OT@@@OT@@QEBAXPEAUhb_paint_context_t@2@I@Z 00000001800dbb5c     hb-ot-font.obj
 0002:00030b84       $chain$1$?release_scratch@accelerator_t@COLR@OT@@AEBAXPEAUhb_colr_scratch_t@@@Z 00000001800dbb84     hb-ot-font.obj
 0002:00030b9c       $chain$2$?release_scratch@accelerator_t@COLR@OT@@AEBAXPEAUhb_colr_scratch_t@@@Z 00000001800dbb9c     hb-ot-font.obj
 0002:00030bac       $unwind$?get_extents@COLR@OT@@QEBA_NPEAUhb_font_t@@IPEAUhb_glyph_extents_t@@AEAUhb_colr_scratch_t@@@Z 00000001800dbbac     hb-ot-font.obj
 0002:00030bc4       $chain$1$?get_extents@COLR@OT@@QEBA_NPEAUhb_font_t@@IPEAUhb_glyph_extents_t@@AEAUhb_colr_scratch_t@@@Z 00000001800dbbc4     hb-ot-font.obj
 0002:00030bdc       $chain$2$?get_extents@COLR@OT@@QEBA_NPEAUhb_font_t@@IPEAUhb_glyph_extents_t@@AEAUhb_colr_scratch_t@@@Z 00000001800dbbdc     hb-ot-font.obj
 0002:00030bf0       $chain$3$?get_extents@COLR@OT@@QEBA_NPEAUhb_font_t@@IPEAUhb_glyph_extents_t@@AEAUhb_colr_scratch_t@@@Z 00000001800dbbf0     hb-ot-font.obj
 0002:00030c00       $unwind$?paint_glyph@COLR@OT@@QEBA_NPEAUhb_font_t@@IPEAUhb_paint_funcs_t@@PEAXII_NAEAUhb_colr_scratch_t@@@Z 00000001800dbc00     hb-ot-font.obj
 0002:00030c1c       $unwind$?get_png_extents@accelerator_t@sbix@OT@@AEBA_NPEAUhb_font_t@@IPEAUhb_glyph_extents_t@@_N@Z 00000001800dbc1c     hb-ot-font.obj
 0002:00030c34       $chain$0$?acquire_varStore_cache@advance_cache_t@hb_ot_font_t@@QEBAPEAU?$hb_atomic_t@H@@AEBUItemVariationStore@OT@@@Z 00000001800dbc34     hb-ot-font.obj
 0002:00030c48       $chain$1$?acquire_varStore_cache@advance_cache_t@hb_ot_font_t@@QEBAPEAU?$hb_atomic_t@H@@AEBUItemVariationStore@OT@@@Z 00000001800dbc48     hb-ot-font.obj
 0002:00030c58       $chain$2$?acquire_varStore_cache@advance_cache_t@hb_ot_font_t@@QEBAPEAU?$hb_atomic_t@H@@AEBUItemVariationStore@OT@@@Z 00000001800dbc58     hb-ot-font.obj
 0002:00030c6c       $chain$3$?acquire_varStore_cache@advance_cache_t@hb_ot_font_t@@QEBAPEAU?$hb_atomic_t@H@@AEBUItemVariationStore@OT@@@Z 00000001800dbc6c     hb-ot-font.obj
 0002:00030c80       $chain$4$?acquire_varStore_cache@advance_cache_t@hb_ot_font_t@@QEBAPEAU?$hb_atomic_t@H@@AEBUItemVariationStore@OT@@@Z 00000001800dbc80     hb-ot-font.obj
 0002:00030c90       $unwind$?hb_ot_get_nominal_glyphs@@YAIPEAUhb_font_t@@PEAXIPEBIIPEAII1@Z 00000001800dbc90     hb-ot-font.obj
 0002:00030ca0       $chain$2$?hb_ot_get_nominal_glyphs@@YAIPEAUhb_font_t@@PEAXIPEBIIPEAII1@Z 00000001800dbca0     hb-ot-font.obj
 0002:00030cbc       $chain$3$?hb_ot_get_nominal_glyphs@@YAIPEAUhb_font_t@@PEAXIPEBIIPEAII1@Z 00000001800dbcbc     hb-ot-font.obj
 0002:00030ccc       $unwind$?hb_ot_get_glyph_h_advances@@YAXPEAUhb_font_t@@PEAXIPEBIIPEAHI1@Z 00000001800dbccc     hb-ot-font.obj
 0002:00030cd4       $chain$8$?hb_ot_get_glyph_h_advances@@YAXPEAUhb_font_t@@PEAXIPEBIIPEAHI1@Z 00000001800dbcd4     hb-ot-font.obj
 0002:00030d08       $chain$9$?hb_ot_get_glyph_h_advances@@YAXPEAUhb_font_t@@PEAXIPEBIIPEAHI1@Z 00000001800dbd08     hb-ot-font.obj
 0002:00030d18       $unwind$?hb_ot_get_glyph_v_advances@@YAXPEAUhb_font_t@@PEAXIPEBIIPEAHI1@Z 00000001800dbd18     hb-ot-font.obj
 0002:00030d3c       $chain$0$?hb_ot_get_glyph_v_advances@@YAXPEAUhb_font_t@@PEAXIPEBIIPEAHI1@Z 00000001800dbd3c     hb-ot-font.obj
 0002:00030d50       $chain$1$?hb_ot_get_glyph_v_advances@@YAXPEAUhb_font_t@@PEAXIPEBIIPEAHI1@Z 00000001800dbd50     hb-ot-font.obj
 0002:00030d60       $unwind$?hb_ot_get_glyph_v_origin@@YAHPEAUhb_font_t@@PEAXIPEAH21@Z 00000001800dbd60     hb-ot-font.obj
 0002:00030d80       $chain$0$?hb_ot_get_glyph_v_origin@@YAHPEAUhb_font_t@@PEAXIPEAH21@Z 00000001800dbd80     hb-ot-font.obj
 0002:00030d94       $chain$2$?hb_ot_get_glyph_v_origin@@YAHPEAUhb_font_t@@PEAXIPEAH21@Z 00000001800dbd94     hb-ot-font.obj
 0002:00030da8       $chain$3$?hb_ot_get_glyph_v_origin@@YAHPEAUhb_font_t@@PEAXIPEAH21@Z 00000001800dbda8     hb-ot-font.obj
 0002:00030db8       $unwind$?hb_ot_get_glyph_extents@@YAHPEAUhb_font_t@@PEAXIPEAUhb_glyph_extents_t@@1@Z 00000001800dbdb8     hb-ot-font.obj
 0002:00030dd4       $unwind$?hb_ot_get_glyph_name@@YAHPEAUhb_font_t@@PEAXIPEADI1@Z 00000001800dbdd4     hb-ot-font.obj
 0002:00030de8       $unwind$?hb_ot_draw_glyph_or_fail@@YAHPEAUhb_font_t@@PEAXIPEAUhb_draw_funcs_t@@11@Z 00000001800dbde8     hb-ot-font.obj
 0002:00030e04       $chain$1$?hb_ot_draw_glyph_or_fail@@YAHPEAUhb_font_t@@PEAXIPEAUhb_draw_funcs_t@@11@Z 00000001800dbe04     hb-ot-font.obj
 0002:00030e1c       $chain$2$?hb_ot_draw_glyph_or_fail@@YAHPEAUhb_font_t@@PEAXIPEAUhb_draw_funcs_t@@11@Z 00000001800dbe1c     hb-ot-font.obj
 0002:00030e30       $chain$3$?hb_ot_draw_glyph_or_fail@@YAHPEAUhb_font_t@@PEAXIPEAUhb_draw_funcs_t@@11@Z 00000001800dbe30     hb-ot-font.obj
 0002:00030e40       $chain$4$?hb_ot_draw_glyph_or_fail@@YAHPEAUhb_font_t@@PEAXIPEAUhb_draw_funcs_t@@11@Z 00000001800dbe40     hb-ot-font.obj
 0002:00030e50       $unwind$?hb_ot_paint_glyph_or_fail@@YAHPEAUhb_font_t@@PEAXIPEAUhb_paint_funcs_t@@1II1@Z 00000001800dbe50     hb-ot-font.obj
 0002:00030e78       $chain$0$??$sanitize@Uhb_sanitize_context_t@@@?$hb_array_t@$$CBE@@QEBA_NPEAUhb_sanitize_context_t@@@Z 00000001800dbe78     hb-ot-font.obj
 0002:00030e8c       $chain$1$??$sanitize@Uhb_sanitize_context_t@@@?$hb_array_t@$$CBE@@QEBA_NPEAUhb_sanitize_context_t@@@Z 00000001800dbe8c     hb-ot-font.obj
 0002:00030e9c       $unwind$?interpret@?$dict_interpreter_t@Ucff1_font_dict_opset_t@CFF@@Ucff1_font_dict_values_t@2@U?$interp_env_t@Unumber_t@CFF@@@2@@CFF@@QEAA_NAEAUcff1_font_dict_values_t@2@@Z 00000001800dbe9c     hb-ot-font.obj
 0002:00030e9c       $unwind$?interpret@?$dict_interpreter_t@Ucff2_font_dict_opset_t@CFF@@Ucff2_font_dict_values_t@2@U?$interp_env_t@Unumber_t@CFF@@@2@@CFF@@QEAA_NAEAUcff2_font_dict_values_t@2@@Z 00000001800dbe9c     hb-ot-font.obj
 0002:00030e9c       $unwind$?_apply@?$ContextFormat2_5@USmallTypes@Layout@OT@@@OT@@QEBA_NPEAUhb_ot_apply_context_t@2@_N@Z 00000001800dbe9c     hb-ot-layout.obj
 0002:00030e9c       $unwind$?has_feature@hb_ot_map_builder_t@@QEAA_NI@Z 00000001800dbe9c     hb-ot-map.obj
 0002:00030e9c       $unwind$?get_var@MVAR@OT@@QEBAMIPEBHI@Z 00000001800dbe9c     hb-ot-metrics.obj
 0002:00030e9c       $unwind$?would_substitute@hb_indic_would_substitute_feature_t@@QEBA_NPEBIIPEAUhb_face_t@@@Z 00000001800dbe9c     hb-ot-shaper-indic.obj
 0002:00030eb4       $unwind$?interpret@?$dict_interpreter_t@Ucff1_private_dict_opset_t@CFF@@U?$cff1_private_dict_values_base_t@Udict_val_t@CFF@@@2@U?$interp_env_t@Unumber_t@CFF@@@2@@CFF@@QEAA_NAEAU?$cff1_private_dict_values_base_t@Udict_val_t@CFF@@@2@@Z 00000001800dbeb4     hb-ot-font.obj
 0002:00030eb4       $unwind$?interpret@?$dict_interpreter_t@Ucff2_private_dict_opset_t@CFF@@U?$cff2_private_dict_values_base_t@Udict_val_t@CFF@@@2@Ucff2_priv_dict_interp_env_t@2@@CFF@@QEAA_NAEAU?$cff2_private_dict_values_base_t@Udict_val_t@CFF@@@2@@Z 00000001800dbeb4     hb-ot-font.obj
 0002:00030ecc       $unwind$??$sanitize_blob@Ucff1@OT@@@hb_sanitize_context_t@@QEAAPEAUhb_blob_t@@PEAU1@@Z 00000001800dbecc     hb-ot-font.obj
 0002:00030ecc       $unwind$??$sanitize_blob@Ucff2@OT@@@hb_sanitize_context_t@@QEAAPEAUhb_blob_t@@PEAU1@@Z 00000001800dbecc     hb-ot-font.obj
 0002:00030ee8       $unwind$hb_ot_layout_collect_features_map 00000001800dbee8     hb-ot-layout.obj
 0002:00030ef8       $chain$2$hb_ot_layout_collect_features_map 00000001800dbef8     hb-ot-layout.obj
 0002:00030f14       $chain$3$hb_ot_layout_collect_features_map 00000001800dbf14     hb-ot-layout.obj
 0002:00030f24       $unwind$hb_ot_layout_table_find_feature_variations 00000001800dbf24     hb-ot-layout.obj
 0002:00030f38       $unwind$hb_ot_layout_lookup_would_substitute 00000001800dbf38     hb-ot-layout.obj
 0002:00030f4c       $chain$2$hb_ot_layout_lookup_would_substitute 00000001800dbf4c     hb-ot-layout.obj
 0002:00030f64       $chain$3$hb_ot_layout_lookup_would_substitute 00000001800dbf64     hb-ot-layout.obj
 0002:00030f74       $unwind$?_set_glyph_flags@hb_buffer_t@@QEAAXIII_N0@Z 00000001800dbf74     hb-ot-layout.obj
 0002:00030f88       $chain$0$?_set_glyph_flags@hb_buffer_t@@QEAAXIII_N0@Z 00000001800dbf88     hb-ot-layout.obj
 0002:00030f9c       $chain$1$?_set_glyph_flags@hb_buffer_t@@QEAAXIII_N0@Z 00000001800dbf9c     hb-ot-layout.obj
 0002:00030fac       $unwind$?position@hb_ot_map_t@@QEBAXPEBUhb_ot_shape_plan_t@@PEAUhb_font_t@@PEAUhb_buffer_t@@@Z 00000001800dbfac     hb-ot-layout.obj
 0002:00030fac       $unwind$?substitute@hb_ot_map_t@@QEBAXPEBUhb_ot_shape_plan_t@@PEAUhb_font_t@@PEAUhb_buffer_t@@@Z 00000001800dbfac     hb-ot-layout.obj
 0002:00030fc0       $unwind$?get_stored@?$hb_lazy_loader_t@UGPOS_accelerator_t@OT@@U?$hb_face_lazy_loader_t@UGPOS_accelerator_t@OT@@$0BK@@@Uhb_face_t@@$0BK@U12@@@QEBAPEAUGPOS_accelerator_t@OT@@XZ 00000001800dbfc0     hb-ot-layout.obj
 0002:00030fc0       $unwind$?get_stored@?$hb_lazy_loader_t@UGSUB_accelerator_t@OT@@U?$hb_face_lazy_loader_t@UGSUB_accelerator_t@OT@@$0BJ@@@Uhb_face_t@@$0BJ@U12@@@QEBAPEAUGSUB_accelerator_t@OT@@XZ 00000001800dbfc0     hb-ot-layout.obj
 0002:00030fdc       $unwind$?process_@hb_bit_set_t@@QEAAXP6A?AU?$hb_vector_size_t@_K$0EA@@@AEBU2@0@Z_N2AEBU1@@Z 00000001800dbfdc     hb-ot-layout.obj
 0002:00030ff0       $chain$5$?process_@hb_bit_set_t@@QEAAXP6A?AU?$hb_vector_size_t@_K$0EA@@@AEBU2@0@Z_N2AEBU1@@Z 00000001800dbff0     hb-ot-layout.obj
 0002:00031018       $chain$6$?process_@hb_bit_set_t@@QEAAXP6A?AU?$hb_vector_size_t@_K$0EA@@@AEBU2@0@Z_N2AEBU1@@Z 00000001800dc018     hb-ot-layout.obj
 0002:00031028       $unwind$?hb_ot_layout_kern@@YAXPEBUhb_ot_shape_plan_t@@PEAUhb_font_t@@PEAUhb_buffer_t@@@Z 00000001800dc028     hb-ot-layout.obj
 0002:00031040       $unwind$?_apply@?$ChainContextFormat2_5@USmallTypes@Layout@OT@@@OT@@QEBA_NPEAUhb_ot_apply_context_t@2@_N@Z 00000001800dc040     hb-ot-layout.obj
 0002:00031040       $unwind$?get_indexes@IndexArray@OT@@QEBAIIPEAI0@Z 00000001800dc040     hb-ot-layout.obj
 0002:00031058       $unwind$??$evaluate@UItemVarStoreInstancer@OT@@@Condition@OT@@QEBA_NPEBHIPEAUItemVarStoreInstancer@1@@Z 00000001800dc058     hb-ot-layout.obj
 0002:00031068       $chain$2$??$evaluate@UItemVarStoreInstancer@OT@@@Condition@OT@@QEBA_NPEBHIPEAUItemVarStoreInstancer@1@@Z 00000001800dc068     hb-ot-layout.obj
 0002:00031084       $chain$4$??$evaluate@UItemVarStoreInstancer@OT@@@Condition@OT@@QEBA_NPEBHIPEAUItemVarStoreInstancer@1@@Z 00000001800dc084     hb-ot-layout.obj
 0002:000310a0       $chain$5$??$evaluate@UItemVarStoreInstancer@OT@@@Condition@OT@@QEBA_NPEBHIPEAUItemVarStoreInstancer@1@@Z 00000001800dc0a0     hb-ot-layout.obj
 0002:000310b0       $unwind$?get_delta@HintingDevice@OT@@AEBAHIH@Z 00000001800dc0b0     hb-ot-layout.obj
 0002:000310c0       $chain$1$?get_delta@HintingDevice@OT@@AEBAHIH@Z 00000001800dc0c0     hb-ot-layout.obj
 0002:000310d8       $chain$2$?get_delta@HintingDevice@OT@@AEBAHIH@Z 00000001800dc0d8     hb-ot-layout.obj
 0002:000310ec       $chain$3$?get_delta@HintingDevice@OT@@AEBAHIH@Z 00000001800dc0ec     hb-ot-layout.obj
 0002:000310fc       $unwind$?get_glyph_props@accelerator_t@GDEF@OT@@QEBAII@Z 00000001800dc0fc     hb-ot-layout.obj
 0002:0003110c       $chain$3$?get_glyph_props@accelerator_t@GDEF@OT@@QEBAII@Z 00000001800dc10c     hb-ot-layout.obj
 0002:00031128       $chain$4$?get_glyph_props@accelerator_t@GDEF@OT@@QEBAII@Z 00000001800dc128     hb-ot-layout.obj
 0002:00031138       $unwind$?ligate_input@OT@@YA_NPEAUhb_ot_apply_context_t@1@IPEBIIII@Z 00000001800dc138     hb-ot-layout.obj
 0002:00031150       $unwind$?apply_lookup@OT@@YAXPEAUhb_ot_apply_context_t@1@IPEAIIQEBULookupRecord@1@I@Z 00000001800dc150     hb-ot-layout.obj
 0002:00031164       $chain$2$?apply_lookup@OT@@YAXPEAUhb_ot_apply_context_t@1@IPEAIIQEBULookupRecord@1@I@Z 00000001800dc164     hb-ot-layout.obj
 0002:00031180       $chain$3$?apply_lookup@OT@@YAXPEAUhb_ot_apply_context_t@1@IPEAIIQEBULookupRecord@1@I@Z 00000001800dc180     hb-ot-layout.obj
 0002:00031190       $chain$4$?apply_lookup@OT@@YAXPEAUhb_ot_apply_context_t@1@IPEAIIQEBULookupRecord@1@I@Z 00000001800dc190     hb-ot-layout.obj
 0002:000311ac       $unwind$?would_apply@?$ChainRuleSet@USmallTypes@Layout@OT@@@OT@@QEBA_NPEAUhb_would_apply_context_t@2@AEBUChainContextApplyLookupContext@2@@Z 00000001800dc1ac     hb-ot-layout.obj
 0002:000311ac       $unwind$?would_apply@?$RuleSet@USmallTypes@Layout@OT@@@OT@@QEBA_NPEAUhb_would_apply_context_t@2@AEBUContextApplyLookupContext@2@@Z 00000001800dc1ac     hb-ot-layout.obj
 0002:000311cc       $unwind$?apply@?$RuleSet@USmallTypes@Layout@OT@@@OT@@QEBA_NPEAUhb_ot_apply_context_t@2@AEBUContextApplyLookupContext@2@@Z 00000001800dc1cc     hb-ot-layout.obj
 0002:000311e4       $unwind$?apply@?$Rule@USmallTypes@Layout@OT@@@OT@@QEBA_NPEAUhb_ot_apply_context_t@2@AEBUContextApplyLookupContext@2@@Z 00000001800dc1e4     hb-ot-layout.obj
 0002:00031200       $chain$0$?apply@?$Rule@USmallTypes@Layout@OT@@@OT@@QEBA_NPEAUhb_ot_apply_context_t@2@AEBUContextApplyLookupContext@2@@Z 00000001800dc200     hb-ot-layout.obj
 0002:00031214       $chain$2$?apply@?$Rule@USmallTypes@Layout@OT@@@OT@@QEBA_NPEAUhb_ot_apply_context_t@2@AEBUContextApplyLookupContext@2@@Z 00000001800dc214     hb-ot-layout.obj
 0002:0003122c       $chain$3$?apply@?$Rule@USmallTypes@Layout@OT@@@OT@@QEBA_NPEAUhb_ot_apply_context_t@2@AEBUContextApplyLookupContext@2@@Z 00000001800dc22c     hb-ot-layout.obj
 0002:0003123c       $chain$4$?apply@?$Rule@USmallTypes@Layout@OT@@@OT@@QEBA_NPEAUhb_ot_apply_context_t@2@AEBUContextApplyLookupContext@2@@Z 00000001800dc23c     hb-ot-layout.obj
 0002:0003124c       $chain$5$?apply@?$Rule@USmallTypes@Layout@OT@@@OT@@QEBA_NPEAUhb_ot_apply_context_t@2@AEBUContextApplyLookupContext@2@@Z 00000001800dc24c     hb-ot-layout.obj
 0002:00031268       $unwind$?apply@ContextFormat3@OT@@QEBA_NPEAUhb_ot_apply_context_t@2@@Z 00000001800dc268     hb-ot-layout.obj
 0002:00031280       $chain$0$?apply@ContextFormat3@OT@@QEBA_NPEAUhb_ot_apply_context_t@2@@Z 00000001800dc280     hb-ot-layout.obj
 0002:00031294       $chain$2$?apply@ContextFormat3@OT@@QEBA_NPEAUhb_ot_apply_context_t@2@@Z 00000001800dc294     hb-ot-layout.obj
 0002:000312ac       $chain$4$?apply@ContextFormat3@OT@@QEBA_NPEAUhb_ot_apply_context_t@2@@Z 00000001800dc2ac     hb-ot-layout.obj
 0002:000312c4       $chain$5$?apply@ContextFormat3@OT@@QEBA_NPEAUhb_ot_apply_context_t@2@@Z 00000001800dc2c4     hb-ot-layout.obj
 0002:000312d4       $chain$6$?apply@ContextFormat3@OT@@QEBA_NPEAUhb_ot_apply_context_t@2@@Z 00000001800dc2d4     hb-ot-layout.obj
 0002:000312e4       $chain$7$?apply@ContextFormat3@OT@@QEBA_NPEAUhb_ot_apply_context_t@2@@Z 00000001800dc2e4     hb-ot-layout.obj
 0002:000312f4       $chain$8$?apply@ContextFormat3@OT@@QEBA_NPEAUhb_ot_apply_context_t@2@@Z 00000001800dc2f4     hb-ot-layout.obj
 0002:00031318       $unwind$?apply@?$ChainRuleSet@USmallTypes@Layout@OT@@@OT@@QEBA_NPEAUhb_ot_apply_context_t@2@AEBUChainContextApplyLookupContext@2@@Z 00000001800dc318     hb-ot-layout.obj
 0002:00031330       $unwind$?apply@?$ChainRule@USmallTypes@Layout@OT@@@OT@@QEBA_NPEAUhb_ot_apply_context_t@2@AEBUChainContextApplyLookupContext@2@@Z 00000001800dc330     hb-ot-layout.obj
 0002:00031348       $chain$0$?apply@?$ChainRule@USmallTypes@Layout@OT@@@OT@@QEBA_NPEAUhb_ot_apply_context_t@2@AEBUChainContextApplyLookupContext@2@@Z 00000001800dc348     hb-ot-layout.obj
 0002:0003135c       $chain$3$?apply@?$ChainRule@USmallTypes@Layout@OT@@@OT@@QEBA_NPEAUhb_ot_apply_context_t@2@AEBUChainContextApplyLookupContext@2@@Z 00000001800dc35c     hb-ot-layout.obj
 0002:00031378       $chain$4$?apply@?$ChainRule@USmallTypes@Layout@OT@@@OT@@QEBA_NPEAUhb_ot_apply_context_t@2@AEBUChainContextApplyLookupContext@2@@Z 00000001800dc378     hb-ot-layout.obj
 0002:0003138c       $chain$5$?apply@?$ChainRule@USmallTypes@Layout@OT@@@OT@@QEBA_NPEAUhb_ot_apply_context_t@2@AEBUChainContextApplyLookupContext@2@@Z 00000001800dc38c     hb-ot-layout.obj
 0002:0003139c       $chain$6$?apply@?$ChainRule@USmallTypes@Layout@OT@@@OT@@QEBA_NPEAUhb_ot_apply_context_t@2@AEBUChainContextApplyLookupContext@2@@Z 00000001800dc39c     hb-ot-layout.obj
 0002:000313ac       $chain$7$?apply@?$ChainRule@USmallTypes@Layout@OT@@@OT@@QEBA_NPEAUhb_ot_apply_context_t@2@AEBUChainContextApplyLookupContext@2@@Z 00000001800dc3ac     hb-ot-layout.obj
 0002:000313cc       $chain$1$?apply@ChainContextFormat3@OT@@QEBA_NPEAUhb_ot_apply_context_t@2@@Z 00000001800dc3cc     hb-ot-layout.obj
 0002:000313e4       $chain$2$?apply@ChainContextFormat3@OT@@QEBA_NPEAUhb_ot_apply_context_t@2@@Z 00000001800dc3e4     hb-ot-layout.obj
 0002:000313f8       $chain$4$?apply@ChainContextFormat3@OT@@QEBA_NPEAUhb_ot_apply_context_t@2@@Z 00000001800dc3f8     hb-ot-layout.obj
 0002:00031410       $chain$5$?apply@ChainContextFormat3@OT@@QEBA_NPEAUhb_ot_apply_context_t@2@@Z 00000001800dc410     hb-ot-layout.obj
 0002:00031424       $chain$6$?apply@ChainContextFormat3@OT@@QEBA_NPEAUhb_ot_apply_context_t@2@@Z 00000001800dc424     hb-ot-layout.obj
 0002:00031434       $chain$7$?apply@ChainContextFormat3@OT@@QEBA_NPEAUhb_ot_apply_context_t@2@@Z 00000001800dc434     hb-ot-layout.obj
 0002:00031444       $chain$8$?apply@ChainContextFormat3@OT@@QEBA_NPEAUhb_ot_apply_context_t@2@@Z 00000001800dc444     hb-ot-layout.obj
 0002:00031454       $chain$9$?apply@ChainContextFormat3@OT@@QEBA_NPEAUhb_ot_apply_context_t@2@@Z 00000001800dc454     hb-ot-layout.obj
 0002:00031478       $unwind$?apply@?$ChainContextFormat1_4@USmallTypes@Layout@OT@@@OT@@QEBA_NPEAUhb_ot_apply_context_t@2@@Z 00000001800dc478     hb-ot-layout.obj
 0002:00031490       $unwind$?get_lookup@GSUBGPOS@OT@@QEBAAEBULookup@2@I@Z 00000001800dc490     hb-ot-layout.obj
 0002:000314a0       $unwind$?find_variations_index@GSUBGPOS@OT@@QEBA_NPEBHIPEAIPEAUItemVarStoreInstancer@2@@Z 00000001800dc4a0     hb-ot-layout.obj
 0002:000314c0       $unwind$?get_feature_variation@GSUBGPOS@OT@@QEBAAEBUFeature@2@II@Z 00000001800dc4c0     hb-ot-layout.obj
 0002:000314cc       $unwind$?apply_value@ValueFormat@GPOS_impl@Layout@OT@@QEBA_NPEAUhb_ot_apply_context_t@4@PEBUValueBase@234@PEBU?$IntType@G$01@4@AEAUhb_glyph_position_t@@@Z 00000001800dc4cc     hb-ot-layout.obj
 0002:000314e8       $unwind$?sanitize_values_stride_unsafe@ValueFormat@GPOS_impl@Layout@OT@@QEBA_NPEAUhb_sanitize_context_t@@PEBUValueBase@234@PEBU?$IntType@G$01@4@II@Z 00000001800dc4e8     hb-ot-layout.obj
 0002:00031504       $unwind$?apply@SinglePosFormat2@GPOS_impl@Layout@OT@@QEBA_NPEAUhb_ot_apply_context_t@4@@Z 00000001800dc504     hb-ot-layout.obj
 0002:00031518       $unwind$?sanitize@?$PairSet@USmallTypes@Layout@OT@@@GPOS_impl@Layout@OT@@QEBA_NPEAUhb_sanitize_context_t@@PEBUsanitize_closure_t@1234@@Z 00000001800dc518     hb-ot-layout.obj
 0002:00031530       $unwind$?apply@?$PairSet@USmallTypes@Layout@OT@@@GPOS_impl@Layout@OT@@QEBA_NPEAUhb_ot_apply_context_t@4@PEBUValueFormat@234@I@Z 00000001800dc530     hb-ot-layout.obj
 0002:00031548       $unwind$?sanitize@?$PairPosFormat1_3@USmallTypes@Layout@OT@@@GPOS_impl@Layout@OT@@QEBA_NPEAUhb_sanitize_context_t@@@Z 00000001800dc548     hb-ot-layout.obj
 0002:00031564       $unwind$?_apply@?$PairPosFormat1_3@USmallTypes@Layout@OT@@@GPOS_impl@Layout@OT@@QEBA_NPEAUhb_ot_apply_context_t@4@_N@Z 00000001800dc564     hb-ot-layout.obj
 0002:0003157c       $chain$0$?_apply@?$PairPosFormat1_3@USmallTypes@Layout@OT@@@GPOS_impl@Layout@OT@@QEBA_NPEAUhb_ot_apply_context_t@4@_N@Z 00000001800dc57c     hb-ot-layout.obj
 0002:00031590       $chain$0$?sanitize@?$PairPosFormat2_4@USmallTypes@Layout@OT@@@GPOS_impl@Layout@OT@@QEBA_NPEAUhb_sanitize_context_t@@@Z 00000001800dc590     hb-ot-layout.obj
 0002:000315a4       $chain$2$?sanitize@?$PairPosFormat2_4@USmallTypes@Layout@OT@@@GPOS_impl@Layout@OT@@QEBA_NPEAUhb_sanitize_context_t@@@Z 00000001800dc5a4     hb-ot-layout.obj
 0002:000315b8       $chain$3$?sanitize@?$PairPosFormat2_4@USmallTypes@Layout@OT@@@GPOS_impl@Layout@OT@@QEBA_NPEAUhb_sanitize_context_t@@@Z 00000001800dc5b8     hb-ot-layout.obj
 0002:000315c8       $unwind$?cache_cost@?$PairPosFormat2_4@USmallTypes@Layout@OT@@@GPOS_impl@Layout@OT@@QEBAIXZ 00000001800dc5c8     hb-ot-layout.obj
 0002:000315d8       $unwind$?_apply@?$PairPosFormat2_4@USmallTypes@Layout@OT@@@GPOS_impl@Layout@OT@@QEBA_NPEAUhb_ot_apply_context_t@4@_N@Z 00000001800dc5d8     hb-ot-layout.obj
 0002:000315ec       $chain$0$?_apply@?$PairPosFormat2_4@USmallTypes@Layout@OT@@@GPOS_impl@Layout@OT@@QEBA_NPEAUhb_ot_apply_context_t@4@_N@Z 00000001800dc5ec     hb-ot-layout.obj
 0002:00031600       $unwind$?get_anchor@AnchorFormat2@GPOS_impl@Layout@OT@@QEBAXPEAUhb_ot_apply_context_t@4@IPEAM1@Z 00000001800dc600     hb-ot-layout.obj
 0002:00031614       $chain$0$?get_anchor@AnchorFormat2@GPOS_impl@Layout@OT@@QEBAXPEAUhb_ot_apply_context_t@4@IPEAM1@Z 00000001800dc614     hb-ot-layout.obj
 0002:00031628       $chain$1$?get_anchor@AnchorFormat2@GPOS_impl@Layout@OT@@QEBAXPEAUhb_ot_apply_context_t@4@IPEAM1@Z 00000001800dc628     hb-ot-layout.obj
 0002:00031638       $chain$0$?sanitize@Anchor@GPOS_impl@Layout@OT@@QEBA_NPEAUhb_sanitize_context_t@@@Z 00000001800dc638     hb-ot-layout.obj
 0002:0003164c       $chain$2$?sanitize@Anchor@GPOS_impl@Layout@OT@@QEBA_NPEAUhb_sanitize_context_t@@@Z 00000001800dc64c     hb-ot-layout.obj
 0002:00031660       $chain$3$?sanitize@Anchor@GPOS_impl@Layout@OT@@QEBA_NPEAUhb_sanitize_context_t@@@Z 00000001800dc660     hb-ot-layout.obj
 0002:00031670       $unwind$?reverse_cursive_minor_offset@GPOS_impl@Layout@OT@@YAXPEAUhb_glyph_position_t@@IW4hb_direction_t@@I@Z 00000001800dc670     hb-ot-layout.obj
 0002:00031684       $chain$0$?reverse_cursive_minor_offset@GPOS_impl@Layout@OT@@YAXPEAUhb_glyph_position_t@@IW4hb_direction_t@@I@Z 00000001800dc684     hb-ot-layout.obj
 0002:00031698       $chain$1$?reverse_cursive_minor_offset@GPOS_impl@Layout@OT@@YAXPEAUhb_glyph_position_t@@IW4hb_direction_t@@I@Z 00000001800dc698     hb-ot-layout.obj
 0002:000316a8       $unwind$?sanitize@CursivePosFormat1@GPOS_impl@Layout@OT@@QEBA_NPEAUhb_sanitize_context_t@@@Z 00000001800dc6a8     hb-ot-layout.obj
 0002:000316b8       $chain$2$?sanitize@CursivePosFormat1@GPOS_impl@Layout@OT@@QEBA_NPEAUhb_sanitize_context_t@@@Z 00000001800dc6b8     hb-ot-layout.obj
 0002:000316d4       $chain$4$?sanitize@CursivePosFormat1@GPOS_impl@Layout@OT@@QEBA_NPEAUhb_sanitize_context_t@@@Z 00000001800dc6d4     hb-ot-layout.obj
 0002:000316f0       $chain$5$?sanitize@CursivePosFormat1@GPOS_impl@Layout@OT@@QEBA_NPEAUhb_sanitize_context_t@@@Z 00000001800dc6f0     hb-ot-layout.obj
 0002:00031700       $unwind$?apply@CursivePosFormat1@GPOS_impl@Layout@OT@@QEBA_NPEAUhb_ot_apply_context_t@4@@Z 00000001800dc700     hb-ot-layout.obj
 0002:0003171c       $chain$5$?apply@CursivePosFormat1@GPOS_impl@Layout@OT@@QEBA_NPEAUhb_ot_apply_context_t@4@@Z 00000001800dc71c     hb-ot-layout.obj
 0002:00031740       $chain$6$?apply@CursivePosFormat1@GPOS_impl@Layout@OT@@QEBA_NPEAUhb_ot_apply_context_t@4@@Z 00000001800dc740     hb-ot-layout.obj
 0002:00031750       $unwind$?apply@MarkArray@GPOS_impl@Layout@OT@@QEBA_NPEAUhb_ot_apply_context_t@4@IIAEBUAnchorMatrix@234@II@Z 00000001800dc750     hb-ot-layout.obj
 0002:0003176c       $chain$6$?apply@MarkArray@GPOS_impl@Layout@OT@@QEBA_NPEAUhb_ot_apply_context_t@4@IIAEBUAnchorMatrix@234@II@Z 00000001800dc76c     hb-ot-layout.obj
 0002:0003178c       $chain$7$?apply@MarkArray@GPOS_impl@Layout@OT@@QEBA_NPEAUhb_ot_apply_context_t@4@IIAEBUAnchorMatrix@234@II@Z 00000001800dc78c     hb-ot-layout.obj
 0002:0003179c       $unwind$?apply@?$MarkBasePosFormat1_2@USmallTypes@Layout@OT@@@GPOS_impl@Layout@OT@@QEBA_NPEAUhb_ot_apply_context_t@4@@Z 00000001800dc79c     hb-ot-layout.obj
 0002:000317b8       $unwind$?sanitize@?$MarkLigPosFormat1_2@USmallTypes@Layout@OT@@@GPOS_impl@Layout@OT@@QEBA_NPEAUhb_sanitize_context_t@@@Z 00000001800dc7b8     hb-ot-layout.obj
 0002:000317cc       $unwind$?apply@?$MarkLigPosFormat1_2@USmallTypes@Layout@OT@@@GPOS_impl@Layout@OT@@QEBA_NPEAUhb_ot_apply_context_t@4@@Z 00000001800dc7cc     hb-ot-layout.obj
 0002:000317e8       $unwind$?apply@?$MarkMarkPosFormat1_2@USmallTypes@Layout@OT@@@GPOS_impl@Layout@OT@@QEBA_NPEAUhb_ot_apply_context_t@4@@Z 00000001800dc7e8     hb-ot-layout.obj
 0002:00031804       $unwind$?propagate_attachment_offsets@Layout@OT@@YAXPEAUhb_glyph_position_t@@IIW4hb_direction_t@@I@Z 00000001800dc804     hb-ot-layout.obj
 0002:00031818       $chain$0$?propagate_attachment_offsets@Layout@OT@@YAXPEAUhb_glyph_position_t@@IIW4hb_direction_t@@I@Z 00000001800dc818     hb-ot-layout.obj
 0002:0003182c       $chain$1$?propagate_attachment_offsets@Layout@OT@@YAXPEAUhb_glyph_position_t@@IIW4hb_direction_t@@I@Z 00000001800dc82c     hb-ot-layout.obj
 0002:0003183c       $unwind$?position_finish_offsets@GPOS@Layout@OT@@SAXPEAUhb_font_t@@PEAUhb_buffer_t@@@Z 00000001800dc83c     hb-ot-layout.obj
 0002:0003184c       $chain$0$?position_finish_offsets@GPOS@Layout@OT@@SAXPEAUhb_font_t@@PEAUhb_buffer_t@@@Z 00000001800dc84c     hb-ot-layout.obj
 0002:00031860       $chain$2$?position_finish_offsets@GPOS@Layout@OT@@SAXPEAUhb_font_t@@PEAUhb_buffer_t@@@Z 00000001800dc860     hb-ot-layout.obj
 0002:00031878       $chain$3$?position_finish_offsets@GPOS@Layout@OT@@SAXPEAUhb_font_t@@PEAUhb_buffer_t@@@Z 00000001800dc878     hb-ot-layout.obj
 0002:00031888       $chain$4$?position_finish_offsets@GPOS@Layout@OT@@SAXPEAUhb_font_t@@PEAUhb_buffer_t@@@Z 00000001800dc888     hb-ot-layout.obj
 0002:00031898       $chain$5$?position_finish_offsets@GPOS@Layout@OT@@SAXPEAUhb_font_t@@PEAUhb_buffer_t@@@Z 00000001800dc898     hb-ot-layout.obj
 0002:000318ac       $chain$6$?position_finish_offsets@GPOS@Layout@OT@@SAXPEAUhb_font_t@@PEAUhb_buffer_t@@@Z 00000001800dc8ac     hb-ot-layout.obj
 0002:000318bc       $unwind$??$dispatch_recurse_func@Uhb_ot_apply_context_t@OT@@@PosLookup@GPOS_impl@Layout@OT@@SA_NPEAUhb_ot_apply_context_t@3@I@Z 00000001800dc8bc     hb-ot-layout.obj
 0002:000318bc       $unwind$??$dispatch_recurse_func@Uhb_ot_apply_context_t@OT@@@SubstLookup@GSUB_impl@Layout@OT@@SA_NPEAUhb_ot_apply_context_t@3@I@Z 00000001800dc8bc     hb-ot-layout.obj
 0002:000318d8       $unwind$?apply@?$KerxTable@UKernAAT@OT@@@AAT@@QEBA_NPEAUhb_aat_apply_context_t@2@AEBUkern_accelerator_data_t@2@@Z 00000001800dc8d8     hb-ot-layout.obj
 0002:000318d8       $unwind$?apply@?$KerxTable@UKernOT@OT@@@AAT@@QEBA_NPEAUhb_aat_apply_context_t@2@AEBUkern_accelerator_data_t@2@@Z 00000001800dc8d8     hb-ot-layout.obj
 0002:000318f0       $unwind$??0accelerator_t@kern@OT@@QEAA@PEAUhb_face_t@@@Z 00000001800dc8f0     hb-ot-layout.obj
 0002:00031904       $chain$0$??0accelerator_t@kern@OT@@QEAA@PEAUhb_face_t@@@Z 00000001800dc904     hb-ot-layout.obj
 0002:00031918       $chain$1$??0accelerator_t@kern@OT@@QEAA@PEAUhb_face_t@@@Z 00000001800dc918     hb-ot-layout.obj
 0002:0003192c       $chain$2$??0accelerator_t@kern@OT@@QEAA@PEAUhb_face_t@@@Z 00000001800dc92c     hb-ot-layout.obj
 0002:0003193c       $chain$3$??0accelerator_t@kern@OT@@QEAA@PEAUhb_face_t@@@Z 00000001800dc93c     hb-ot-layout.obj
 0002:0003194c       $unwind$?apply@?$SingleSubstFormat2_4@USmallTypes@Layout@OT@@@GSUB_impl@Layout@OT@@QEBA_NPEAUhb_ot_apply_context_t@4@@Z 00000001800dc94c     hb-ot-layout.obj
 0002:00031960       $unwind$?apply@?$Sequence@USmallTypes@Layout@OT@@@GSUB_impl@Layout@OT@@QEBA_NPEAUhb_ot_apply_context_t@4@@Z 00000001800dc960     hb-ot-layout.obj
 0002:0003197c       $chain$1$?apply@?$Sequence@USmallTypes@Layout@OT@@@GSUB_impl@Layout@OT@@QEBA_NPEAUhb_ot_apply_context_t@4@@Z 00000001800dc97c     hb-ot-layout.obj
 0002:00031994       $chain$2$?apply@?$Sequence@USmallTypes@Layout@OT@@@GSUB_impl@Layout@OT@@QEBA_NPEAUhb_ot_apply_context_t@4@@Z 00000001800dc994     hb-ot-layout.obj
 0002:000319a8       $chain$3$?apply@?$Sequence@USmallTypes@Layout@OT@@@GSUB_impl@Layout@OT@@QEBA_NPEAUhb_ot_apply_context_t@4@@Z 00000001800dc9a8     hb-ot-layout.obj
 0002:000319b8       $chain$4$?apply@?$Sequence@USmallTypes@Layout@OT@@@GSUB_impl@Layout@OT@@QEBA_NPEAUhb_ot_apply_context_t@4@@Z 00000001800dc9b8     hb-ot-layout.obj
 0002:000319c8       $unwind$?apply@?$AlternateSet@USmallTypes@Layout@OT@@@GSUB_impl@Layout@OT@@QEBA_NPEAUhb_ot_apply_context_t@4@@Z 00000001800dc9c8     hb-ot-layout.obj
 0002:000319d8       $unwind$?apply@?$Ligature@USmallTypes@Layout@OT@@@GSUB_impl@Layout@OT@@QEBA_NPEAUhb_ot_apply_context_t@4@@Z 00000001800dc9d8     hb-ot-layout.obj
 0002:000319fc       $unwind$?apply@?$LigatureSet@USmallTypes@Layout@OT@@@GSUB_impl@Layout@OT@@QEBA_NPEAUhb_ot_apply_context_t@4@@Z 00000001800dc9fc     hb-ot-layout.obj
 0002:00031a14       $unwind$?would_apply@?$LigatureSubstFormat1_2@USmallTypes@Layout@OT@@@GSUB_impl@Layout@OT@@QEBA_NPEAUhb_would_apply_context_t@4@@Z 00000001800dca14     hb-ot-layout.obj
 0002:00031a28       $chain$1$?would_apply@?$LigatureSubstFormat1_2@USmallTypes@Layout@OT@@@GSUB_impl@Layout@OT@@QEBA_NPEAUhb_would_apply_context_t@4@@Z 00000001800dca28     hb-ot-layout.obj
 0002:00031a40       $chain$2$?would_apply@?$LigatureSubstFormat1_2@USmallTypes@Layout@OT@@@GSUB_impl@Layout@OT@@QEBA_NPEAUhb_would_apply_context_t@4@@Z 00000001800dca40     hb-ot-layout.obj
 0002:00031a50       $unwind$?apply@ReverseChainSingleSubstFormat1@GSUB_impl@Layout@OT@@QEBA_NPEAUhb_ot_apply_context_t@4@@Z 00000001800dca50     hb-ot-layout.obj
 0002:00031a70       $unwind$?_hb_ot_layout_set_glyph_props@@YAXPEAUhb_font_t@@PEAUhb_buffer_t@@@Z 00000001800dca70     hb-ot-layout.obj
 0002:00031a7c       $chain$4$?_hb_ot_layout_set_glyph_props@@YAXPEAUhb_font_t@@PEAUhb_buffer_t@@@Z 00000001800dca7c     hb-ot-layout.obj
 0002:00031aa0       $chain$5$?_hb_ot_layout_set_glyph_props@@YAXPEAUhb_font_t@@PEAUhb_buffer_t@@@Z 00000001800dcaa0     hb-ot-layout.obj
 0002:00031ab0       $unwind$?apply_forward@@YA_NPEAUhb_ot_apply_context_t@OT@@AEBUhb_ot_layout_lookup_accelerator_t@2@I@Z 00000001800dcab0     hb-ot-layout.obj
 0002:00031ac0       $chain$2$?apply_forward@@YA_NPEAUhb_ot_apply_context_t@OT@@AEBUhb_ot_layout_lookup_accelerator_t@2@I@Z 00000001800dcac0     hb-ot-layout.obj
 0002:00031adc       $chain$3$?apply_forward@@YA_NPEAUhb_ot_apply_context_t@OT@@AEBUhb_ot_layout_lookup_accelerator_t@2@I@Z 00000001800dcadc     hb-ot-layout.obj
 0002:00031af0       $chain$4$?apply_forward@@YA_NPEAUhb_ot_apply_context_t@OT@@AEBUhb_ot_layout_lookup_accelerator_t@2@I@Z 00000001800dcaf0     hb-ot-layout.obj
 0002:00031b00       $chain$5$?apply_forward@@YA_NPEAUhb_ot_apply_context_t@OT@@AEBUhb_ot_layout_lookup_accelerator_t@2@I@Z 00000001800dcb00     hb-ot-layout.obj
 0002:00031b10       $unwind$?apply_backward@@YA_NPEAUhb_ot_apply_context_t@OT@@AEBUhb_ot_layout_lookup_accelerator_t@2@I@Z 00000001800dcb10     hb-ot-layout.obj
 0002:00031b28       $unwind$??$apply@UGSUBProxy@@@hb_ot_map_t@@QEBAXAEBUGSUBProxy@@PEBUhb_ot_shape_plan_t@@PEAUhb_font_t@@PEAUhb_buffer_t@@@Z 00000001800dcb28     hb-ot-layout.obj
 0002:00031b48       $unwind$??$apply@UGPOSProxy@@@hb_ot_map_t@@QEBAXAEBUGPOSProxy@@PEBUhb_ot_shape_plan_t@@PEAUhb_font_t@@PEAUhb_buffer_t@@@Z 00000001800dcb48     hb-ot-layout.obj
 0002:00031b68       $chain$0$??$apply_string@UGSUBProxy@@@@YA_NPEAUhb_ot_apply_context_t@OT@@AEBUSubstLookup@GSUB_impl@Layout@1@AEBUhb_ot_layout_lookup_accelerator_t@1@@Z 00000001800dcb68     hb-ot-layout.obj
 0002:00031b7c       $chain$2$??$apply_string@UGSUBProxy@@@@YA_NPEAUhb_ot_apply_context_t@OT@@AEBUSubstLookup@GSUB_impl@Layout@1@AEBUhb_ot_layout_lookup_accelerator_t@1@@Z 00000001800dcb7c     hb-ot-layout.obj
 0002:00031b90       $chain$3$??$apply_string@UGSUBProxy@@@@YA_NPEAUhb_ot_apply_context_t@OT@@AEBUSubstLookup@GSUB_impl@Layout@1@AEBUhb_ot_layout_lookup_accelerator_t@1@@Z 00000001800dcb90     hb-ot-layout.obj
 0002:00031ba0       $unwind$??$create@UPosLookup@GPOS_impl@Layout@OT@@@hb_ot_layout_lookup_accelerator_t@OT@@SAPEAU01@AEBUPosLookup@GPOS_impl@Layout@1@@Z 00000001800dcba0     hb-ot-layout.obj
 0002:00031ba0       $unwind$??$create@USubstLookup@GSUB_impl@Layout@OT@@@hb_ot_layout_lookup_accelerator_t@OT@@SAPEAU01@AEBUSubstLookup@GSUB_impl@Layout@1@@Z 00000001800dcba0     hb-ot-layout.obj
 0002:00031bb0       $chain$4$??$create@USubstLookup@GSUB_impl@Layout@OT@@@hb_ot_layout_lookup_accelerator_t@OT@@SAPEAU01@AEBUSubstLookup@GSUB_impl@Layout@1@@Z 00000001800dcbb0     hb-ot-layout.obj
 0002:00031bd0       $chain$5$??$create@USubstLookup@GSUB_impl@Layout@OT@@@hb_ot_layout_lookup_accelerator_t@OT@@SAPEAU01@AEBUSubstLookup@GSUB_impl@Layout@1@@Z 00000001800dcbd0     hb-ot-layout.obj
 0002:00031be4       $chain$6$??$create@USubstLookup@GSUB_impl@Layout@OT@@@hb_ot_layout_lookup_accelerator_t@OT@@SAPEAU01@AEBUSubstLookup@GSUB_impl@Layout@1@@Z 00000001800dcbe4     hb-ot-layout.obj
 0002:00031bf4       $chain$0$??$collect_glyphs@Uhb_bit_set_t@@@?$KernSubTable@UKernAATSubTableHeader@OT@@@OT@@QEBAXAEAUhb_bit_set_t@@0I@Z 00000001800dcbf4     hb-ot-layout.obj
 0002:00031c08       $chain$1$??$collect_glyphs@Uhb_bit_set_t@@@?$KernSubTable@UKernAATSubTableHeader@OT@@@OT@@QEBAXAEAUhb_bit_set_t@@0I@Z 00000001800dcc08     hb-ot-layout.obj
 0002:00031c18       $chain$0$??$collect_glyphs@Uhb_bit_set_t@@@?$KernSubTable@UKernOTSubTableHeader@OT@@@OT@@QEBAXAEAUhb_bit_set_t@@0I@Z 00000001800dcc18     hb-ot-layout.obj
 0002:00031c2c       $chain$1$??$collect_glyphs@Uhb_bit_set_t@@@?$KernSubTable@UKernOTSubTableHeader@OT@@@OT@@QEBAXAEAUhb_bit_set_t@@0I@Z 00000001800dcc2c     hb-ot-layout.obj
 0002:00031c3c       $chain$4$??$create@UPosLookup@GPOS_impl@Layout@OT@@@hb_ot_layout_lookup_accelerator_t@OT@@SAPEAU01@AEBUPosLookup@GPOS_impl@Layout@1@@Z 00000001800dcc3c     hb-ot-layout.obj
 0002:00031c5c       $chain$5$??$create@UPosLookup@GPOS_impl@Layout@OT@@@hb_ot_layout_lookup_accelerator_t@OT@@SAPEAU01@AEBUPosLookup@GPOS_impl@Layout@1@@Z 00000001800dcc5c     hb-ot-layout.obj
 0002:00031c70       $chain$6$??$create@UPosLookup@GPOS_impl@Layout@OT@@@hb_ot_layout_lookup_accelerator_t@OT@@SAPEAU01@AEBUPosLookup@GPOS_impl@Layout@1@@Z 00000001800dcc70     hb-ot-layout.obj
 0002:00031c80       $unwind$??$would_match_input@U?$IntType@G$01@OT@@@OT@@YA_NPEAUhb_would_apply_context_t@0@IQEBU?$IntType@G$01@0@P6A_NAEAUhb_glyph_info_t@@IPEBX@Z3@Z 00000001800dcc80     hb-ot-layout.obj
 0002:00031c9c       $chain$4$??$dispatch@U?$List16OfOffsetTo@UPosLookup@GPOS_impl@Layout@OT@@U?$IntType@G$01@4@@OT@@$$V@hb_sanitize_context_t@@QEAA_NAEBU?$List16OfOffsetTo@UPosLookup@GPOS_impl@Layout@OT@@U?$IntType@G$01@4@@OT@@@Z 00000001800dcc9c     hb-ot-layout.obj
 0002:00031cc0       $chain$6$??$dispatch@U?$List16OfOffsetTo@UPosLookup@GPOS_impl@Layout@OT@@U?$IntType@G$01@4@@OT@@$$V@hb_sanitize_context_t@@QEAA_NAEBU?$List16OfOffsetTo@UPosLookup@GPOS_impl@Layout@OT@@U?$IntType@G$01@4@@OT@@@Z 00000001800dccc0     hb-ot-layout.obj
 0002:00031ce4       $unwind$??$collect_coverage@Uhb_set_digest_t@@@Coverage@Common@Layout@OT@@QEBA_NPEAUhb_set_digest_t@@@Z 00000001800dcce4     hb-ot-layout.obj
 0002:00031cf0       $unwind$??$collect_glyphs@Uhb_bit_set_t@@@?$ClassTable@U?$IntType@G$01@OT@@@AAT@@QEBAXAEAUhb_bit_set_t@@I@Z 00000001800dccf0     hb-ot-layout.obj
 0002:00031d00       $chain$1$??$collect_glyphs@Uhb_bit_set_t@@@?$ClassTable@U?$IntType@G$01@OT@@@AAT@@QEBAXAEAUhb_bit_set_t@@I@Z 00000001800dcd00     hb-ot-layout.obj
 0002:00031d18       $chain$2$??$collect_glyphs@Uhb_bit_set_t@@@?$ClassTable@U?$IntType@G$01@OT@@@AAT@@QEBAXAEAUhb_bit_set_t@@I@Z 00000001800dcd18     hb-ot-layout.obj
 0002:00031d28       $unwind$??$dispatch@Uhb_would_apply_context_t@OT@@$$V@Context@OT@@QEBA_NPEAUhb_would_apply_context_t@1@@Z 00000001800dcd28     hb-ot-layout.obj
 0002:00031d3c       $chain$0$??$dispatch@Uhb_would_apply_context_t@OT@@$$V@Context@OT@@QEBA_NPEAUhb_would_apply_context_t@1@@Z 00000001800dcd3c     hb-ot-layout.obj
 0002:00031d50       $chain$1$??$dispatch@Uhb_would_apply_context_t@OT@@$$V@Context@OT@@QEBA_NPEAUhb_would_apply_context_t@1@@Z 00000001800dcd50     hb-ot-layout.obj
 0002:00031d60       $unwind$??$dispatch@Uhb_would_apply_context_t@OT@@$$V@ChainContext@OT@@QEBA_NPEAUhb_would_apply_context_t@1@@Z 00000001800dcd60     hb-ot-layout.obj
 0002:00031d70       $chain$2$??$dispatch@Uhb_would_apply_context_t@OT@@$$V@ChainContext@OT@@QEBA_NPEAUhb_would_apply_context_t@1@@Z 00000001800dcd70     hb-ot-layout.obj
 0002:00031d8c       $chain$3$??$dispatch@Uhb_would_apply_context_t@OT@@$$V@ChainContext@OT@@QEBA_NPEAUhb_would_apply_context_t@1@@Z 00000001800dcd8c     hb-ot-layout.obj
 0002:00031d9c       $unwind$??$dispatch@Uhb_sanitize_context_t@@$$V@?$KernSubTable@UKernAATSubTableHeader@OT@@@OT@@QEBA_NPEAUhb_sanitize_context_t@@@Z 00000001800dcd9c     hb-ot-layout.obj
 0002:00031d9c       $unwind$??$dispatch@Uhb_sanitize_context_t@@$$V@?$KernSubTable@UKernOTSubTableHeader@OT@@@OT@@QEBA_NPEAUhb_sanitize_context_t@@@Z 00000001800dcd9c     hb-ot-layout.obj
 0002:00031da8       $chain$1$??$dispatch@Uhb_sanitize_context_t@@$$V@?$KernSubTable@UKernAATSubTableHeader@OT@@@OT@@QEBA_NPEAUhb_sanitize_context_t@@@Z 00000001800dcda8     hb-ot-layout.obj
 0002:00031dc0       $chain$3$??$dispatch@Uhb_sanitize_context_t@@$$V@?$KernSubTable@UKernAATSubTableHeader@OT@@@OT@@QEBA_NPEAUhb_sanitize_context_t@@@Z 00000001800dcdc0     hb-ot-layout.obj
 0002:00031dd8       $chain$4$??$dispatch@Uhb_sanitize_context_t@@$$V@?$KernSubTable@UKernAATSubTableHeader@OT@@@OT@@QEBA_NPEAUhb_sanitize_context_t@@@Z 00000001800dcdd8     hb-ot-layout.obj
 0002:00031dec       $chain$6$??$dispatch@Uhb_sanitize_context_t@@$$V@?$KernSubTable@UKernAATSubTableHeader@OT@@@OT@@QEBA_NPEAUhb_sanitize_context_t@@@Z 00000001800dcdec     hb-ot-layout.obj
 0002:00031e00       $chain$7$??$dispatch@Uhb_sanitize_context_t@@$$V@?$KernSubTable@UKernAATSubTableHeader@OT@@@OT@@QEBA_NPEAUhb_sanitize_context_t@@@Z 00000001800dce00     hb-ot-layout.obj
 0002:00031e10       $chain$8$??$dispatch@Uhb_sanitize_context_t@@$$V@?$KernSubTable@UKernAATSubTableHeader@OT@@@OT@@QEBA_NPEAUhb_sanitize_context_t@@@Z 00000001800dce10     hb-ot-layout.obj
 0002:00031e20       $chain$1$??$dispatch@Uhb_sanitize_context_t@@$$V@?$KernSubTable@UKernOTSubTableHeader@OT@@@OT@@QEBA_NPEAUhb_sanitize_context_t@@@Z 00000001800dce20     hb-ot-layout.obj
 0002:00031e38       $chain$3$??$dispatch@Uhb_sanitize_context_t@@$$V@?$KernSubTable@UKernOTSubTableHeader@OT@@@OT@@QEBA_NPEAUhb_sanitize_context_t@@@Z 00000001800dce38     hb-ot-layout.obj
 0002:00031e50       $chain$4$??$dispatch@Uhb_sanitize_context_t@@$$V@?$KernSubTable@UKernOTSubTableHeader@OT@@@OT@@QEBA_NPEAUhb_sanitize_context_t@@@Z 00000001800dce50     hb-ot-layout.obj
 0002:00031e64       $chain$6$??$dispatch@Uhb_sanitize_context_t@@$$V@?$KernSubTable@UKernOTSubTableHeader@OT@@@OT@@QEBA_NPEAUhb_sanitize_context_t@@@Z 00000001800dce64     hb-ot-layout.obj
 0002:00031e78       $chain$7$??$dispatch@Uhb_sanitize_context_t@@$$V@?$KernSubTable@UKernOTSubTableHeader@OT@@@OT@@QEBA_NPEAUhb_sanitize_context_t@@@Z 00000001800dce78     hb-ot-layout.obj
 0002:00031e88       $chain$8$??$dispatch@Uhb_sanitize_context_t@@$$V@?$KernSubTable@UKernOTSubTableHeader@OT@@@OT@@QEBA_NPEAUhb_sanitize_context_t@@@Z 00000001800dce88     hb-ot-layout.obj
 0002:00031e98       $unwind$??$dispatch@Uhb_accelerate_subtables_context_t@OT@@$$V@ChainContext@OT@@QEBA?AUhb_empty_t@@PEAUhb_accelerate_subtables_context_t@1@@Z 00000001800dce98     hb-ot-layout.obj
 0002:00031eac       $unwind$?kern@?$hb_kern_machine_t@U?$KernSubTableFormat3@UKernAATSubTableHeader@OT@@@OT@@@OT@@QEBAXPEAUhb_font_t@@PEAUhb_buffer_t@@I_N@Z 00000001800dceac     hb-ot-layout.obj
 0002:00031eac       $unwind$?kern@?$hb_kern_machine_t@U?$KernSubTableFormat3@UKernOTSubTableHeader@OT@@@OT@@@OT@@QEBAXPEAUhb_font_t@@PEAUhb_buffer_t@@I_N@Z 00000001800dceac     hb-ot-layout.obj
 0002:00031ec8       $chain$1$?kern@?$hb_kern_machine_t@U?$KernSubTableFormat3@UKernAATSubTableHeader@OT@@@OT@@@OT@@QEBAXPEAUhb_font_t@@PEAUhb_buffer_t@@I_N@Z 00000001800dcec8     hb-ot-layout.obj
 0002:00031ee0       $chain$2$?kern@?$hb_kern_machine_t@U?$KernSubTableFormat3@UKernAATSubTableHeader@OT@@@OT@@@OT@@QEBAXPEAUhb_font_t@@PEAUhb_buffer_t@@I_N@Z 00000001800dcee0     hb-ot-layout.obj
 0002:00031ef4       $chain$3$?kern@?$hb_kern_machine_t@U?$KernSubTableFormat3@UKernAATSubTableHeader@OT@@@OT@@@OT@@QEBAXPEAUhb_font_t@@PEAUhb_buffer_t@@I_N@Z 00000001800dcef4     hb-ot-layout.obj
 0002:00031f04       $chain$4$?kern@?$hb_kern_machine_t@U?$KernSubTableFormat3@UKernAATSubTableHeader@OT@@@OT@@@OT@@QEBAXPEAUhb_font_t@@PEAUhb_buffer_t@@I_N@Z 00000001800dcf04     hb-ot-layout.obj
 0002:00031f14       $chain$0$?kern@?$hb_kern_machine_t@Uaccelerator_t@?$KerxSubTableFormat2@UKernAATSubTableHeader@OT@@@AAT@@@OT@@QEBAXPEAUhb_font_t@@PEAUhb_buffer_t@@I_N@Z 00000001800dcf14     hb-ot-layout.obj
 0002:00031f28       $chain$3$?kern@?$hb_kern_machine_t@Uaccelerator_t@?$KerxSubTableFormat2@UKernAATSubTableHeader@OT@@@AAT@@@OT@@QEBAXPEAUhb_font_t@@PEAUhb_buffer_t@@I_N@Z 00000001800dcf28     hb-ot-layout.obj
 0002:00031f44       $chain$4$?kern@?$hb_kern_machine_t@Uaccelerator_t@?$KerxSubTableFormat2@UKernAATSubTableHeader@OT@@@AAT@@@OT@@QEBAXPEAUhb_font_t@@PEAUhb_buffer_t@@I_N@Z 00000001800dcf44     hb-ot-layout.obj
 0002:00031f54       $chain$5$?kern@?$hb_kern_machine_t@Uaccelerator_t@?$KerxSubTableFormat2@UKernAATSubTableHeader@OT@@@AAT@@@OT@@QEBAXPEAUhb_font_t@@PEAUhb_buffer_t@@I_N@Z 00000001800dcf54     hb-ot-layout.obj
 0002:00031f64       $unwind$?transition@driver_context_t@?$KerxSubTableFormat1@UKernAATSubTableHeader@OT@@@AAT@@QEAAXPEAUhb_buffer_t@@PEAU?$StateTableDriver@UObsoleteTypes@AAT@@XW4Flags@?$KerxSubTableFormat1@UKernAATSubTableHeader@OT@@@2@@3@AEBU?$Entry@X@3@@Z 00000001800dcf64     hb-ot-layout.obj
 0002:00031f64       $unwind$?transition@driver_context_t@?$KerxSubTableFormat1@UKernOTSubTableHeader@OT@@@AAT@@QEAAXPEAUhb_buffer_t@@PEAU?$StateTableDriver@UObsoleteTypes@AAT@@XW4Flags@?$KerxSubTableFormat1@UKernOTSubTableHeader@OT@@@2@@3@AEBU?$Entry@X@3@@Z 00000001800dcf64     hb-ot-layout.obj
 0002:00031f78       $chain$0$?transition@driver_context_t@?$KerxSubTableFormat1@UKernAATSubTableHeader@OT@@@AAT@@QEAAXPEAUhb_buffer_t@@PEAU?$StateTableDriver@UObsoleteTypes@AAT@@XW4Flags@?$KerxSubTableFormat1@UKernAATSubTableHeader@OT@@@2@@3@AEBU?$Entry@X@3@@Z 00000001800dcf78     hb-ot-layout.obj
 0002:00031f8c       $chain$1$?transition@driver_context_t@?$KerxSubTableFormat1@UKernAATSubTableHeader@OT@@@AAT@@QEAAXPEAUhb_buffer_t@@PEAU?$StateTableDriver@UObsoleteTypes@AAT@@XW4Flags@?$KerxSubTableFormat1@UKernAATSubTableHeader@OT@@@2@@3@AEBU?$Entry@X@3@@Z 00000001800dcf8c     hb-ot-layout.obj
 0002:00031f9c       $unwind$??$drive@Udriver_context_t@?$KerxSubTableFormat1@UKernAATSubTableHeader@OT@@@AAT@@@?$StateTableDriver@UObsoleteTypes@AAT@@XW4Flags@?$KerxSubTableFormat1@UKernAATSubTableHeader@OT@@@2@@AAT@@QEAAXPEAUdriver_context_t@?$KerxSubTableFormat1@UKernAATSubTableHeader@OT@@@1@PEAUhb_aat_apply_context_t@1@@Z 00000001800dcf9c     hb-ot-layout.obj
 0002:00031f9c       $unwind$??$drive@Udriver_context_t@?$KerxSubTableFormat1@UKernOTSubTableHeader@OT@@@AAT@@@?$StateTableDriver@UObsoleteTypes@AAT@@XW4Flags@?$KerxSubTableFormat1@UKernOTSubTableHeader@OT@@@2@@AAT@@QEAAXPEAUdriver_context_t@?$KerxSubTableFormat1@UKernOTSubTableHeader@OT@@@1@PEAUhb_aat_apply_context_t@1@@Z 00000001800dcf9c     hb-ot-layout.obj
 0002:00031fac       $chain$3$??$drive@Udriver_context_t@?$KerxSubTableFormat1@UKernAATSubTableHeader@OT@@@AAT@@@?$StateTableDriver@UObsoleteTypes@AAT@@XW4Flags@?$KerxSubTableFormat1@UKernAATSubTableHeader@OT@@@2@@AAT@@QEAAXPEAUdriver_context_t@?$KerxSubTableFormat1@UKernAATSubTableHeader@OT@@@1@PEAUhb_aat_apply_context_t@1@@Z 00000001800dcfac     hb-ot-layout.obj
 0002:00031fcc       $chain$4$??$drive@Udriver_context_t@?$KerxSubTableFormat1@UKernAATSubTableHeader@OT@@@AAT@@@?$StateTableDriver@UObsoleteTypes@AAT@@XW4Flags@?$KerxSubTableFormat1@UKernAATSubTableHeader@OT@@@2@@AAT@@QEAAXPEAUdriver_context_t@?$KerxSubTableFormat1@UKernAATSubTableHeader@OT@@@1@PEAUhb_aat_apply_context_t@1@@Z 00000001800dcfcc     hb-ot-layout.obj
 0002:00031fdc       $chain$0$?kern@?$hb_kern_machine_t@Uaccelerator_t@?$KerxSubTableFormat0@UKernAATSubTableHeader@OT@@@AAT@@@OT@@QEBAXPEAUhb_font_t@@PEAUhb_buffer_t@@I_N@Z 00000001800dcfdc     hb-ot-layout.obj
 0002:00031ff0       $chain$3$?kern@?$hb_kern_machine_t@Uaccelerator_t@?$KerxSubTableFormat0@UKernAATSubTableHeader@OT@@@AAT@@@OT@@QEBAXPEAUhb_font_t@@PEAUhb_buffer_t@@I_N@Z 00000001800dcff0     hb-ot-layout.obj
 0002:0003200c       $chain$4$?kern@?$hb_kern_machine_t@Uaccelerator_t@?$KerxSubTableFormat0@UKernAATSubTableHeader@OT@@@AAT@@@OT@@QEBAXPEAUhb_font_t@@PEAUhb_buffer_t@@I_N@Z 00000001800dd00c     hb-ot-layout.obj
 0002:0003201c       $chain$5$?kern@?$hb_kern_machine_t@Uaccelerator_t@?$KerxSubTableFormat0@UKernAATSubTableHeader@OT@@@AAT@@@OT@@QEBAXPEAUhb_font_t@@PEAUhb_buffer_t@@I_N@Z 00000001800dd01c     hb-ot-layout.obj
 0002:0003202c       $chain$1$?kern@?$hb_kern_machine_t@U?$KernSubTableFormat3@UKernOTSubTableHeader@OT@@@OT@@@OT@@QEBAXPEAUhb_font_t@@PEAUhb_buffer_t@@I_N@Z 00000001800dd02c     hb-ot-layout.obj
 0002:00032044       $chain$2$?kern@?$hb_kern_machine_t@U?$KernSubTableFormat3@UKernOTSubTableHeader@OT@@@OT@@@OT@@QEBAXPEAUhb_font_t@@PEAUhb_buffer_t@@I_N@Z 00000001800dd044     hb-ot-layout.obj
 0002:00032058       $chain$3$?kern@?$hb_kern_machine_t@U?$KernSubTableFormat3@UKernOTSubTableHeader@OT@@@OT@@@OT@@QEBAXPEAUhb_font_t@@PEAUhb_buffer_t@@I_N@Z 00000001800dd058     hb-ot-layout.obj
 0002:00032068       $chain$4$?kern@?$hb_kern_machine_t@U?$KernSubTableFormat3@UKernOTSubTableHeader@OT@@@OT@@@OT@@QEBAXPEAUhb_font_t@@PEAUhb_buffer_t@@I_N@Z 00000001800dd068     hb-ot-layout.obj
 0002:00032078       $chain$0$?kern@?$hb_kern_machine_t@Uaccelerator_t@?$KerxSubTableFormat2@UKernOTSubTableHeader@OT@@@AAT@@@OT@@QEBAXPEAUhb_font_t@@PEAUhb_buffer_t@@I_N@Z 00000001800dd078     hb-ot-layout.obj
 0002:0003208c       $chain$3$?kern@?$hb_kern_machine_t@Uaccelerator_t@?$KerxSubTableFormat2@UKernOTSubTableHeader@OT@@@AAT@@@OT@@QEBAXPEAUhb_font_t@@PEAUhb_buffer_t@@I_N@Z 00000001800dd08c     hb-ot-layout.obj
 0002:000320a8       $chain$4$?kern@?$hb_kern_machine_t@Uaccelerator_t@?$KerxSubTableFormat2@UKernOTSubTableHeader@OT@@@AAT@@@OT@@QEBAXPEAUhb_font_t@@PEAUhb_buffer_t@@I_N@Z 00000001800dd0a8     hb-ot-layout.obj
 0002:000320b8       $chain$5$?kern@?$hb_kern_machine_t@Uaccelerator_t@?$KerxSubTableFormat2@UKernOTSubTableHeader@OT@@@AAT@@@OT@@QEBAXPEAUhb_font_t@@PEAUhb_buffer_t@@I_N@Z 00000001800dd0b8     hb-ot-layout.obj
 0002:000320c8       $chain$0$?transition@driver_context_t@?$KerxSubTableFormat1@UKernOTSubTableHeader@OT@@@AAT@@QEAAXPEAUhb_buffer_t@@PEAU?$StateTableDriver@UObsoleteTypes@AAT@@XW4Flags@?$KerxSubTableFormat1@UKernOTSubTableHeader@OT@@@2@@3@AEBU?$Entry@X@3@@Z 00000001800dd0c8     hb-ot-layout.obj
 0002:000320dc       $chain$1$?transition@driver_context_t@?$KerxSubTableFormat1@UKernOTSubTableHeader@OT@@@AAT@@QEAAXPEAUhb_buffer_t@@PEAU?$StateTableDriver@UObsoleteTypes@AAT@@XW4Flags@?$KerxSubTableFormat1@UKernOTSubTableHeader@OT@@@2@@3@AEBU?$Entry@X@3@@Z 00000001800dd0dc     hb-ot-layout.obj
 0002:000320ec       $chain$3$??$drive@Udriver_context_t@?$KerxSubTableFormat1@UKernOTSubTableHeader@OT@@@AAT@@@?$StateTableDriver@UObsoleteTypes@AAT@@XW4Flags@?$KerxSubTableFormat1@UKernOTSubTableHeader@OT@@@2@@AAT@@QEAAXPEAUdriver_context_t@?$KerxSubTableFormat1@UKernOTSubTableHeader@OT@@@1@PEAUhb_aat_apply_context_t@1@@Z 00000001800dd0ec     hb-ot-layout.obj
 0002:0003210c       $chain$4$??$drive@Udriver_context_t@?$KerxSubTableFormat1@UKernOTSubTableHeader@OT@@@AAT@@@?$StateTableDriver@UObsoleteTypes@AAT@@XW4Flags@?$KerxSubTableFormat1@UKernOTSubTableHeader@OT@@@2@@AAT@@QEAAXPEAUdriver_context_t@?$KerxSubTableFormat1@UKernOTSubTableHeader@OT@@@1@PEAUhb_aat_apply_context_t@1@@Z 00000001800dd10c     hb-ot-layout.obj
 0002:0003211c       $chain$0$?kern@?$hb_kern_machine_t@Uaccelerator_t@?$KerxSubTableFormat0@UKernOTSubTableHeader@OT@@@AAT@@@OT@@QEBAXPEAUhb_font_t@@PEAUhb_buffer_t@@I_N@Z 00000001800dd11c     hb-ot-layout.obj
 0002:00032130       $chain$3$?kern@?$hb_kern_machine_t@Uaccelerator_t@?$KerxSubTableFormat0@UKernOTSubTableHeader@OT@@@AAT@@@OT@@QEBAXPEAUhb_font_t@@PEAUhb_buffer_t@@I_N@Z 00000001800dd130     hb-ot-layout.obj
 0002:0003214c       $chain$4$?kern@?$hb_kern_machine_t@Uaccelerator_t@?$KerxSubTableFormat0@UKernOTSubTableHeader@OT@@@AAT@@@OT@@QEBAXPEAUhb_font_t@@PEAUhb_buffer_t@@I_N@Z 00000001800dd14c     hb-ot-layout.obj
 0002:0003215c       $chain$5$?kern@?$hb_kern_machine_t@Uaccelerator_t@?$KerxSubTableFormat0@UKernOTSubTableHeader@OT@@@AAT@@@OT@@QEBAXPEAUhb_font_t@@PEAUhb_buffer_t@@I_N@Z 00000001800dd15c     hb-ot-layout.obj
 0002:0003216c       $unwind$??$dispatch@U?$ContextFormat2_5@USmallTypes@Layout@OT@@@OT@@@hb_accelerate_subtables_context_t@OT@@QEAA?AUhb_empty_t@@AEBU?$ContextFormat2_5@USmallTypes@Layout@OT@@@1@@Z 00000001800dd16c     hb-ot-layout.obj
 0002:0003216c       $unwind$??$dispatch@U?$LigatureSubstFormat1_2@USmallTypes@Layout@OT@@@GSUB_impl@Layout@OT@@@hb_accelerate_subtables_context_t@OT@@QEAA?AUhb_empty_t@@AEBU?$LigatureSubstFormat1_2@USmallTypes@Layout@OT@@@GSUB_impl@Layout@1@@Z 00000001800dd16c     hb-ot-layout.obj
 0002:0003216c       $unwind$??$dispatch@U?$PairPosFormat1_3@USmallTypes@Layout@OT@@@GPOS_impl@Layout@OT@@@hb_accelerate_subtables_context_t@OT@@QEAA?AUhb_empty_t@@AEBU?$PairPosFormat1_3@USmallTypes@Layout@OT@@@GPOS_impl@Layout@1@@Z 00000001800dd16c     hb-ot-layout.obj
 0002:00032188       $chain$0$??$dispatch@Uhb_sanitize_context_t@@$$V@?$Extension@UExtensionPos@GPOS_impl@Layout@OT@@@OT@@QEBA_NPEAUhb_sanitize_context_t@@@Z 00000001800dd188     hb-ot-layout.obj
 0002:0003219c       $chain$1$??$dispatch@Uhb_sanitize_context_t@@$$V@?$Extension@UExtensionPos@GPOS_impl@Layout@OT@@@OT@@QEBA_NPEAUhb_sanitize_context_t@@@Z 00000001800dd19c     hb-ot-layout.obj
 0002:000321ac       $unwind$??$dispatch@UMarkArray@GPOS_impl@Layout@OT@@$$V@hb_sanitize_context_t@@QEAA_NAEBUMarkArray@GPOS_impl@Layout@OT@@@Z 00000001800dd1ac     hb-ot-layout.obj
 0002:000321b8       $chain$5$??$dispatch@UMarkArray@GPOS_impl@Layout@OT@@$$V@hb_sanitize_context_t@@QEAA_NAEBUMarkArray@GPOS_impl@Layout@OT@@@Z 00000001800dd1b8     hb-ot-layout.obj
 0002:000321e0       $chain$7$??$dispatch@UMarkArray@GPOS_impl@Layout@OT@@$$V@hb_sanitize_context_t@@QEAA_NAEBUMarkArray@GPOS_impl@Layout@OT@@@Z 00000001800dd1e0     hb-ot-layout.obj
 0002:00032208       $unwind$??$dispatch@ULigatureArray@GPOS_impl@Layout@OT@@I@hb_sanitize_context_t@@QEAA_NAEBULigatureArray@GPOS_impl@Layout@OT@@$$QEAI@Z 00000001800dd208     hb-ot-layout.obj
 0002:00032214       $chain$4$??$dispatch@ULigatureArray@GPOS_impl@Layout@OT@@I@hb_sanitize_context_t@@QEAA_NAEBULigatureArray@GPOS_impl@Layout@OT@@$$QEAI@Z 00000001800dd214     hb-ot-layout.obj
 0002:00032238       $chain$6$??$dispatch@ULigatureArray@GPOS_impl@Layout@OT@@I@hb_sanitize_context_t@@QEAA_NAEBULigatureArray@GPOS_impl@Layout@OT@@$$QEAI@Z 00000001800dd238     hb-ot-layout.obj
 0002:0003225c       $chain$0$?alloc@?$hb_vector_t@Ulookup_map_t@hb_ot_map_t@@$0A@@@QEAA_NI_N@Z 00000001800dd25c     hb-ot-map.obj
 0002:0003225c       $chain$0$?alloc@?$hb_vector_t@Uhb_outline_point_t@@$0A@@@QEAA_NI_N@Z 00000001800dd25c     hb-outline.obj
 0002:00032270       $chain$2$?alloc@?$hb_vector_t@Ulookup_map_t@hb_ot_map_t@@$0A@@@QEAA_NI_N@Z 00000001800dd270     hb-ot-map.obj
 0002:00032270       $chain$4$?alloc@?$hb_vector_t@Ulookup_map_t@hb_ot_map_t@@$0A@@@QEAA_NI_N@Z 00000001800dd270     hb-ot-map.obj
 0002:00032270       $chain$2$?alloc@?$hb_vector_t@Uhb_outline_point_t@@$0A@@@QEAA_NI_N@Z 00000001800dd270     hb-outline.obj
 0002:00032270       $chain$4$?alloc@?$hb_vector_t@Uhb_outline_point_t@@$0A@@@QEAA_NI_N@Z 00000001800dd270     hb-outline.obj
 0002:00032284       $unwind$??0hb_ot_map_builder_t@@QEAA@PEAUhb_face_t@@AEBUhb_segment_properties_t@@@Z 00000001800dd284     hb-ot-map.obj
 0002:000322a4       $unwind$?add_feature@hb_ot_map_builder_t@@QEAAXIW4hb_ot_map_feature_flags_t@@I@Z 00000001800dd2a4     hb-ot-map.obj
 0002:000322b4       $chain$3$?add_feature@hb_ot_map_builder_t@@QEAAXIW4hb_ot_map_feature_flags_t@@I@Z 00000001800dd2b4     hb-ot-map.obj
 0002:000322d4       $chain$4$?add_feature@hb_ot_map_builder_t@@QEAAXIW4hb_ot_map_feature_flags_t@@I@Z 00000001800dd2d4     hb-ot-map.obj
 0002:000322e4       $chain$5$?add_feature@hb_ot_map_builder_t@@QEAAXIW4hb_ot_map_feature_flags_t@@I@Z 00000001800dd2e4     hb-ot-map.obj
 0002:00032304       $unwind$?compile@hb_ot_map_builder_t@@QEAAXAEAUhb_ot_map_t@@AEBUhb_ot_shape_plan_key_t@@@Z 00000001800dd304     hb-ot-map.obj
 0002:00032320       $unwind$?add_lookups@hb_ot_map_builder_t@@AEAAXAEAUhb_ot_map_t@@IIII_N111I@Z 00000001800dd320     hb-ot-map.obj
 0002:00032340       $chain$0$?alloc@?$hb_vector_t@Ufeature_info_t@hb_ot_map_builder_t@@$0A@@@QEAA_NI_N@Z 00000001800dd340     hb-ot-map.obj
 0002:00032354       $chain$2$?alloc@?$hb_vector_t@Ufeature_info_t@hb_ot_map_builder_t@@$0A@@@QEAA_NI_N@Z 00000001800dd354     hb-ot-map.obj
 0002:00032354       $chain$4$?alloc@?$hb_vector_t@Ufeature_info_t@hb_ot_map_builder_t@@$0A@@@QEAA_NI_N@Z 00000001800dd354     hb-ot-map.obj
 0002:00032368       $chain$1$??C?$hb_lazy_loader_t@UOS2@OT@@U?$hb_table_lazy_loader_t@UOS2@OT@@$05$00@@Uhb_face_t@@$05Uhb_blob_t@@@@QEBAPEBUOS2@OT@@XZ 00000001800dd368     hb-ot-metrics.obj
 0002:00032380       $chain$2$??C?$hb_lazy_loader_t@UOS2@OT@@U?$hb_table_lazy_loader_t@UOS2@OT@@$05$00@@Uhb_face_t@@$05Uhb_blob_t@@@@QEBAPEBUOS2@OT@@XZ 00000001800dd380     hb-ot-metrics.obj
 0002:00032390       $chain$1$?get@?$hb_lazy_loader_t@UMVAR@OT@@U?$hb_table_lazy_loader_t@UMVAR@OT@@$0BG@$00@@Uhb_face_t@@$0BG@Uhb_blob_t@@@@QEBAPEBUMVAR@OT@@XZ 00000001800dd390     hb-ot-metrics.obj
 0002:000323a8       $chain$2$?get@?$hb_lazy_loader_t@UMVAR@OT@@U?$hb_table_lazy_loader_t@UMVAR@OT@@$0BG@$00@@Uhb_face_t@@$0BG@Uhb_blob_t@@@@QEBAPEBUMVAR@OT@@XZ 00000001800dd3a8     hb-ot-metrics.obj
 0002:000323b8       $unwind$??$sanitize_blob@UMVAR@OT@@@hb_sanitize_context_t@@QEAAPEAUhb_blob_t@@PEAU1@@Z 00000001800dd3b8     hb-ot-metrics.obj
 0002:000323d4       $unwind$?_hb_ot_shape_fallback_mark_position@@YAXPEBUhb_ot_shape_plan_t@@PEAUhb_font_t@@PEAUhb_buffer_t@@_N@Z 00000001800dd3d4     hb-ot-shape-fallback.obj
 0002:000323e4       $chain$2$?_hb_ot_shape_fallback_mark_position@@YAXPEBUhb_ot_shape_plan_t@@PEAUhb_font_t@@PEAUhb_buffer_t@@_N@Z 00000001800dd3e4     hb-ot-shape-fallback.obj
 0002:00032400       $chain$3$?_hb_ot_shape_fallback_mark_position@@YAXPEBUhb_ot_shape_plan_t@@PEAUhb_font_t@@PEAUhb_buffer_t@@_N@Z 00000001800dd400     hb-ot-shape-fallback.obj
 0002:00032410       $chain$2$?_hb_ot_shape_fallback_mark_position_recategorize_marks@@YAXPEBUhb_ot_shape_plan_t@@PEAUhb_font_t@@PEAUhb_buffer_t@@@Z 00000001800dd410     hb-ot-shape-fallback.obj
 0002:0003242c       $chain$3$?_hb_ot_shape_fallback_mark_position_recategorize_marks@@YAXPEBUhb_ot_shape_plan_t@@PEAUhb_font_t@@PEAUhb_buffer_t@@@Z 00000001800dd42c     hb-ot-shape-fallback.obj
 0002:0003243c       $unwind$?_hb_ot_shape_fallback_kern@@YAXPEBUhb_ot_shape_plan_t@@PEAUhb_font_t@@PEAUhb_buffer_t@@@Z 00000001800dd43c     hb-ot-shape-fallback.obj
 0002:0003244c       $chain$0$?_hb_ot_shape_fallback_kern@@YAXPEBUhb_ot_shape_plan_t@@PEAUhb_font_t@@PEAUhb_buffer_t@@@Z 00000001800dd44c     hb-ot-shape-fallback.obj
 0002:00032460       $chain$1$?_hb_ot_shape_fallback_kern@@YAXPEBUhb_ot_shape_plan_t@@PEAUhb_font_t@@PEAUhb_buffer_t@@@Z 00000001800dd460     hb-ot-shape-fallback.obj
 0002:00032470       $unwind$?_hb_ot_shape_fallback_spaces@@YAXPEBUhb_ot_shape_plan_t@@PEAUhb_font_t@@PEAUhb_buffer_t@@@Z 00000001800dd470     hb-ot-shape-fallback.obj
 0002:0003247c       $chain$4$?_hb_ot_shape_fallback_spaces@@YAXPEBUhb_ot_shape_plan_t@@PEAUhb_font_t@@PEAUhb_buffer_t@@@Z 00000001800dd47c     hb-ot-shape-fallback.obj
 0002:000324a0       $chain$5$?_hb_ot_shape_fallback_spaces@@YAXPEBUhb_ot_shape_plan_t@@PEAUhb_font_t@@PEAUhb_buffer_t@@@Z 00000001800dd4a0     hb-ot-shape-fallback.obj
 0002:000324b0       $chain$6$?_hb_ot_shape_fallback_spaces@@YAXPEBUhb_ot_shape_plan_t@@PEAUhb_font_t@@PEAUhb_buffer_t@@@Z 00000001800dd4b0     hb-ot-shape-fallback.obj
 0002:000324d4       $unwind$?position_mark@@YAXPEBUhb_ot_shape_plan_t@@PEAUhb_font_t@@PEAUhb_buffer_t@@AEAUhb_glyph_extents_t@@II@Z 00000001800dd4d4     hb-ot-shape-fallback.obj
 0002:000324ec       $unwind$?position_around_base@@YAXPEBUhb_ot_shape_plan_t@@PEAUhb_font_t@@PEAUhb_buffer_t@@II_N@Z 00000001800dd4ec     hb-ot-shape-fallback.obj
 0002:0003250c       $chain$1$?position_around_base@@YAXPEBUhb_ot_shape_plan_t@@PEAUhb_font_t@@PEAUhb_buffer_t@@II_N@Z 00000001800dd50c     hb-ot-shape-fallback.obj
 0002:00032524       $chain$2$?position_around_base@@YAXPEBUhb_ot_shape_plan_t@@PEAUhb_font_t@@PEAUhb_buffer_t@@II_N@Z 00000001800dd524     hb-ot-shape-fallback.obj
 0002:00032534       $unwind$?position_cluster@@YAXPEBUhb_ot_shape_plan_t@@PEAUhb_font_t@@PEAUhb_buffer_t@@II_N@Z 00000001800dd534     hb-ot-shape-fallback.obj
 0002:00032544       $chain$0$?position_cluster@@YAXPEBUhb_ot_shape_plan_t@@PEAUhb_font_t@@PEAUhb_buffer_t@@II_N@Z 00000001800dd544     hb-ot-shape-fallback.obj
 0002:00032558       $chain$2$?position_cluster@@YAXPEBUhb_ot_shape_plan_t@@PEAUhb_font_t@@PEAUhb_buffer_t@@II_N@Z 00000001800dd558     hb-ot-shape-fallback.obj
 0002:00032570       $chain$3$?position_cluster@@YAXPEBUhb_ot_shape_plan_t@@PEAUhb_font_t@@PEAUhb_buffer_t@@II_N@Z 00000001800dd570     hb-ot-shape-fallback.obj
 0002:00032580       $chain$4$?position_cluster@@YAXPEBUhb_ot_shape_plan_t@@PEAUhb_font_t@@PEAUhb_buffer_t@@II_N@Z 00000001800dd580     hb-ot-shape-fallback.obj
 0002:00032590       $unwind$?kern@?$hb_kern_machine_t@Uhb_ot_shape_fallback_kern_driver_t@@@OT@@QEBAXPEAUhb_font_t@@PEAUhb_buffer_t@@I_N@Z 00000001800dd590     hb-ot-shape-fallback.obj
 0002:000325a8       $chain$0$?kern@?$hb_kern_machine_t@Uhb_ot_shape_fallback_kern_driver_t@@@OT@@QEBAXPEAUhb_font_t@@PEAUhb_buffer_t@@I_N@Z 00000001800dd5a8     hb-ot-shape-fallback.obj
 0002:000325bc       $chain$3$?kern@?$hb_kern_machine_t@Uhb_ot_shape_fallback_kern_driver_t@@@OT@@QEBAXPEAUhb_font_t@@PEAUhb_buffer_t@@I_N@Z 00000001800dd5bc     hb-ot-shape-fallback.obj
 0002:000325d8       $chain$4$?kern@?$hb_kern_machine_t@Uhb_ot_shape_fallback_kern_driver_t@@@OT@@QEBAXPEAUhb_font_t@@PEAUhb_buffer_t@@I_N@Z 00000001800dd5d8     hb-ot-shape-fallback.obj
 0002:000325e8       $chain$5$?kern@?$hb_kern_machine_t@Uhb_ot_shape_fallback_kern_driver_t@@@OT@@QEBAXPEAUhb_font_t@@PEAUhb_buffer_t@@I_N@Z 00000001800dd5e8     hb-ot-shape-fallback.obj
 0002:000325f8       $unwind$?_hb_ot_shape_normalize@@YAXPEBUhb_ot_shape_plan_t@@PEAUhb_buffer_t@@PEAUhb_font_t@@@Z 00000001800dd5f8     hb-ot-shape-normalize.obj
 0002:00032608       $chain$4$?_hb_ot_shape_normalize@@YAXPEBUhb_ot_shape_plan_t@@PEAUhb_buffer_t@@PEAUhb_font_t@@@Z 00000001800dd608     hb-ot-shape-normalize.obj
 0002:0003262c       $chain$5$?_hb_ot_shape_normalize@@YAXPEBUhb_ot_shape_plan_t@@PEAUhb_buffer_t@@PEAUhb_font_t@@@Z 00000001800dd62c     hb-ot-shape-normalize.obj
 0002:0003263c       $unwind$?decompose@@YAIPEBUhb_ot_shape_normalize_context_t@@_NI@Z 00000001800dd63c     hb-ot-shape-normalize.obj
 0002:00032650       $unwind$?decompose_current_character@@YAXPEBUhb_ot_shape_normalize_context_t@@_N@Z 00000001800dd650     hb-ot-shape-normalize.obj
 0002:00032664       $unwind$?handle_variation_selector_cluster@@YAXPEBUhb_ot_shape_normalize_context_t@@I_N@Z 00000001800dd664     hb-ot-shape-normalize.obj
 0002:00032670       $chain$1$?handle_variation_selector_cluster@@YAXPEBUhb_ot_shape_normalize_context_t@@I_N@Z 00000001800dd670     hb-ot-shape-normalize.obj
 0002:00032688       $chain$4$?handle_variation_selector_cluster@@YAXPEBUhb_ot_shape_normalize_context_t@@I_N@Z 00000001800dd688     hb-ot-shape-normalize.obj
 0002:000326a4       $chain$5$?handle_variation_selector_cluster@@YAXPEBUhb_ot_shape_normalize_context_t@@I_N@Z 00000001800dd6a4     hb-ot-shape-normalize.obj
 0002:000326b4       $chain$6$?handle_variation_selector_cluster@@YAXPEBUhb_ot_shape_normalize_context_t@@I_N@Z 00000001800dd6b4     hb-ot-shape-normalize.obj
 0002:000326c4       $unwind$?init0@hb_ot_shape_plan_t@@QEAA_NPEAUhb_face_t@@PEBUhb_shape_plan_key_t@@@Z 00000001800dd6c4     hb-ot-shape.obj
 0002:000326e4       $unwind$?compile@hb_ot_shape_planner_t@@QEAAXAEAUhb_ot_shape_plan_t@@AEBUhb_ot_shape_plan_key_t@@@Z 00000001800dd6e4     hb-ot-shape.obj
 0002:000326f8       $chain$0$?compile@hb_ot_shape_planner_t@@QEAAXAEAUhb_ot_shape_plan_t@@AEBUhb_ot_shape_plan_key_t@@@Z 00000001800dd6f8     hb-ot-shape.obj
 0002:0003270c       $chain$1$?compile@hb_ot_shape_planner_t@@QEAAXAEAUhb_ot_shape_plan_t@@AEBUhb_ot_shape_plan_key_t@@@Z 00000001800dd70c     hb-ot-shape.obj
 0002:00032720       $chain$2$?compile@hb_ot_shape_planner_t@@QEAAXAEAUhb_ot_shape_plan_t@@AEBUhb_ot_shape_plan_key_t@@@Z 00000001800dd720     hb-ot-shape.obj
 0002:00032730       $chain$3$?compile@hb_ot_shape_planner_t@@QEAAXAEAUhb_ot_shape_plan_t@@AEBUhb_ot_shape_plan_key_t@@@Z 00000001800dd730     hb-ot-shape.obj
 0002:00032744       $chain$4$?compile@hb_ot_shape_planner_t@@QEAAXAEAUhb_ot_shape_plan_t@@AEBUhb_ot_shape_plan_key_t@@@Z 00000001800dd744     hb-ot-shape.obj
 0002:00032758       $unwind$_hb_ot_shaper_font_data_create 00000001800dd758     hb-ot-shape.obj
 0002:00032764       $chain$3$_hb_ot_shaper_font_data_create 00000001800dd764     hb-ot-shape.obj
 0002:00032780       $chain$4$_hb_ot_shaper_font_data_create 00000001800dd780     hb-ot-shape.obj
 0002:00032794       $chain$5$_hb_ot_shaper_font_data_create 00000001800dd794     hb-ot-shape.obj
 0002:000327a4       $chain$6$_hb_ot_shaper_font_data_create 00000001800dd7a4     hb-ot-shape.obj
 0002:000327bc       $unwind$?hb_ot_shape_collect_features@@YAXPEAUhb_ot_shape_planner_t@@PEBUhb_feature_t@@I@Z 00000001800dd7bc     hb-ot-shape.obj
 0002:000327d8       $unwind$?hb_set_unicode_props@@YAXPEAUhb_buffer_t@@@Z 00000001800dd7d8     hb-ot-shape.obj
 0002:000327e8       $chain$3$?hb_set_unicode_props@@YAXPEAUhb_buffer_t@@@Z 00000001800dd7e8     hb-ot-shape.obj
 0002:00032808       $chain$4$?hb_set_unicode_props@@YAXPEAUhb_buffer_t@@@Z 00000001800dd808     hb-ot-shape.obj
 0002:00032818       $chain$2$?hb_form_clusters@@YAXPEAUhb_buffer_t@@@Z 00000001800dd818     hb-ot-shape.obj
 0002:00032834       $chain$3$?hb_form_clusters@@YAXPEAUhb_buffer_t@@@Z 00000001800dd834     hb-ot-shape.obj
 0002:00032848       $chain$4$?hb_form_clusters@@YAXPEAUhb_buffer_t@@@Z 00000001800dd848     hb-ot-shape.obj
 0002:0003285c       $chain$5$?hb_form_clusters@@YAXPEAUhb_buffer_t@@@Z 00000001800dd85c     hb-ot-shape.obj
 0002:0003286c       $chain$6$?hb_form_clusters@@YAXPEAUhb_buffer_t@@@Z 00000001800dd86c     hb-ot-shape.obj
 0002:0003287c       $chain$7$?hb_form_clusters@@YAXPEAUhb_buffer_t@@@Z 00000001800dd87c     hb-ot-shape.obj
 0002:0003288c       $unwind$?hb_ot_rotate_chars@@YAXPEBUhb_ot_shape_context_t@@@Z 00000001800dd88c     hb-ot-shape.obj
 0002:000328a0       $chain$0$?hb_ot_rotate_chars@@YAXPEBUhb_ot_shape_context_t@@@Z 00000001800dd8a0     hb-ot-shape.obj
 0002:000328b4       $chain$1$?hb_ot_rotate_chars@@YAXPEBUhb_ot_shape_context_t@@@Z 00000001800dd8b4     hb-ot-shape.obj
 0002:000328c8       $chain$2$?hb_ot_rotate_chars@@YAXPEBUhb_ot_shape_context_t@@@Z 00000001800dd8c8     hb-ot-shape.obj
 0002:000328d8       $chain$3$?hb_ot_rotate_chars@@YAXPEBUhb_ot_shape_context_t@@@Z 00000001800dd8d8     hb-ot-shape.obj
 0002:000328e8       $unwind$?hb_ot_shape_setup_masks_fraction@@YAXPEBUhb_ot_shape_context_t@@@Z 00000001800dd8e8     hb-ot-shape.obj
 0002:000328f0       $chain$2$?hb_ot_shape_setup_masks_fraction@@YAXPEBUhb_ot_shape_context_t@@@Z 00000001800dd8f0     hb-ot-shape.obj
 0002:0003290c       $chain$6$?hb_ot_shape_setup_masks_fraction@@YAXPEBUhb_ot_shape_context_t@@@Z 00000001800dd90c     hb-ot-shape.obj
 0002:0003292c       $chain$7$?hb_ot_shape_setup_masks_fraction@@YAXPEBUhb_ot_shape_context_t@@@Z 00000001800dd92c     hb-ot-shape.obj
 0002:0003293c       $chain$8$?hb_ot_shape_setup_masks_fraction@@YAXPEBUhb_ot_shape_context_t@@@Z 00000001800dd93c     hb-ot-shape.obj
 0002:0003294c       $chain$9$?hb_ot_shape_setup_masks_fraction@@YAXPEBUhb_ot_shape_context_t@@@Z 00000001800dd94c     hb-ot-shape.obj
 0002:00032978       $chain$0$?hb_ot_substitute_default@@YAXPEBUhb_ot_shape_context_t@@@Z 00000001800dd978     hb-ot-shape.obj
 0002:0003298c       $chain$3$?hb_ot_substitute_default@@YAXPEBUhb_ot_shape_context_t@@@Z 00000001800dd98c     hb-ot-shape.obj
 0002:000329a8       $chain$5$?hb_ot_substitute_default@@YAXPEBUhb_ot_shape_context_t@@@Z 00000001800dd9a8     hb-ot-shape.obj
 0002:000329c0       $chain$6$?hb_ot_substitute_default@@YAXPEBUhb_ot_shape_context_t@@@Z 00000001800dd9c0     hb-ot-shape.obj
 0002:000329d0       $chain$7$?hb_ot_substitute_default@@YAXPEBUhb_ot_shape_context_t@@@Z 00000001800dd9d0     hb-ot-shape.obj
 0002:000329e0       $chain$8$?hb_ot_substitute_default@@YAXPEBUhb_ot_shape_context_t@@@Z 00000001800dd9e0     hb-ot-shape.obj
 0002:000329f0       $chain$9$?hb_ot_substitute_default@@YAXPEBUhb_ot_shape_context_t@@@Z 00000001800dd9f0     hb-ot-shape.obj
 0002:00032a18       $unwind$?hb_ot_substitute_post@@YAXPEBUhb_ot_shape_context_t@@@Z 00000001800dda18     hb-ot-shape.obj
 0002:00032a24       $chain$2$?hb_ot_substitute_post@@YAXPEBUhb_ot_shape_context_t@@@Z 00000001800dda24     hb-ot-shape.obj
 0002:00032a40       $chain$3$?hb_ot_substitute_post@@YAXPEBUhb_ot_shape_context_t@@@Z 00000001800dda40     hb-ot-shape.obj
 0002:00032a50       $unwind$?hb_ot_position_default@@YAXPEBUhb_ot_shape_context_t@@@Z 00000001800dda50     hb-ot-shape.obj
 0002:00032a5c       $chain$5$?hb_ot_position_default@@YAXPEBUhb_ot_shape_context_t@@@Z 00000001800dda5c     hb-ot-shape.obj
 0002:00032a84       $chain$6$?hb_ot_position_default@@YAXPEBUhb_ot_shape_context_t@@@Z 00000001800dda84     hb-ot-shape.obj
 0002:00032a94       $unwind$?hb_ot_position_plan@@YAXPEBUhb_ot_shape_context_t@@@Z 00000001800dda94     hb-ot-shape.obj
 0002:00032aac       $unwind$?hb_propagate_flags@@YAXPEAUhb_buffer_t@@@Z 00000001800ddaac     hb-ot-shape.obj
 0002:00032ab4       $chain$2$?hb_propagate_flags@@YAXPEAUhb_buffer_t@@@Z 00000001800ddab4     hb-ot-shape.obj
 0002:00032ad0       $chain$7$?hb_propagate_flags@@YAXPEAUhb_buffer_t@@@Z 00000001800ddad0     hb-ot-shape.obj
 0002:00032af4       $chain$8$?hb_propagate_flags@@YAXPEAUhb_buffer_t@@@Z 00000001800ddaf4     hb-ot-shape.obj
 0002:00032b04       $chain$9$?hb_propagate_flags@@YAXPEAUhb_buffer_t@@@Z 00000001800ddb04     hb-ot-shape.obj
 0002:00032b14       $unwind$??$dispatch@UAxisValueOffsetArray@OT@@AEBU?$IntType@G$01@2@PEBU12@@hb_sanitize_context_t@@QEAA_NAEBUAxisValueOffsetArray@OT@@AEBU?$IntType@G$01@2@$$QEAPEBU12@@Z 00000001800ddb14     hb-ot-shape.obj
 0002:00032b24       $chain$3$??$dispatch@UAxisValueOffsetArray@OT@@AEBU?$IntType@G$01@2@PEBU12@@hb_sanitize_context_t@@QEAA_NAEBUAxisValueOffsetArray@OT@@AEBU?$IntType@G$01@2@$$QEAPEBU12@@Z 00000001800ddb24     hb-ot-shape.obj
 0002:00032b44       $chain$5$??$dispatch@UAxisValueOffsetArray@OT@@AEBU?$IntType@G$01@2@PEBU12@@hb_sanitize_context_t@@QEAA_NAEBUAxisValueOffsetArray@OT@@AEBU?$IntType@G$01@2@$$QEAPEBU12@@Z 00000001800ddb44     hb-ot-shape.obj
 0002:00032b64       $unwind$??$sanitize_blob@USTAT@OT@@@hb_sanitize_context_t@@QEAAPEAUhb_blob_t@@PEAU1@@Z 00000001800ddb64     hb-ot-shape.obj
 0002:00032b80       $unwind$?safe_to_insert_tatweel@hb_buffer_t@@QEAAXII@Z 00000001800ddb80     hb-ot-shaper-arabic.obj
 0002:00032b90       $chain$4$?discard_stale_objects@hb_serialize_context_t@@QEAAXXZ 00000001800ddb90     hb-ot-shaper-arabic.obj
 0002:00032bb4       $chain$5$?discard_stale_objects@hb_serialize_context_t@@QEAAXXZ 00000001800ddbb4     hb-ot-shaper-arabic.obj
 0002:00032bc4       $unwind$?data_create_arabic@@YAPEAXPEBUhb_ot_shape_plan_t@@@Z 00000001800ddbc4     hb-ot-shaper-arabic.obj
 0002:00032be0       $unwind$?arabic_fallback_shape@@YA_NPEBUhb_ot_shape_plan_t@@PEAUhb_font_t@@PEAUhb_buffer_t@@@Z 00000001800ddbe0     hb-ot-shaper-arabic.obj
 0002:00032bf8       $chain$3$?arabic_fallback_shape@@YA_NPEBUhb_ot_shape_plan_t@@PEAUhb_font_t@@PEAUhb_buffer_t@@@Z 00000001800ddbf8     hb-ot-shaper-arabic.obj
 0002:00032c18       $chain$4$?arabic_fallback_shape@@YA_NPEBUhb_ot_shape_plan_t@@PEAUhb_font_t@@PEAUhb_buffer_t@@@Z 00000001800ddc18     hb-ot-shaper-arabic.obj
 0002:00032c28       $unwind$?serialize@?$ArrayOf@UHBGlyphID16@OT@@U?$IntType@G$01@2@@OT@@QEAA_NPEAUhb_serialize_context_t@@I_N@Z 00000001800ddc28     hb-ot-shaper-arabic.obj
 0002:00032c28       $unwind$?serialize@?$HeadlessArrayOf@UHBGlyphID16@OT@@U?$IntType@G$01@2@@OT@@QEAA_NPEAUhb_serialize_context_t@@I_N@Z 00000001800ddc28     hb-ot-shaper-arabic.obj
 0002:00032c3c       $unwind$?serialize@?$SortedArrayOf@U?$RangeRecord@USmallTypes@Layout@OT@@@Common@Layout@OT@@U?$IntType@G$01@4@@OT@@QEAA_NPEAUhb_serialize_context_t@@I@Z 00000001800ddc3c     hb-ot-shaper-arabic.obj
 0002:00032c50       $chain$0$??$extend_min@U?$IntType@G$01@OT@@@hb_serialize_context_t@@QEAAPEAU?$IntType@G$01@OT@@AEAU12@@Z 00000001800ddc50     hb-ot-shaper-arabic.obj
 0002:00032c50       $chain$0$??$extend_min@U?$LigatureSet@USmallTypes@Layout@OT@@@GSUB_impl@Layout@OT@@@hb_serialize_context_t@@QEAAPEAU?$LigatureSet@USmallTypes@Layout@OT@@@GSUB_impl@Layout@OT@@PEAU1234@@Z 00000001800ddc50     hb-ot-shaper-arabic.obj
 0002:00032c50       $chain$0$??$extend_min@UCoverage@Common@Layout@OT@@@hb_serialize_context_t@@QEAAPEAUCoverage@Common@Layout@OT@@PEAU1234@@Z 00000001800ddc50     hb-ot-shaper-arabic.obj
 0002:00032c64       $chain$2$??$extend_min@U?$IntType@G$01@OT@@@hb_serialize_context_t@@QEAAPEAU?$IntType@G$01@OT@@AEAU12@@Z 00000001800ddc64     hb-ot-shaper-arabic.obj
 0002:00032c64       $chain$2$??$extend_min@U?$LigatureSet@USmallTypes@Layout@OT@@@GSUB_impl@Layout@OT@@@hb_serialize_context_t@@QEAAPEAU?$LigatureSet@USmallTypes@Layout@OT@@@GSUB_impl@Layout@OT@@PEAU1234@@Z 00000001800ddc64     hb-ot-shaper-arabic.obj
 0002:00032c64       $chain$2$??$extend_min@UCoverage@Common@Layout@OT@@@hb_serialize_context_t@@QEAAPEAUCoverage@Common@Layout@OT@@PEAU1234@@Z 00000001800ddc64     hb-ot-shaper-arabic.obj
 0002:00032c78       $chain$0$??$extend_min@U?$LigatureSubstFormat1_2@USmallTypes@Layout@OT@@@GSUB_impl@Layout@OT@@@hb_serialize_context_t@@QEAAPEAU?$LigatureSubstFormat1_2@USmallTypes@Layout@OT@@@GSUB_impl@Layout@OT@@PEAU1234@@Z 00000001800ddc78     hb-ot-shaper-arabic.obj
 0002:00032c78       $chain$0$??$extend_min@U?$SingleSubstFormat1_3@USmallTypes@Layout@OT@@@GSUB_impl@Layout@OT@@@hb_serialize_context_t@@QEAAPEAU?$SingleSubstFormat1_3@USmallTypes@Layout@OT@@@GSUB_impl@Layout@OT@@PEAU1234@@Z 00000001800ddc78     hb-ot-shaper-arabic.obj
 0002:00032c78       $chain$0$??$extend_min@U?$SingleSubstFormat2_4@USmallTypes@Layout@OT@@@GSUB_impl@Layout@OT@@@hb_serialize_context_t@@QEAAPEAU?$SingleSubstFormat2_4@USmallTypes@Layout@OT@@@GSUB_impl@Layout@OT@@PEAU1234@@Z 00000001800ddc78     hb-ot-shaper-arabic.obj
 0002:00032c78       $chain$0$??$extend_min@ULookup@OT@@@hb_serialize_context_t@@QEAAPEAULookup@OT@@PEAU12@@Z 00000001800ddc78     hb-ot-shaper-arabic.obj
 0002:00032c8c       $chain$2$??$extend_min@U?$LigatureSubstFormat1_2@USmallTypes@Layout@OT@@@GSUB_impl@Layout@OT@@@hb_serialize_context_t@@QEAAPEAU?$LigatureSubstFormat1_2@USmallTypes@Layout@OT@@@GSUB_impl@Layout@OT@@PEAU1234@@Z 00000001800ddc8c     hb-ot-shaper-arabic.obj
 0002:00032c8c       $chain$2$??$extend_min@U?$SingleSubstFormat1_3@USmallTypes@Layout@OT@@@GSUB_impl@Layout@OT@@@hb_serialize_context_t@@QEAAPEAU?$SingleSubstFormat1_3@USmallTypes@Layout@OT@@@GSUB_impl@Layout@OT@@PEAU1234@@Z 00000001800ddc8c     hb-ot-shaper-arabic.obj
 0002:00032c8c       $chain$2$??$extend_min@U?$SingleSubstFormat2_4@USmallTypes@Layout@OT@@@GSUB_impl@Layout@OT@@@hb_serialize_context_t@@QEAAPEAU?$SingleSubstFormat2_4@USmallTypes@Layout@OT@@@GSUB_impl@Layout@OT@@PEAU1234@@Z 00000001800ddc8c     hb-ot-shaper-arabic.obj
 0002:00032c8c       $chain$2$??$extend_min@ULookup@OT@@@hb_serialize_context_t@@QEAAPEAULookup@OT@@PEAU12@@Z 00000001800ddc8c     hb-ot-shaper-arabic.obj
 0002:00032ca0       $unwind$?serialize@?$LigatureSet@USmallTypes@Layout@OT@@@GSUB_impl@Layout@OT@@QEAA_NPEAUhb_serialize_context_t@@U?$hb_array_t@$$CBUHBGlyphID16@OT@@@@U?$hb_array_t@$$CBI@@AEAU6@@Z 00000001800ddca0     hb-ot-shaper-arabic.obj
 0002:00032cb8       $unwind$?serialize@?$LigatureSubstFormat1_2@USmallTypes@Layout@OT@@@GSUB_impl@Layout@OT@@QEAA_NPEAUhb_serialize_context_t@@U?$hb_sorted_array_t@$$CBUHBGlyphID16@OT@@@@U?$hb_array_t@$$CBI@@U?$hb_array_t@$$CBUHBGlyphID16@OT@@@@23@Z 00000001800ddcb8     hb-ot-shaper-arabic.obj
 0002:00032cd4       $unwind$?arabic_fallback_synthesize_lookup_single@@YAPEAUSubstLookup@GSUB_impl@Layout@OT@@PEBUhb_ot_shape_plan_t@@PEAUhb_font_t@@I@Z 00000001800ddcd4     hb-ot-shaper-arabic.obj
 0002:00032cf4       $chain$0$?arabic_fallback_synthesize_lookup_single@@YAPEAUSubstLookup@GSUB_impl@Layout@OT@@PEBUhb_ot_shape_plan_t@@PEAUhb_font_t@@I@Z 00000001800ddcf4     hb-ot-shaper-arabic.obj
 0002:00032d08       $chain$1$?arabic_fallback_synthesize_lookup_single@@YAPEAUSubstLookup@GSUB_impl@Layout@OT@@PEBUhb_ot_shape_plan_t@@PEAUhb_font_t@@I@Z 00000001800ddd08     hb-ot-shaper-arabic.obj
 0002:00032d18       $unwind$??$arabic_fallback_synthesize_lookup_ligature@$$BY00Uligature_3_set_t@@@@YAPEAUSubstLookup@GSUB_impl@Layout@OT@@PEBUhb_ot_shape_plan_t@@PEAUhb_font_t@@AEAY00$$CBUligature_3_set_t@@I@Z 00000001800ddd18     hb-ot-shaper-arabic.obj
 0002:00032d38       $chain$0$??$arabic_fallback_synthesize_lookup_ligature@$$BY00Uligature_3_set_t@@@@YAPEAUSubstLookup@GSUB_impl@Layout@OT@@PEBUhb_ot_shape_plan_t@@PEAUhb_font_t@@AEAY00$$CBUligature_3_set_t@@I@Z 00000001800ddd38     hb-ot-shaper-arabic.obj
 0002:00032d4c       $chain$1$??$arabic_fallback_synthesize_lookup_ligature@$$BY00Uligature_3_set_t@@@@YAPEAUSubstLookup@GSUB_impl@Layout@OT@@PEBUhb_ot_shape_plan_t@@PEAUhb_font_t@@AEAY00$$CBUligature_3_set_t@@I@Z 00000001800ddd4c     hb-ot-shaper-arabic.obj
 0002:00032d5c       $unwind$??$arabic_fallback_synthesize_lookup_ligature@$$BY0BC@Uligature_set_t@@@@YAPEAUSubstLookup@GSUB_impl@Layout@OT@@PEBUhb_ot_shape_plan_t@@PEAUhb_font_t@@AEAY0BC@$$CBUligature_set_t@@I@Z 00000001800ddd5c     hb-ot-shaper-arabic.obj
 0002:00032d80       $unwind$??$arabic_fallback_synthesize_lookup_ligature@$$BY00Uligature_mark_set_t@@@@YAPEAUSubstLookup@GSUB_impl@Layout@OT@@PEBUhb_ot_shape_plan_t@@PEAUhb_font_t@@AEAY00$$CBUligature_mark_set_t@@I@Z 00000001800ddd80     hb-ot-shaper-arabic.obj
 0002:00032da0       $chain$0$??$arabic_fallback_synthesize_lookup_ligature@$$BY00Uligature_mark_set_t@@@@YAPEAUSubstLookup@GSUB_impl@Layout@OT@@PEBUhb_ot_shape_plan_t@@PEAUhb_font_t@@AEAY00$$CBUligature_mark_set_t@@I@Z 00000001800ddda0     hb-ot-shaper-arabic.obj
 0002:00032db4       $chain$1$??$arabic_fallback_synthesize_lookup_ligature@$$BY00Uligature_mark_set_t@@@@YAPEAUSubstLookup@GSUB_impl@Layout@OT@@PEBUhb_ot_shape_plan_t@@PEAUhb_font_t@@AEAY00$$CBUligature_mark_set_t@@I@Z 00000001800dddb4     hb-ot-shaper-arabic.obj
 0002:00032dc4       $unwind$?arabic_fallback_plan_init_win1256@@YA_NPEAUarabic_fallback_plan_t@@PEBUhb_ot_shape_plan_t@@PEAUhb_font_t@@@Z 00000001800dddc4     hb-ot-shaper-arabic.obj
 0002:00032dd0       $chain$4$?arabic_fallback_plan_init_win1256@@YA_NPEAUarabic_fallback_plan_t@@PEBUhb_ot_shape_plan_t@@PEAUhb_font_t@@@Z 00000001800dddd0     hb-ot-shaper-arabic.obj
 0002:00032df4       $chain$6$?arabic_fallback_plan_init_win1256@@YA_NPEAUarabic_fallback_plan_t@@PEBUhb_ot_shape_plan_t@@PEAUhb_font_t@@@Z 00000001800dddf4     hb-ot-shaper-arabic.obj
 0002:00032e18       $chain$7$?arabic_fallback_plan_init_win1256@@YA_NPEAUarabic_fallback_plan_t@@PEBUhb_ot_shape_plan_t@@PEAUhb_font_t@@@Z 00000001800dde18     hb-ot-shaper-arabic.obj
 0002:00032e28       $unwind$?arabic_fallback_plan_init_unicode@@YA_NPEAUarabic_fallback_plan_t@@PEBUhb_ot_shape_plan_t@@PEAUhb_font_t@@@Z 00000001800dde28     hb-ot-shaper-arabic.obj
 0002:00032e44       $chain$0$?arabic_fallback_plan_destroy@@YAXPEAUarabic_fallback_plan_t@@@Z 00000001800dde44     hb-ot-shaper-arabic.obj
 0002:00032e58       $chain$2$?arabic_fallback_plan_destroy@@YAXPEAUarabic_fallback_plan_t@@@Z 00000001800dde58     hb-ot-shaper-arabic.obj
 0002:00032e70       $chain$3$?arabic_fallback_plan_destroy@@YAXPEAUarabic_fallback_plan_t@@@Z 00000001800dde70     hb-ot-shaper-arabic.obj
 0002:00032e80       $chain$4$?arabic_fallback_plan_destroy@@YAXPEAUarabic_fallback_plan_t@@@Z 00000001800dde80     hb-ot-shaper-arabic.obj
 0002:00032e90       $unwind$?arabic_joining@@YAXPEAUhb_buffer_t@@@Z 00000001800dde90     hb-ot-shaper-arabic.obj
 0002:00032ea8       $unwind$?apply_stch@@YAXPEBUhb_ot_shape_plan_t@@PEAUhb_buffer_t@@PEAUhb_font_t@@@Z 00000001800ddea8     hb-ot-shaper-arabic.obj
 0002:00032eb4       $chain$5$?apply_stch@@YAXPEBUhb_ot_shape_plan_t@@PEAUhb_buffer_t@@PEAUhb_font_t@@@Z 00000001800ddeb4     hb-ot-shaper-arabic.obj
 0002:00032edc       $chain$6$?apply_stch@@YAXPEBUhb_ot_shape_plan_t@@PEAUhb_buffer_t@@PEAUhb_font_t@@@Z 00000001800ddedc     hb-ot-shaper-arabic.obj
 0002:00032eec       $unwind$?reorder_marks_arabic@@YAXPEBUhb_ot_shape_plan_t@@PEAUhb_buffer_t@@II@Z 00000001800ddeec     hb-ot-shaper-arabic.obj
 0002:00032f10       $unwind$??$serialize_serialize@AEAU?$hb_sorted_array_t@$$CBUHBGlyphID16@OT@@@@@?$OffsetTo@UCoverage@Common@Layout@OT@@U?$IntType@G$01@4@X$00@OT@@QEAA_NPEAUhb_serialize_context_t@@AEAU?$hb_sorted_array_t@$$CBUHBGlyphID16@OT@@@@@Z 00000001800ddf10     hb-ot-shaper-arabic.obj
 0002:00032f20       $unwind$??$serialize@U?$hb_zip_iter_t@U?$hb_sorted_array_t@UHBGlyphID16@OT@@@@U?$hb_array_t@UHBGlyphID16@OT@@@@@@$0A@@SingleSubst@GSUB_impl@Layout@OT@@QEAA_NPEAUhb_serialize_context_t@@U?$hb_zip_iter_t@U?$hb_sorted_array_t@UHBGlyphID16@OT@@@@U?$hb_array_t@UHBGlyphID16@OT@@@@@@@Z 00000001800ddf20     hb-ot-shaper-arabic.obj
 0002:00032f38       $chain$3$??$serialize@U?$hb_zip_iter_t@U?$hb_sorted_array_t@UHBGlyphID16@OT@@@@U?$hb_array_t@UHBGlyphID16@OT@@@@@@$0A@@SingleSubst@GSUB_impl@Layout@OT@@QEAA_NPEAUhb_serialize_context_t@@U?$hb_zip_iter_t@U?$hb_sorted_array_t@UHBGlyphID16@OT@@@@U?$hb_array_t@UHBGlyphID16@OT@@@@@@@Z 00000001800ddf38     hb-ot-shaper-arabic.obj
 0002:00032f50       $chain$4$??$serialize@U?$hb_zip_iter_t@U?$hb_sorted_array_t@UHBGlyphID16@OT@@@@U?$hb_array_t@UHBGlyphID16@OT@@@@@@$0A@@SingleSubst@GSUB_impl@Layout@OT@@QEAA_NPEAUhb_serialize_context_t@@U?$hb_zip_iter_t@U?$hb_sorted_array_t@UHBGlyphID16@OT@@@@U?$hb_array_t@UHBGlyphID16@OT@@@@@@@Z 00000001800ddf50     hb-ot-shaper-arabic.obj
 0002:00032f64       $unwind$??$hb_stable_sort@UHBGlyphID16@OT@@U?$IntType@G$01@2@I@@YAXPEAUHBGlyphID16@OT@@IP6AHPEBU?$IntType@G$01@1@1@ZPEAI@Z 00000001800ddf64     hb-ot-shaper-arabic.obj
 0002:00032f70       $chain$5$??$hb_stable_sort@UHBGlyphID16@OT@@U?$IntType@G$01@2@I@@YAXPEAUHBGlyphID16@OT@@IP6AHPEBU?$IntType@G$01@1@1@ZPEAI@Z 00000001800ddf70     hb-ot-shaper-arabic.obj
 0002:00032f98       $chain$6$??$hb_stable_sort@UHBGlyphID16@OT@@U?$IntType@G$01@2@I@@YAXPEAUHBGlyphID16@OT@@IP6AHPEBU?$IntType@G$01@1@1@ZPEAI@Z 00000001800ddf98     hb-ot-shaper-arabic.obj
 0002:00032fa8       $unwind$??$serialize@U?$hb_sorted_array_t@$$CBUHBGlyphID16@OT@@@@$0A@@Coverage@Common@Layout@OT@@QEAA_NPEAUhb_serialize_context_t@@U?$hb_sorted_array_t@$$CBUHBGlyphID16@OT@@@@@Z 00000001800ddfa8     hb-ot-shaper-arabic.obj
 0002:00032fb4       $chain$4$??$serialize@U?$hb_sorted_array_t@$$CBUHBGlyphID16@OT@@@@$0A@@Coverage@Common@Layout@OT@@QEAA_NPEAUhb_serialize_context_t@@U?$hb_sorted_array_t@$$CBUHBGlyphID16@OT@@@@@Z 00000001800ddfb4     hb-ot-shaper-arabic.obj
 0002:00032fd8       $chain$5$??$serialize@U?$hb_sorted_array_t@$$CBUHBGlyphID16@OT@@@@$0A@@Coverage@Common@Layout@OT@@QEAA_NPEAUhb_serialize_context_t@@U?$hb_sorted_array_t@$$CBUHBGlyphID16@OT@@@@@Z 00000001800ddfd8     hb-ot-shaper-arabic.obj
 0002:00032fe8       $chain$0$??$extend_min@U?$CoverageFormat2_4@USmallTypes@Layout@OT@@@Common@Layout@OT@@@hb_serialize_context_t@@QEAAPEAU?$CoverageFormat2_4@USmallTypes@Layout@OT@@@Common@Layout@OT@@PEAU1234@@Z 00000001800ddfe8     hb-ot-shaper-arabic.obj
 0002:00032fe8       $chain$0$??$extend_min@U?$Ligature@USmallTypes@Layout@OT@@@GSUB_impl@Layout@OT@@@hb_serialize_context_t@@QEAAPEAU?$Ligature@USmallTypes@Layout@OT@@@GSUB_impl@Layout@OT@@PEAU1234@@Z 00000001800ddfe8     hb-ot-shaper-arabic.obj
 0002:00032ffc       $chain$2$??$extend_min@U?$CoverageFormat2_4@USmallTypes@Layout@OT@@@Common@Layout@OT@@@hb_serialize_context_t@@QEAAPEAU?$CoverageFormat2_4@USmallTypes@Layout@OT@@@Common@Layout@OT@@PEAU1234@@Z 00000001800ddffc     hb-ot-shaper-arabic.obj
 0002:00032ffc       $chain$2$??$extend_min@U?$Ligature@USmallTypes@Layout@OT@@@GSUB_impl@Layout@OT@@@hb_serialize_context_t@@QEAAPEAU?$Ligature@USmallTypes@Layout@OT@@@GSUB_impl@Layout@OT@@PEAU1234@@Z 00000001800ddffc     hb-ot-shaper-arabic.obj
 0002:00033010       $unwind$??$serialize_serialize@AEAU?$hb_map_iter_t@U?$hb_zip_iter_t@U?$hb_sorted_array_t@UHBGlyphID16@OT@@@@U?$hb_array_t@UHBGlyphID16@OT@@@@@@AEBU<unnamed-type-hb_first>@@$00$0A@@@@?$OffsetTo@UCoverage@Common@Layout@OT@@U?$IntType@G$01@4@X$00@OT@@QEAA_NPEAUhb_serialize_context_t@@AEAU?$hb_map_iter_t@U?$hb_zip_iter_t@U?$hb_sorted_array_t@UHBGlyphID16@OT@@@@U?$hb_array_t@UHBGlyphID16@OT@@@@@@AEBU<unnamed-type-hb_first>@@$00$0A@@@@Z 00000001800de010     hb-ot-shaper-arabic.obj
 0002:00033020       $unwind$??$serialize@U?$hb_map_iter_t@U?$hb_zip_iter_t@U?$hb_sorted_array_t@UHBGlyphID16@OT@@@@U?$hb_array_t@UHBGlyphID16@OT@@@@@@AEBU<unnamed-type-hb_first>@@$00$0A@@@$0A@@Coverage@Common@Layout@OT@@QEAA_NPEAUhb_serialize_context_t@@U?$hb_map_iter_t@U?$hb_zip_iter_t@U?$hb_sorted_array_t@UHBGlyphID16@OT@@@@U?$hb_array_t@UHBGlyphID16@OT@@@@@@AEBU<unnamed-type-hb_first>@@$00$0A@@@@Z 00000001800de020     hb-ot-shaper-arabic.obj
 0002:00033034       $chain$0$??$serialize@U?$hb_map_iter_t@U?$hb_zip_iter_t@U?$hb_sorted_array_t@UHBGlyphID16@OT@@@@U?$hb_array_t@UHBGlyphID16@OT@@@@@@AEBU<unnamed-type-hb_first>@@$00$0A@@@$0A@@Coverage@Common@Layout@OT@@QEAA_NPEAUhb_serialize_context_t@@U?$hb_map_iter_t@U?$hb_zip_iter_t@U?$hb_sorted_array_t@UHBGlyphID16@OT@@@@U?$hb_array_t@UHBGlyphID16@OT@@@@@@AEBU<unnamed-type-hb_first>@@$00$0A@@@@Z 00000001800de034     hb-ot-shaper-arabic.obj
 0002:00033048       $chain$2$??$serialize@U?$hb_map_iter_t@U?$hb_zip_iter_t@U?$hb_sorted_array_t@UHBGlyphID16@OT@@@@U?$hb_array_t@UHBGlyphID16@OT@@@@@@AEBU<unnamed-type-hb_first>@@$00$0A@@@$0A@@Coverage@Common@Layout@OT@@QEAA_NPEAUhb_serialize_context_t@@U?$hb_map_iter_t@U?$hb_zip_iter_t@U?$hb_sorted_array_t@UHBGlyphID16@OT@@@@U?$hb_array_t@UHBGlyphID16@OT@@@@@@AEBU<unnamed-type-hb_first>@@$00$0A@@@@Z 00000001800de048     hb-ot-shaper-arabic.obj
 0002:00033060       $chain$3$??$serialize@U?$hb_map_iter_t@U?$hb_zip_iter_t@U?$hb_sorted_array_t@UHBGlyphID16@OT@@@@U?$hb_array_t@UHBGlyphID16@OT@@@@@@AEBU<unnamed-type-hb_first>@@$00$0A@@@$0A@@Coverage@Common@Layout@OT@@QEAA_NPEAUhb_serialize_context_t@@U?$hb_map_iter_t@U?$hb_zip_iter_t@U?$hb_sorted_array_t@UHBGlyphID16@OT@@@@U?$hb_array_t@UHBGlyphID16@OT@@@@@@AEBU<unnamed-type-hb_first>@@$00$0A@@@@Z 00000001800de060     hb-ot-shaper-arabic.obj
 0002:00033070       $chain$4$??$serialize@U?$hb_map_iter_t@U?$hb_zip_iter_t@U?$hb_sorted_array_t@UHBGlyphID16@OT@@@@U?$hb_array_t@UHBGlyphID16@OT@@@@@@AEBU<unnamed-type-hb_first>@@$00$0A@@@$0A@@Coverage@Common@Layout@OT@@QEAA_NPEAUhb_serialize_context_t@@U?$hb_map_iter_t@U?$hb_zip_iter_t@U?$hb_sorted_array_t@UHBGlyphID16@OT@@@@U?$hb_array_t@UHBGlyphID16@OT@@@@@@AEBU<unnamed-type-hb_first>@@$00$0A@@@@Z 00000001800de070     hb-ot-shaper-arabic.obj
 0002:00033080       $unwind$??$serialize@U?$hb_map_iter_t@U?$hb_zip_iter_t@U?$hb_sorted_array_t@UHBGlyphID16@OT@@@@U?$hb_array_t@UHBGlyphID16@OT@@@@@@AEBU<unnamed-type-hb_first>@@$00$0A@@@$0A@@?$CoverageFormat2_4@USmallTypes@Layout@OT@@@Common@Layout@OT@@AEAA_NPEAUhb_serialize_context_t@@U?$hb_map_iter_t@U?$hb_zip_iter_t@U?$hb_sorted_array_t@UHBGlyphID16@OT@@@@U?$hb_array_t@UHBGlyphID16@OT@@@@@@AEBU<unnamed-type-hb_first>@@$00$0A@@@@Z 00000001800de080     hb-ot-shaper-arabic.obj
 0002:00033098       $unwind$?data_create_hangul@@YAPEAXPEBUhb_ot_shape_plan_t@@@Z 00000001800de098     hb-ot-shaper-hangul.obj
 0002:000330a8       $unwind$?preprocess_text_hangul@@YAXPEBUhb_ot_shape_plan_t@@PEAUhb_buffer_t@@PEAUhb_font_t@@@Z 00000001800de0a8     hb-ot-shaper-hangul.obj
 0002:000330c0       $chain$3$?preprocess_text_hangul@@YAXPEBUhb_ot_shape_plan_t@@PEAUhb_buffer_t@@PEAUhb_font_t@@@Z 00000001800de0c0     hb-ot-shaper-hangul.obj
 0002:000330e0       $chain$4$?preprocess_text_hangul@@YAXPEBUhb_ot_shape_plan_t@@PEAUhb_buffer_t@@PEAUhb_font_t@@@Z 00000001800de0e0     hb-ot-shaper-hangul.obj
 0002:000330f0       $unwind$?compose_hebrew@@YA_NPEBUhb_ot_shape_normalize_context_t@@IIPEAI@Z 00000001800de0f0     hb-ot-shaper-hebrew.obj
 0002:000330f0       $unwind$?compose_khmer@@YA_NPEBUhb_ot_shape_normalize_context_t@@IIPEAI@Z 00000001800de0f0     hb-ot-shaper-khmer.obj
 0002:000330f0       $unwind$?compose_use@@YA_NPEBUhb_ot_shape_normalize_context_t@@IIPEAI@Z 00000001800de0f0     hb-ot-shaper-use.obj
 0002:00033104       $unwind$?reorder_marks_hebrew@@YAXPEBUhb_ot_shape_plan_t@@PEAUhb_buffer_t@@II@Z 00000001800de104     hb-ot-shaper-hebrew.obj
 0002:00033110       $chain$2$?reorder_marks_hebrew@@YAXPEBUhb_ot_shape_plan_t@@PEAUhb_buffer_t@@II@Z 00000001800de110     hb-ot-shaper-hebrew.obj
 0002:0003312c       $chain$3$?reorder_marks_hebrew@@YAXPEBUhb_ot_shape_plan_t@@PEAUhb_buffer_t@@II@Z 00000001800de12c     hb-ot-shaper-hebrew.obj
 0002:0003313c       $unwind$?find_syllables_indic@@YAXPEAUhb_buffer_t@@@Z 00000001800de13c     hb-ot-shaper-indic.obj
 0002:0003313c       $unwind$?find_syllables_khmer@@YAXPEAUhb_buffer_t@@@Z 00000001800de13c     hb-ot-shaper-khmer.obj
 0002:0003313c       $unwind$?find_syllables_myanmar@@YAXPEAUhb_buffer_t@@@Z 00000001800de13c     hb-ot-shaper-myanmar.obj
 0002:0003313c       $unwind$?__forward__@?$hb_iter_fallback_mixin_t@U?$hb_filter_iter_t@U?$hb_filter_iter_t@U?$hb_zip_iter_t@U?$hb_iota_iter_t@II@@U?$hb_array_t@Uhb_glyph_info_t@@@@@@V<lambda_e52748becc06432fe81365edeb8c4003>@@AEBU<unnamed-type-hb_second>@@$0A@@@V<lambda_a2885d5959499a7c5bcf896c0de144bb>@@AEBU<unnamed-type-hb_identity>@@$0A@@@U?$hb_pair_t@IAEAUhb_glyph_info_t@@@@@@QEAAXI@Z 00000001800de13c     hb-ot-shaper-use.obj
 0002:0003313c       $unwind$?__rewind__@?$hb_iter_fallback_mixin_t@U?$hb_filter_iter_t@U?$hb_filter_iter_t@U?$hb_zip_iter_t@U?$hb_iota_iter_t@II@@U?$hb_array_t@Uhb_glyph_info_t@@@@@@V<lambda_e52748becc06432fe81365edeb8c4003>@@AEBU<unnamed-type-hb_second>@@$0A@@@V<lambda_a2885d5959499a7c5bcf896c0de144bb>@@AEBU<unnamed-type-hb_identity>@@$0A@@@U?$hb_pair_t@IAEAUhb_glyph_info_t@@@@@@QEAAXI@Z 00000001800de13c     hb-ot-shaper-use.obj
 0002:00033158       $unwind$?setup_syllables_indic@@YA_NPEBUhb_ot_shape_plan_t@@PEAUhb_font_t@@PEAUhb_buffer_t@@@Z 00000001800de158     hb-ot-shaper-indic.obj
 0002:00033158       $unwind$?setup_syllables_khmer@@YA_NPEBUhb_ot_shape_plan_t@@PEAUhb_font_t@@PEAUhb_buffer_t@@@Z 00000001800de158     hb-ot-shaper-khmer.obj
 0002:00033158       $unwind$?setup_syllables_myanmar@@YA_NPEBUhb_ot_shape_plan_t@@PEAUhb_font_t@@PEAUhb_buffer_t@@@Z 00000001800de158     hb-ot-shaper-myanmar.obj
 0002:00033164       $chain$2$?setup_syllables_indic@@YA_NPEBUhb_ot_shape_plan_t@@PEAUhb_font_t@@PEAUhb_buffer_t@@@Z 00000001800de164     hb-ot-shaper-indic.obj
 0002:00033180       $chain$4$?setup_syllables_indic@@YA_NPEBUhb_ot_shape_plan_t@@PEAUhb_font_t@@PEAUhb_buffer_t@@@Z 00000001800de180     hb-ot-shaper-indic.obj
 0002:00033194       $chain$5$?setup_syllables_indic@@YA_NPEBUhb_ot_shape_plan_t@@PEAUhb_font_t@@PEAUhb_buffer_t@@@Z 00000001800de194     hb-ot-shaper-indic.obj
 0002:000331a4       $unwind$?initial_reordering_indic@@YA_NPEBUhb_ot_shape_plan_t@@PEAUhb_font_t@@PEAUhb_buffer_t@@@Z 00000001800de1a4     hb-ot-shaper-indic.obj
 0002:000331c0       $chain$4$?initial_reordering_indic@@YA_NPEBUhb_ot_shape_plan_t@@PEAUhb_font_t@@PEAUhb_buffer_t@@@Z 00000001800de1c0     hb-ot-shaper-indic.obj
 0002:000331d4       $chain$5$?initial_reordering_indic@@YA_NPEBUhb_ot_shape_plan_t@@PEAUhb_font_t@@PEAUhb_buffer_t@@@Z 00000001800de1d4     hb-ot-shaper-indic.obj
 0002:000331e4       $unwind$?final_reordering_indic@@YA_NPEBUhb_ot_shape_plan_t@@PEAUhb_font_t@@PEAUhb_buffer_t@@@Z 00000001800de1e4     hb-ot-shaper-indic.obj
 0002:000331f4       $chain$0$?final_reordering_indic@@YA_NPEBUhb_ot_shape_plan_t@@PEAUhb_font_t@@PEAUhb_buffer_t@@@Z 00000001800de1f4     hb-ot-shaper-indic.obj
 0002:00033208       $chain$1$?final_reordering_indic@@YA_NPEBUhb_ot_shape_plan_t@@PEAUhb_font_t@@PEAUhb_buffer_t@@@Z 00000001800de208     hb-ot-shaper-indic.obj
 0002:0003321c       $chain$2$?final_reordering_indic@@YA_NPEBUhb_ot_shape_plan_t@@PEAUhb_font_t@@PEAUhb_buffer_t@@@Z 00000001800de21c     hb-ot-shaper-indic.obj
 0002:0003322c       $chain$3$?final_reordering_indic@@YA_NPEBUhb_ot_shape_plan_t@@PEAUhb_font_t@@PEAUhb_buffer_t@@@Z 00000001800de22c     hb-ot-shaper-indic.obj
 0002:0003323c       $unwind$?data_create_indic@@YAPEAXPEBUhb_ot_shape_plan_t@@@Z 00000001800de23c     hb-ot-shaper-indic.obj
 0002:0003324c       $chain$1$?data_create_indic@@YAPEAXPEBUhb_ot_shape_plan_t@@@Z 00000001800de24c     hb-ot-shaper-indic.obj
 0002:00033264       $chain$3$?data_create_indic@@YAPEAXPEBUhb_ot_shape_plan_t@@@Z 00000001800de264     hb-ot-shaper-indic.obj
 0002:0003327c       $unwind$?consonant_position_from_face@@YA?AW4ot_position_t@@PEBUindic_shape_plan_t@@IIPEAUhb_face_t@@@Z 00000001800de27c     hb-ot-shaper-indic.obj
 0002:00033294       $chain$0$?setup_masks_indic@@YAXPEBUhb_ot_shape_plan_t@@PEAUhb_buffer_t@@PEAUhb_font_t@@@Z 00000001800de294     hb-ot-shaper-indic.obj
 0002:000332a8       $chain$1$?setup_masks_indic@@YAXPEBUhb_ot_shape_plan_t@@PEAUhb_buffer_t@@PEAUhb_font_t@@@Z 00000001800de2a8     hb-ot-shaper-indic.obj
 0002:000332b8       $unwind$?initial_reordering_consonant_syllable@@YAXPEBUhb_ot_shape_plan_t@@PEAUhb_face_t@@PEAUhb_buffer_t@@II@Z 00000001800de2b8     hb-ot-shaper-indic.obj
 0002:000332d8       $unwind$?final_reordering_syllable_indic@@YAXPEBUhb_ot_shape_plan_t@@PEAUhb_buffer_t@@II@Z 00000001800de2d8     hb-ot-shaper-indic.obj
 0002:000332e4       $chain$4$?final_reordering_syllable_indic@@YAXPEBUhb_ot_shape_plan_t@@PEAUhb_buffer_t@@II@Z 00000001800de2e4     hb-ot-shaper-indic.obj
 0002:00033308       $chain$5$?final_reordering_syllable_indic@@YAXPEBUhb_ot_shape_plan_t@@PEAUhb_buffer_t@@II@Z 00000001800de308     hb-ot-shaper-indic.obj
 0002:0003331c       $chain$6$?final_reordering_syllable_indic@@YAXPEBUhb_ot_shape_plan_t@@PEAUhb_buffer_t@@II@Z 00000001800de31c     hb-ot-shaper-indic.obj
 0002:0003332c       $chain$2$?setup_syllables_khmer@@YA_NPEBUhb_ot_shape_plan_t@@PEAUhb_font_t@@PEAUhb_buffer_t@@@Z 00000001800de32c     hb-ot-shaper-khmer.obj
 0002:00033348       $chain$4$?setup_syllables_khmer@@YA_NPEBUhb_ot_shape_plan_t@@PEAUhb_font_t@@PEAUhb_buffer_t@@@Z 00000001800de348     hb-ot-shaper-khmer.obj
 0002:0003335c       $chain$5$?setup_syllables_khmer@@YA_NPEBUhb_ot_shape_plan_t@@PEAUhb_font_t@@PEAUhb_buffer_t@@@Z 00000001800de35c     hb-ot-shaper-khmer.obj
 0002:0003336c       $unwind$?reorder_khmer@@YA_NPEBUhb_ot_shape_plan_t@@PEAUhb_font_t@@PEAUhb_buffer_t@@@Z 00000001800de36c     hb-ot-shaper-khmer.obj
 0002:0003337c       $chain$1$?reorder_khmer@@YA_NPEBUhb_ot_shape_plan_t@@PEAUhb_font_t@@PEAUhb_buffer_t@@@Z 00000001800de37c     hb-ot-shaper-khmer.obj
 0002:00033394       $chain$2$?reorder_khmer@@YA_NPEBUhb_ot_shape_plan_t@@PEAUhb_font_t@@PEAUhb_buffer_t@@@Z 00000001800de394     hb-ot-shaper-khmer.obj
 0002:000333a4       $unwind$?data_create_khmer@@YAPEAXPEBUhb_ot_shape_plan_t@@@Z 00000001800de3a4     hb-ot-shaper-khmer.obj
 0002:000333b0       $chain$2$?data_create_khmer@@YAPEAXPEBUhb_ot_shape_plan_t@@@Z 00000001800de3b0     hb-ot-shaper-khmer.obj
 0002:000333cc       $chain$4$?data_create_khmer@@YAPEAXPEBUhb_ot_shape_plan_t@@@Z 00000001800de3cc     hb-ot-shaper-khmer.obj
 0002:000333e8       $chain$0$?setup_masks_khmer@@YAXPEBUhb_ot_shape_plan_t@@PEAUhb_buffer_t@@PEAUhb_font_t@@@Z 00000001800de3e8     hb-ot-shaper-khmer.obj
 0002:000333fc       $chain$1$?setup_masks_khmer@@YAXPEBUhb_ot_shape_plan_t@@PEAUhb_buffer_t@@PEAUhb_font_t@@@Z 00000001800de3fc     hb-ot-shaper-khmer.obj
 0002:0003340c       $unwind$?reorder_consonant_syllable@@YAXPEBUhb_ot_shape_plan_t@@PEAUhb_face_t@@PEAUhb_buffer_t@@II@Z 00000001800de40c     hb-ot-shaper-khmer.obj
 0002:00033418       $chain$4$?reorder_consonant_syllable@@YAXPEBUhb_ot_shape_plan_t@@PEAUhb_face_t@@PEAUhb_buffer_t@@II@Z 00000001800de418     hb-ot-shaper-khmer.obj
 0002:0003343c       $chain$5$?reorder_consonant_syllable@@YAXPEBUhb_ot_shape_plan_t@@PEAUhb_face_t@@PEAUhb_buffer_t@@II@Z 00000001800de43c     hb-ot-shaper-khmer.obj
 0002:0003344c       $chain$2$?setup_syllables_myanmar@@YA_NPEBUhb_ot_shape_plan_t@@PEAUhb_font_t@@PEAUhb_buffer_t@@@Z 00000001800de44c     hb-ot-shaper-myanmar.obj
 0002:00033468       $chain$4$?setup_syllables_myanmar@@YA_NPEBUhb_ot_shape_plan_t@@PEAUhb_font_t@@PEAUhb_buffer_t@@@Z 00000001800de468     hb-ot-shaper-myanmar.obj
 0002:0003347c       $chain$5$?setup_syllables_myanmar@@YA_NPEBUhb_ot_shape_plan_t@@PEAUhb_font_t@@PEAUhb_buffer_t@@@Z 00000001800de47c     hb-ot-shaper-myanmar.obj
 0002:0003348c       $unwind$?reorder_myanmar@@YA_NPEBUhb_ot_shape_plan_t@@PEAUhb_font_t@@PEAUhb_buffer_t@@@Z 00000001800de48c     hb-ot-shaper-myanmar.obj
 0002:0003348c       $unwind$?reorder_use@@YA_NPEBUhb_ot_shape_plan_t@@PEAUhb_font_t@@PEAUhb_buffer_t@@@Z 00000001800de48c     hb-ot-shaper-use.obj
 0002:0003349c       $chain$1$?reorder_myanmar@@YA_NPEBUhb_ot_shape_plan_t@@PEAUhb_font_t@@PEAUhb_buffer_t@@@Z 00000001800de49c     hb-ot-shaper-myanmar.obj
 0002:000334b4       $chain$2$?reorder_myanmar@@YA_NPEBUhb_ot_shape_plan_t@@PEAUhb_font_t@@PEAUhb_buffer_t@@@Z 00000001800de4b4     hb-ot-shaper-myanmar.obj
 0002:000334c4       $chain$0$?setup_masks_myanmar@@YAXPEBUhb_ot_shape_plan_t@@PEAUhb_buffer_t@@PEAUhb_font_t@@@Z 00000001800de4c4     hb-ot-shaper-myanmar.obj
 0002:000334d8       $chain$1$?setup_masks_myanmar@@YAXPEBUhb_ot_shape_plan_t@@PEAUhb_buffer_t@@PEAUhb_font_t@@@Z 00000001800de4d8     hb-ot-shaper-myanmar.obj
 0002:000334e8       $unwind$?hb_syllabic_insert_dotted_circles@@YA_NPEAUhb_font_t@@PEAUhb_buffer_t@@IIHH@Z 00000001800de4e8     hb-ot-shaper-syllabic.obj
 0002:000334f8       $chain$1$?hb_syllabic_insert_dotted_circles@@YA_NPEAUhb_font_t@@PEAUhb_buffer_t@@IIHH@Z 00000001800de4f8     hb-ot-shaper-syllabic.obj
 0002:00033510       $chain$2$?hb_syllabic_insert_dotted_circles@@YA_NPEAUhb_font_t@@PEAUhb_buffer_t@@IIHH@Z 00000001800de510     hb-ot-shaper-syllabic.obj
 0002:00033520       $unwind$?do_thai_pua_shaping@@YAXPEBUhb_ot_shape_plan_t@@PEAUhb_buffer_t@@PEAUhb_font_t@@@Z 00000001800de520     hb-ot-shaper-thai.obj
 0002:00033530       $chain$3$?do_thai_pua_shaping@@YAXPEBUhb_ot_shape_plan_t@@PEAUhb_buffer_t@@PEAUhb_font_t@@@Z 00000001800de530     hb-ot-shaper-thai.obj
 0002:00033550       $chain$4$?do_thai_pua_shaping@@YAXPEBUhb_ot_shape_plan_t@@PEAUhb_buffer_t@@PEAUhb_font_t@@@Z 00000001800de550     hb-ot-shaper-thai.obj
 0002:00033560       $unwind$?preprocess_text_thai@@YAXPEBUhb_ot_shape_plan_t@@PEAUhb_buffer_t@@PEAUhb_font_t@@@Z 00000001800de560     hb-ot-shaper-thai.obj
 0002:0003356c       $chain$1$?preprocess_text_thai@@YAXPEBUhb_ot_shape_plan_t@@PEAUhb_buffer_t@@PEAUhb_font_t@@@Z 00000001800de56c     hb-ot-shaper-thai.obj
 0002:00033584       $chain$4$?preprocess_text_thai@@YAXPEBUhb_ot_shape_plan_t@@PEAUhb_buffer_t@@PEAUhb_font_t@@@Z 00000001800de584     hb-ot-shaper-thai.obj
 0002:000335a0       $chain$5$?preprocess_text_thai@@YAXPEBUhb_ot_shape_plan_t@@PEAUhb_buffer_t@@PEAUhb_font_t@@@Z 00000001800de5a0     hb-ot-shaper-thai.obj
 0002:000335b0       $chain$6$?preprocess_text_thai@@YAXPEBUhb_ot_shape_plan_t@@PEAUhb_buffer_t@@PEAUhb_font_t@@@Z 00000001800de5b0     hb-ot-shaper-thai.obj
 0002:000335c0       $unwind$?find_syllables_use@@YAXPEAUhb_buffer_t@@@Z 00000001800de5c0     hb-ot-shaper-use.obj
 0002:000335e8       $unwind$??D?$hb_iter_t@U?$hb_zip_iter_t@U?$hb_iota_iter_t@II@@U?$hb_filter_iter_t@U?$hb_filter_iter_t@U?$hb_zip_iter_t@U?$hb_iota_iter_t@II@@U?$hb_array_t@Uhb_glyph_info_t@@@@@@V<lambda_e52748becc06432fe81365edeb8c4003>@@AEBU<unnamed-type-hb_second>@@$0A@@@V<lambda_a2885d5959499a7c5bcf896c0de144bb>@@AEBU<unnamed-type-hb_identity>@@$0A@@@@@U?$hb_pair_t@IU?$hb_pair_t@IAEAUhb_glyph_info_t@@@@@@@@QEBA?AU?$hb_pair_t@IU?$hb_pair_t@IAEAUhb_glyph_info_t@@@@@@XZ 00000001800de5e8     hb-ot-shaper-use.obj
 0002:000335f0       $unwind$?setup_syllables_use@@YA_NPEBUhb_ot_shape_plan_t@@PEAUhb_font_t@@PEAUhb_buffer_t@@@Z 00000001800de5f0     hb-ot-shaper-use.obj
 0002:00033604       $chain$1$?setup_syllables_use@@YA_NPEBUhb_ot_shape_plan_t@@PEAUhb_font_t@@PEAUhb_buffer_t@@@Z 00000001800de604     hb-ot-shaper-use.obj
 0002:0003361c       $chain$2$?setup_syllables_use@@YA_NPEBUhb_ot_shape_plan_t@@PEAUhb_font_t@@PEAUhb_buffer_t@@@Z 00000001800de61c     hb-ot-shaper-use.obj
 0002:0003362c       $unwind$?record_rphf_use@@YA_NPEBUhb_ot_shape_plan_t@@PEAUhb_font_t@@PEAUhb_buffer_t@@@Z 00000001800de62c     hb-ot-shaper-use.obj
 0002:00033638       $chain$1$?record_rphf_use@@YA_NPEBUhb_ot_shape_plan_t@@PEAUhb_font_t@@PEAUhb_buffer_t@@@Z 00000001800de638     hb-ot-shaper-use.obj
 0002:00033650       $chain$2$?record_rphf_use@@YA_NPEBUhb_ot_shape_plan_t@@PEAUhb_font_t@@PEAUhb_buffer_t@@@Z 00000001800de650     hb-ot-shaper-use.obj
 0002:00033660       $chain$1$?reorder_use@@YA_NPEBUhb_ot_shape_plan_t@@PEAUhb_font_t@@PEAUhb_buffer_t@@@Z 00000001800de660     hb-ot-shaper-use.obj
 0002:00033678       $chain$2$?reorder_use@@YA_NPEBUhb_ot_shape_plan_t@@PEAUhb_font_t@@PEAUhb_buffer_t@@@Z 00000001800de678     hb-ot-shaper-use.obj
 0002:00033688       $unwind$?setup_topographical_masks@@YAXPEBUhb_ot_shape_plan_t@@PEAUhb_buffer_t@@@Z 00000001800de688     hb-ot-shaper-use.obj
 0002:00033698       $chain$4$?setup_topographical_masks@@YAXPEBUhb_ot_shape_plan_t@@PEAUhb_buffer_t@@@Z 00000001800de698     hb-ot-shaper-use.obj
 0002:000336bc       $chain$6$?setup_topographical_masks@@YAXPEBUhb_ot_shape_plan_t@@PEAUhb_buffer_t@@@Z 00000001800de6bc     hb-ot-shaper-use.obj
 0002:000336d4       $chain$10$?setup_topographical_masks@@YAXPEBUhb_ot_shape_plan_t@@PEAUhb_buffer_t@@@Z 00000001800de6d4     hb-ot-shaper-use.obj
 0002:000336d4       $chain$7$?setup_topographical_masks@@YAXPEBUhb_ot_shape_plan_t@@PEAUhb_buffer_t@@@Z 00000001800de6d4     hb-ot-shaper-use.obj
 0002:000336e4       $chain$8$?setup_topographical_masks@@YAXPEBUhb_ot_shape_plan_t@@PEAUhb_buffer_t@@@Z 00000001800de6e4     hb-ot-shaper-use.obj
 0002:000336fc       $chain$9$?setup_topographical_masks@@YAXPEBUhb_ot_shape_plan_t@@PEAUhb_buffer_t@@@Z 00000001800de6fc     hb-ot-shaper-use.obj
 0002:00033710       $chain$11$?setup_topographical_masks@@YAXPEBUhb_ot_shape_plan_t@@PEAUhb_buffer_t@@@Z 00000001800de710     hb-ot-shaper-use.obj
 0002:00033720       $unwind$?reorder_syllable_use@@YAXPEAUhb_buffer_t@@II@Z 00000001800de720     hb-ot-shaper-use.obj
 0002:00033730       $chain$1$?reorder_syllable_use@@YAXPEAUhb_buffer_t@@II@Z 00000001800de730     hb-ot-shaper-use.obj
 0002:00033748       $chain$2$?reorder_syllable_use@@YAXPEAUhb_buffer_t@@II@Z 00000001800de748     hb-ot-shaper-use.obj
 0002:0003375c       $chain$3$?reorder_syllable_use@@YAXPEAUhb_buffer_t@@II@Z 00000001800de75c     hb-ot-shaper-use.obj
 0002:0003375c       $chain$5$?reorder_syllable_use@@YAXPEAUhb_buffer_t@@II@Z 00000001800de75c     hb-ot-shaper-use.obj
 0002:0003376c       $chain$4$?reorder_syllable_use@@YAXPEAUhb_buffer_t@@II@Z 00000001800de76c     hb-ot-shaper-use.obj
 0002:00033780       $chain$6$?reorder_syllable_use@@YAXPEAUhb_buffer_t@@II@Z 00000001800de780     hb-ot-shaper-use.obj
 0002:00033790       $chain$2$?_hb_preprocess_text_vowel_constraints@@YAXPEBUhb_ot_shape_plan_t@@PEAUhb_buffer_t@@PEAUhb_font_t@@@Z 00000001800de790     hb-ot-shaper-vowel-constraints.obj
 0002:000337ac       $chain$3$?_hb_preprocess_text_vowel_constraints@@YAXPEBUhb_ot_shape_plan_t@@PEAUhb_buffer_t@@PEAUhb_font_t@@@Z 00000001800de7ac     hb-ot-shaper-vowel-constraints.obj
 0002:000337bc       $unwind$hb_ot_tags_from_script_and_language 00000001800de7bc     hb-ot-tag.obj
 0002:000337cc       $chain$3$hb_ot_tags_from_script_and_language 00000001800de7cc     hb-ot-tag.obj
 0002:000337ec       $chain$4$hb_ot_tags_from_script_and_language 00000001800de7ec     hb-ot-tag.obj
 0002:000337ec       $chain$6$hb_ot_tags_from_script_and_language 00000001800de7ec     hb-ot-tag.obj
 0002:000337fc       $chain$5$hb_ot_tags_from_script_and_language 00000001800de7fc     hb-ot-tag.obj
 0002:0003381c       $unwind$hb_ot_tag_to_language 00000001800de81c     hb-ot-tag.obj
 0002:0003382c       $unwind$?hb_ot_tags_from_complex_language@@YA_NPEBD0PEAI1@Z 00000001800de82c     hb-ot-tag.obj
 0002:00033840       $chain$0$?hb_ot_tags_from_complex_language@@YA_NPEBD0PEAI1@Z 00000001800de840     hb-ot-tag.obj
 0002:00033854       $chain$2$?hb_ot_tags_from_complex_language@@YA_NPEBD0PEAI1@Z 00000001800de854     hb-ot-tag.obj
 0002:00033868       $unwind$?hb_ot_tags_from_language@@YAXPEBD0PEAI1@Z 00000001800de868     hb-ot-tag.obj
 0002:00033878       $chain$3$?hb_ot_tags_from_language@@YAXPEBD0PEAI1@Z 00000001800de878     hb-ot-tag.obj
 0002:00033898       $chain$4$?hb_ot_tags_from_language@@YAXPEBD0PEAI1@Z 00000001800de898     hb-ot-tag.obj
 0002:000338a8       $unwind$hb_ot_var_normalize_coords 00000001800de8a8     hb-ot-var.obj
 0002:000338bc       $chain$4$hb_ot_var_normalize_coords 00000001800de8bc     hb-ot-var.obj
 0002:000338e0       $chain$5$hb_ot_var_normalize_coords 00000001800de8e0     hb-ot-var.obj
 0002:000338f0       $chain$1$??C?$hb_lazy_loader_t@Uavar@OT@@U?$hb_table_lazy_loader_t@Uavar@OT@@$0BD@$00@@Uhb_face_t@@$0BD@Uhb_blob_t@@@@QEBAPEBUavar@OT@@XZ 00000001800de8f0     hb-ot-var.obj
 0002:00033908       $chain$2$??C?$hb_lazy_loader_t@Uavar@OT@@U?$hb_table_lazy_loader_t@Uavar@OT@@$0BD@$00@@Uhb_face_t@@$0BD@Uhb_blob_t@@@@QEBAPEBUavar@OT@@XZ 00000001800de908     hb-ot-var.obj
 0002:00033918       $unwind$?map_coords@avar@OT@@QEBAXPEAHI@Z 00000001800de918     hb-ot-var.obj
 0002:00033928       $chain$1$?map_coords@avar@OT@@QEBAXPEAHI@Z 00000001800de928     hb-ot-var.obj
 0002:00033940       $chain$3$?map_coords@avar@OT@@QEBAXPEAHI@Z 00000001800de940     hb-ot-var.obj
 0002:00033958       $chain$4$?map_coords@avar@OT@@QEBAXPEAHI@Z 00000001800de958     hb-ot-var.obj
 0002:00033958       $chain$6$?map_coords@avar@OT@@QEBAXPEAHI@Z 00000001800de958     hb-ot-var.obj
 0002:00033968       $chain$5$?map_coords@avar@OT@@QEBAXPEAHI@Z 00000001800de968     hb-ot-var.obj
 0002:00033980       $chain$7$?map_coords@avar@OT@@QEBAXPEAHI@Z 00000001800de980     hb-ot-var.obj
 0002:00033990       $unwind$?replay@hb_outline_t@@QEBAXPEAUhb_draw_funcs_t@@PEAX@Z 00000001800de990     hb-outline.obj
 0002:000339a8       $chain$5$?replay@hb_outline_t@@QEBAXPEAUhb_draw_funcs_t@@PEAX@Z 00000001800de9a8     hb-outline.obj
 0002:000339d0       $chain$6$?replay@hb_outline_t@@QEBAXPEAUhb_draw_funcs_t@@PEAX@Z 00000001800de9d0     hb-outline.obj
 0002:000339e0       $unwind$?control_area@hb_outline_t@@QEBAMXZ 00000001800de9e0     hb-outline.obj
 0002:000339ec       $chain$4$?control_area@hb_outline_t@@QEBAMXZ 00000001800de9ec     hb-outline.obj
 0002:00033a10       $chain$5$?control_area@hb_outline_t@@QEBAMXZ 00000001800dea10     hb-outline.obj
 0002:00033a20       $unwind$?embolden@hb_outline_t@@QEAAXMMMM@Z 00000001800dea20     hb-outline.obj
 0002:00033a34       $chain$1$?embolden@hb_outline_t@@QEAAXMMMM@Z 00000001800dea34     hb-outline.obj
 0002:00033a4c       $chain$14$?embolden@hb_outline_t@@QEAAXMMMM@Z 00000001800dea4c     hb-outline.obj
 0002:00033a90       $chain$15$?embolden@hb_outline_t@@QEAAXMMMM@Z 00000001800dea90     hb-outline.obj
 0002:00033aa0       $chain$16$?embolden@hb_outline_t@@QEAAXMMMM@Z 00000001800deaa0     hb-outline.obj
 0002:00033ab0       $chain$0$?hb_outline_recording_pen_get_funcs@@YAPEAUhb_draw_funcs_t@@XZ 00000001800deab0     hb-outline.obj
 0002:00033ac4       $chain$2$?hb_outline_recording_pen_get_funcs@@YAPEAUhb_draw_funcs_t@@XZ 00000001800deac4     hb-outline.obj
 0002:00033ad8       $chain$3$?hb_outline_recording_pen_get_funcs@@YAPEAUhb_draw_funcs_t@@XZ 00000001800dead8     hb-outline.obj
 0002:00033ae8       $unwind$?hb_outline_recording_pen_cubic_to@@YAXPEAUhb_draw_funcs_t@@PEAXPEAUhb_draw_state_t@@MMMMMM1@Z 00000001800deae8     hb-outline.obj
 0002:00033ae8       $unwind$?hb_outline_recording_pen_line_to@@YAXPEAUhb_draw_funcs_t@@PEAXPEAUhb_draw_state_t@@MM1@Z 00000001800deae8     hb-outline.obj
 0002:00033ae8       $unwind$?hb_outline_recording_pen_move_to@@YAXPEAUhb_draw_funcs_t@@PEAXPEAUhb_draw_state_t@@MM1@Z 00000001800deae8     hb-outline.obj
 0002:00033ae8       $unwind$?hb_outline_recording_pen_quadratic_to@@YAXPEAUhb_draw_funcs_t@@PEAXPEAUhb_draw_state_t@@MMMM1@Z 00000001800deae8     hb-outline.obj
 0002:00033af4       $chain$0$?hb_paint_bounded_get_funcs@@YAPEAUhb_paint_funcs_t@@XZ 00000001800deaf4     hb-paint-bounded.obj
 0002:00033b08       $chain$2$?hb_paint_bounded_get_funcs@@YAPEAUhb_paint_funcs_t@@XZ 00000001800deb08     hb-paint-bounded.obj
 0002:00033b1c       $chain$3$?hb_paint_bounded_get_funcs@@YAPEAUhb_paint_funcs_t@@XZ 00000001800deb1c     hb-paint-bounded.obj
 0002:00033b2c       $unwind$?transform_extents@hb_transform_t@@QEBAXAEAUhb_extents_t@@@Z 00000001800deb2c     hb-paint-extents.obj
 0002:00033b44       $chain$0$?intersect@hb_bounds_t@@QEAAXAEBU1@@Z 00000001800deb44     hb-paint-extents.obj
 0002:00033b58       $chain$1$?intersect@hb_bounds_t@@QEAAXAEBU1@@Z 00000001800deb58     hb-paint-extents.obj
 0002:00033b68       $chain$0$?pop_group@hb_paint_extents_context_t@@QEAAXW4hb_paint_composite_mode_t@@@Z 00000001800deb68     hb-paint-extents.obj
 0002:00033b7c       $chain$2$?pop_group@hb_paint_extents_context_t@@QEAAXW4hb_paint_composite_mode_t@@@Z 00000001800deb7c     hb-paint-extents.obj
 0002:00033b90       $chain$3$?pop_group@hb_paint_extents_context_t@@QEAAXW4hb_paint_composite_mode_t@@@Z 00000001800deb90     hb-paint-extents.obj
 0002:00033ba0       $chain$0$?hb_paint_extents_get_funcs@@YAPEAUhb_paint_funcs_t@@XZ 00000001800deba0     hb-paint-extents.obj
 0002:00033bb4       $chain$2$?hb_paint_extents_get_funcs@@YAPEAUhb_paint_funcs_t@@XZ 00000001800debb4     hb-paint-extents.obj
 0002:00033bc8       $chain$3$?hb_paint_extents_get_funcs@@YAPEAUhb_paint_funcs_t@@XZ 00000001800debc8     hb-paint-extents.obj
 0002:00033bd8       $unwind$?hb_paint_extents_push_transform@@YAXPEAUhb_paint_funcs_t@@PEAXMMMMMM1@Z 00000001800debd8     hb-paint-extents.obj
 0002:00033bec       $chain$5$?hb_paint_extents_push_transform@@YAXPEAUhb_paint_funcs_t@@PEAXMMMMMM1@Z 00000001800debec     hb-paint-extents.obj
 0002:00033c14       $chain$6$?hb_paint_extents_push_transform@@YAXPEAUhb_paint_funcs_t@@PEAXMMMMMM1@Z 00000001800dec14     hb-paint-extents.obj
 0002:00033c24       $chain$1$hb_paint_funcs_destroy 00000001800dec24     hb-paint.obj
 0002:00033c3c       $chain$2$hb_paint_funcs_destroy 00000001800dec3c     hb-paint.obj
 0002:00033c50       $chain$3$hb_paint_funcs_destroy 00000001800dec50     hb-paint.obj
 0002:00033c60       $chain$0$hb_paint_funcs_set_push_transform_func 00000001800dec60     hb-paint.obj
 0002:00033c74       $chain$1$hb_paint_funcs_set_push_transform_func 00000001800dec74     hb-paint.obj
 0002:00033c84       $chain$0$hb_paint_funcs_set_pop_transform_func 00000001800dec84     hb-paint.obj
 0002:00033c98       $chain$1$hb_paint_funcs_set_pop_transform_func 00000001800dec98     hb-paint.obj
 0002:00033ca8       $chain$0$hb_paint_funcs_set_push_clip_glyph_func 00000001800deca8     hb-paint.obj
 0002:00033cbc       $chain$1$hb_paint_funcs_set_push_clip_glyph_func 00000001800decbc     hb-paint.obj
 0002:00033ccc       $chain$0$hb_paint_funcs_set_push_clip_rectangle_func 00000001800deccc     hb-paint.obj
 0002:00033ce0       $chain$1$hb_paint_funcs_set_push_clip_rectangle_func 00000001800dece0     hb-paint.obj
 0002:00033cf0       $chain$0$hb_paint_funcs_set_pop_clip_func 00000001800decf0     hb-paint.obj
 0002:00033d04       $chain$1$hb_paint_funcs_set_pop_clip_func 00000001800ded04     hb-paint.obj
 0002:00033d14       $chain$0$hb_paint_funcs_set_color_func 00000001800ded14     hb-paint.obj
 0002:00033d28       $chain$1$hb_paint_funcs_set_color_func 00000001800ded28     hb-paint.obj
 0002:00033d38       $chain$0$hb_paint_funcs_set_image_func 00000001800ded38     hb-paint.obj
 0002:00033d4c       $chain$1$hb_paint_funcs_set_image_func 00000001800ded4c     hb-paint.obj
 0002:00033d5c       $chain$0$hb_paint_funcs_set_linear_gradient_func 00000001800ded5c     hb-paint.obj
 0002:00033d70       $chain$1$hb_paint_funcs_set_linear_gradient_func 00000001800ded70     hb-paint.obj
 0002:00033d80       $chain$0$hb_paint_funcs_set_radial_gradient_func 00000001800ded80     hb-paint.obj
 0002:00033d94       $chain$1$hb_paint_funcs_set_radial_gradient_func 00000001800ded94     hb-paint.obj
 0002:00033da4       $chain$0$hb_paint_funcs_set_sweep_gradient_func 00000001800deda4     hb-paint.obj
 0002:00033db8       $chain$1$hb_paint_funcs_set_sweep_gradient_func 00000001800dedb8     hb-paint.obj
 0002:00033dc8       $chain$0$hb_paint_funcs_set_push_group_func 00000001800dedc8     hb-paint.obj
 0002:00033ddc       $chain$1$hb_paint_funcs_set_push_group_func 00000001800deddc     hb-paint.obj
 0002:00033dec       $chain$0$hb_paint_funcs_set_pop_group_func 00000001800dedec     hb-paint.obj
 0002:00033e00       $chain$1$hb_paint_funcs_set_pop_group_func 00000001800dee00     hb-paint.obj
 0002:00033e10       $unwind$hb_shape_plan_create2 00000001800dee10     hb-shape-plan.obj
 0002:00033e28       $chain$0$hb_shape_plan_create2 00000001800dee28     hb-shape-plan.obj
 0002:00033e3c       $chain$1$hb_shape_plan_create2 00000001800dee3c     hb-shape-plan.obj
 0002:00033e4c       $chain$2$hb_shape_plan_create2 00000001800dee4c     hb-shape-plan.obj
 0002:00033e60       $unwind$hb_shape_plan_create_cached2 00000001800dee60     hb-shape-plan.obj
 0002:00033e80       $chain$0$hb_shape_plan_destroy 00000001800dee80     hb-shape-plan.obj
 0002:00033e94       $chain$1$hb_shape_plan_destroy 00000001800dee94     hb-shape-plan.obj
 0002:00033ea4       $unwind$??1?$hb_vector_t@U?$hb_vector_t@Urange_flags_t@hb_aat_map_t@@$00@@$0A@@@QEAA@XZ 00000001800deea4     hb-shape-plan.obj
 0002:00033eb4       $chain$1$??1?$hb_vector_t@U?$hb_vector_t@Urange_flags_t@hb_aat_map_t@@$00@@$0A@@@QEAA@XZ 00000001800deeb4     hb-shape-plan.obj
 0002:00033ecc       $chain$3$??1?$hb_vector_t@U?$hb_vector_t@Urange_flags_t@hb_aat_map_t@@$00@@$0A@@@QEAA@XZ 00000001800deecc     hb-shape-plan.obj
 0002:00033ee4       $chain$4$??1?$hb_vector_t@U?$hb_vector_t@Urange_flags_t@hb_aat_map_t@@$00@@$0A@@@QEAA@XZ 00000001800deee4     hb-shape-plan.obj
 0002:00033ef4       $chain$5$??1?$hb_vector_t@U?$hb_vector_t@Urange_flags_t@hb_aat_map_t@@$00@@$0A@@@QEAA@XZ 00000001800deef4     hb-shape-plan.obj
 0002:00033f04       $unwind$?init@hb_shape_plan_key_t@@QEAA_N_NPEAUhb_face_t@@PEBUhb_segment_properties_t@@PEBUhb_feature_t@@IPEBHIPEBQEBD@Z 00000001800def04     hb-shape-plan.obj
 0002:00033f1c       $chain$0$?init@hb_shape_plan_key_t@@QEAA_N_NPEAUhb_face_t@@PEBUhb_segment_properties_t@@PEBUhb_feature_t@@IPEBHIPEBQEBD@Z 00000001800def1c     hb-shape-plan.obj
 0002:00033f30       $chain$1$?init@hb_shape_plan_key_t@@QEAA_N_NPEAUhb_face_t@@PEBUhb_segment_properties_t@@PEBUhb_feature_t@@IPEBHIPEBQEBD@Z 00000001800def30     hb-shape-plan.obj
 0002:00033f40       $unwind$?_hb_shape_plan_execute_internal@@YA_NPEAUhb_shape_plan_t@@PEAUhb_font_t@@PEAUhb_buffer_t@@PEBUhb_feature_t@@I@Z 00000001800def40     hb-shape-plan.obj
 0002:00033f54       $unwind$hb_shape_full      00000001800def54     hb-shape.obj
 0002:00033f6c       $chain$3$hb_shape_full     00000001800def6c     hb-shape.obj
 0002:00033f84       $chain$4$hb_shape_full     00000001800def84     hb-shape.obj
 0002:00033f98       $unwind$?get_stored@?$hb_lazy_loader_t@Uhb_shaper_entry_t@@Uhb_shapers_lazy_loader_t@@X$0A@U1@@@QEBAPEAUhb_shaper_entry_t@@XZ 00000001800def98     hb-shaper.obj
 0002:00033fa0       $chain$6$?get_stored@?$hb_lazy_loader_t@Uhb_shaper_entry_t@@Uhb_shapers_lazy_loader_t@@X$0A@U1@@@QEBAPEAUhb_shaper_entry_t@@XZ 00000001800defa0     hb-shaper.obj
 0002:00033fcc       $chain$7$?get_stored@?$hb_lazy_loader_t@Uhb_shaper_entry_t@@Uhb_shapers_lazy_loader_t@@X$0A@U1@@@QEBAPEAUhb_shaper_entry_t@@XZ 00000001800defcc     hb-shaper.obj
 0002:00033fdc       $chain$0$hb_ucd_get_unicode_funcs 00000001800defdc     hb-ucd.obj
 0002:00033ff0       $chain$2$hb_ucd_get_unicode_funcs 00000001800deff0     hb-ucd.obj
 0002:00034004       $chain$3$hb_ucd_get_unicode_funcs 00000001800df004     hb-ucd.obj
 0002:00034014       $chain$1$?hb_ucd_compose@@YAHPEAUhb_unicode_funcs_t@@IIPEAIPEAX@Z 00000001800df014     hb-ucd.obj
 0002:0003402c       $chain$3$?hb_ucd_compose@@YAHPEAUhb_unicode_funcs_t@@IIPEAIPEAX@Z 00000001800df02c     hb-ucd.obj
 0002:0003402c       $chain$5$?hb_ucd_compose@@YAHPEAUhb_unicode_funcs_t@@IIPEAIPEAX@Z 00000001800df02c     hb-ucd.obj
 0002:00034044       $chain$0$hb_unicode_funcs_destroy 00000001800df044     hb-unicode.obj
 0002:00034058       $chain$1$hb_unicode_funcs_destroy 00000001800df058     hb-unicode.obj
 0002:00034068       $unwind$Java_sun_font_FileFontStrike__1getGlyphImageFromWindows 00000001800df068     lcdglyph.obj
 0002:00034094       $unwind$Java_sun_font_StrikeCache_freeIntMemory 00000001800df094     sunFont.obj
 0002:00034094       $unwind$Java_sun_font_StrikeCache_freeLongMemory 00000001800df094     sunFont.obj
 0002:00034094       $unwind$?filt$0@?0??dllmain_dispatch@@YAHQEAUHINSTANCE__@@KQEAX@Z@4HA 00000001800df094     MSVCRT:dll_dllmain.obj
 0002:0003409c       $chain$3$Java_sun_font_StrikeCache_freeIntMemory 00000001800df09c     sunFont.obj
 0002:000340bc       $chain$4$Java_sun_font_StrikeCache_freeIntMemory 00000001800df0bc     sunFont.obj
 0002:000340d0       $chain$5$Java_sun_font_StrikeCache_freeIntMemory 00000001800df0d0     sunFont.obj
 0002:000340e4       $chain$6$Java_sun_font_StrikeCache_freeIntMemory 00000001800df0e4     sunFont.obj
 0002:000340f4       $chain$7$Java_sun_font_StrikeCache_freeIntMemory 00000001800df0f4     sunFont.obj
 0002:00034104       $chain$8$Java_sun_font_StrikeCache_freeIntMemory 00000001800df104     sunFont.obj
 0002:00034114       $chain$3$Java_sun_font_StrikeCache_freeLongMemory 00000001800df114     sunFont.obj
 0002:00034134       $chain$4$Java_sun_font_StrikeCache_freeLongMemory 00000001800df134     sunFont.obj
 0002:00034148       $chain$5$Java_sun_font_StrikeCache_freeLongMemory 00000001800df148     sunFont.obj
 0002:0003415c       $chain$6$Java_sun_font_StrikeCache_freeLongMemory 00000001800df15c     sunFont.obj
 0002:0003416c       $chain$7$Java_sun_font_StrikeCache_freeLongMemory 00000001800df16c     sunFont.obj
 0002:0003417c       $chain$8$Java_sun_font_StrikeCache_freeLongMemory 00000001800df17c     sunFont.obj
 0002:0003418c       $chain$0$initFontIDs       00000001800df18c     sunFont.obj
 0002:000341a0       $chain$1$initFontIDs       00000001800df1a0     sunFont.obj
 0002:000341b0       $xdatasym                  00000001800df1b0     MSVCRT:amdsecgs.obj
 0002:000341b4       $unwind$__report_securityfailure 00000001800df1b4     MSVCRT:gs_report.obj
 0002:000341bc       $unwind$__report_gsfailure 00000001800df1bc     MSVCRT:gs_report.obj
 0002:000341c4       $unwind$capture_current_context 00000001800df1c4     MSVCRT:gs_report.obj
 0002:000341d0       $unwind$capture_previous_context 00000001800df1d0     MSVCRT:gs_report.obj
 0002:000341e0       $xdatasym                  00000001800df1e0     MSVCRT:chkstk.obj
 0002:000341e8       $unwind$?dllmain_crt_process_attach@@YAHQEAUHINSTANCE__@@QEAX@Z 00000001800df1e8     MSVCRT:dll_dllmain.obj
 0002:00034224       $unwind$?fin$0@?0??dllmain_crt_process_attach@@YAHQEAUHINSTANCE__@@QEAX@Z@4HA 00000001800df224     MSVCRT:dll_dllmain.obj
 0002:00034224       $unwind$?fin$0@?0??dllmain_crt_process_detach@@YAH_N@Z@4HA 00000001800df224     MSVCRT:dll_dllmain.obj
 0002:00034224       $unwind$?fin$1@?0??dllmain_crt_process_detach@@YAH_N@Z@4HA 00000001800df224     MSVCRT:dll_dllmain.obj
 0002:0003422c       $unwind$?dllmain_crt_process_detach@@YAH_N@Z 00000001800df22c     MSVCRT:dll_dllmain.obj
 0002:00034280       $unwind$?dllmain_dispatch@@YAHQEAUHINSTANCE__@@KQEAX@Z 00000001800df280     MSVCRT:dll_dllmain.obj
 0002:000342a8       $unwind$__isa_available_init 00000001800df2a8     MSVCRT:cpu_disp.obj
 0002:000342b8       $unwind$__security_init_cookie 00000001800df2b8     MSVCRT:gs_support.obj
 0002:000342c4       $unwind$__scrt_is_nonwritable_in_current_image 00000001800df2c4     MSVCRT:utility.obj
 0002:000342e4       $unwind$__scrt_fastfail    00000001800df2e4     MSVCRT:utility_desktop.obj
 0002:000342f8       $xdatasym                  00000001800df2f8     MSVCRT:guard_dispatch.obj
 0002:00034300       $xdatasym                  00000001800df300     MSVCRT:guard_xfg_dispatch.obj
 0002:00034310       .edata                     00000001800df310     fontmanager.exp
 0002:00034338       rgpv                       00000001800df338     fontmanager.exp
 0002:000343d4       rgszName                   00000001800df3d4     fontmanager.exp
 0002:00034470       rgwOrd                     00000001800df470     fontmanager.exp
 0002:000344be       szName                     00000001800df4be     fontmanager.exp
 0002:000344ce       $N00001                    00000001800df4ce     fontmanager.exp
 0002:000344db       $N00002                    00000001800df4db     fontmanager.exp
 0002:000344ed       $N00003                    00000001800df4ed     fontmanager.exp
 0002:000344fb       $N00004                    00000001800df4fb     fontmanager.exp
 0002:00034525       $N00005                    00000001800df525     fontmanager.exp
 0002:0003455c       $N00006                    00000001800df55c     fontmanager.exp
 0002:00034588       $N00007                    00000001800df588     fontmanager.exp
 0002:000345bc       $N00008                    00000001800df5bc     fontmanager.exp
 0002:000345f4       $N00009                    00000001800df5f4     fontmanager.exp
 0002:0003462f       $N00010                    00000001800df62f     fontmanager.exp
 0002:00034664       $N00011                    00000001800df664     fontmanager.exp
 0002:0003469a       $N00012                    00000001800df69a     fontmanager.exp
 0002:000346d1       $N00013                    00000001800df6d1     fontmanager.exp
 0002:00034705       $N00014                    00000001800df705     fontmanager.exp
 0002:0003473a       $N00015                    00000001800df73a     fontmanager.exp
 0002:00034771       $N00016                    00000001800df771     fontmanager.exp
 0002:000347ae       $N00017                    00000001800df7ae     fontmanager.exp
 0002:000347e5       $N00018                    00000001800df7e5     fontmanager.exp
 0002:0003481a       $N00019                    00000001800df81a     fontmanager.exp
 0002:00034857       $N00020                    00000001800df857     fontmanager.exp
 0002:00034892       $N00021                    00000001800df892     fontmanager.exp
 0002:000348c6       $N00022                    00000001800df8c6     fontmanager.exp
 0002:000348fb       $N00023                    00000001800df8fb     fontmanager.exp
 0002:00034924       $N00024                    00000001800df924     fontmanager.exp
 0002:00034956       $N00025                    00000001800df956     fontmanager.exp
 0002:00034981       $N00026                    00000001800df981     fontmanager.exp
 0002:000349b3       $N00027                    00000001800df9b3     fontmanager.exp
 0002:000349db       $N00028                    00000001800df9db     fontmanager.exp
 0002:00034a04       $N00029                    00000001800dfa04     fontmanager.exp
 0002:00034a2d       $N00030                    00000001800dfa2d     fontmanager.exp
 0002:00034a57       $N00031                    00000001800dfa57     fontmanager.exp
 0002:00034a86       $N00032                    00000001800dfa86     fontmanager.exp
 0002:00034aab       $N00033                    00000001800dfaab     fontmanager.exp
 0002:00034ad4       $N00034                    00000001800dfad4     fontmanager.exp
 0002:00034afe       $N00035                    00000001800dfafe     fontmanager.exp
 0002:00034b22       $N00036                    00000001800dfb22     fontmanager.exp
 0002:00034b58       $N00037                    00000001800dfb58     fontmanager.exp
 0002:00034b90       $N00038                    00000001800dfb90     fontmanager.exp
 0002:00034bc2       $N00039                    00000001800dfbc2     fontmanager.exp
 0002:000352cc       .idata$6                   00000001800e02cc     awt:awt.dll
 0002:0003536a       .idata$6                   00000001800e036a     java:java.dll
 0002:00035504       .idata$6                   00000001800e0504     freetype:freetype.dll
 0002:00035554       .idata$6                   00000001800e0554     advapi32:ADVAPI32.dll
 0002:0003567a       .idata$6                   00000001800e067a     gdi32:GDI32.dll
 0002:000356de       .idata$6                   00000001800e06de     user32:USER32.dll
 0002:0003593e       .idata$6                   00000001800e093e     kernel32:KERNEL32.dll
 0002:000359de       .idata$6                   00000001800e09de     vcruntime:VCRUNTIME140.dll
 0002:00035bd8       .idata$6                   00000001800e0bd8     ucrt:api-ms-win-crt-heap-l1-1-0.dll
 0002:00035bf8       .idata$6                   00000001800e0bf8     ucrt:api-ms-win-crt-math-l1-1-0.dll
 0002:00035c18       .idata$6                   00000001800e0c18     ucrt:api-ms-win-crt-environment-l1-1-0.dll
 0002:00035c3e       .idata$6                   00000001800e0c3e     ucrt:api-ms-win-crt-convert-l1-1-0.dll
 0002:00035c60       .idata$6                   00000001800e0c60     ucrt:api-ms-win-crt-stdio-l1-1-0.dll
 0002:00035c80       .idata$6                   00000001800e0c80     ucrt:api-ms-win-crt-string-l1-1-0.dll
 0002:00035ca2       .idata$6                   00000001800e0ca2     ucrt:api-ms-win-crt-runtime-l1-1-0.dll
 0003:00000200       gvdClassName               00000001800e1200     HBShaper.obj
 0003:00000208       ?PADBYTES@?1??getGlyphImageNativeInternal@@9@9 00000001800e1208     freetypeScaler.obj
 0003:00000210       ?_hb_buffer_serialize_formats@@3PAPEBDA 00000001800e1210     hb-buffer-serialize.obj
 0003:00000538       ?supported_face_loaders@@3PAUsupported_face_loaders_t@@A 00000001800e1538     hb-face.obj
 0003:000006e0       ?_hb_draw_funcs_default@@3Uhb_draw_funcs_t@@B 00000001800e16e0     hb-font.obj
 0003:00000728       ?supported_font_funcs@@3PAUsupported_font_funcs_t@@A 00000001800e1728     hb-font.obj
 0003:00000740       ?_hb_font_funcs_default@@3Uhb_font_funcs_t@@B 00000001800e1740     hb-font.obj
 0003:000007f8       ?modifier_combining_marks@@3PAIA 00000001800e17f8     hb-ot-shaper-arabic.obj
 0003:00000830       ?thai_above_start_state@@3PAW4thai_above_state_t@@A 00000001800e1830     hb-ot-shaper-thai.obj
 0003:00000848       ?thai_below_start_state@@3PAW4thai_below_state_t@@A 00000001800e1848     hb-ot-shaper-thai.obj
 0003:00000b00       gvdClass                   00000001800e1b00     HBShaper.obj
 0003:00000b08       gvdCountFID                00000001800e1b08     HBShaper.obj
 0003:00000b10       gvdFlagsFID                00000001800e1b10     HBShaper.obj
 0003:00000b18       gvdGlyphsFID               00000001800e1b18     HBShaper.obj
 0003:00000b20       gvdPositionsFID            00000001800e1b20     HBShaper.obj
 0003:00000b28       gvdIndicesFID              00000001800e1b28     HBShaper.obj
 0003:00000b30       gvdGrowMID                 00000001800e1b30     HBShaper.obj
 0003:00000b38       jniInited                  00000001800e1b38     HBShaper.obj
 0003:00000b40       screenDC                   00000001800e1b40     fontpath.obj
 0003:00000b48       invalidateScalerMID        00000001800e1b48     freetypeScaler.obj
 0003:00000b50       debugFonts                 00000001800e1b50     freetypeScaler.obj
 0003:00000de8       ?langs@@3U?$hb_atomic_t@PEAUhb_language_item_t@@@@A 00000001800e1de8     hb-common.obj
 0003:00000df0       ?static_draw_extents_funcs@@3Uhb_draw_extents_funcs_lazy_loader_t@@A 00000001800e1df0     hb-draw.obj
 0003:00000df8       ?static_face_loader_list@@3Uhb_face_loader_list_lazy_loader_t@@A 00000001800e1df8     hb-face.obj
 0003:00000e00       ?static_funcs_name@?1??get_default_funcs_name@@YAPEBDXZ@4U?$hb_atomic_t@PEBD@@A 00000001800e1e00     hb-font.obj
 0003:00000e08       ?static_font_funcs_list@@3Uhb_font_funcs_list_lazy_loader_t@@A 00000001800e1e08     hb-font.obj
 0003:00000e10       ?jdk_ffuncs@?1??_hb_jdk_get_font_funcs@@YAPEAUhb_font_funcs_t@@XZ@4PEAU2@EA 00000001800e1e10     hb-jdk-font.obj
 0003:00000e18       ?static_ot_funcs@@3Uhb_ot_font_funcs_lazy_loader_t@@A 00000001800e1e18     hb-ot-font.obj
 0003:00000e20       ?last_tag_idx@?4??hb_ot_tags_from_language@@YAXPEBD0PEAI1@Z@4U?$hb_atomic_t@I@@A 00000001800e1e20     hb-ot-tag.obj
 0003:00000e28       ?static_outline_recording_pen_funcs@@3Uhb_outline_recording_pen_funcs_lazy_loader_t@@A 00000001800e1e28     hb-outline.obj
 0003:00000e30       ?static_paint_bounded_funcs@@3Uhb_paint_bounded_funcs_lazy_loader_t@@A 00000001800e1e30     hb-paint-bounded.obj
 0003:00000e38       ?static_paint_extents_funcs@@3Uhb_paint_extents_funcs_lazy_loader_t@@A 00000001800e1e38     hb-paint-extents.obj
 0003:00000e40       ?static_shaper_list@@3Uhb_shaper_list_lazy_loader_t@@A 00000001800e1e40     hb-shape.obj
 0003:00000e48       ?static_shapers@@3Uhb_shapers_lazy_loader_t@@A 00000001800e1e48     hb-shaper.obj
 0003:00000e50       ?static_ucd_funcs@@3Uhb_ucd_unicode_funcs_lazy_loader_t@@A 00000001800e1e50     hb-ucd.obj
 0003:00000e60       igLUTable                  00000001800e1e60     lcdglyph.obj
 0003:00001228       theNullScalerContext       00000001800e2228     sunFont.obj
 0003:00001230       initialisedFontIDs         00000001800e2230     sunFont.obj
 0003:00001240       GS_ExceptionRecord         00000001800e2240     MSVCRT:gs_report.obj
 0003:000012e0       GS_ContextRecord           00000001800e22e0     MSVCRT:gs_report.obj
 0003:000017b0       ?__proc_attached@@3HA      00000001800e27b0     MSVCRT:dll_dllmain.obj
 0003:000017e8       ?is_initialized_as_dll@@3_NA 00000001800e27e8     MSVCRT:utility.obj
 0003:000017e9       ?module_local_atexit_table_initialized@@3_NA 00000001800e27e9     MSVCRT:utility.obj
 0003:000017f0       ?module_local_atexit_table@@3U_onexit_table_t@@A 00000001800e27f0     MSVCRT:utility.obj
 0003:00001808       ?module_local_at_quick_exit_table@@3U_onexit_table_t@@A 00000001800e2808     MSVCRT:utility.obj
 0005:00000000       _2il0floatpacket$0         00000001800ec000     MSVCRT:svml_sfloorf4_sse2.obj
 0005:00000010       _2il0floatpacket$1         00000001800ec010     MSVCRT:svml_sfloorf4_sse2.obj
 0005:00000020       _2il0floatpacket$2         00000001800ec020     MSVCRT:svml_sfloorf4_sse2.obj
 0006:00000060       $R000000                   00000001800ed060     fontmanager.dll.res
